 vbsp

 Timestamp is 47b58f03 (Fri Feb 15 14:09:23 2008)

 Preferred load address is 00400000

 Start         Length     Name                   Class
 0001:00000000 000974dcH .text                   CODE
 0001:000974e0 000002c3H .text$x                 CODE
 0001:000977b0 00000cabH .text$yc                CODE
 0001:00098460 00000a22H .text$yd                CODE
 0002:00000000 0000024cH .idata$5                DATA
 0002:0000024c 00000004H .CRT$XCA                DATA
 0002:00000250 0000000cH .CRT$XCC                DATA
 0002:0000025c 00000224H .CRT$XCU                DATA
 0002:00000480 00000004H .CRT$XCZ                DATA
 0002:00000484 00000004H .CRT$XIA                DATA
 0002:00000488 00000014H .CRT$XIC                DATA
 0002:0000049c 00000004H .CRT$XIY                DATA
 0002:000004a0 00000004H .CRT$XIZ                DATA
 0002:000004a4 00000004H .CRT$XPA                DATA
 0002:000004a8 00000008H .CRT$XPX                DATA
 0002:000004b0 00000004H .CRT$XPXA               DATA
 0002:000004b4 00000004H .CRT$XPZ                DATA
 0002:000004b8 00000004H .CRT$XTA                DATA
 0002:000004bc 00000004H .CRT$XTZ                DATA
 0002:000004c0 00052794H .rdata                  DATA
 0002:00052c54 00000043H .rdata$debug            DATA
 0002:00052c98 00000dacH .rdata$r                DATA
 0002:00053a44 00000004H .rtc$IAA                DATA
 0002:00053a48 00000004H .rtc$IZZ                DATA
 0002:00053a4c 00000004H .rtc$TAA                DATA
 0002:00053a50 00000004H .rtc$TZZ                DATA
 0002:00053a58 00000f8cH .xdata$x                DATA
 0002:000549e4 00000050H .idata$2                DATA
 0002:00054a34 00000014H .idata$3                DATA
 0002:00054a48 0000024cH .idata$4                DATA
 0002:00054c94 00000b42H .idata$6                DATA
 0002:000557e0 0000004bH .edata                  DATA
 0003:00000000 000097d8H .data                   DATA
 0003:000097e0 06b50818H .bss                    DATA

  Address         Publics by Value              Rva+Base       Lib:Object

 0000:00000000       ___safe_se_handler_table   00000000     <absolute>
 0000:00000000       __except_list              00000000     <absolute>
 0000:00000000       ___safe_se_handler_count   00000000     <absolute>
 0000:00000000       ___ImageBase               00400000     <linker-defined>
 0001:00000000       ??0Vector2D@@QAE@XZ        00401000 f i collisionutils.obj
 0001:00000000       ??0cplane_t@@QAE@XZ        00401000 f i collisionutils.obj
 0001:00000000       ??0Vector@@QAE@XZ          00401000 f i brushbsp.obj
 0001:00000010       ??AVector@@QAEAAMH@Z       00401010 f i brushbsp.obj
 0001:00000020       ??AVector@@QBEMH@Z         00401020 f i brushbsp.obj
 0001:00000030       ??_H@YGXPAXIHP6EPAX0@Z@Z   00401030 f i brushbsp.obj
 0001:00000070       ?VectorLength@@YAMABVVector@@@Z 00401070 f i brushbsp.obj
 0001:000000a0       ??HVector@@QBE?AV0@ABV0@@Z 004010a0 f i brushbsp.obj
 0001:000000d0       ??DVector@@QBE?AV0@M@Z     004010d0 f i brushbsp.obj
 0001:00000100       ?BoundBrush@@YAXPAUbspbrush_t@@@Z 00401100 f   brushbsp.obj
 0001:00000190       ?PointInsideBrush@@YA?AVVector@@PAUbspbrush_t@@@Z 00401190 f   brushbsp.obj
 0001:00000420       ?CreateBrushWindings@@YAXPAUbspbrush_t@@@Z 00401420 f   brushbsp.obj
 0001:000005b0       ?BrushVolume@@YAMPAUbspbrush_t@@@Z 004015b0 f   brushbsp.obj
 0001:00000680       ?CountBrushList@@YAHPAUbspbrush_t@@@Z 00401680 f   brushbsp.obj
 0001:000006a0       ?AllocTree@@YAPAUtree_t@@XZ 004016a0 f   brushbsp.obj
 0001:000006d0       ?AllocNode@@YAPAUnode_t@@XZ 004016d0 f   brushbsp.obj
 0001:00000710       ?AllocBrush@@YAPAUbspbrush_t@@H@Z 00401710 f   brushbsp.obj
 0001:00000760       ?FreeBrush@@YAXPAUbspbrush_t@@@Z 00401760 f   brushbsp.obj
 0001:000007b0       ?FreeBrushList@@YAXPAUbspbrush_t@@@Z 004017b0 f   brushbsp.obj
 0001:000007e0       ?CopyBrush@@YAPAUbspbrush_t@@PAU1@@Z 004017e0 f   brushbsp.obj
 0001:00000870       ?PointInLeaf@@YAPAUnode_t@@PAU1@AAVVector@@@Z 00401870 f   brushbsp.obj
 0001:000008e0       ?BrushBspBoxOnPlaneSide@@YAHABVVector@@0PAUdplane_t@@@Z 004018e0 f   brushbsp.obj
 0001:000009d0       ?TestBrushToPlanenum@@YAHPAUbspbrush_t@@HPAH11@Z 004019d0 f   brushbsp.obj
 0001:00000da0       ?WindingIsTiny@@YAHPAUwinding_t@@@Z 00401da0 f   brushbsp.obj
 0001:00000e30       ?WindingIsHuge@@YAHPAUwinding_t@@@Z 00401e30 f   brushbsp.obj
 0001:00000eb0       ?LeafNode@@YAXPAUnode_t@@PAUbspbrush_t@@@Z 00401eb0 f   brushbsp.obj
 0001:00000f20       ?RemoveAreaPortalBrushes_R@@YAXPAUnode_t@@@Z 00401f20 f   brushbsp.obj
 0001:00000f70       ?BrushMostlyOnSide@@YAHPAUbspbrush_t@@PAUplane_t@@@Z 00401f70 f   brushbsp.obj
 0001:00001170       ?BrushFromBounds@@YAPAUbspbrush_t@@AAVVector@@0@Z 00402170 f   brushbsp.obj
 0001:00001260       ??4?$CUtlVector@HV?$CUtlMemory@HH@@@@QAEAAV0@ABV0@@Z 00402260 f i brushbsp.obj
 0001:000012a0       ??4side_t@@QAEAAU0@ABU0@@Z 004022a0 f i brushbsp.obj
 0001:00001320       ?SplitBrush@@YAXPAUbspbrush_t@@HPAPAU1@1@Z 00402320 f   brushbsp.obj
 0001:00001aa0       ?SplitBrushList@@YAXPAUbspbrush_t@@PAUnode_t@@PAPAU1@2@Z 00402aa0 f   brushbsp.obj
 0001:00001b80       ?SelectSplitSide@@YAPAUside_t@@PAUbspbrush_t@@PAUnode_t@@@Z 00402b80 f   brushbsp.obj
 0001:00001e70       ?BuildTree_r@@YAPAUnode_t@@PAU1@PAUbspbrush_t@@@Z 00402e70 f   brushbsp.obj
 0001:00001f90       ?BrushBSP@@YAPAUtree_t@@PAUbspbrush_t@@AAVVector@@1@Z 00402f90 f   brushbsp.obj
 0001:00002150       ?fabs@@YAMM@Z              00403150 f i collisionutils.obj
 0001:00002160       ?Vector2DSubtract@@YAXABVVector2D@@0AAV1@@Z 00403160 f i collisionutils.obj
 0001:00002180       ?Init@Vector@@QAEXMMM@Z    00403180 f i collisionutils.obj
 0001:000021a0       ??4Vector@@QAEAAV0@ABV0@@Z 004031a0 f i collisionutils.obj
 0001:000021c0       ?Dot@Vector@@QBEMABV1@@Z   004031c0 f i collisionutils.obj
 0001:000021e0       ?CrossProduct@@YAXABVVector@@0AAV1@@Z 004031e0 f i collisionutils.obj
 0001:00002220       ?Length@Vector@@QBEMXZ     00403220 f i collisionutils.obj
 0001:00002250       ??GVector@@QBE?AV0@ABV0@@Z 00403250 f i collisionutils.obj
 0001:00002280       ?IsBoxIntersectingBox@@YA_NABVVector@@000@Z 00403280 f   collisionutils.obj
 0001:000022f0       ?PointInQuadFromBarycentric@@YAXABVVector@@000ABVVector2D@@AAV1@@Z 004032f0 f   collisionutils.obj
 0001:00002380       ?SubtractBrush@@YAPAUbspbrush_t@@PAU1@0@Z 00403380 f   csg.obj
 0001:00002430       ?IntersectBrush@@YAPAUbspbrush_t@@PAU1@0@Z 00403430 f   csg.obj
 0001:000024b0       ?BrushesDisjoint@@YAHPAUbspbrush_t@@0@Z 004034b0 f   csg.obj
 0001:00002560       ?ClipBrushToBox@@YAPAUbspbrush_t@@PAU1@ABVVector@@1@Z 00403560 f   csg.obj
 0001:00002820       ?MakeBspBrushList@@YAPAUbspbrush_t@@HHABVVector@@0H@Z 00403820 f   csg.obj
 0001:000028b0       ?MakeBspBrushList@@YAPAUbspbrush_t@@PAPAUmapbrush_t@@HABVVector@@1@Z 004038b0 f   csg.obj
 0001:00002920       ?PrintBrushContentsToString@@YAXHPADH@Z 00403920 f   csg.obj
 0001:00002bb0       ?ChopBrushes@@YAPAUbspbrush_t@@PAU1@@Z 00403bb0 f   csg.obj
 0001:00002ef0       ?CopyMatchingTexinfos@@YAXPAUside_t@@HPBUbspbrush_t@@@Z 00403ef0 f   csg.obj
 0001:00003010       ?FixupAreaportalWaterBrushes@@YAXPAUbspbrush_t@@@Z 00404010 f   csg.obj
 0001:000030b0       ?VectorScale@@YAXABVVector@@MAAV1@@Z 004040b0 f i cubemap.obj
 0001:00003100       ?Cubemap_InsertSample@@YAXABVVector@@H@Z 00404100 f   cubemap.obj
 0001:000034e0       ?DoesMaterialOrDependentsUseEnvmap@@YA_NPBD@Z 004044e0 f   cubemap.obj
 0001:00003530       ?Cubemap_FindClosestCubemap@@YAHABVVector@@PAUside_t@@@Z 00404530 f   cubemap.obj
 0001:00003730       ?Purge@?$CUtlMemory@EH@@QAEXXZ 00404730 f i cubemap.obj
 0001:00003760       ?Links@?$CUtlRBTree@UCubemapInfo_t@@GP6A_NABU1@0@ZV?$CUtlMemory@U?$UtlRBTreeNode_t@UCubemapInfo_t@@G@@G@@@@IBEABU?$UtlRBTreeLinks_t@G@@G@Z 00404760 f i cubemap.obj
 0001:000037c0       ?Next@?$CUtlMemory@U?$UtlLinkedListElem_t@UGameLump_t@@G@@G@@QBE?AVIterator_t@1@ABV21@@Z 004047c0 f i bsplib.obj
 0001:000037c0       ?Next@?$CUtlMemory@U?$UtlRBTreeNode_t@UStaticPropLookup_t@@G@@G@@QBE?AVIterator_t@1@ABV21@@Z 004047c0 f i detailobjects.obj
 0001:000037c0       ?Next@?$CUtlMemory@U?$UtlRBTreeNode_t@VCStringPoolIndex@CUtlSymbolTable@@G@@G@@QBE?AVIterator_t@1@ABV21@@Z 004047c0 f i tier1:utlsymbol.obj
 0001:000037c0       ?Next@?$CUtlMemory@U?$UtlRBTreeNode_t@UModelCollisionLookup_t@@G@@G@@QBE?AVIterator_t@1@ABV21@@Z 004047c0 f i staticprop.obj
 0001:000037c0       ?Next@?$CUtlMemory@U?$UtlRBTreeNode_t@UCubemapInfo_t@@G@@G@@QBE?AVIterator_t@1@ABV21@@Z 004047c0 f i cubemap.obj
 0001:000037c0       ?Next@?$CUtlMemory@U?$UtlLinkedListElem_t@PAVCZip@@G@@G@@QBE?AVIterator_t@1@ABV21@@Z 004047c0 f i zip_utils.obj
 0001:00003800       ?Grow@?$CUtlMemory@Utexinfo_s@@H@@QAEXH@Z 00404800 f i cubemap.obj
 0001:000038a0       ?Grow@?$CUtlMemory@U?$UtlRBTreeNode_t@UCubemapInfo_t@@G@@G@@QAEXH@Z 004048a0 f i cubemap.obj
 0001:000038a0       ?Grow@?$CUtlMemory@U?$UtlRBTreeNode_t@UModelCollisionLookup_t@@G@@G@@QAEXH@Z 004048a0 f i staticprop.obj
 0001:00003960       ?Purge@?$CUtlVector@HV?$CUtlMemory@HH@@@@QAEXXZ 00404960 f i cubemap.obj
 0001:000039b0       ?FindInsertionPosition@?$CUtlRBTree@UCubemapInfo_t@@GP6A_NABU1@0@ZV?$CUtlMemory@U?$UtlRBTreeNode_t@UCubemapInfo_t@@G@@G@@@@IAEXABUCubemapInfo_t@@AAGAA_N@Z 004049b0 f i cubemap.obj
 0001:00003ac0       ?NewNode@?$CUtlRBTree@UCubemapInfo_t@@GP6A_NABU1@0@ZV?$CUtlMemory@U?$UtlRBTreeNode_t@UCubemapInfo_t@@G@@G@@@@QAEGXZ 00404ac0 f i cubemap.obj
 0001:00003bb0       ?RotateLeft@?$CUtlRBTree@UCubemapInfo_t@@GP6A_NABU1@0@ZV?$CUtlMemory@U?$UtlRBTreeNode_t@UCubemapInfo_t@@G@@G@@@@IAEXG@Z 00404bb0 f i cubemap.obj
 0001:00003ca0       ?RotateRight@?$CUtlRBTree@UCubemapInfo_t@@GP6A_NABU1@0@ZV?$CUtlMemory@U?$UtlRBTreeNode_t@UCubemapInfo_t@@G@@G@@@@IAEXG@Z 00404ca0 f i cubemap.obj
 0001:00003da0       ??0?$CUtlRBTree@UCubemapInfo_t@@GP6A_NABU1@0@ZV?$CUtlMemory@U?$UtlRBTreeNode_t@UCubemapInfo_t@@G@@G@@@@QAE@HHABQ6A_NABUCubemapInfo_t@@0@Z@Z 00404da0 f i cubemap.obj
 0001:00003e00       ?Find@?$CUtlRBTree@UCubemapInfo_t@@GP6A_NABU1@0@ZV?$CUtlMemory@U?$UtlRBTreeNode_t@UCubemapInfo_t@@G@@G@@@@QBEGABUCubemapInfo_t@@@Z 00404e00 f i cubemap.obj
 0001:00003f00       ?RemoveAll@?$CUtlRBTree@UCubemapInfo_t@@GP6A_NABU1@0@ZV?$CUtlMemory@U?$UtlRBTreeNode_t@UCubemapInfo_t@@G@@G@@@@QAEXXZ 00404f00 f i cubemap.obj
 0001:00003fc0       ?InsertRebalance@?$CUtlRBTree@UCubemapInfo_t@@GP6A_NABU1@0@ZV?$CUtlMemory@U?$UtlRBTreeNode_t@UCubemapInfo_t@@G@@G@@@@IAEXG@Z 00404fc0 f i cubemap.obj
 0001:000048a0       ?CreateDefaultCubemaps@@YAX_N@Z 004058a0 f   cubemap.obj
 0001:00004c90       ?Cubemap_CreateDefaultCubemaps@@YAXXZ 00405c90 f   cubemap.obj
 0001:00004cb0       ?InsertBefore@?$CUtlVector@Utexinfo_s@@V?$CUtlMemory@Utexinfo_s@@H@@@@QAEHHABUtexinfo_s@@@Z 00405cb0 f i cubemap.obj
 0001:00004d30       ?InsertBefore@?$CUtlVector@V?$CUtlVector@HV?$CUtlMemory@HH@@@@V?$CUtlMemory@V?$CUtlVector@HV?$CUtlMemory@HH@@@@H@@@@QAEHH@Z 00405d30 f i cubemap.obj
 0001:00004db0       ?LinkToParent@?$CUtlRBTree@UCubemapInfo_t@@GP6A_NABU1@0@ZV?$CUtlMemory@U?$UtlRBTreeNode_t@UCubemapInfo_t@@G@@G@@@@IAEXGG_N@Z 00405db0 f i cubemap.obj
 0001:00004e20       ?Cubemap_AddUnreferencedCubemaps@@YAXXZ 00405e20 f   cubemap.obj
 0001:00004fb0       ?RemoveAll@?$CUtlVector@Ucluster_portals_t@@V?$CUtlMemory@Ucluster_portals_t@@H@@@@QAEXXZ 00405fb0 f i prtfile.obj
 0001:00004fb0       ?RemoveAll@?$CUtlVector@V?$CUtlVector@HV?$CUtlMemory@HH@@@@V?$CUtlMemory@V?$CUtlVector@HV?$CUtlMemory@HH@@@@H@@@@QAEXXZ 00405fb0 f i cubemap.obj
 0001:00005040       ?Cubemap_SaveBrushSides@@YAXPBD@Z 00406040 f   cubemap.obj
 0001:000053d0       ?Cubemap_FixupBrushSidesMaterials@@YAXXZ 004063d0 f   cubemap.obj
 0001:000054e0       ?Insert@?$CUtlRBTree@UCubemapInfo_t@@GP6A_NABU1@0@ZV?$CUtlMemory@U?$UtlRBTreeNode_t@UCubemapInfo_t@@G@@G@@@@QAEGABUCubemapInfo_t@@@Z 004064e0 f i cubemap.obj
 0001:00005550       ?Cubemap_InitCubemapSideData@@YAXXZ 00406550 f   cubemap.obj
 0001:000056f0       ?Cubemap_AttachDefaultCubemapToSpecularSides@@YAXXZ 004066f0 f   cubemap.obj
 0001:00005870       ??1?$CUtlVector@V?$CUtlVector@HV?$CUtlMemory@HH@@@@V?$CUtlMemory@V?$CUtlVector@HV?$CUtlMemory@HH@@@@H@@@@QAE@XZ 00406870 f i cubemap.obj
 0001:00005870       ??1?$CUtlVector@Ucluster_portals_t@@V?$CUtlMemory@Ucluster_portals_t@@H@@@@QAE@XZ 00406870 f i prtfile.obj
 0001:000058d0       ?MergeBrush_r@@YAXPAUnode_t@@PAUbspbrush_t@@@Z 004068d0 f   detail.obj
 0001:00005950       ?MergeFace_r@@YA_NPAUnode_t@@PAUface_t@@1@Z 00406950 f   detail.obj
 0001:00005af0       ?FilterFacesIntoTree@@YAPAUface_t@@PAUtree_t@@PAU1@@Z 00406af0 f   detail.obj
 0001:00005b80       ?TryMergeFaceList@@YAXPAPAUface_t@@@Z 00406b80 f   detail.obj
 0001:00005c90       ?FilterBrushesIntoTree@@YAXPAUtree_t@@PAUbspbrush_t@@@Z 00406c90 f   detail.obj
 0001:00005cc0       ?BrushBoxOverlap@@YA_NPAUbspbrush_t@@0@Z 00406cc0 f   detail.obj
 0001:00005d10       ?FindOriginalSide@@YAPAUside_t@@PAUmapbrush_t@@PAU1@@Z 00406d10 f   detail.obj
 0001:00005de0       ?ClipFaceToBrush@@YA_NPAUface_t@@PAUbspbrush_t@@PAPAU1@@Z 00406de0 f   detail.obj
 0001:000060f0       ?GetListOfCutBrushes@@YAHAAV?$CUtlVector@PAUbspbrush_t@@V?$CUtlMemory@PAUbspbrush_t@@H@@@@PAUbspbrush_t@@1@Z 004070f0 f   detail.obj
 0001:00006240       ?ComputeVisibleBrushSides@@YAPAUface_t@@PAUbspbrush_t@@@Z 00407240 f   detail.obj
 0001:00006410       ?MergeDetailTree@@YAPAUface_t@@PAUtree_t@@HH@Z 00407410 f   detail.obj
 0001:00006550       ?Init@Vector2D@@QAEXMM@Z   00407550 f i detailobjects.obj
 0001:00006760       ?Links@?$CUtlRBTree@UStaticPropLookup_t@@GP6A_NABU1@0@ZV?$CUtlMemory@U?$UtlRBTreeNode_t@UStaticPropLookup_t@@G@@G@@@@IBEABU?$UtlRBTreeLinks_t@G@@G@Z 00407760 f i detailobjects.obj
 0001:000067c0       ?Grow@?$CUtlMemory@U?$UtlRBTreeNode_t@UStaticPropLookup_t@@G@@G@@QAEXH@Z 004077c0 f i detailobjects.obj
 0001:000067c0       ?Grow@?$CUtlMemory@U?$UtlRBTreeNode_t@VCStringPoolIndex@CUtlSymbolTable@@G@@G@@QAEXH@Z 004077c0 f i tier1:utlsymbol.obj
 0001:00006880       ?Grow@?$CUtlMemory@UDetailObjectDictLump_t@@H@@QAEXH@Z 00407880 f i detailobjects.obj
 0001:00006880       ?Grow@?$CUtlMemory@UStaticPropDictLump_t@@H@@QAEXH@Z 00407880 f i staticprop.obj
 0001:00006930       ?Grow@?$CUtlMemory@UDetailObjectLump_t@@H@@QAEXH@Z 00407930 f i detailobjects.obj
 0001:000069e0       ?Grow@?$CUtlMemory@UDetailSpriteDictLump_t@@H@@QAEXH@Z 004079e0 f i detailobjects.obj
 0001:000069e0       ?Grow@?$CUtlMemory@Udtexdata_t@@H@@QAEXH@Z 004079e0 f i writebsp.obj
 0001:00006b90       ??$PutTypeBin@H@CUtlBuffer@@IAEXH@Z 00407b90 f i detailobjects.obj
 0001:00006bf0       ?FindInsertionPosition@?$CUtlRBTree@UStaticPropLookup_t@@GP6A_NABU1@0@ZV?$CUtlMemory@U?$UtlRBTreeNode_t@UStaticPropLookup_t@@G@@G@@@@IAEXABUStaticPropLookup_t@@AAGAA_N@Z 00407bf0 f i detailobjects.obj
 0001:00006d00       ?NewNode@?$CUtlRBTree@UStaticPropLookup_t@@GP6A_NABU1@0@ZV?$CUtlMemory@U?$UtlRBTreeNode_t@UStaticPropLookup_t@@G@@G@@@@QAEGXZ 00407d00 f i detailobjects.obj
 0001:00006e00       ?RotateLeft@?$CUtlRBTree@UStaticPropLookup_t@@GP6A_NABU1@0@ZV?$CUtlMemory@U?$UtlRBTreeNode_t@UStaticPropLookup_t@@G@@G@@@@IAEXG@Z 00407e00 f i detailobjects.obj
 0001:00006f00       ?RotateRight@?$CUtlRBTree@UStaticPropLookup_t@@GP6A_NABU1@0@ZV?$CUtlMemory@U?$UtlRBTreeNode_t@UStaticPropLookup_t@@G@@G@@@@IAEXG@Z 00407f00 f i detailobjects.obj
 0001:00007000       ?Find@?$CUtlRBTree@UStaticPropLookup_t@@GP6A_NABU1@0@ZV?$CUtlMemory@U?$UtlRBTreeNode_t@UStaticPropLookup_t@@G@@G@@@@QBEGABUStaticPropLookup_t@@@Z 00408000 f i detailobjects.obj
 0001:00007110       ?InsertBefore@?$CUtlVector@UDetailObjectLump_t@@V?$CUtlMemory@UDetailObjectLump_t@@H@@@@QAEHH@Z 00408110 f i detailobjects.obj
 0001:00007170       ?InsertBefore@?$CUtlVector@UDetailSpriteDictLump_t@@V?$CUtlMemory@UDetailSpriteDictLump_t@@H@@@@QAEHHABUDetailSpriteDictLump_t@@@Z 00408170 f i detailobjects.obj
 0001:00007210       ?RemoveAll@?$CUtlRBTree@UStaticPropLookup_t@@GP6A_NABU1@0@ZV?$CUtlMemory@U?$UtlRBTreeNode_t@UStaticPropLookup_t@@G@@G@@@@QAEXXZ 00408210 f i detailobjects.obj
 0001:000072d0       ?InsertRebalance@?$CUtlRBTree@UStaticPropLookup_t@@GP6A_NABU1@0@ZV?$CUtlMemory@U?$UtlRBTreeNode_t@UStaticPropLookup_t@@G@@G@@@@IAEXG@Z 004082d0 f i detailobjects.obj
 0001:000079e0       ?InsertBefore@?$CUtlVector@UDetailModel_t@@V?$CUtlMemory@UDetailModel_t@@H@@@@QAEHH@Z 004089e0 f i detailobjects.obj
 0001:00007a60       ?LinkToParent@?$CUtlRBTree@UStaticPropLookup_t@@GP6A_NABU1@0@ZV?$CUtlMemory@U?$UtlRBTreeNode_t@UStaticPropLookup_t@@G@@G@@@@IAEXGG_N@Z 00408a60 f i detailobjects.obj
 0001:00007e20       ??1?$CUtlRBTree@UStaticPropLookup_t@@GP6A_NABU1@0@ZV?$CUtlMemory@U?$UtlRBTreeNode_t@UStaticPropLookup_t@@G@@G@@@@QAE@XZ 00408e20 f i detailobjects.obj
 0001:00007e80       ?Insert@?$CUtlRBTree@UStaticPropLookup_t@@GP6A_NABU1@0@ZV?$CUtlMemory@U?$UtlRBTreeNode_t@UStaticPropLookup_t@@G@@G@@@@QAEGABUStaticPropLookup_t@@@Z 00408e80 f i detailobjects.obj
 0001:00008c90       ?EmitDetailModels@@YAXXZ   00409c90 f   detailobjects.obj
 0001:00009040       ?EmitDetailObjects@@YAXXZ  0040a040 f   detailobjects.obj
 0001:00009070       ?InsertBefore@?$CUtlVector@UDetailObject_t@@V?$CUtlMemory@UDetailObject_t@@H@@@@QAEHH@Z 0040a070 f i detailobjects.obj
 0001:00009100       ?RemoveAll@?$CUtlVector@UDetailObject_t@@V?$CUtlMemory@UDetailObject_t@@H@@@@QAEXXZ 0040a100 f i detailobjects.obj
 0001:00009270       ?LoadEmitDetailObjectDictionary@@YAXPBD@Z 0040a270 f   detailobjects.obj
 0001:000092c0       ??1?$CUtlVector@UDetailObject_t@@V?$CUtlMemory@UDetailObject_t@@H@@@@QAE@XZ 0040a2c0 f i detailobjects.obj
 0001:00009320       ??9CVertIndex@@QBE_NABV0@@Z 0040a320 f i disp_common.obj
 0001:00009350       ?VectorMin@@YAXABVVector@@0AAV1@@Z 0040a350 f i disp_common.obj
 0001:000093b0       ?VectorMax@@YAXABVVector@@0AAV1@@Z 0040a3b0 f i disp_common.obj
 0001:00009410       ?SetInvalid@CDispNeighbor@@QAEXXZ 0040a410 f i disp_common.obj
 0001:00009420       ?SetInvalid@CDispCornerNeighbors@@QAEXXZ 0040a420 f i disp_common.obj
 0001:00009430       ?GetPoint@CCoreDispSurface@@QBEXHAAVVector@@@Z 0040a430 f i disp_common.obj
 0001:00009460       ?GetSurface@CCoreDispInfo@@QAEPAVCCoreDispSurface@@XZ 0040a460 f i disp_common.obj
 0001:000094c0       ?GetEdgeIndexFromPoint@@YAHABVCVertIndex@@H@Z 0040a4c0 f   disp_common.obj
 0001:00009510       ?GetSubNeighborIndex@@YAHPAVCDispUtilsHelper@@HABVCVertIndex@@@Z 0040a510 f   disp_common.obj
 0001:00009590       ?SetupSpan@@YAXHHW4NeighborSpan@@AAVCVertIndex@@1@Z 0040a590 f   disp_common.obj
 0001:00009650       ?ClearNeighborData@@YAXPAVCCoreDispInfo@@@Z 0040a650 f   disp_common.obj
 0001:00009690       ?GetDispBox@@YAXPAVCCoreDispInfo@@AAVCDispBox@@@Z 0040a690 f   disp_common.obj
 0001:00009760       ?FindEdge@@YA_NPAVCCoreDispInfo@@ABVVector@@1AAH@Z 0040a760 f   disp_common.obj
 0001:00009820       ?AddNeighbor@@YAXPAVCCoreDispInfo@@HHW4NeighborSpan@@0H1@Z 0040a820 f   disp_common.obj
 0001:00009910       ?SetupEdgeNeighbors@@YAXPAVCCoreDispInfo@@0@Z 0040a910 f   disp_common.obj
 0001:00009b20       ?HasEdgeNeighbor@@YA_NPBVCCoreDispInfo@@H@Z 0040ab20 f   disp_common.obj
 0001:00009b90       ?IsCorner@@YAHABVCVertIndex@@H@Z 0040ab90 f   disp_common.obj
 0001:00009be0       ?TransformIntoSubNeighbor@@YAPAVCDispUtilsHelper@@PAV1@HHABVCVertIndex@@AAV2@@Z 0040abe0 f   disp_common.obj
 0001:00009cf0       ?TransformIntoNeighbor@@YAPAVCDispUtilsHelper@@PAV1@HABVCVertIndex@@AAV2@@Z 0040acf0 f   disp_common.obj
 0001:00009d50       ?SetupCornerNeighbors@@YAXPAVCCoreDispInfo@@0PAH@Z 0040ad50 f   disp_common.obj
 0001:00009ef0       ?VerifyNeighborVertConnection@@YA_NPAVCDispUtilsHelper@@ABVCVertIndex@@PBV1@1H@Z 0040aef0 f   disp_common.obj
 0001:00009fb0       ?SetupEdgeIncrements@@YAPAVCDispUtilsHelper@@PAV1@HHAAVCVertIndex@@111AAH2@Z 0040afb0 f   disp_common.obj
 0001:0000a140       ?Next@CDispEdgeIterator@@QAE_NXZ 0040b140 f   disp_common.obj
 0001:0000a200       ?VerifyNeighborConnections@@YAXPAPAVCCoreDispInfo@@H@Z 0040b200 f   disp_common.obj
 0001:0000a3e0       ?IsVertAllowed@@YA_NPAVCDispUtilsHelper@@ABVCVertIndex@@H@Z 0040b3e0 f   disp_common.obj
 0001:0000a500       ?UnallowVerts_R@@YAXPAVCDispUtilsHelper@@ABVCVertIndex@@AAH@Z 0040b500 f   disp_common.obj
 0001:0000a5a0       ?DisableUnallowedVerts_R@@YAXPAVCDispUtilsHelper@@ABVCVertIndex@@HAAH@Z 0040b5a0 f   disp_common.obj
 0001:0000a650       ?SetupAllowedVerts@@YAXPAPAVCCoreDispInfo@@H@Z 0040b650 f   disp_common.obj
 0001:0000a6f0       ?InsertMultipleBefore@?$CUtlVector@VCDispBox@@V?$CUtlMemory@VCDispBox@@H@@@@QAEHHHPBVCDispBox@@@Z 0040b6f0 f i disp_common.obj
 0001:0000a8b0       ?FindNeighboringDispSurfs@@YAXPAPAVCCoreDispInfo@@H@Z 0040b8b0 f   disp_common.obj
 0001:0000aa40       ?GetBoundingBox@CCoreDispNode@@QAEXAAVVector@@0@Z 0040ba40 f i disp_ivp.obj
 0001:0000aa70       ?Disp_GridIndex@@YAHPAVCCoreDispInfo@@@Z 0040ba70 f   disp_ivp.obj
 0001:0000aae0       ?GetTrianglesInSphere@CDispMeshEvent@@UAEXPAXABVVector@@MPAUvirtualmeshtrianglelist_t@@@Z 0040bae0 f   disp_ivp.obj
 0001:0000ab20       ?Grow@?$CUtlMemory@UResourceMemorySection@CVTFTexture@@H@@QAEXH@Z 0040bb20 f i vtf:vtf.obj
 0001:0000ab20       ?Grow@?$CUtlMemory@Udoccluderpolydata_t@@H@@QAEXH@Z 0040bb20 f i vbsp.obj
 0001:0000ab20       ?Grow@?$CUtlMemory@VVector@@H@@QAEXH@Z 0040bb20 f i disp_ivp.obj
 0001:0000abc0       ?Grow@?$CUtlMemory@UDetailObjectGroup_t@@H@@QAEXH@Z 0040bbc0 f i detailobjects.obj
 0001:0000abc0       ?Grow@?$CUtlMemory@UfileList_t@@H@@QAEXH@Z 0040bbc0 f i scriplib.obj
 0001:0000abc0       ?Grow@?$CUtlMemory@Udisp_grid_t@@H@@QAEXH@Z 0040bbc0 f i disp_ivp.obj
 0001:0000abc0       ?Grow@?$CUtlMemory@U?$UtlRBTreeNode_t@UNode_t@?$CUtlMap@PBDHH@@H@@H@@QAEXH@Z 0040bbc0 f i writebsp.obj
 0001:0000abc0       ?Grow@?$CUtlMemory@VCDispBox@@H@@QAEXH@Z 0040bbc0 f i disp_common.obj
 0001:0000ac60       ?GetVirtualMesh@CDispMeshEvent@@UAEXPAXPAUvirtualmeshlist_t@@@Z 0040bc60 f   disp_ivp.obj
 0001:0000acc0       ?GetWorldspaceBounds@CDispMeshEvent@@UAEXPAXPAVVector@@1@Z 0040bcc0 f   disp_ivp.obj
 0001:0000ad10       ??$PutObjects@Udphysdisp_t@@@CUtlBuffer@@QAEXPAUdphysdisp_t@@H@Z 0040bd10 f i disp_ivp.obj
 0001:0000ad80       ?InsertMultipleBefore@?$CUtlVector@DV?$CUtlMemory@DH@@@@QAEHHHPBD@Z 0040bd80 f i disp_ivp.obj
 0001:0000ae10       ?InsertMultipleBefore@?$CUtlVector@VVector@@V?$CUtlMemory@VVector@@H@@@@QAEHHHPBVVector@@@Z 0040be10 f i disp_ivp.obj
 0001:0000af60       ?InsertBefore@?$CUtlVector@UStaticPropLeafLump_t@@V?$CUtlMemory@UStaticPropLeafLump_t@@H@@@@QAEHHABUStaticPropLeafLump_t@@@Z 0040bf60 f i staticprop.obj
 0001:0000af60       ?InsertBefore@?$CUtlVector@GV?$CUtlMemory@GH@@@@QAEHHABG@Z 0040bf60 f i disp_ivp.obj
 0001:0000afd0       ??0CDispMeshEvent@@QAE@PAGHPAVCCoreDispInfo@@@Z 0040bfd0 f   disp_ivp.obj
 0001:0000b180       ??$InternalEndTriangle@VCVBSPTesselateHelper@@@@YAXPAVCVBSPTesselateHelper@@ABVCVertIndex@@AAH@Z 0040c180 f i disp_ivp.obj
 0001:0000b1f0       ?InsertBefore@?$CUtlVector@UDetailObjectGroup_t@@V?$CUtlMemory@UDetailObjectGroup_t@@H@@@@QAEHH@Z 0040c1f0 f i detailobjects.obj
 0001:0000b1f0       ?InsertBefore@?$CUtlVector@Udisp_grid_t@@V?$CUtlMemory@Udisp_grid_t@@H@@@@QAEHH@Z 0040c1f0 f i disp_ivp.obj
 0001:0000b270       ??$TesselateDisplacementNode@VCVBSPTesselateHelper@@@@YAXPAVCVBSPTesselateHelper@@ABVCVertIndex@@HPAH@Z 0040c270 f i disp_ivp.obj
 0001:0000b3b0       ??$TesselateDisplacement_R@VCVBSPTesselateHelper@@@@YAXPAVCVBSPTesselateHelper@@ABVCVertIndex@@HH@Z 0040c3b0 f i disp_ivp.obj
 0001:0000b4e0       ?FindOrInsertGrid@@YAAAUdisp_grid_t@@H@Z 0040c4e0 f   disp_ivp.obj
 0001:0000b540       ??1?$CUtlVector@UDetailObjectGroup_t@@V?$CUtlMemory@UDetailObjectGroup_t@@H@@@@QAE@XZ 0040c540 f i detailobjects.obj
 0001:0000b540       ??1?$CUtlVector@Udisp_grid_t@@V?$CUtlMemory@Udisp_grid_t@@H@@@@QAE@XZ 0040c540 f i disp_ivp.obj
 0001:0000b540       ??1?$CUtlVector@Uclusterlist_t@@V?$CUtlMemory@Uclusterlist_t@@H@@@@QAE@XZ 0040c540 f i bsplib.obj
 0001:0000b5a0       ?Disp_AddCollisionModels@@YAXAAV?$CUtlVector@PAVCPhysCollisionEntry@@V?$CUtlMemory@PAVCPhysCollisionEntry@@H@@@@PAUdmodel_t@@H@Z 0040c5a0 f   disp_ivp.obj
 0001:0000bac0       ?Disp_BuildVirtualMesh@@YAXH@Z 0040cac0 f   disp_ivp.obj
 0001:0000c650       ?GetPowerInfo@@YAPBVCPowerInfo@@H@Z 0040d650 f   disp_powerinfo.obj
 0001:0000c660       ?GetCornerPointIndex@CPowerInfo@@QBEABVCVertIndex@@H@Z 0040d660 f   disp_powerinfo.obj
 0001:0000c670       ??0CVertInfo@@QAE@XZ       0040d670 f   disp_powerinfo.obj
 0001:0000c830       ?InitPowerInfo@@YAXPAVCPowerInfo@@H@Z 0040d830 f   disp_powerinfo.obj
 0001:0000cde0       ??0CPowerInfoInitializer@@QAE@XZ 0040dde0 f i disp_powerinfo.obj
 0001:0000ce20       ?Vector2DCopy@@YAXABVVector2D@@AAV1@@Z 0040de20 f i disp_vbsp.obj
 0001:0000ce40       ?GetBarycentricCoords2D@@YAXABVVector2D@@000QAM@Z 0040de40 f i disp_vbsp.obj
 0001:0000cee0       ?GetSize@CCoreDispInfo@@QBEHXZ 0040dee0 f i disp_vbsp.obj
 0001:0000cf00       ?GetBarycentricCoordsFromLightmapCoords@@YA_NQAVVector2D@@ABV1@QAM@Z 0040df00 f   disp_vbsp.obj
 0001:0000cf80       ?FindTriIndexMapByUV@@YA_NPAVCCoreDispInfo@@ABVVector2D@@AAHQAM@Z 0040df80 f   disp_vbsp.obj
 0001:0000d070       ?GetDispInfoEntityNum@@YAHPAUmapdispinfo_t@@@Z 0040e070 f   disp_vbsp.obj
 0001:0000d080       ?ExportCoreDispNeighborData@@YAXPBVCCoreDispInfo@@PAVddispinfo_t@@@Z 0040e080 f   disp_vbsp.obj
 0001:0000d170       ?DispGetFaceInfo@@YAXPAUmapbrush_t@@@Z 0040e170 f   disp_vbsp.obj
 0001:0000d270       ?HasDispInfo@@YA_NPAUmapbrush_t@@@Z 0040e270 f   disp_vbsp.obj
 0001:0000d2a0       ??4ddispinfo_t@@QAEAAV0@ABV0@@Z 0040e2a0 f i disp_vbsp.obj
 0001:0000d410       ?Grow@?$CUtlMemory@Vddispinfo_t@@H@@QAEXH@Z 0040e410 f i disp_vbsp.obj
 0001:0000d4c0       ?Grow@?$CUtlMemory@DH@@QAEXH@Z 0040e4c0 f i disp_ivp.obj
 0001:0000d4c0       ?Grow@?$CUtlMemory@_NH@@QAEXH@Z 0040e4c0 f i disp_vbsp.obj
 0001:0000d4c0       ?Grow@?$CUtlMemory@EH@@QAEXH@Z 0040e4c0 f i disp_vbsp.obj
 0001:0000d570       ?ExportCoreDispAllowedVertList@@YAXPBVCCoreDispInfo@@PAVddispinfo_t@@@Z 0040e570 f   disp_vbsp.obj
 0001:0000d600       ?FindEnclosingTri@@YA_NABVVector2D@@AAV?$CUtlVector@VVector2D@@V?$CUtlMemory@VVector2D@@H@@@@AAV?$CUtlVector@GV?$CUtlMemory@GH@@@@PAHQAM@Z 0040e600 f   disp_vbsp.obj
 0001:0000d6c0       ?InsertMultipleBefore@?$CUtlVector@Vddispinfo_t@@V?$CUtlMemory@Vddispinfo_t@@H@@@@QAEHHHPBVddispinfo_t@@@Z 0040e6c0 f i disp_vbsp.obj
 0001:0000d770       ?InsertMultipleBefore@?$CUtlVector@VVector2D@@V?$CUtlMemory@VVector2D@@H@@@@QAEHHHPBVVector2D@@@Z 0040e770 f i disp_vbsp.obj
 0001:0000d890       ?InsertMultipleBefore@?$CUtlVector@VCDispVert@@V?$CUtlMemory@VCDispVert@@H@@@@QAEHHHPBVCDispVert@@@Z 0040e890 f i disp_vbsp.obj
 0001:0000da30       ?CalculateLightmapSamplePositions@@YAXPAVCCoreDispInfo@@PBUdface_t@@AAV?$CUtlVector@EV?$CUtlMemory@EH@@@@@Z 0040ea30 f   disp_vbsp.obj
 0001:0000de00       ?DispMapToCoreDispInfo@@YAXPAUmapdispinfo_t@@PAVCCoreDispInfo@@PAUdface_t@@PAH@Z 0040ee00 f   disp_vbsp.obj
 0001:0000e280       ?ComputeDispInfoBounds@@YAXHAAVVector@@0@Z 0040f280 f   disp_vbsp.obj
 0001:0000e310       ?EmitInitialDispInfos@@YAXXZ 0040f310 f   disp_vbsp.obj
 0001:0000e620       ?SnapRemainingVertsToSurface@@YAXPAVCCoreDispInfo@@PAVddispinfo_t@@@Z 0040f620 f   disp_vbsp.obj
 0001:0000ea10       ?EmitDispLMAlphaAndNeighbors@@YAXXZ 0040fa10 f   disp_vbsp.obj
 0001:0000edd0       ?GetVertexnum@@YAHAAVVector@@@Z 0040fdd0 f   faces.obj
 0001:0000ef90       ?FindEdgeVerts@@YAXAAVVector@@0@Z 0040ff90 f   faces.obj
 0001:0000f080       ?TestEdge@@YAXMMHHH@Z      00410080 f   faces.obj
 0001:0000f240       ?AllocFace@@YAPAUface_t@@XZ 00410240 f   faces.obj
 0001:0000f280       ?NewFaceFromFace@@YAPAUface_t@@PAU1@@Z 00410280 f   faces.obj
 0001:0000f2e0       ?FreeFace@@YAXPAUface_t@@@Z 004102e0 f   faces.obj
 0001:0000f310       ?FreeFaceList@@YAXPAUface_t@@@Z 00410310 f   faces.obj
 0001:0000f350       ?TryMergeWinding@@YAPAUwinding_t@@PAU1@0AAVVector@@@Z 00410350 f   faces.obj
 0001:0000f6e0       ?FaceOnWaterBrush@@YA_NPAUface_t@@@Z 004106e0 f   faces.obj
 0001:0000f700       ?FaceFromSuperverts@@YAXPAPAUface_t@@PAU1@H@Z 00410700 f   faces.obj
 0001:0000f8a0       ?EmitFaceVertexes@@YAXPAPAUface_t@@PAU1@@Z 004108a0 f   faces.obj
 0001:0000f990       ?EmitNodeFaceVertexes_r@@YAXPAUnode_t@@@Z 00410990 f   faces.obj
 0001:0000f9e0       ?Grow@?$CUtlMemory@VVector2D@@H@@QAEXH@Z 004109e0 f i disp_vbsp.obj
 0001:0000f9e0       ?Grow@?$CUtlMemory@Uface_vert_table_t@@H@@QAEXH@Z 004109e0 f i faces.obj
 0001:0000f9e0       ?Grow@?$CUtlMemory@UentitySideList_t@@H@@QAEXH@Z 004109e0 f i worldvertextransitionfixup.obj
 0001:0000f9e0       ?Grow@?$CUtlMemory@UResourceEntryInfo@@H@@QAEXH@Z 004109e0 f i vtf:vtf.obj
 0001:0000fa90       ?IntSort@@YAXAAV?$CUtlVector@HV?$CUtlMemory@HH@@@@@Z 00410a90 f   faces.obj
 0001:0000fae0       ?SubdivideFace@@YAXPAPAUface_t@@PAU1@@Z 00410ae0 f   faces.obj
 0001:0000fdd0       ?SubdivideFaceList@@YAXPAPAUface_t@@@Z 00410dd0 f   faces.obj
 0001:0000ff60       ?FaceFromPortal@@YAPAUface_t@@PAUportal_t@@H@Z 00410f60 f   faces.obj
 0001:000100f0       ?GetEdge2_InitOptimizedList@@YAXXZ 004110f0 f   faces.obj
 0001:00010120       ?OverlaysAreEqual@@YA_NPAUface_t@@0@Z 00411120 f   faces.obj
 0001:000101a0       ?TryMerge@@YAPAUface_t@@PAU1@0AAVVector@@@Z 004111a0 f   faces.obj
 0001:00010270       ?MergeFaceList@@YAXPAPAUface_t@@@Z 00411270 f   faces.obj
 0001:00010300       ?MakeFaces_r@@YAXPAUnode_t@@@Z 00411300 f   faces.obj
 0001:000103b0       ?MakeFaces@@YAXPAUnode_t@@@Z 004113b0 f   faces.obj
 0001:00010410       ?InsertMultipleBefore@?$CUtlVector@Uface_vert_table_t@@V?$CUtlMemory@Uface_vert_table_t@@H@@@@QAEHHHPBUface_vert_table_t@@@Z 00411410 f i faces.obj
 0001:000104e0       ?Triangulate_r@@YAXAAV?$CUtlVector@HV?$CUtlMemory@HH@@@@ABV1@ABV?$CUtlVector@Uface_vert_table_t@@V?$CUtlMemory@Uface_vert_table_t@@H@@@@@Z 004114e0 f   faces.obj
 0001:00010890       ?FixFaceEdges@@YAXPAPAUface_t@@PAU1@@Z 00411890 f   faces.obj
 0001:00010d10       ?FixEdges_r@@YAXPAUnode_t@@@Z 00411d10 f   faces.obj
 0001:00010d60       ?FixLeafFaceEdges@@YAXPAPAUface_t@@@Z 00411d60 f   faces.obj
 0001:00010d90       ?FixTjuncs@@YAPAUface_t@@PAUnode_t@@PAU1@@Z 00411d90 f   faces.obj
 0001:00010f10       ?AddEdge@@YAHHHPAUface_t@@@Z 00411f10 f   faces.obj
 0001:00010fc0       ?GetEdge2@@YAHHHPAUface_t@@@Z 00411fc0 f   faces.obj
 0001:00011060       ?OutputWinding@@YAXPAUwinding_t@@PAX@Z 00412060 f   glfile.obj
 0001:00011110       ?OutputPortal@@YAXPAUportal_t@@PAX@Z 00412110 f   glfile.obj
 0001:00011180       ?WriteGLView_r@@YAXPAUnode_t@@PAX@Z 00412180 f   glfile.obj
 0001:000111d0       ?WriteGLView@@YAXPAUtree_t@@PAD@Z 004121d0 f   glfile.obj
 0001:00011280       ?DumpCollideToGlView@@YAXPAVCPhysCollide@@PBD@Z 00412280 f   ivp.obj
 0001:000113c0       ??0CPhysCollisionEntryStaticMesh@@QAE@PAVCPhysCollide@@PBD@Z 004123c0 f   ivp.obj
 0001:000113e0       ??0CPhysCollisionEntryFluid@@QAE@PAVCPhysCollide@@PBDMABVVector@@MH@Z 004123e0 f   ivp.obj
 0001:00011460       ?GetFirstBrushSide@CPlaneList@@QAEHXZ 00412460 f   ivp.obj
 0001:000114d0       ?ZipFileLessFunc@CZipEntry@CZipFile@@SA_NABV12@0@Z 004124d0 f   zip_utils.obj
 0001:000114d0       ?WaterLessFunc@@YA_NABUWaterTexInfo@@0@Z 004124d0 f   ivp.obj
 0001:000114f0       ?GetWaterTextureName@@YAXPBD0HPAD@Z 004124f0 f   ivp.obj
 0001:00011550       ?EmitWaterMaterialFile@@YAXPAUWaterTexInfo@@@Z 00412550 f   ivp.obj
 0001:00011730       ?FirstWaterTexinfo@@YAHPAUbspbrush_t@@H@Z 00412730 f   ivp.obj
 0001:00011930       ?Links@?$CUtlRBTree@UWaterTexInfo@@HP6A_NABU1@0@ZV?$CUtlMemory@U?$UtlRBTreeNode_t@UWaterTexInfo@@H@@H@@@@IBEABU?$UtlRBTreeLinks_t@H@@H@Z 00412930 f i ivp.obj
 0001:00011980       ?Grow@?$CUtlMemory@U?$UtlRBTreeNode_t@VCZipEntry@CZipFile@@H@@H@@QAEXH@Z 00412980 f i zip_utils.obj
 0001:00011980       ?Grow@?$CUtlMemory@Uwaterleaf_t@@H@@QAEXH@Z 00412980 f i ivp.obj
 0001:00011a30       ?Grow@?$CUtlMemory@UDetailObject_t@@H@@QAEXH@Z 00412a30 f i detailobjects.obj
 0001:00011a30       ?Grow@?$CUtlMemory@U?$UtlRBTreeNode_t@UWaterTexInfo@@H@@H@@QAEXH@Z 00412a30 f i ivp.obj
 0001:00011a30       ?Grow@?$CUtlMemory@Udleafambientlighting_t@@H@@QAEXH@Z 00412a30 f i bsplib.obj
 0001:00011af0       ?Grow@?$CUtlMemory@UDetailModel_t@@H@@QAEXH@Z 00412af0 f i detailobjects.obj
 0001:00011af0       ?Grow@?$CUtlMemory@Uwatermodel_t@@H@@QAEXH@Z 00412af0 f i ivp.obj
 0001:00011ba0       ?DumpCollideToPHY@@YAXPAVCPhysCollide@@PAVCTextBuffer@@PBD@Z 00412ba0 f   ivp.obj
 0001:00011c80       ?DumpCollideFileName@CPhysCollisionEntry@@IAEXPBDHPAVCTextBuffer@@@Z 00412c80 f   ivp.obj
 0001:00011cf0       ?DumpCollide@CPhysCollisionEntrySolid@@UAEXPAVCTextBuffer@@HH@Z 00412cf0 f   ivp.obj
 0001:00011d10       ?DumpCollide@CPhysCollisionEntryStaticSolid@@UAEXPAVCTextBuffer@@HH@Z 00412d10 f   ivp.obj
 0001:00011d60       ?DumpCollide@CPhysCollisionEntryStaticMesh@@UAEXPAVCTextBuffer@@HH@Z 00412d60 f   ivp.obj
 0001:00011db0       ?DumpCollide@CPhysCollisionEntryFluid@@UAEXPAVCTextBuffer@@HH@Z 00412db0 f   ivp.obj
 0001:00011e00       ?IsLeafReferenced@CPlaneList@@QAE_NH@Z 00412e00 f   ivp.obj
 0001:00011f70       ?FindInsertionPosition@?$CUtlRBTree@UWaterTexInfo@@HP6A_NABU1@0@ZV?$CUtlMemory@U?$UtlRBTreeNode_t@UWaterTexInfo@@H@@H@@@@IAEXABUWaterTexInfo@@AAHAA_N@Z 00412f70 f i ivp.obj
 0001:00012060       ?NewNode@?$CUtlRBTree@UWaterTexInfo@@HP6A_NABU1@0@ZV?$CUtlMemory@U?$UtlRBTreeNode_t@UWaterTexInfo@@H@@H@@@@QAEHXZ 00413060 f i ivp.obj
 0001:00012150       ?RotateLeft@?$CUtlRBTree@UWaterTexInfo@@HP6A_NABU1@0@ZV?$CUtlMemory@U?$UtlRBTreeNode_t@UWaterTexInfo@@H@@H@@@@IAEXH@Z 00413150 f i ivp.obj
 0001:00012240       ?RotateRight@?$CUtlRBTree@UWaterTexInfo@@HP6A_NABU1@0@ZV?$CUtlMemory@U?$UtlRBTreeNode_t@UWaterTexInfo@@H@@H@@@@IAEXH@Z 00413240 f i ivp.obj
 0001:00012340       ?Find@?$CUtlRBTree@UWaterTexInfo@@HP6A_NABU1@0@ZV?$CUtlMemory@U?$UtlRBTreeNode_t@UWaterTexInfo@@H@@H@@@@QBEHABUWaterTexInfo@@@Z 00413340 f i ivp.obj
 0001:00012430       ?InsertBefore@?$CUtlVector@Uwaterleaf_t@@V?$CUtlMemory@Uwaterleaf_t@@H@@@@QAEHHABUwaterleaf_t@@@Z 00413430 f i ivp.obj
 0001:000124a0       ?InsertBefore@?$CUtlVector@PAUnode_t@@V?$CUtlMemory@PAUnode_t@@H@@@@QAEHHABQAUnode_t@@@Z 004134a0 f i ivp.obj
 0001:000124a0       ?InsertBefore@?$CUtlVector@PAUStringPool_t@CUtlSymbolTable@@V?$CUtlMemory@PAUStringPool_t@CUtlSymbolTable@@H@@@@QAEHHABQAUStringPool_t@CUtlSymbolTable@@@Z 004134a0 f i tier1:utlsymbol.obj
 0001:000124a0       ?InsertBefore@?$CUtlVector@PAUbspbrush_t@@V?$CUtlMemory@PAUbspbrush_t@@H@@@@QAEHHABQAUbspbrush_t@@@Z 004134a0 f i detail.obj
 0001:000124a0       ?InsertBefore@?$CUtlVector@PAVCPhysConvex@@V?$CUtlMemory@PAVCPhysConvex@@H@@@@QAEHHABQAVCPhysConvex@@@Z 004134a0 f i ivp.obj
 0001:000124a0       ?InsertBefore@?$CUtlVector@HV?$CUtlMemory@HH@@@@QAEHHABH@Z 004134a0 f i cubemap.obj
 0001:000124a0       ?InsertBefore@?$CUtlVector@PAUportal_t@@V?$CUtlMemory@PAUportal_t@@H@@@@QAEHHABQAUportal_t@@@Z 004134a0 f i portals.obj
 0001:000124a0       ?InsertBefore@?$CUtlVector@PAVKeyValues@@V?$CUtlMemory@PAVKeyValues@@H@@@@QAEHHABQAVKeyValues@@@Z 004134a0 f i tier1:KeyValues.obj
 0001:00012510       ?InsertBefore@?$CUtlVector@Uwatermodel_t@@V?$CUtlMemory@Uwatermodel_t@@H@@@@QAEHHABUwatermodel_t@@@Z 00413510 f i ivp.obj
 0001:00012590       ?RemoveAll@?$CUtlRBTree@UWaterTexInfo@@HP6A_NABU1@0@ZV?$CUtlMemory@U?$UtlRBTreeNode_t@UWaterTexInfo@@H@@H@@@@QAEXXZ 00413590 f i ivp.obj
 0001:00012620       ?InsertRebalance@?$CUtlRBTree@UWaterTexInfo@@HP6A_NABU1@0@ZV?$CUtlMemory@U?$UtlRBTreeNode_t@UWaterTexInfo@@H@@H@@@@IAEXH@Z 00413620 f i ivp.obj
 0001:00012c40       ?LinkToParent@?$CUtlRBTree@UWaterTexInfo@@HP6A_NABU1@0@ZV?$CUtlMemory@U?$UtlRBTreeNode_t@UWaterTexInfo@@H@@H@@@@IAEXHH_N@Z 00413c40 f i ivp.obj
 0001:00012cb0       ?CopyData@CTextBuffer@@AAEXPBDH@Z 00413cb0 f   ivp.obj
 0001:00012db0       ?RemapWorldMaterial@@YAHH@Z 00413db0 f   ivp.obj
 0001:00012dd0       ??0CPlaneList@@QAE@MM@Z    00413dd0 f   ivp.obj
 0001:00012e60       ?BuildConvexForBrush@CPlaneList@@AAEPAVCPhysConvex@@HMPAVCPhysCollide@@M@Z 00413e60 f   ivp.obj
 0001:00013060       ?AddBrushes@CPlaneList@@QAEHXZ 00414060 f   ivp.obj
 0001:00013170       ?EnumLeaves_r@@YAXAAV?$CUtlVector@PAUnode_t@@V?$CUtlMemory@PAUnode_t@@H@@@@PAUnode_t@@H@Z 00414170 f   ivp.obj
 0001:00013f00       ??1?$CUtlRBTree@UWaterTexInfo@@HP6A_NABU1@0@ZV?$CUtlMemory@U?$UtlRBTreeNode_t@UWaterTexInfo@@H@@H@@@@QAE@XZ 00414f00 f i ivp.obj
 0001:00013f60       ?WriteIntKey@CTextBuffer@@QAEXPBDH@Z 00414f60 f   ivp.obj
 0001:00013ff0       ?WriteFloatKey@CTextBuffer@@QAEXPBDM@Z 00414ff0 f   ivp.obj
 0001:00014090       ?WriteFloatArrayKey@CTextBuffer@@QAEXPBDPBMH@Z 00415090 f   ivp.obj
 0001:000141b0       ?CopyStringQuotes@CTextBuffer@@QAEXPBD@Z 004151b0 f   ivp.obj
 0001:00014280       ?WriteToTextBuffer@CPhysCollisionEntryStaticSolid@@UAEXPAVCTextBuffer@@HH@Z 00415280 f   ivp.obj
 0001:000142d0       ?WriteToTextBuffer@CPhysCollisionEntryStaticMesh@@UAEXPAVCTextBuffer@@HH@Z 004152d0 f   ivp.obj
 0001:00014310       ?EmitPhysCollision@@YAXXZ  00415310 f   ivp.obj
 0001:00014880       ?Insert@?$CUtlRBTree@UWaterTexInfo@@HP6A_NABU1@0@ZV?$CUtlMemory@U?$UtlRBTreeNode_t@UWaterTexInfo@@H@@H@@@@QAEHABUWaterTexInfo@@@Z 00415880 f i ivp.obj
 0001:00014900       ?WriteStringKey@CTextBuffer@@QAEXPBD0@Z 00415900 f   ivp.obj
 0001:000149c0       ?WriteToTextBuffer@CPhysCollisionEntrySolid@@UAEXPAVCTextBuffer@@HH@Z 004159c0 f   ivp.obj
 0001:00014a40       ?WriteToTextBuffer@CPhysCollisionEntryFluid@@UAEXPAVCTextBuffer@@HH@Z 00415a40 f   ivp.obj
 0001:00014b00       ?FindOrCreateWaterTexInfo@@YAHPAUtexinfo_s@@M@Z 00415b00 f   ivp.obj
 0001:00014c60       ?EmitWaterVolumesForBSP@@YAXPAUdmodel_t@@PAUnode_t@@@Z 00415c60 f   ivp.obj
 0001:00014fc0       ?LeakFile@@YAXPAUtree_t@@@Z 00415fc0 f   leakfile.obj
 0001:00015190       ?AreaportalLeakFile@@YAXPAUtree_t@@PAUportal_t@@1PAUnode_t@@@Z 00416190 f   leakfile.obj
 0001:00015620       ?LoadCmdLineFromFile@@YAXAAHAAPAPADPBD2@Z 00416620 f   loadcmdline.obj
 0001:00015700       ?DeleteCmdLine@@YAXHPAPAD@Z 00416700 f   loadcmdline.obj
 0001:00015740       ?ReportError@CMapError@@QAEXPBD@Z 00416740 f i map.obj
 0001:00015770       ?ReportWarning@CMapError@@QAEXPBD@Z 00416770 f i map.obj
 0001:00015790       ?PlaneTypeForNormal@@YAHAAVVector@@@Z 00416790 f   map.obj
 0001:00015850       ?SnapVector@@YA_NAAVVector@@@Z 00416850 f   map.obj
 0001:000158c0       ?SnapPlane@@YAXAAVVector@@AAMABV1@22@Z 004168c0 f   map.obj
 0001:00015980       ?BrushContents@@YAHPAUmapbrush_t@@@Z 00416980 f   map.obj
 0001:000159c0       ?IsAreaPortal@@YA_NPBD@Z   004169c0 f   map.obj
 0001:000159f0       ??4brush_texture_t@@QAEAAU0@ABU0@@Z 004169f0 f i map.obj
 0001:00015a70       ?MakeBrushWindings@@YAHPAUmapbrush_t@@@Z 00416a70 f   map.obj
 0001:00015c10       ?MoveBrushesToWorld@@YAXPAUentity_t@@@Z 00416c10 f   map.obj
 0001:00015cd0       ?RemoveContentsDetailFromEntity@@YAXPAUentity_t@@@Z 00416cd0 f   map.obj
 0001:00015d30       ?LoadDispDistancesKeyCallback@@YA?AW4ChunkFileResult_t@@PBD0PAUmapdispinfo_t@@@Z 00416d30 f   map.obj
 0001:00015df0       ?LoadDispInfoKeyCallback@@YA?AW4ChunkFileResult_t@@PBD0PAUmapdispinfo_t@@@Z 00416df0 f   map.obj
 0001:00015f40       ?LoadDispNormalsKeyCallback@@YA?AW4ChunkFileResult_t@@PBD0PAUmapdispinfo_t@@@Z 00416f40 f   map.obj
 0001:00016070       ?LoadDispOffsetsKeyCallback@@YA?AW4ChunkFileResult_t@@PBD0PAUmapdispinfo_t@@@Z 00417070 f   map.obj
 0001:000161a0       ?LoadDispAlphasKeyCallback@@YA?AW4ChunkFileResult_t@@PBD0PAUmapdispinfo_t@@@Z 004171a0 f   map.obj
 0001:00016260       ?LoadDispTriangleTagsKeyCallback@@YA?AW4ChunkFileResult_t@@PBD0PAUmapdispinfo_t@@@Z 00417260 f   map.obj
 0001:00016360       ?ConvertSideList@@YAXPAUentity_t@@PAD@Z 00417360 f   map.obj
 0001:000164d0       ?AddLadderKeys@@YAXPAUentity_t@@@Z 004174d0 f   map.obj
 0001:00016650       ?EntityByName@@YAPAUentity_t@@PBD@Z 00417650 f   map.obj
 0001:000166b0       ?ForceFuncAreaPortalWindowContents@@YAXXZ 004176b0 f   map.obj
 0001:000167c0       ?LoadSideKeyCallback@@YA?AW4ChunkFileResult_t@@PBD0PAULoadSide_t@@@Z 004177c0 f   map.obj
 0001:00016ae0       ?LoadConnectionsKeyCallback@@YA?AW4ChunkFileResult_t@@PBD0PAULoadEntity_t@@@Z 00417ae0 f   map.obj
 0001:00016ba0       ?LoadSolidKeyCallback@@YA?AW4ChunkFileResult_t@@PBD0PAUmapbrush_t@@@Z 00417ba0 f   map.obj
 0001:00016be0       ?LoadDispDistancesCallback@@YA?AW4ChunkFileResult_t@@PAVCChunkFile@@PAUmapdispinfo_t@@@Z 00417be0 f   map.obj
 0001:00016c00       ?LoadDispNormalsCallback@@YA?AW4ChunkFileResult_t@@PAVCChunkFile@@PAUmapdispinfo_t@@@Z 00417c00 f   map.obj
 0001:00016c20       ?LoadDispOffsetsCallback@@YA?AW4ChunkFileResult_t@@PAVCChunkFile@@PAUmapdispinfo_t@@@Z 00417c20 f   map.obj
 0001:00016c40       ?LoadDispAlphasCallback@@YA?AW4ChunkFileResult_t@@PAVCChunkFile@@PAUmapdispinfo_t@@@Z 00417c40 f   map.obj
 0001:00016c60       ?LoadDispTriangleTagsCallback@@YA?AW4ChunkFileResult_t@@PAVCChunkFile@@PAUmapdispinfo_t@@@Z 00417c60 f   map.obj
 0001:00016c80       ?LoadConnectionsCallback@@YA?AW4ChunkFileResult_t@@PAVCChunkFile@@PAULoadEntity_t@@@Z 00417c80 f   map.obj
 0001:00016ca0       ?Grow@?$CUtlMemory@Umapoverlay_t@@H@@QAEXH@Z 00417ca0 f i map.obj
 0001:00016d40       ?CreateNewFloatPlane@@YAHAAVVector@@M@Z 00417d40 f   map.obj
 0001:00016f60       ?FindFloatPlane@@YAHAAVVector@@M@Z 00417f60 f   map.obj
 0001:00017070       ?PlaneFromPoints@@YAHABVVector@@00@Z 00418070 f   map.obj
 0001:00017130       ?LoadDispInfoCallback@@YA?AW4ChunkFileResult_t@@PAVCChunkFile@@PAPAUmapdispinfo_t@@@Z 00418130 f   map.obj
 0001:00017240       ?LoadSideCallback@@YA?AW4ChunkFileResult_t@@PAVCChunkFile@@PAULoadSide_t@@@Z 00418240 f   map.obj
 0001:000174b0       ?HandleNoDynamicShadowsEnt@@YA?AW4ChunkFileResult_t@@PAUentity_t@@@Z 004184b0 f   map.obj
 0001:00017900       ?InsertBefore@?$CUtlVector@Umapoverlay_t@@V?$CUtlMemory@Umapoverlay_t@@H@@@@QAEHH@Z 00418900 f i map.obj
 0001:000179b0       ?AddBrushBevels@@YAXPAUmapbrush_t@@@Z 004189b0 f   map.obj
 0001:000181a0       ?LoadSolidCallback@@YA?AW4ChunkFileResult_t@@PAVCChunkFile@@PAULoadEntity_t@@@Z 004191a0 f   map.obj
 0001:00018490       ?LoadEntityCallback@@YA?AW4ChunkFileResult_t@@PAVCChunkFile@@H@Z 00419490 f   map.obj
 0001:00018a40       ?LoadMapFile@@YAXPBD@Z     00419a40 f   map.obj
 0001:00018d10       ?CreateMaterialPatchRecursive@@YAXPAVKeyValues@@0HPBUMaterialPatchInfo_t@@@Z 00419d10 f   materialpatch.obj
 0001:00018f60       ?Parent@?$CUtlRBTree@UNameTranslationLookup_t@@HP6A_NABU1@0@ZV?$CUtlMemory@U?$UtlRBTreeNode_t@UNameTranslationLookup_t@@H@@H@@@@QBEHH@Z 00419f60 f i materialpatch.obj
 0001:00018fb0       ?LeftChild@?$CUtlRBTree@UNameTranslationLookup_t@@HP6A_NABU1@0@ZV?$CUtlMemory@U?$UtlRBTreeNode_t@UNameTranslationLookup_t@@H@@H@@@@QBEHH@Z 00419fb0 f i materialpatch.obj
 0001:00019000       ?RightChild@?$CUtlRBTree@UNameTranslationLookup_t@@HP6A_NABU1@0@ZV?$CUtlMemory@U?$UtlRBTreeNode_t@UNameTranslationLookup_t@@H@@H@@@@QBEHH@Z 0041a000 f i materialpatch.obj
 0001:00019050       ?FindInsertionPosition@?$CUtlRBTree@UNameTranslationLookup_t@@HP6A_NABU1@0@ZV?$CUtlMemory@U?$UtlRBTreeNode_t@UNameTranslationLookup_t@@H@@H@@@@IAEXABUNameTranslationLookup_t@@AAHAA_N@Z 0041a050 f i materialpatch.obj
 0001:00019140       ?NewNode@?$CUtlRBTree@UNameTranslationLookup_t@@HP6A_NABU1@0@ZV?$CUtlMemory@U?$UtlRBTreeNode_t@UNameTranslationLookup_t@@H@@H@@@@QAEHXZ 0041a140 f i materialpatch.obj
 0001:00019220       ?IsLeftChild@?$CUtlRBTree@UNameTranslationLookup_t@@HP6A_NABU1@0@ZV?$CUtlMemory@U?$UtlRBTreeNode_t@UNameTranslationLookup_t@@H@@H@@@@QBE_NH@Z 0041a220 f i materialpatch.obj
 0001:00019290       ?RotateLeft@?$CUtlRBTree@UNameTranslationLookup_t@@HP6A_NABU1@0@ZV?$CUtlMemory@U?$UtlRBTreeNode_t@UNameTranslationLookup_t@@H@@H@@@@IAEXH@Z 0041a290 f i materialpatch.obj
 0001:000193c0       ?RotateRight@?$CUtlRBTree@UNameTranslationLookup_t@@HP6A_NABU1@0@ZV?$CUtlMemory@U?$UtlRBTreeNode_t@UNameTranslationLookup_t@@H@@H@@@@IAEXH@Z 0041a3c0 f i materialpatch.obj
 0001:000194c0       ?LoadKeyValuesFromPackOrFile@@YA_NPBDPAVKeyValues@@@Z 0041a4c0 f   materialpatch.obj
 0001:00019690       ?LoadMaterialKeyValues@@YAPAVKeyValues@@PBDI@Z 0041a690 f   materialpatch.obj
 0001:00019720       ?WriteMaterialKeyValuesToPak@@YAXPBDPAVKeyValues@@@Z 0041a720 f   materialpatch.obj
 0001:000197c0       ?GetValueFromPatchedMaterial@@YA_NPBD0PADH@Z 0041a7c0 f   materialpatch.obj
 0001:00019880       ?Find@?$CUtlRBTree@UNameTranslationLookup_t@@HP6A_NABU1@0@ZV?$CUtlMemory@U?$UtlRBTreeNode_t@UNameTranslationLookup_t@@H@@H@@@@QBEHABUNameTranslationLookup_t@@@Z 0041a880 f i materialpatch.obj
 0001:00019970       ?RemoveAll@?$CUtlRBTree@UNameTranslationLookup_t@@HP6A_NABU1@0@ZV?$CUtlMemory@U?$UtlRBTreeNode_t@UNameTranslationLookup_t@@H@@H@@@@QAEXXZ 0041a970 f i materialpatch.obj
 0001:00019a00       ?InsertRebalance@?$CUtlRBTree@UNameTranslationLookup_t@@HP6A_NABU1@0@ZV?$CUtlMemory@U?$UtlRBTreeNode_t@UNameTranslationLookup_t@@H@@H@@@@IAEXH@Z 0041aa00 f i materialpatch.obj
 0001:00019f40       ?GetOriginalMaterialNameForPatchedMaterial@@YAPBDPBD@Z 0041af40 f   materialpatch.obj
 0001:00019fd0       ?DoesMaterialHaveKey@@YA_NPBD0@Z 0041afd0 f   materialpatch.obj
 0001:0001a070       ?DoesMaterialHaveKeyValuePair@@YA_NPBD00@Z 0041b070 f   materialpatch.obj
 0001:0001a110       ?GetValueFromMaterial@@YA_NPBD0PADH@Z 0041b110 f   materialpatch.obj
 0001:0001a1d0       ?FindOriginalMaterial@@YAPAXPBDPA_N_N@Z 0041b1d0 f   materialpatch.obj
 0001:0001a200       ?LinkToParent@?$CUtlRBTree@UNameTranslationLookup_t@@HP6A_NABU1@0@ZV?$CUtlMemory@U?$UtlRBTreeNode_t@UNameTranslationLookup_t@@H@@H@@@@IAEXHH_N@Z 0041b200 f i materialpatch.obj
 0001:0001a270       ??1?$CUtlRBTree@UNameTranslationLookup_t@@HP6A_NABU1@0@ZV?$CUtlMemory@U?$UtlRBTreeNode_t@UNameTranslationLookup_t@@H@@H@@@@QAE@XZ 0041b270 f i materialpatch.obj
 0001:0001a2d0       ?Insert@?$CUtlRBTree@UNameTranslationLookup_t@@HP6A_NABU1@0@ZV?$CUtlMemory@U?$UtlRBTreeNode_t@UNameTranslationLookup_t@@H@@H@@@@QAEHABUNameTranslationLookup_t@@@Z 0041b2d0 f i materialpatch.obj
 0001:0001a330       ?AddNewTranslation@@YAXPBD0@Z 0041b330 f   materialpatch.obj
 0001:0001a390       ?CreateMaterialPatch@@YAXPBD0HPBUMaterialPatchInfo_t@@W4MaterialPatchType_t@@@Z 0041b390 f   materialpatch.obj
 0001:0001a580       ?CreateMaterialPatch@@YAXPBD000W4MaterialPatchType_t@@@Z 0041b580 f   materialpatch.obj
 0001:0001a5c0       ?LoadMaterialReplacementKeys@@YAXPBD0@Z 0041b5c0 f   materialsub.obj
 0001:0001a6f0       ?DeleteMaterialReplacementKeys@@YAXXZ 0041b6f0 f   materialsub.obj
 0001:0001a710       ?ReplaceMaterialName@@YAPBDPBD@Z 0041b710 f   materialsub.obj
 0001:0001a760       ?MakeModuleFileName@@YAPBDXZ 0041b760 f   memoverride.obj
 0001:0001a7f0       _calloc                    0041b7f0 f   memoverride.obj
 0001:0001a870       __calloc_base              0041b870 f   memoverride.obj
 0001:0001a8f0       __realloc_base             0041b8f0 f   memoverride.obj
 0001:0001a8f0       _realloc                   0041b8f0 f   memoverride.obj
 0001:0001a950       __recalloc_base            0041b950 f   memoverride.obj
 0001:0001a9d0       ??_U@YAPAXI@Z              0041b9d0 f   memoverride.obj
 0001:0001a9d0       ??2@YAPAXI@Z               0041b9d0 f   memoverride.obj
 0001:0001a9d0       _malloc                    0041b9d0 f   memoverride.obj
 0001:0001a9d0       __malloc_crt               0041b9d0 f   memoverride.obj
 0001:0001aa30       __calloc_crt               0041ba30 f   memoverride.obj
 0001:0001aa50       __realloc_crt              0041ba50 f   memoverride.obj
 0001:0001aa60       __recalloc_crt             0041ba60 f   memoverride.obj
 0001:0001aa80       __msize                    0041ba80 f   memoverride.obj
 0001:0001aaa0       __heap_init                0041baa0 f   memoverride.obj
 0001:0001aab0       ??_V@YAXPAX@Z              0041bab0 f   memoverride.obj
 0001:0001aab0       ??3@YAXPAX@Z               0041bab0 f   memoverride.obj
 0001:0001aab0       _free                      0041bab0 f   memoverride.obj
 0001:0001aad0       __strdup                   0041bad0 f   memoverride.obj
 0001:0001ab50       ??1bad_alloc@std@@UAE@XZ   0041bb50 f i mstristrip.obj
 0001:0001ab60       ??_Gbad_alloc@std@@UAEPAXI@Z 0041bb60 f i mstristrip.obj
 0001:0001ab60       ??_Ebad_alloc@std@@UAEPAXI@Z 0041bb60 f i mstristrip.obj
 0001:0001ab90       ??$_Allocate@D@std@@YAPADIPAD@Z 0041bb90 f i mstristrip.obj
 0001:0001abf0       ??0bad_alloc@std@@QAE@ABV01@@Z 0041bbf0 f i mstristrip.obj
 0001:0001ac10       ?allocate@?$allocator@D@std@@QAEPADI@Z 0041bc10 f i mstristrip.obj
 0001:0001ac30       ?_Tidy@?$basic_string@DU?$char_traits@D@std@@V?$allocator@D@2@@std@@IAEX_NI@Z 0041bc30 f i mstristrip.obj
 0001:0001ac80       ?erase@?$basic_string@DU?$char_traits@D@std@@V?$allocator@D@2@@std@@QAEAAV12@II@Z 0041bc80 f i mstristrip.obj
 0001:0001ad10       ?_Copy@?$basic_string@DU?$char_traits@D@std@@V?$allocator@D@2@@std@@IAEXII@Z 0041bd10 f i mstristrip.obj
 0001:0001ae60       ??1?$basic_string@DU?$char_traits@D@std@@V?$allocator@D@2@@std@@QAE@XZ 0041be60 f i mstristrip.obj
 0001:0001ae90       ??1logic_error@std@@UAE@XZ 0041be90 f i mstristrip.obj
 0001:0001ae90       ??1length_error@std@@UAE@XZ 0041be90 f i mstristrip.obj
 0001:0001aed0       ?what@logic_error@std@@UBEPBDXZ 0041bed0 f i mstristrip.obj
 0001:0001aed0       ?what@runtime_error@std@@UBEPBDXZ 0041bed0 f i chunkfile.obj
 0001:0001aee0       ??_Glength_error@std@@UAEPAXI@Z 0041bee0 f i mstristrip.obj
 0001:0001aee0       ??_Glogic_error@std@@UAEPAXI@Z 0041bee0 f i mstristrip.obj
 0001:0001aee0       ??_Elength_error@std@@UAEPAXI@Z 0041bee0 f i mstristrip.obj
 0001:0001aee0       ??_Elogic_error@std@@UAEPAXI@Z 0041bee0 f i mstristrip.obj
 0001:0001af30       ?assign@?$basic_string@DU?$char_traits@D@std@@V?$allocator@D@2@@std@@QAEAAV12@ABV12@II@Z 0041bf30 f i mstristrip.obj
 0001:0001b010       ?assign@?$basic_string@DU?$char_traits@D@std@@V?$allocator@D@2@@std@@QAEAAV12@PBDI@Z 0041c010 f i mstristrip.obj
 0001:0001b0e0       ?assign@?$basic_string@DU?$char_traits@D@std@@V?$allocator@D@2@@std@@QAEAAV12@PBD@Z 0041c0e0 f i mstristrip.obj
 0001:0001b110       ??0logic_error@std@@QAE@ABV?$basic_string@DU?$char_traits@D@std@@V?$allocator@D@2@@1@@Z 0041c110 f i mstristrip.obj
 0001:0001b150       ??0?$basic_string@DU?$char_traits@D@std@@V?$allocator@D@2@@std@@QAE@PBD@Z 0041c150 f i mstristrip.obj
 0001:0001b190       ??0logic_error@std@@QAE@ABV01@@Z 0041c190 f i mstristrip.obj
 0001:0001b1d0       ??0length_error@std@@QAE@ABV01@@Z 0041c1d0 f i mstristrip.obj
 0001:0001b210       ?SaveVertexNormals@@YAXXZ  0041c210 f   normals.obj
 0001:0001b300       ?Overlay_EmitOverlayFace@@YAXPAUmapoverlay_t@@@Z 0041c300 f   overlay.obj
 0001:0001b620       ?OverlayTransition_EmitOverlayFace@@YAXPAUmapoverlay_t@@@Z 0041c620 f   overlay.obj
 0001:0001b920       ?Overlay_EmitOverlayFaces@@YAXXZ 0041c920 f   overlay.obj
 0001:0001b950       ?OverlayTransition_EmitOverlayFaces@@YAXXZ 0041c950 f   overlay.obj
 0001:0001b980       ?Overlay_UpdateSideLists@@YAXXZ 0041c980 f   overlay.obj
 0001:0001bab0       ?OverlayTransition_UpdateSideLists@@YAXXZ 0041cab0 f   overlay.obj
 0001:0001bbe0       ?Overlay_AddFaceToLists@@YAXHPAUside_t@@@Z 0041cbe0 f   overlay.obj
 0001:0001bc50       ?OverlayTransition_AddFaceToLists@@YAXHPAUside_t@@@Z 0041cc50 f   overlay.obj
 0001:0001bce0       ?RemoveAll@?$CUtlVector@Umapoverlay_t@@V?$CUtlMemory@Umapoverlay_t@@H@@@@QAEXXZ 0041cce0 f i overlay.obj
 0001:0001be00       ?Overlay_GetFromEntity@@YAHPAUentity_t@@@Z 0041ce00 f   overlay.obj
 0001:0001c0f0       ??1?$CUtlVector@Umapoverlay_t@@V?$CUtlMemory@Umapoverlay_t@@H@@@@QAE@XZ 0041d0f0 f i overlay.obj
 0001:0001c150       ?GetPhysicsFactory@@YAP6APAXPBDPAH@ZXZ 0041d150 f   physdll.obj
 0001:0001c190       _PhysicsDLLPath            0041d190 f   physdll.obj
 0001:0001c1c0       ?AllocPortal@@YAPAUportal_t@@XZ 0041d1c0 f   portals.obj
 0001:0001c210       ?FreePortal@@YAXPAUportal_t@@@Z 0041d210 f   portals.obj
 0001:0001c250       ?VisibleContents@@YAHH@Z   0041d250 f   portals.obj
 0001:0001c270       ?ClusterContents@@YAHPAUnode_t@@@Z 0041d270 f   portals.obj
 0001:0001c2b0       ?Portal_VisFlood@@YAHPAUportal_t@@@Z 0041d2b0 f   portals.obj
 0001:0001c390       ?RemovePortalFromNode@@YAXPAUportal_t@@PAUnode_t@@@Z 0041d390 f   portals.obj
 0001:0001c410       ?AreaportalBrushForNode@@YAPAUbspbrush_t@@PAUnode_t@@@Z 0041d410 f   portals.obj
 0001:0001c430       ?BaseWindingForNode@@YAPAUwinding_t@@PAUnode_t@@@Z 0041d430 f   portals.obj
 0001:0001c510       ?CalcNodeBounds@@YAXPAUnode_t@@@Z 0041d510 f   portals.obj
 0001:0001c590       ?FloodPortals_r@@YAXPAUnode_t@@H@Z 0041d590 f   portals.obj
 0001:0001c620       ?FloodAreaLeak_r@@YAXPAUnode_t@@H@Z 0041d620 f   portals.obj
 0001:0001c6d0       ?ClearOccupied_r@@YAXPAUnode_t@@@Z 0041d6d0 f   portals.obj
 0001:0001c700       ?PlaceOccupant@@YAHPAUnode_t@@AAVVector@@PAUentity_t@@@Z 0041d700 f   portals.obj
 0001:0001c780       ?FloodEntities@@YAHPAUtree_t@@@Z 0041d780 f   portals.obj
 0001:0001c950       ?FloodAreas_r@@YAXPAUnode_t@@PAUportal_t@@@Z 0041d950 f   portals.obj
 0001:0001ca60       ?FindAreas_r@@YAXPAUnode_t@@@Z 0041da60 f   portals.obj
 0001:0001cac0       ?ReportAreaportalLeak@@YAXPAUtree_t@@PAUnode_t@@@Z 0041dac0 f   portals.obj
 0001:0001cbe0       ?SetAreaPortalAreas_r@@YAXPAUtree_t@@PAUnode_t@@@Z 0041dbe0 f   portals.obj
 0001:0001cc70       ?FindUniquePoints@@YAHPBVVector2D@@HPAHHM@Z 0041dc70 f   portals.obj
 0001:0001cde0       ?Convex2D@@YAHPBVVector2D@@HPAHH@Z 0041dde0 f   portals.obj
 0001:0001d1a0       ?SetNodeAreaIndices_R@@YAXPAUnode_t@@@Z 0041e1a0 f   portals.obj
 0001:0001d1e0       ?FloodAreas@@YAXPAUtree_t@@@Z 0041e1e0 f   portals.obj
 0001:0001d250       ?FillOutside_r@@YAXPAUnode_t@@@Z 0041e250 f   portals.obj
 0001:0001d2b0       ?FillOutside@@YAXPAUnode_t@@@Z 0041e2b0 f   portals.obj
 0001:0001d360       ??0?$CFmtStrN@$0BAA@@@QAA@PBDZZ 0041e360 f i portals.obj
 0001:0001d390       ?MakeNodePortal@@YAXPAUnode_t@@@Z 0041e390 f   portals.obj
 0001:0001d560       ??4portal_t@@QAEAAU0@ABU0@@Z 0041e560 f i portals.obj
 0001:0001d5d0       ?MakeHeadnodePortals@@YAXPAUtree_t@@@Z 0041e5d0 f   portals.obj
 0001:0001d830       ?SplitNodePortals@@YAXPAUnode_t@@@Z 0041e830 f   portals.obj
 0001:0001dba0       ?MakeTreePortals_r@@YAXPAUnode_t@@@Z 0041eba0 f   portals.obj
 0001:0001dcd0       ?MakeTreePortals@@YAXPAUtree_t@@@Z 0041ecd0 f   portals.obj
 0001:0001dcf0       ?InsertBefore@?$CUtlVector@VVector@@V?$CUtlMemory@VVector@@H@@@@QAEHHABVVector@@@Z 0041ecf0 f i portals.obj
 0001:0001dcf0       ?InsertBefore@?$CUtlVector@UResourceMemorySection@CVTFTexture@@V?$CUtlMemory@UResourceMemorySection@CVTFTexture@@H@@@@QAEHHABUResourceMemorySection@CVTFTexture@@@Z 0041ecf0 f i vtf:vtf.obj
 0001:0001dd70       ?FindPortalsLeadingToArea_R@@YAXPAUnode_t@@HHPAUplane_t@@AAV?$CUtlVector@PAUportal_t@@V?$CUtlMemory@PAUportal_t@@H@@@@@Z 0041ed70 f   portals.obj
 0001:0001ded0       ?EmitClipPortalGeometry@@YAXPAUnode_t@@PAUportal_t@@HPAUdareaportal_t@@@Z 0041eed0 f   portals.obj
 0001:0001e380       ?EmitAreaPortals@@YAXPAUnode_t@@@Z 0041f380 f   portals.obj
 0001:0001e770       ?FindPortalSide@@YAXPAUportal_t@@@Z 0041f770 f   portals.obj
 0001:0001e930       ?MarkVisibleSides_r@@YAXPAUnode_t@@@Z 0041f930 f   portals.obj
 0001:0001e9a0       ?MarkVisibleSides@@YAXPAUtree_t@@HHH@Z 0041f9a0 f   portals.obj
 0001:0001ea20       ?MarkVisibleSides@@YAXPAUtree_t@@PAPAUmapbrush_t@@H@Z 0041fa20 f   portals.obj
 0001:0001ea80       ?VolumeOfIntersection@@YAMPAUbspbrush_t@@PAUnode_t@@@Z 0041fa80 f   prtfile.obj
 0001:0001eb00       ?CreateVisPortals_r@@YAXPAUnode_t@@@Z 0041fb00 f   prtfile.obj
 0001:0001eb40       ?SaveClusters_r@@YAXPAUnode_t@@@Z 0041fb40 f   prtfile.obj
 0001:0001eb90       ?Grow@?$CUtlMemory@V?$CUtlVector@HV?$CUtlMemory@HH@@@@H@@QAEXH@Z 0041fb90 f i cubemap.obj
 0001:0001eb90       ?Grow@?$CUtlMemory@U?$UtlRBTreeNode_t@UNameTranslationLookup_t@@H@@H@@QAEXH@Z 0041fb90 f i materialpatch.obj
 0001:0001eb90       ?Grow@?$CUtlMemory@VCDispVert@@H@@QAEXH@Z 0041fb90 f i disp_vbsp.obj
 0001:0001eb90       ?Grow@?$CUtlMemory@Ucluster_portals_t@@H@@QAEXH@Z 0041fb90 f i prtfile.obj
 0001:0001ec30       ?WritePortalFile@@YAXPAU_iobuf@@ABV?$CUtlVector@Ucluster_portals_t@@V?$CUtlMemory@Ucluster_portals_t@@H@@@@@Z 0041fc30 f   prtfile.obj
 0001:0001eea0       ?GetVisCluster@@YAHPAUnode_t@@@Z 0041fea0 f   prtfile.obj
 0001:0001ef10       ?NumberLeafs@@YAXABV?$CUtlVector@PAUnode_t@@V?$CUtlMemory@PAUnode_t@@H@@@@@Z 0041ff10 f   prtfile.obj
 0001:0001efd0       ?InsertBefore@?$CUtlVector@Uviscluster_t@@V?$CUtlMemory@Uviscluster_t@@H@@@@QAEHHABUviscluster_t@@@Z 0041ffd0 f i prtfile.obj
 0001:0001efd0       ?InsertBefore@?$CUtlVector@Ulistplane_t@@V?$CUtlMemory@Ulistplane_t@@H@@@@QAEHHABUlistplane_t@@@Z 0041ffd0 f i ivp.obj
 0001:0001f050       ?AddVisCluster@@YAXPAUentity_t@@@Z 00420050 f   prtfile.obj
 0001:0001f0e0       ?BuildVisLeafList_r@@YAXPAUnode_t@@AAV?$CUtlVector@PAUnode_t@@V?$CUtlMemory@PAUnode_t@@H@@@@@Z 004200e0 f   prtfile.obj
 0001:0001f140       ?BuildPortalList@@YAHAAV?$CUtlVector@Ucluster_portals_t@@V?$CUtlMemory@Ucluster_portals_t@@H@@@@ABV?$CUtlVector@PAUnode_t@@V?$CUtlMemory@PAUnode_t@@H@@@@@Z 00420140 f   prtfile.obj
 0001:0001f230       ?InsertMultipleBefore@?$CUtlVector@Ucluster_portals_t@@V?$CUtlMemory@Ucluster_portals_t@@H@@@@QAEHHHPBUcluster_portals_t@@@Z 00420230 f i prtfile.obj
 0001:0001f380       ?WritePortalFile@@YAXPAUtree_t@@@Z 00420380 f   prtfile.obj
 0001:0001f540       ?CopyArray@?$CUtlVector@DV?$CUtlMemory@DH@@@@QAEXPBDH@Z 00420540 f i scratchpad3d.obj
 0001:0001f5b0       ?Studio_ConvertStudioHdrToNewVersion@@YA_NPAUstudiohdr_t@@@Z 004205b0 f i staticprop.obj
 0001:0001f6f0       ?IsStaticProp@@YA?AW4isstaticprop_ret@@PAUstudiohdr_t@@@Z 004206f0 f   staticprop.obj
 0001:0001f790       ?CacheVertexData@mstudiomodel_t@@QAEPBUvertexFileHeader_t@@PAX@Z 00420790 f   staticprop.obj
 0001:0001f930       ?GetVertexData@mstudiomodel_t@@QAEPBUmstudio_modelvertexdata_t@@PAX@Z 00420930 f i staticprop.obj
 0001:0001f9a0       ?LoadStudioModel@@YA_NPBD0AAVCUtlBuffer@@@Z 004209a0 f   staticprop.obj
 0001:0001fd30       ?Links@?$CUtlRBTree@UModelCollisionLookup_t@@GP6A_NABU1@0@ZV?$CUtlMemory@U?$UtlRBTreeNode_t@UModelCollisionLookup_t@@G@@G@@@@IBEABU?$UtlRBTreeLinks_t@G@@G@Z 00420d30 f i staticprop.obj
 0001:0001fd90       ?Grow@?$CUtlMemory@UStaticPropLump_t@@H@@QAEXH@Z 00420d90 f i staticprop.obj
 0001:0001ff60       ?FindInsertionPosition@?$CUtlRBTree@UModelCollisionLookup_t@@GP6A_NABU1@0@ZV?$CUtlMemory@U?$UtlRBTreeNode_t@UModelCollisionLookup_t@@G@@G@@@@IAEXABUModelCollisionLookup_t@@AAGAA_N@Z 00420f60 f i staticprop.obj
 0001:00020070       ?NewNode@?$CUtlRBTree@UModelCollisionLookup_t@@GP6A_NABU1@0@ZV?$CUtlMemory@U?$UtlRBTreeNode_t@UModelCollisionLookup_t@@G@@G@@@@QAEGXZ 00421070 f i staticprop.obj
 0001:00020170       ?RotateLeft@?$CUtlRBTree@UModelCollisionLookup_t@@GP6A_NABU1@0@ZV?$CUtlMemory@U?$UtlRBTreeNode_t@UModelCollisionLookup_t@@G@@G@@@@IAEXG@Z 00421170 f i staticprop.obj
 0001:00020260       ?RotateRight@?$CUtlRBTree@UModelCollisionLookup_t@@GP6A_NABU1@0@ZV?$CUtlMemory@U?$UtlRBTreeNode_t@UModelCollisionLookup_t@@G@@G@@@@IAEXG@Z 00421260 f i staticprop.obj
 0001:00020360       ?Find@?$CUtlRBTree@UModelCollisionLookup_t@@GP6A_NABU1@0@ZV?$CUtlMemory@U?$UtlRBTreeNode_t@UModelCollisionLookup_t@@G@@G@@@@QBEGABUModelCollisionLookup_t@@@Z 00421360 f i staticprop.obj
 0001:00020460       ?InsertBefore@?$CUtlVector@UStaticPropLump_t@@V?$CUtlMemory@UStaticPropLump_t@@H@@@@QAEHH@Z 00421460 f i staticprop.obj
 0001:000204c0       ?RemoveAll@?$CUtlRBTree@UModelCollisionLookup_t@@GP6A_NABU1@0@ZV?$CUtlMemory@U?$UtlRBTreeNode_t@UModelCollisionLookup_t@@G@@G@@@@QAEXXZ 004214c0 f i staticprop.obj
 0001:00020580       ?InsertRebalance@?$CUtlRBTree@UModelCollisionLookup_t@@GP6A_NABU1@0@ZV?$CUtlMemory@U?$UtlRBTreeNode_t@UModelCollisionLookup_t@@G@@G@@@@IAEXG@Z 00421580 f i staticprop.obj
 0001:00020ce0       ?LinkToParent@?$CUtlRBTree@UModelCollisionLookup_t@@GP6A_NABU1@0@ZV?$CUtlMemory@U?$UtlRBTreeNode_t@UModelCollisionLookup_t@@G@@G@@@@IAEXGG_N@Z 00421ce0 f i staticprop.obj
 0001:00020ec0       ?ComputeConvexHull@@YAPAVCPhysCollide@@PAUstudiohdr_t@@@Z 00421ec0 f   staticprop.obj
 0001:00021270       ??1?$CUtlRBTree@UModelCollisionLookup_t@@GP6A_NABU1@0@ZV?$CUtlMemory@U?$UtlRBTreeNode_t@UModelCollisionLookup_t@@G@@G@@@@QAE@XZ 00422270 f i staticprop.obj
 0001:000212d0       ?Insert@?$CUtlRBTree@UModelCollisionLookup_t@@GP6A_NABU1@0@ZV?$CUtlMemory@U?$UtlRBTreeNode_t@UModelCollisionLookup_t@@G@@G@@@@QAEGABUModelCollisionLookup_t@@@Z 004222d0 f i staticprop.obj
 0001:000216c0       ?EmitStaticProps@@YAXXZ    004226c0 f   staticprop.obj
 0001:000219d0       _cosf                      004229d0 f i textures.obj
 0001:000219e0       ?GetTexData@@YAPAUdtexdata_t@@H@Z 004229e0 f   textures.obj
 0001:00021a30       ?FindMiptex@@YAHPBD@Z      00422a30 f   textures.obj
 0001:000221e0       ?TextureAxisFromPlane@@YAXPAUplane_t@@AAVVector@@1@Z 004231e0 f   textures.obj
 0001:00022360       ?GetSurfaceProperties@@YAHPAXPBD@Z 00423360 f   textures.obj
 0001:000223e0       ?GetSurfaceProperties2@@YAHPAXPBD@Z 004233e0 f   textures.obj
 0001:00022450       ?FindAliasedTexData@@YAHPBDPAUdtexdata_t@@@Z 00423450 f   textures.obj
 0001:000225e0       ?FindTexData@@YAHPBD@Z     004235e0 f   textures.obj
 0001:00022640       ?FindOrCreateTexData@@YAHPBD@Z 00423640 f   textures.obj
 0001:00022750       ?LoadSurfacePropFile@@YAXPBD@Z 00423750 f   textures.obj
 0001:000227d0       ?LoadSurfaceProperties@@YAXXZ 004237d0 f   textures.obj
 0001:00022880       ?AddCloneTexData@@YAHPAUdtexdata_t@@PBD@Z 00423880 f   textures.obj
 0001:00022910       ?FindTexInfo@@YAHABUtexinfo_s@@@Z 00423910 f   textures.obj
 0001:000229f0       ?FindOrCreateTexInfo@@YAHABUtexinfo_s@@@Z 004239f0 f   textures.obj
 0001:00022a30       ?TexinfoForBrushTexture@@YAHPAUplane_t@@PAUbrush_texture_t@@ABVVector@@@Z 00423a30 f   textures.obj
 0001:00022d90       ?NodeForPoint@@YAPAUnode_t@@PAU1@AAVVector@@@Z 00423d90 f   tree.obj
 0001:00022df0       ?FreeTreePortals_r@@YAXPAUnode_t@@@Z 00423df0 f   tree.obj
 0001:00022e60       ?FreeTree_r@@YAXPAUnode_t@@@Z 00423e60 f   tree.obj
 0001:00022ee0       ?FreeTree@@YAXPAUtree_t@@@Z 00423ee0 f   tree.obj
 0001:00022f10       ?PruneNodes_r@@YAXPAUnode_t@@@Z 00423f10 f   tree.obj
 0001:00022fd0       ?PruneNodes@@YAXPAUnode_t@@@Z 00423fd0 f   tree.obj
 0001:00023010       ??0MaterialSystem_Config_t@@QAE@XZ 00424010 f i utilmatlib.obj
 0001:00023110       ?LoadMaterialSystemInterface@@YAXP6APAXPBDPAH@Z@Z 00424110 f   utilmatlib.obj
 0001:000231b0       ?InitMaterialSystem@@YAXPBDP6APAX0PAH@Z@Z 004241b0 f   utilmatlib.obj
 0001:000231e0       ?ShutdownMaterialSystem@@YAXXZ 004241e0 f   utilmatlib.obj
 0001:00023200       ?FindMaterial@@YAPAXPBDPA_N_N@Z 00424200 f   utilmatlib.obj
 0001:00023250       ?GetMaterialDimensions@@YAXPAXPAH1@Z 00424250 f   utilmatlib.obj
 0001:00023290       ?GetMaterialReflectivity@@YAXPAXPAM@Z 00424290 f   utilmatlib.obj
 0001:00023300       ?GetMaterialShaderPropertyBool@@YAHPAXH@Z 00424300 f   utilmatlib.obj
 0001:00023340       ?GetMaterialShaderPropertyInt@@YAHPAXH@Z 00424340 f   utilmatlib.obj
 0001:00023380       ?GetMaterialVar@@YAPBDPAXPBD@Z 00424380 f   utilmatlib.obj
 0001:000233b0       ?GetMaterialShaderName@@YAPBDPAX@Z 004243b0 f   utilmatlib.obj
 0001:000233c0       ?BlockTree@@YAPAUnode_t@@HHHH@Z 004243c0 f   vbsp.obj
 0001:000234f0       ?ProcessBlock_Thread@@YAXHH@Z 004244f0 f   vbsp.obj
 0001:00023620       ?ProcessSubModel@@YAXXZ    00424620 f   vbsp.obj
 0001:00023720       ?IsFuncOccluder@@YA_NH@Z   00424720 f   vbsp.obj
 0001:00023760       ?FixupOnlyEntsOccluderEntities@@YAXXZ 00424760 f   vbsp.obj
 0001:00023800       ?PrintCommandLine@@YAXHPAPAD@Z 00424800 f   vbsp.obj
 0001:00023850       ?Grow@?$CUtlMemory@Udoccluderdata_t@@H@@QAEXH@Z 00424850 f i vbsp.obj
 0001:000238f0       ?AssignAreaToOccluder@@YAXHPAUtree_t@@_N@Z 004248f0 f   vbsp.obj
 0001:00023ae0       ?AssignOccluderAreas@@YAXPAUtree_t@@@Z 00424ae0 f   vbsp.obj
 0001:00023b30       ?MarkNoDynamicShadowSides@@YAXXZ 00424b30 f   vbsp.obj
 0001:00023b90       ?Is3DSkyboxArea@@YA_NH@Z   00424b90 f   vbsp.obj
 0001:00023bc0       ?InsertBefore@?$CUtlVector@Udoccluderdata_t@@V?$CUtlMemory@Udoccluderdata_t@@H@@@@QAEHH@Z 00424bc0 f i vbsp.obj
 0001:00023c20       ?InsertBefore@?$CUtlVector@Udoccluderpolydata_t@@V?$CUtlMemory@Udoccluderpolydata_t@@H@@@@QAEHH@Z 00424c20 f i vbsp.obj
 0001:000240b0       ?ProcessWorldModel@@YAXXZ  004250b0 f   vbsp.obj
 0001:00024890       ?ProcessModels@@YAXXZ      00425890 f   vbsp.obj
 0001:00024930       ?RunVBSP@@YAHHPAPAD@Z      00425930 f   vbsp.obj
 0001:000257b0       _main                      004267b0 f   vbsp.obj
 0001:00025810       ?CreateWorldVertexTransitionPatchedMaterial@@YAXPBD0@Z 00426810 f   worldvertextransitionfixup.obj
 0001:00025990       ?CreateBrushVersionOfWorldVertexTransitionMaterial@@YAHH@Z 00426990 f   worldvertextransitionfixup.obj
 0001:00025a80       ?WorldVertexTransitionFixup@@YAXXZ 00426a80 f   worldvertextransitionfixup.obj
 0001:00025bf0       ?MemAlloc_StrDup@@YAPADPBD@Z 00426bf0 f i writebsp.obj
 0001:00025c50       ?CaselessStringLessThan@@YA_NABQBD0@Z 00426c50 f i writebsp.obj
 0001:00025c70       ?SetDynamicShadowsEnabled@dface_t@@QAEX_N@Z 00426c70 f i writebsp.obj
 0001:00025c90       ?EmitPlanes@@YAXXZ         00426c90 f   writebsp.obj
 0001:00025dc0       ?EmitMarkFace@@YAXPAUdleaf_t@@PAUface_t@@@Z 00426dc0 f   writebsp.obj
 0001:00025e70       ?EmitLeaf@@YAXPAUnode_t@@@Z 00426e70 f   writebsp.obj
 0001:00026030       ?CreateOrigFace@@YAHPAUface_t@@@Z 00427030 f   writebsp.obj
 0001:00026290       ?FindOrigFace@@YAHPAUface_t@@@Z 00427290 f   writebsp.obj
 0001:000262f0       ?FindOrCreateOrigFace@@YAHPAUface_t@@@Z 004272f0 f   writebsp.obj
 0001:00026320       ?FreeLeafFaces@@YAXPAUface_t@@@Z 00427320 f   writebsp.obj
 0001:00026350       ?SetModelNumbers@@YAXXZ    00427350 f   writebsp.obj
 0001:000263e0       ?SetLightStyles@@YAXXZ     004273e0 f   writebsp.obj
 0001:00026570       ?EmitBrushes@@YAXXZ        00427570 f   writebsp.obj
 0001:00026750       ?BeginBSPFile@@YAXXZ       00427750 f   writebsp.obj
 0001:00026790       ?EnsurePresenceOfWaterLODControlEntity@@YAXXZ 00427790 f   writebsp.obj
 0001:00026860       ?BeginModel@@YAXXZ         00427860 f   writebsp.obj
 0001:00026960       ?EndModel@@YAXXZ           00427960 f   writebsp.obj
 0001:00026990       ?Grow@?$CUtlMemory@VCDispTri@@H@@QAEXH@Z 00427990 f i disp_vbsp.obj
 0001:00026990       ?Grow@?$CUtlMemory@GH@@QAEXH@Z 00427990 f i disp_ivp.obj
 0001:00026990       ?Grow@?$CUtlMemory@UStaticPropLeafLump_t@@H@@QAEXH@Z 00427990 f i staticprop.obj
 0001:00026990       ?Grow@?$CUtlMemory@VCFaceMacroTextureInfo@@H@@QAEXH@Z 00427990 f i writebsp.obj
 0001:00026990       ?Grow@?$CUtlMemory@Udfaceid_t@@H@@QAEXH@Z 00427990 f i writebsp.obj
 0001:00026a40       ?Parent@?$CUtlRBTree@UNode_t@?$CUtlMap@PBDHH@@HVCKeyLess@2@V?$CUtlMemory@U?$UtlRBTreeNode_t@UNode_t@?$CUtlMap@PBDHH@@H@@H@@@@QBEHH@Z 00427a40 f i writebsp.obj
 0001:00026a90       ?FindMatchingBrushSideTexinfo@@YAHHPBUtexinfomap_t@@@Z 00427a90 f   writebsp.obj
 0001:00026c90       ?IsBoxInsideWorld@@YA_NHAAV?$CUtlVector@HV?$CUtlMemory@HH@@@@ABVVector@@1@Z 00427c90 f   writebsp.obj
 0001:00026d50       ?AddDispsToBounds@@YAXHAAV?$CUtlVector@HV?$CUtlMemory@HH@@@@AAVVector@@1@Z 00427d50 f   writebsp.obj
 0001:00026dd0       ?ComputeBoundsNoSkybox@@YAXXZ 00427dd0 f   writebsp.obj
 0001:00026f00       ?LeftChild@?$CUtlRBTree@UNode_t@?$CUtlMap@PBDHH@@HVCKeyLess@2@V?$CUtlMemory@U?$UtlRBTreeNode_t@UNode_t@?$CUtlMap@PBDHH@@H@@H@@@@QBEHH@Z 00427f00 f i writebsp.obj
 0001:00026f50       ?RightChild@?$CUtlRBTree@UNode_t@?$CUtlMap@PBDHH@@HVCKeyLess@2@V?$CUtlMemory@U?$UtlRBTreeNode_t@UNode_t@?$CUtlMap@PBDHH@@H@@H@@@@QBEHH@Z 00427f50 f i writebsp.obj
 0001:00026fa0       ?FindInsertionPosition@?$CUtlRBTree@UNode_t@?$CUtlMap@PBDHH@@HVCKeyLess@2@V?$CUtlMemory@U?$UtlRBTreeNode_t@UNode_t@?$CUtlMap@PBDHH@@H@@H@@@@IAEXABUNode_t@?$CUtlMap@PBDHH@@AAHAA_N@Z 00427fa0 f i writebsp.obj
 0001:00027090       ?NewNode@?$CUtlRBTree@UNode_t@?$CUtlMap@PBDHH@@HVCKeyLess@2@V?$CUtlMemory@U?$UtlRBTreeNode_t@UNode_t@?$CUtlMap@PBDHH@@H@@H@@@@QAEHXZ 00428090 f i writebsp.obj
 0001:00027160       ?FirstInorder@?$CUtlRBTree@UNode_t@?$CUtlMap@PBDHH@@HVCKeyLess@2@V?$CUtlMemory@U?$UtlRBTreeNode_t@UNode_t@?$CUtlMap@PBDHH@@H@@H@@@@QBEHXZ 00428160 f i writebsp.obj
 0001:00027200       ?InsertMultipleBefore@?$CUtlVector@Utexinfo_s@@V?$CUtlMemory@Utexinfo_s@@H@@@@QAEHHHPBUtexinfo_s@@@Z 00428200 f i writebsp.obj
 0001:000272c0       ?IsLeftChild@?$CUtlRBTree@UNode_t@?$CUtlMap@PBDHH@@HVCKeyLess@2@V?$CUtlMemory@U?$UtlRBTreeNode_t@UNode_t@?$CUtlMap@PBDHH@@H@@H@@@@QBE_NH@Z 004282c0 f i writebsp.obj
 0001:00027330       ?RotateLeft@?$CUtlRBTree@UNode_t@?$CUtlMap@PBDHH@@HVCKeyLess@2@V?$CUtlMemory@U?$UtlRBTreeNode_t@UNode_t@?$CUtlMap@PBDHH@@H@@H@@@@IAEXH@Z 00428330 f i writebsp.obj
 0001:00027460       ?RotateRight@?$CUtlRBTree@UNode_t@?$CUtlMap@PBDHH@@HVCKeyLess@2@V?$CUtlMemory@U?$UtlRBTreeNode_t@UNode_t@?$CUtlMap@PBDHH@@H@@H@@@@IAEXH@Z 00428460 f i writebsp.obj
 0001:00027560       ??1?$CUtlVector@Udleafambientindex_t@@V?$CUtlMemory@Udleafambientindex_t@@H@@@@QAE@XZ 00428560 f i bsplib.obj
 0001:00027560       ??1?$CUtlVector@UDetailObjectDictLump_t@@V?$CUtlMemory@UDetailObjectDictLump_t@@H@@@@QAE@XZ 00428560 f i detailobjects.obj
 0001:00027560       ??1?$CUtlVector@Uvariable_t@@V?$CUtlMemory@Uvariable_t@@H@@@@QAE@XZ 00428560 f i scriplib.obj
 0001:00027560       ??1?$CUtlVector@Utexinfo_s@@V?$CUtlMemory@Utexinfo_s@@H@@@@QAE@XZ 00428560 f i writebsp.obj
 0001:00027560       ??1?$CUtlVector@UResourceEntryInfo@@V?$CUtlMemory@UResourceEntryInfo@@H@@@@QAE@XZ 00428560 f i vtf:vtf.obj
 0001:00027560       ??1?$CUtlVector@PAUStringPool_t@CUtlSymbolTable@@V?$CUtlMemory@PAUStringPool_t@CUtlSymbolTable@@H@@@@QAE@XZ 00428560 f i tier1:utlsymbol.obj
 0001:00027560       ??1?$CUtlVector@EV?$CUtlMemory@EH@@@@QAE@XZ 00428560 f i bsplib.obj
 0001:00027560       ??1?$CUtlVector@VS3RGBA@@V?$CUtlMemory@VS3RGBA@@H@@@@QAE@XZ 00428560 f i vtf:vtf.obj
 0001:00027560       ??1?$CUtlVector@Udoccluderpolydata_t@@V?$CUtlMemory@Udoccluderpolydata_t@@H@@@@QAE@XZ 00428560 f i bsplib.obj
 0001:00027560       ??1?$CUtlVector@PAUnode_t@@V?$CUtlMemory@PAUnode_t@@H@@@@QAE@XZ 00428560 f i ivp.obj
 0001:00027560       ??1?$CUtlVector@Vddispinfo_t@@V?$CUtlMemory@Vddispinfo_t@@H@@@@QAE@XZ 00428560 f i bsplib.obj
 0001:00027560       ??1?$CUtlVector@UOccluderInfo_t@@V?$CUtlMemory@UOccluderInfo_t@@H@@@@QAE@XZ 00428560 f i vbsp.obj
 0001:00027560       ??1?$CUtlVector@DV?$CUtlMemory@DH@@@@QAE@XZ 00428560 f i disp_ivp.obj
 0001:00027560       ??1?$CUtlVector@UDetailObjectLump_t@@V?$CUtlMemory@UDetailObjectLump_t@@H@@@@QAE@XZ 00428560 f i detailobjects.obj
 0001:00027560       ??1?$CUtlVector@Uwatermodel_t@@V?$CUtlMemory@Uwatermodel_t@@H@@@@QAE@XZ 00428560 f i ivp.obj
 0001:00027560       ??1?$CUtlVector@VCDispVert@@V?$CUtlMemory@VCDispVert@@H@@@@QAE@XZ 00428560 f i bsplib.obj
 0001:00027560       ??1?$CUtlVector@HV?$CUtlMemory@HH@@@@QAE@XZ 00428560 f i cubemap.obj
 0001:00027560       ??1?$CUtlVector@UDetailSpriteDictLump_t@@V?$CUtlMemory@UDetailSpriteDictLump_t@@H@@@@QAE@XZ 00428560 f i detailobjects.obj
 0001:00027560       ??1?$CUtlVector@UStaticPropDictLump_t@@V?$CUtlMemory@UStaticPropDictLump_t@@H@@@@QAE@XZ 00428560 f i staticprop.obj
 0001:00027560       ??1?$CUtlVector@GV?$CUtlMemory@GH@@@@QAE@XZ 00428560 f i disp_ivp.obj
 0001:00027560       ??1?$CUtlVector@VCFaceMacroTextureInfo@@V?$CUtlMemory@VCFaceMacroTextureInfo@@H@@@@QAE@XZ 00428560 f i bsplib.obj
 0001:00027560       ??1?$CUtlVector@Uviscluster_t@@V?$CUtlMemory@Uviscluster_t@@H@@@@QAE@XZ 00428560 f i prtfile.obj
 0001:00027560       ??1?$CUtlVector@Udoccluderdata_t@@V?$CUtlMemory@Udoccluderdata_t@@H@@@@QAE@XZ 00428560 f i bsplib.obj
 0001:00027560       ??1?$CUtlVector@UStaticPropLeafLump_t@@V?$CUtlMemory@UStaticPropLeafLump_t@@H@@@@QAE@XZ 00428560 f i staticprop.obj
 0001:00027560       ??1?$CUtlVector@Udleafambientlighting_t@@V?$CUtlMemory@Udleafambientlighting_t@@H@@@@QAE@XZ 00428560 f i bsplib.obj
 0001:00027560       ??1?$CUtlVector@PADV?$CUtlMemory@PADH@@@@QAE@XZ 00428560 f i cubemap.obj
 0001:00027560       ??1?$CUtlVector@UResourceMemorySection@CVTFTexture@@V?$CUtlMemory@UResourceMemorySection@CVTFTexture@@H@@@@QAE@XZ 00428560 f i vtf:vtf.obj
 0001:00027560       ??1?$CUtlVector@PAVCCoreDispInfo@@V?$CUtlMemory@PAVCCoreDispInfo@@H@@@@QAE@XZ 00428560 f i disp_vbsp.obj
 0001:00027560       ??1?$CUtlVector@VCDispTri@@V?$CUtlMemory@VCDispTri@@H@@@@QAE@XZ 00428560 f i bsplib.obj
 0001:00027560       ??1?$CUtlVector@Udfaceid_t@@V?$CUtlMemory@Udfaceid_t@@H@@@@QAE@XZ 00428560 f i bsplib.obj
 0001:00027560       ??1?$CUtlVector@UStaticPropLump_t@@V?$CUtlMemory@UStaticPropLump_t@@H@@@@QAE@XZ 00428560 f i staticprop.obj
 0001:000275d0       ?Find@?$CUtlRBTree@UNode_t@?$CUtlMap@PBDHH@@HVCKeyLess@2@V?$CUtlMemory@U?$UtlRBTreeNode_t@UNode_t@?$CUtlMap@PBDHH@@H@@H@@@@QBEHABUNode_t@?$CUtlMap@PBDHH@@@Z 004285d0 f i writebsp.obj
 0001:000276c0       ?RemoveAll@?$CUtlRBTree@UNode_t@?$CUtlMap@PBDHH@@HVCKeyLess@2@V?$CUtlMemory@U?$UtlRBTreeNode_t@UNode_t@?$CUtlMap@PBDHH@@H@@H@@@@QAEXXZ 004286c0 f i writebsp.obj
 0001:00027750       ?NextInorder@?$CUtlRBTree@UNode_t@?$CUtlMap@PBDHH@@HVCKeyLess@2@V?$CUtlMemory@U?$UtlRBTreeNode_t@UNode_t@?$CUtlMap@PBDHH@@H@@H@@@@QBEHH@Z 00428750 f i writebsp.obj
 0001:000278e0       ?InsertMultipleBefore@?$CUtlVector@Udtexdata_t@@V?$CUtlMemory@Udtexdata_t@@H@@@@QAEHHHPBUdtexdata_t@@@Z 004288e0 f i writebsp.obj
 0001:00027af0       ?InsertRebalance@?$CUtlRBTree@UNode_t@?$CUtlMap@PBDHH@@HVCKeyLess@2@V?$CUtlMemory@U?$UtlRBTreeNode_t@UNode_t@?$CUtlMap@PBDHH@@H@@H@@@@IAEXH@Z 00428af0 f i writebsp.obj
 0001:00028030       ?LinkToParent@?$CUtlRBTree@UNode_t@?$CUtlMap@PBDHH@@HVCKeyLess@2@V?$CUtlMemory@U?$UtlRBTreeNode_t@UNode_t@?$CUtlMap@PBDHH@@H@@H@@@@IAEXHH_N@Z 00429030 f i writebsp.obj
 0001:000280a0       ?RemoveAll@?$CUtlDict@HH@@QAEXXZ 004290a0 f i writebsp.obj
 0001:000280f0       ?EmitFace@@YAXPAUface_t@@H@Z 004290f0 f   writebsp.obj
 0001:00028360       ?EmitDrawNode_r@@YAHPAUnode_t@@@Z 00429360 f   writebsp.obj
 0001:000284d0       ?WriteBSP@@YAXPAUnode_t@@PAUface_t@@@Z 004294d0 f   writebsp.obj
 0001:00028620       ?CopyArray@?$CUtlVector@Utexinfo_s@@V?$CUtlMemory@Utexinfo_s@@H@@@@QAEXPBUtexinfo_s@@H@Z 00429620 f i writebsp.obj
 0001:00028670       ?Insert@?$CUtlRBTree@UNode_t@?$CUtlMap@PBDHH@@HVCKeyLess@2@V?$CUtlMemory@U?$UtlRBTreeNode_t@UNode_t@?$CUtlMap@PBDHH@@H@@H@@@@QAEHABUNode_t@?$CUtlMap@PBDHH@@@Z 00429670 f i writebsp.obj
 0001:000286d0       ?ComapctTexinfoArray@@YAXPAUtexinfomap_t@@@Z 004296d0 f   writebsp.obj
 0001:000287c0       ?CopyArray@?$CUtlVector@Udtexdata_t@@V?$CUtlMemory@Udtexdata_t@@H@@@@QAEXPBUdtexdata_t@@H@Z 004297c0 f i writebsp.obj
 0001:00028980       ?CompactTexdataArray@@YAXPAUtexdatamap_t@@@Z 00429980 f   writebsp.obj
 0001:00028b50       ?CompactTexinfos@@YAXXZ    00429b50 f   writebsp.obj
 0001:00028f00       ?DiscoverMacroTextures@@YAXXZ 00429f00 f   writebsp.obj
 0001:00029090       ?EndBSPFile@@YAXXZ         0042a090 f   writebsp.obj
 0001:00029140       ?CreateTempFile@CWin32File@@SAPAXAAVCUtlString@@0@Z 0042a140 f i zip_utils.obj
 0001:00029260       ?FileSeek@CWin32File@@SAIPAXIK@Z 0042a260 f i zip_utils.obj
 0001:000292b0       ?FileTell@CWin32File@@SAIPAX@Z 0042a2b0 f i zip_utils.obj
 0001:00029300       ?FileWrite@CWin32File@@SA_NPAX0I@Z 0042a300 f i zip_utils.obj
 0001:00029340       ?Put@CFileStream@@UAEXPBXH@Z 0042a340 f i zip_utils.obj
 0001:00029380       ?Tell@CFileStream@@UAEIXZ  0042a380 f i zip_utils.obj
 0001:000293a0       ??0CZipEntry@CZipFile@@QAE@ABV01@@Z 0042a3a0 f   zip_utils.obj
 0001:00029410       ?ZipFileLessFunc_CaselessSort@CZipEntry@CZipFile@@SA_NABV12@0@Z 0042a410 f   zip_utils.obj
 0001:00029470       ?ParseXZipCommentString@CZipFile@@AAEXPBD@Z 0042a470 f   zip_utils.obj
 0001:000294d0       ?SetBigEndian@CZip@@UAEX_N@Z 0042a4d0 f   zip_utils.obj
 0001:00029500       ?ActivateByteSwapping@CZip@@UAEX_N@Z 0042a500 f   zip_utils.obj
 0001:00029530       ?ForceAlignment@CZip@@UAEX_N0I@Z 0042a530 f   zip_utils.obj
 0001:00029560       ?GetAlignment@CZip@@UAEIXZ 0042a560 f   zip_utils.obj
 0001:00029570       ?Put@CBufferStream@@UAEXPBXH@Z 0042a570 f i zip_utils.obj
 0001:00029580       ?Tell@CBufferStream@@UAEIXZ 0042a580 f i zip_utils.obj
 0001:00029590       ?Color@?$CUtlRBTree@VCZipEntry@CZipFile@@HP6A_NABV12@0@ZV?$CUtlMemory@U?$UtlRBTreeNode_t@VCZipEntry@CZipFile@@H@@H@@@@IBE?AW4NodeColor_t@1@H@Z 0042a590 f i zip_utils.obj
 0001:000295e0       ?Grow@?$CUtlMemory@U?$UtlLinkedListElem_t@PAVCZip@@G@@G@@QAEXH@Z 0042a5e0 f i zip_utils.obj
 0001:000296b0       ??$PutTypeBin@D@CUtlBuffer@@IAEXD@Z 0042a6b0 f i zip_utils.obj
 0001:000296e0       ??$GetObjects@UZIP_EndOfCentralDirRecord@@@CUtlBuffer@@QAEXPAUZIP_EndOfCentralDirRecord@@H@Z 0042a6e0 f i zip_utils.obj
 0001:00029760       ??$GetObjects@UZIP_FileHeader@@@CUtlBuffer@@QAEXPAUZIP_FileHeader@@H@Z 0042a760 f i zip_utils.obj
 0001:000297d0       ?Parent@?$CUtlRBTree@VCZipEntry@CZipFile@@HP6A_NABV12@0@ZV?$CUtlMemory@U?$UtlRBTreeNode_t@VCZipEntry@CZipFile@@H@@H@@@@QBEHH@Z 0042a7d0 f i zip_utils.obj
 0001:00029820       ?LeftChild@?$CUtlRBTree@VCZipEntry@CZipFile@@HP6A_NABV12@0@ZV?$CUtlMemory@U?$UtlRBTreeNode_t@VCZipEntry@CZipFile@@H@@H@@@@QBEHH@Z 0042a820 f i zip_utils.obj
 0001:00029870       ?RightChild@?$CUtlRBTree@VCZipEntry@CZipFile@@HP6A_NABV12@0@ZV?$CUtlMemory@U?$UtlRBTreeNode_t@VCZipEntry@CZipFile@@H@@H@@@@QBEHH@Z 0042a870 f i zip_utils.obj
 0001:000298c0       ?IsRightChild@?$CUtlRBTree@VCZipEntry@CZipFile@@HP6A_NABV12@0@ZV?$CUtlMemory@U?$UtlRBTreeNode_t@VCZipEntry@CZipFile@@H@@H@@@@QBE_NH@Z 0042a8c0 f i zip_utils.obj
 0001:00029970       ?FindInsertionPosition@?$CUtlRBTree@VCZipEntry@CZipFile@@HP6A_NABV12@0@ZV?$CUtlMemory@U?$UtlRBTreeNode_t@VCZipEntry@CZipFile@@H@@H@@@@IAEXABVCZipEntry@CZipFile@@AAHAA_N@Z 0042a970 f i zip_utils.obj
 0001:00029a60       ?NewNode@?$CUtlRBTree@VCZipEntry@CZipFile@@HP6A_NABV12@0@ZV?$CUtlMemory@U?$UtlRBTreeNode_t@VCZipEntry@CZipFile@@H@@H@@@@QAEHXZ 0042aa60 f i zip_utils.obj
 0001:00029b70       ?AllocInternal@?$CUtlLinkedList@PAVCZip@@G$0A@GV?$CUtlMemory@U?$UtlLinkedListElem_t@PAVCZip@@G@@G@@@@IAEG_N@Z 0042ab70 f i zip_utils.obj
 0001:00029c90       ?IsLeftChild@?$CUtlRBTree@VCZipEntry@CZipFile@@HP6A_NABV12@0@ZV?$CUtlMemory@U?$UtlRBTreeNode_t@VCZipEntry@CZipFile@@H@@H@@@@QBE_NH@Z 0042ac90 f i zip_utils.obj
 0001:00029d40       ?RotateLeft@?$CUtlRBTree@VCZipEntry@CZipFile@@HP6A_NABV12@0@ZV?$CUtlMemory@U?$UtlRBTreeNode_t@VCZipEntry@CZipFile@@H@@H@@@@IAEXH@Z 0042ad40 f i zip_utils.obj
 0001:00029eb0       ?RotateRight@?$CUtlRBTree@VCZipEntry@CZipFile@@HP6A_NABV12@0@ZV?$CUtlMemory@U?$UtlRBTreeNode_t@VCZipEntry@CZipFile@@H@@H@@@@IAEXH@Z 0042aeb0 f i zip_utils.obj
 0001:0002a030       ?PutTabs@CUtlBuffer@@IAEXXZ 0042b030 f i zip_utils.obj
 0001:0002a1a0       ?Find@?$CUtlRBTree@VCZipEntry@CZipFile@@HP6A_NABV12@0@ZV?$CUtlMemory@U?$UtlRBTreeNode_t@VCZipEntry@CZipFile@@H@@H@@@@QBEHABVCZipEntry@CZipFile@@@Z 0042b1a0 f i zip_utils.obj
 0001:0002a290       ?RemoveAll@?$CUtlRBTree@VCZipEntry@CZipFile@@HP6A_NABV12@0@ZV?$CUtlMemory@U?$UtlRBTreeNode_t@VCZipEntry@CZipFile@@H@@H@@@@QAEXXZ 0042b290 f i zip_utils.obj
 0001:0002a330       ?FirstInorder@?$CUtlRBTree@VCZipEntry@CZipFile@@HP6A_NABV12@0@ZV?$CUtlMemory@U?$UtlRBTreeNode_t@VCZipEntry@CZipFile@@H@@H@@@@QBEHXZ 0042b330 f i zip_utils.obj
 0001:0002a3c0       ?NextInorder@?$CUtlRBTree@VCZipEntry@CZipFile@@HP6A_NABV12@0@ZV?$CUtlMemory@U?$UtlRBTreeNode_t@VCZipEntry@CZipFile@@H@@H@@@@QBEHH@Z 0042b3c0 f i zip_utils.obj
 0001:0002a510       ?InsertRebalance@?$CUtlRBTree@VCZipEntry@CZipFile@@HP6A_NABV12@0@ZV?$CUtlMemory@U?$UtlRBTreeNode_t@VCZipEntry@CZipFile@@H@@H@@@@IAEXH@Z 0042b510 f i zip_utils.obj
 0001:0002a940       ?RemoveRebalance@?$CUtlRBTree@VCZipEntry@CZipFile@@HP6A_NABV12@0@ZV?$CUtlMemory@U?$UtlRBTreeNode_t@VCZipEntry@CZipFile@@H@@H@@@@IAEXH@Z 0042b940 f i zip_utils.obj
 0001:0002b240       ?Unlink@?$CUtlLinkedList@PAVCZip@@G$0A@GV?$CUtlMemory@U?$UtlLinkedListElem_t@PAVCZip@@G@@G@@@@QAEXG@Z 0042c240 f i zip_utils.obj
 0001:0002b2d0       ??1CDatadescGeneratedNameHolder@@QAE@XZ 0042c2d0 f i zip_utils.obj
 0001:0002b350       ?ReadFileFromZip@CZipFile@@QAE_NPBD_NAAVCUtlBuffer@@@Z 0042c350 f   zip_utils.obj
 0001:0002b470       ?ReadFileFromZip@CZipFile@@QAE_NPAXPBD_NAAVCUtlBuffer@@@Z 0042c470 f   zip_utils.obj
 0001:0002b600       ?FileExistsInZip@CZipFile@@QAE_NPBD@Z 0042c600 f   zip_utils.obj
 0001:0002b6c0       ?CalculateSize@CZipFile@@QAEIXZ 0042c6c0 f   zip_utils.obj
 0001:0002b7c0       ?PrintDirectory@CZipFile@@QAEXXZ 0042c7c0 f   zip_utils.obj
 0001:0002b810       ?GetNextFilename@CZipFile@@QAEHHPADHAAH@Z 0042c810 f   zip_utils.obj
 0001:0002b880       ?SaveDirectory@CZipFile@@AAEXAAVIWriteStream@@@Z 0042c880 f   zip_utils.obj
 0001:0002bde0       ?FileExistsInZip@CZip@@UAE_NPBD@Z 0042cde0 f   zip_utils.obj
 0001:0002bdf0       ?ReadFileFromZip@CZip@@UAE_NPBD_NAAVCUtlBuffer@@@Z 0042cdf0 f   zip_utils.obj
 0001:0002be00       ?ReadFileFromZip@CZip@@UAE_NPAXPBD_NAAVCUtlBuffer@@@Z 0042ce00 f   zip_utils.obj
 0001:0002be10       ?GetNextFilename@CZip@@UAEHHPADHAAH@Z 0042ce10 f   zip_utils.obj
 0001:0002be20       ?PrintDirectory@CZip@@UAEXXZ 0042ce20 f   zip_utils.obj
 0001:0002be30       ?Reset@CZip@@UAEXXZ        0042ce30 f   zip_utils.obj
 0001:0002be80       ?EstimateSize@CZip@@UAEIXZ 0042ce80 f   zip_utils.obj
 0001:0002be90       ??1?$CUtlRBTree@VCZipEntry@CZipFile@@HP6A_NABV12@0@ZV?$CUtlMemory@U?$UtlRBTreeNode_t@VCZipEntry@CZipFile@@H@@H@@@@QAE@XZ 0042ce90 f i zip_utils.obj
 0001:0002bef0       ?LinkToParent@?$CUtlRBTree@VCZipEntry@CZipFile@@HP6A_NABV12@0@ZV?$CUtlMemory@U?$UtlRBTreeNode_t@VCZipEntry@CZipFile@@H@@H@@@@IAEXHH_N@Z 0042cef0 f i zip_utils.obj
 0001:0002bf60       ?Unlink@?$CUtlRBTree@VCZipEntry@CZipFile@@HP6A_NABV12@0@ZV?$CUtlMemory@U?$UtlRBTreeNode_t@VCZipEntry@CZipFile@@H@@H@@@@IAEXH@Z 0042cf60 f i zip_utils.obj
 0001:0002c190       ??$DataMapInit@UZIP_EndOfCentralDirRecord@@@@YAPAUdatamap_t@@PAUZIP_EndOfCentralDirRecord@@@Z 0042d190 f   zip_utils.obj
 0001:0002c210       ??$DataMapInit@UZIP_FileHeader@@@@YAPAUdatamap_t@@PAUZIP_FileHeader@@@Z 0042d210 f   zip_utils.obj
 0001:0002c290       ??$DataMapInit@UZIP_LocalFileHeader@@@@YAPAUdatamap_t@@PAUZIP_LocalFileHeader@@@Z 0042d290 f   zip_utils.obj
 0001:0002c310       ??$DataMapInit@UZIP_PreloadHeader@@@@YAPAUdatamap_t@@PAUZIP_PreloadHeader@@@Z 0042d310 f   zip_utils.obj
 0001:0002c390       ??$DataMapInit@UZIP_PreloadDirectoryEntry@@@@YAPAUdatamap_t@@PAUZIP_PreloadDirectoryEntry@@@Z 0042d390 f   zip_utils.obj
 0001:0002c410       ??0CZipFile@@QAE@PBD_N@Z   0042d410 f   zip_utils.obj
 0001:0002c4c0       ??1CZipFile@@QAE@XZ        0042d4c0 f   zip_utils.obj
 0001:0002c560       ??0CZip@@QAE@PBD_N@Z       0042d560 f   zip_utils.obj
 0001:0002c5d0       ?SaveToBuffer@CZip@@UAEXAAVCUtlBuffer@@@Z 0042d5d0 f   zip_utils.obj
 0001:0002c600       ?SaveToDisk@CZip@@UAEXPAU_iobuf@@@Z 0042d600 f   zip_utils.obj
 0001:0002c630       ?SaveToDisk@CZip@@UAEXPAX@Z 0042d630 f   zip_utils.obj
 0001:0002c660       ?RemoveAt@?$CUtlRBTree@VCZipEntry@CZipFile@@HP6A_NABV12@0@ZV?$CUtlMemory@U?$UtlRBTreeNode_t@VCZipEntry@CZipFile@@H@@H@@@@QAEXH@Z 0042d660 f i zip_utils.obj
 0001:0002c6b0       ??_GCZip@@UAEPAXI@Z        0042d6b0 f i zip_utils.obj
 0001:0002c6b0       ??_ECZip@@UAEPAXI@Z        0042d6b0 f i zip_utils.obj
 0001:0002c6e0       ?Insert@?$CUtlRBTree@VCZipEntry@CZipFile@@HP6A_NABV12@0@ZV?$CUtlMemory@U?$UtlRBTreeNode_t@VCZipEntry@CZipFile@@H@@H@@@@QAEHABVCZipEntry@CZipFile@@@Z 0042d6e0 f i zip_utils.obj
 0001:0002c740       ?AddToTail@?$CUtlLinkedList@PAVCZip@@G$0A@GV?$CUtlMemory@U?$UtlLinkedListElem_t@PAVCZip@@G@@G@@@@QAEGABQAVCZip@@@Z 0042d740 f i zip_utils.obj
 0001:0002c7b0       ?FindAndRemove@?$CUtlLinkedList@PAVCZip@@G$0A@GV?$CUtlMemory@U?$UtlLinkedListElem_t@PAVCZip@@G@@G@@@@QAE_NABQAVCZip@@@Z 0042d7b0 f i zip_utils.obj
 0001:0002c820       ?ParseFromBuffer@CZipFile@@QAEXPAXH@Z 0042d820 f   zip_utils.obj
 0001:0002cc70       ?ParseFromDisk@CZipFile@@QAEPAXPBD@Z 0042dc70 f   zip_utils.obj
 0001:0002d030       ?AddBufferToZip@CZipFile@@QAEXPBDPAXH_N@Z 0042e030 f   zip_utils.obj
 0001:0002d270       ?AddFileToZip@CZipFile@@QAEXPBD0@Z 0042e270 f   zip_utils.obj
 0001:0002d2f0       ?RemoveFileFromZip@CZipFile@@QAEXPBD@Z 0042e2f0 f   zip_utils.obj
 0001:0002d3c0       ?CreateZip@IZip@@SAPAV1@PBD_N@Z 0042e3c0 f   zip_utils.obj
 0001:0002d400       ?ReleaseZip@IZip@@SAXPAV1@@Z 0042e400 f   zip_utils.obj
 0001:0002d430       ?AddFileToZip@CZip@@UAEXPBD0@Z 0042e430 f   zip_utils.obj
 0001:0002d440       ?RemoveFileFromZip@CZip@@UAEXPBD@Z 0042e440 f   zip_utils.obj
 0001:0002d450       ?AddBufferToZip@CZip@@UAEXPBDPAXH_N@Z 0042e450 f   zip_utils.obj
 0001:0002d460       ?ParseFromBuffer@CZip@@UAEXPAXH@Z 0042e460 f   zip_utils.obj
 0001:0002d4c0       ?ParseFromDisk@CZip@@UAEPAXPBD@Z 0042e4c0 f   zip_utils.obj
 0001:0002d520       ?GetPakFile@@YAPAVIZip@@XZ 0042e520 f   bsplib.obj
 0001:0002d540       ?ReleasePakFileLumps@@YAXXZ 0042e540 f   bsplib.obj
 0001:0002d560       ?AddBufferToPak@@YAXPAVIZip@@PBDPAXH_N@Z 0042e560 f   bsplib.obj
 0001:0002d580       ?FileExistsInPak@@YA_NPAVIZip@@PBD@Z 0042e580 f   bsplib.obj
 0001:0002d5a0       ?ReadFileFromPak@@YA_NPAVIZip@@PBD_NAAVCUtlBuffer@@@Z 0042e5a0 f   bsplib.obj
 0001:0002d5c0       ?InvalidGameLump@CGameLump@@QAEGXZ 0042e5c0 f   bsplib.obj
 0001:0002d5d0       ?SetKeyValue@@YAXPAUentity_t@@PBD1@Z 0042e5d0 f   bsplib.obj
 0001:0002d650       ?ValueForKey@@YAPADPAUentity_t@@PAD@Z 0042e650 f   bsplib.obj
 0001:0002d690       ?FloatForKey@@YAMPAUentity_t@@PAD@Z 0042e690 f   bsplib.obj
 0001:0002d6b0       ?IntForKey@@YAHPAUentity_t@@PAD@Z 0042e6b0 f   bsplib.obj
 0001:0002d6d0       ?GetVectorForKey@@YAXPAUentity_t@@PADAAVVector@@@Z 0042e6d0 f   bsplib.obj
 0001:0002d6d0       ?GetAnglesForKey@@YAXPAUentity_t@@PADAAVQAngle@@@Z 0042e6d0 f   bsplib.obj
 0001:0002d730       ?GetVector2DForKey@@YAXPAUentity_t@@PADAAVVector2D@@@Z 0042e730 f   bsplib.obj
 0001:0002d780       ?CalcTextureCoordsAtPoints@@YAXQAY03$$CBMQBHPBVVector@@HPAVVector2D@@@Z 0042e780 f   bsplib.obj
 0001:0002d810       ?GetPlatformMapPath@@YAXPBDPADHH@Z 0042e810 f   bsplib.obj
 0001:0002d840       ??$SwapFieldsToTargetEndian@UStaticPropDictLump_t@@@CByteswap@@QAEXPAUStaticPropDictLump_t@@PAXI@Z 0042e840 f i bsplib.obj
 0001:0002d880       ??$SwapFieldsToTargetEndian@UStaticPropLeafLump_t@@@CByteswap@@QAEXPAUStaticPropLeafLump_t@@PAXI@Z 0042e880 f i bsplib.obj
 0001:0002d8c0       ??$SwapFieldsToTargetEndian@UDetailObjectDictLump_t@@@CByteswap@@QAEXPAUDetailObjectDictLump_t@@PAXI@Z 0042e8c0 f i bsplib.obj
 0001:0002d900       ??$SwapFieldsToTargetEndian@UDetailPropLightstylesLump_t@@@CByteswap@@QAEXPAUDetailPropLightstylesLump_t@@PAXI@Z 0042e900 f i bsplib.obj
 0001:0002d940       ??$SwapFieldsToTargetEndian@Udgamelumpheader_t@@@CByteswap@@QAEXPAUdgamelumpheader_t@@PAXI@Z 0042e940 f i bsplib.obj
 0001:0002d980       ??$SwapFieldsToTargetEndian@Udgamelump_t@@@CByteswap@@QAEXPAUdgamelump_t@@PAXI@Z 0042e980 f i bsplib.obj
 0001:0002d9c0       ??$SwapFieldsToTargetEndian@Udheader_t@@@CByteswap@@QAEXPAUdheader_t@@PAXI@Z 0042e9c0 f i bsplib.obj
 0001:0002da00       ??$SwapFieldsToTargetEndian@Udleafambientlighting_t@@@CByteswap@@QAEXPAUdleafambientlighting_t@@PAXI@Z 0042ea00 f i bsplib.obj
 0001:0002da40       ??$SwapFieldsToTargetEndian@Udleafambientindex_t@@@CByteswap@@QAEXPAUdleafambientindex_t@@PAXI@Z 0042ea40 f i bsplib.obj
 0001:0002da80       ??$SwapFieldsToTargetEndian@Udleaf_t@@@CByteswap@@QAEXPAUdleaf_t@@PAXI@Z 0042ea80 f i bsplib.obj
 0001:0002dac0       ??$SwapFieldsToTargetEndian@Udflagslump_t@@@CByteswap@@QAEXPAUdflagslump_t@@PAXI@Z 0042eac0 f i bsplib.obj
 0001:0002db00       ??$SwapFieldsToTargetEndian@Udface_t@@@CByteswap@@QAEXPAUdface_t@@PAXI@Z 0042eb00 f i bsplib.obj
 0001:0002db40       ??$SwapFieldsToTargetEndian@Udworldlight_t@@@CByteswap@@QAEXPAUdworldlight_t@@PAXI@Z 0042eb40 f i bsplib.obj
 0001:0002db80       ??$SwapFieldsToTargetEndian@Udmodel_t@@@CByteswap@@QAEXPAUdmodel_t@@PAXI@Z 0042eb80 f i bsplib.obj
 0001:0002dbc0       ??$SwapFieldsToTargetEndian@Udvertex_t@@@CByteswap@@QAEXPAUdvertex_t@@PAXI@Z 0042ebc0 f i bsplib.obj
 0001:0002dc00       ??$SwapFieldsToTargetEndian@Udplane_t@@@CByteswap@@QAEXPAUdplane_t@@PAXI@Z 0042ec00 f i bsplib.obj
 0001:0002dc40       ??$SwapFieldsToTargetEndian@Udnode_t@@@CByteswap@@QAEXPAUdnode_t@@PAXI@Z 0042ec40 f i bsplib.obj
 0001:0002dc80       ??$SwapFieldsToTargetEndian@Utexinfo_s@@@CByteswap@@QAEXPAUtexinfo_s@@PAXI@Z 0042ec80 f i bsplib.obj
 0001:0002dcc0       ??$SwapFieldsToTargetEndian@Udtexdata_t@@@CByteswap@@QAEXPAUdtexdata_t@@PAXI@Z 0042ecc0 f i bsplib.obj
 0001:0002dd00       ??$SwapFieldsToTargetEndian@Vddispinfo_t@@@CByteswap@@QAEXPAVddispinfo_t@@PAXI@Z 0042ed00 f i bsplib.obj
 0001:0002dd40       ??$SwapFieldsToTargetEndian@VCDispVert@@@CByteswap@@QAEXPAVCDispVert@@PAXI@Z 0042ed40 f i bsplib.obj
 0001:0002dd80       ??$SwapFieldsToTargetEndian@VCDispTri@@@CByteswap@@QAEXPAVCDispTri@@PAXI@Z 0042ed80 f i bsplib.obj
 0001:0002ddc0       ??$SwapFieldsToTargetEndian@VCFaceMacroTextureInfo@@@CByteswap@@QAEXPAVCFaceMacroTextureInfo@@PAXI@Z 0042edc0 f i bsplib.obj
 0001:0002de00       ??$SwapFieldsToTargetEndian@Udprimitive_t@@@CByteswap@@QAEXPAUdprimitive_t@@PAXI@Z 0042ee00 f i bsplib.obj
 0001:0002de40       ??$SwapFieldsToTargetEndian@Udprimvert_t@@@CByteswap@@QAEXPAUdprimvert_t@@PAXI@Z 0042ee40 f i bsplib.obj
 0001:0002de80       ??$SwapFieldsToTargetEndian@Udedge_t@@@CByteswap@@QAEXPAUdedge_t@@PAXI@Z 0042ee80 f i bsplib.obj
 0001:0002dec0       ??$SwapFieldsToTargetEndian@Udbrush_t@@@CByteswap@@QAEXPAUdbrush_t@@PAXI@Z 0042eec0 f i bsplib.obj
 0001:0002df00       ??$SwapFieldsToTargetEndian@Udbrushside_t@@@CByteswap@@QAEXPAUdbrushside_t@@PAXI@Z 0042ef00 f i bsplib.obj
 0001:0002df40       ??$SwapFieldsToTargetEndian@Udarea_t@@@CByteswap@@QAEXPAUdarea_t@@PAXI@Z 0042ef40 f i bsplib.obj
 0001:0002df80       ??$SwapFieldsToTargetEndian@Udareaportal_t@@@CByteswap@@QAEXPAUdareaportal_t@@PAXI@Z 0042ef80 f i bsplib.obj
 0001:0002dfc0       ??$SwapFieldsToTargetEndian@Udleafwaterdata_t@@@CByteswap@@QAEXPAUdleafwaterdata_t@@PAXI@Z 0042efc0 f i bsplib.obj
 0001:0002e000       ??$SwapFieldsToTargetEndian@Udcubemapsample_t@@@CByteswap@@QAEXPAUdcubemapsample_t@@PAXI@Z 0042f000 f i bsplib.obj
 0001:0002e040       ??$SwapFieldsToTargetEndian@Udoverlay_t@@@CByteswap@@QAEXPAUdoverlay_t@@PAXI@Z 0042f040 f i bsplib.obj
 0001:0002e080       ??$SwapFieldsToTargetEndian@Udwateroverlay_t@@@CByteswap@@QAEXPAUdwateroverlay_t@@PAXI@Z 0042f080 f i bsplib.obj
 0001:0002e0c0       ??$SwapFieldsToTargetEndian@Udoverlayfade_t@@@CByteswap@@QAEXPAUdoverlayfade_t@@PAXI@Z 0042f0c0 f i bsplib.obj
 0001:0002e100       ??$SwapFieldsToTargetEndian@Udoccluderdata_t@@@CByteswap@@QAEXPAUdoccluderdata_t@@PAXI@Z 0042f100 f i bsplib.obj
 0001:0002e140       ??$SwapFieldsToTargetEndian@Udoccluderpolydata_t@@@CByteswap@@QAEXPAUdoccluderpolydata_t@@PAXI@Z 0042f140 f i bsplib.obj
 0001:0002e180       ??$SwapFieldsToTargetEndian@Udfaceid_t@@@CByteswap@@QAEXPAUdfaceid_t@@PAXI@Z 0042f180 f i bsplib.obj
 0001:0002e1c0       ?Grow@?$CUtlMemory@Uviscluster_t@@H@@QAEXH@Z 0042f1c0 f i prtfile.obj
 0001:0002e1c0       ?Grow@?$CUtlMemory@VCUtlString@@H@@QAEXH@Z 0042f1c0 f i bsplib.obj
 0001:0002e1c0       ?Grow@?$CUtlMemory@Ulistplane_t@@H@@QAEXH@Z 0042f1c0 f i ivp.obj
 0001:0002e270       ?ShiftElementsRight@?$CUtlVector@Udleafambientlighting_t@@V?$CUtlMemory@Udleafambientlighting_t@@H@@@@IAEXHH@Z 0042f270 f i bsplib.obj
 0001:0002e2d0       ?Grow@?$CUtlMemory@VS3RGBA@@H@@QAEXH@Z 0042f2d0 f i vtf:vtf.obj
 0001:0002e2d0       ?Grow@?$CUtlMemory@PAUnode_t@@H@@QAEXH@Z 0042f2d0 f i ivp.obj
 0001:0002e2d0       ?Grow@?$CUtlMemory@Udleafambientindex_t@@H@@QAEXH@Z 0042f2d0 f i bsplib.obj
 0001:0002e2d0       ?Grow@?$CUtlMemory@PAUface_t@@H@@QAEXH@Z 0042f2d0 f i vbsp.obj
 0001:0002e2d0       ?Grow@?$CUtlMemory@PAVCPhysCollide@@H@@QAEXH@Z 0042f2d0 f i disp_ivp.obj
 0001:0002e2d0       ?Grow@?$CUtlMemory@PAVKeyValues@@H@@QAEXH@Z 0042f2d0 f i tier1:KeyValues.obj
 0001:0002e2d0       ?Grow@?$CUtlMemory@PADH@@QAEXH@Z 0042f2d0 f i cubemap.obj
 0001:0002e2d0       ?Grow@?$CUtlMemory@PAUmapbrush_t@@H@@QAEXH@Z 0042f2d0 f i vbsp.obj
 0001:0002e2d0       ?Grow@?$CUtlMemory@PAVCPhysCollisionEntry@@H@@QAEXH@Z 0042f2d0 f i disp_ivp.obj
 0001:0002e2d0       ?Grow@?$CUtlMemory@PAVCCoreDispInfo@@H@@QAEXH@Z 0042f2d0 f i disp_vbsp.obj
 0001:0002e2d0       ?Grow@?$CUtlMemory@UOccluderInfo_t@@H@@QAEXH@Z 0042f2d0 f i vbsp.obj
 0001:0002e2d0       ?Grow@?$CUtlMemory@HH@@QAEXH@Z 0042f2d0 f i brushbsp.obj
 0001:0002e2d0       ?Grow@?$CUtlMemory@PAVCPhysConvex@@H@@QAEXH@Z 0042f2d0 f i ivp.obj
 0001:0002e2d0       ?Grow@?$CUtlMemory@PAUside_t@@H@@QAEXH@Z 0042f2d0 f i vbsp.obj
 0001:0002e2d0       ?Grow@?$CUtlMemory@PAUbspbrush_t@@H@@QAEXH@Z 0042f2d0 f i detail.obj
 0001:0002e2d0       ?Grow@?$CUtlMemory@PAUdface_t@@H@@QAEXH@Z 0042f2d0 f i disp_vbsp.obj
 0001:0002e2d0       ?Grow@?$CUtlMemory@PAUStringPool_t@CUtlSymbolTable@@H@@QAEXH@Z 0042f2d0 f i tier1:utlsymbol.obj
 0001:0002e2d0       ?Grow@?$CUtlMemory@PAUportal_t@@H@@QAEXH@Z 0042f2d0 f i portals.obj
 0001:0002e480       ?EnsureCapacity@?$CUtlMemory@EH@@QAEXH@Z 0042f480 f i bsplib.obj
 0001:0002e4d0       ??$SwapBufferToTargetEndian@M@CByteswap@@QAEXPAM0H@Z 0042f4d0 f i bsplib.obj
 0001:0002e560       ??$SwapBufferToTargetEndian@G@CByteswap@@QAEXPAG0H@Z 0042f560 f i bsplib.obj
 0001:0002e560       ??$SwapBufferToTargetEndian@F@CByteswap@@QAEXPAF0H@Z 0042f560 f i disp_ivp.obj
 0001:0002e5e0       ??$GetTypeBin@H@CUtlBuffer@@IAEXAAH@Z 0042f5e0 f i bsplib.obj
 0001:0002e640       ??$GetObject@Udoccluderdata_t@@@CUtlBuffer@@IAEXPAUdoccluderdata_t@@@Z 0042f640 f i bsplib.obj
 0001:0002e6c0       ??$CopyLumpInternal@Udleaf_t@@@@YAHHPAUdleaf_t@@H@Z 0042f6c0 f i bsplib.obj
 0001:0002e770       ??$CopyLumpInternal@Udleafambientlighting_t@@@@YAHHPAUdleafambientlighting_t@@H@Z 0042f770 f i bsplib.obj
 0001:0002e840       ??$CopyLumpInternal@Udleafambientindex_t@@@@YAHHPAUdleafambientindex_t@@H@Z 0042f840 f i bsplib.obj
 0001:0002e8f0       ??$CopyLumpInternal@Udmodel_t@@@@YAHHPAUdmodel_t@@H@Z 0042f8f0 f i bsplib.obj
 0001:0002e9b0       ??$CopyLumpInternal@Udvertex_t@@@@YAHHPAUdvertex_t@@H@Z 0042f9b0 f i bsplib.obj
 0001:0002ea70       ??$CopyLumpInternal@Udplane_t@@@@YAHHPAUdplane_t@@H@Z 0042fa70 f i bsplib.obj
 0001:0002eb40       ??$CopyLumpInternal@Udnode_t@@@@YAHHPAUdnode_t@@H@Z 0042fb40 f i bsplib.obj
 0001:0002ebf0       ??$CopyLumpInternal@Utexinfo_s@@@@YAHHPAUtexinfo_s@@H@Z 0042fbf0 f i bsplib.obj
 0001:0002ecc0       ??$CopyLumpInternal@Udtexdata_t@@@@YAHHPAUdtexdata_t@@H@Z 0042fcc0 f i bsplib.obj
 0001:0002ed70       ??$CopyLumpInternal@Vddispinfo_t@@@@YAHHPAVddispinfo_t@@H@Z 0042fd70 f i bsplib.obj
 0001:0002ee40       ??$CopyLumpInternal@VCDispVert@@@@YAHHPAVCDispVert@@H@Z 0042fe40 f i bsplib.obj
 0001:0002ef10       ??$CopyLumpInternal@VCDispTri@@@@YAHHPAVCDispTri@@H@Z 0042ff10 f i bsplib.obj
 0001:0002efc0       ??$CopyLumpInternal@VCFaceMacroTextureInfo@@@@YAHHPAVCFaceMacroTextureInfo@@H@Z 0042ffc0 f i bsplib.obj
 0001:0002f070       ??$CopyLumpInternal@Udface_t@@@@YAHHPAUdface_t@@H@Z 00430070 f i bsplib.obj
 0001:0002f150       ??$CopyLumpInternal@Udfaceid_t@@@@YAHHPAUdfaceid_t@@H@Z 00430150 f i bsplib.obj
 0001:0002f200       ??$CopyLumpInternal@Udprimitive_t@@@@YAHHPAUdprimitive_t@@H@Z 00430200 f i bsplib.obj
 0001:0002f2c0       ??$CopyLumpInternal@Udprimvert_t@@@@YAHHPAUdprimvert_t@@H@Z 004302c0 f i bsplib.obj
 0001:0002f380       ??$CopyLumpInternal@Udedge_t@@@@YAHHPAUdedge_t@@H@Z 00430380 f i bsplib.obj
 0001:0002f430       ??$CopyLumpInternal@Udbrush_t@@@@YAHHPAUdbrush_t@@H@Z 00430430 f i bsplib.obj
 0001:0002f4f0       ??$CopyLumpInternal@Udbrushside_t@@@@YAHHPAUdbrushside_t@@H@Z 004304f0 f i bsplib.obj
 0001:0002f5a0       ??$CopyLumpInternal@Udarea_t@@@@YAHHPAUdarea_t@@H@Z 004305a0 f i bsplib.obj
 0001:0002f650       ??$CopyLumpInternal@Udareaportal_t@@@@YAHHPAUdareaportal_t@@H@Z 00430650 f i bsplib.obj
 0001:0002f710       ??$CopyLumpInternal@Udworldlight_t@@@@YAHHPAUdworldlight_t@@H@Z 00430710 f i bsplib.obj
 0001:0002f7e0       ??$CopyLumpInternal@Udleafwaterdata_t@@@@YAHHPAUdleafwaterdata_t@@H@Z 004307e0 f i bsplib.obj
 0001:0002f8a0       ??$CopyLumpInternal@Udcubemapsample_t@@@@YAHHPAUdcubemapsample_t@@H@Z 004308a0 f i bsplib.obj
 0001:0002f950       ??$CopyLumpInternal@Udoverlay_t@@@@YAHHPAUdoverlay_t@@H@Z 00430950 f i bsplib.obj
 0001:0002fa20       ??$CopyLumpInternal@Udwateroverlay_t@@@@YAHHPAUdwateroverlay_t@@H@Z 00430a20 f i bsplib.obj
 0001:0002fb00       ??$CopyLumpInternal@Udoverlayfade_t@@@@YAHHPAUdoverlayfade_t@@H@Z 00430b00 f i bsplib.obj
 0001:0002fbb0       ??$CopyLumpInternal@Udflagslump_t@@@@YAHHPAUdflagslump_t@@H@Z 00430bb0 f i bsplib.obj
 0001:0002fc60       ?Grow@?$CUtlMemory@U?$UtlLinkedListElem_t@UGameLump_t@@G@@G@@QAEXH@Z 00430c60 f i bsplib.obj
 0001:0002fd20       ?GetGameLump@CGameLump@@QAEPAXG@Z 00430d20 f   bsplib.obj
 0001:0002fd40       ?SwapGameLump@CGameLump@@QAEXHHPAE0H@Z 00430d40 f   bsplib.obj
 0001:000300e0       ?TexDataStringTable_GetString@@YAPBDH@Z 004310e0 f   bsplib.obj
 0001:000306b0       ?Lumps_Write@@YAXXZ        004316b0 f   bsplib.obj
 0001:00030720       ?OpenBSPFile@@YAXPBD@Z     00431720 f   bsplib.obj
 0001:000307e0       ?CalcFaceExtents@@YAXPAUdface_t@@QAH1@Z 004317e0 f   bsplib.obj
 0001:00030a90       ?UpdateAllFaceLightmapExtents@@YAXXZ 00431a90 f   bsplib.obj
 0001:00030ae0       ??$GetObjects@Udoccluderpolydata_t@@@CUtlBuffer@@QAEXPAUdoccluderpolydata_t@@H@Z 00431ae0 f i bsplib.obj
 0001:00030b40       ??$CopyLumpInternal@D@@YAHHHPADH@Z 00431b40 f i bsplib.obj
 0001:00030b40       ??$CopyLumpInternal@E@@YAHHHPAEH@Z 00431b40 f i bsplib.obj
 0001:00030c80       ?InsertMultipleBefore@?$CUtlVector@Udoccluderdata_t@@V?$CUtlMemory@Udoccluderdata_t@@H@@@@QAEHHHPBUdoccluderdata_t@@@Z 00431c80 f i bsplib.obj
 0001:00030ed0       ?InsertMultipleBefore@?$CUtlVector@Udoccluderpolydata_t@@V?$CUtlMemory@Udoccluderpolydata_t@@H@@@@QAEHHHPBUdoccluderpolydata_t@@@Z 00431ed0 f i bsplib.obj
 0001:00030f80       ?AllocInternal@?$CUtlLinkedList@UGameLump_t@@G$0A@GV?$CUtlMemory@U?$UtlLinkedListElem_t@UGameLump_t@@G@@G@@@@IAEG_N@Z 00431f80 f i bsplib.obj
 0001:000310a0       ?InsertMultipleBefore@?$CUtlVector@HV?$CUtlMemory@HH@@@@QAEHHHPBH@Z 004320a0 f i brushbsp.obj
 0001:000310a0       ?InsertMultipleBefore@?$CUtlVector@VS3RGBA@@V?$CUtlMemory@VS3RGBA@@H@@@@QAEHHHPBVS3RGBA@@@Z 004320a0 f i vtf:vtf.obj
 0001:000310a0       ?InsertMultipleBefore@?$CUtlVector@PAVCPhysCollide@@V?$CUtlMemory@PAVCPhysCollide@@H@@@@QAEHHHPBQAVCPhysCollide@@@Z 004320a0 f i disp_ivp.obj
 0001:000310a0       ?InsertMultipleBefore@?$CUtlVector@Udleafambientindex_t@@V?$CUtlMemory@Udleafambientindex_t@@H@@@@QAEHHHPBUdleafambientindex_t@@@Z 004320a0 f i bsplib.obj
 0001:00031140       ?InsertMultipleBefore@?$CUtlVector@VCDispTri@@V?$CUtlMemory@VCDispTri@@H@@@@QAEHHHPBVCDispTri@@@Z 00432140 f i disp_vbsp.obj
 0001:00031140       ?InsertMultipleBefore@?$CUtlVector@VCFaceMacroTextureInfo@@V?$CUtlMemory@VCFaceMacroTextureInfo@@H@@@@QAEHHHPBVCFaceMacroTextureInfo@@@Z 00432140 f i writebsp.obj
 0001:00031140       ?InsertMultipleBefore@?$CUtlVector@Udfaceid_t@@V?$CUtlMemory@Udfaceid_t@@H@@@@QAEHHHPBUdfaceid_t@@@Z 00432140 f i bsplib.obj
 0001:000311e0       ?GetGameLumpHandle@CGameLump@@QAEGH@Z 004321e0 f   bsplib.obj
 0001:00031220       ?ComputeGameLumpSizeAndCount@CGameLump@@QAEXAAH0@Z 00432220 f   bsplib.obj
 0001:00031710       ?Unlink@?$CUtlLinkedList@UGameLump_t@@G$0A@GV?$CUtlMemory@U?$UtlLinkedListElem_t@UGameLump_t@@G@@G@@@@QAEXG@Z 00432710 f i bsplib.obj
 0001:00031870       ?TexDataStringTable_AddOrFindString@@YAHPBD@Z 00432870 f   bsplib.obj
 0001:00031950       ?Lumps_Parse@@YAXXZ        00432950 f   bsplib.obj
 0001:000319b0       ?LoadBSPFile_FileSystemOnly@@YAXPBD@Z 004329b0 f   bsplib.obj
 0001:00031b00       ?WriteBSPFile@@YAXPBDPAD@Z 00432b00 f   bsplib.obj
 0001:00032210       ?SetCount@?$CUtlVector@Udleafambientlighting_t@@V?$CUtlMemory@Udleafambientlighting_t@@H@@@@QAEXH@Z 00433210 f i bsplib.obj
 0001:00032250       ??$DataMapInit@Udheader_t@@@@YAPAUdatamap_t@@PAUdheader_t@@@Z 00433250 f   bsplib.obj
 0001:000322d0       ??$DataMapInit@Ulump_t@@@@YAPAUdatamap_t@@PAUlump_t@@@Z 004332d0 f   bsplib.obj
 0001:00032350       ??$DataMapInit@Udflagslump_t@@@@YAPAUdatamap_t@@PAUdflagslump_t@@@Z 00433350 f   bsplib.obj
 0001:000323d0       ??$DataMapInit@Udplane_t@@@@YAPAUdatamap_t@@PAUdplane_t@@@Z 004333d0 f   bsplib.obj
 0001:00032450       ??$DataMapInit@Udleaf_version_0_t@@@@YAPAUdatamap_t@@PAUdleaf_version_0_t@@@Z 00433450 f   bsplib.obj
 0001:000324d0       ??$DataMapInit@Udleaf_t@@@@YAPAUdatamap_t@@PAUdleaf_t@@@Z 004334d0 f   bsplib.obj
 0001:00032550       ??$DataMapInit@UCompressedLightCube@@@@YAPAUdatamap_t@@PAUCompressedLightCube@@@Z 00433550 f   bsplib.obj
 0001:000325d0       ??$DataMapInit@Udleafambientindex_t@@@@YAPAUdatamap_t@@PAUdleafambientindex_t@@@Z 004335d0 f   bsplib.obj
 0001:00032650       ??$DataMapInit@Udleafambientlighting_t@@@@YAPAUdatamap_t@@PAUdleafambientlighting_t@@@Z 00433650 f   bsplib.obj
 0001:000326d0       ??$DataMapInit@Udvertex_t@@@@YAPAUdatamap_t@@PAUdvertex_t@@@Z 004336d0 f   bsplib.obj
 0001:00032750       ??$DataMapInit@Udnode_t@@@@YAPAUdatamap_t@@PAUdnode_t@@@Z 00433750 f   bsplib.obj
 0001:000327d0       ??$DataMapInit@Utexinfo_s@@@@YAPAUdatamap_t@@PAUtexinfo_s@@@Z 004337d0 f   bsplib.obj
 0001:00032850       ??$DataMapInit@Udtexdata_t@@@@YAPAUdatamap_t@@PAUdtexdata_t@@@Z 00433850 f   bsplib.obj
 0001:000328d0       ??$DataMapInit@Vddispinfo_t@@@@YAPAUdatamap_t@@PAVddispinfo_t@@@Z 004338d0 f   bsplib.obj
 0001:00032950       ??$DataMapInit@VCDispNeighbor@@@@YAPAUdatamap_t@@PAVCDispNeighbor@@@Z 00433950 f   bsplib.obj
 0001:000329d0       ??$DataMapInit@VCDispCornerNeighbors@@@@YAPAUdatamap_t@@PAVCDispCornerNeighbors@@@Z 004339d0 f   bsplib.obj
 0001:00032a50       ??$DataMapInit@UCDispSubNeighbor@@@@YAPAUdatamap_t@@PAUCDispSubNeighbor@@@Z 00433a50 f   bsplib.obj
 0001:00032ad0       ??$DataMapInit@VCDispVert@@@@YAPAUdatamap_t@@PAVCDispVert@@@Z 00433ad0 f   bsplib.obj
 0001:00032b50       ??$DataMapInit@VCDispTri@@@@YAPAUdatamap_t@@PAVCDispTri@@@Z 00433b50 f   bsplib.obj
 0001:00032bd0       ??$DataMapInit@VCFaceMacroTextureInfo@@@@YAPAUdatamap_t@@PAVCFaceMacroTextureInfo@@@Z 00433bd0 f   bsplib.obj
 0001:00032c50       ??$DataMapInit@Udprimitive_t@@@@YAPAUdatamap_t@@PAUdprimitive_t@@@Z 00433c50 f   bsplib.obj
 0001:00032cd0       ??$DataMapInit@Udprimvert_t@@@@YAPAUdatamap_t@@PAUdprimvert_t@@@Z 00433cd0 f   bsplib.obj
 0001:00032d50       ??$DataMapInit@Udface_t@@@@YAPAUdatamap_t@@PAUdface_t@@@Z 00433d50 f   bsplib.obj
 0001:00032dd0       ??$DataMapInit@Udfaceid_t@@@@YAPAUdatamap_t@@PAUdfaceid_t@@@Z 00433dd0 f   bsplib.obj
 0001:00032e50       ??$DataMapInit@Udbrush_t@@@@YAPAUdatamap_t@@PAUdbrush_t@@@Z 00433e50 f   bsplib.obj
 0001:00032ed0       ??$DataMapInit@Udbrushside_t@@@@YAPAUdatamap_t@@PAUdbrushside_t@@@Z 00433ed0 f   bsplib.obj
 0001:00032f50       ??$DataMapInit@Udedge_t@@@@YAPAUdatamap_t@@PAUdedge_t@@@Z 00433f50 f   bsplib.obj
 0001:00032fd0       ??$DataMapInit@Udmodel_t@@@@YAPAUdatamap_t@@PAUdmodel_t@@@Z 00433fd0 f   bsplib.obj
 0001:00033050       ??$DataMapInit@Udphysmodel_t@@@@YAPAUdatamap_t@@PAUdphysmodel_t@@@Z 00434050 f   bsplib.obj
 0001:000330d0       ??$DataMapInit@Udphysdisp_t@@@@YAPAUdatamap_t@@PAUdphysdisp_t@@@Z 004340d0 f   bsplib.obj
 0001:00033150       ??$DataMapInit@Udarea_t@@@@YAPAUdatamap_t@@PAUdarea_t@@@Z 00434150 f   bsplib.obj
 0001:000331d0       ??$DataMapInit@Udareaportal_t@@@@YAPAUdatamap_t@@PAUdareaportal_t@@@Z 004341d0 f   bsplib.obj
 0001:00033250       ??$DataMapInit@Udworldlight_t@@@@YAPAUdatamap_t@@PAUdworldlight_t@@@Z 00434250 f   bsplib.obj
 0001:000332d0       ??$DataMapInit@Udleafwaterdata_t@@@@YAPAUdatamap_t@@PAUdleafwaterdata_t@@@Z 004342d0 f   bsplib.obj
 0001:00033350       ??$DataMapInit@Udoccluderdata_t@@@@YAPAUdatamap_t@@PAUdoccluderdata_t@@@Z 00434350 f   bsplib.obj
 0001:000333d0       ??$DataMapInit@Udoccluderpolydata_t@@@@YAPAUdatamap_t@@PAUdoccluderpolydata_t@@@Z 004343d0 f   bsplib.obj
 0001:00033450       ??$DataMapInit@Udcubemapsample_t@@@@YAPAUdatamap_t@@PAUdcubemapsample_t@@@Z 00434450 f   bsplib.obj
 0001:000334d0       ??$DataMapInit@Udoverlay_t@@@@YAPAUdatamap_t@@PAUdoverlay_t@@@Z 004344d0 f   bsplib.obj
 0001:00033550       ??$DataMapInit@Udwateroverlay_t@@@@YAPAUdatamap_t@@PAUdwateroverlay_t@@@Z 00434550 f   bsplib.obj
 0001:000335d0       ??$DataMapInit@Udoverlayfade_t@@@@YAPAUdatamap_t@@PAUdoverlayfade_t@@@Z 004345d0 f   bsplib.obj
 0001:00033650       ??$DataMapInit@Udgamelumpheader_t@@@@YAPAUdatamap_t@@PAUdgamelumpheader_t@@@Z 00434650 f   bsplib.obj
 0001:000336d0       ??$DataMapInit@Udgamelump_t@@@@YAPAUdatamap_t@@PAUdgamelump_t@@@Z 004346d0 f   bsplib.obj
 0001:00033750       ??$DataMapInit@UStaticPropDictLump_t@@@@YAPAUdatamap_t@@PAUStaticPropDictLump_t@@@Z 00434750 f   bsplib.obj
 0001:000337d0       ??$DataMapInit@UStaticPropLump_t@@@@YAPAUdatamap_t@@PAUStaticPropLump_t@@@Z 004347d0 f   bsplib.obj
 0001:00033850       ??$DataMapInit@UStaticPropLumpV4_t@@@@YAPAUdatamap_t@@PAUStaticPropLumpV4_t@@@Z 00434850 f   bsplib.obj
 0001:000338d0       ??$DataMapInit@UStaticPropLumpV5_t@@@@YAPAUdatamap_t@@PAUStaticPropLumpV5_t@@@Z 004348d0 f   bsplib.obj
 0001:00033950       ??$DataMapInit@UStaticPropLeafLump_t@@@@YAPAUdatamap_t@@PAUStaticPropLeafLump_t@@@Z 00434950 f   bsplib.obj
 0001:000339d0       ??$DataMapInit@UDetailObjectDictLump_t@@@@YAPAUdatamap_t@@PAUDetailObjectDictLump_t@@@Z 004349d0 f   bsplib.obj
 0001:00033a50       ??$DataMapInit@UDetailObjectLump_t@@@@YAPAUdatamap_t@@PAUDetailObjectLump_t@@@Z 00434a50 f   bsplib.obj
 0001:00033ad0       ??$DataMapInit@UDetailSpriteDictLump_t@@@@YAPAUdatamap_t@@PAUDetailSpriteDictLump_t@@@Z 00434ad0 f   bsplib.obj
 0001:00033b50       ??$DataMapInit@UDetailPropLightstylesLump_t@@@@YAPAUdatamap_t@@PAUDetailPropLightstylesLump_t@@@Z 00434b50 f   bsplib.obj
 0001:00033bd0       ??$DataMapInit@UMeshHeader_t@HardwareVerts@@@HardwareVerts@@YAPAUdatamap_t@@PAUMeshHeader_t@0@@Z 00434bd0 f   bsplib.obj
 0001:00033c50       ??$DataMapInit@UFileHeader_t@HardwareVerts@@@HardwareVerts@@YAPAUdatamap_t@@PAUFileHeader_t@0@@Z 00434c50 f   bsplib.obj
 0001:00033ec0       ??$DataMapInit@Uswapcollideheader_t@@@@YAPAUdatamap_t@@PAUswapcollideheader_t@@@Z 00434ec0 f   bsplib.obj
 0001:00033f40       ??$DataMapInit@Uswapcompactsurfaceheader_t@@@@YAPAUdatamap_t@@PAUswapcompactsurfaceheader_t@@@Z 00434f40 f   bsplib.obj
 0001:00033fd0       ??$DataMapInit@Uswapmoppsurfaceheader_t@@@@YAPAUdatamap_t@@PAUswapmoppsurfaceheader_t@@@Z 00434fd0 f   bsplib.obj
 0001:00034060       ?LoadLeafs@@YAHXZ          00435060 f   bsplib.obj
 0001:00034210       ?UnparseEntities@@YAXXZ    00435210 f   bsplib.obj
 0001:00034440       ?RemoveAll@?$CUtlLinkedList@UGameLump_t@@G$0A@GV?$CUtlMemory@U?$UtlLinkedListElem_t@UGameLump_t@@G@@G@@@@QAEXXZ 00435440 f i bsplib.obj
 0001:000344f0       ??$CopyOptionalLump@Udleafambientlighting_t@@@@YAXHAAV?$CUtlVector@Udleafambientlighting_t@@V?$CUtlMemory@Udleafambientlighting_t@@H@@@@H@Z 004354f0 f i bsplib.obj
 0001:00034570       ??$CopyOptionalLump@Udleafambientindex_t@@@@YAXHAAV?$CUtlVector@Udleafambientindex_t@@V?$CUtlMemory@Udleafambientindex_t@@H@@@@H@Z 00435570 f i bsplib.obj
 0001:000345c0       ?SetSize@?$CUtlVector@DV?$CUtlMemory@DH@@@@QAEXH@Z 004355c0 f i scratchpad3d.obj
 0001:000345c0       ?SetSize@?$CUtlVector@EV?$CUtlMemory@EH@@@@QAEXH@Z 004355c0 f i bsplib.obj
 0001:00034610       ?Free@?$CUtlLinkedList@UGameLump_t@@G$0A@GV?$CUtlMemory@U?$UtlLinkedListElem_t@UGameLump_t@@G@@G@@@@QAEXG@Z 00435610 f i bsplib.obj
 0001:00034670       ?LoadLeafAmbientLighting@@YAXH@Z 00435670 f   bsplib.obj
 0001:000348b0       ?AddToTail@?$CUtlLinkedList@UGameLump_t@@G$0A@GV?$CUtlMemory@U?$UtlLinkedListElem_t@UGameLump_t@@G@@G@@@@QAEGXZ 004358b0 f i bsplib.obj
 0001:00034930       ??$CopyLump@D@@YAXHHAAV?$CUtlVector@DV?$CUtlMemory@DH@@@@H@Z 00435930 f i bsplib.obj
 0001:00034930       ??$CopyLump@E@@YAXHHAAV?$CUtlVector@EV?$CUtlMemory@EH@@@@H@Z 00435930 f i bsplib.obj
 0001:000349b0       ?RemoveAll@?$CUtlVector@Udisp_grid_t@@V?$CUtlMemory@Udisp_grid_t@@H@@@@QAEXXZ 004359b0 f i disp_ivp.obj
 0001:000349b0       ?RemoveAll@?$CUtlVector@UDetailObjectGroup_t@@V?$CUtlMemory@UDetailObjectGroup_t@@H@@@@QAEXXZ 004359b0 f i detailobjects.obj
 0001:000349b0       ?RemoveAll@?$CUtlVector@Uclusterlist_t@@V?$CUtlMemory@Uclusterlist_t@@H@@@@QAEXXZ 004359b0 f i bsplib.obj
 0001:00034a50       ?RemoveAll@?$CUtlVector@VCUtlString@@V?$CUtlMemory@VCUtlString@@H@@@@QAEXXZ 00435a50 f i bsplib.obj
 0001:00034ab0       ?CreateGameLump@CGameLump@@QAEGHHHH@Z 00435ab0 f   bsplib.obj
 0001:00034b40       ?DestroyGameLump@CGameLump@@QAEXG@Z 00435b40 f   bsplib.obj
 0001:00034b50       ?ParseGameLump@CGameLump@@QAEXPAUdheader_t@@@Z 00435b50 f   bsplib.obj
 0001:00034c50       ?LoadBSPFile@@YAXPBD@Z     00435c50 f   bsplib.obj
 0001:000357e0       ??1?$CUtlVector@VCUtlString@@V?$CUtlMemory@VCUtlString@@H@@@@QAE@XZ 004367e0 f i bsplib.obj
 0001:00035840       ?Vector2DClear@@YAXAAVVector2D@@@Z 00436840 f i builddisp.obj
 0001:00035850       ?Vector2DAdd@@YAXABVVector2D@@0AAV1@@Z 00436850 f i builddisp.obj
 0001:00035870       ?Vector2DMultiply@@YAXABVVector2D@@MAAV1@@Z 00436870 f i builddisp.obj
 0001:00035890       ?GetCornerNeighbors@CCoreDispSurface@@QAEPAVCDispCornerNeighbors@@H@Z 00436890 f i builddisp.obj
 0001:000358b0       ?GetEdgeNeighbor@CCoreDispSurface@@QAEPAVCDispNeighbor@@H@Z 004368b0 f i builddisp.obj
 0001:000358c0       ?GetType@CCodec@ATI_Compress@@UBE?AW4_CodecType@@XZ 004368c0 f i bitmap:Codec.obj
 0001:000358c0       ?GetPointCount@CCoreDispSurface@@QBEHXZ 004368c0 f i builddisp.obj
 0001:000358d0       ?GetTexCoord@CCoreDispSurface@@QBEXHAAVVector2D@@@Z 004368d0 f i builddisp.obj
 0001:000358f0       ?GetLuxelCoord@CCoreDispSurface@@QBEXHHAAVVector2D@@@Z 004368f0 f i builddisp.obj
 0001:00035920       ?SetFlags@CCoreDispSurface@@QAEXH@Z 00436920 f i builddisp.obj
 0001:00035930       ?GetSAxis@CCoreDispSurface@@QAEXAAVVector@@@Z 00436930 f i builddisp.obj
 0001:00035960       ?GetTAxis@CCoreDispSurface@@QAEXAAVVector@@@Z 00436960 f i builddisp.obj
 0001:00035990       ?GetPointStartIndex@CCoreDispSurface@@QAEHXZ 00436990 f i builddisp.obj
 0001:000359a0       ?GetNormal@CCoreDispSurface@@QAEXAAVVector@@@Z 004369a0 f i builddisp.obj
 0001:00035a00       ?SetBoundingBox@CCoreDispNode@@QAEXABVVector@@0@Z 00436a00 f i builddisp.obj
 0001:00035a30       ?SetErrorTerm@CCoreDispNode@@QAEXM@Z 00436a30 f i builddisp.obj
 0001:00035a40       ?GetErrorTerm@CCoreDispNode@@QAEMXZ 00436a40 f i builddisp.obj
 0001:00035a50       ?GetBufferType@CCodecBuffer_Block@@UBE?BW4_CodecBufferType@@XZ 00436a50 f i bitmap:CodecBuffer_Block.obj
 0001:00035a50       ?MipCount@CVTFTexture@@UBEHXZ 00436a50 f i vtf:vtf.obj
 0001:00035a50       ?GetCenterVertIndex@CCoreDispNode@@QAEHXZ 00436a50 f i builddisp.obj
 0001:00035a60       ?SetNeighborVertIndex@CCoreDispNode@@QAEXHH@Z 00436a60 f i builddisp.obj
 0001:00035a70       ?GetNeighborVertIndex@CCoreDispNode@@QAEHH@Z 00436a70 f i builddisp.obj
 0001:00035a80       ?SetTriBoundingBox@CCoreDispNode@@QAEXHABVVector@@0@Z 00436a80 f i builddisp.obj
 0001:00035ac0       ?GetTriBoundingBox@CCoreDispNode@@QAEXHAAVVector@@0@Z 00436ac0 f i builddisp.obj
 0001:00035b00       ?SetTriPlane@CCoreDispNode@@QAEXHABVVector@@M@Z 00436b00 f i builddisp.obj
 0001:00035b40       ?SetRayBoundingBox@CCoreDispNode@@QAEXHABVVector@@0@Z 00436b40 f i builddisp.obj
 0001:00035b90       ?GetPostSpacing@CCoreDispInfo@@QAEHXZ 00436b90 f i builddisp.obj
 0001:00035ba0       ?GetNodeLevel@@YAHH@Z      00436ba0 f   builddisp.obj
 0001:00035be0       ?GetNodeCount@@YAHH@Z      00436be0 f   builddisp.obj
 0001:00035c00       ?GetNodeChild@@YAHHHH@Z    00436c00 f   builddisp.obj
 0001:00035c10       ?CalcBarycentricCooefs@@YA_NABVVector@@000AAM11@Z 00436c10 f   builddisp.obj
 0001:00035e10       ?Init@CCoreDispSurface@@QAEXXZ 00436e10 f   builddisp.obj
 0001:00035fd0       ?FindSurfPointStartIndex@CCoreDispSurface@@QAEHXZ 00436fd0 f   builddisp.obj
 0001:000360c0       ?AdjustSurfPointData@CCoreDispSurface@@QAEXXZ 004370c0 f   builddisp.obj
 0001:00036370       ?LongestInU@CCoreDispSurface@@IAE_NABVVector@@0@Z 00437370 f   builddisp.obj
 0001:000364d0       ?CalcLuxelCoords@CCoreDispSurface@@QAE_NH_NABVVector@@1@Z 004374d0 f   builddisp.obj
 0001:000368e0       ?Init@CCoreDispNode@@QAEXXZ 004378e0 f   builddisp.obj
 0001:00036a10       ??1CCoreDispInfo@@QAE@XZ   00437a10 f   builddisp.obj
 0001:00036ab0       ??0CoreDispVert_t@@QAE@XZ  00437ab0 f i builddisp.obj
 0001:00036b40       ?SetDispUtilsHelperInfo@CCoreDispInfo@@QAEXPAPAV1@H@Z 00437b40 f   builddisp.obj
 0001:00036b70       ?GetPowerInfo@CCoreDispInfo@@UBEPBVCPowerInfo@@XZ 00437b70 f   builddisp.obj
 0001:00036b90       ?GetEdgeNeighbor@CCoreDispInfo@@UAEPAVCDispNeighbor@@H@Z 00437b90 f   builddisp.obj
 0001:00036bb0       ?GetCornerNeighbors@CCoreDispInfo@@UAEPAVCDispCornerNeighbors@@H@Z 00437bb0 f   builddisp.obj
 0001:00036bd0       ?GetDispUtilsByIndex@CCoreDispInfo@@UAEPAVCDispUtilsHelper@@H@Z 00437bd0 f   builddisp.obj
 0001:00036c10       ?BuildTriTLtoBR@CCoreDispInfo@@AAEXH@Z 00437c10 f   builddisp.obj
 0001:00036d10       ?BuildTriBLtoTR@CCoreDispInfo@@AAEXH@Z 00437d10 f   builddisp.obj
 0001:00036e10       ?GenerateCollisionSurface@CCoreDispInfo@@AAEXXZ 00437e10 f   builddisp.obj
 0001:00036ee0       ?GenerateCollisionData@CCoreDispInfo@@AAEXXZ 00437ee0 f   builddisp.obj
 0001:00036f00       ?CalcTriSurfPlanes@CCoreDispInfo@@AAEXHQAY02H@Z 00437f00 f   builddisp.obj
 0001:000370f0       ?CalcRayBoundingBoxes@CCoreDispInfo@@AAEXHQAY02H@Z 004380f0 f   builddisp.obj
 0001:00037850       ?CalcTriSurfBoundingBoxes@CCoreDispInfo@@AAEXHQAY02H@Z 00438850 f   builddisp.obj
 0001:00037bd0       ?CalcTriSurfIndices@CCoreDispInfo@@AAEXHQAY02H@Z 00438bd0 f   builddisp.obj
 0001:00037e30       ?CalcTriSurfInfoAtNode@CCoreDispInfo@@AAEXH@Z 00438e30 f   builddisp.obj
 0001:00037e80       ?CalcMinMaxBoundingBoxAtNode@CCoreDispInfo@@AAEXHAAVVector@@0@Z 00438e80 f   builddisp.obj
 0001:000380a0       ?CalcBoundingBoxAtNode@CCoreDispInfo@@AAEXH@Z 004390a0 f   builddisp.obj
 0001:00038650       ?GetMaxErrorFromChildren@CCoreDispInfo@@AAEMHH@Z 00439650 f   builddisp.obj
 0001:000386e0       ?CalcErrorTermAtNode@CCoreDispInfo@@AAEXHH@Z 004396e0 f   builddisp.obj
 0001:00038cf0       ?CalcNeighborVertIndicesAtNode@CCoreDispInfo@@AAEXHH@Z 00439cf0 f   builddisp.obj
 0001:00038e80       ?CalcNodeInfo@CCoreDispInfo@@AAEXHH@Z 00439e80 f   builddisp.obj
 0001:00038f30       ?GetNodeVertIndexFromParentIndex@CCoreDispInfo@@AAEHHHH@Z 00439f30 f   builddisp.obj
 0001:00039010       ?CalcVertIndicesAtNodes@CCoreDispInfo@@AAEXH@Z 0043a010 f   builddisp.obj
 0001:000390f0       ?GenerateLODTree@CCoreDispInfo@@AAEXXZ 0043a0f0 f   builddisp.obj
 0001:00039160       ?CalcDispSurfCoords@CCoreDispInfo@@QAEX_NH@Z 0043a160 f   builddisp.obj
 0001:00039470       ?GenerateDispSurfTangentSpaces@CCoreDispInfo@@AAEXXZ 0043a470 f   builddisp.obj
 0001:000396e0       ?CalcNormalFromEdges@CCoreDispInfo@@AAEXHHQA_NAAVVector@@@Z 0043a6e0 f   builddisp.obj
 0001:0003a2f0       ?DoesEdgeExist@CCoreDispInfo@@AAE_NHHHH@Z 0043b2f0 f   builddisp.obj
 0001:0003a380       ?GenerateDispSurfNormals@CCoreDispInfo@@AAEXXZ 0043b380 f   builddisp.obj
 0001:0003a480       ?GenerateDispSurf@CCoreDispInfo@@AAEXXZ 0043b480 f   builddisp.obj
 0001:0003a9c0       ?DispUVToSurf_TriTLToBR_2@CCoreDispInfo@@AAEXABVVector@@HHHHAAV2@PAV2@PAM_N@Z 0043b9c0 f   builddisp.obj
 0001:0003b030       ?DispUVToSurf_TriBLToTR_2@CCoreDispInfo@@AAEXABVVector@@HHHHAAV2@PAV2@PAM_N@Z 0043c030 f   builddisp.obj
 0001:0003b690       ?GetTriCount@CCoreDispInfo@@QAEHXZ 0043c690 f   builddisp.obj
 0001:0003b6a0       ?InitTris@CCoreDispInfo@@AAEXXZ 0043c6a0 f   builddisp.obj
 0001:0003b6f0       ?CreateTris@CCoreDispInfo@@AAEXXZ 0043c6f0 f   builddisp.obj
 0001:0003b770       ??0CCoreDispSurface@@QAE@XZ 0043c770 f   builddisp.obj
 0001:0003b810       ??0CCoreDispNode@@QAE@XZ   0043c810 f i builddisp.obj
 0001:0003b880       ?Create@CCoreDispInfo@@QAE_NXZ 0043c880 f   builddisp.obj
 0001:0003b910       ?DispUVToSurf_TriTLToBR_1@CCoreDispInfo@@AAEXABVVector@@HHHHAAV2@PAV2@PAM_N@Z 0043c910 f   builddisp.obj
 0001:0003bf30       ?DispUVToSurf_TriTLToBR@CCoreDispInfo@@AAEXAAVVector@@PAV2@PAMMMABV2@@Z 0043cf30 f   builddisp.obj
 0001:0003bfd0       ?DispUVToSurf_TriBLToTR_1@CCoreDispInfo@@AAEXABVVector@@HHHHAAV2@PAV2@PAM_N@Z 0043cfd0 f   builddisp.obj
 0001:0003c600       ?DispUVToSurf_TriBLToTR@CCoreDispInfo@@AAEXAAVVector@@PAV2@PAMMMABV2@@Z 0043d600 f   builddisp.obj
 0001:0003c690       ?DispUVToSurf@CCoreDispInfo@@QAEXABVVector2D@@AAVVector@@PAV3@PAM@Z 0043d690 f   builddisp.obj
 0001:0003c7c0       ?InitDispInfo@CCoreDispInfo@@QAEXHHMPAMPAVVector@@0@Z 0043d7c0 f   builddisp.obj
 0001:0003ccb0       ?GetPositionOnSurface@CCoreDispInfo@@QAEXMMAAVVector@@PAV2@PAM@Z 0043dcb0 f   builddisp.obj
 0001:0003ccf0       ??0?$CBitVec@$0BCB@@@QAE@XZ 0043dcf0 f i builddisp.obj
 0001:0003cd20       ??0CCoreDispInfo@@QAE@XZ   0043dd20 f   builddisp.obj
 0001:0003ce00       ?_Decref@facet@locale@std@@QAEPAV123@XZ 0043de00 f i chunkfile.obj
 0001:0003ce40       ??1locale@std@@QAE@XZ      0043de40 f i chunkfile.obj
 0001:0003ce90       ??_Eios_base@std@@UAEPAXI@Z 0043de90 f i chunkfile.obj
 0001:0003ce90       ??_Gios_base@std@@UAEPAXI@Z 0043de90 f i chunkfile.obj
 0001:0003ce90       ??_G?$basic_ios@DU?$char_traits@D@std@@@std@@UAEPAXI@Z 0043de90 f i tier1:tokenreader.obj
 0001:0003ce90       ??_E?$basic_ios@DU?$char_traits@D@std@@@std@@UAEPAXI@Z 0043de90 f i tier1:tokenreader.obj
 0001:0003cec0       ??0CChunkHandlerMap@@QAE@XZ 0043dec0 f   chunkfile.obj
 0001:0003ced0       ??1CChunkHandlerMap@@QAE@XZ 0043ded0 f   chunkfile.obj
 0001:0003cef0       ?AddHandler@CChunkHandlerMap@@QAEXPBDP6A?AW4ChunkFileResult_t@@PAVCChunkFile@@PAX@Z2@Z 0043def0 f   chunkfile.obj
 0001:0003cf50       ?GetHandler@CChunkHandlerMap@@QAEP6A?AW4ChunkFileResult_t@@PAVCChunkFile@@PAX@ZPBDPAPAX@Z 0043df50 f   chunkfile.obj
 0001:0003cf90       ?GetErrorText@CChunkFile@@QAEPBDW4ChunkFileResult_t@@@Z 0043df90 f   chunkfile.obj
 0001:0003d090       ?Open@CChunkFile@@QAE?AW4ChunkFileResult_t@@PBDW4ChunkFileOpenMode_t@@@Z 0043e090 f   chunkfile.obj
 0001:0003d0f0       ?PopHandlers@CChunkFile@@QAEXXZ 0043e0f0 f   chunkfile.obj
 0001:0003d110       ?PushHandlers@CChunkFile@@QAEXPAVCChunkHandlerMap@@@Z 0043e110 f   chunkfile.obj
 0001:0003d130       ?ReadNext@CChunkFile@@QAE?AW4ChunkFileResult_t@@PAD0HAAW4ChunkType_t@@@Z 0043e130 f   chunkfile.obj
 0001:0003d2f0       ?ReadKeyValueFloat@CChunkFile@@SA_NPBDAAM@Z 0043e2f0 f   chunkfile.obj
 0001:0003d310       ?ReadKeyValueInt@CChunkFile@@SA_NPBDAAH@Z 0043e310 f   chunkfile.obj
 0001:0003d330       ?ReadKeyValueVector3@CChunkFile@@SA_NPBDAAVVector@@@Z 0043e330 f   chunkfile.obj
 0001:0003d370       ?HandleChunk@CChunkFile@@QAE?AW4ChunkFileResult_t@@PBD@Z 0043e370 f   chunkfile.obj
 0001:0003d480       ?ReadChunk@CChunkFile@@QAE?AW4ChunkFileResult_t@@P6A?AW42@PBD0PAX@Z1@Z 0043e480 f   chunkfile.obj
 0001:0003d510       ??1?$basic_streambuf@DU?$char_traits@D@std@@@std@@UAE@XZ 0043e510 f i chunkfile.obj
 0001:0003d590       ?pbackfail@?$basic_streambuf@DU?$char_traits@D@std@@@std@@MAEHH@Z 0043e590 f i chunkfile.obj
 0001:0003d590       ?overflow@?$basic_streambuf@DU?$char_traits@D@std@@@std@@MAEHH@Z 0043e590 f i chunkfile.obj
 0001:0003d5a0       ?underflow@?$basic_streambuf@DU?$char_traits@D@std@@@std@@MAEHXZ 0043e5a0 f i chunkfile.obj
 0001:0003d5b0       ?xsgetn@?$basic_streambuf@DU?$char_traits@D@std@@@std@@MAEHPADH@Z 0043e5b0 f i chunkfile.obj
 0001:0003d5d0       ?setbuf@?$basic_streambuf@DU?$char_traits@D@std@@@std@@MAEPAV12@PADH@Z 0043e5d0 f i chunkfile.obj
 0001:0003d5e0       ?imbue@?$basic_streambuf@DU?$char_traits@D@std@@@std@@MAEXABVlocale@2@@Z 0043e5e0 f i chunkfile.obj
 0001:0003d5f0       ?_Gnavail@?$basic_streambuf@DU?$char_traits@D@std@@@std@@IBEHXZ 0043e5f0 f i chunkfile.obj
 0001:0003d610       ?_Pnavail@?$basic_streambuf@DU?$char_traits@D@std@@@std@@IBEHXZ 0043e610 f i chunkfile.obj
 0001:0003d630       ?uflow@?$basic_streambuf@DU?$char_traits@D@std@@@std@@MAEHXZ 0043e630 f i chunkfile.obj
 0001:0003d660       ?seekoff@?$basic_streambuf@DU?$char_traits@D@std@@@std@@MAE?AV?$fpos@H@2@JHH@Z 0043e660 f i chunkfile.obj
 0001:0003d680       ?seekpos@?$basic_streambuf@DU?$char_traits@D@std@@@std@@MAE?AV?$fpos@H@2@V32@H@Z 0043e680 f i chunkfile.obj
 0001:0003d6a0       ??_E?$basic_istream@DU?$char_traits@D@std@@@std@@UAEPAXI@Z 0043e6a0 f i chunkfile.obj
 0001:0003d6a0       ??_G?$basic_istream@DU?$char_traits@D@std@@@std@@UAEPAXI@Z 0043e6a0 f i chunkfile.obj
 0001:0003d6e0       ??_G?$basic_streambuf@DU?$char_traits@D@std@@@std@@UAEPAXI@Z 0043e6e0 f i chunkfile.obj
 0001:0003d6e0       ??_E?$basic_streambuf@DU?$char_traits@D@std@@@std@@UAEPAXI@Z 0043e6e0 f i chunkfile.obj
 0001:0003d700       ??D?$_String_iterator@DU?$char_traits@D@std@@V?$allocator@D@2@@std@@QBEAADXZ 0043e700 f i chunkfile.obj
 0001:0003d740       ?_Chassign@?$basic_string@DU?$char_traits@D@std@@V?$allocator@D@2@@std@@IAEXIID@Z 0043e740 f i chunkfile.obj
 0001:0003d7a0       ?_Init@?$basic_streambuf@DU?$char_traits@D@std@@@std@@IAEXXZ 0043e7a0 f i chunkfile.obj
 0001:0003d800       ??0?$_String_const_iterator@DU?$char_traits@D@std@@V?$allocator@D@2@@std@@QAE@PBDPBU_Container_base@1@@Z 0043e800 f i chunkfile.obj
 0001:0003d860       ?_Xsgetn_s@?$basic_streambuf@DU?$char_traits@D@std@@@std@@MAEHPADIH@Z 0043e860 f i chunkfile.obj
 0001:0003d900       ?xsputn@?$basic_streambuf@DU?$char_traits@D@std@@@std@@MAEHPBDH@Z 0043e900 f i chunkfile.obj
 0001:0003d9a0       ?begin@?$basic_string@DU?$char_traits@D@std@@V?$allocator@D@2@@std@@QAE?AV?$_String_iterator@DU?$char_traits@D@std@@V?$allocator@D@2@@2@XZ 0043e9a0 f i chunkfile.obj
 0001:0003d9e0       ?append@?$basic_string@DU?$char_traits@D@std@@V?$allocator@D@2@@std@@QAEAAV12@ID@Z 0043e9e0 f i chunkfile.obj
 0001:0003da90       ?_Endwrite@?$basic_filebuf@DU?$char_traits@D@std@@@std@@IAE_NXZ 0043ea90 f i chunkfile.obj
 0001:0003dd80       ?close@?$basic_filebuf@DU?$char_traits@D@std@@@std@@QAEPAV12@XZ 0043ed80 f i chunkfile.obj
 0001:0003ddd0       ?_Incref@facet@locale@std@@QAEXXZ 0043edd0 f i chunkfile.obj
 0001:0003de00       ??1facet@locale@std@@UAE@XZ 0043ee00 f i chunkfile.obj
 0001:0003de10       ??_E?$codecvt@DDH@std@@MAEPAXI@Z 0043ee10 f i chunkfile.obj
 0001:0003de10       ??_Efacet@locale@std@@UAEPAXI@Z 0043ee10 f i chunkfile.obj
 0001:0003de10       ??_G?$codecvt@DDH@std@@MAEPAXI@Z 0043ee10 f i chunkfile.obj
 0001:0003de10       ??_Gfacet@locale@std@@UAEPAXI@Z 0043ee10 f i chunkfile.obj
 0001:0003de30       ?do_always_noconv@codecvt_base@std@@MBE_NXZ 0043ee30 f i chunkfile.obj
 0001:0003de40       ?GetBufferType@CCodecBuffer_RGBA8888@@UBE?BW4_CodecBufferType@@XZ 0043ee40 f i bitmap:CodecBuffer_RGBA8888.obj
 0001:0003de40       ?do_encoding@codecvt_base@std@@MBEHXZ 0043ee40 f i chunkfile.obj
 0001:0003de40       ?GetBlockHeight@CCodec@ATI_Compress@@UAEKXZ 0043ee40 f i bitmap:Codec.obj
 0001:0003de40       ?do_max_length@codecvt_base@std@@MBEHXZ 0043ee40 f i chunkfile.obj
 0001:0003de50       ??$_Fputc@D@std@@YA_NDPAU_iobuf@@@Z 0043ee50 f i chunkfile.obj
 0001:0003de70       ?sync@?$basic_filebuf@DU?$char_traits@D@std@@@std@@MAEHXZ 0043ee70 f i chunkfile.obj
 0001:0003dea0       ?pbackfail@?$basic_filebuf@DU?$char_traits@D@std@@@std@@MAEHH@Z 0043eea0 f i chunkfile.obj
 0001:0003df10       ?underflow@?$basic_filebuf@DU?$char_traits@D@std@@@std@@MAEHXZ 0043ef10 f i chunkfile.obj
 0001:0003df60       ?setbuf@?$basic_filebuf@DU?$char_traits@D@std@@@std@@MAEPAV?$basic_streambuf@DU?$char_traits@D@std@@@2@PADH@Z 0043ef60 f i chunkfile.obj
 0001:0003dfe0       ??1_Locinfo@std@@QAE@XZ    0043efe0 f i chunkfile.obj
 0001:0003e070       ?uflow@?$basic_filebuf@DU?$char_traits@D@std@@@std@@MAEHXZ 0043f070 f i chunkfile.obj
 0001:0003e3a0       ??_Gruntime_error@std@@UAEPAXI@Z 0043f3a0 f i chunkfile.obj
 0001:0003e3a0       ??_Efailure@ios_base@std@@UAEPAXI@Z 0043f3a0 f i tier1:tokenreader.obj
 0001:0003e3a0       ??_Gfailure@ios_base@std@@UAEPAXI@Z 0043f3a0 f i tier1:tokenreader.obj
 0001:0003e3a0       ??_Eruntime_error@std@@UAEPAXI@Z 0043f3a0 f i chunkfile.obj
 0001:0003e3f0       ?overflow@?$basic_filebuf@DU?$char_traits@D@std@@@std@@MAEHH@Z 0043f3f0 f i chunkfile.obj
 0001:0003e790       ?seekoff@?$basic_filebuf@DU?$char_traits@D@std@@@std@@MAE?AV?$fpos@H@2@JHH@Z 0043f790 f i chunkfile.obj
 0001:0003e870       ?seekpos@?$basic_filebuf@DU?$char_traits@D@std@@@std@@MAE?AV?$fpos@H@2@V32@H@Z 0043f870 f i chunkfile.obj
 0001:0003e960       ??0_Locinfo@std@@QAE@PBD@Z 0043f960 f i chunkfile.obj
 0001:0003ea10       ??0runtime_error@std@@QAE@ABV01@@Z 0043fa10 f i chunkfile.obj
 0001:0003ea50       ??_G?$basic_filebuf@DU?$char_traits@D@std@@@std@@UAEPAXI@Z 0043fa50 f i chunkfile.obj
 0001:0003ea50       ??_E?$basic_filebuf@DU?$char_traits@D@std@@@std@@UAEPAXI@Z 0043fa50 f i chunkfile.obj
 0001:0003ea90       ??0?$codecvt@DDH@std@@QAE@I@Z 0043fa90 f i chunkfile.obj
 0001:0003ead0       ?do_out@?$codecvt@DDH@std@@MBEHAAHPBD1AAPBDPAD3AAPAD@Z 0043fad0 f i chunkfile.obj
 0001:0003ead0       ?do_in@?$codecvt@DDH@std@@MBEHAAHPBD1AAPBDPAD3AAPAD@Z 0043fad0 f i chunkfile.obj
 0001:0003eaf0       ?do_unshift@?$codecvt@DDH@std@@MBEHAAHPAD1AAPAD@Z 0043faf0 f i chunkfile.obj
 0001:0003eb10       ?do_length@?$codecvt@DDH@std@@MBEHABHPBD1I@Z 0043fb10 f i chunkfile.obj
 0001:0003eb30       ??_D?$basic_ifstream@DU?$char_traits@D@std@@@std@@QAEXXZ 0043fb30 f i chunkfile.obj
 0001:0003eb80       ??_G?$basic_ifstream@DU?$char_traits@D@std@@@std@@UAEPAXI@Z 0043fb80 f i chunkfile.obj
 0001:0003eb80       ??_E?$basic_ifstream@DU?$char_traits@D@std@@@std@@UAEPAXI@Z 0043fb80 f i chunkfile.obj
 0001:0003ebb0       ??$use_facet@V?$codecvt@DDH@std@@@std@@YAABV?$codecvt@DDH@0@ABVlocale@0@@Z 0043fbb0 f i chunkfile.obj
 0001:0003eca0       ??_DTokenReader@@QAEXXZ    0043fca0 f i chunkfile.obj
 0001:0003ed00       ??0CChunkFile@@QAE@XZ      0043fd00 f   chunkfile.obj
 0001:0003ed30       ??1CChunkFile@@QAE@XZ      0043fd30 f   chunkfile.obj
 0001:0003ed50       ?imbue@?$basic_filebuf@DU?$char_traits@D@std@@@std@@MAEXABVlocale@2@@Z 0043fd50 f i chunkfile.obj
 0001:0003ee10       ?SetConsoleTextColor@@YAGHHHH@Z 0043fe10 f   cmdlib.obj
 0001:0003eea0       ?CmdLib_Exit@@YAXH@Z       0043fea0 f   cmdlib.obj
 0001:0003eeb0       ?qprintf@@YAXPADZZ         0043feb0 f   cmdlib.obj
 0001:0003ef00       ?ExpandArg@@YAPADPAD@Z     0043ff00 f   cmdlib.obj
 0001:0003ef80       ?copystring@@YAPADPBD@Z    0043ff80 f   cmdlib.obj
 0001:0003efc0       ?GetHourMinuteSecondsString@@YAXHPADH@Z 0043ffc0 f   cmdlib.obj
 0001:0003f0d0       ?CmdLib_InitFileSystem@@YAXPBDH@Z 004400d0 f   cmdlib.obj
 0001:0003f100       ?CmdLib_GetFileSystemFactory@@YAP6APAXPBDPAH@ZXZ 00440100 f   cmdlib.obj
 0001:0003f110       ?SafeOpenWrite@@YAPAXPBD@Z 00440110 f   cmdlib.obj
 0001:0003f150       ?CmdLib_HasBasePath@@YA_NPBDAAH@Z 00440150 f   cmdlib.obj
 0001:0003f220       ?SafeOpenRead@@YAPAXPBD@Z  00440220 f   cmdlib.obj
 0001:0003f340       ?SafeWrite@@YAXPAX0H@Z     00440340 f   cmdlib.obj
 0001:0003f370       ?FileExists@@YAHPBD@Z      00440370 f   cmdlib.obj
 0001:0003f3b0       ?LoadFile@@YAHPBDPAPAX@Z   004403b0 f   cmdlib.obj
 0001:0003f430       ?RemoveAll@?$CUtlLinkedList@PAVCZip@@G$0A@GV?$CUtlMemory@U?$UtlLinkedListElem_t@PAVCZip@@G@@G@@@@QAEXXZ 00440430 f i zip_utils.obj
 0001:0003f430       ?RemoveAll@?$CUtlLinkedList@P6AXXZG$0A@GV?$CUtlMemory@U?$UtlLinkedListElem_t@P6AXXZG@@G@@@@QAEXXZ 00440430 f i cmdlib.obj
 0001:0003f430       ?RemoveAll@?$CUtlLinkedList@P6AXPBD@ZG$0A@GV?$CUtlMemory@U?$UtlLinkedListElem_t@P6AXPBD@ZG@@G@@@@QAEXXZ 00440430 f i cmdlib.obj
 0001:0003f4a0       ?CmdLib_Cleanup@@YAXXZ     004404a0 f   cmdlib.obj
 0001:0003f510       ?CmdLib_FPrintf@@YAXPAXPBDZZ 00440510 f   cmdlib.obj
 0001:0003f6a0       ?CmdLib_SpewOutputFunc@@YA?AW4SpewRetval_t@@W4SpewType_t@@PBD@Z 004406a0 f   cmdlib.obj
 0001:0003f990       ?InstallSpewFunction@@YAXXZ 00440990 f   cmdlib.obj
 0001:0003f9d0       ?SetSpewFunctionLogFile@@YAXPBD@Z 004409d0 f   cmdlib.obj
 0001:0003fa20       ?SetValue@CTempEnvVar@@QAAXPBDZZ 00440a20 f i filesystem_init.obj
 0001:0003fa90       ?Q_getwd@@YAXPADH@Z        00440a90 f   filesystem_init.obj
 0001:0003fac0       ??0CFSSearchPathsInit@@QAE@XZ 00440ac0 f   filesystem_init.obj
 0001:0003fad0       ??0CFSLoadModuleInfo@@QAE@XZ 00440ad0 f   filesystem_init.obj
 0001:0003fb00       ??0CFSMountContentInfo@@QAE@XZ 00440b00 f   filesystem_init.obj
 0001:0003fb10       ?AddLanguageGameDir@@YAXPAVIFileSystem@@PBD1@Z 00440b10 f   filesystem_init.obj
 0001:0003fbe0       ?GetVProjectCmdLineValue@@YAPBDXZ 00440be0 f   filesystem_init.obj
 0001:0003fc20       ?IsLowViolenceBuild@@YA_NXZ 00440c20 f   filesystem_init.obj
 0001:0003fe90       ?DoesFileExistIn@@YA_NPBD0@Z 00440e90 f   filesystem_init.obj
 0001:0003ff00       ?DoesPathExistAlready@@YA_NPBD0@Z 00440f00 f   filesystem_init.obj
 0001:00040040       ?SetSteamUserPassphrase@@YAXPAVKeyValues@@AAVCSteamEnvVars@@@Z 00441040 f   filesystem_init.obj
 0001:000400a0       ?FileSystem_AddSearchPath_Platform@@YAXPAVIFileSystem@@PBD@Z 004410a0 f   filesystem_init.obj
 0001:00040130       ?FileSystem_GetExecutableDir@@YA_NPADH@Z 00441130 f   filesystem_init.obj
 0001:00040250       ?LaunchVConfig@@YAXXZ      00441250 f   filesystem_init.obj
 0001:000402c0       ?SetupFileSystemError@@YA?AW4FSReturnCode_t@@_NW41@PBDZZ 004412c0 f   filesystem_init.obj
 0001:00040350       ?FileSystem_IsHldsUpdateToolDedicatedServer@@YA_NXZ 00441350 f   filesystem_init.obj
 0001:000403d0       ?SetSteamInstallPath@@YA?AW4FSReturnCode_t@@PADHAAVCSteamEnvVars@@_N@Z 004413d0 f   filesystem_init.obj
 0001:00040530       ?FileSystem_SetBasePaths@@YA?AW4FSReturnCode_t@@PAVIFileSystem@@@Z 00441530 f   filesystem_init.obj
 0001:000405a0       ?FileSystem_GetFileSystemDLLName@@YA?AW4FSReturnCode_t@@PADHAA_N@Z 004415a0 f   filesystem_init.obj
 0001:00040670       ??1CTempEnvVar@@QAE@XZ     00441670 f i filesystem_init.obj
 0001:000408b0       ?LocateGameInfoFile@@YA?AW4FSReturnCode_t@@ABVCFSSteamSetupInfo@@PADH@Z 004418b0 f   filesystem_init.obj
 0001:00040ab0       ??1CSteamEnvVars@@QAE@XZ   00441ab0 f i filesystem_init.obj
 0001:00040ae0       ??0CTempEnvVar@@QAE@PBD@Z  00441ae0 f i filesystem_init.obj
 0001:00040b80       ?ReadKeyValuesFile@@YAPAVKeyValues@@PBD@Z 00441b80 f   filesystem_init.obj
 0001:00040c60       ?LoadGameInfoFile@@YA?AW4FSReturnCode_t@@PBDAAPAVKeyValues@@11@Z 00441c60 f   filesystem_init.obj
 0001:00040d50       ?FileSystem_LoadSearchPaths@@YA?AW4FSReturnCode_t@@AAVCFSSearchPathsInit@@@Z 00441d50 f   filesystem_init.obj
 0001:00040f50       ?SetSteamAppUser@@YAXPAVKeyValues@@PBDAAVCSteamEnvVars@@@Z 00441f50 f   filesystem_init.obj
 0001:00041080       ?SetupSteamStartupEnvironment@@YA?AW4FSReturnCode_t@@PAVKeyValues@@PBDAAVCSteamEnvVars@@@Z 00442080 f   filesystem_init.obj
 0001:00041170       ?GetSteamExtraAppId@@YA?AW4FSReturnCode_t@@PBDPAH@Z 00442170 f   filesystem_init.obj
 0001:000411c0       ?FileSystem_SetupSteamInstallPath@@YA?AW4FSReturnCode_t@@XZ 004421c0 f   filesystem_init.obj
 0001:00041250       ?FileSystem_SetupSteamEnvironment@@YA?AW4FSReturnCode_t@@AAVCFSSteamSetupInfo@@@Z 00442250 f   filesystem_init.obj
 0001:000413c0       ?FileSystem_LoadFileSystemModule@@YA?AW4FSReturnCode_t@@AAVCFSLoadModuleInfo@@@Z 004423c0 f   filesystem_init.obj
 0001:00041480       ?FileSystem_MountContent@@YA?AW4FSReturnCode_t@@AAVCFSMountContentInfo@@@Z 00442480 f   filesystem_init.obj
 0001:000415a0       ?FileSystem_SetupStandardDirectories@@YAXPBD0@Z 004425a0 f   filesystem_tools.obj
 0001:00041620       ?FileSystem_Init_Normal@@YA_NPBDW4FSInitType_t@@_N@Z 00442620 f   filesystem_tools.obj
 0001:00041830       ?FileSystem_Init@@YA_NPBDHW4FSInitType_t@@_N@Z 00442830 f   filesystem_tools.obj
 0001:00041850       ?FileSystem_Term@@YAXXZ    00442850 f   filesystem_tools.obj
 0001:000418a0       ?FileSystem_GetFactory@@YAP6APAXPBDPAH@ZXZ 004428a0 f   filesystem_tools.obj
 0001:000418b0       ?LoadEntityKeyCallback@@YA?AW4ChunkFileResult_t@@PBD0PAULoadEntity_t@@@Z 004428b0 f   map_shared.obj
 0001:000419c0       ?UpdatePacifier@@YAXM@Z    004429c0 f   pacifier.obj
 0001:00041a50       ?EndPacifier@@YAX_N@Z      00442a50 f   pacifier.obj
 0001:00041a80       ?StartPacifier@@YAXPBD@Z   00442a80 f   pacifier.obj
 0001:00041ab0       ?AllocWinding@@YAPAUwinding_t@@H@Z 00442ab0 f   polylib.obj
 0001:00041b40       ?FreeWinding@@YAXPAUwinding_t@@@Z 00442b40 f   polylib.obj
 0001:00041b80       ?WindingPlane@@YAXPAUwinding_t@@AAVVector@@PAM@Z 00442b80 f   polylib.obj
 0001:00041c10       ?WindingArea@@YAMPAUwinding_t@@@Z 00442c10 f   polylib.obj
 0001:00041cc0       ?WindingCenter@@YAXPAUwinding_t@@AAVVector@@@Z 00442cc0 f   polylib.obj
 0001:00041d40       ?BaseWindingForPlane@@YAPAUwinding_t@@ABVVector@@M@Z 00442d40 f   polylib.obj
 0001:00041fb0       ?CopyWinding@@YAPAUwinding_t@@PAU1@@Z 00442fb0 f   polylib.obj
 0001:00041ff0       ?ReverseWinding@@YAPAUwinding_t@@PAU1@@Z 00442ff0 f   polylib.obj
 0001:00042050       ?ClipWindingEpsilon@@YAXPAUwinding_t@@ABVVector@@MMPAPAU1@2@Z 00443050 f   polylib.obj
 0001:00042650       ?ClassifyWindingEpsilon@@YAXPAUwinding_t@@ABVVector@@MMPAPAU1@22@Z 00443650 f   polylib.obj
 0001:00042a30       ?ChopWindingInPlace@@YAXPAPAUwinding_t@@ABVVector@@MM@Z 00443a30 f   polylib.obj
 0001:00042d40       ?WindingOnPlaneSide@@YAHPAUwinding_t@@ABVVector@@M@Z 00443d40 f   polylib.obj
 0001:00042df0       ?TranslateWinding@@YAXPAUwinding_t@@ABVVector@@@Z 00443df0 f   polylib.obj
 0001:00042e30       ?ClipWindingEpsilon_Offset@@YAXPAUwinding_t@@ABVVector@@MMPAPAU1@21@Z 00443e30 f   polylib.obj
 0001:00042f20       ?ClassifyWindingEpsilon_Offset@@YAXPAUwinding_t@@ABVVector@@MMPAPAU1@221@Z 00443f20 f   polylib.obj
 0001:00043050       ?DefaultScriptLoadedCallback@@YAXPBD0H@Z 00444050 f   scriplib.obj
 0001:00043060       ?DoesFileExist@CScriptLib@@UAE_NPBD@Z 00444060 f   scriplib.obj
 0001:00043080       ?ReadFileToBuffer@CScriptLib@@UAE_NPBDAAVCUtlBuffer@@_N2@Z 00444080 f   scriplib.obj
 0001:00043100       ?WriteBufferToFile@CScriptLib@@UAE_NPBDAAVCUtlBuffer@@W4DiskWriteMode_t@@@Z 00444100 f   scriplib.obj
 0001:000431d0       ?CompareFileTime@CScriptLib@@UAEHPBD0@Z 004441d0 f   scriplib.obj
 0001:00043230       ?MakeTemporaryFilename@CScriptLib@@UAEPADPBDPADH@Z 00444230 f   scriplib.obj
 0001:000432b0       ?InsertBefore@?$CUtlVector@VCUtlString@@V?$CUtlMemory@VCUtlString@@H@@@@QAEHH@Z 004442b0 f i scriplib.obj
 0001:00043320       ?InsertBefore@?$CUtlVector@UfileList_t@@V?$CUtlMemory@UfileList_t@@H@@@@QAEHH@Z 00444320 f i scriplib.obj
 0001:00043390       ?InsertMultipleBefore@?$CUtlVector@UfileList_t@@V?$CUtlMemory@UfileList_t@@H@@@@QAEHHHPBUfileList_t@@@Z 00444390 f i scriplib.obj
 0001:00043480       ?RemoveAll@?$CUtlVector@UfileList_t@@V?$CUtlMemory@UfileList_t@@H@@@@QAEXXZ 00444480 f i scriplib.obj
 0001:000434f0       ?GetFileList@CScriptLib@@AAEHPBD0AAV?$CUtlVector@UfileList_t@@V?$CUtlMemory@UfileList_t@@H@@@@@Z 004444f0 f   scriplib.obj
 0001:00043770       ??1?$CUtlVector@UfileList_t@@V?$CUtlMemory@UfileList_t@@H@@@@QAE@XZ 00444770 f i scriplib.obj
 0001:000437d0       ?DeleteTemporaryFiles@CScriptLib@@UAEXPBD@Z 004447d0 f   scriplib.obj
 0001:00043910       ?RecurseFileTree_r@CScriptLib@@AAEXPBDHAAV?$CUtlVector@VCUtlString@@V?$CUtlMemory@VCUtlString@@H@@@@@Z 00444910 f   scriplib.obj
 0001:00043a00       ?FindFiles@CScriptLib@@UAEHPAD_NAAV?$CUtlVector@UfileList_t@@V?$CUtlMemory@UfileList_t@@H@@@@@Z 00444a00 f   scriplib.obj
 0001:00043d10       ?SetLowPriority@@YAXXZ     00444d10 f   threads.obj
 0001:00043d20       ?ThreadSetDefault@@YAXXZ   00444d20 f   threads.obj
 0001:00043d70       ?ThreadLock@@YAXXZ         00444d70 f   threads.obj
 0001:00043db0       ?ThreadUnlock@@YAXXZ       00444db0 f   threads.obj
 0001:00043df0       ?InternalRunThreadsFn@@YGKPAX@Z 00444df0 f   threads.obj
 0001:00043e10       ?RunThreads_Start@@YAXP6AXHPAX@Z0W4ERunThreadsPriority@@@Z 00444e10 f   threads.obj
 0001:00043eb0       ?RunThreads_End@@YAXXZ     00444eb0 f   threads.obj
 0001:00043f10       ?RunThreadsOn@@YAXHHP6AXHPAX@Z0@Z 00444f10 f   threads.obj
 0001:00043f90       ?GetThreadWork@@YAHXZ      00444f90 f   threads.obj
 0001:00044070       ?ThreadWorkerFunction@@YAXHPAX@Z 00445070 f   threads.obj
 0001:000440a0       ?RunThreadsOnIndividual@@YAXHHP6AXHH@Z@Z 004450a0 f   threads.obj
 0001:00044110       ?EnableFullMinidumps@@YAX_N@Z 00445110 f   tools_minidump.obj
 0001:00044120       ?SetupDefaultToolsMinidumpHandler@@YAXXZ 00445120 f   tools_minidump.obj
 0001:00044130       ?V_strncmp@@YAHPBD0H@Z     00445130 f   tier1:strtools.obj
 0001:00044190       ?V_strncasecmp@@YAHPBD0H@Z 00445190 f   tier1:strtools.obj
 0001:00044210       ?V_strcasecmp@@YAHPBD0@Z   00445210 f   tier1:strtools.obj
 0001:00044240       ?V_strnicmp@@YAHPBD0H@Z    00445240 f   tier1:strtools.obj
 0001:00044280       ?V_stristr@@YAPBDPBD0@Z    00445280 f   tier1:strtools.obj
 0001:00044350       ?V_stristr@@YAPADPADPBD@Z  00445350 f   tier1:strtools.obj
 0001:00044380       ?V_strncat@@YAPADPADPBDIH@Z 00445380 f   tier1:strtools.obj
 0001:00044410       ?V_StripTrailingSlash@@YAXPAD@Z 00445410 f   tier1:strtools.obj
 0001:00044450       ?V_DefaultExtension@@YAXPADPBDH@Z 00445450 f   tier1:strtools.obj
 0001:00044500       ?V_StripFilename@@YAXPAD@Z 00445500 f   tier1:strtools.obj
 0001:00044540       ?V_FixSlashes@@YAXPADD@Z   00445540 f   tier1:strtools.obj
 0001:00044570       ?V_UnqualifiedFileName@@YAPBDPBD@Z 00445570 f   tier1:strtools.obj
 0001:000445b0       ?V_GetFileExtension@@YAPBDPBD@Z 004455b0 f   tier1:strtools.obj
 0001:00044600       ?V_RemoveDotSlashes@@YA_NPADD@Z 00445600 f   tier1:strtools.obj
 0001:00044760       ?V_AppendSlash@@YAXPADH@Z  00445760 f   tier1:strtools.obj
 0001:000447c0       ?V_IsAbsolutePath@@YA_NPBD@Z 004457c0 f   tier1:strtools.obj
 0001:000447e0       ?V_StrSlice@@YAXPBDHHPADH@Z 004457e0 f   tier1:strtools.obj
 0001:000448a0       ?V_strncpy@@YAXPADPBDH@Z   004458a0 f   tier1:strtools.obj
 0001:000448e0       ?V_snprintf@@YAHPADHPBDZZ  004458e0 f   tier1:strtools.obj
 0001:00044930       ?V_vsnprintf@@YAHPADHPBD0@Z 00445930 f   tier1:strtools.obj
 0001:00044980       ?V_FileBase@@YAXPBDPADH@Z  00445980 f   tier1:strtools.obj
 0001:00044a40       ?V_StripExtension@@YAXPBDPADH@Z 00445a40 f   tier1:strtools.obj
 0001:00044af0       ?V_StripLastDir@@YA_NPADH@Z 00445af0 f   tier1:strtools.obj
 0001:00044b90       ?V_ComposeFileName@@YAXPBD0PADH@Z 00445b90 f   tier1:strtools.obj
 0001:00044c50       ?V_ExtractFileExtension@@YAXPBDPADH@Z 00445c50 f   tier1:strtools.obj
 0001:00044ca0       ?V_MakeAbsolutePath@@YAXPADHPBD1@Z 00445ca0 f   tier1:strtools.obj
 0001:00044dc0       ?V_StrRight@@YAXPBDHPADH@Z 00445dc0 f   tier1:strtools.obj
 0001:00044e50       ?GetCStringCharConversion@@YAPAVCUtlCharConversion@@XZ 00445e50 f   tier1:utlbuffer.obj
 0001:00044e60       ?GetNoEscCharConversion@@YAPAVCUtlCharConversion@@XZ 00445e60 f   tier1:utlbuffer.obj
 0001:00044e70       ?FindConversion@CUtlCStringConversion@@UAEDPBDPAH@Z 00445e70 f   tier1:utlbuffer.obj
 0001:00044e90       ??0CUtlCharConversion@@QAE@DPBDHPAUConversionArray_t@0@@Z 00445e90 f   tier1:utlbuffer.obj
 0001:00044f40       ?FindConversion@CUtlCharConversion@@UAEDPBDPAH@Z 00445f40 f   tier1:utlbuffer.obj
 0001:00044fc0       ?SetBufferType@CUtlBuffer@@QAEX_N0@Z 00445fc0 f   tier1:utlbuffer.obj
 0001:00044ff0       ?GetOverflow@CUtlBuffer@@IAE_NH@Z 00445ff0 f   tier1:utlbuffer.obj
 0001:00045000       ?ActivateByteSwapping@CUtlBuffer@@QAEX_N@Z 00446000 f   tier1:utlbuffer.obj
 0001:00045030       ?FindConversion@CUtlNoEscConversion@@UAEDPBDPAH@Z 00446030 f i tier1:utlbuffer.obj
 0001:00045040       ?CheckGet@CUtlBuffer@@IAE_NH@Z 00446040 f   tier1:utlbuffer.obj
 0001:000450a0       ?CheckArbitraryPeekGet@CUtlBuffer@@IAE_NHAAH@Z 004460a0 f   tier1:utlbuffer.obj
 0001:00045110       ?PeekGet@CUtlBuffer@@QAEPBXHH@Z 00446110 f   tier1:utlbuffer.obj
 0001:00045150       ?SeekGet@CUtlBuffer@@QAEXW4SeekType_t@1@H@Z 00446150 f   tier1:utlbuffer.obj
 0001:000451b0       ?CheckPut@CUtlBuffer@@IAE_NH@Z 004461b0 f   tier1:utlbuffer.obj
 0001:00045200       ?AddNullTermination@CUtlBuffer@@IAEXXZ 00446200 f   tier1:utlbuffer.obj
 0001:00045250       ?ConvertToGrowableMemory@?$CUtlMemory@EH@@QAEXH@Z 00446250 f i tier1:utlbuffer.obj
 0001:000452a0       ?EnsureCapacity@CUtlBuffer@@QAEXH@Z 004462a0 f   tier1:utlbuffer.obj
 0001:00045300       ?Get@CUtlBuffer@@QAEXPAXH@Z 00446300 f   tier1:utlbuffer.obj
 0001:00045340       ?EatWhiteSpace@CUtlBuffer@@QAEXXZ 00446340 f   tier1:utlbuffer.obj
 0001:000453b0       ?PeekWhiteSpace@CUtlBuffer@@IAEHH@Z 004463b0 f   tier1:utlbuffer.obj
 0001:00045450       ?PeekStringLength@CUtlBuffer@@QAEHXZ 00446450 f   tier1:utlbuffer.obj
 0001:000455b0       ?PeekStringMatch@CUtlBuffer@@IAE_NHPBDH@Z 004465b0 f   tier1:utlbuffer.obj
 0001:00045610       ?Put@CUtlBuffer@@QAEXPBXH@Z 00446610 f   tier1:utlbuffer.obj
 0001:00045680       ?PutOverflow@CUtlBuffer@@IAE_NH@Z 00446680 f   tier1:utlbuffer.obj
 0001:000456d0       ?SeekPut@CUtlBuffer@@QAEXW4SeekType_t@1@H@Z 004466d0 f   tier1:utlbuffer.obj
 0001:00045750       ??0CUtlBuffer@@QAE@HHH@Z   00446750 f   tier1:utlbuffer.obj
 0001:000457d0       ??0CUtlBuffer@@QAE@PBXHH@Z 004467d0 f   tier1:utlbuffer.obj
 0001:00045850       ?PutString@CUtlBuffer@@QAEXPBD@Z 00446850 f   tier1:utlbuffer.obj
 0001:00045950       ?Printf@CUtlBuffer@@QAAXPBDZZ 00446950 f   tier1:utlbuffer.obj
 0001:00045990       ?GetChar@CUtlBuffer@@QAEDXZ 00446990 f i tier1:utlbuffer.obj
 0001:000459e0       ?EatCPPComment@CUtlBuffer@@QAE_NXZ 004469e0 f   tier1:utlbuffer.obj
 0001:00045a50       ?GetString@CUtlBuffer@@QAEXPADH@Z 00446a50 f   tier1:utlbuffer.obj
 0001:00045b10       ?GetDelimitedCharInternal@CUtlBuffer@@IAEDPAVCUtlCharConversion@@@Z 00446b10 f   tier1:utlbuffer.obj
 0001:00045ba0       ?GetDelimitedString@CUtlBuffer@@QAEXPAVCUtlCharConversion@@PADH@Z 00446ba0 f   tier1:utlbuffer.obj
 0001:00045cd0       ?VaScanf@CUtlBuffer@@QAEHPBDPAD@Z 00446cd0 f   tier1:utlbuffer.obj
 0001:00045ff0       ?Scanf@CUtlBuffer@@QAAHPBDZZ 00446ff0 f   tier1:utlbuffer.obj
 0001:00046010       ?NewNode@?$CUtlRBTree@VCStringPoolIndex@CUtlSymbolTable@@GVCLess@2@V?$CUtlMemory@U?$UtlRBTreeNode_t@VCStringPoolIndex@CUtlSymbolTable@@G@@G@@@@QAEGXZ 00447010 f i tier1:utlsymbol.obj
 0001:00046100       ?Links@?$CUtlRBTree@VCStringPoolIndex@CUtlSymbolTable@@GVCLess@2@V?$CUtlMemory@U?$UtlRBTreeNode_t@VCStringPoolIndex@CUtlSymbolTable@@G@@G@@@@IBEABU?$UtlRBTreeLinks_t@G@@G@Z 00447100 f i tier1:utlsymbol.obj
 0001:00046160       ??RCLess@CUtlSymbolTable@@QBE_NABVCStringPoolIndex@1@0@Z 00447160 f   tier1:utlsymbol.obj
 0001:00046220       ?FindPoolWithSpace@CUtlSymbolTable@@ABEHH@Z 00447220 f   tier1:utlsymbol.obj
 0001:00046260       ?FindInsertionPosition@?$CUtlRBTree@VCStringPoolIndex@CUtlSymbolTable@@GVCLess@2@V?$CUtlMemory@U?$UtlRBTreeNode_t@VCStringPoolIndex@CUtlSymbolTable@@G@@G@@@@IAEXABVCStringPoolIndex@CUtlSymbolTable@@AAGAA_N@Z 00447260 f i tier1:utlsymbol.obj
 0001:00046370       ?RotateLeft@?$CUtlRBTree@VCStringPoolIndex@CUtlSymbolTable@@GVCLess@2@V?$CUtlMemory@U?$UtlRBTreeNode_t@VCStringPoolIndex@CUtlSymbolTable@@G@@G@@@@IAEXG@Z 00447370 f i tier1:utlsymbol.obj
 0001:00046470       ?RotateRight@?$CUtlRBTree@VCStringPoolIndex@CUtlSymbolTable@@GVCLess@2@V?$CUtlMemory@U?$UtlRBTreeNode_t@VCStringPoolIndex@CUtlSymbolTable@@G@@G@@@@IAEXG@Z 00447470 f i tier1:utlsymbol.obj
 0001:00046570       ?String@CUtlSymbolTable@@QBEPBDVCUtlSymbol@@@Z 00447570 f   tier1:utlsymbol.obj
 0001:000465b0       ??0?$CUtlRBTree@VCStringPoolIndex@CUtlSymbolTable@@GVCLess@2@V?$CUtlMemory@U?$UtlRBTreeNode_t@VCStringPoolIndex@CUtlSymbolTable@@G@@G@@@@QAE@HHABVCLess@CUtlSymbolTable@@@Z 004475b0 f i tier1:utlsymbol.obj
 0001:00046610       ?Find@?$CUtlRBTree@VCStringPoolIndex@CUtlSymbolTable@@GVCLess@2@V?$CUtlMemory@U?$UtlRBTreeNode_t@VCStringPoolIndex@CUtlSymbolTable@@G@@G@@@@QBEGABVCStringPoolIndex@CUtlSymbolTable@@@Z 00447610 f i tier1:utlsymbol.obj
 0001:00046720       ?RemoveAll@?$CUtlRBTree@VCStringPoolIndex@CUtlSymbolTable@@GVCLess@2@V?$CUtlMemory@U?$UtlRBTreeNode_t@VCStringPoolIndex@CUtlSymbolTable@@G@@G@@@@QAEXXZ 00447720 f i tier1:utlsymbol.obj
 0001:000467e0       ?InsertRebalance@?$CUtlRBTree@VCStringPoolIndex@CUtlSymbolTable@@GVCLess@2@V?$CUtlMemory@U?$UtlRBTreeNode_t@VCStringPoolIndex@CUtlSymbolTable@@G@@G@@@@IAEXG@Z 004477e0 f i tier1:utlsymbol.obj
 0001:00046d50       ?String@CUtlSymbolTableMT@@QBEPBDVCUtlSymbol@@@Z 00447d50 f i tier1:utlsymbol.obj
 0001:00046db0       ?LinkToParent@?$CUtlRBTree@VCStringPoolIndex@CUtlSymbolTable@@GVCLess@2@V?$CUtlMemory@U?$UtlRBTreeNode_t@VCStringPoolIndex@CUtlSymbolTable@@G@@G@@@@IAEXGG_N@Z 00447db0 f i tier1:utlsymbol.obj
 0001:00046e20       ?RemoveAll@CUtlSymbolTable@@QAEXXZ 00447e20 f   tier1:utlsymbol.obj
 0001:00046ea0       ??1?$CUtlRBTree@VCStringPoolIndex@CUtlSymbolTable@@GVCLess@2@V?$CUtlMemory@U?$UtlRBTreeNode_t@VCStringPoolIndex@CUtlSymbolTable@@G@@G@@@@QAE@XZ 00447ea0 f i tier1:utlsymbol.obj
 0001:00046f00       ??1CUtlSymbolTable@@QAE@XZ 00447f00 f   tier1:utlsymbol.obj
 0001:00046f20       ?Insert@?$CUtlRBTree@VCStringPoolIndex@CUtlSymbolTable@@GVCLess@2@V?$CUtlMemory@U?$UtlRBTreeNode_t@VCStringPoolIndex@CUtlSymbolTable@@G@@G@@@@QAEGABVCStringPoolIndex@CUtlSymbolTable@@@Z 00447f20 f i tier1:utlsymbol.obj
 0001:00046f80       ??0CUtlSymbolTable@@QAE@HH_N@Z 00447f80 f   tier1:utlsymbol.obj
 0001:00046fc0       ?AddString@CUtlSymbolTable@@QAE?AVCUtlSymbol@@PBD@Z 00447fc0 f   tier1:utlsymbol.obj
 0001:000470c0       ?Initialize@CUtlSymbol@@KAXXZ 004480c0 f   tier1:utlsymbol.obj
 0001:00047160       ??0CUtlSymbol@@QAE@PBD@Z   00448160 f   tier1:utlsymbol.obj
 0001:000471b0       ?String@CUtlSymbol@@QBEPBDXZ 004481b0 f   tier1:utlsymbol.obj
 0001:000471d0       ?ReportError@CKeyValuesErrorStack@@QAEXPBD@Z 004481d0 f i tier1:KeyValues.obj
 0001:00047260       ?ChainKeyValue@KeyValues@@QAEXPAV1@@Z 00448260 f   tier1:KeyValues.obj
 0001:00047260       ?SetCenterVertIndex@CCoreDispNode@@QAEXH@Z 00448260 f   builddisp.obj
 0001:00047270       ?GetName@KeyValues@@QBEPBDXZ 00448270 f   tier1:KeyValues.obj
 0001:00047290       ?ReadToken@KeyValues@@AAEPBDAAVCUtlBuffer@@AA_N1@Z 00448290 f   tier1:KeyValues.obj
 0001:00047420       ?InternalWrite@KeyValues@@AAEXPAVIBaseFileSystem@@PAXPAVCUtlBuffer@@PBXH@Z 00448420 f   tier1:KeyValues.obj
 0001:00047460       ?RemoveSubKey@KeyValues@@QAEXPAV1@@Z 00448460 f   tier1:KeyValues.obj
 0001:000474b0       ?GetFirstSubKey@KeyValues@@QAEPAV1@XZ 004484b0 f   tier1:KeyValues.obj
 0001:000474b0       ?Format@CVTFTexture@@UBE?AW4ImageFormat@@XZ 004484b0 f   vtf:vtf.obj
 0001:000474c0       ?GetNextKey@KeyValues@@QAEPAV1@XZ 004484c0 f   tier1:KeyValues.obj
 0001:000474c0       ?Depth@CVTFTexture@@UBEHXZ 004484c0 f   vtf:vtf.obj
 0001:000474d0       ?GetFirstTrueSubKey@KeyValues@@QAEPAV1@XZ 004484d0 f   tier1:KeyValues.obj
 0001:000474f0       ?GetNextTrueSubKey@KeyValues@@QAEPAV1@XZ 004484f0 f   tier1:KeyValues.obj
 0001:00047510       ?GetFirstValue@KeyValues@@QAEPAV1@XZ 00448510 f   tier1:KeyValues.obj
 0001:00047530       ?GetNextValue@KeyValues@@QAEPAV1@XZ 00448530 f   tier1:KeyValues.obj
 0001:00047550       ?SetName@KeyValues@@QAEXPBD@Z 00448550 f   tier1:KeyValues.obj
 0001:00047570       ?CopySubkeys@KeyValues@@QBEXPAV1@@Z 00448570 f   tier1:KeyValues.obj
 0001:000475b0       ??2KeyValues@@SAPAXI@Z     004485b0 f   tier1:KeyValues.obj
 0001:000475d0       ??0KeyValues@@QAE@PBD@Z    004485d0 f   tier1:KeyValues.obj
 0001:00047620       ?LoadFromFile@KeyValues@@QAE_NPAVIBaseFileSystem@@PBD1@Z 00448620 f   tier1:KeyValues.obj
 0001:00047770       ?WriteIndents@KeyValues@@AAEXPAVIBaseFileSystem@@PAXPAVCUtlBuffer@@H@Z 00448770 f   tier1:KeyValues.obj
 0001:000477d0       ?WriteConvertedString@KeyValues@@AAEXPAVIBaseFileSystem@@PAXPAVCUtlBuffer@@PBD@Z 004487d0 f   tier1:KeyValues.obj
 0001:00047870       ?RecursiveSaveToFile@KeyValues@@AAEXPAVIBaseFileSystem@@PAXPAVCUtlBuffer@@H@Z 00448870 f   tier1:KeyValues.obj
 0001:00047f20       ?FindKey@KeyValues@@QAEPAV1@PBD_N@Z 00448f20 f   tier1:KeyValues.obj
 0001:00048060       ?GetInt@KeyValues@@QAEHPBDH@Z 00449060 f   tier1:KeyValues.obj
 0001:000480e0       ?GetPtr@KeyValues@@QAEPAXPBDPAX@Z 004490e0 f   tier1:KeyValues.obj
 0001:00048110       ?GetFloat@KeyValues@@QAEMPBDM@Z 00449110 f   tier1:KeyValues.obj
 0001:000481e0       ?SetString@KeyValues@@QAEXPBD0@Z 004491e0 f   tier1:KeyValues.obj
 0001:00048250       ?SetInt@KeyValues@@QAEXPBDH@Z 00449250 f   tier1:KeyValues.obj
 0001:00048270       ?SetFloat@KeyValues@@QAEXPBDM@Z 00449270 f   tier1:KeyValues.obj
 0001:00048290       ?SetPtr@KeyValues@@QAEXPBDPAX@Z 00449290 f   tier1:KeyValues.obj
 0001:000482b0       ?RecursiveCopyKeyValues@KeyValues@@AAEXAAV1@@Z 004492b0 f   tier1:KeyValues.obj
 0001:000484c0       ?MakeCopy@KeyValues@@QBEPAV1@XZ 004494c0 f   tier1:KeyValues.obj
 0001:000486b0       ?GetDataType@KeyValues@@QAE?AW4types_t@1@PBD@Z 004496b0 f   tier1:KeyValues.obj
 0001:000486d0       ?deleteThis@KeyValues@@QAEXXZ 004496d0 f   tier1:KeyValues.obj
 0001:000486f0       ?RecursiveMergeKeyValues@KeyValues@@AAEXPAV1@@Z 004496f0 f   tier1:KeyValues.obj
 0001:000487c0       ??$SwapBufferToTargetEndian@I@CByteswap@@QAEXPAI0H@Z 004497c0 f i tier1:KeyValues.obj
 0001:000487c0       ??$SwapBufferToTargetEndian@H@CByteswap@@QAEXPAH0H@Z 004497c0 f i detailobjects.obj
 0001:00048850       ?RemoveEverything@KeyValues@@AAEXXZ 00449850 f   tier1:KeyValues.obj
 0001:000488e0       ?RecursiveSaveToFile@KeyValues@@QAEXAAVCUtlBuffer@@H@Z 004498e0 f   tier1:KeyValues.obj
 0001:00048900       ?CreateKey@KeyValues@@AAEPAV1@PBD@Z 00449900 f   tier1:KeyValues.obj
 0001:000489a0       ?GetString@KeyValues@@QAEPBDPBD0@Z 004499a0 f   tier1:KeyValues.obj
 0001:00048b00       ??4KeyValues@@QAEAAV0@AAV0@@Z 00449b00 f   tier1:KeyValues.obj
 0001:00048b40       ?AppendIncludedKeys@KeyValues@@AAEXAAV?$CUtlVector@PAVKeyValues@@V?$CUtlMemory@PAVKeyValues@@H@@@@@Z 00449b40 f   tier1:KeyValues.obj
 0001:00048b90       ?RecursiveLoadFromBuffer@KeyValues@@AAEXPBDAAVCUtlBuffer@@@Z 00449b90 f   tier1:KeyValues.obj
 0001:00048f00       ?ParseIncludedKeys@KeyValues@@AAEXPBD0PAVIBaseFileSystem@@0AAV?$CUtlVector@PAVKeyValues@@V?$CUtlMemory@PAVKeyValues@@H@@@@@Z 00449f00 f   tier1:KeyValues.obj
 0001:00049030       ?LoadFromBuffer@KeyValues@@QAE_NPBDAAVCUtlBuffer@@PAVIBaseFileSystem@@0@Z 0044a030 f   tier1:KeyValues.obj
 0001:000493b0       ?LoadFromBuffer@KeyValues@@QAE_NPBD0PAVIBaseFileSystem@@0@Z 0044a3b0 f   tier1:KeyValues.obj
 0001:00049430       ??$SwapBufferToTargetEndian@D@CByteswap@@QAEXPAD0H@Z 0044a430 f i zip_utils.obj
 0001:00049430       ??$SwapBufferToTargetEndian@_N@CByteswap@@QAEXPA_N0H@Z 0044a430 f i tier1:byteswap.obj
 0001:00049460       ?SwapFieldToTargetEndian@CByteswap@@QAEXPAX0PAUtypedescription_t@@@Z 0044a460 f   tier1:byteswap.obj
 0001:000495b0       ?SwapFieldsToTargetEndian@CByteswap@@QAEXPAX0PAUdatamap_t@@@Z 0044a5b0 f   tier1:byteswap.obj
 0001:00049610       _CreateInterface           0044a610 f   tier1:interface.obj
 0001:00049680       ?ThreadedLoadLibraryFunc@@YAIPAX@Z 0044a680 f   tier1:interface.obj
 0001:000496a0       ?Sys_LoadLibrary@@YAPAUHINSTANCE__@@PBD@Z 0044a6a0 f   tier1:interface.obj
 0001:000497a0       ?Sys_LoadModule@@YAPAVCSysModule@@PBD@Z 0044a7a0 f   tier1:interface.obj
 0001:000498f0       ?Sys_UnloadModule@@YAXPAVCSysModule@@@Z 0044a8f0 f   tier1:interface.obj
 0001:00049900       ?Sys_GetFactory@@YAP6APAXPBDPAH@ZPAVCSysModule@@@Z 0044a900 f   tier1:interface.obj
 0001:00049920       ?Sys_GetFactoryThis@@YAP6APAXPBDPAH@ZXZ 0044a920 f   tier1:interface.obj
 0001:00049930       ?Sys_LoadInterface@@YA_NPBD0PAPAVCSysModule@@PAPAX@Z 0044a930 f   tier1:interface.obj
 0001:00049990       ?Length@CUtlString@@QBEHXZ 0044a990 f   tier1:utlstring.obj
 0001:000499a0       ?Get@CUtlString@@QBEPBDXZ  0044a9a0 f   tier1:utlstring.obj
 0001:000499b0       ?Set@CUtlBinaryBlock@@QAEXPBXH@Z 0044a9b0 f   tier1:utlstring.obj
 0001:00049a20       ?Set@CUtlString@@QAEXPBD@Z 0044aa20 f   tier1:utlstring.obj
 0001:00049a60       ??4CUtlString@@QAEAAV0@ABV0@@Z 0044aa60 f   tier1:utlstring.obj
 0001:00049a80       ??4CUtlString@@QAEAAV0@PBD@Z 0044aa80 f   tier1:utlstring.obj
 0001:00049ad0       ??0CUtlString@@QAE@XZ      0044aad0 f   tier1:utlstring.obj
 0001:00049ae0       ?CRC32_Init@@YAXPAK@Z      0044aae0 f   tier1:checksum_crc.obj
 0001:00049af0       ?CRC32_Final@@YAXPAK@Z     0044aaf0 f   tier1:checksum_crc.obj
 0001:00049b00       ?CRC32_ProcessBuffer@@YAXPAKPBXH@Z 0044ab00 f   tier1:checksum_crc.obj
 0001:00049ce0       ?getloc@ios_base@std@@QBE?AVlocale@2@XZ 0044ace0 f i tier1:tokenreader.obj
 0001:00049d20       ?Error@TokenReader@@QAAPBDPADZZ 0044ad20 f   tier1:tokenreader.obj
 0001:00049d70       ?sgetc@?$basic_streambuf@DU?$char_traits@D@std@@@std@@QAEHXZ 0044ad70 f i tier1:tokenreader.obj
 0001:00049d90       ?sbumpc@?$basic_streambuf@DU?$char_traits@D@std@@@std@@QAEHXZ 0044ad90 f i tier1:tokenreader.obj
 0001:00049dc0       ?sputbackc@?$basic_streambuf@DU?$char_traits@D@std@@@std@@QAEHD@Z 0044adc0 f i tier1:tokenreader.obj
 0001:00049e00       ?snextc@?$basic_streambuf@DU?$char_traits@D@std@@@std@@QAEHXZ 0044ae00 f i tier1:tokenreader.obj
 0001:00049e80       ??0?$basic_streambuf@DU?$char_traits@D@std@@@std@@IAE@XZ 0044ae80 f i tier1:tokenreader.obj
 0001:00049f00       ??0failure@ios_base@std@@QAE@ABV?$basic_string@DU?$char_traits@D@std@@V?$allocator@D@2@@2@@Z 0044af00 f i tier1:tokenreader.obj
 0001:00049f40       ??1runtime_error@std@@UAE@XZ 0044af40 f i chunkfile.obj
 0001:00049f40       ??1failure@ios_base@std@@UAE@XZ 0044af40 f i tier1:tokenreader.obj
 0001:00049f80       ?do_tolower@?$ctype@D@std@@MBEDD@Z 0044af80 f i tier1:tokenreader.obj
 0001:00049fa0       ?do_tolower@?$ctype@D@std@@MBEPBDPADPBD@Z 0044afa0 f i tier1:tokenreader.obj
 0001:00049fd0       ?do_toupper@?$ctype@D@std@@MBEDD@Z 0044afd0 f i tier1:tokenreader.obj
 0001:00049ff0       ?do_toupper@?$ctype@D@std@@MBEPBDPADPBD@Z 0044aff0 f i tier1:tokenreader.obj
 0001:0004a020       ?do_widen@?$ctype@D@std@@MBEDD@Z 0044b020 f i tier1:tokenreader.obj
 0001:0004a030       ?do_widen@?$ctype@D@std@@MBEPBDPBD0PAD@Z 0044b030 f i tier1:tokenreader.obj
 0001:0004a060       ?_Do_widen_s@?$ctype@D@std@@MBEPBDPBD0PADI@Z 0044b060 f i tier1:tokenreader.obj
 0001:0004a0a0       ?do_narrow@?$ctype@D@std@@MBEDDD@Z 0044b0a0 f i tier1:tokenreader.obj
 0001:0004a0b0       ?do_narrow@?$ctype@D@std@@MBEPBDPBD0DPAD@Z 0044b0b0 f i tier1:tokenreader.obj
 0001:0004a0e0       ?_Do_narrow_s@?$ctype@D@std@@MBEPBDPBD0DPADI@Z 0044b0e0 f i tier1:tokenreader.obj
 0001:0004a120       ??_G?$ctype@D@std@@MAEPAXI@Z 0044b120 f i tier1:tokenreader.obj
 0001:0004a120       ??_E?$ctype@D@std@@MAEPAXI@Z 0044b120 f i tier1:tokenreader.obj
 0001:0004a170       ?_Getcat@?$ctype@D@std@@SAIPAPBVfacet@locale@2@@Z 0044b170 f i tier1:tokenreader.obj
 0001:0004a210       ?clear@ios_base@std@@QAEXH_N@Z 0044b210 f i tier1:tokenreader.obj
 0001:0004a2d0       ??0failure@ios_base@std@@QAE@ABV012@@Z 0044b2d0 f i tier1:tokenreader.obj
 0001:0004a310       ?_Init@ios_base@std@@IAEXXZ 0044b310 f i tier1:tokenreader.obj
 0001:0004a390       ?setstate@?$basic_ios@DU?$char_traits@D@std@@@std@@QAEXH_N@Z 0044b390 f i tier1:tokenreader.obj
 0001:0004a3c0       ??$use_facet@V?$ctype@D@std@@@std@@YAABV?$ctype@D@0@ABVlocale@0@@Z 0044b3c0 f i tier1:tokenreader.obj
 0001:0004a4c0       ?flush@?$basic_ostream@DU?$char_traits@D@std@@@std@@QAEAAV12@XZ 0044b4c0 f i tier1:tokenreader.obj
 0001:0004a510       ?_Ipfx@?$basic_istream@DU?$char_traits@D@std@@@std@@QAE_N_N@Z 0044b510 f i tier1:tokenreader.obj
 0001:0004a670       ?widen@?$basic_ios@DU?$char_traits@D@std@@@std@@QBEDD@Z 0044b670 f i tier1:tokenreader.obj
 0001:0004a710       ?get@?$basic_istream@DU?$char_traits@D@std@@@std@@QAEHXZ 0044b710 f i tier1:tokenreader.obj
 0001:0004a830       ?get@?$basic_istream@DU?$char_traits@D@std@@@std@@QAEAAV12@PADHD@Z 0044b830 f i tier1:tokenreader.obj
 0001:0004a990       ?ignore@?$basic_istream@DU?$char_traits@D@std@@@std@@QAEAAV12@HH@Z 0044b990 f i tier1:tokenreader.obj
 0001:0004aac0       ?peek@?$basic_istream@DU?$char_traits@D@std@@@std@@QAEHXZ 0044bac0 f i tier1:tokenreader.obj
 0001:0004abe0       ?putback@?$basic_istream@DU?$char_traits@D@std@@@std@@QAEAAV12@D@Z 0044bbe0 f i tier1:tokenreader.obj
 0001:0004acf0       ?open@?$basic_filebuf@DU?$char_traits@D@std@@@std@@QAEPAV12@PBDHH@Z 0044bcf0 f i tier1:tokenreader.obj
 0001:0004ade0       ?SkipWhiteSpace@TokenReader@@AAE_NXZ 0044bde0 f   tier1:tokenreader.obj
 0001:0004ae70       ??0?$basic_ifstream@DU?$char_traits@D@std@@@std@@QAE@XZ 0044be70 f i tier1:tokenreader.obj
 0001:0004af20       ??0TokenReader@@QAE@XZ     0044bf20 f   tier1:tokenreader.obj
 0001:0004af70       ??_GTokenReader@@UAEPAXI@Z 0044bf70 f i tier1:tokenreader.obj
 0001:0004af70       ??_ETokenReader@@UAEPAXI@Z 0044bf70 f i tier1:tokenreader.obj
 0001:0004afa0       ?Open@TokenReader@@QAE_NPBD@Z 0044bfa0 f   tier1:tokenreader.obj
 0001:0004b010       ?GetString@TokenReader@@AAE?AW4trtoken_t@@PADH@Z 0044c010 f   tier1:tokenreader.obj
 0001:0004b160       ?NextToken@TokenReader@@QAE?AW4trtoken_t@@PADH@Z 0044c160 f   tier1:tokenreader.obj
 0001:0004b390       ?SinCos@@YAXMPAM0@Z        0044c390 f i mathlib:mathlib_base.obj
 0001:0004b3b0       ?_sqrtf@@YAMM@Z            0044c3b0 f   mathlib:mathlib_base.obj
 0001:0004b3c0       ?_rsqrtf@@YAMM@Z           0044c3c0 f   mathlib:mathlib_base.obj
 0001:0004b3d0       ?_VectorNormalize@@YIMAAVVector@@@Z 0044c3d0 f   mathlib:mathlib_base.obj
 0001:0004b410       ?_VectorNormalizeFast@@YIXAAVVector@@@Z 0044c410 f   mathlib:mathlib_base.obj
 0001:0004b450       ?_InvRSquared@@YAMPBM@Z    0044c450 f   mathlib:mathlib_base.obj
 0001:0004b480       ?InitSinCosTable@@YAXXZ    0044c480 f   mathlib:mathlib_base.obj
 0001:0004b4b0       ?AngleVectors@@YAXABVQAngle@@PAVVector@@11@Z 0044c4b0 f   mathlib:mathlib_base.obj
 0001:0004b600       ?VectorAngles@@YAXABVVector@@AAVQAngle@@@Z 0044c600 f   mathlib:mathlib_base.obj
 0001:0004b6e0       ?ClearBounds@@YAXAAVVector@@0@Z 0044c6e0 f   mathlib:mathlib_base.obj
 0001:0004b710       ?AddPointToBounds@@YAXABVVector@@AAV1@1@Z 0044c710 f   mathlib:mathlib_base.obj
 0001:0004b780       ?MathLib_Init@@YAXMMMH_N000@Z 0044c780 f   mathlib:mathlib_base.obj
 0001:0004b920       ??4VMatrix@@QAEAAV0@ABV0@@Z 0044c920 f   mathlib:vmatrix.obj
 0001:0004b990       ?MatrixMul@VMatrix@@QBEXABV1@AAV1@@Z 0044c990 f   mathlib:vmatrix.obj
 0001:0004bc00       ??DVMatrix@@QBE?AV0@ABV0@@Z 0044cc00 f   mathlib:vmatrix.obj
 0001:0004bc20       ?MatrixSetIdentity@@YAXAAVVMatrix@@@Z 0044cc20 f   mathlib:vmatrix.obj
 0001:0004bc60       ?MatrixToAngles@@YAXABVVMatrix@@AAVQAngle@@@Z 0044cc60 f   mathlib:vmatrix.obj
 0001:0004bd10       ?SetupMatrixAxisRot@@YA?AVVMatrix@@ABVVector@@M@Z 0044cd10 f   mathlib:vmatrix.obj
 0001:0004bdd0       ?Transpose@VMatrix@@QBE?AV1@XZ 0044cdd0 f   mathlib:vmatrix.obj
 0001:0004be40       ?TextureToLinear@@YAMH@Z   0044ce40 f   mathlib:color_conversion.obj
 0001:0004be60       ?BuildGammaTable@@YAXMMMH@Z 0044ce60 f   mathlib:color_conversion.obj
 0001:0004c120       ?_SSE_Sqrt@@YAMM@Z         0044d120 f   mathlib:sse.obj
 0001:0004c140       ?_SSE_RSqrtAccurate@@YAMM@Z 0044d140 f   mathlib:sse.obj
 0001:0004c190       ?_SSE_RSqrtFast@@YAMM@Z    0044d190 f   mathlib:sse.obj
 0001:0004c1b0       ?_SSE_VectorNormalizeFast@@YIXAAVVector@@@Z 0044d1b0 f   mathlib:sse.obj
 0001:0004c240       ?_SSE_InvRSquared@@YAMPBM@Z 0044d240 f   mathlib:sse.obj
 0001:0004c280       ?_SSE_SinCos@@YAXMPAM0@Z   0044d280 f   mathlib:sse.obj
 0001:0004c3c0       ?_SSE_cos@@YAMM@Z          0044d3c0 f   mathlib:sse.obj
 0001:0004c490       ?_SSE2_SinCos@@YAXMPAM0@Z  0044d490 f   mathlib:sse.obj
 0001:0004c5b0       ?_SSE2_cos@@YAMM@Z         0044d5b0 f   mathlib:sse.obj
 0001:0004c680       ?_3DNow_Sqrt@@YAMM@Z       0044d680 f   mathlib:3dnow.obj
 0001:0004c6b0       ?_3DNow_RSqrt@@YAMM@Z      0044d6b0 f   mathlib:3dnow.obj
 0001:0004c6d0       ?_3DNow_VectorNormalize@@YIMAAVVector@@@Z 0044d6d0 f   mathlib:3dnow.obj
 0001:0004c750       ?_3DNow_VectorNormalizeFast@@YIXAAVVector@@@Z 0044d750 f   mathlib:3dnow.obj
 0001:0004c760       ?_3DNow_InvRSquared@@YAMPBM@Z 0044d760 f   mathlib:3dnow.obj
 0001:0004c7a0       ?SizeInBytes@ImageLoader@@YAHW4ImageFormat@@@Z 0044d7a0 f i vtf:vtf.obj
 0001:0004c7c0       ?DestroyVTFTexture@@YAXPAVIVTFTexture@@@Z 0044d7c0 f   vtf:vtf.obj
 0001:0004c7e0       ?ComputeMipCount@CVTFTexture@@ABEHXZ 0044d7e0 f   vtf:vtf.obj
 0001:0004c800       ?AllocateImageData@CVTFTexture@@AAEXH@Z 0044d800 f   vtf:vtf.obj
 0001:0004c830       ?SetBumpScale@CVTFTexture@@UAEXM@Z 0044d830 f   vtf:vtf.obj
 0001:0004c840       ?SetReflectivity@CVTFTexture@@UAEXABVVector@@@Z 0044d840 f   vtf:vtf.obj
 0001:0004c860       ?SetAlphaTestThreshholds@CVTFTexture@@UAEXMM@Z 0044d860 f   vtf:vtf.obj
 0001:0004c880       ?LoadLowResData@CVTFTexture@@AAE_NAAVCUtlBuffer@@@Z 0044d880 f   vtf:vtf.obj
 0001:0004c8d0       ?LoadImageData@CVTFTexture@@AAE_NAAVCUtlBuffer@@ABUVTFFileHeader_t@@H@Z 0044d8d0 f   vtf:vtf.obj
 0001:0004ca10       ?WriteData@ResourceMemorySection@CVTFTexture@@QBE_NAAVCUtlBuffer@@@Z 0044da10 f   vtf:vtf.obj
 0001:0004cab0       ?WriteImageData@CVTFTexture@@AAE_NAAVCUtlBuffer@@@Z 0044dab0 f   vtf:vtf.obj
 0001:0004cb30       ?Width@CVTFTexture@@UBEHXZ 0044db30 f   vtf:vtf.obj
 0001:0004cb30       ?GetPower@CCoreDispInfo@@QBEHXZ 0044db30 f   disp_vbsp.obj
 0001:0004cb40       ?Height@CVTFTexture@@UBEHXZ 0044db40 f   vtf:vtf.obj
 0001:0004cb50       ?FaceCount@CVTFTexture@@UBEHXZ 0044db50 f   vtf:vtf.obj
 0001:0004cb60       ?FrameCount@CVTFTexture@@UBEHXZ 0044db60 f   vtf:vtf.obj
 0001:0004cb70       ?Flags@CVTFTexture@@UBEHXZ 0044db70 f   vtf:vtf.obj
 0001:0004cb80       ?IsCubeMap@CVTFTexture@@UBE_NXZ 0044db80 f   vtf:vtf.obj
 0001:0004cb90       ?IsNormalMap@CVTFTexture@@UBE_NXZ 0044db90 f   vtf:vtf.obj
 0001:0004cba0       ?IsVolumeTexture@CVTFTexture@@UBE_NXZ 0044dba0 f   vtf:vtf.obj
 0001:0004cbb0       ?BumpScale@CVTFTexture@@UBEMXZ 0044dbb0 f   vtf:vtf.obj
 0001:0004cbc0       ?Reflectivity@CVTFTexture@@UBEABVVector@@XZ 0044dbc0 f   vtf:vtf.obj
 0001:0004cbd0       ?ImageData@CVTFTexture@@UAEPAEXZ 0044dbd0 f   vtf:vtf.obj
 0001:0004cbe0       ?LowResWidth@CVTFTexture@@UBEHXZ 0044dbe0 f   vtf:vtf.obj
 0001:0004cbf0       ?LowResHeight@CVTFTexture@@UBEHXZ 0044dbf0 f   vtf:vtf.obj
 0001:0004cc00       ?LowResFormat@CVTFTexture@@UBE?AW4ImageFormat@@XZ 0044dc00 f   vtf:vtf.obj
 0001:0004cc10       ?LowResImageData@CVTFTexture@@UAEPAEXZ 0044dc10 f   vtf:vtf.obj
 0001:0004cc20       ?RowSizeInBytes@CVTFTexture@@UBEHH@Z 0044dc20 f   vtf:vtf.obj
 0001:0004cc50       ?FaceSizeInBytes@CVTFTexture@@UBEHH@Z 0044dc50 f   vtf:vtf.obj
 0001:0004cc90       ?ImageData@CVTFTexture@@UAEPAEHHHHHH@Z 0044dc90 f   vtf:vtf.obj
 0001:0004cd00       ?ComputeMipSize@CVTFTexture@@UBEHH@Z 0044dd00 f   vtf:vtf.obj
 0001:0004cd50       ?ComputeFaceSize@CVTFTexture@@ABEHHW4ImageFormat@@@Z 0044dd50 f i vtf:vtf.obj
 0001:0004cde0       ?ComputeFaceSize@CVTFTexture@@UBEHH@Z 0044dde0 f   vtf:vtf.obj
 0001:0004ce00       ?ComputeTotalSize@CVTFTexture@@UBEHXZ 0044de00 f   vtf:vtf.obj
 0001:0004ce20       ?GetImageOffset@CVTFTexture@@ABEHHHHW4ImageFormat@@@Z 0044de20 f   vtf:vtf.obj
 0001:0004cea0       ?ComputeMipLevelDimensions@CVTFTexture@@UBEXHPAH00@Z 0044dea0 f   vtf:vtf.obj
 0001:0004cef0       ?ComputeMipLevelSubRect@CVTFTexture@@UBEXPAURect_t@@H0@Z 0044def0 f   vtf:vtf.obj
 0001:0004cfb0       ?ConvertImageFormat@CVTFTexture@@UAEXW4ImageFormat@@_N@Z 0044dfb0 f   vtf:vtf.obj
 0001:0004d710       ?ComputeHemispheremapFrame@CVTFTexture@@AAEXPAPAEPAEW4LookDir_t@@@Z 0044e710 f   vtf:vtf.obj
 0001:0004d8e0       ?GenerateHemisphereMap@CVTFTexture@@UAEXPAEHHW4LookDir_t@@H@Z 0044e8e0 f   vtf:vtf.obj
 0001:0004d9e0       ?FixCubemapFaceOrientation@CVTFTexture@@UAEXXZ 0044e9e0 f   vtf:vtf.obj
 0001:0004dab0       ?NormalizeTopMipLevel@CVTFTexture@@UAEXXZ 0044eab0 f   vtf:vtf.obj
 0001:0004db40       ?PutOneOverMipLevelInAlpha@CVTFTexture@@UAEXXZ 0044eb40 f   vtf:vtf.obj
 0001:0004dc30       ?ComputeReflectivity@CVTFTexture@@UAEXXZ 0044ec30 f   vtf:vtf.obj
 0001:0004dd80       ?ComputeAlphaFlags@CVTFTexture@@UAEXXZ 0044ed80 f   vtf:vtf.obj
 0001:0004ded0       ?PostProcess@CVTFTexture@@UAEX_NW4LookDir_t@@0@Z 0044eed0 f   vtf:vtf.obj
 0001:0004df60       ?SetPostProcessingSettings@CVTFTexture@@UAEXPBUVtfProcessingOptions@@@Z 0044ef60 f   vtf:vtf.obj
 0001:0004dfb0       ?SetupFaceVert@CVTFTexture@@AAEXHHAAVCEdgePos@@@Z 0044efb0 f   vtf:vtf.obj
 0001:0004e010       ?SetupTextureEdgeIncrements@CVTFTexture@@AAEXHHH_NPAVCEdgeIncrements@@@Z 0044f010 f   vtf:vtf.obj
 0001:0004e130       ?BlendTexels@@YAXPAPAEH@Z  0044f130 f   vtf:vtf.obj
 0001:0004e1e0       ?BlendCubeMapFaceCorners@CVTFTexture@@AAEXHHPBVCCornerMatch@@@Z 0044f1e0 f   vtf:vtf.obj
 0001:0004e3c0       ?BuildCubeMapMatchLists@CVTFTexture@@AAEXQAVCEdgeMatch@@QAVCCornerMatch@@_N@Z 0044f3c0 f   vtf:vtf.obj
 0001:0004e640       ??9CEdgePos@@QAE_NABV0@@Z  0044f640 f i vtf:vtf.obj
 0001:0004e680       ?ImageData@CVTFTexture@@UAEPAEHHH@Z 0044f680 f   vtf:vtf.obj
 0001:0004e6b0       ?ComputeSpheremapFrame@CVTFTexture@@AAEXPAPAEPAEW4LookDir_t@@@Z 0044f6b0 f   vtf:vtf.obj
 0001:0004e880       ?GenerateSpheremap@CVTFTexture@@UAEXW4LookDir_t@@@Z 0044f880 f   vtf:vtf.obj
 0001:0004e960       ?GenerateMipmaps@CVTFTexture@@UAEXXZ 0044f960 f   vtf:vtf.obj
 0001:0004edb0       ?BlendCubeMapFaceEdges@CVTFTexture@@AAEXHHPBVCEdgeMatch@@@Z 0044fdb0 f   vtf:vtf.obj
 0001:0004ef80       ?ReleaseResources@CVTFTexture@@AAEXXZ 0044ff80 f   vtf:vtf.obj
 0001:0004f000       ?GetResourceTypes@CVTFTexture@@UBEIPAIH@Z 00450000 f   vtf:vtf.obj
 0001:0004f050       ?LoadData@ResourceMemorySection@CVTFTexture@@QAE_NAAVCUtlBuffer@@AAVCByteswap@@@Z 00450050 f   vtf:vtf.obj
 0001:0004f0f0       ?ReadHeader@CVTFTexture@@AAE_NAAVCUtlBuffer@@AAUVTFFileHeader_t@@@Z 004500f0 f   vtf:vtf.obj
 0001:0004f1d0       ?LoadNewResources@CVTFTexture@@AAE_NAAVCUtlBuffer@@@Z 004501d0 f   vtf:vtf.obj
 0001:0004f250       ?FindResourceEntryInfo@CVTFTexture@@ABEPBUResourceEntryInfo@@I@Z 00450250 f   vtf:vtf.obj
 0001:0004f2c0       ?BlendCubeMapEdgePalettes@CVTFTexture@@AAEXHHPBVCEdgeMatch@@@Z 004502c0 f   vtf:vtf.obj
 0001:0004f4e0       ?BlendCubeMapCornerPalettes@CVTFTexture@@AAEXHHPBVCCornerMatch@@@Z 004504e0 f   vtf:vtf.obj
 0001:0004f640       ?MatchCubeMapS3TCPalettes@CVTFTexture@@AAEXQAVCEdgeMatch@@QAVCCornerMatch@@@Z 00450640 f   vtf:vtf.obj
 0001:0004f6c0       ?EnsureCapacity@?$CUtlVector@UResourceMemorySection@CVTFTexture@@V?$CUtlMemory@UResourceMemorySection@CVTFTexture@@H@@@@QAEXH@Z 004506c0 f i vtf:vtf.obj
 0001:0004f720       ?InsertMultipleBefore@?$CUtlVector@UentitySideList_t@@V?$CUtlMemory@UentitySideList_t@@H@@@@QAEHHHPBUentitySideList_t@@@Z 00450720 f i worldvertextransitionfixup.obj
 0001:0004f720       ?InsertMultipleBefore@?$CUtlVector@UResourceEntryInfo@@V?$CUtlMemory@UResourceEntryInfo@@H@@@@QAEHHHPBUResourceEntryInfo@@@Z 00450720 f i vtf:vtf.obj
 0001:0004f7c0       ?InsertMultipleBefore@?$CUtlVector@UResourceMemorySection@CVTFTexture@@V?$CUtlMemory@UResourceMemorySection@CVTFTexture@@H@@@@QAEHHHPBUResourceMemorySection@CVTFTexture@@@Z 004507c0 f i vtf:vtf.obj
 0001:0004f8a0       ?LowResFileInfo@CVTFTexture@@UBEXPAH0@Z 004508a0 f   vtf:vtf.obj
 0001:0004f900       ?ImageFileInfo@CVTFTexture@@UBEXHHHPAH0@Z 00450900 f   vtf:vtf.obj
 0001:0004fa00       ?FileSize@CVTFTexture@@UBEHH@Z 00450a00 f   vtf:vtf.obj
 0001:0004fa40       ?GetResourceData@CVTFTexture@@UBEPAXIPAI@Z 00450a40 f   vtf:vtf.obj
 0001:0004fab0       ?HasResourceEntry@CVTFTexture@@UBE_NI@Z 00450ab0 f   vtf:vtf.obj
 0001:0004fad0       ?ConstructLowResImage@CVTFTexture@@UAE_NXZ 00450ad0 f   vtf:vtf.obj
 0001:0004fc10       ?InsertBefore@?$CUtlVector@UResourceMemorySection@CVTFTexture@@V?$CUtlMemory@UResourceMemorySection@CVTFTexture@@H@@@@QAEHH@Z 00450c10 f i vtf:vtf.obj
 0001:0004fc80       ??0CVTFTexture@@QAE@XZ     00450c80 f   vtf:vtf.obj
 0001:0004fd80       ??1CVTFTexture@@UAE@XZ     00450d80 f   vtf:vtf.obj
 0001:0004fde0       ?FindOrCreateResourceEntryInfo@CVTFTexture@@AAEPAUResourceEntryInfo@@I@Z 00450de0 f   vtf:vtf.obj
 0001:0004ff10       ?Serialize@CVTFTexture@@UAE_NAAVCUtlBuffer@@@Z 00450f10 f   vtf:vtf.obj
 0001:00050140       ??$DataMapInit@UVTFFileBaseHeader_t@@@@YAPAUdatamap_t@@PAUVTFFileBaseHeader_t@@@Z 00451140 f   vtf:vtf.obj
 0001:000501c0       ??$DataMapInit@UVTFFileHeaderV7_1_t@@@@YAPAUdatamap_t@@PAUVTFFileHeaderV7_1_t@@@Z 004511c0 f   vtf:vtf.obj
 0001:00050250       ??$DataMapInit@UVTFFileHeaderV7_2_t@@@@YAPAUdatamap_t@@PAUVTFFileHeaderV7_2_t@@@Z 00451250 f   vtf:vtf.obj
 0001:000502e0       ??$DataMapInit@UVTFFileHeaderV7_3_t@@@@YAPAUdatamap_t@@PAUVTFFileHeaderV7_3_t@@@Z 004512e0 f   vtf:vtf.obj
 0001:00050370       ??$DataMapInit@UVTFFileHeader_t@@@@YAPAUdatamap_t@@PAUVTFFileHeader_t@@@Z 00451370 f   vtf:vtf.obj
 0001:00050400       ??$DataMapInit@UVTFFileHeaderX360_t@@@@YAPAUdatamap_t@@PAUVTFFileHeaderX360_t@@@Z 00451400 f   vtf:vtf.obj
 0001:00050490       ?CreateVTFTexture@@YAPAVIVTFTexture@@XZ 00451490 f   vtf:vtf.obj
 0001:000504b0       ??_ECVTFTexture@@UAEPAXI@Z 004514b0 f i vtf:vtf.obj
 0001:000504b0       ??_GCVTFTexture@@UAEPAXI@Z 004514b0 f i vtf:vtf.obj
 0001:000504d0       ?Unserialize@CVTFTexture@@UAE_NAAVCUtlBuffer@@_NH@Z 004514d0 f   vtf:vtf.obj
 0001:000507b0       ?RemoveResourceEntryInfo@CVTFTexture@@AAE_NI@Z 004517b0 f   vtf:vtf.obj
 0001:000508a0       ?Init@CVTFTexture@@UAE_NHHHW4ImageFormat@@HHH@Z 004518a0 f   vtf:vtf.obj
 0001:000509f0       ?InitLowResImage@CVTFTexture@@UAEXHHW4ImageFormat@@@Z 004519f0 f   vtf:vtf.obj
 0001:00050a60       ?SetResourceData@CVTFTexture@@UAEPAXIPBXI@Z 00451a60 f   vtf:vtf.obj
 0001:00050b00       ?MatchCubeMapBorders@CVTFTexture@@UAEXHW4ImageFormat@@_N@Z 00451b00 f   vtf:vtf.obj
 0001:00050c90       ?WriteBitInt@@YAXPADHHH@Z  00451c90 f   vtf:s3tc_decode.obj
 0001:00050ce0       ?S3TC_GetPixelPaletteIndex@@YA?AVS3PaletteIndex@@W4ImageFormat@@PBDHH@Z 00451ce0 f   vtf:s3tc_decode.obj
 0001:00050d40       ?S3TC_SetPixelPaletteIndex@@YAXW4ImageFormat@@PADHHVS3PaletteIndex@@@Z 00451d40 f   vtf:s3tc_decode.obj
 0001:00050db0       ?S3TC_GetBlock@@YAPADPAXW4ImageFormat@@HHH@Z 00451db0 f   vtf:s3tc_decode.obj
 0001:00050de0       ?S3TC_MergeBlocks@@YAXPAPADPAPAVS3RGBA@@HHW4ImageFormat@@@Z 00451de0 f   vtf:s3tc_decode.obj
 0001:00051120       ?S3TC_GetPaletteIndex@@YA?AVS3PaletteIndex@@PAEW4ImageFormat@@HHH@Z 00452120 f   vtf:s3tc_decode.obj
 0001:00051180       ?S3TC_SetPaletteIndex@@YAXPAEW4ImageFormat@@HHHVS3PaletteIndex@@@Z 00452180 f   vtf:s3tc_decode.obj
 0001:000511d9       __cfltcvt_init             004521d9 f   LIBCMT:fpinit.obj
 0001:00051239       __fpmath                   00452239 f   LIBCMT:fpinit.obj
 0001:00051260       _memmove                   00452260 f   LIBCMT:memmove.obj
 0001:000515d0       _memset                    004525d0 f   LIBCMT:memset.obj
 0001:00051650       _memcpy                    00452650 f   LIBCMT:memcpy.obj
 0001:000519c0       __ftol2_sse                004529c0 f   LIBCMT:ftol2.obj
 0001:000519c9       __ftol2_pentium4           004529c9 f   LIBCMT:ftol2.obj
 0001:000519dc       __ftol2_sse_excpt          004529dc f   LIBCMT:ftol2.obj
 0001:000519f6       __ftol2                    004529f6 f   LIBCMT:ftol2.obj
 0001:00051a6b       __fclose_nolock            00452a6b f   LIBCMT:fclose.obj
 0001:00051add       _fclose                    00452add f   LIBCMT:fclose.obj
 0001:00051b59       _fprintf                   00452b59 f   LIBCMT:fprintf.obj
 0001:00051ca8       __fsopen                   00452ca8 f   LIBCMT:fopen.obj
 0001:00051d6c       _fopen                     00452d6c f   LIBCMT:fopen.obj
 0001:00051d7f       _sprintf                   00452d7f f   LIBCMT:sprintf.obj
 0001:00051e62       _sscanf                    00452e62 f   LIBCMT:sscanf.obj
 0001:00051e81       _strtok                    00452e81 f   LIBCMT:strtok.obj
 0001:00051f40       __alloca_probe_16          00452f40 f   LIBCMT:alloca16.obj
 0001:00051f56       __alloca_probe_8           00452f56     LIBCMT:alloca16.obj
 0001:00052025       ___onexitinit              00453025 f   LIBCMT:onexit.obj
 0001:00052054       __onexit                   00453054 f   LIBCMT:onexit.obj
 0001:00052090       _atexit                    00453090 f   LIBCMT:onexit.obj
 0001:000520a2       _srand                     004530a2 f   LIBCMT:rand.obj
 0001:000520af       _rand                      004530af f   LIBCMT:rand.obj
 0001:000521a0       _qsort                     004531a0 f   LIBCMT:qsort.obj
 0001:00052450       _strncpy                   00453450 f   LIBCMT:strncpy.obj
 0001:00052574       ??1type_info@@UAE@XZ       00453574 f   LIBCMT:typinfo.obj
 0001:00052582       ??_Etype_info@@UAEPAXI@Z   00453582 f i LIBCMT:typinfo.obj
 0001:00052582       ??_Gtype_info@@UAEPAXI@Z   00453582 f i LIBCMT:typinfo.obj
 0001:0005259e       ??8type_info@@QBE_NABV0@@Z 0045359e f   LIBCMT:typinfo.obj
 0001:000525b9       __purecall                 004535b9 f   LIBCMT:purevirt.obj
 0001:000525f0       __chkstk                   004535f0 f   LIBCMT:chkstk.obj
 0001:000525f0       __alloca_probe             004535f0     LIBCMT:chkstk.obj
 0001:0005261b       ??0_LocaleUpdate@@QAE@PAUlocaleinfo_struct@@@Z 0045361b f i LIBCMT:atof.obj
 0001:0005269d       __atof_l                   0045369d f   LIBCMT:atof.obj
 0001:00052746       _atof                      00453746 f   LIBCMT:atof.obj
 0001:00052754       __fwrite_nolock            00453754 f   LIBCMT:fwrite.obj
 0001:000528b3       _fwrite                    004538b3 f   LIBCMT:fwrite.obj
 0001:00052940       _floor                     00453940 f   LIBCMT:floor_pentium4.obj
 0001:00052980       __floor_pentium4           00453980 f   LIBCMT:floor_pentium4.obj
 0001:00052a61       _printf                    00453a61 f   LIBCMT:printf.obj
 0001:00052b10       __get_printf_count_output  00453b10 f   LIBCMT:printf.obj
 0001:00052b26       _atol                      00453b26 f   LIBCMT:atox.obj
 0001:00052b37       _atoi                      00453b37 f   LIBCMT:atox.obj
 0001:00052b40       _strrchr                   00453b40 f   LIBCMT:strrchr.obj
 0001:00052b6d       __vsnprintf_l              00453b6d f   LIBCMT:vsnprint.obj
 0001:00052c1e       __vsnprintf                00453c1e f   LIBCMT:vsnprint.obj
 0001:00052c39       _memcpy_s                  00453c39 f   LIBCMT:memcpy_s.obj
 0001:00052cb4       _memmove_s                 00453cb4 f   LIBCMT:memmove_s.obj
 0001:00052d0f       ??0exception@std@@QAE@XZ   00453d0f f   LIBCMT:stdexcpt.obj
 0001:00052d20       ??0exception@std@@QAE@ABQBD@Z 00453d20 f   LIBCMT:stdexcpt.obj
 0001:00052d6e       ??0exception@std@@QAE@ABV01@@Z 00453d6e f   LIBCMT:stdexcpt.obj
 0001:00052dc6       ??1exception@std@@UAE@XZ   00453dc6 f   LIBCMT:stdexcpt.obj
 0001:00052ddc       ?what@exception@std@@UBEPBDXZ 00453ddc f   LIBCMT:stdexcpt.obj
 0001:00052de9       ??0bad_cast@std@@QAE@PBD@Z 00453de9 f   LIBCMT:stdexcpt.obj
 0001:00052e02       ??0bad_cast@std@@QAE@ABV01@@Z 00453e02 f   LIBCMT:stdexcpt.obj
 0001:00052e1a       ??1bad_cast@std@@UAE@XZ    00453e1a f   LIBCMT:stdexcpt.obj
 0001:00052e25       ??_Gexception@std@@UAEPAXI@Z 00453e25 f i LIBCMT:stdexcpt.obj
 0001:00052e25       ??_Eexception@std@@UAEPAXI@Z 00453e25 f i LIBCMT:stdexcpt.obj
 0001:00052e41       ??_Ebad_cast@std@@UAEPAXI@Z 00453e41 f i LIBCMT:stdexcpt.obj
 0001:00052e41       ??_Gbad_cast@std@@UAEPAXI@Z 00453e41 f i LIBCMT:stdexcpt.obj
 0001:00052e63       __initp_misc_invarg        00453e63 f   LIBCMT:invarg.obj
 0001:00052e6d       __invoke_watson            00453e6d f   LIBCMT:invarg.obj
 0001:00052f69       __invalid_parameter        00453f69 f   LIBCMT:invarg.obj
 0001:00052f8d       __invalid_parameter_noinfo 00453f8d f   LIBCMT:invarg.obj
 0001:00052f9d       __CxxThrowException@8      00453f9d f   LIBCMT:throw.obj
 0001:00052fe7       ?_JumpToContinuation@@YGXPAXPAUEHRegistrationNode@@@Z 00453fe7 f   LIBCMT:trnsctrl.obj
 0001:00053017       ?_CallMemberFunction2@@YGXPAX00H@Z 00454017 f   LIBCMT:trnsctrl.obj
 0001:00053017       ?_CallMemberFunction0@@YGXPAX0@Z 00454017 f   LIBCMT:trnsctrl.obj
 0001:00053017       ?_CallMemberFunction1@@YGXPAX00@Z 00454017 f   LIBCMT:trnsctrl.obj
 0001:0005301e       ?_UnwindNestedFrames@@YGXPAUEHRegistrationNode@@PAUEHExceptionRecord@@@Z 0045401e f   LIBCMT:trnsctrl.obj
 0001:00053070       ___CxxFrameHandler3        00454070 f   LIBCMT:trnsctrl.obj
 0001:000530d6       ?_CallSETranslator@@YAHPAUEHExceptionRecord@@PAUEHRegistrationNode@@PAX2PBU_s_FuncInfo@@H1@Z 004540d6 f   LIBCMT:trnsctrl.obj
 0001:00053248       ?_GetRangeOfTrysToCheck@@YAPBU_s_TryBlockMapEntry@@PBU_s_FuncInfo@@HHPAI1@Z 00454248 f   LIBCMT:trnsctrl.obj
 0001:000532bb       __CreateFrameInfo          004542bb f   LIBCMT:trnsctrl.obj
 0001:000532e3       __IsExceptionObjectToBeDestroyed 004542e3 f   LIBCMT:trnsctrl.obj
 0001:00053304       __FindAndUnlinkFrame       00454304 f   LIBCMT:trnsctrl.obj
 0001:00053350       ?_CallCatchBlock2@@YAPAXPAUEHRegistrationNode@@PBU_s_FuncInfo@@PAXHK@Z 00454350 f   LIBCMT:trnsctrl.obj
 0001:000533b0       _fmod                      004543b0 f   LIBCMT:87fmod.obj
 0001:000533ba       __CIfmod                   004543ba f   LIBCMT:87fmod.obj
 0001:00053400       _strchr                    00454400 f   LIBCMT:strchr.obj
 0001:00053406       ___from_strstr_to_strchr   00454406     LIBCMT:strchr.obj
 0001:000534be       _strncmp                   004544be f   LIBCMT:strncmp.obj
 0001:0005357c       __freea                    0045457c f i LIBCMT:strlwr.obj
 0001:00053597       ?_strlwr_s_l_stat@@YAHPADIPAUlocaleinfo_struct@@@Z 00454597 f   LIBCMT:strlwr.obj
 0001:00053718       __strlwr_s_l               00454718 f   LIBCMT:strlwr.obj
 0001:0005374a       __strlwr                   0045474a f   LIBCMT:strlwr.obj
 0001:0005374a       _strlwr                    0045474a f   LIBCMT:strlwr.obj
 0001:000537ac       __amsg_exit                004547ac f   LIBCMT:crt0dat.obj
 0001:000537d0       ___crtCorExitProcess       004547d0 f   LIBCMT:crt0dat.obj
 0001:000537f6       ___crtExitProcess          004547f6 f   LIBCMT:crt0dat.obj
 0001:0005380b       __lockexit                 0045480b f   LIBCMT:crt0dat.obj
 0001:00053814       __unlockexit               00454814 f   LIBCMT:crt0dat.obj
 0001:00053835       __initterm_e               00454835 f   LIBCMT:crt0dat.obj
 0001:00053855       __get_osplatform           00454855 f   LIBCMT:crt0dat.obj
 0001:0005388c       __get_winmajor             0045488c f   LIBCMT:crt0dat.obj
 0001:000538c8       __cinit                    004548c8 f   LIBCMT:crt0dat.obj
 0001:00053a3c       _exit                      00454a3c f   LIBCMT:crt0dat.obj
 0001:00053a4d       __exit                     00454a4d f   LIBCMT:crt0dat.obj
 0001:00053a5e       __cexit                    00454a5e f   LIBCMT:crt0dat.obj
 0001:00053a6d       __c_exit                   00454a6d f   LIBCMT:crt0dat.obj
 0001:00053a7c       __init_pointers            00454a7c f   LIBCMT:crt0dat.obj
 0001:00053ac8       _remove                    00454ac8 f   LIBCMT:unlink.obj
 0001:00053af2       __unlink                   00454af2 f   LIBCMT:unlink.obj
 0001:00053af7       __snprintf                 00454af7 f   LIBCMT:snprintf.obj
 0001:00053cf9       __tmpnam_helper            00454cf9 f   LIBCMT:tmpfile.obj
 0001:00053e38       _tmpnam                    00454e38 f   LIBCMT:tmpfile.obj
 0001:00053e5d       __ftell_nolock             00454e5d f   LIBCMT:ftell.obj
 0001:00053ff5       _ftell                     00454ff5 f   LIBCMT:ftell.obj
 0001:00054063       __fread_nolock_s           00455063 f   LIBCMT:fread.obj
 0001:00054269       _fread_s                   00455269 f   LIBCMT:fread.obj
 0001:000542ff       _fread                     004552ff f   LIBCMT:fread.obj
 0001:0005431a       __fseek_nolock             0045531a f   LIBCMT:fseek.obj
 0001:000543a1       _fseek                     004553a1 f   LIBCMT:fseek.obj
 0001:00054430       _ceil                      00455430 f   LIBCMT:ceil_pentium4.obj
 0001:00054470       __ceil_pentium4            00455470 f   LIBCMT:ceil_pentium4.obj
 0001:0005454d       ___iob_func                0045554d f   LIBCMT:_file.obj
 0001:00054553       ___initstdio               00455553 f   LIBCMT:_file.obj
 0001:00054604       ___endstdio                00455604 f   LIBCMT:_file.obj
 0001:00054624       __lock_file                00455624 f   LIBCMT:_file.obj
 0001:00054660       __lock_file2               00455660 f   LIBCMT:_file.obj
 0001:0005468e       __unlock_file              0045568e f   LIBCMT:_file.obj
 0001:000546c4       __unlock_file2             004556c4 f   LIBCMT:_file.obj
 0001:000546ee       __get_sys_err_msg          004556ee f i LIBCMT:strerror.obj
 0001:00054711       _strerror                  00455711 f   LIBCMT:strerror.obj
 0001:00054778       __get_errno_from_oserr     00455778 f   LIBCMT:dosmap.obj
 0001:000547b3       __errno                    004557b3 f   LIBCMT:dosmap.obj
 0001:000547c6       ___doserrno                004557c6 f   LIBCMT:dosmap.obj
 0001:000547d9       __dosmaperr                004557d9 f   LIBCMT:dosmap.obj
 0001:000547f7       _fgetc                     004557f7 f   LIBCMT:fgetc.obj
 0001:0005492e       _fputc                     0045592e f   LIBCMT:fputc.obj
 0001:00054a6d       __ungetc_nolock            00455a6d f   LIBCMT:ungetc.obj
 0001:00054b8b       _ungetc                    00455b8b f   LIBCMT:ungetc.obj
 0001:00054bfd       __flush                    00455bfd f   LIBCMT:fflush.obj
 0001:00054c5f       __fflush_nolock            00455c5f f   LIBCMT:fflush.obj
 0001:00054d7b       _fflush                    00455d7b f   LIBCMT:fflush.obj
 0001:00054dce       __flushall                 00455dce f   LIBCMT:fflush.obj
 0001:00054dd7       _setvbuf                   00455dd7 f   LIBCMT:setvbuf.obj
 0001:00054ed5       _fgetpos                   00455ed5 f   LIBCMT:fgetpos.obj
 0001:00054f40       _fsetpos                   00455f40 f   LIBCMT:fsetpos.obj
 0001:00054f90       _strstr                    00455f90 f   LIBCMT:strstr.obj
 0001:00055016       __initp_heap_handler       00456016 f   LIBCMT:handler.obj
 0001:00055020       __validdrive               00456020 f   LIBCMT:getcwd.obj
 0001:00055057       __getdcwd_nolock           00456057 f   LIBCMT:getcwd.obj
 0001:0005518c       __getcwd                   0045618c f   LIBCMT:getcwd.obj
 0001:000551d5       _mkdir                     004561d5 f   LIBCMT:mkdir.obj
 0001:000551d5       __mkdir                    004561d5 f   LIBCMT:mkdir.obj
 0001:00055201       __findclose                00456201 f   LIBCMT:findfile.obj
 0001:00055221       ___time64_t_from_ft        00456221 f   LIBCMT:findfi32.obj
 0001:00055287       __findfirst64i32           00456287 f   LIBCMT:findfi32.obj
 0001:000553b7       __findnext64i32            004563b7 f   LIBCMT:findfi32.obj
 0001:000556f5       __putenv                   004566f5 f   LIBCMT:putenv.obj
 0001:0005573a       __access_s                 0045673a f   LIBCMT:access.obj
 0001:000557c1       __access                   004567c1 f   LIBCMT:access.obj
 0001:000557d5       __getenv_helper_nolock     004567d5 f   LIBCMT:getenv.obj
 0001:00055856       _getenv                    00456856 f   LIBCMT:getenv.obj
 0001:000558d9       __dupenv_s                 004568d9 f   LIBCMT:getenv.obj
 0001:000559bf       __spawnv                   004569bf f   LIBCMT:spawnv.obj
 0001:00055a0e       __chdir                    00456a0e f   LIBCMT:chdir.obj
 0001:00055b31       __tempnam                  00456b31 f   LIBCMT:tempnam.obj
 0001:00055dc7       __isalpha_l                00456dc7 f i LIBCMT:_ctype.obj
 0001:00055e1b       _isalpha                   00456e1b f i LIBCMT:_ctype.obj
 0001:00055e46       __isupper_l                00456e46 f i LIBCMT:_ctype.obj
 0001:00055e95       _isupper                   00456e95 f i LIBCMT:_ctype.obj
 0001:00055ebe       __islower_l                00456ebe f i LIBCMT:_ctype.obj
 0001:00055f0d       _islower                   00456f0d f i LIBCMT:_ctype.obj
 0001:00055f36       __isdigit_l                00456f36 f i LIBCMT:_ctype.obj
 0001:00055f85       _isdigit                   00456f85 f i LIBCMT:_ctype.obj
 0001:00055fae       __isxdigit_l               00456fae f i LIBCMT:_ctype.obj
 0001:00056002       _isxdigit                  00457002 f i LIBCMT:_ctype.obj
 0001:0005602d       __isspace_l                0045702d f i LIBCMT:_ctype.obj
 0001:0005607c       _isspace                   0045707c f i LIBCMT:_ctype.obj
 0001:000562c0       _mainCRTStartup            004572c0 f   LIBCMT:crt0.obj
 0001:000562ca       __tolower_l                004572ca f   LIBCMT:tolower.obj
 0001:000563e1       _tolower                   004573e1 f   LIBCMT:tolower.obj
 0001:00056410       _strncat                   00457410 f   LIBCMT:strncat.obj
 0001:00056550       __allrem                   00457550 f   LIBCMT:llrem.obj
 0001:00056610       __alldiv                   00457610 f   LIBCMT:lldiv.obj
 0001:000566ba       __strtod_l                 004576ba f   LIBCMT:strtod.obj
 0001:000567d5       _strtod                    004577d5 f   LIBCMT:strtod.obj
 0001:00056a13       _strtol                    00457a13 f   LIBCMT:strtol.obj
 0001:00056a3c       _strtoul                   00457a3c f   LIBCMT:strtol.obj
 0001:00056a66       __wtol                     00457a66 f   LIBCMT:wtox.obj
 0001:00056a77       __wtoi                     00457a77 f   LIBCMT:wtox.obj
 0001:00056a7c       __wtof_l                   00457a7c f   LIBCMT:wtof.obj
 0001:00056b06       __wtof                     00457b06 f   LIBCMT:wtof.obj
 0001:00056b20       __allmul                   00457b20 f   LIBCMT:llmul.obj
 0001:00056b54       __toupper_l                00457b54 f   LIBCMT:toupper.obj
 0001:00056c6c       _toupper                   00457c6c f   LIBCMT:toupper.obj
 0001:00056ca0       _acos                      00457ca0 f   LIBCMT:acos.obj
 0001:00056ce0       __CIacos                   00457ce0 f   LIBCMT:acos.obj
 0001:00056d1b       __CIacos_default           00457d1b f   LIBCMT:acos.obj
 0001:00056d2f       __acos_default             00457d2f     LIBCMT:acos.obj
 0001:00056df0       _asin                      00457df0 f   LIBCMT:asin.obj
 0001:00056e30       __CIasin                   00457e30 f   LIBCMT:asin.obj
 0001:00056e6b       __CIasin_default           00457e6b f   LIBCMT:asin.obj
 0001:00056e7f       __asin_default             00457e7f     LIBCMT:asin.obj
 0001:00056f40       _pow                       00457f40 f   LIBCMT:pow.obj
 0001:00056f80       __CIpow                    00457f80 f   LIBCMT:pow.obj
 0001:00056fbb       __CIpow_default            00457fbb f   LIBCMT:pow.obj
 0001:00056fd4       __pow_default              00457fd4     LIBCMT:pow.obj
 0001:000571d0       __allshr                   004581d0 f   LIBCMT:llshr.obj
 0001:000571f1       __forcdecpt_l              004581f1 f   LIBCMT:cvt.obj
 0001:00057262       __cropzeros_l              00458262 f   LIBCMT:cvt.obj
 0001:000572e2       __positive                 004582e2 f   LIBCMT:cvt.obj
 0001:000572f8       __fassign_l                004582f8 f   LIBCMT:cvt.obj
 0001:00057338       __fassign                  00458338 f   LIBCMT:cvt.obj
 0001:0005736c       __forcdecpt                0045836c f   LIBCMT:cvt.obj
 0001:0005737a       __cropzeros                0045837a f   LIBCMT:cvt.obj
 0001:000574f5       __cftoe_l                  004584f5 f   LIBCMT:cvt.obj
 0001:000575c3       __cftoe                    004585c3 f   LIBCMT:cvt.obj
 0001:000575e1       __cftoa_l                  004585e1 f   LIBCMT:cvt.obj
 0001:00057a47       __cftof_l                  00458a47 f   LIBCMT:cvt.obj
 0001:00057b00       __cftog_l                  00458b00 f   LIBCMT:cvt.obj
 0001:00057bf8       __cfltcvt_l                00458bf8 f   LIBCMT:cvt.obj
 0001:00057c7e       __cfltcvt                  00458c7e f   LIBCMT:cvt.obj
 0001:00057c9f       __initp_misc_cfltcvt_tab   00458c9f f   LIBCMT:cmiscdat.obj
 0001:00057cbe       __setdefaultprecision      00458cbe f   LIBCMT:fp8.obj
 0001:00057ce7       __ms_p5_test_fdiv          00458ce7 f   LIBCMT:testfdiv.obj
 0001:00057d23       __ms_p5_mp_test_fdiv       00458d23 f   LIBCMT:testfdiv.obj
 0001:00057dd3       __VEC_memcpy               00458dd3 f   LIBCMT:p4_memcpy.obj
 0001:00057eb6       __sse2_mathfcns_init       00458eb6 f   LIBCMT:mathfcns.obj
 0001:00057f21       __VEC_memzero              00458f21 f   LIBCMT:p4_memset.obj
 0001:00057fb0       __close_nolock             00458fb0 f   LIBCMT:close.obj
 0001:00058044       __close                    00459044 f   LIBCMT:close.obj
 0001:00058111       __fileno                   00459111 f   LIBCMT:fileno.obj
 0001:0005813e       __freebuf                  0045913e f   LIBCMT:_freebuf.obj
 0001:0005816c       __SEH_prolog4              0045916c f   LIBCMT:sehprolg4.obj
 0001:000581b1       __SEH_epilog4              004591b1 f   LIBCMT:sehprolg4.obj
 0001:000581d0       __except_handler4          004591d0 f   LIBCMT:chandler4.obj
 0001:00058366       __stbuf                    00459366 f   LIBCMT:_sftbuf.obj
 0001:000583fc       __ftbuf                    004593fc f   LIBCMT:_sftbuf.obj
 0001:000584cc       __output_l                 004594cc f   LIBCMT:output.obj
 0001:00058e60       __ioinit                   00459e60 f   LIBCMT:ioinit.obj
 0001:000590a0       __openfile                 0045a0a0 f   LIBCMT:_open.obj
 0001:00059340       __getstream                0045a340 f   LIBCMT:stream.obj
 0001:00059470       __local_unwind4            0045a470 f   LIBCMT:exsup4.obj
 0001:00059546       __seh_longjmp_unwind4@4    0045a546 f   LIBCMT:exsup4.obj
 0001:00059562       @_EH4_CallFilterFunc@8     0045a562 f   LIBCMT:exsup4.obj
 0001:00059579       @_EH4_TransferToHandler@8  0045a579 f   LIBCMT:exsup4.obj
 0001:00059592       @_EH4_GlobalUnwind@4       0045a592 f   LIBCMT:exsup4.obj
 0001:000595ac       @_EH4_LocalUnwind@16       0045a5ac f   LIBCMT:exsup4.obj
 0001:000595c3       __flsbuf                   0045a5c3 f   LIBCMT:_flsbuf.obj
 0001:00059730       _strlen                    0045a730 f   LIBCMT:strlen.obj
 0001:0005984a       __input_l                  0045a84a f   LIBCMT:input.obj
 0001:0005a503       __encode_pointer           0045b503 f   LIBCMT:tidtable.obj
 0001:0005a571       __encoded_null             0045b571 f   LIBCMT:tidtable.obj
 0001:0005a57a       __decode_pointer           0045b57a f   LIBCMT:tidtable.obj
 0001:0005a5e8       ___crtTlsAlloc@4           0045b5e8 f   LIBCMT:tidtable.obj
 0001:0005a5f1       ___set_flsgetvalue         0045b5f1 f   LIBCMT:tidtable.obj
 0001:0005a623       __mtterm                   0045b623 f   LIBCMT:tidtable.obj
 0001:0005a660       __initptd                  0045b660 f   LIBCMT:tidtable.obj
 0001:0005a71f       __getptd_noexit            0045b71f f   LIBCMT:tidtable.obj
 0001:0005a796       __getptd                   0045b796 f   LIBCMT:tidtable.obj
 0001:0005a7ae       __freefls@4                0045b7ae f   LIBCMT:tidtable.obj
 0001:0005a8cf       __mtinit                   0045b8cf f   LIBCMT:tidtable.obj
 0001:0005aa53       @__security_check_cookie@4 0045ba53 f   LIBCMT:secchk.obj
 0001:0005aa62       ?_Type_info_dtor@type_info@@CAXPAV1@@Z 0045ba62 f   LIBCMT:typname.obj
 0001:0005aae0       _strcmp                    0045bae0 f   LIBCMT:strcmp.obj
 0001:0005ab68       _abort                     0045bb68 f   LIBCMT:abort.obj
 0001:0005ac5b       __set_abort_behavior       0045bc5b f   LIBCMT:abort.obj
 0001:0005ac79       __NMSG_WRITE               0045bc79 f   LIBCMT:crt0msg.obj
 0001:0005ae19       __FF_MSGBANNER             0045be19 f   LIBCMT:crt0msg.obj
 0001:0005ae52       ___getlocaleinfo           0045be52 f   LIBCMT:inithelp.obj
 0001:0005afac       __initp_misc_purevirt      0045bfac f   LIBCMT:inithelp.obj
 0001:0005b1c4       ___updatetmbcinfo          0045c1c4 f   LIBCMT:mbctype.obj
 0001:0005b2e2       __setmbcp_nolock           0045c2e2 f   LIBCMT:mbctype.obj
 0001:0005b4bb       __setmbcp                  0045c4bb f   LIBCMT:mbctype.obj
 0001:0005b655       ___initmbctable            0045c655 f   LIBCMT:mbctype.obj
 0001:0005b673       ___freetlocinfo            0045c673 f   LIBCMT:setlocal.obj
 0001:0005b7b3       ___addlocaleref            0045c7b3 f   LIBCMT:setlocal.obj
 0001:0005b839       ___removelocaleref         0045c839 f   LIBCMT:setlocal.obj
 0001:0005b927       ___updatetlocinfo          0045c927 f   LIBCMT:setlocal.obj
 0001:0005b9f0       __strcats                  0045c9f0 f   LIBCMT:setlocal.obj
 0001:0005ba2e       ___lc_strtolc              0045ca2e f   LIBCMT:setlocal.obj
 0001:0005bb57       ___lc_lctostr              0045cb57 f   LIBCMT:setlocal.obj
 0001:0005bd33       __expandlocale             0045cd33 f   LIBCMT:setlocal.obj
 0001:0005c3cb       _setlocale                 0045d3cb f   LIBCMT:setlocal.obj
 0001:0005c53b       __fltin2                   0045d53b f   LIBCMT:cfin.obj
 0001:0005c5e0       __isctype_l                0045d5e0 f   LIBCMT:isctype.obj
 0001:0005c696       ___strgtold12_l            0045d696 f   LIBCMT:strgtold.obj
 0001:0005cd56       __write_nolock             0045dd56 f   LIBCMT:write.obj
 0001:0005d31c       __write                    0045e31c f   LIBCMT:write.obj
 0001:0005d3f8       ___libm_error_support      0045e3f8 f   LIBCMT:libm_error.obj
 0001:0005d6a8       __floor_default            0045e6a8 f   LIBCMT:floor.obj
 0001:0005d779       _strcpy_s                  0045e779 f   LIBCMT:strcpy_s.obj
 0001:0005d7de       __crt_debugger_hook        0045e7de f   LIBCMT:dbghook.obj
 0001:0005d7e6       ??1bad_exception@std@@UAE@XZ 0045e7e6 f i LIBCMT:frame.obj
 0001:0005d7f1       ??_Ebad_exception@std@@UAEPAXI@Z 0045e7f1 f i LIBCMT:frame.obj
 0001:0005d7f1       ??_Gbad_exception@std@@UAEPAXI@Z 0045e7f1 f i LIBCMT:frame.obj
 0001:0005d813       ___TypeMatch               0045e813 f   LIBCMT:frame.obj
 0001:0005d86f       ___FrameUnwindFilter       0045e86f f   LIBCMT:frame.obj
 0001:0005d8b3       ___FrameUnwindToState      0045e8b3 f   LIBCMT:frame.obj
 0001:0005d9d9       ___DestructExceptionObject 0045e9d9 f   LIBCMT:frame.obj
 0001:0005da2d       ___AdjustPointer           0045ea2d f   LIBCMT:frame.obj
 0001:0005dcb0       ___BuildCatchObjectHelper  0045ecb0 f   LIBCMT:frame.obj
 0001:0005de2f       ___BuildCatchObject        0045ee2f f   LIBCMT:frame.obj
 0001:0005e374       ??0bad_exception@std@@QAE@ABV01@@Z 0045f374 f i LIBCMT:frame.obj
 0001:0005e38c       ___InternalCxxFrameHandler 0045f38c f   LIBCMT:frame.obj
 0001:0005e470       ?terminate@@YAXXZ          0045f470 f   LIBCMT:hooks.obj
 0001:0005e4a9       ?unexpected@@YAXXZ         0045f4a9 f   LIBCMT:hooks.obj
 0001:0005e4bc       ?_inconsistency@@YAXXZ     0045f4bc f   LIBCMT:hooks.obj
 0001:0005e4f3       __initp_eh_hooks           0045f4f3 f   LIBCMT:hooks.obj
 0001:0005e510       __CallSettingFrame@12      0045f510 f   LIBCMT:lowhelpr.obj
 0001:0005e537       __NLG_Return               0045f537     LIBCMT:lowhelpr.obj
 0001:0005e560       __cintrindisp2             0045f560 f   LIBCMT:87cdisp.obj
 0001:0005e59e       __cintrindisp1             0045f59e f   LIBCMT:87cdisp.obj
 0001:0005e5db       __ctrandisp2               0045f5db f   LIBCMT:87cdisp.obj
 0001:0005e771       __ctrandisp1               0045f771 f   LIBCMT:87cdisp.obj
 0001:0005e7a4       __fload                    0045f7a4 f   LIBCMT:87cdisp.obj
 0001:0005e7e0       __trandisp1                0045f7e0 f   LIBCMT:87disp.obj
 0001:0005e847       __trandisp2                0045f847 f   LIBCMT:87disp.obj
 0001:0005e8d3       __rttospopde               0045f8d3     LIBCMT:87disp.obj
 0001:0005e8d8       __rttospop                 0045f8d8     LIBCMT:87disp.obj
 0001:0005e8da       __rtnospop                 0045f8da     LIBCMT:87disp.obj
 0001:0005e8dc       __rttosnpop                0045f8dc     LIBCMT:87disp.obj
 0001:0005e8dd       __rtnospopde               0045f8dd     LIBCMT:87disp.obj
 0001:0005e8e4       __rtzeropop                0045f8e4     LIBCMT:87disp.obj
 0001:0005e8e6       __rtzeronpop               0045f8e6     LIBCMT:87disp.obj
 0001:0005e8eb       __rtonepop                 0045f8eb     LIBCMT:87disp.obj
 0001:0005e8ed       __rtonenpop                0045f8ed     LIBCMT:87disp.obj
 0001:0005e8f2       __tosnan1                  0045f8f2     LIBCMT:87disp.obj
 0001:0005e91d       __nosnan2                  0045f91d     LIBCMT:87disp.obj
 0001:0005e91f       __tosnan2                  0045f91f     LIBCMT:87disp.obj
 0001:0005e947       __nan2                     0045f947     LIBCMT:87disp.obj
 0001:0005e986       __rtindfpop                0045f986     LIBCMT:87disp.obj
 0001:0005e988       __rtindfnpop               0045f988     LIBCMT:87disp.obj
 0001:0005e999       __rttosnpopde              0045f999     LIBCMT:87disp.obj
 0001:0005e9a3       __rtchsifneg               0045f9a3     LIBCMT:87disp.obj
 0001:0005e9b0       _fdiv_main_routine         0045f9b0 f   LIBCMT:adj_fdiv.obj
 0001:0005eac7       __adj_fdiv_r               0045fac7 f   LIBCMT:adj_fdiv.obj
 0001:0005ef66       __fdivp_sti_st             0045ff66 f   LIBCMT:adj_fdiv.obj
 0001:0005ef79       __fdivrp_sti_st            0045ff79 f   LIBCMT:adj_fdiv.obj
 0001:0005ef8c       __adj_fdiv_m32             0045ff8c f   LIBCMT:adj_fdiv.obj
 0001:0005efd8       __adj_fdiv_m64             0045ffd8 f   LIBCMT:adj_fdiv.obj
 0001:0005f024       __adj_fdiv_m16i            00460024 f   LIBCMT:adj_fdiv.obj
 0001:0005f058       __adj_fdiv_m32i            00460058 f   LIBCMT:adj_fdiv.obj
 0001:0005f08c       __adj_fdivr_m32            0046008c f   LIBCMT:adj_fdiv.obj
 0001:0005f0d8       __adj_fdivr_m64            004600d8 f   LIBCMT:adj_fdiv.obj
 0001:0005f124       __adj_fdivr_m16i           00460124 f   LIBCMT:adj_fdiv.obj
 0001:0005f158       __adj_fdivr_m32i           00460158 f   LIBCMT:adj_fdiv.obj
 0001:0005f18c       __safe_fdiv                0046018c f   LIBCMT:adj_fdiv.obj
 0001:0005f1a1       __safe_fdivr               004601a1 f   LIBCMT:adj_fdiv.obj
 0001:0005f1b6       __fprem_common             004601b6 f   LIBCMT:adj_fdiv.obj
 0001:0005f3bc       __adj_fprem                004603bc f   LIBCMT:adj_fdiv.obj
 0001:0005f46e       __fprem1_common            0046046e f   LIBCMT:adj_fdiv.obj
 0001:0005f674       __adj_fprem1               00460674 f   LIBCMT:adj_fdiv.obj
 0001:0005f729       __safe_fprem               00460729 f   LIBCMT:adj_fdiv.obj
 0001:0005f72f       __safe_fprem1              0046072f f   LIBCMT:adj_fdiv.obj
 0001:0005f735       __adj_fpatan               00460735 f   LIBCMT:adj_fdiv.obj
 0001:0005f738       __adj_fptan                00460738 f   LIBCMT:adj_fdiv.obj
 0001:0005fadd       ___crtLCMapStringA         00460add f   LIBCMT:a_map.obj
 0001:0005fb20       _strnlen                   00460b20 f   LIBCMT:strlen_s.obj
 0001:0005fb3a       __mtinitlocks              00460b3a f   LIBCMT:mlock.obj
 0001:0005fb83       __mtdeletelocks            00460b83 f   LIBCMT:mlock.obj
 0001:0005fbd8       __unlock                   00460bd8 f   LIBCMT:mlock.obj
 0001:0005fbed       __mtinitlocknum            00460bed f   LIBCMT:mlock.obj
 0001:0005fcb0       __lock                     00460cb0 f   LIBCMT:mlock.obj
 0001:0005fce1       __RTC_Initialize           00460ce1 f   LIBCMT:initsect.obj
 0001:0005fd05       __RTC_Terminate            00460d05 f   LIBCMT:initsect.obj
 0001:0005fd30       __ValidateImageBase        00460d30 f   LIBCMT:pesect.obj
 0001:0005fd60       __FindPESection            00460d60 f   LIBCMT:pesect.obj
 0001:0005fdb0       __IsNonwritableInCurrentImage 00460db0 f   LIBCMT:pesect.obj
 0001:0005fe6b       __initp_misc_winxfltr      00460e6b f   LIBCMT:winxfltr.obj
 0001:0005fe6b       __fpclear                  00460e6b f   LIBCMT:fpinit.obj
 0001:0005fe6c       __XcptFilter               00460e6c f   LIBCMT:winxfltr.obj
 0001:0005ffca       __initp_misc_winsig        00460fca f   LIBCMT:winsig.obj
 0001:00060017       ___get_sigabrt             00461017 f   LIBCMT:winsig.obj
 0001:00060024       _raise                     00461024 f   LIBCMT:winsig.obj
 0001:000601d4       __initp_misc_rand_s        004611d4 f   LIBCMT:rand_s.obj
 0001:000601de       __initp_misc_initcrit      004611de f   LIBCMT:initcrit.obj
 0001:000601f8       ___crtInitCritSecAndSpinCount 004611f8 f   LIBCMT:initcrit.obj
 0001:000602bd       _strcat_s                  004612bd f   LIBCMT:strcat_s.obj
 0001:00060409       __itoa_s                   00461409 f   LIBCMT:xtoas.obj
 0001:00060431       __ultoa_s                  00461431 f   LIBCMT:xtoas.obj
 0001:00060449       __getpid                   00461449 f   LIBCMT:getpid.obj
 0001:0006044f       __mbsrchr_l                0046144f f   LIBCMT:mbsrchr.obj
 0001:0006050f       __mbsrchr                  0046150f f   LIBCMT:mbsrchr.obj
 0001:00060522       __rmtmp                    00461522 f   LIBCMT:rmtmp.obj
 0001:00060d24       __sopen_helper             00461d24 f   LIBCMT:open.obj
 0001:00060df0       __sopen_s                  00461df0 f   LIBCMT:open.obj
 0001:00060e0e       __lseek_nolock             00461e0e f   LIBCMT:lseek.obj
 0001:00060e80       __lseek                    00461e80 f   LIBCMT:lseek.obj
 0001:00060f5c       __filbuf                   00461f5c f   LIBCMT:_filbuf.obj
 0001:0006107c       __read_nolock              0046207c f   LIBCMT:read.obj
 0001:0006163d       __read                     0046263d f   LIBCMT:read.obj
 0001:0006173a       __ceil_default             0046273a f   LIBCMT:ceil.obj
 0001:0006180b       __fcloseall                0046280b f   LIBCMT:closeall.obj
 0001:000618aa       ___sys_nerr                004628aa f   LIBCMT:syserr.obj
 0001:000618b0       ___sys_errlist             004628b0 f   LIBCMT:syserr.obj
 0001:000618b6       _strncpy_s                 004628b6 f   LIBCMT:strncpy_s.obj
 0001:00061969       __getbuf                   00462969 f   LIBCMT:_getbuf.obj
 0001:000619ad       __commit                   004629ad f   LIBCMT:commit.obj
 0001:00061a8e       __ftelli64_nolock          00462a8e f   LIBCMT:ftelli64.obj
 0001:00061d6a       __ftelli64                 00462d6a f   LIBCMT:ftelli64.obj
 0001:00061db4       __fseeki64_nolock          00462db4 f   LIBCMT:fseeki64.obj
 0001:00061e4d       __fseeki64                 00462e4d f   LIBCMT:fseeki64.obj
 0001:00061e9c       ___loctotime64_t           00462e9c f   LIBCMT:dtoxtm64.obj
 0001:00062105       __getdrive                 00463105 f   LIBCMT:drive.obj
 0001:00062279       ___crtwsetenv              00463279 f   LIBCMT:wsetenv.obj
 0001:000625df       _wcslen                    004635df f   LIBCMT:wcslen.obj
 0001:0006269f       ___crtsetenv               0046369f f   LIBCMT:setenv.obj
 0001:000628eb       __mbschr_l                 004638eb f   LIBCMT:mbschr.obj
 0001:000629a5       __mbschr                   004639a5 f   LIBCMT:mbschr.obj
 0001:000629b8       __mbsnbicoll_l             004639b8 f   LIBCMT:mbsnbico.obj
 0001:00062aa4       __mbsnbicoll               00463aa4 f   LIBCMT:mbsnbico.obj
 0001:00062abb       ___wtomb_environ           00463abb f   LIBCMT:wtombenv.obj
 0001:00062bc8       __spawnve                  00463bc8 f   LIBCMT:spawnve.obj
 0001:00062de7       __mbctoupper_l             00463de7 f   LIBCMT:mbtoupr.obj
 0001:00062e8b       __mbctoupper               00463e8b f   LIBCMT:mbtoupr.obj
 0001:00062e99       ?__CxxUnhandledExceptionFilter@@YGJPAU_EXCEPTION_POINTERS@@@Z 00463e99 f   LIBCMT:unhandld.obj
 0001:00062ed6       ___CxxSetUnhandledExceptionFilter 00463ed6 f   LIBCMT:unhandld.obj
 0001:00062ee4       __setenvp                  00463ee4 f   LIBCMT:stdenvp.obj
 0001:00063157       __setargv                  00464157 f   LIBCMT:stdargv.obj
 0001:00063210       ___crtGetEnvironmentStringsA 00464210 f   LIBCMT:a_env.obj
 0001:00063345       ___security_init_cookie    00464345 f   LIBCMT:gs_support.obj
 0001:000633d9       __isleadbyte_l             004643d9 f i LIBCMT:_wctype.obj
 0001:0006340f       _isleadbyte                0046440f f i LIBCMT:_wctype.obj
 0001:00063617       _wcstol                    00464617 f   LIBCMT:wcstol.obj
 0001:00063640       __wfltin2                  00464640 f   LIBCMT:wcfin.obj
 0001:000636e7       __iswctype_l               004646e7 f   LIBCMT:iswctype.obj
 0001:00063769       ___wstrgtold12_l           00464769 f   LIBCMT:wstrgtold.obj
 0001:00063e90       __CIacos_pentium4          00464e90 f   LIBCMT:acos_pentium4.obj
 0001:00063ea8       __acos_pentium4            00464ea8     LIBCMT:acos_pentium4.obj
 0001:000643f0       __startTwoArgErrorHandling 004653f0 f   LIBCMT:genexcep.obj
 0001:00064407       __startOneArgErrorHandling 00465407 f   LIBCMT:genexcep.obj
 0001:00064450       __twoToTOS                 00465450 f   LIBCMT:common.obj
 0001:00064465       __load_CW                  00465465 f   LIBCMT:common.obj
 0001:0006447c       __convertTOStoQNaN         0046547c f   LIBCMT:common.obj
 0001:00064495       __fload_withFB             00465495 f   LIBCMT:common.obj
 0001:000644d8       __checkTOS_withFB          004654d8 f   LIBCMT:common.obj
 0001:000644ee       __fast_exit                004654ee f   LIBCMT:common.obj
 0001:000644fb       __math_exit                004654fb f   LIBCMT:common.obj
 0001:00064525       __check_overflow_exit      00465525 f   LIBCMT:common.obj
 0001:00064539       __check_range_exit         00465539 f   LIBCMT:common.obj
 0001:000645e0       __CIasin_pentium4          004655e0 f   LIBCMT:asin_pentium4.obj
 0001:000645f8       __asin_pentium4            004655f8     LIBCMT:asin_pentium4.obj
 0001:00064b60       __CIpow_pentium4           00465b60 f   LIBCMT:pow_pentium4.obj
 0001:00064b79       __pow_pentium4             00465b79     LIBCMT:pow_pentium4.obj
 0001:000656d1       __fFEXP                    004666d1     LIBCMT:87tran.obj
 0001:00065738       __rtinfpopse               00466738     LIBCMT:87tran.obj
 0001:0006573a       __rtinfnpopse              0046673a     LIBCMT:87tran.obj
 0001:0006574a       __fFLN                     0046674a     LIBCMT:87tran.obj
 0001:000657ff       __rtinfpop                 004667ff     LIBCMT:87tran.obj
 0001:00065801       __rtinfnpop                00466801     LIBCMT:87tran.obj
 0001:0006581e       __ffexpm1                  0046681e     LIBCMT:87tran.obj
 0001:000658c7       __d_inttype                004668c7 f   LIBCMT:powhlp.obj
 0001:0006592b       __powhlp                   0046692b f   LIBCMT:powhlp.obj
 0001:00065a69       __atodbl_l                 00466a69 f   LIBCMT:atodbl.obj
 0001:00065b0f       __atoflt_l                 00466b0f f   LIBCMT:atodbl.obj
 0001:00065bb5       __fptostr                  00466bb5 f   LIBCMT:_fptostr.obj
 0001:00065c72       ___dtold                   00466c72 f   LIBCMT:cfout.obj
 0001:00065d2d       __fltout2                  00466d2d f   LIBCMT:cfout.obj
 0001:00065dc0       __alldvrm                  00466dc0 f   LIBCMT:lldvrm.obj
 0001:00065ea0       __aullshr                  00466ea0 f   LIBCMT:ullshr.obj
 0001:00065ebf       __fptrap                   00466ebf f   LIBCMT:crt0fp.obj
 0001:00065ec8       __controlfp_s              00466ec8 f   LIBCMT:contrlfp.obj
 0001:00065f82       __get_sse2_info            00466f82 f   LIBCMT:cpu_disp.obj
 0001:00065fe2       ___sse2_available_init     00466fe2 f   LIBCMT:cpu_disp.obj
 0001:00065fef       __set_osfhnd               00466fef f   LIBCMT:osfinfo.obj
 0001:0006606c       __free_osfhnd              0046706c f   LIBCMT:osfinfo.obj
 0001:000660ed       __get_osfhandle            004670ed f   LIBCMT:osfinfo.obj
 0001:0006615e       ___lock_fhandle            0046715e f   LIBCMT:osfinfo.obj
 0001:000661fe       __unlock_fhandle           004671fe f   LIBCMT:osfinfo.obj
 0001:00066220       __alloc_osfhnd             00467220 f   LIBCMT:osfinfo.obj
 0001:000663bf       __isatty                   004673bf f   LIBCMT:isatty.obj
 0001:0006641d       __wctomb_s_l               0046741d f   LIBCMT:wctomb.obj
 0001:0006657c       _wctomb_s                  0046757c f   LIBCMT:wctomb.obj
 0001:000665a0       __aulldvrm                 004675a0 f   LIBCMT:ulldvrm.obj
 0001:00066635       __mbsicmp_l                00467635 f   LIBCMT:mbsicmp.obj
 0001:0006684f       __mbsicmp                  0046784f f   LIBCMT:mbsicmp.obj
 0001:00066862       __mbsnbcmp_l               00467862 f   LIBCMT:mbsnbcmp.obj
 0001:000669cb       __mbsnbcmp                 004679cb f   LIBCMT:mbsnbcmp.obj
 0001:000669e4       __global_unwind2           004679e4 f   LIBCMT:exsup.obj
 0001:00066a49       __local_unwind2            00467a49 f   LIBCMT:exsup.obj
 0001:00066acd       __abnormal_termination     00467acd f   LIBCMT:exsup.obj
 0001:00066af0       __NLG_Notify1              00467af0 f   LIBCMT:exsup.obj
 0001:00066af9       __NLG_Notify               00467af9 f   LIBCMT:exsup.obj
 0001:00066b10       __NLG_Dispatch2            00467b10     LIBCMT:exsup.obj
 0001:00066b10       __NLG_Dispatch             00467b10     LIBCMT:exsup.obj
 0001:00066b18       __NLG_Call                 00467b18 f   LIBCMT:exsup.obj
 0001:00066b1a       __NLG_Return2              00467b1a     LIBCMT:exsup.obj
 0001:00066b1b       __lseeki64_nolock          00467b1b f   LIBCMT:lseeki64.obj
 0001:00066b9e       __lseeki64                 00467b9e f   LIBCMT:lseeki64.obj
 0001:00066cb7       __mbtowc_l                 00467cb7 f   LIBCMT:mbtowc.obj
 0001:00066dca       _mbtowc                    00467dca f   LIBCMT:mbtowc.obj
 0001:00066de1       ___report_gsfailure        00467de1 f   LIBCMT:gs_report.obj
 0001:00066ee5       ___crtMessageBoxA          00467ee5 f   LIBCMT:crtmbox.obj
 0001:000670a2       __set_error_mode           004680a2 f   LIBCMT:errmode.obj
 0001:00067223       ___crtGetLocaleInfoW       00468223 f   LIBCMT:w_loc.obj
 0001:0006739b       ___crtGetLocaleInfoA       0046839b f   LIBCMT:a_loc.obj
 0001:0006758e       ___crtGetStringTypeA       0046858e f   LIBCMT:a_str.obj
 0001:000675ce       ___pctype_func             004685ce f   LIBCMT:ctype.obj
 0001:00067a10       ___free_lc_time            00468a10 f   LIBCMT:inittime.obj
 0001:00067ba0       ___init_time               00468ba0 f   LIBCMT:inittime.obj
 0001:00067c13       ___free_lconv_num          00468c13 f   LIBCMT:initnum.obj
 0001:00067c53       ___init_numeric            00468c53 f   LIBCMT:initnum.obj
 0001:00067e1b       ___free_lconv_mon          00468e1b f   LIBCMT:initmon.obj
 0001:00067ea4       ___init_monetary           00468ea4 f   LIBCMT:initmon.obj
 0001:00068168       ___init_ctype              00469168 f   LIBCMT:initctyp.obj
 0001:000684fd       ____lc_codepage_func       004694fd f   LIBCMT:initctyp.obj
 0001:00068523       ____lc_handle_func         00469523 f   LIBCMT:initctyp.obj
 0001:00068550       _strcspn                   00469550 f   LIBCMT:strcspn.obj
 0001:00068b10       ___get_qualified_locale    00469b10 f   LIBCMT:getqloc.obj
 0001:00068cf3       _memcmp                    00469cf3 f   LIBCMT:memcmp.obj
 0001:0006a380       _strpbrk                   0046b380 f   LIBCMT:strpbrk.obj
 0001:0006a3c0       __ld12tod                  0046b3c0 f   LIBCMT:intrncvt.obj
 0001:0006a902       __ld12tof                  0046b902 f   LIBCMT:intrncvt.obj
 0001:0006ae44       ___mtold12                 0046be44 f   LIBCMT:mantold.obj
 0001:0006b010       __putwch_nolock            0046c010 f   LIBCMT:putwch.obj
 0001:0006b0d2       ___init_collate            0046c0d2 f   LIBCMT:initcoll.obj
 0001:0006b0d2       __matherr                  0046c0d2 f   LIBCMT:matherr.obj
 0001:0006b0d2       ___init_dummy              0046c0d2 f   LIBCMT:setlocal.obj
 0001:0006b0d5       __raise_exc_ex             0046c0d5 f   LIBCMT:fpexcept.obj
 0001:0006b3af       __raise_exc                0046c3af f   LIBCMT:fpexcept.obj
 0001:0006b3d0       __handle_exc               0046c3d0 f   LIBCMT:fpexcept.obj
 0001:0006b5b1       __set_errno_from_matherr   0046c5b1 f   LIBCMT:fpexcept.obj
 0001:0006b5d9       __errcode                  0046c5d9 f   LIBCMT:fpexcept.obj
 0001:0006b606       __umatherr                 0046c606 f   LIBCMT:fpexcept.obj
 0001:0006b6a4       __handle_qnan1             0046c6a4 f   LIBCMT:fpexcept.obj
 0001:0006b6f7       __except1                  0046c6f7 f   LIBCMT:fpexcept.obj
 0001:0006b7b1       __frnd                     0046c7b1 f   LIBCMT:frnd.obj
 0001:0006b7c2       __set_exp                  0046c7c2 f   LIBCMT:util.obj
 0001:0006b7ec       __sptype                   0046c7ec f   LIBCMT:util.obj
 0001:0006b847       __decomp                   0046c847 f   LIBCMT:util.obj
 0001:0006b8f6       __statfp                   0046c8f6 f   LIBCMT:fpctrl.obj
 0001:0006b901       __clrfp                    0046c901 f   LIBCMT:fpctrl.obj
 0001:0006b90d       __ctrlfp                   0046c90d f   LIBCMT:fpctrl.obj
 0001:0006b934       __set_statfp               0046c934 f   LIBCMT:fpctrl.obj
 0001:0006b98a       ___set_fpsr_sse2           0046c98a f   LIBCMT:fpctrl.obj
 0001:0006b9fc       __EH_prolog3               0046c9fc f   LIBCMT:ehprolg3.obj
 0001:0006ba2f       __EH_prolog3_catch         0046ca2f f   LIBCMT:ehprolg3.obj
 0001:0006ba65       __EH_epilog3               0046ca65 f   LIBCMT:ehprolg3.obj
 0001:0006ba79       ?_ValidateRead@@YAHPBXI@Z  0046ca79 f   LIBCMT:validate.obj
 0001:0006ba79       ?_ValidateWrite@@YAHPAXI@Z 0046ca79 f   LIBCMT:validate.obj
 0001:0006ba79       ?_ValidateExecute@@YAHP6GHXZ@Z 0046ca79 f   LIBCMT:validate.obj
 0001:0006ba86       __87except                 0046ca86 f   LIBCMT:87except.obj
 0001:0006bb82       ___ansicp                  0046cb82 f   LIBCMT:convrtcp.obj
 0001:0006bbc9       ___convertcp               0046cbc9 f   LIBCMT:convrtcp.obj
 0001:0006bd7b       __chsize_nolock            0046cd7b f   LIBCMT:chsize.obj
 0001:0006bf2f       __setmode_nolock           0046cf2f f   LIBCMT:setmode.obj
 0001:0006bfeb       __get_fmode                0046cfeb f   LIBCMT:setmode.obj
 0001:0006c70b       ___tzset                   0046d70b f   LIBCMT:tzset.obj
 0001:0006c75a       __isindst                  0046d75a f   LIBCMT:tzset.obj
 0001:0006c79b       __get_daylight             0046d79b f   LIBCMT:timeset.obj
 0001:0006c7cf       __get_dstbias              0046d7cf f   LIBCMT:timeset.obj
 0001:0006c803       __get_timezone             0046d803 f   LIBCMT:timeset.obj
 0001:0006c837       ___daylight                0046d837 f   LIBCMT:timeset.obj
 0001:0006c83d       ___dstbias                 0046d83d f   LIBCMT:timeset.obj
 0001:0006c843       ___timezone                0046d843 f   LIBCMT:timeset.obj
 0001:0006c849       ___tzname                  0046d849 f   LIBCMT:timeset.obj
 0001:0006c84f       __wcsnicoll_l              0046d84f f   LIBCMT:wcsnicol.obj
 0001:0006c990       __wcsnicoll                0046d990 f   LIBCMT:wcsnicol.obj
 0001:0006ca32       _wcscpy_s                  0046da32 f   LIBCMT:wcscpy_s.obj
 0001:0006ca9e       ___mbtow_environ           0046da9e f   LIBCMT:mbtowenv.obj
 0001:0006cb23       __wsetenvp                 0046db23 f   LIBCMT:wstdenvp.obj
 0001:0006cbfd       ___crtGetEnvironmentStringsW 0046dbfd f   LIBCMT:w_env.obj
 0001:0006cd5e       _wcschr                    0046dd5e f   LIBCMT:wcschr.obj
 0001:0006d109       ___crtCompareStringA       0046e109 f   LIBCMT:a_cmp.obj
 0001:0006d149       __strnicoll_l              0046e149 f   LIBCMT:strnicol.obj
 0001:0006d241       __dospawn                  0046e241 f   LIBCMT:dospawn.obj
 0001:0006d44e       __cenvarg                  0046e44e f   LIBCMT:cenvarg.obj
 0001:0006d876       __ismbblead                0046e876 f   LIBCMT:ismbbyte.obj
 0001:0006d889       __wchartodigit             0046e889 f   LIBCMT:wchtodig.obj
 0001:0006dc2f       ___crtGetStringTypeW       0046ec2f f   LIBCMT:w_str.obj
 0001:0006dc6d       __fpclass                  0046ec6d f   LIBCMT:ieeemisc.obj
 0001:0006dd01       _$I10_OUTPUT               0046ed01 f   LIBCMT:x10fout.obj
 0001:0006e6f5       __control87                0046f6f5 f i LIBCMT:ieee87.obj
 0001:0006e9f8       __controlfp                0046f9f8 f   LIBCMT:ieee87.obj
 0001:0006ed01       ___ascii_stricmp           0046fd01 f   LIBCMT:stricmp.obj
 0001:0006ed36       __stricmp_l                0046fd36 f   LIBCMT:stricmp.obj
 0001:0006ee09       _stricmp                   0046fe09 f   LIBCMT:stricmp.obj
 0001:0006ee09       __stricmp                  0046fe09 f   LIBCMT:stricmp.obj
 0001:0006ee09       _strcmpi                   0046fe09 f   LIBCMT:stricmp.obj
 0001:0006ee59       __strnicmp_l               0046fe59 f   LIBCMT:strnicmp.obj
 0001:0006ef49       _strnicmp                  0046ff49 f   LIBCMT:strnicmp.obj
 0001:0006ef49       __strnicmp                 0046ff49 f   LIBCMT:strnicmp.obj
 0001:0006efa5       ___initconin               0046ffa5 f   LIBCMT:initcon.obj
 0001:0006efc4       ___initconout              0046ffc4 f   LIBCMT:initcon.obj
 0001:0006efe3       ___termcon                 0046ffe3 f   LIBCMT:initcon.obj
 0001:0006f27c       ___crtCompareStringW       0047027c f   LIBCMT:w_cmp.obj
 0001:0006f2bc       __mbsnicmp_l               004702bc f   LIBCMT:mbsnicmp.obj
 0001:0006f485       __mbsnicmp                 00470485 f   LIBCMT:mbsnicmp.obj
 0001:0006f4a0       ___ascii_strnicmp          004704a0 f   LIBCMT:_strnicm.obj
 0001:0006f501       ??1out_of_range@std@@UAE@XZ 00470501 f i libcpmt:string.obj
 0001:0006f50c       ??_Gout_of_range@std@@UAEPAXI@Z 0047050c f i libcpmt:string.obj
 0001:0006f50c       ??_Eout_of_range@std@@UAEPAXI@Z 0047050c f i libcpmt:string.obj
 0001:0006f52e       ?_Xlen@_String_base@std@@SAXXZ 0047052e f   libcpmt:string.obj
 0001:0006f56d       ?_Xran@_String_base@std@@SAXXZ 0047056d f   libcpmt:string.obj
 0001:0006f5ac       ??0out_of_range@std@@QAE@ABV01@@Z 004705ac f i libcpmt:string.obj
 0001:0006f5c4       ??0_Init_locks@std@@QAE@XZ 004705c4 f   libcpmt:xlock.obj
 0001:0006f5f3       ??1_Init_locks@std@@QAE@XZ 004705f3 f   libcpmt:xlock.obj
 0001:0006f61c       ??0_Lockit@std@@QAE@H@Z    0047061c f   libcpmt:xlock.obj
 0001:0006f63d       ??1_Lockit@std@@QAE@XZ     0047063d f   libcpmt:xlock.obj
 0001:0006f64f       ?_Callfns@ios_base@std@@AAEXW4event@12@@Z 0047064f f i libcpmt:ios.obj
 0001:0006f671       ?_Tidy@ios_base@std@@AAAXXZ 00470671 f i libcpmt:ios.obj
 0001:0006f6b7       ?_Ios_base_dtor@ios_base@std@@CAXPAV12@@Z 004706b7 f   libcpmt:ios.obj
 0001:0006f6f5       ??0_Mutex@std@@QAE@XZ      004706f5 f   libcpmt:xmutex.obj
 0001:0006f70d       ??1_Mutex@std@@QAE@XZ      0047070d f   libcpmt:xmutex.obj
 0001:0006f722       ?_Lock@_Mutex@std@@QAEXXZ  00470722 f   libcpmt:xmutex.obj
 0001:0006f72b       ?_Unlock@_Mutex@std@@QAEXXZ 0047072b f   libcpmt:xmutex.obj
 0001:0006f734       ??1_Fac_node@std@@QAE@XZ   00470734 f i libcpmt:locale0.obj
 0001:0006f749       __Deletegloballocale       00470749 f   libcpmt:locale0.obj
 0001:0006f78f       ?_Getgloballocale@locale@std@@CAPAV_Locimp@12@XZ 0047078f f   libcpmt:locale0.obj
 0001:0006f795       ?_Setgloballocale@locale@std@@CAXPAX@Z 00470795 f   libcpmt:locale0.obj
 0001:0006f7ba       ?_Locimp_dtor@_Locimp@locale@std@@CAXPAV123@@Z 004707ba f   libcpmt:locale0.obj
 0001:0006f81a       __Fac_tidy                 0047081a f   libcpmt:locale0.obj
 0001:0006f85d       ?facet_Register@facet@locale@std@@CAXPAV123@@Z 0047085d f   libcpmt:locale0.obj
 0001:0006f896       ?_Locinfo_dtor@_Locinfo@std@@SAXPAV12@@Z 00470896 f   libcpmt:locale0.obj
 0001:0006f8b9       ??0_Locimp@locale@std@@AAE@_N@Z 004708b9 f i libcpmt:locale0.obj
 0001:0006f902       ??1_Locimp@locale@std@@MAE@XZ 00470902 f i libcpmt:locale0.obj
 0001:0006f93f       ??_E_Locimp@locale@std@@MAEPAXI@Z 0047093f f i libcpmt:locale0.obj
 0001:0006f93f       ??_G_Locimp@locale@std@@MAEPAXI@Z 0047093f f i libcpmt:locale0.obj
 0001:0006f95b       ?_Init@locale@std@@CAPAV_Locimp@12@XZ 0047095b f   libcpmt:locale0.obj
 0001:0006f9f5       ?_Locinfo_ctor@_Locinfo@std@@SAXPAV12@PBD@Z 004709f5 f   libcpmt:locale0.obj
 0001:0006fa3f       __Tolower                  00470a3f f   libcpmt:_tolower.obj
 0001:0006fb4e       __Getctype                 00470b4e f   libcpmt:_tolower.obj
 0001:0006fba9       __Toupper                  00470ba9 f   libcpmt:_toupper.obj
 0001:0006fcbd       ?_Xfsopen@std@@YAPAU_iobuf@@PB_W0H@Z 00470cbd f   libcpmt:fiopen.obj
 0001:0006fd72       ?_Fiopen@std@@YAPAU_iobuf@@PB_WHH@Z 00470d72 f   libcpmt:fiopen.obj
 0001:0006fe27       ?_Fiopen@std@@YAPAU_iobuf@@PBDHH@Z 00470e27 f   libcpmt:fiopen.obj
 0001:0006fe82       __Mtxinit                  00470e82 f   libcpmt:xmtx.obj
 0001:0006fe8d       __Mtxdst                   00470e8d f   libcpmt:xmtx.obj
 0001:0006fe98       __Mtxlock                  00470e98 f   libcpmt:xmtx.obj
 0001:0006fea3       __Mtxunlock                00470ea3 f   libcpmt:xmtx.obj
 0001:0006feae       ?_Atexit@@YAXP6AXXZ@Z      00470eae f   libcpmt:iosptrs.obj
 0001:0006fece       ??1_Init_atexit@@QAE@XZ    00470ece f i libcpmt:iosptrs.obj
 0001:0006fef4       _RtlUnwind@16              00470ef4 f   kernel32:KERNEL32.dll
 0001:0006ff00       ?ImageFormatInfo@ImageLoader@@YAABUImageFormatInfo_t@@W4ImageFormat@@@Z 00470f00 f   bitmap:imageformat.obj
 0001:0006ff20       ?GetNumMipMapLevels@ImageLoader@@YAHHHH@Z 00470f20 f   bitmap:imageformat.obj
 0001:0006ff90       ?GetMemRequired@ImageLoader@@YAHHHHW4ImageFormat@@_N@Z 00470f90 f   bitmap:imageformat.obj
 0001:000700d0       ??4BGRA5551_t@@QAEAAU0@ABUBGRA8888_t@@@Z 004710d0 f i bitmap:colorconversion.obj
 0001:00070150       ??4BGRA4444_t@@QAEAAU0@ABUBGRA8888_t@@@Z 00471150 f i bitmap:colorconversion.obj
 0001:000701d0       ?ConvertFloatTo16bits@float16@@KAGM@Z 004711d0 f i bitmap:colorconversion.obj
 0001:00070310       ?Convert16bitFloatTo32bits@float16@@KAMG@Z 00471310 f i bitmap:colorconversion.obj
 0001:000703e0       ?PixRGBAF_to_8@@YA?AUPixRGBA8@@ABUPixRGBAF@@@Z 004713e0 f i bitmap:colorconversion.obj
 0001:00070750       ?ConvertToATIxN@ImageLoader@@YA_NPBEW4ImageFormat@@PAE1HHHH@Z 00471750 f   bitmap:colorconversion.obj
 0001:00070860       ?ConvertToDXT@ImageLoader@@YA_NPBEW4ImageFormat@@PAE1HHHH@Z 00471860 f   bitmap:colorconversion.obj
 0001:00070a40       ?ConvertImageFormat_RGBA16161616_To_RGB323232F@ImageLoader@@YAXPAGPAMHH@Z 00471a40 f   bitmap:colorconversion.obj
 0001:00070ba0       ?ConvertImageFormat_RGB323232F_To_RGBA16161616@ImageLoader@@YAXPAMPAGHH@Z 00471ba0 f   bitmap:colorconversion.obj
 0001:00070cb0       ?ConvertImageFormat_RGB323232F_To_RGBA8888@ImageLoader@@YAXPAMPAEHH@Z 00471cb0 f   bitmap:colorconversion.obj
 0001:00070f70       ?ConvertImageFormat_RGB323232F_To_BGRA8888@ImageLoader@@YAXPAMPAEHH@Z 00471f70 f   bitmap:colorconversion.obj
 0001:00071230       ?ConvertNormalMapRGBA8888ToDUDVMapUVWQ8888@ImageLoader@@YAXPBEHHPAE@Z 00472230 f   bitmap:colorconversion.obj
 0001:00071290       ?ConvertNormalMapRGBA8888ToDUDVMapUVLX8888@ImageLoader@@YAXPBEHHPAE@Z 00472290 f   bitmap:colorconversion.obj
 0001:000712e0       ?ConvertNormalMapRGBA8888ToDUDVMapUV88@ImageLoader@@YAXPBEHHPAE@Z 004722e0 f   bitmap:colorconversion.obj
 0001:00071320       ?NormalizeNormalMapRGBA8888@ImageLoader@@YAXPAEH@Z 00472320 f   bitmap:colorconversion.obj
 0001:00071450       ?RotateImageLeft@ImageLoader@@YA_NPBEPAEHW4ImageFormat@@@Z 00472450 f   bitmap:colorconversion.obj
 0001:00071600       ?RotateImage180@ImageLoader@@YA_NPBEPAEHW4ImageFormat@@@Z 00472600 f   bitmap:colorconversion.obj
 0001:00071640       ?FlipImageVertically@ImageLoader@@YA_NPAX0HHW4ImageFormat@@H@Z 00472640 f   bitmap:colorconversion.obj
 0001:00071720       ?FlipImageHorizontally@ImageLoader@@YA_NPAX0HHW4ImageFormat@@H@Z 00472720 f   bitmap:colorconversion.obj
 0001:000739d0       ?ConvertImageFormat_RGBA16161616F_To_RGB323232F@ImageLoader@@YAXPAVfloat16@@PAMHH@Z 004749d0 f   bitmap:colorconversion.obj
 0001:00073a30       ?ConvertImageFormat_RGBA16161616F_To_RGBA323232F@ImageLoader@@YAXPAVfloat16@@PAMHHI@Z 00474a30 f   bitmap:colorconversion.obj
 0001:00073ad0       ?ConvertImageFormat_RGB323232F_To_RGBA16161616F@ImageLoader@@YAXPAMPAVfloat16@@HH@Z 00474ad0 f   bitmap:colorconversion.obj
 0001:00073b30       ?ConvertImageFormat_RGBA16161616_To_RGBA16161616F@ImageLoader@@YAXPAGPAMHH@Z 00474b30 f   bitmap:colorconversion.obj
 0001:00073bf0       ?ConvertImageFormat_RGBA16161616F_To_RGBA16161616@ImageLoader@@YAXPAVfloat16@@PAGHH@Z 00474bf0 f   bitmap:colorconversion.obj
 0001:000750e0       ?ConvertImageFormat@ImageLoader@@YA_NPBEW4ImageFormat@@PAE1HHHH@Z 004760e0 f   bitmap:colorconversion.obj
 0001:00075850       ?ConstructGammaTable@ImageLoader@@YAXPAEMM@Z 00476850 f   bitmap:resample.obj
 0001:000758c0       ?GammaCorrectRGBA8888@ImageLoader@@YAXPAE0HHH0@Z 004768c0 f   bitmap:resample.obj
 0001:000759a0       ?GammaCorrectRGBA8888@ImageLoader@@YAXPAE0HHHMM@Z 004769a0 f   bitmap:resample.obj
 0001:00075e00       ?ResampleRGBA8888@ImageLoader@@YA_NABUResampleInfo_t@1@@Z 00476e00 f   bitmap:resample.obj
 0001:000761c0       ?ResampleRGB323232F@ImageLoader@@YA_NABUResampleInfo_t@1@@Z 004771c0 f   bitmap:resample.obj
 0001:00076360       ?ComputeAveragedColor@?$CKernelWrapper@$0A@$0A@@ImageLoader@@SAXABUKernelInfo_t@2@ABUResampleInfo_t@2@HHHPAM2@Z 00477360 f i bitmap:resample.obj
 0001:00076530       ?ComputeAveragedColor@?$CKernelWrapper@$00$0A@@ImageLoader@@SAXABUKernelInfo_t@2@ABUResampleInfo_t@2@HHHPAM2@Z 00477530 f i bitmap:resample.obj
 0001:00076700       ?ComputeAveragedColor@?$CKernelWrapper@$01$0A@@ImageLoader@@SAXABUKernelInfo_t@2@ABUResampleInfo_t@2@HHHPAM2@Z 00477700 f i bitmap:resample.obj
 0001:000768b0       ?AddAlphaToAlphaResult@?$CKernelWrapper@$01$0A@@ImageLoader@@SAXABUKernelInfo_t@2@ABUResampleInfo_t@2@HHHMPAM@Z 004778b0 f i bitmap:resample.obj
 0001:000769f0       ?AdjustAlphaChannel@?$CKernelWrapper@$01$0A@@ImageLoader@@SAXABUKernelInfo_t@2@ABUResampleInfo_t@2@HHHPAM@Z 004779f0 f i bitmap:resample.obj
 0001:000769f0       ?AdjustAlphaChannel@?$CKernelWrapper@$01$00@ImageLoader@@SAXABUKernelInfo_t@2@ABUResampleInfo_t@2@HHHPAM@Z 004779f0 f i bitmap:resample.obj
 0001:00076e50       ?ComputeAveragedColor@?$CKernelWrapper@$0A@$00@ImageLoader@@SAXABUKernelInfo_t@2@ABUResampleInfo_t@2@HHHPAM2@Z 00477e50 f i bitmap:resample.obj
 0001:00077030       ?ComputeAveragedColor@?$CKernelWrapper@$00$00@ImageLoader@@SAXABUKernelInfo_t@2@ABUResampleInfo_t@2@HHHPAM2@Z 00478030 f i bitmap:resample.obj
 0001:00077210       ?ComputeAveragedColor@?$CKernelWrapper@$01$00@ImageLoader@@SAXABUKernelInfo_t@2@ABUResampleInfo_t@2@HHHPAM2@Z 00478210 f i bitmap:resample.obj
 0001:00077400       ?AddAlphaToAlphaResult@?$CKernelWrapper@$01$00@ImageLoader@@SAXABUKernelInfo_t@2@ABUResampleInfo_t@2@HHHMPAM@Z 00478400 f i bitmap:resample.obj
 0001:00077570       ?ApplyKernel@?$CKernelWrapper@$0A@$0A@@ImageLoader@@SAXABUKernelInfo_t@2@ABUResampleInfo_t@2@HHHPAM2@Z 00478570 f i bitmap:resample.obj
 0001:00077750       ?ApplyKernel@?$CKernelWrapper@$00$0A@@ImageLoader@@SAXABUKernelInfo_t@2@ABUResampleInfo_t@2@HHHPAM2@Z 00478750 f i bitmap:resample.obj
 0001:000778d0       ?ApplyKernel@?$CKernelWrapper@$01$0A@@ImageLoader@@SAXABUKernelInfo_t@2@ABUResampleInfo_t@2@HHHPAM2@Z 004788d0 f i bitmap:resample.obj
 0001:00077b40       ?ApplyKernel@?$CKernelWrapper@$0A@$00@ImageLoader@@SAXABUKernelInfo_t@2@ABUResampleInfo_t@2@HHHPAM2@Z 00478b40 f i bitmap:resample.obj
 0001:00077d20       ?ApplyKernel@?$CKernelWrapper@$00$00@ImageLoader@@SAXABUKernelInfo_t@2@ABUResampleInfo_t@2@HHHPAM2@Z 00478d20 f i bitmap:resample.obj
 0001:00077ea0       ?ApplyKernel@?$CKernelWrapper@$01$00@ImageLoader@@SAXABUKernelInfo_t@2@ABUResampleInfo_t@2@HHHPAM2@Z 00478ea0 f i bitmap:resample.obj
 0001:00078110       ?GenerateMipmapLevels@ImageLoader@@YAXPAE0HHHW4ImageFormat@@MMH@Z 00479110 f   bitmap:resample.obj
 0001:000782b0       ?GetProcessorCount@@YAKXZ  004792b0 f   bitmap:ATI_Compress.obj
 0001:000782d0       ?GetCodecType@@YA?AW4_CodecType@@W4ATI_TC_FORMAT@@@Z 004792d0 f   bitmap:ATI_Compress.obj
 0001:00078380       ?GetError@@YA?AW4ATI_TC_ERROR@@W4_CODECError@@@Z 00479380 f   bitmap:ATI_Compress.obj
 0001:000783b0       ?CalcBufferSize@@YAKW4ATI_TC_FORMAT@@KKK@Z 004793b0 f   bitmap:ATI_Compress.obj
 0001:00078440       ?CompressTexture@@YA?AW4ATI_TC_ERROR@@PBU_ATI_TC_Texture@@PAU2@PBU_ATI_TC_CompressOptions@@P6A_NMKK@ZKKW4_CodecType@@@Z 00479440 f   bitmap:ATI_Compress.obj
 0001:000786d0       ??0CATICompressThreadData@@QAE@XZ 004796d0 f   bitmap:ATI_Compress.obj
 0001:000786e0       ??1CATICompressThreadData@@QAE@XZ 004796e0 f   bitmap:ATI_Compress.obj
 0001:00078730       ?ThreadedCompressProc@@YGKPAX@Z 00479730 f   bitmap:ATI_Compress.obj
 0001:00078790       ?ThreadedCompressTexture@@YA?AW4ATI_TC_ERROR@@PBU_ATI_TC_Texture@@PAU2@PBU_ATI_TC_CompressOptions@@P6A_NMKK@ZKKW4_CodecType@@@Z 00479790 f   bitmap:ATI_Compress.obj
 0001:00078c10       _ATI_TC_CalculateBufferSize 00479c10 f   bitmap:ATI_Compress.obj
 0001:00078c50       ?CheckTexture@@YA?AW4ATI_TC_ERROR@@PBU_ATI_TC_Texture@@_N@Z 00479c50 f   bitmap:ATI_Compress.obj
 0001:00078cd0       _ATI_TC_ConvertTexture     00479cd0 f   bitmap:ATI_Compress.obj
 0001:00079220       ?S3TCencode@@YAXPAU_DDSURFACEDESC@@PAUtagPALETTEENTRY@@0PAXIPAM@Z 0047a220 f   bitmap:S3_intrf.obj
 0001:00079f40       ??0FloatBitMap_t@@QAE@HH@Z 0047af40 f   bitmap:float_bm.obj
 0001:00079f90       ??1FloatBitMap_t@@QAE@XZ   0047af90 f   bitmap:float_bm.obj
 0001:00079fa0       ?CompressTo8Bits@FloatBitMap_t@@QAEXM@Z 0047afa0 f   bitmap:float_bm2.obj
 0001:0007a290       ??0CCodec@ATI_Compress@@QAE@W4_CodecType@@@Z 0047b290 f   bitmap:Codec.obj
 0001:0007a2b0       ??1CCodec@ATI_Compress@@UAE@XZ 0047b2b0 f   bitmap:Codec.obj
 0001:0007a2c0       ?SetParameter@CCodec@ATI_Compress@@UAE_NPBDK@Z 0047b2c0 f   bitmap:Codec.obj
 0001:0007a2d0       ?GetParameter@CCodec@ATI_Compress@@UAE_NPBDAAK@Z 0047b2d0 f   bitmap:Codec.obj
 0001:0007a2e0       ?SetParameter@CCodec@ATI_Compress@@UAE_NPBDM@Z 0047b2e0 f   bitmap:Codec.obj
 0001:0007a2f0       ?GetParameter@CCodec@ATI_Compress@@UAE_NPBDAAM@Z 0047b2f0 f   bitmap:Codec.obj
 0001:0007a300       ?SupportsSSE2@@YA_NXZ      0047b300 f   bitmap:Codec.obj
 0001:0007a310       ?CreateCodec@@YAPAVCCodec@ATI_Compress@@W4_CodecType@@@Z 0047b310 f   bitmap:Codec.obj
 0001:0007a640       ?CalcBufferSize@@YAKW4_CodecType@@KK@Z 0047b640 f   bitmap:Codec.obj
 0001:0007a6b0       ?DeriveB@@YAEEE@Z          0047b6b0 f   bitmap:Codec.obj
 0001:0007a7c0       ?DeriveB@@YAMMM@Z          0047b7c0 f   bitmap:Codec.obj
 0001:0007a850       ??_GCCodec@ATI_Compress@@UAEPAXI@Z 0047b850 f i bitmap:Codec.obj
 0001:0007a850       ??_ECCodec@ATI_Compress@@UAEPAXI@Z 0047b850 f i bitmap:Codec.obj
 0001:0007a870       ??0half@@QAE@M@Z           0047b870 f i bitmap:CodecBuffer.obj
 0001:0007a8e0       ?CreateCodecBuffer@@YAPAVCCodecBuffer@@W4_CodecBufferType@@KKKPAE@Z 0047b8e0 f   bitmap:CodecBuffer.obj
 0001:0007ab10       ??0CCodecBuffer@@QAE@KKKPAE@Z 0047bb10 f   bitmap:CodecBuffer.obj
 0001:0007ab50       ??1CCodecBuffer@@UAE@XZ    0047bb50 f   bitmap:CodecBuffer.obj
 0001:0007ab80       ?Copy@CCodecBuffer@@UAEXAAV1@@Z 0047bb80 f   bitmap:CodecBuffer.obj
 0001:0007ac40       ?WriteBlock@CCodecBuffer@@UAE_NKKPAKK@Z 0047bc40 f   bitmap:CodecBuffer.obj
 0001:0007ac50       ?ReadBlock@CCodecBuffer@@UAE_NKKPAKK@Z 0047bc50 f   bitmap:CodecBuffer.obj
 0001:0007ac60       ?ConvertBlock@CCodecBuffer@@IAEXQANQAMK@Z 0047bc60 f   bitmap:CodecBuffer.obj
 0001:0007ace0       ?ConvertBlock@CCodecBuffer@@IAEXQANQAVhalf@@K@Z 0047bce0 f   bitmap:CodecBuffer.obj
 0001:0007ad90       ?ConvertBlock@CCodecBuffer@@IAEXQANQAGK@Z 0047bd90 f   bitmap:CodecBuffer.obj
 0001:0007ae60       ?ConvertBlock@CCodecBuffer@@IAEXQANQAEK@Z 0047be60 f   bitmap:CodecBuffer.obj
 0001:0007af20       ?ConvertBlock@CCodecBuffer@@IAEXQAMQANK@Z 0047bf20 f   bitmap:CodecBuffer.obj
 0001:0007afa0       ?ConvertBlock@CCodecBuffer@@IAEXQAMQAVhalf@@K@Z 0047bfa0 f   bitmap:CodecBuffer.obj
 0001:0007b050       ?ConvertBlock@CCodecBuffer@@IAEXQAMQAGK@Z 0047c050 f   bitmap:CodecBuffer.obj
 0001:0007b120       ?ConvertBlock@CCodecBuffer@@IAEXQAMQAEK@Z 0047c120 f   bitmap:CodecBuffer.obj
 0001:0007b1e0       ?ConvertBlock@CCodecBuffer@@IAEXQAVhalf@@QANK@Z 0047c1e0 f   bitmap:CodecBuffer.obj
 0001:0007b230       ?ConvertBlock@CCodecBuffer@@IAEXQAVhalf@@QAMK@Z 0047c230 f   bitmap:CodecBuffer.obj
 0001:0007b280       ?ConvertBlock@CCodecBuffer@@IAEXQAVhalf@@QAGK@Z 0047c280 f   bitmap:CodecBuffer.obj
 0001:0007b2e0       ?ConvertBlock@CCodecBuffer@@IAEXQAVhalf@@QAEK@Z 0047c2e0 f   bitmap:CodecBuffer.obj
 0001:0007b340       ?ConvertBlock@CCodecBuffer@@IAEXQAGQANK@Z 0047c340 f   bitmap:CodecBuffer.obj
 0001:0007b3b0       ?ConvertBlock@CCodecBuffer@@IAEXQAGQAMK@Z 0047c3b0 f   bitmap:CodecBuffer.obj
 0001:0007b420       ?ConvertBlock@CCodecBuffer@@IAEXQAGQAVhalf@@K@Z 0047c420 f   bitmap:CodecBuffer.obj
 0001:0007b490       ?ConvertBlock@CCodecBuffer@@IAEXQAGQAEK@Z 0047c490 f   bitmap:CodecBuffer.obj
 0001:0007b4d0       ?ConvertBlock@CCodecBuffer@@IAEXQAEQANK@Z 0047c4d0 f   bitmap:CodecBuffer.obj
 0001:0007b540       ?ConvertBlock@CCodecBuffer@@IAEXQAEQAMK@Z 0047c540 f   bitmap:CodecBuffer.obj
 0001:0007b5b0       ?ConvertBlock@CCodecBuffer@@IAEXQAEQAVhalf@@K@Z 0047c5b0 f   bitmap:CodecBuffer.obj
 0001:0007b630       ?ConvertBlock@CCodecBuffer@@IAEXQAEQAGK@Z 0047c630 f   bitmap:CodecBuffer.obj
 0001:0007b6b0       ?SwizzleBlock@CCodecBuffer@@IAEXQANK@Z 0047c6b0 f   bitmap:CodecBuffer.obj
 0001:0007b750       ?SwizzleBlock@CCodecBuffer@@IAEXQAMK@Z 0047c750 f   bitmap:CodecBuffer.obj
 0001:0007b810       ?SwizzleBlock@CCodecBuffer@@IAEXQAVhalf@@K@Z 0047c810 f   bitmap:CodecBuffer.obj
 0001:0007b850       ?SwizzleBlock@CCodecBuffer@@IAEXQAGK@Z 0047c850 f   bitmap:CodecBuffer.obj
 0001:0007b890       ?ReadBlockR@CCodecBuffer@@UAE_NKKEEQAE@Z 0047c890 f   bitmap:CodecBuffer.obj
 0001:0007ba50       ?ReadBlockG@CCodecBuffer@@UAE_NKKEEQAE@Z 0047ca50 f   bitmap:CodecBuffer.obj
 0001:0007bc10       ?ReadBlockB@CCodecBuffer@@UAE_NKKEEQAE@Z 0047cc10 f   bitmap:CodecBuffer.obj
 0001:0007bdd0       ?ReadBlockA@CCodecBuffer@@UAE_NKKEEQAE@Z 0047cdd0 f   bitmap:CodecBuffer.obj
 0001:0007bf90       ?ReadBlockR@CCodecBuffer@@UAE_NKKEEQAG@Z 0047cf90 f   bitmap:CodecBuffer.obj
 0001:0007c170       ?ReadBlockG@CCodecBuffer@@UAE_NKKEEQAG@Z 0047d170 f   bitmap:CodecBuffer.obj
 0001:0007c350       ?ReadBlockB@CCodecBuffer@@UAE_NKKEEQAG@Z 0047d350 f   bitmap:CodecBuffer.obj
 0001:0007c530       ?ReadBlockA@CCodecBuffer@@UAE_NKKEEQAG@Z 0047d530 f   bitmap:CodecBuffer.obj
 0001:0007c710       ?ReadBlockR@CCodecBuffer@@UAE_NKKEEQAVhalf@@@Z 0047d710 f   bitmap:CodecBuffer.obj
 0001:0007c910       ?ReadBlockG@CCodecBuffer@@UAE_NKKEEQAVhalf@@@Z 0047d910 f   bitmap:CodecBuffer.obj
 0001:0007cb10       ?ReadBlockB@CCodecBuffer@@UAE_NKKEEQAVhalf@@@Z 0047db10 f   bitmap:CodecBuffer.obj
 0001:0007cd10       ?ReadBlockA@CCodecBuffer@@UAE_NKKEEQAVhalf@@@Z 0047dd10 f   bitmap:CodecBuffer.obj
 0001:0007cf10       ?ReadBlockR@CCodecBuffer@@UAE_NKKEEQAM@Z 0047df10 f   bitmap:CodecBuffer.obj
 0001:0007d070       ?ReadBlockG@CCodecBuffer@@UAE_NKKEEQAM@Z 0047e070 f   bitmap:CodecBuffer.obj
 0001:0007d1d0       ?ReadBlockB@CCodecBuffer@@UAE_NKKEEQAM@Z 0047e1d0 f   bitmap:CodecBuffer.obj
 0001:0007d330       ?ReadBlockA@CCodecBuffer@@UAE_NKKEEQAM@Z 0047e330 f   bitmap:CodecBuffer.obj
 0001:0007d490       ?ReadBlockR@CCodecBuffer@@UAE_NKKEEQAN@Z 0047e490 f   bitmap:CodecBuffer.obj
 0001:0007d5e0       ?ReadBlockG@CCodecBuffer@@UAE_NKKEEQAN@Z 0047e5e0 f   bitmap:CodecBuffer.obj
 0001:0007d730       ?ReadBlockB@CCodecBuffer@@UAE_NKKEEQAN@Z 0047e730 f   bitmap:CodecBuffer.obj
 0001:0007d880       ?ReadBlockA@CCodecBuffer@@UAE_NKKEEQAN@Z 0047e880 f   bitmap:CodecBuffer.obj
 0001:0007d9d0       ?WriteBlockR@CCodecBuffer@@UAE_NKKEEQAE@Z 0047e9d0 f   bitmap:CodecBuffer.obj
 0001:0007db50       ?WriteBlockG@CCodecBuffer@@UAE_NKKEEQAE@Z 0047eb50 f   bitmap:CodecBuffer.obj
 0001:0007dcd0       ?WriteBlockB@CCodecBuffer@@UAE_NKKEEQAE@Z 0047ecd0 f   bitmap:CodecBuffer.obj
 0001:0007de60       ?WriteBlockA@CCodecBuffer@@UAE_NKKEEQAE@Z 0047ee60 f   bitmap:CodecBuffer.obj
 0001:0007dff0       ?WriteBlockR@CCodecBuffer@@UAE_NKKEEQAG@Z 0047eff0 f   bitmap:CodecBuffer.obj
 0001:0007e180       ?WriteBlockG@CCodecBuffer@@UAE_NKKEEQAG@Z 0047f180 f   bitmap:CodecBuffer.obj
 0001:0007e310       ?WriteBlockB@CCodecBuffer@@UAE_NKKEEQAG@Z 0047f310 f   bitmap:CodecBuffer.obj
 0001:0007e4b0       ?WriteBlockA@CCodecBuffer@@UAE_NKKEEQAG@Z 0047f4b0 f   bitmap:CodecBuffer.obj
 0001:0007e650       ?WriteBlockR@CCodecBuffer@@UAE_NKKEEQAVhalf@@@Z 0047f650 f   bitmap:CodecBuffer.obj
 0001:0007e790       ?WriteBlockG@CCodecBuffer@@UAE_NKKEEQAVhalf@@@Z 0047f790 f   bitmap:CodecBuffer.obj
 0001:0007e8d0       ?WriteBlockB@CCodecBuffer@@UAE_NKKEEQAVhalf@@@Z 0047f8d0 f   bitmap:CodecBuffer.obj
 0001:0007ea10       ?WriteBlockA@CCodecBuffer@@UAE_NKKEEQAVhalf@@@Z 0047fa10 f   bitmap:CodecBuffer.obj
 0001:0007eb50       ?WriteBlockR@CCodecBuffer@@UAE_NKKEEQAM@Z 0047fb50 f   bitmap:CodecBuffer.obj
 0001:0007ed40       ?WriteBlockG@CCodecBuffer@@UAE_NKKEEQAM@Z 0047fd40 f   bitmap:CodecBuffer.obj
 0001:0007ef40       ?WriteBlockB@CCodecBuffer@@UAE_NKKEEQAM@Z 0047ff40 f   bitmap:CodecBuffer.obj
 0001:0007f140       ?WriteBlockA@CCodecBuffer@@UAE_NKKEEQAM@Z 00480140 f   bitmap:CodecBuffer.obj
 0001:0007f340       ?WriteBlockR@CCodecBuffer@@UAE_NKKEEQAN@Z 00480340 f   bitmap:CodecBuffer.obj
 0001:0007f520       ?WriteBlockG@CCodecBuffer@@UAE_NKKEEQAN@Z 00480520 f   bitmap:CodecBuffer.obj
 0001:0007f700       ?WriteBlockB@CCodecBuffer@@UAE_NKKEEQAN@Z 00480700 f   bitmap:CodecBuffer.obj
 0001:0007f8f0       ?WriteBlockA@CCodecBuffer@@UAE_NKKEEQAN@Z 004808f0 f   bitmap:CodecBuffer.obj
 0001:0007fae0       ?WriteBlockRGBA@CCodecBuffer@@UAE_NKKEEQAK@Z 00480ae0 f   bitmap:CodecBuffer.obj
 0001:0007fcd0       ?ReadBlockRGBA@CCodecBuffer@@UAE_NKKEEQAK@Z 00480cd0 f   bitmap:CodecBuffer.obj
 0001:0007fed0       ?WriteBlockRGBA@CCodecBuffer@@UAE_NKKEEQAG@Z 00480ed0 f   bitmap:CodecBuffer.obj
 0001:00080060       ?ReadBlockRGBA@CCodecBuffer@@UAE_NKKEEQAG@Z 00481060 f   bitmap:CodecBuffer.obj
 0001:00080220       ?WriteBlockRGBA@CCodecBuffer@@UAE_NKKEEQAVhalf@@@Z 00481220 f   bitmap:CodecBuffer.obj
 0001:000803b0       ?ReadBlockRGBA@CCodecBuffer@@UAE_NKKEEQAVhalf@@@Z 004813b0 f   bitmap:CodecBuffer.obj
 0001:00080570       ?WriteBlockRGBA@CCodecBuffer@@UAE_NKKEEQAM@Z 00481570 f   bitmap:CodecBuffer.obj
 0001:00080700       ?ReadBlockRGBA@CCodecBuffer@@UAE_NKKEEQAM@Z 00481700 f   bitmap:CodecBuffer.obj
 0001:000808c0       ?WriteBlockRGBA@CCodecBuffer@@UAE_NKKEEQAN@Z 004818c0 f   bitmap:CodecBuffer.obj
 0001:00080a50       ?ReadBlockRGBA@CCodecBuffer@@UAE_NKKEEQAN@Z 00481a50 f   bitmap:CodecBuffer.obj
 0001:00080c10       ?sync@?$basic_streambuf@DU?$char_traits@D@std@@@std@@MAEHXZ 00481c10 f i chunkfile.obj
 0001:00080c10       ?GetBufferType@CCodecBuffer@@UBE?BW4_CodecBufferType@@XZ 00481c10 f i bitmap:CodecBuffer.obj
 0001:00080c10       ?showmanyc@?$basic_streambuf@DU?$char_traits@D@std@@@std@@MAEHXZ 00481c10 f i chunkfile.obj
 0001:00080c10       __wcsdup                   00481c10 f i memoverride.obj
 0001:00080c20       ??_GCCodecBuffer@@UAEPAXI@Z 00481c20 f i bitmap:CodecBuffer.obj
 0001:00080c20       ??_ECCodecBuffer@@UAEPAXI@Z 00481c20 f i bitmap:CodecBuffer.obj
 0001:00080c60       _CodeRGBBlock              00481c60 f   bitmap:S3_quant.obj
 0001:00083c80       _CodeAlphaBlock            00484c80 f   bitmap:S3_quant.obj
 0001:00084a30       ??0CCodec_ATI2N_DXT5@@QAE@XZ 00485a30 f   bitmap:Codec_ATI2N_DXT5.obj
 0001:00084a50       ??1CCodec_ATI2N_DXT5@@UAE@XZ 00485a50 f   bitmap:Codec_ATI2N_DXT5.obj
 0001:00084a60       ?Compress@CCodec_ATI2N_DXT5@@UAE?AW4_CODECError@@AAVCCodecBuffer@@0P6A_NMKK@ZKK@Z 00485a60 f   bitmap:Codec_ATI2N_DXT5.obj
 0001:00084cf0       ?Decompress@CCodec_ATI2N_DXT5@@UAE?AW4_CODECError@@AAVCCodecBuffer@@0@Z 00485cf0 f   bitmap:Codec_ATI2N_DXT5.obj
 0001:00084ee0       ?GetBlockHeight@CCodec_Block_4x4@@UAEKXZ 00485ee0 f i bitmap:Codec_ATI2N_DXT5.obj
 0001:00084ee0       ?GetBufferType@CCodecBuffer_RGBA16F@@UBE?BW4_CodecBufferType@@XZ 00485ee0 f i bitmap:CodecBuffer_RGBA16F.obj
 0001:00084ef0       ??_GCCodec_ATI2N_DXT5@@UAEPAXI@Z 00485ef0 f i bitmap:Codec_ATI2N_DXT5.obj
 0001:00084ef0       ??_ECCodec_ATI2N_DXT5@@UAEPAXI@Z 00485ef0 f i bitmap:Codec_ATI2N_DXT5.obj
 0001:00084f20       ??0CCodec_ATI2N@@QAE@W4_CodecType@@@Z 00485f20 f   bitmap:Codec_ATI2N.obj
 0001:00084f40       ??1CCodec_ATI2N@@UAE@XZ    00485f40 f   bitmap:Codec_ATI2N.obj
 0001:00084f50       ?Compress@CCodec_ATI2N@@UAE?AW4_CODECError@@AAVCCodecBuffer@@0P6A_NMKK@ZKK@Z 00485f50 f   bitmap:Codec_ATI2N.obj
 0001:000851c0       ?Decompress@CCodec_ATI2N@@UAE?AW4_CODECError@@AAVCCodecBuffer@@0@Z 004861c0 f   bitmap:Codec_ATI2N.obj
 0001:00085490       ?DeriveBlockB@CCodec_ATI2N@@MAEXQAE00@Z 00486490 f   bitmap:Codec_ATI2N.obj
 0001:000854e0       ?DeriveBlockB@CCodec_ATI2N@@MAEXQAM00@Z 004864e0 f   bitmap:Codec_ATI2N.obj
 0001:00085530       ??_ECCodec_ATI2N@@UAEPAXI@Z 00486530 f i bitmap:Codec_ATI2N.obj
 0001:00085530       ??_GCCodec_ATI2N@@UAEPAXI@Z 00486530 f i bitmap:Codec_ATI2N.obj
 0001:00085560       ??0CCodec_ATI1N@@QAE@W4_CodecType@@@Z 00486560 f   bitmap:Codec_ATI1N.obj
 0001:00085580       ??1CCodec_ATI1N@@UAE@XZ    00486580 f   bitmap:Codec_ATI1N.obj
 0001:00085590       ?CreateBuffer@CCodec_ATI1N@@UBEPAVCCodecBuffer@@KKKPAE@Z 00486590 f   bitmap:Codec_ATI1N.obj
 0001:000855c0       ?Compress@CCodec_ATI1N@@UAE?AW4_CODECError@@AAVCCodecBuffer@@0P6A_NMKK@ZKK@Z 004865c0 f   bitmap:Codec_ATI1N.obj
 0001:000857b0       ?Decompress@CCodec_ATI1N@@UAE?AW4_CODECError@@AAVCCodecBuffer@@0@Z 004867b0 f   bitmap:Codec_ATI1N.obj
 0001:00085990       ??_GCCodec_ATI1N@@UAEPAXI@Z 00486990 f i bitmap:Codec_ATI1N.obj
 0001:00085990       ??_ECCodec_ATI1N@@UAEPAXI@Z 00486990 f i bitmap:Codec_ATI1N.obj
 0001:000859c0       ??0CCodec_DXT5_xGxR@@QAE@XZ 004869c0 f   bitmap:Codec_DXT5_xGxR.obj
 0001:000859e0       ??1CCodec_DXT5_xGxR@@UAE@XZ 004869e0 f   bitmap:Codec_DXT5_xGxR.obj
 0001:000859f0       ?ReadBlock@CCodec_DXT5_xGxR@@MAEXAAVCCodecBuffer@@KKQAK@Z 004869f0 f   bitmap:Codec_DXT5_xGxR.obj
 0001:00085ab0       ?WriteBlock@CCodec_DXT5_xGxR@@MAEXAAVCCodecBuffer@@KKQAK@Z 00486ab0 f   bitmap:Codec_DXT5_xGxR.obj
 0001:00085b70       ?ReadBlock@CCodec_DXT5_xGxR@@MAEXAAVCCodecBuffer@@KKQAM@Z 00486b70 f   bitmap:Codec_DXT5_xGxR.obj
 0001:00085be0       ?WriteBlock@CCodec_DXT5_xGxR@@MAEXAAVCCodecBuffer@@KKQAM@Z 00486be0 f   bitmap:Codec_DXT5_xGxR.obj
 0001:00085c60       ??_ECCodec_DXT5_xGxR@@UAEPAXI@Z 00486c60 f i bitmap:Codec_DXT5_xGxR.obj
 0001:00085c60       ??_GCCodec_DXT5_xGxR@@UAEPAXI@Z 00486c60 f i bitmap:Codec_DXT5_xGxR.obj
 0001:00085c90       ??0CCodec_DXT5_RGxB@@QAE@XZ 00486c90 f   bitmap:Codec_DXT5_RGxB.obj
 0001:00085cb0       ??1CCodec_DXT5_RGxB@@UAE@XZ 00486cb0 f   bitmap:Codec_DXT5_RGxB.obj
 0001:00085cc0       ?ReadBlock@CCodec_DXT5_RGxB@@MAEXAAVCCodecBuffer@@KKQAK@Z 00486cc0 f   bitmap:Codec_DXT5_RGxB.obj
 0001:00085dc0       ?WriteBlock@CCodec_DXT5_RGxB@@MAEXAAVCCodecBuffer@@KKQAK@Z 00486dc0 f   bitmap:Codec_DXT5_RGxB.obj
 0001:00085ea0       ?ReadBlock@CCodec_DXT5_RGxB@@MAEXAAVCCodecBuffer@@KKQAM@Z 00486ea0 f   bitmap:Codec_DXT5_RGxB.obj
 0001:00085f20       ?WriteBlock@CCodec_DXT5_RGxB@@MAEXAAVCCodecBuffer@@KKQAM@Z 00486f20 f   bitmap:Codec_DXT5_RGxB.obj
 0001:00085fb0       ??_GCCodec_DXT5_RGxB@@UAEPAXI@Z 00486fb0 f i bitmap:Codec_DXT5_RGxB.obj
 0001:00085fb0       ??_ECCodec_DXT5_RGxB@@UAEPAXI@Z 00486fb0 f i bitmap:Codec_DXT5_RGxB.obj
 0001:00085fe0       ??0CCodec_DXT5_xRBG@@QAE@XZ 00486fe0 f   bitmap:Codec_DXT5_xRBG.obj
 0001:00086000       ??1CCodec_DXT5_xRBG@@UAE@XZ 00487000 f   bitmap:Codec_DXT5_xRBG.obj
 0001:00086010       ?ReadBlock@CCodec_DXT5_xRBG@@MAEXAAVCCodecBuffer@@KKQAK@Z 00487010 f   bitmap:Codec_DXT5_xRBG.obj
 0001:00086100       ?WriteBlock@CCodec_DXT5_xRBG@@MAEXAAVCCodecBuffer@@KKQAK@Z 00487100 f   bitmap:Codec_DXT5_xRBG.obj
 0001:000861e0       ?ReadBlock@CCodec_DXT5_xRBG@@MAEXAAVCCodecBuffer@@KKQAM@Z 004871e0 f   bitmap:Codec_DXT5_xRBG.obj
 0001:00086260       ?WriteBlock@CCodec_DXT5_xRBG@@MAEXAAVCCodecBuffer@@KKQAM@Z 00487260 f   bitmap:Codec_DXT5_xRBG.obj
 0001:000862e0       ?SetParameter@CCodec_DXT5_xRBG@@UAE_NPBDM@Z 004872e0 f   bitmap:Codec_DXT5_xRBG.obj
 0001:00086370       ?GetParameter@CCodec_DXT5_xRBG@@UAE_NPBDAAM@Z 00487370 f   bitmap:Codec_DXT5_xRBG.obj
 0001:000863f0       ??_ECCodec_DXT5_xRBG@@UAEPAXI@Z 004873f0 f i bitmap:Codec_DXT5_xRBG.obj
 0001:000863f0       ??_GCCodec_DXT5_xRBG@@UAEPAXI@Z 004873f0 f i bitmap:Codec_DXT5_xRBG.obj
 0001:00086420       ??0CCodec_DXT5_RBxG@@QAE@XZ 00487420 f   bitmap:Codec_DXT5_RBxG.obj
 0001:00086440       ??1CCodec_DXT5_RBxG@@UAE@XZ 00487440 f   bitmap:Codec_DXT5_RBxG.obj
 0001:00086450       ?ReadBlock@CCodec_DXT5_RBxG@@MAEXAAVCCodecBuffer@@KKQAK@Z 00487450 f   bitmap:Codec_DXT5_RBxG.obj
 0001:00086540       ?WriteBlock@CCodec_DXT5_RBxG@@MAEXAAVCCodecBuffer@@KKQAK@Z 00487540 f   bitmap:Codec_DXT5_RBxG.obj
 0001:00086620       ?ReadBlock@CCodec_DXT5_RBxG@@MAEXAAVCCodecBuffer@@KKQAM@Z 00487620 f   bitmap:Codec_DXT5_RBxG.obj
 0001:000866a0       ?WriteBlock@CCodec_DXT5_RBxG@@MAEXAAVCCodecBuffer@@KKQAM@Z 004876a0 f   bitmap:Codec_DXT5_RBxG.obj
 0001:00086720       ?SetParameter@CCodec_DXT5_RBxG@@UAE_NPBDM@Z 00487720 f   bitmap:Codec_DXT5_RBxG.obj
 0001:000867b0       ?GetParameter@CCodec_DXT5_RBxG@@UAE_NPBDAAM@Z 004877b0 f   bitmap:Codec_DXT5_RBxG.obj
 0001:00086830       ??_ECCodec_DXT5_RBxG@@UAEPAXI@Z 00487830 f i bitmap:Codec_DXT5_RBxG.obj
 0001:00086830       ??_GCCodec_DXT5_RBxG@@UAEPAXI@Z 00487830 f i bitmap:Codec_DXT5_RBxG.obj
 0001:00086860       ??0CCodec_DXT5_RxBG@@QAE@XZ 00487860 f   bitmap:Codec_DXT5_RxBG.obj
 0001:00086880       ??1CCodec_DXT5_RxBG@@UAE@XZ 00487880 f   bitmap:Codec_DXT5_RxBG.obj
 0001:00086890       ?ReadBlock@CCodec_DXT5_RxBG@@MAEXAAVCCodecBuffer@@KKQAK@Z 00487890 f   bitmap:Codec_DXT5_RxBG.obj
 0001:00086970       ?WriteBlock@CCodec_DXT5_RxBG@@MAEXAAVCCodecBuffer@@KKQAK@Z 00487970 f   bitmap:Codec_DXT5_RxBG.obj
 0001:00086a50       ?ReadBlock@CCodec_DXT5_RxBG@@MAEXAAVCCodecBuffer@@KKQAM@Z 00487a50 f   bitmap:Codec_DXT5_RxBG.obj
 0001:00086ad0       ?WriteBlock@CCodec_DXT5_RxBG@@MAEXAAVCCodecBuffer@@KKQAM@Z 00487ad0 f   bitmap:Codec_DXT5_RxBG.obj
 0001:00086b50       ??_GCCodec_DXT5_RxBG@@UAEPAXI@Z 00487b50 f i bitmap:Codec_DXT5_RxBG.obj
 0001:00086b50       ??_ECCodec_DXT5_RxBG@@UAEPAXI@Z 00487b50 f i bitmap:Codec_DXT5_RxBG.obj
 0001:00086b80       ??0CCodec_DXT5_xGBR@@QAE@XZ 00487b80 f   bitmap:Codec_DXT5_xGBR.obj
 0001:00086ba0       ??1CCodec_DXT5_xGBR@@UAE@XZ 00487ba0 f   bitmap:Codec_DXT5_xGBR.obj
 0001:00086bb0       ?ReadBlock@CCodec_DXT5_xGBR@@MAEXAAVCCodecBuffer@@KKQAK@Z 00487bb0 f   bitmap:Codec_DXT5_xGBR.obj
 0001:00086ca0       ?WriteBlock@CCodec_DXT5_xGBR@@MAEXAAVCCodecBuffer@@KKQAK@Z 00487ca0 f   bitmap:Codec_DXT5_xGBR.obj
 0001:00086d80       ?ReadBlock@CCodec_DXT5_xGBR@@MAEXAAVCCodecBuffer@@KKQAM@Z 00487d80 f   bitmap:Codec_DXT5_xGBR.obj
 0001:00086e00       ?WriteBlock@CCodec_DXT5_xGBR@@MAEXAAVCCodecBuffer@@KKQAM@Z 00487e00 f   bitmap:Codec_DXT5_xGBR.obj
 0001:00086e90       ??_ECCodec_DXT5_xGBR@@UAEPAXI@Z 00487e90 f i bitmap:Codec_DXT5_xGBR.obj
 0001:00086e90       ??_GCCodec_DXT5_xGBR@@UAEPAXI@Z 00487e90 f i bitmap:Codec_DXT5_xGBR.obj
 0001:00086ec0       ??0CCodec_DXT5@@QAE@XZ     00487ec0 f   bitmap:Codec_DXT5.obj
 0001:00086ee0       ??1CCodec_DXT5@@UAE@XZ     00487ee0 f   bitmap:Codec_DXT5.obj
 0001:00086ef0       ?Compress@CCodec_DXT5@@UAE?AW4_CODECError@@AAVCCodecBuffer@@0P6A_NMKK@ZKK@Z 00487ef0 f   bitmap:Codec_DXT5.obj
 0001:000870d0       ?Decompress@CCodec_DXT5@@UAE?AW4_CODECError@@AAVCCodecBuffer@@0@Z 004880d0 f   bitmap:Codec_DXT5.obj
 0001:00087210       ??_GCCodec_DXT5@@UAEPAXI@Z 00488210 f i bitmap:Codec_DXT5.obj
 0001:00087210       ??_ECCodec_DXT5@@UAEPAXI@Z 00488210 f i bitmap:Codec_DXT5.obj
 0001:00087240       ??0CCodec_DXT3@@QAE@XZ     00488240 f   bitmap:Codec_DXT3.obj
 0001:00087260       ??1CCodec_DXT3@@UAE@XZ     00488260 f   bitmap:Codec_DXT3.obj
 0001:00087270       ?Compress@CCodec_DXT3@@UAE?AW4_CODECError@@AAVCCodecBuffer@@0P6A_NMKK@ZKK@Z 00488270 f   bitmap:Codec_DXT3.obj
 0001:00087450       ?Decompress@CCodec_DXT3@@UAE?AW4_CODECError@@AAVCCodecBuffer@@0@Z 00488450 f   bitmap:Codec_DXT3.obj
 0001:00087590       ??_GCCodec_DXT3@@UAEPAXI@Z 00488590 f i bitmap:Codec_DXT3.obj
 0001:00087590       ??_ECCodec_DXT3@@UAEPAXI@Z 00488590 f i bitmap:Codec_DXT3.obj
 0001:000875c0       ??0CCodec_DXT1@@QAE@XZ     004885c0 f   bitmap:Codec_DXT1.obj
 0001:000875e0       ??1CCodec_DXT1@@UAE@XZ     004885e0 f   bitmap:Codec_DXT1.obj
 0001:000875f0       ?CreateBuffer@CCodec_DXT1@@UBEPAVCCodecBuffer@@KKKPAE@Z 004885f0 f   bitmap:Codec_DXT1.obj
 0001:00087620       ?Compress@CCodec_DXT1@@UAE?AW4_CODECError@@AAVCCodecBuffer@@0P6A_NMKK@ZKK@Z 00488620 f   bitmap:Codec_DXT1.obj
 0001:00087840       ?Decompress@CCodec_DXT1@@UAE?AW4_CODECError@@AAVCCodecBuffer@@0@Z 00488840 f   bitmap:Codec_DXT1.obj
 0001:00087980       ?SetParameter@CCodec_DXT1@@UAE_NPBDK@Z 00488980 f   bitmap:Codec_DXT1.obj
 0001:000879e0       ?GetParameter@CCodec_DXT1@@UAE_NPBDAAK@Z 004889e0 f   bitmap:Codec_DXT1.obj
 0001:00087a50       ??_GCCodec_DXT1@@UAEPAXI@Z 00488a50 f i bitmap:Codec_DXT1.obj
 0001:00087a50       ??_ECCodec_DXT1@@UAEPAXI@Z 00488a50 f i bitmap:Codec_DXT1.obj
 0001:00087a80       ?overflow@half@@CAMXZ      00488a80 f   bitmap:half.obj
 0001:00087ab0       ?convert@half@@CAFH@Z      00488ab0 f   bitmap:half.obj
 0001:00087b70       ??0CCodecBuffer_Block@@QAE@W4_CodecBufferType@@KKKPAE@Z 00488b70 f   bitmap:CodecBuffer_Block.obj
 0001:00087c90       ??1CCodecBuffer_Block@@UAE@XZ 00488c90 f   bitmap:CodecBuffer_Block.obj
 0001:00087ca0       ?ReadBlock@CCodecBuffer_Block@@UAE_NKKPAKK@Z 00488ca0 f   bitmap:CodecBuffer_Block.obj
 0001:00087d10       ?WriteBlock@CCodecBuffer_Block@@UAE_NKKPAKK@Z 00488d10 f   bitmap:CodecBuffer_Block.obj
 0001:00087d80       ??_ECCodecBuffer_Block@@UAEPAXI@Z 00488d80 f i bitmap:CodecBuffer_Block.obj
 0001:00087d80       ??_GCCodecBuffer_Block@@UAEPAXI@Z 00488d80 f i bitmap:CodecBuffer_Block.obj
 0001:00087db0       ??0CCodecBuffer_RGBA32F@@QAE@KKKPAE@Z 00488db0 f   bitmap:CodecBuffer_RGBA32F.obj
 0001:00087e10       ??1CCodecBuffer_RGBA32F@@UAE@XZ 00488e10 f   bitmap:CodecBuffer_RGBA32F.obj
 0001:00087e20       ?Copy@CCodecBuffer_RGBA32F@@UAEXAAVCCodecBuffer@@@Z 00488e20 f   bitmap:CodecBuffer_RGBA32F.obj
 0001:00087ee0       ?WriteBlock@CCodecBuffer_RGBA32F@@MAE_NKKEEQAMK@Z 00488ee0 f   bitmap:CodecBuffer_RGBA32F.obj
 0001:00088050       ?ReadBlockA@CCodecBuffer_RGBA32F@@UAE_NKKEEQAM@Z 00489050 f   bitmap:CodecBuffer_RGBA32F.obj
 0001:00088080       ?ReadBlockR@CCodecBuffer_RGBA32F@@UAE_NKKEEQAM@Z 00489080 f   bitmap:CodecBuffer_RGBA32F.obj
 0001:000880b0       ?ReadBlockG@CCodecBuffer_RGBA32F@@UAE_NKKEEQAM@Z 004890b0 f   bitmap:CodecBuffer_RGBA32F.obj
 0001:000880e0       ?ReadBlockB@CCodecBuffer_RGBA32F@@UAE_NKKEEQAM@Z 004890e0 f   bitmap:CodecBuffer_RGBA32F.obj
 0001:00088110       ?WriteBlockA@CCodecBuffer_RGBA32F@@UAE_NKKEEQAM@Z 00489110 f   bitmap:CodecBuffer_RGBA32F.obj
 0001:00088140       ?WriteBlockR@CCodecBuffer_RGBA32F@@UAE_NKKEEQAM@Z 00489140 f   bitmap:CodecBuffer_RGBA32F.obj
 0001:00088170       ?WriteBlockG@CCodecBuffer_RGBA32F@@UAE_NKKEEQAM@Z 00489170 f   bitmap:CodecBuffer_RGBA32F.obj
 0001:000881a0       ?WriteBlockB@CCodecBuffer_RGBA32F@@UAE_NKKEEQAM@Z 004891a0 f   bitmap:CodecBuffer_RGBA32F.obj
 0001:000881d0       ?WriteBlockRGBA@CCodecBuffer_RGBA32F@@UAE_NKKEEQAM@Z 004891d0 f   bitmap:CodecBuffer_RGBA32F.obj
 0001:00088270       ?ReadBlock@CCodecBuffer_RGBA32F@@MAE_NKKEEQAMK@Z 00489270 f   bitmap:CodecBuffer_RGBA32F.obj
 0001:00088490       ?ReadBlockRGBA@CCodecBuffer_RGBA32F@@UAE_NKKEEQAM@Z 00489490 f   bitmap:CodecBuffer_RGBA32F.obj
 0001:000885f0       ?GetBufferType@CCodecBuffer_RGBA32F@@UBE?BW4_CodecBufferType@@XZ 004895f0 f i bitmap:CodecBuffer_RGBA32F.obj
 0001:00088600       ??_ECCodecBuffer_RGBA32F@@UAEPAXI@Z 00489600 f i bitmap:CodecBuffer_RGBA32F.obj
 0001:00088600       ??_GCCodecBuffer_RGBA32F@@UAEPAXI@Z 00489600 f i bitmap:CodecBuffer_RGBA32F.obj
 0001:00088630       ??0CCodecBuffer_RGBA16F@@QAE@KKKPAE@Z 00489630 f   bitmap:CodecBuffer_RGBA16F.obj
 0001:00088690       ??1CCodecBuffer_RGBA16F@@UAE@XZ 00489690 f   bitmap:CodecBuffer_RGBA16F.obj
 0001:000886a0       ?WriteBlock@CCodecBuffer_RGBA16F@@MAE_NKKEEQAVhalf@@K@Z 004896a0 f   bitmap:CodecBuffer_RGBA16F.obj
 0001:00088740       ?ReadBlockA@CCodecBuffer_RGBA16F@@UAE_NKKEEQAVhalf@@@Z 00489740 f   bitmap:CodecBuffer_RGBA16F.obj
 0001:00088770       ?ReadBlockR@CCodecBuffer_RGBA16F@@UAE_NKKEEQAVhalf@@@Z 00489770 f   bitmap:CodecBuffer_RGBA16F.obj
 0001:000887a0       ?ReadBlockG@CCodecBuffer_RGBA16F@@UAE_NKKEEQAVhalf@@@Z 004897a0 f   bitmap:CodecBuffer_RGBA16F.obj
 0001:000887d0       ?ReadBlockB@CCodecBuffer_RGBA16F@@UAE_NKKEEQAVhalf@@@Z 004897d0 f   bitmap:CodecBuffer_RGBA16F.obj
 0001:00088800       ?WriteBlockA@CCodecBuffer_RGBA16F@@UAE_NKKEEQAVhalf@@@Z 00489800 f   bitmap:CodecBuffer_RGBA16F.obj
 0001:00088830       ?WriteBlockR@CCodecBuffer_RGBA16F@@UAE_NKKEEQAVhalf@@@Z 00489830 f   bitmap:CodecBuffer_RGBA16F.obj
 0001:00088860       ?WriteBlockG@CCodecBuffer_RGBA16F@@UAE_NKKEEQAVhalf@@@Z 00489860 f   bitmap:CodecBuffer_RGBA16F.obj
 0001:00088890       ?WriteBlockB@CCodecBuffer_RGBA16F@@UAE_NKKEEQAVhalf@@@Z 00489890 f   bitmap:CodecBuffer_RGBA16F.obj
 0001:000888c0       ?WriteBlockRGBA@CCodecBuffer_RGBA16F@@UAE_NKKEEQAVhalf@@@Z 004898c0 f   bitmap:CodecBuffer_RGBA16F.obj
 0001:00088960       ?Copy@CCodecBuffer_RGBA16F@@UAEXAAVCCodecBuffer@@@Z 00489960 f   bitmap:CodecBuffer_RGBA16F.obj
 0001:00088a40       ?ReadBlock@CCodecBuffer_RGBA16F@@MAE_NKKEEQAVhalf@@K@Z 00489a40 f   bitmap:CodecBuffer_RGBA16F.obj
 0001:00088b80       ?ReadBlockRGBA@CCodecBuffer_RGBA16F@@UAE_NKKEEQAVhalf@@@Z 00489b80 f   bitmap:CodecBuffer_RGBA16F.obj
 0001:00088cc0       ??$PadBlock@G@@YAXKEEQAG@Z 00489cc0 f i bitmap:CodecBuffer_RGBA16.obj
 0001:00088cc0       ??$PadBlock@Vhalf@@@@YAXKEEQAVhalf@@@Z 00489cc0 f i bitmap:CodecBuffer_RGBA16F.obj
 0001:00088d10       ??_ECCodecBuffer_RGBA16F@@UAEPAXI@Z 00489d10 f i bitmap:CodecBuffer_RGBA16F.obj
 0001:00088d10       ??_GCCodecBuffer_RGBA16F@@UAEPAXI@Z 00489d10 f i bitmap:CodecBuffer_RGBA16F.obj
 0001:00088d40       ??0CCodecBuffer_RGBA16@@QAE@KKKPAE@Z 00489d40 f   bitmap:CodecBuffer_RGBA16.obj
 0001:00088da0       ??1CCodecBuffer_RGBA16@@UAE@XZ 00489da0 f   bitmap:CodecBuffer_RGBA16.obj
 0001:00088db0       ?Copy@CCodecBuffer_RGBA16@@UAEXAAVCCodecBuffer@@@Z 00489db0 f   bitmap:CodecBuffer_RGBA16.obj
 0001:00088e90       ?WriteBlock@CCodecBuffer_RGBA16@@MAE_NKKEEQAGK@Z 00489e90 f   bitmap:CodecBuffer_RGBA16.obj
 0001:00088f30       ?ReadBlockA@CCodecBuffer_RGBA16@@UAE_NKKEEQAG@Z 00489f30 f   bitmap:CodecBuffer_RGBA16.obj
 0001:00088f60       ?ReadBlockR@CCodecBuffer_RGBA16@@UAE_NKKEEQAG@Z 00489f60 f   bitmap:CodecBuffer_RGBA16.obj
 0001:00088f90       ?ReadBlockG@CCodecBuffer_RGBA16@@UAE_NKKEEQAG@Z 00489f90 f   bitmap:CodecBuffer_RGBA16.obj
 0001:00088fc0       ?ReadBlockB@CCodecBuffer_RGBA16@@UAE_NKKEEQAG@Z 00489fc0 f   bitmap:CodecBuffer_RGBA16.obj
 0001:00088ff0       ?WriteBlockA@CCodecBuffer_RGBA16@@UAE_NKKEEQAG@Z 00489ff0 f   bitmap:CodecBuffer_RGBA16.obj
 0001:00089020       ?WriteBlockR@CCodecBuffer_RGBA16@@UAE_NKKEEQAG@Z 0048a020 f   bitmap:CodecBuffer_RGBA16.obj
 0001:00089050       ?WriteBlockG@CCodecBuffer_RGBA16@@UAE_NKKEEQAG@Z 0048a050 f   bitmap:CodecBuffer_RGBA16.obj
 0001:00089080       ?WriteBlockB@CCodecBuffer_RGBA16@@UAE_NKKEEQAG@Z 0048a080 f   bitmap:CodecBuffer_RGBA16.obj
 0001:000890b0       ?WriteBlockRGBA@CCodecBuffer_RGBA16@@UAE_NKKEEQAG@Z 0048a0b0 f   bitmap:CodecBuffer_RGBA16.obj
 0001:00089150       ?ReadBlock@CCodecBuffer_RGBA16@@MAE_NKKEEQAGK@Z 0048a150 f   bitmap:CodecBuffer_RGBA16.obj
 0001:00089290       ?ReadBlockRGBA@CCodecBuffer_RGBA16@@UAE_NKKEEQAG@Z 0048a290 f   bitmap:CodecBuffer_RGBA16.obj
 0001:000893d0       ?GetBufferType@CCodecBuffer_RGBA16@@UBE?BW4_CodecBufferType@@XZ 0048a3d0 f i bitmap:CodecBuffer_RGBA16.obj
 0001:000893e0       ??$PadLine@G@@YAXKEQAG@Z   0048a3e0 f i bitmap:CodecBuffer_RGBA16.obj
 0001:000893e0       ??$PadLine@Vhalf@@@@YAXKEQAVhalf@@@Z 0048a3e0 f i bitmap:CodecBuffer_RGBA16F.obj
 0001:00089420       ??_GCCodecBuffer_RGBA16@@UAEPAXI@Z 0048a420 f i bitmap:CodecBuffer_RGBA16.obj
 0001:00089420       ??_ECCodecBuffer_RGBA16@@UAEPAXI@Z 0048a420 f i bitmap:CodecBuffer_RGBA16.obj
 0001:00089450       ??0CCodecBuffer_RGBA2101010@@QAE@KKKPAE@Z 0048a450 f   bitmap:CodecBuffer_RGBA2101010.obj
 0001:000894b0       ??1CCodecBuffer_RGBA2101010@@UAE@XZ 0048a4b0 f   bitmap:CodecBuffer_RGBA2101010.obj
 0001:000894c0       ?Copy@CCodecBuffer_RGBA2101010@@UAEXAAVCCodecBuffer@@@Z 0048a4c0 f   bitmap:CodecBuffer_RGBA2101010.obj
 0001:00089580       ?WriteBlock@CCodecBuffer_RGBA2101010@@MAE_NKKEEQAGKK@Z 0048a580 f   bitmap:CodecBuffer_RGBA2101010.obj
 0001:00089640       ?ReadBlockA@CCodecBuffer_RGBA2101010@@UAE_NKKEEQAG@Z 0048a640 f   bitmap:CodecBuffer_RGBA2101010.obj
 0001:00089670       ?ReadBlockR@CCodecBuffer_RGBA2101010@@UAE_NKKEEQAG@Z 0048a670 f   bitmap:CodecBuffer_RGBA2101010.obj
 0001:000896a0       ?ReadBlockG@CCodecBuffer_RGBA2101010@@UAE_NKKEEQAG@Z 0048a6a0 f   bitmap:CodecBuffer_RGBA2101010.obj
 0001:000896d0       ?ReadBlockB@CCodecBuffer_RGBA2101010@@UAE_NKKEEQAG@Z 0048a6d0 f   bitmap:CodecBuffer_RGBA2101010.obj
 0001:00089700       ?WriteBlockA@CCodecBuffer_RGBA2101010@@UAE_NKKEEQAG@Z 0048a700 f   bitmap:CodecBuffer_RGBA2101010.obj
 0001:00089730       ?WriteBlockR@CCodecBuffer_RGBA2101010@@UAE_NKKEEQAG@Z 0048a730 f   bitmap:CodecBuffer_RGBA2101010.obj
 0001:00089760       ?WriteBlockG@CCodecBuffer_RGBA2101010@@UAE_NKKEEQAG@Z 0048a760 f   bitmap:CodecBuffer_RGBA2101010.obj
 0001:00089790       ?WriteBlockB@CCodecBuffer_RGBA2101010@@UAE_NKKEEQAG@Z 0048a790 f   bitmap:CodecBuffer_RGBA2101010.obj
 0001:000897c0       ?WriteBlockRGBA@CCodecBuffer_RGBA2101010@@UAE_NKKEEQAK@Z 0048a7c0 f   bitmap:CodecBuffer_RGBA2101010.obj
 0001:00089880       ?WriteBlockRGBA@CCodecBuffer_RGBA2101010@@UAE_NKKEEQAG@Z 0048a880 f   bitmap:CodecBuffer_RGBA2101010.obj
 0001:00089980       ?ReadBlock@CCodecBuffer_RGBA2101010@@MAE_NKKEEQAGKK@Z 0048a980 f   bitmap:CodecBuffer_RGBA2101010.obj
 0001:00089ad0       ?ReadBlockRGBA@CCodecBuffer_RGBA2101010@@UAE_NKKEEQAK@Z 0048aad0 f   bitmap:CodecBuffer_RGBA2101010.obj
 0001:00089c10       ?ReadBlockRGBA@CCodecBuffer_RGBA2101010@@UAE_NKKEEQAG@Z 0048ac10 f   bitmap:CodecBuffer_RGBA2101010.obj
 0001:00089de0       ?GetBufferType@CCodecBuffer_RGBA2101010@@UBE?BW4_CodecBufferType@@XZ 0048ade0 f i bitmap:CodecBuffer_RGBA2101010.obj
 0001:00089df0       ??$PadLine@M@@YAXKEQAM@Z   0048adf0 f i bitmap:CodecBuffer_RGBA32F.obj
 0001:00089df0       ??$PadLine@K@@YAXKEQAK@Z   0048adf0 f i bitmap:CodecBuffer_RGBA2101010.obj
 0001:00089e30       ??$PadBlock@M@@YAXKEEQAM@Z 0048ae30 f i bitmap:CodecBuffer_RGBA32F.obj
 0001:00089e30       ??$PadBlock@K@@YAXKEEQAK@Z 0048ae30 f i bitmap:CodecBuffer_RGBA2101010.obj
 0001:00089e80       ??_ECCodecBuffer_RGBA2101010@@UAEPAXI@Z 0048ae80 f i bitmap:CodecBuffer_RGBA2101010.obj
 0001:00089e80       ??_GCCodecBuffer_RGBA2101010@@UAEPAXI@Z 0048ae80 f i bitmap:CodecBuffer_RGBA2101010.obj
 0001:00089eb0       ??0CCodecBuffer_RGBA8888@@QAE@KKKPAE@Z 0048aeb0 f   bitmap:CodecBuffer_RGBA8888.obj
 0001:00089f10       ??1CCodecBuffer_RGBA8888@@UAE@XZ 0048af10 f   bitmap:CodecBuffer_RGBA8888.obj
 0001:00089f20       ?Copy@CCodecBuffer_RGBA8888@@UAEXAAVCCodecBuffer@@@Z 0048af20 f   bitmap:CodecBuffer_RGBA8888.obj
 0001:00089fe0       ?WriteBlock@CCodecBuffer_RGBA8888@@MAE_NKKEEQAEK@Z 0048afe0 f   bitmap:CodecBuffer_RGBA8888.obj
 0001:0008a0a0       ?ReadBlockA@CCodecBuffer_RGBA8888@@UAE_NKKEEQAE@Z 0048b0a0 f   bitmap:CodecBuffer_RGBA8888.obj
 0001:0008a0d0       ?ReadBlockR@CCodecBuffer_RGBA8888@@UAE_NKKEEQAE@Z 0048b0d0 f   bitmap:CodecBuffer_RGBA8888.obj
 0001:0008a100       ?ReadBlockG@CCodecBuffer_RGBA8888@@UAE_NKKEEQAE@Z 0048b100 f   bitmap:CodecBuffer_RGBA8888.obj
 0001:0008a130       ?ReadBlockB@CCodecBuffer_RGBA8888@@UAE_NKKEEQAE@Z 0048b130 f   bitmap:CodecBuffer_RGBA8888.obj
 0001:0008a160       ?WriteBlockA@CCodecBuffer_RGBA8888@@UAE_NKKEEQAE@Z 0048b160 f   bitmap:CodecBuffer_RGBA8888.obj
 0001:0008a190       ?WriteBlockR@CCodecBuffer_RGBA8888@@UAE_NKKEEQAE@Z 0048b190 f   bitmap:CodecBuffer_RGBA8888.obj
 0001:0008a1c0       ?WriteBlockG@CCodecBuffer_RGBA8888@@UAE_NKKEEQAE@Z 0048b1c0 f   bitmap:CodecBuffer_RGBA8888.obj
 0001:0008a1f0       ?WriteBlockB@CCodecBuffer_RGBA8888@@UAE_NKKEEQAE@Z 0048b1f0 f   bitmap:CodecBuffer_RGBA8888.obj
 0001:0008a220       ?WriteBlockRGBA@CCodecBuffer_RGBA8888@@UAE_NKKEEQAK@Z 0048b220 f   bitmap:CodecBuffer_RGBA8888.obj
 0001:0008a2e0       ?ReadBlock@CCodecBuffer_RGBA8888@@MAE_NKKEEQAEK@Z 0048b2e0 f   bitmap:CodecBuffer_RGBA8888.obj
 0001:0008a430       ?ReadBlockRGBA@CCodecBuffer_RGBA8888@@UAE_NKKEEQAK@Z 0048b430 f   bitmap:CodecBuffer_RGBA8888.obj
 0001:0008a570       ??$PadLine@E@@YAXKEQAE@Z   0048b570 f i bitmap:CodecBuffer_RGBA8888.obj
 0001:0008a5b0       ??$PadBlock@E@@YAXKEEQAE@Z 0048b5b0 f i bitmap:CodecBuffer_RGBA8888.obj
 0001:0008a600       ??_ECCodecBuffer_RGBA8888@@UAEPAXI@Z 0048b600 f i bitmap:CodecBuffer_RGBA8888.obj
 0001:0008a600       ??_GCCodecBuffer_RGBA8888@@UAEPAXI@Z 0048b600 f i bitmap:CodecBuffer_RGBA8888.obj
 0001:0008a630       ??0CCodec_DXTC@@QAE@W4_CodecType@@@Z 0048b630 f   bitmap:Codec_DXTC.obj
 0001:0008a6d0       ??1CCodec_DXTC@@UAE@XZ     0048b6d0 f   bitmap:Codec_DXTC.obj
 0001:0008a6e0       ?SetParameter@CCodec_DXTC@@UAE_NPBDK@Z 0048b6e0 f   bitmap:Codec_DXTC.obj
 0001:0008a7e0       ?GetParameter@CCodec_DXTC@@UAE_NPBDAAK@Z 0048b7e0 f   bitmap:Codec_DXTC.obj
 0001:0008a8d0       ?SetParameter@CCodec_DXTC@@UAE_NPBDM@Z 0048b8d0 f   bitmap:Codec_DXTC.obj
 0001:0008a980       ?GetParameter@CCodec_DXTC@@UAE_NPBDAAM@Z 0048b980 f   bitmap:Codec_DXTC.obj
 0001:0008aa30       ??_GCCodec_DXTC@@UAEPAXI@Z 0048ba30 f i bitmap:Codec_DXTC.obj
 0001:0008aa30       ??_ECCodec_DXTC@@UAEPAXI@Z 0048ba30 f i bitmap:Codec_DXTC.obj
 0001:0008aa60       ??0CCodec_Block_4x4@@QAE@W4_CodecType@@@Z 0048ba60 f   bitmap:Codec_Block_4x4.obj
 0001:0008aa80       ??1CCodec_Block_4x4@@UAE@XZ 0048ba80 f   bitmap:Codec_Block_4x4.obj
 0001:0008aa90       ?CreateBuffer@CCodec_Block_4x4@@UBEPAVCCodecBuffer@@KKKPAE@Z 0048ba90 f   bitmap:Codec_Block_4x4.obj
 0001:0008aac0       ??_ECCodec_Block_4x4@@UAEPAXI@Z 0048bac0 f i bitmap:Codec_Block_4x4.obj
 0001:0008aac0       ??_GCCodec_Block_4x4@@UAEPAXI@Z 0048bac0 f i bitmap:Codec_Block_4x4.obj
 0001:0008aaf0       ?EncodeAlphaBlock@CCodec_DXTC@@IAEXQAKQAE1@Z 0048baf0 f   bitmap:Codec_DXTC_Alpha.obj
 0001:0008ac50       ?CompressExplicitAlphaBlock@CCodec_DXTC@@MAE?AW4_CODECError@@QAEQAK@Z 0048bc50 f   bitmap:Codec_DXTC_Alpha.obj
 0001:0008ade0       ?CompressExplicitAlphaBlock@CCodec_DXTC@@MAE?AW4_CODECError@@QAMQAK@Z 0048bde0 f   bitmap:Codec_DXTC_Alpha.obj
 0001:0008ae80       ?DecompressExplicitAlphaBlock@CCodec_DXTC@@MAEXQAEQAK@Z 0048be80 f   bitmap:Codec_DXTC_Alpha.obj
 0001:0008aec0       ?DecompressExplicitAlphaBlock@CCodec_DXTC@@MAEXQAMQAK@Z 0048bec0 f   bitmap:Codec_DXTC_Alpha.obj
 0001:0008b090       ?GetCompressedAlphaRamp@CCodec_DXTC@@IAEXQAEQAK@Z 0048c090 f   bitmap:Codec_DXTC_Alpha.obj
 0001:0008b200       ?GetCompressedAlphaRamp@CCodec_DXTC@@IAEXQAMQAK@Z 0048c200 f   bitmap:Codec_DXTC_Alpha.obj
 0001:0008b320       ?CompressAlphaBlock@CCodec_DXTC@@MAE?AW4_CODECError@@QAEQAK@Z 0048c320 f   bitmap:Codec_DXTC_Alpha.obj
 0001:0008b3f0       ?CompressAlphaBlock@CCodec_DXTC@@MAE?AW4_CODECError@@QAMQAK@Z 0048c3f0 f   bitmap:Codec_DXTC_Alpha.obj
 0001:0008b4c0       ?DecompressAlphaBlock@CCodec_DXTC@@MAEXQAEQAK@Z 0048c4c0 f   bitmap:Codec_DXTC_Alpha.obj
 0001:0008b660       ?DecompressAlphaBlock@CCodec_DXTC@@MAEXQAMQAK@Z 0048c660 f   bitmap:Codec_DXTC_Alpha.obj
 0001:0008b900       ?CompressRGBABlock@CCodec_DXTC@@MAE?AW4_CODECError@@QAK0PAM@Z 0048c900 f   bitmap:Codec_DXTC_RGBA.obj
 0001:0008b970       ?DecompressRGBABlock@CCodec_DXTC@@MAEXQAK0@Z 0048c970 f   bitmap:Codec_DXTC_RGBA.obj
 0001:0008ba30       ?CompressRGBABlock_ExplicitAlpha@CCodec_DXTC@@MAE?AW4_CODECError@@QAK0PAM@Z 0048ca30 f   bitmap:Codec_DXTC_RGBA.obj
 0001:0008baa0       ?DecompressRGBABlock_ExplicitAlpha@CCodec_DXTC@@MAEXQAK0@Z 0048caa0 f   bitmap:Codec_DXTC_RGBA.obj
 0001:0008bb60       ?CompressRGBBlock@CCodec_DXTC@@MAE?AW4_CODECError@@QAK0PAM_N2E@Z 0048cb60 f   bitmap:Codec_DXTC_RGBA.obj
 0001:0008be20       ?CompressRGBABlock@CCodec_DXTC@@MAE?AW4_CODECError@@QAMQAKPAM@Z 0048ce20 f   bitmap:Codec_DXTC_RGBA.obj
 0001:0008bec0       ?CompressRGBABlock_ExplicitAlpha@CCodec_DXTC@@MAE?AW4_CODECError@@QAMQAKPAM@Z 0048cec0 f   bitmap:Codec_DXTC_RGBA.obj
 0001:0008bf60       ?CompressRGBBlock@CCodec_DXTC@@MAE?AW4_CODECError@@QAMQAKPAM_N3M@Z 0048cf60 f   bitmap:Codec_DXTC_RGBA.obj
 0001:0008c220       ?DecompressRGBABlock@CCodec_DXTC@@MAEXQAMQAK@Z 0048d220 f   bitmap:Codec_DXTC_RGBA.obj
 0001:0008c2a0       ?DecompressRGBABlock_ExplicitAlpha@CCodec_DXTC@@MAEXQAMQAK@Z 0048d2a0 f   bitmap:Codec_DXTC_RGBA.obj
 0001:0008c320       ?DecompressRGBBlock@CCodec_DXTC@@MAEXQAK0_N@Z 0048d320 f   bitmap:Codec_DXTC_RGBA.obj
 0001:0008c560       ?DecompressRGBBlock@CCodec_DXTC@@MAEXQAMQAK_N@Z 0048d560 f   bitmap:Codec_DXTC_RGBA.obj
 0001:0008c8d0       ?CalculateColourWeightings@CCodec_DXTC@@IAEPAMQAK@Z 0048d8d0 f   bitmap:Codec_DXTC_RGBA.obj
 0001:0008ccb0       ?CalculateColourWeightings@CCodec_DXTC@@IAEPAMQAM@Z 0048dcb0 f   bitmap:Codec_DXTC_RGBA.obj
 0001:0008cfe0       ??0CCodec_DXT5_Swizzled@@QAE@W4_CodecType@@@Z 0048dfe0 f   bitmap:Codec_DXT5_Swizzled.obj
 0001:0008d000       ??1CCodec_DXT5_Swizzled@@UAE@XZ 0048e000 f   bitmap:Codec_DXT5_Swizzled.obj
 0001:0008d010       ?Compress@CCodec_DXT5_Swizzled@@UAE?AW4_CODECError@@AAVCCodecBuffer@@0P6A_NMKK@ZKK@Z 0048e010 f   bitmap:Codec_DXT5_Swizzled.obj
 0001:0008d1e0       ?Decompress@CCodec_DXT5_Swizzled@@UAE?AW4_CODECError@@AAVCCodecBuffer@@0@Z 0048e1e0 f   bitmap:Codec_DXT5_Swizzled.obj
 0001:0008d320       ??_GCCodec_DXT5_Swizzled@@UAEPAXI@Z 0048e320 f i bitmap:Codec_DXT5_Swizzled.obj
 0001:0008d320       ??_ECCodec_DXT5_Swizzled@@UAEPAXI@Z 0048e320 f i bitmap:Codec_DXT5_Swizzled.obj
 0001:0008d350       ??0CCodec_Block@@QAE@W4_CodecType@@@Z 0048e350 f   bitmap:Codec_Block.obj
 0001:0008d370       ??1CCodec_Block@@UAE@XZ    0048e370 f   bitmap:Codec_Block.obj
 0001:0008d380       ??_ECCodec_Block@@UAEPAXI@Z 0048e380 f i bitmap:Codec_Block.obj
 0001:0008d380       ??_GCCodec_Block@@UAEPAXI@Z 0048e380 f i bitmap:Codec_Block.obj
 0001:0008d3b0       ?ConstructColor@@YAKEEEEEE@Z 0048e3b0 f   bitmap:ATiXCodec.obj
 0001:0008ee50       ?CompBlock1X@@YAMPAMGQAEPAEE_N3HH3@Z 0048fe50 f   bitmap:ATiXCodec.obj
 0001:0008ef30       ?CompBlock1X@@YAMPAEGQAE0E_N2HH2@Z 0048ff30 f   bitmap:ATiXCodec.obj
 0001:0008f2a0       ?Clstr@@YAMQAKGQAY01EPAEEPAM_NEEEE@Z 004902a0 f   bitmap:ATiXCodec.obj
 0001:0008f660       ?Clstr@@YAMQAMGQAY01EPAEEPAM_NMEEE@Z 00490660 f   bitmap:ATiXCodec.obj
 0001:00093c60       ?CompressRGBBlockXSSE2@@YAXQAY01MQAY03MQAMHE_NEPAMEEE@Z 00494c60 f   bitmap:ATiXCodec.obj
 0001:00094e20       ?CompRGBBlock@@YAMPAMGEEEQAY01EPAEE_N3E03M@Z 00495e20 f   bitmap:ATiXCodec.obj
 0001:000953a0       ?CompRGBBlock@@YAMPAKGEEEQAY01EPAEE_N3EPAM3E@Z 004963a0 f   bitmap:ATiXCodec.obj
 0001:000956e0       ?MkWkRmpPts@@YAXPA_NQAY01M1EEE@Z 004966e0 f i bitmap:ATiXCodec.obj
 0001:00095840       ?BldClrRmp@@YAXQAM0E@Z     00496840 f i bitmap:ATiXCodec.obj
 0001:00095953       __itoa                     00496953 f   LIBCMT:xtoa.obj
 0001:00095953       _itoa                      00496953 f   LIBCMT:xtoa.obj
 0001:0009597b       __getextendedkeycode       0049697b f   LIBCMT:getch.obj
 0001:00095a28       __getch_nolock             00496a28 f   LIBCMT:getch.obj
 0001:00095aeb       _getch                     00496aeb f   LIBCMT:getch.obj
 0001:00095aeb       __getch                    00496aeb f   LIBCMT:getch.obj
 0001:00095b29       __wcstombs_l_helper        00496b29 f   LIBCMT:wcstombs.obj
 0001:00095d6f       __wcstombs_s_l             00496d6f f   LIBCMT:wcstombs.obj
 0001:00095e20       _wcstombs_s                00496e20 f   LIBCMT:wcstombs.obj
 0001:00095e3e       __wfsopen                  00496e3e f   LIBCMT:wfopen.obj
 0001:00095f04       __mbstowcs_l_helper        00496f04 f   LIBCMT:mbstowcs.obj
 0001:0009608c       __mbstowcs_s_l             0049708c f   LIBCMT:mbstowcs.obj
 0001:00096182       _mbstowcs_s                00497182 f   LIBCMT:mbstowcs.obj
 0001:000961a0       ?__ArrayUnwind@@YGXPAXIHP6EX0@Z@Z 004971a0 f   LIBCMT:ehvecdtr.obj
 0001:000961fe       ??_M@YGXPAXIHP6EX0@Z@Z     004971fe f   LIBCMT:ehvecdtr.obj
 0001:00096261       ??_L@YGXPAXIHP6EX0@Z1@Z    00497261 f   LIBCMT:ehvecctr.obj
 0001:000962d0       __ftol                     004972d0 f   LIBCMT:ftol.obj
 0001:00096300       __CIsqrt                   00497300 f   LIBCMT:sqrt.obj
 0001:00096314       _sqrt                      00497314     LIBCMT:sqrt.obj
 0001:000963ba       __mbscmp_l                 004973ba f   LIBCMT:mbscmp.obj
 0001:000964d6       __mbscmp                   004974d6 f   LIBCMT:mbscmp.obj
 0001:000964e9       __wopenfile                004974e9 f   LIBCMT:_wopen.obj
 0001:00096ecf       __wsopen_helper            00497ecf f   LIBCMT:wopen.obj
 0001:00096f9b       __wsopen_s                 00497f9b f   LIBCMT:wopen.obj
 0001:00096fb9       __wcsicmp_l                00497fb9 f   LIBCMT:wcsicmp.obj
 0001:000970c8       __wcsicmp                  004980c8 f   LIBCMT:wcsicmp.obj
 0001:00097159       _wcsncmp                   00498159 f   LIBCMT:wcsncmp.obj
 0001:0009718e       __towlower_l               0049818e f   LIBCMT:towlower.obj
 0001:0009749c       ___crtLCMapStringW         0049849c f   LIBCMT:w_map.obj
 0002:00000000       __imp__RegQueryValueExA@24 0049a000     advapi32:ADVAPI32.dll
 0002:00000004       __imp__RegCloseKey@4       0049a004     advapi32:ADVAPI32.dll
 0002:00000008       __imp__RegOpenKeyExA@20    0049a008     advapi32:ADVAPI32.dll
 0002:0000000c       \177ADVAPI32_NULL_THUNK_DATA 0049a00c     advapi32:ADVAPI32.dll
 0002:00000010       __imp__CreateFileA@28      0049a010     kernel32:KERNEL32.dll
 0002:00000014       __imp__GetLocalTime@4      0049a014     kernel32:KERNEL32.dll
 0002:00000018       __imp__GetLastError@0      0049a018     kernel32:KERNEL32.dll
 0002:0000001c       __imp__SetFilePointer@16   0049a01c     kernel32:KERNEL32.dll
 0002:00000020       __imp__ReadFile@20         0049a020     kernel32:KERNEL32.dll
 0002:00000024       __imp__WriteFile@20        0049a024     kernel32:KERNEL32.dll
 0002:00000028       __imp__DeleteFileA@4       0049a028     kernel32:KERNEL32.dll
 0002:0000002c       __imp__CloseHandle@4       0049a02c     kernel32:KERNEL32.dll
 0002:00000030       __imp__FlushFileBuffers@4  0049a030     kernel32:KERNEL32.dll
 0002:00000034       __imp__GetConsoleScreenBufferInfo@8 0049a034     kernel32:KERNEL32.dll
 0002:00000038       __imp__GetStdHandle@4      0049a038     kernel32:KERNEL32.dll
 0002:0000003c       __imp__SetConsoleTextAttribute@8 0049a03c     kernel32:KERNEL32.dll
 0002:00000040       __imp__GetProcessHeap@0    0049a040     kernel32:KERNEL32.dll
 0002:00000044       __imp__GetCurrentProcess@0 0049a044     kernel32:KERNEL32.dll
 0002:00000048       __imp__LeaveCriticalSection@4 0049a048     kernel32:KERNEL32.dll
 0002:0000004c       __imp__OutputDebugStringA@4 0049a04c     kernel32:KERNEL32.dll
 0002:00000050       __imp__EnterCriticalSection@4 0049a050     kernel32:KERNEL32.dll
 0002:00000054       __imp__InitializeCriticalSection@4 0049a054     kernel32:KERNEL32.dll
 0002:00000058       __imp__GetEnvironmentVariableA@12 0049a058     kernel32:KERNEL32.dll
 0002:0000005c       __imp__GetModuleHandleA@4  0049a05c     kernel32:KERNEL32.dll
 0002:00000060       __imp__SetPriorityClass@8  0049a060     kernel32:KERNEL32.dll
 0002:00000064       __imp__GetSystemInfo@4     0049a064     kernel32:KERNEL32.dll
 0002:00000068       __imp__SetThreadPriority@8 0049a068     kernel32:KERNEL32.dll
 0002:0000006c       __imp__CreateThread@24     0049a06c     kernel32:KERNEL32.dll
 0002:00000070       __imp__WaitForMultipleObjects@16 0049a070     kernel32:KERNEL32.dll
 0002:00000074       __imp__SetUnhandledExceptionFilter@4 0049a074     kernel32:KERNEL32.dll
 0002:00000078       __imp__HeapAlloc@12        0049a078     kernel32:KERNEL32.dll
 0002:0000007c       __imp__VirtualQuery@12     0049a07c     kernel32:KERNEL32.dll
 0002:00000080       __imp__TerminateProcess@8  0049a080     kernel32:KERNEL32.dll
 0002:00000084       __imp__GetModuleFileNameA@12 0049a084     kernel32:KERNEL32.dll
 0002:00000088       __imp__SetConsoleMode@8    0049a088     kernel32:KERNEL32.dll
 0002:0000008c       __imp__ReadConsoleInputA@16 0049a08c     kernel32:KERNEL32.dll
 0002:00000090       __imp__IsProcessorFeaturePresent@4 0049a090     kernel32:KERNEL32.dll
 0002:00000094       __imp__ResumeThread@4      0049a094     kernel32:KERNEL32.dll
 0002:00000098       __imp__GetExitCodeThread@8 0049a098     kernel32:KERNEL32.dll
 0002:0000009c       __imp__CreateProcessA@40   0049a09c     kernel32:KERNEL32.dll
 0002:000000a0       __imp__WaitForSingleObject@8 0049a0a0     kernel32:KERNEL32.dll
 0002:000000a4       __imp__GetExitCodeProcess@8 0049a0a4     kernel32:KERNEL32.dll
 0002:000000a8       __imp__CompareStringW@24   0049a0a8     kernel32:KERNEL32.dll
 0002:000000ac       __imp__CompareStringA@24   0049a0ac     kernel32:KERNEL32.dll
 0002:000000b0       __imp__GetTimeZoneInformation@4 0049a0b0     kernel32:KERNEL32.dll
 0002:000000b4       __imp__SetEndOfFile@4      0049a0b4     kernel32:KERNEL32.dll
 0002:000000b8       __imp__WriteConsoleW@20    0049a0b8     kernel32:KERNEL32.dll
 0002:000000bc       __imp__GetConsoleOutputCP@0 0049a0bc     kernel32:KERNEL32.dll
 0002:000000c0       __imp__WriteConsoleA@20    0049a0c0     kernel32:KERNEL32.dll
 0002:000000c4       __imp__IsValidLocale@8     0049a0c4     kernel32:KERNEL32.dll
 0002:000000c8       __imp__EnumSystemLocalesA@8 0049a0c8     kernel32:KERNEL32.dll
 0002:000000cc       __imp__GetUserDefaultLCID@0 0049a0cc     kernel32:KERNEL32.dll
 0002:000000d0       __imp__GetStringTypeW@16   0049a0d0     kernel32:KERNEL32.dll
 0002:000000d4       __imp__GetStringTypeA@20   0049a0d4     kernel32:KERNEL32.dll
 0002:000000d8       __imp__GetLocaleInfoW@16   0049a0d8     kernel32:KERNEL32.dll
 0002:000000dc       __imp__GetLocaleInfoA@16   0049a0dc     kernel32:KERNEL32.dll
 0002:000000e0       __imp__SetStdHandle@8      0049a0e0     kernel32:KERNEL32.dll
 0002:000000e4       __imp__GetSystemTimeAsFileTime@4 0049a0e4     kernel32:KERNEL32.dll
 0002:000000e8       __imp__GetTickCount@0      0049a0e8     kernel32:KERNEL32.dll
 0002:000000ec       __imp__QueryPerformanceCounter@4 0049a0ec     kernel32:KERNEL32.dll
 0002:000000f0       __imp__GetEnvironmentStringsW@0 0049a0f0     kernel32:KERNEL32.dll
 0002:000000f4       __imp__FreeEnvironmentStringsW@4 0049a0f4     kernel32:KERNEL32.dll
 0002:000000f8       __imp__MultiByteToWideChar@24 0049a0f8     kernel32:KERNEL32.dll
 0002:000000fc       __imp__WideCharToMultiByte@32 0049a0fc     kernel32:KERNEL32.dll
 0002:00000100       __imp__GetProcAddress@8    0049a100     kernel32:KERNEL32.dll
 0002:00000104       __imp__LoadLibraryExA@12   0049a104     kernel32:KERNEL32.dll
 0002:00000108       __imp__FreeLibrary@4       0049a108     kernel32:KERNEL32.dll
 0002:0000010c       __imp__UnhandledExceptionFilter@4 0049a10c     kernel32:KERNEL32.dll
 0002:00000110       __imp__IsDebuggerPresent@0 0049a110     kernel32:KERNEL32.dll
 0002:00000114       __imp__RaiseException@16   0049a114     kernel32:KERNEL32.dll
 0002:00000118       __imp__RtlUnwind@16        0049a118     kernel32:KERNEL32.dll
 0002:0000011c       __imp__ExitProcess@4       0049a11c     kernel32:KERNEL32.dll
 0002:00000120       __imp__FindClose@4         0049a120     kernel32:KERNEL32.dll
 0002:00000124       __imp__FileTimeToSystemTime@8 0049a124     kernel32:KERNEL32.dll
 0002:00000128       __imp__FileTimeToLocalFileTime@8 0049a128     kernel32:KERNEL32.dll
 0002:0000012c       __imp__GetDriveTypeA@4     0049a12c     kernel32:KERNEL32.dll
 0002:00000130       __imp__FindFirstFileA@8    0049a130     kernel32:KERNEL32.dll
 0002:00000134       __imp__GetFullPathNameA@16 0049a134     kernel32:KERNEL32.dll
 0002:00000138       __imp__CreateDirectoryA@8  0049a138     kernel32:KERNEL32.dll
 0002:0000013c       __imp__FindNextFileA@8     0049a13c     kernel32:KERNEL32.dll
 0002:00000140       __imp__GetFileAttributesA@4 0049a140     kernel32:KERNEL32.dll
 0002:00000144       __imp__SetEnvironmentVariableA@8 0049a144     kernel32:KERNEL32.dll
 0002:00000148       __imp__GetCurrentDirectoryA@8 0049a148     kernel32:KERNEL32.dll
 0002:0000014c       __imp__SetCurrentDirectoryA@4 0049a14c     kernel32:KERNEL32.dll
 0002:00000150       __imp__GetCommandLineA@0   0049a150     kernel32:KERNEL32.dll
 0002:00000154       __imp__HeapFree@12         0049a154     kernel32:KERNEL32.dll
 0002:00000158       __imp__GetVersionExA@4     0049a158     kernel32:KERNEL32.dll
 0002:0000015c       __imp__SetHandleCount@4    0049a15c     kernel32:KERNEL32.dll
 0002:00000160       __imp__GetFileType@4       0049a160     kernel32:KERNEL32.dll
 0002:00000164       __imp__GetStartupInfoA@4   0049a164     kernel32:KERNEL32.dll
 0002:00000168       __imp__DeleteCriticalSection@4 0049a168     kernel32:KERNEL32.dll
 0002:0000016c       __imp__TlsGetValue@4       0049a16c     kernel32:KERNEL32.dll
 0002:00000170       __imp__TlsAlloc@0          0049a170     kernel32:KERNEL32.dll
 0002:00000174       __imp__TlsSetValue@8       0049a174     kernel32:KERNEL32.dll
 0002:00000178       __imp__TlsFree@4           0049a178     kernel32:KERNEL32.dll
 0002:0000017c       __imp__InterlockedIncrement@4 0049a17c     kernel32:KERNEL32.dll
 0002:00000180       __imp__SetLastError@4      0049a180     kernel32:KERNEL32.dll
 0002:00000184       __imp__GetCurrentThreadId@0 0049a184     kernel32:KERNEL32.dll
 0002:00000188       __imp__InterlockedDecrement@4 0049a188     kernel32:KERNEL32.dll
 0002:0000018c       __imp__GetCPInfo@8         0049a18c     kernel32:KERNEL32.dll
 0002:00000190       __imp__GetACP@0            0049a190     kernel32:KERNEL32.dll
 0002:00000194       __imp__GetOEMCP@0          0049a194     kernel32:KERNEL32.dll
 0002:00000198       __imp__IsValidCodePage@4   0049a198     kernel32:KERNEL32.dll
 0002:0000019c       __imp__GetConsoleCP@0      0049a19c     kernel32:KERNEL32.dll
 0002:000001a0       __imp__GetConsoleMode@8    0049a1a0     kernel32:KERNEL32.dll
 0002:000001a4       __imp__LCMapStringA@24     0049a1a4     kernel32:KERNEL32.dll
 0002:000001a8       __imp__LCMapStringW@24     0049a1a8     kernel32:KERNEL32.dll
 0002:000001ac       __imp__LoadLibraryA@4      0049a1ac     kernel32:KERNEL32.dll
 0002:000001b0       __imp__GetCurrentProcessId@0 0049a1b0     kernel32:KERNEL32.dll
 0002:000001b4       __imp__SetEnvironmentVariableW@8 0049a1b4     kernel32:KERNEL32.dll
 0002:000001b8       __imp__FreeEnvironmentStringsA@4 0049a1b8     kernel32:KERNEL32.dll
 0002:000001bc       __imp__GetEnvironmentStrings@0 0049a1bc     kernel32:KERNEL32.dll
 0002:000001c0       __imp__CreateFileW@28      0049a1c0     kernel32:KERNEL32.dll
 0002:000001c4       \177KERNEL32_NULL_THUNK_DATA 0049a1c4     kernel32:KERNEL32.dll
 0002:000001c8       __imp__Msg                 0049a1c8     tier0:tier0.dll
 0002:000001cc       __imp__Error               0049a1cc     tier0:tier0.dll
 0002:000001d0       __imp__g_pMemAlloc         0049a1d0     tier0:tier0.dll
 0002:000001d4       __imp__GetCPUInformation   0049a1d4     tier0:tier0.dll
 0002:000001d8       __imp__GetThreadedLoadLibraryFunc 0049a1d8     tier0:tier0.dll
 0002:000001dc       __imp__CreateSimpleThread  0049a1dc     tier0:tier0.dll
 0002:000001e0       __imp__ReleaseThreadHandle 0049a1e0     tier0:tier0.dll
 0002:000001e4       __imp__Plat_IsInDebugSession 0049a1e4     tier0:tier0.dll
 0002:000001e8       __imp__ThreadWaitForObjects 0049a1e8     tier0:tier0.dll
 0002:000001ec       __imp__DevMsg              0049a1ec     tier0:tier0.dll
 0002:000001f0       __imp_??0CThreadSpinRWLock@@QAE@XZ 0049a1f0     tier0:tier0.dll
 0002:000001f4       __imp_?LockForWrite@CThreadSpinRWLock@@QAEXXZ 0049a1f4     tier0:tier0.dll
 0002:000001f8       __imp_?UnlockWrite@CThreadSpinRWLock@@QAEXXZ 0049a1f8     tier0:tier0.dll
 0002:000001fc       __imp_?LockForRead@CThreadSpinRWLock@@QAEXXZ 0049a1fc     tier0:tier0.dll
 0002:00000200       __imp_?UnlockRead@CThreadSpinRWLock@@QAEXXZ 0049a200     tier0:tier0.dll
 0002:00000204       __imp___AssertValidWritePtr 0049a204     tier0:tier0.dll
 0002:00000208       __imp__AssertValidStringPtr 0049a208     tier0:tier0.dll
 0002:0000020c       __imp__WriteMiniDumpUsingExceptionInfo 0049a20c     tier0:tier0.dll
 0002:00000210       __imp__SpewOutputFunc      0049a210     tier0:tier0.dll
 0002:00000214       __imp__GetSpewOutputColor  0049a214     tier0:tier0.dll
 0002:00000218       __imp_?DevMsg@@YAXPBDZZ    0049a218     tier0:tier0.dll
 0002:0000021c       __imp__CommandLine_Tier0   0049a21c     tier0:tier0.dll
 0002:00000220       __imp__MemFreeScratch      0049a220     tier0:tier0.dll
 0002:00000224       __imp__MemAllocScratch     0049a224     tier0:tier0.dll
 0002:00000228       __imp__SpewActivate        0049a228     tier0:tier0.dll
 0002:0000022c       __imp__ColorSpewMessage    0049a22c     tier0:tier0.dll
 0002:00000230       __imp__Plat_FloatTime      0049a230     tier0:tier0.dll
 0002:00000234       __imp__Warning             0049a234     tier0:tier0.dll
 0002:00000238       \177tier0_NULL_THUNK_DATA  0049a238     tier0:tier0.dll
 0002:0000023c       __imp__RandomSeed          0049a23c     vstdlib:vstdlib.dll
 0002:00000240       __imp__KeyValuesSystem     0049a240     vstdlib:vstdlib.dll
 0002:00000244       __imp__RandomGaussianFloat 0049a244     vstdlib:vstdlib.dll
 0002:00000248       \177vstdlib_NULL_THUNK_DATA 0049a248     vstdlib:vstdlib.dll
 0002:0000024c       ___xc_a                    0049a24c     LIBCMT:crt0init.obj
 0002:00000480       ___xc_z                    0049a480     LIBCMT:crt0init.obj
 0002:00000484       ___xi_a                    0049a484     LIBCMT:crt0init.obj
 0002:000004a0       ___xi_z                    0049a4a0     LIBCMT:crt0init.obj
 0002:000004a4       ___xp_a                    0049a4a4     LIBCMT:crt0init.obj
 0002:000004b4       ___xp_z                    0049a4b4     LIBCMT:crt0init.obj
 0002:000004b8       ___xt_a                    0049a4b8     LIBCMT:crt0init.obj
 0002:000004bc       ___xt_z                    0049a4bc     LIBCMT:crt0init.obj
 0002:000004dc       ??_C@_01NOFIACDB@w?$AA@    0049a4dc     brushbsp.obj
 0002:000004e0       ??_C@_01EEMJAFIK@?6?$AA@   0049a4e0     brushbsp.obj
 0002:000004e4       __real@3eaaaaab            0049a4e4     brushbsp.obj
 0002:000004e8       __real@3f50624dd2f1a9fc    0049a4e8     brushbsp.obj
 0002:000004f0       ??_C@_0N@OCBJIIGD@bad?5planenum?$AA@ 0049a4f0     brushbsp.obj
 0002:00000500       __real@bf800000            0049a500     brushbsp.obj
 0002:00000504       __real@3f800000            0049a504     brushbsp.obj
 0002:00000508       __real@bfb999999999999a    0049a508     brushbsp.obj
 0002:00000510       __real@3fb999999999999a    0049a510     brushbsp.obj
 0002:00000518       __real@3fc999999999999a    0049a518     brushbsp.obj
 0002:00000520       __real@46800000            0049a520     brushbsp.obj
 0002:00000524       __real@c6800000            0049a524     brushbsp.obj
 0002:00000528       ??_C@_0N@LMFHMMBE@Tried?5parent?$AA@ 0049a528     brushbsp.obj
 0002:00000538       ??_C@_0BJ@MIBLAJDN@split?5not?5on?5both?5sides?6?$AA@ 0049a538     brushbsp.obj
 0002:00000554       ??_C@_0BF@HEKJJEMO@split?5removed?5brush?6?$AA@ 0049a554     brushbsp.obj
 0002:0000056c       ??_C@_0BI@PNMADFKF@bogus?5brush?5after?5clip?6?$AA@ 0049a56c     brushbsp.obj
 0002:00000584       ??_C@_0BH@FEMFMIHD@WARNING?3?5huge?5winding?6?$AA@ 0049a584     brushbsp.obj
 0002:0000059c       __real@bf000000            0049a59c     brushbsp.obj
 0002:000005a0       ??_C@_0BJ@OFPPOJGD@PSIDE_FACING?5with?5splits?$AA@ 0049a5a0     brushbsp.obj
 0002:000005bc       ??_C@_0L@OGLHABIK@?$CF5i?5leafs?6?$AA@ 0049a5bc     brushbsp.obj
 0002:000005c8       ??_C@_0BC@MKFJDBDJ@?$CF5i?5nonvis?5nodes?6?$AA@ 0049a5c8     brushbsp.obj
 0002:000005dc       ??_C@_0BD@NJLKNHAJ@?$CF5i?5visible?5nodes?6?$AA@ 0049a5dc     brushbsp.obj
 0002:000005f0       ??_C@_0BG@KLEEPBIP@?$CF5i?5nonvisible?5faces?6?$AA@ 0049a5f0     brushbsp.obj
 0002:00000608       ??_C@_0BD@GCHPCEAO@?$CF5i?5visible?5faces?6?$AA@ 0049a608     brushbsp.obj
 0002:0000061c       ??_C@_0N@BAHABBPA@?$CF5i?5brushes?6?$AA@ 0049a61c     brushbsp.obj
 0002:0000062c       ??_C@_0BP@JDOEDEKN@Brush?5?$CFi?3?5WARNING?0?5microbrush?6?$AA@ 0049a62c     brushbsp.obj
 0002:0000064c       ??_C@_0BC@FBAFDPHA@?9?9?9?5BrushBSP?5?9?9?9?6?$AA@ 0049a64c     brushbsp.obj
 0002:00000660       __real@3a83126f            0049a660     collisionutils.obj
 0002:00000668       __real@3eb0c6f7a0b5ed8d    0049a668     collisionutils.obj
 0002:00000670       __real@3f000000            0049a670     collisionutils.obj
 0002:00000674       __real@40800000            0049a674     collisionutils.obj
 0002:00000678       __real@40000000            0049a678     collisionutils.obj
 0002:00000680       __real@0000000000000000    0049a680     collisionutils.obj
 0002:00000688       __real@3ee4f8b588e368f1    0049a688     collisionutils.obj
 0002:00000690       __real@3ff0000000000000    0049a690     collisionutils.obj
 0002:00000698       __real@41200000            0049a698     collisionutils.obj
 0002:0000069c       __real@c7c34f80            0049a69c     collisionutils.obj
 0002:000006a0       __real@4010000000000000    0049a6a0     collisionutils.obj
 0002:000006a8       ??_C@_0BB@GFLDGGJL@CONTENTS_HITBOX?5?$AA@ 0049a6a8     csg.obj
 0002:000006bc       ??_C@_0BB@DMKKLEIP@CONTENTS_LADDER?5?$AA@ 0049a6bc     csg.obj
 0002:000006d0       ??_C@_0BG@GBNDOMKC@CONTENTS_TRANSLUCENT?5?$AA@ 0049a6d0     csg.obj
 0002:000006e8       ??_C@_0BB@IMFIDHAA@CONTENTS_DETAIL?5?$AA@ 0049a6e8     csg.obj
 0002:000006fc       ??_C@_0BB@GJONNPJJ@CONTENTS_DEBRIS?5?$AA@ 0049a6fc     csg.obj
 0002:00000710       ??_C@_0BC@JHNGBGJB@CONTENTS_MONSTER?5?$AA@ 0049a710     csg.obj
 0002:00000724       ??_C@_0BB@EAMHLJJN@CONTENTS_ORIGIN?5?$AA@ 0049a724     csg.obj
 0002:00000738       ??_C@_0BH@MCAJFAKC@CONTENTS_CURRENT_DOWN?5?$AA@ 0049a738     csg.obj
 0002:00000750       ??_C@_0BF@BKFOCONM@CONTENTS_CURRENT_UP?5?$AA@ 0049a750     csg.obj
 0002:00000768       ??_C@_0BG@ILDOCDOE@CONTENTS_CURRENT_270?5?$AA@ 0049a768     csg.obj
 0002:00000780       ??_C@_0BG@JEPNEJGC@CONTENTS_CURRENT_180?5?$AA@ 0049a780     csg.obj
 0002:00000798       ??_C@_0BF@CDHJKNEH@CONTENTS_CURRENT_90?5?$AA@ 0049a798     csg.obj
 0002:000007b0       ??_C@_0BE@NOLHPBOB@CONTENTS_CURRENT_0?5?$AA@ 0049a7b0     csg.obj
 0002:000007c4       ??_C@_0BG@KIBJOIGE@CONTENTS_MONSTERCLIP?5?$AA@ 0049a7c4     csg.obj
 0002:000007dc       ??_C@_0BF@HJINIOEE@CONTENTS_PLAYERCLIP?5?$AA@ 0049a7dc     csg.obj
 0002:000007f4       ??_C@_0BF@HGIDDNMO@CONTENTS_AREAPORTAL?5?$AA@ 0049a7f4     csg.obj
 0002:0000080c       ??_C@_0BD@KGKKLEFD@CONTENTS_MOVEABLE?5?$AA@ 0049a80c     csg.obj
 0002:00000820       ??_C@_0BI@HIDMIENL@CONTENTS_TESTFOGVOLUME?5?$AA@ 0049a820     csg.obj
 0002:00000838       ??_C@_0BB@MCDBEPDN@CONTENTS_OPAQUE?5?$AA@ 0049a838     csg.obj
 0002:0000084c       ??_C@_0BD@HKLNCBAK@CONTENTS_BLOCKLOS?5?$AA@ 0049a84c     csg.obj
 0002:00000860       ??_C@_0BA@CLNLOILO@CONTENTS_WATER?5?$AA@ 0049a860     csg.obj
 0002:00000870       ??_C@_0BA@CHKHBBFK@CONTENTS_SLIME?5?$AA@ 0049a870     csg.obj
 0002:00000880       ??_C@_0BA@JAILJJLI@CONTENTS_GRATE?5?$AA@ 0049a880     csg.obj
 0002:00000890       ??_C@_0O@KGHFKPEC@CONTENTS_AUX?5?$AA@ 0049a890     csg.obj
 0002:000008a0       ??_C@_0BB@OGHJNGHM@CONTENTS_WINDOW?5?$AA@ 0049a8a0     csg.obj
 0002:000008b4       ??_C@_0BA@OHHDBBOE@CONTENTS_SOLID?5?$AA@ 0049a8b4     csg.obj
 0002:000008c4       ??_C@_02DKCKIIND@?$CFs?$AA@ 0049a8c4     csg.obj
 0002:000008c8       ??_C@_0BE@HPDKFHIA@output?5brushes?3?5?$CFi?6?$AA@ 0049a8c8     csg.obj
 0002:000008dc       ??_C@_0BG@FLNBNMPG@original?5brushes?3?5?$CFi?6?$AA@ 0049a8dc     csg.obj
 0002:000008f4       ??_C@_0BH@CNPBDCHJ@?9?9?9?9?5ChopBrushes?5?9?9?9?9?6?$AA@ 0049a8f4     csg.obj
 0002:0000090c       ??_C@_0CA@FMJIPOPP@Found?5no?5matching?5plane?5for?5?$CFs?6?$AA@ 0049a90c     csg.obj
 0002:0000092c       ??_C@_02KGHIDFGE@?$HN?6?$AA@ 0049a92c     csg.obj
 0002:00000930       ??_C@_02KCPFEJNG@?$HL?6?$AA@ 0049a930     csg.obj
 0002:00000933       ??_C@_00CNPNBAHC@?$AA@     0049a933     cubemap.obj
 0002:00000934       ??_C@_0BC@KFGKDDMG@$fallbackmaterial?$AA@ 0049a934     cubemap.obj
 0002:00000948       ??_C@_0P@OHFFMJJM@$crackmaterial?$AA@ 0049a948     cubemap.obj
 0002:00000958       ??_C@_0BA@OOJNCPMH@$bottommaterial?$AA@ 0049a958     cubemap.obj
 0002:00000968       ??_C@_07OAIDGMCI@skyname?$AA@ 0049a968     cubemap.obj
 0002:00000970       ??_C@_0L@BIFLFHPF@worldspawn?$AA@ 0049a970     cubemap.obj
 0002:0000097c       ??_C@_09CNJINBGN@classname?$AA@ 0049a97c     cubemap.obj
 0002:00000988       ??_C@_0EI@KOELCBDO@Material?5?$CFs?5is?5depending?5on?5itse@ 0049a988     cubemap.obj
 0002:000009d0       ??_C@_08DJCCKPNK@?4hdr?4vtf?$AA@ 0049a9d0     cubemap.obj
 0002:000009dc       ??_C@_04GJCHGKGK@?4vtf?$AA@ 0049a9dc     cubemap.obj
 0002:000009e4       ??_C@_0DM@NGPBHADK@Generated?5env_cubemap?5patch?5name@ 0049a9e4     cubemap.obj
 0002:00000a20       ??_C@_0BF@KEBGBCLN@maps?1?$CFs?1?$CFs?$CFs?$CFd_?$CFd_?$CFd?$AA@ 0049aa20     cubemap.obj
 0002:00000a38       ??_C@_01IDAFKMJL@_?$AA@    0049aa38     cubemap.obj
 0002:00000a3c       ??_C@_07NFGFKDAC@$envmap?$AA@ 0049aa3c     cubemap.obj
 0002:00000a44       ??_C@_0M@DLHJBNEJ@env_cubemap?$AA@ 0049aa44     cubemap.obj
 0002:00000a50       __real@7f7fffff            0049aa50     cubemap.obj
 0002:00000a54       ??_C@_0BG@EMENODEA@CUtlRBTree?5overflow?$CB?6?$AA@ 0049aa54     cubemap.obj
 0002:00000a70       ??_C@_0GD@NNAGIMAC@?$CK?$CK?$CK?5Error?3?5Skybox?5vtf?5files?5for?5@ 0049aa70     cubemap.obj
 0002:00000ad4       ??_C@_0CM@BJEKPFON@?$CK?$CK?$CK?5Error?5unserializing?5skybox?5t@ 0049aad4     cubemap.obj
 0002:00000b00       ??_C@_0BB@NIFPAOKF@materials?1?$CFs?4vtf?$AA@ 0049ab00     cubemap.obj
 0002:00000b14       ??_C@_0N@NEFMJPPI@$basetexture?$AA@ 0049ab14     cubemap.obj
 0002:00000b24       ??_C@_06BMKANHHL@skybox?$AA@ 0049ab24     cubemap.obj
 0002:00000b2c       ??_C@_04HDOCAJNK@?$CFs?$CFs?$AA@ 0049ab2c     cubemap.obj
 0002:00000b34       ??_C@_02LEBOADDI@dn?$AA@   0049ab34     cubemap.obj
 0002:00000b38       ??_C@_02HNLLPFKA@up?$AA@   0049ab38     cubemap.obj
 0002:00000b3c       ??_C@_02HLHCNIN@ft?$AA@    0049ab3c     cubemap.obj
 0002:00000b40       ??_C@_02MNOEILMP@bk?$AA@   0049ab40     cubemap.obj
 0002:00000b44       ??_C@_02HCNENIII@lf?$AA@   0049ab44     cubemap.obj
 0002:00000b48       ??_C@_02BMJICGCB@rt?$AA@   0049ab48     cubemap.obj
 0002:00000b4c       ??_C@_0CJ@LJOMCNEC@materials?1maps?1?$CFs?1cubemapdefault@ 0049ab4c     cubemap.obj
 0002:00000b78       ??_C@_0CG@CBMBGIFJ@Error?5serializing?5default?5cubema@ 0049ab78     cubemap.obj
 0002:00000ba0       ??_C@_0CF@HMPEADGK@materials?1maps?1?$CFs?1cubemapdefault@ 0049aba0     cubemap.obj
 0002:00000bc8       ??_C@_0JB@DKEDBBNA@Creating?5default?5?$CFscubemaps?5for?5@ 0049abc8     cubemap.obj
 0002:00000c5c       ??_C@_04EKBEKMLM@LDR?5?$AA@ 0049ac5c     cubemap.obj
 0002:00000c64       ??_C@_04LPJEAKHM@HDR?5?$AA@ 0049ac64     cubemap.obj
 0002:00000c6c       ??_C@_0DJ@OHDMOOPJ@Can?8t?5load?5skybox?5file?5?$CFs?5to?5bui@ 0049ac6c     cubemap.obj
 0002:00000ca8       ??_C@_09ICMOGGML@skybox?1?$CFs?$AA@ 0049aca8     cubemap.obj
 0002:00000cb4       ??_C@_01PAPGNFGE@c?$AA@    0049acb4     cubemap.obj
 0002:00000cb8       ??_C@_02DPKJAMEF@?$CFd?$AA@ 0049acb8     cubemap.obj
 0002:00000cbc       ??_C@_01CLKCMJKC@?5?$AA@   0049acbc     cubemap.obj
 0002:00000cc0       ??_C@_09IKJKMKOL@_?$CFd_?$CFd_?$CFd?$AA@ 0049acc0     cubemap.obj
 0002:00000ccc       ??_C@_0DC@KJOJLAEN@Multiple?5references?5for?5cubemap?5@ 0049accc     cubemap.obj
 0002:00000d00       ??_C@_0DN@PGKDBHHE@env_cubemap?5pointing?5at?5deleted?5@ 0049ad00     cubemap.obj
 0002:00000d40       ??_C@_0DD@COIAGLNI@fixing?5up?5env_cubemap?5materials?5@ 0049ad40     cubemap.obj
 0002:00000d74       ??_C@_0BL@EODFEKPD@?6Merged?5?$CFd?5detail?5faces?4?4?4?$AA@ 0049ad74     detail.obj
 0002:00000d90       ??_C@_0BK@ENPICNGK@Split?5face?5in?5merge?5list?$CB?$AA@ 0049ad90     detail.obj
 0002:00000dac       ??_C@_0BH@BFHFPFDM@Bad?5detail?5brush?5side?6?$AA@ 0049adac     detail.obj
 0002:00000dc4       ??_C@_0BD@PAPALJBM@Merging?5details?4?4?4?$AA@ 0049adc4     detail.obj
 0002:00000dd8       ??_C@_0BN@KHGACLOP@Find?5Visible?5Detail?5Sides?4?4?4?$AA@ 0049add8     detail.obj
 0002:00000df8       ??_C@_0L@MGHOLLP@done?5?$CI?$CFd?$CJ?6?$AA@ 0049adf8     detail.obj
 0002:00000e04       ??_C@_0BA@KHMLJCAD@Chop?5Details?4?4?4?$AA@ 0049ae04     detail.obj
 0002:00000e14       ??_C@_0L@NJIBFGO@detailvbsp?$AA@ 0049ae14     detailobjects.obj
 0002:00000e20       ??_C@_0M@BKGGJIMH@detail?4vbsp?$AA@ 0049ae20     detailobjects.obj
 0002:00000e2c       __real@38000100            0049ae2c     detailobjects.obj
 0002:00000e30       ??_C@_0DO@GOPKNNIB@Error?$CB?5Too?5many?5detail?5props?5emi@ 0049ae30     detailobjects.obj
 0002:00000e70       ??_C@_0CC@EGCFEIGF@Error?5loading?5studio?5model?5?$CC?$CFs?$CC?$CB@ 0049ae70     detailobjects.obj
 0002:00000e94       ??_C@_0M@BAHNLOII@detail_prop?$AA@ 0049ae94     detailobjects.obj
 0002:00000ea0       __real@bf50624dd2f1a9fc    0049aea0     detailobjects.obj
 0002:00000ea8       __real@3c340168            0049aea8     detailobjects.obj
 0002:00000eac       __real@3b808081            0049aeac     detailobjects.obj
 0002:00000eb0       ??_C@_0BC@IGEEGACB@detailOrientation?$AA@ 0049aeb0     detailobjects.obj
 0002:00000ec8       __real@3f91df46a2529d39    0049aec8     detailobjects.obj
 0002:00000ed0       ??_C@_08GKKMMBDC@maxAngle?$AA@ 0049aed0     detailobjects.obj
 0002:00000edc       ??_C@_08LNEHHDHD@minAngle?$AA@ 0049aedc     detailobjects.obj
 0002:00000ee8       __real@43340000            0049aee8     detailobjects.obj
 0002:00000eec       ??_C@_07OLKLDPGP@upright?$AA@ 0049aeec     detailobjects.obj
 0002:00000ef4       ??_C@_06LFKBJBLO@amount?$AA@ 0049aef4     detailobjects.obj
 0002:00000efc       ??_C@_0L@ELCGLDIA@shape_size?$AA@ 0049aefc     detailobjects.obj
 0002:00000f08       ??_C@_0M@KEOFPBDM@shape_angle?$AA@ 0049af08     detailobjects.obj
 0002:00000f18       __real@406fe00000000000    0049af18     detailobjects.obj
 0002:00000f20       ??_C@_04MGKPGJHA@sway?$AA@ 0049af20     detailobjects.obj
 0002:00000f28       ??_C@_0BC@KOPCEEPG@spriterandomscale?$AA@ 0049af28     detailobjects.obj
 0002:00000f3c       ??_C@_0M@ONLGMOD@?$CFf?5?$CFf?5?$CFf?5?$CFf?$AA@ 0049af3c     detailobjects.obj
 0002:00000f48       __real@41a00000            0049af48     detailobjects.obj
 0002:00000f4c       __real@c1200000            0049af4c     detailobjects.obj
 0002:00000f50       ??_C@_0L@ONKOJFJJ@spritesize?$AA@ 0049af50     detailobjects.obj
 0002:00000f5c       ??_C@_0DK@BNNOAIGN@Invalid?5arguments?5to?5?$CCsprite?$CC?5in@ 0049af5c     detailobjects.obj
 0002:00000f98       ??_C@_0P@NOPOKGBE@?$CFf?5?$CFf?5?$CFf?5?$CFf?5?$CFf?$AA@ 0049af98     detailobjects.obj
 0002:00000fa8       __real@44000000            0049afa8     detailobjects.obj
 0002:00000fac       __real@42800000            0049afac     detailobjects.obj
 0002:00000fb0       ??_C@_03NJKMHLPI@tri?$AA@  0049afb0     detailobjects.obj
 0002:00000fb4       ??_C@_05HCKPILGO@cross?$AA@ 0049afb4     detailobjects.obj
 0002:00000fbc       ??_C@_0N@FDIPGNCE@sprite_shape?$AA@ 0049afbc     detailobjects.obj
 0002:00000fcc       ??_C@_06DKHPLDLO@sprite?$AA@ 0049afcc     detailobjects.obj
 0002:00000fd4       ??_C@_05NCCFOPHA@model?$AA@ 0049afd4     detailobjects.obj
 0002:00000fdc       ??_C@_05IAEKHIAN@alpha?$AA@ 0049afdc     detailobjects.obj
 0002:00000fe4       ??_C@_0P@NFANEIDG@tex_total_size?$AA@ 0049afe4     detailobjects.obj
 0002:00000ff4       ??_C@_08LHFNKDML@tex_size?$AA@ 0049aff4     detailobjects.obj
 0002:00001000       ??_C@_06ODDDHALK@tex_ul?$AA@ 0049b000     detailobjects.obj
 0002:00001008       ??_C@_0M@KIMMAHMF@position_lr?$AA@ 0049b008     detailobjects.obj
 0002:00001014       ??_C@_0M@GPHKKAOF@position_ul?$AA@ 0049b014     detailobjects.obj
 0002:00001020       ??_C@_06GNEAMJOC@angles?$AA@ 0049b020     detailobjects.obj
 0002:00001028       ??_C@_06NHCMNMEH@origin?$AA@ 0049b028     detailobjects.obj
 0002:00001030       ??_C@_0BD@FCGBCNFD@prop_detail_sprite?$AA@ 0049b030     detailobjects.obj
 0002:00001044       ??_C@_0M@HMCBNKGG@prop_detail?$AA@ 0049b044     detailobjects.obj
 0002:00001050       ??_C@_0DB@BJBIMCHI@Material?5?$CFs?5uses?5unknown?5detail?5@ 0049b050     detailobjects.obj
 0002:00001084       ??_C@_0M@FFHDBFLG@?$CFdetailtype?$AA@ 0049b084     detailobjects.obj
 0002:00001090       ??_C@_0BI@JJLHFIKC@Placing?5detail?5props?5?3?5?$AA@ 0049b090     detailobjects.obj
 0002:000010a8       ??_C@_0EA@HKIIMBGB@Error?$CB?5Too?5many?5detail?5props?5on?5@ 0049b0a8     detailobjects.obj
 0002:000010e8       ??_C@_07HAFFKDBK@density?$AA@ 0049b0e8     detailobjects.obj
 0002:000010f0       __real@e753c21c            0049b0f0     disp_common.obj
 0002:000010f4       __real@6753c21c            0049b0f4     disp_common.obj
 0002:000010f8       __real@3c23d70a            0049b0f8     disp_common.obj
 0002:000010fc       ??_C@_0DK@GOGDGCAF@Found?5a?5displacement?5edge?5abutti@ 0049b0fc     disp_common.obj
 0002:00001138       ??_C@_0EM@MEODGKKJ@Warning?3?5invalid?5neighbor?5connec@ 0049b138     disp_common.obj
 0002:00001184       ??_C@_0DL@OBKBOEFP@Warning?3?5overflowed?5?$CFd?5displacem@ 0049b184     disp_common.obj
 0002:000011c0       __real@39800000            0049b1c0     disp_ivp.obj
 0002:000011c4       __real@39000000            0049b1c4     disp_ivp.obj
 0002:000011cc       ??_7CDispMeshEvent@@6B@    0049b1cc     disp_ivp.obj
 0002:000011d8       ??_C@_0N@KPONPEDB@surfaceprop2?$AA@ 0049b1d8     disp_ivp.obj
 0002:000011e8       __real@43bf4000            0049b1e8     disp_ivp.obj
 0002:000011ec       ??_C@_0DN@FLCJBOKC@Can?8t?5compile?5displacement?5physi@ 0049b1ec     disp_ivp.obj
 0002:0000122c       ??_C@_0DG@FCCGPPB@Displacement?5?$CFd?5has?5bad?5geometry@ 0049b22c     disp_ivp.obj
 0002:00001268       ??_C@_0EB@LNKDGLEF@Trying?5to?5create?5a?5non?9quad?5disp@ 0049b268     disp_vbsp.obj
 0002:000012b0       ??_C@_0FD@ILAEEOJA@Error?3?5displacement?5found?5on?5a?$CIn@ 0049b2b0     disp_vbsp.obj
 0002:00001304       __real@437fe666            0049b304     disp_vbsp.obj
 0002:00001308       ??_C@_0BG@HIJIAFNE@Displacement?5Alpha?5?3?5?$AA@ 0049b308     disp_vbsp.obj
 0002:00001320       ??_C@_0CG@HOOPHLIA@Finding?5lightmap?5sample?5position@ 0049b320     disp_vbsp.obj
 0002:00001348       ??_C@_0CD@BOCMJHJK@Finding?5displacement?5neighbors?4?4@ 0049b348     disp_vbsp.obj
 0002:0000136c       ??_C@_0CD@HHIGMIOB@HashVec?3?5point?5outside?5valid?5ran@ 0049b36c     faces.obj
 0002:00001390       ??_C@_0ED@JPHBHMOE@Too?5many?5unique?5verts?0?5max?5?$DN?5?$CFd?5@ 0049b390     faces.obj
 0002:000013d8       __real@3f847ae147ae147b    0049b3d8     faces.obj
 0002:000013e0       ??_C@_0EO@MBPOMJAM@Edge?5with?5too?5many?5vertices?5due?5@ 0049b3e0     faces.obj
 0002:00001430       __real@3e800000            0049b430     faces.obj
 0002:00001434       ??_C@_0CI@MMDKAFBP@SubdivideFace?3?5didn?8t?5split?5the?5@ 0049b434     faces.obj
 0002:0000145c       __real@3dcccccd            0049b45c     faces.obj
 0002:00001460       __real@c97423f0            0049b460     faces.obj
 0002:00001464       __real@497423f0            0049b464     faces.obj
 0002:00001468       ??_C@_0DD@FLIEHJFO@error?3?5material?5?$CFs?5doesn?8t?5have?5@ 0049b468     faces.obj
 0002:0000149c       ??_C@_09JCAKHELD@toolsskip?$AA@ 0049b49c     faces.obj
 0002:000014a8       ??_C@_06MEFHFNAK@nodraw?$AA@ 0049b4a8     faces.obj
 0002:000014b0       ??_C@_0BA@KCFHMCIO@?$CF5i?5subdivided?6?$AA@ 0049b4b0     faces.obj
 0002:000014c0       ??_C@_0M@LENHICMH@?$CF5i?5merged?6?$AA@ 0049b4c0     faces.obj
 0002:000014cc       ??_C@_0P@JLOIMJEC@?$CF5i?5makefaces?6?$AA@ 0049b4cc     faces.obj
 0002:000014dc       ??_C@_0BD@EJBJJFIN@?9?9?9?5MakeFaces?5?9?9?9?6?$AA@ 0049b4dc     faces.obj
 0002:000014f0       ??_C@_0EK@NDGGJICH@Too?5many?5t?9junctions?5to?5fix?5up?$CB?5@ 0049b4f0     faces.obj
 0002:0000153c       ??_C@_0BF@KDMEAIOC@?$CF5i?5bad?5start?5verts?6?$AA@ 0049b53c     faces.obj
 0002:00001554       ??_C@_0BP@FJGOMCCN@?$CF5i?5faces?5added?5by?5tjunctions?6?$AA@ 0049b554     faces.obj
 0002:00001574       ??_C@_0BP@NMMOJFFM@?$CF5i?5edges?5added?5by?5tjunctions?6?$AA@ 0049b574     faces.obj
 0002:00001594       ??_C@_0BH@MLJGLOGH@?$CF5i?5faces?5degenerated?6?$AA@ 0049b594     faces.obj
 0002:000015ac       ??_C@_0BH@PPDCHOOG@?$CF5i?5edges?5degenerated?6?$AA@ 0049b5ac     faces.obj
 0002:000015c4       ??_C@_0BD@HCGCCAKA@?$CFi?5unique?5from?5?$CFi?6?$AA@ 0049b5c4     faces.obj
 0002:000015d8       ??_C@_0BB@DDDNOAPE@?9?9?9?9?5tjunc?5?9?9?9?9?6?$AA@ 0049b5d8     faces.obj
 0002:000015ec       ??_C@_0BG@DMMDOHDA@?9?9?9?9?5snap?5verts?5?9?9?9?9?6?$AA@ 0049b5ec     faces.obj
 0002:00001604       ??_C@_0CB@LKNAAKJM@Too?5many?5edges?5in?5map?0?5max?5?$DN?$DN?5?$CFd@ 0049b604     faces.obj
 0002:00001628       ??_C@_0CF@MHKAGILO@?$CF6?43f?5?$CF6?43f?5?$CF6?43f?5?$CF6?43f?5?$CF6?43f?5?$CF6@ 0049b628     glfile.obj
 0002:00001650       __real@3f70101010101010    0049b650     glfile.obj
 0002:00001658       ??_C@_03PELOGHMK@?$CFi?6?$AA@ 0049b658     glfile.obj
 0002:0000165c       ??_C@_0P@EGNPLIPA@?$CF5i?5c_glfaces?6?$AA@ 0049b65c     glfile.obj
 0002:0000166c       ??_C@_0BB@MAHHKGJO@Couldn?8t?5open?5?$CFs?$AA@ 0049b66c     glfile.obj
 0002:00001680       ??_C@_0M@BBJDCBAD@Writing?5?$CFs?6?$AA@ 0049b680     glfile.obj
 0002:0000168c       ??_C@_07NLOFKJIL@?$CFs?$CFs?4gl?$AA@ 0049b68c     glfile.obj
 0002:00001698       ??_C@_0BJ@GLFIAOHK@?$CF6?43f?5?$CF6?43f?5?$CF6?43f?50?50?51?6?$AA@ 0049b698     ivp.obj
 0002:000016b4       ??_C@_0BJ@FHPKENPN@?$CF6?43f?5?$CF6?43f?5?$CF6?43f?50?51?50?6?$AA@ 0049b6b4     ivp.obj
 0002:000016d0       ??_C@_0BJ@MMONGPPJ@?$CF6?43f?5?$CF6?43f?5?$CF6?43f?51?50?50?6?$AA@ 0049b6d0     ivp.obj
 0002:000016ec       ??_C@_02NMHMJFKO@3?6?$AA@  0049b6ec     ivp.obj
 0002:000016f0       ??_C@_0P@FLEPLLPM@Writing?5?$CFs?4?4?4?6?$AA@ 0049b6f0     ivp.obj
 0002:00001704       ??_7CPhysCollisionEntrySolid@@6B@ 0049b704     ivp.obj
 0002:00001710       ??_7CPhysCollisionEntryStaticSolid@@6B@ 0049b710     ivp.obj
 0002:0000171c       ??_7CPhysCollisionEntryStaticMesh@@6B@ 0049b71c     ivp.obj
 0002:00001728       ??_7CPhysCollisionEntryFluid@@6B@ 0049b728     ivp.obj
 0002:00001730       ??_C@_0BE@PBEHMONM@maps?1?$CFs?1?$CFs_depth_?$CFi?$AA@ 0049b730     ivp.obj
 0002:00001744       ??_C@_0M@GPMGDIOD@$waterdepth?$AA@ 0049b744     ivp.obj
 0002:00001750       ??_C@_02IKAHHCAI@?$CFi?$AA@ 0049b750     ivp.obj
 0002:00001754       ??_C@_02GMLFBBN@wb?$AA@    0049b754     ivp.obj
 0002:00001758       ??_C@_0L@LCJFBGLL@?$CFs?$CF03d?4txt?$AA@ 0049b758     ivp.obj
 0002:00001764       ??_C@_0L@JEHPFMNB@?$CFs?$CF03d?4phy?$AA@ 0049b764     ivp.obj
 0002:00001770       ??_C@_07ILMJKKDI@collide?$AA@ 0049b770     ivp.obj
 0002:00001778       ??_C@_0L@CACCOGME@static?$CF02d?$AA@ 0049b778     ivp.obj
 0002:00001784       ??_C@_08MKICKDHE@mesh?$CF02d?$AA@ 0049b784     ivp.obj
 0002:00001790       ??_C@_09CLPCALOF@water?$CF02d?$AA@ 0049b790     ivp.obj
 0002:0000179c       __real@40400000            0049b79c     ivp.obj
 0002:000017a0       ??_C@_05ELAABIKM@water?$AA@ 0049b7a0     ivp.obj
 0002:000017a8       __real@378976f3            0049b7a8     ivp.obj
 0002:000017ac       ??_C@_07DLHCIBDH@default?$AA@ 0049b7ac     ivp.obj
 0002:000017b4       __real@44800000            0049b7b4     ivp.obj
 0002:000017b8       ??_C@_0L@GIBLANCP@?$CC?$CFs?$CC?5?$CC?$CFd?$CC?6?$AA@ 0049b7b8     ivp.obj
 0002:000017c4       ??_C@_0CB@EAKJLKK@Error?5writing?5collision?5data?5?$CFs?6@ 0049b7c4     ivp.obj
 0002:000017e8       ??_C@_0L@MCBCMFKE@?$CC?$CFs?$CC?5?$CC?$CFf?$CC?6?$AA@ 0049b7e8     ivp.obj
 0002:000017f4       ??_C@_02MBJIFMOJ@?$CC?6?$AA@ 0049b7f4     ivp.obj
 0002:000017f8       ??_C@_03JAIJOMNP@?$CFf?5?$AA@ 0049b7f8     ivp.obj
 0002:000017fc       ??_C@_06EGGGGBNL@?$CC?$CFs?$CC?5?$CC?$AA@ 0049b7fc     ivp.obj
 0002:00001804       ??_C@_01BJJEKLCA@?$CC?$AA@ 0049b804     ivp.obj
 0002:00001808       ??_C@_01LOCGONAA@?$AA?$AA@ 0049b808     ivp.obj
 0002:0000180c       ??_C@_08ODCIAOPM@contents?$AA@ 0049b80c     ivp.obj
 0002:00001818       ??_C@_05FKHKFDID@index?$AA@ 0049b818     ivp.obj
 0002:00001820       ??_C@_0P@OEGNPKIB@staticsolid?5?$HL?6?$AA@ 0049b820     ivp.obj
 0002:00001830       ??_C@_0BG@MIFABPEL@done?5?$CI?$CFd?$CJ?5?$CI?$CFd?5bytes?$CJ?6?$AA@ 0049b830     ivp.obj
 0002:00001848       ??_C@_0BB@PAFEBCLK@materialtable?5?$HL?6?$AA@ 0049b848     ivp.obj
 0002:0000185c       ??_C@_0BD@BFDMGGNB@virtualterrain?5?$HL?$HN?6?$AA@ 0049b85c     ivp.obj
 0002:00001870       ??_C@_0CE@ILLOBNPM@Building?5Physics?5collision?5data?4@ 0049b870     ivp.obj
 0002:00001894       ??_C@_0CK@PKCCIPMA@?$CB?$CB?$CB?5WARNING?3?5Can?8t?5build?5collisi@ 0049b894     ivp.obj
 0002:000018c0       ??_C@_0BF@PLKAEACL@VPhysicsCollision007?$AA@ 0049b8c0     ivp.obj
 0002:000018d8       ??_C@_06EMCPHFGM@volume?$AA@ 0049b8d8     ivp.obj
 0002:000018e0       ??_C@_0M@CPDICMCJ@surfaceprop?$AA@ 0049b8e0     ivp.obj
 0002:000018ec       ??_C@_04IJEANHEE@mass?$AA@ 0049b8ec     ivp.obj
 0002:000018f4       ??_C@_08NEDFMPNN@solid?5?$HL?6?$AA@ 0049b8f4     ivp.obj
 0002:00001900       ??_C@_0BA@DBPBOMKC@currentvelocity?$AA@ 0049b900     ivp.obj
 0002:00001910       ??_C@_0N@HDKAOPAI@surfaceplane?$AA@ 0049b910     ivp.obj
 0002:00001920       ??_C@_07IANOJGAO@damping?$AA@ 0049b920     ivp.obj
 0002:00001928       ??_C@_08EOKLBGBN@fluid?5?$HL?6?$AA@ 0049b928     ivp.obj
 0002:00001934       ??_C@_0CE@INBCPILM@Entity?5?$CFs?5?$CI?$CF?42f?5?$CF?42f?5?$CF?42f?$CJ?5leake@ 0049b934     leakfile.obj
 0002:00001958       ??_C@_0BE@ONJNDCHC@?$CF5i?5point?5linefile?6?$AA@ 0049b958     leakfile.obj
 0002:0000196c       ??_C@_09MALOBAAJ@?$CFf?5?$CFf?5?$CFf?6?$AA@ 0049b96c     leakfile.obj
 0002:00001978       ??_C@_0BC@ONJICBGP@Couldn?8t?5open?5?$CFs?6?$AA@ 0049b978     leakfile.obj
 0002:0000198c       ??_C@_06MBNJCGIN@?$CFs?4lin?$AA@ 0049b98c     leakfile.obj
 0002:00001994       ??_C@_0BC@LPEHNNEG@?9?9?9?5LeakFile?5?9?9?9?6?$AA@ 0049b994     leakfile.obj
 0002:000019a8       ??_C@_0BM@DFODNGPI@Areaportal?5leak?5?$CB?5File?3?5?$CFs?5?$AA@ 0049b9a8     leakfile.obj
 0002:000019c4       ??_C@_09CKEIHHKG@Wrote?5?$CFs?6?$AA@ 0049b9c4     leakfile.obj
 0002:000019d0       ??_C@_0BI@GJGMGOAA@Command?5Line?5found?3?5?$CFs?6?$AA@ 0049b9d0     loadcmdline.obj
 0002:000019e8       ??_C@_0BH@FPHGKPHF@?$CFs?1cfg?1commandline?4cfg?$AA@ 0049b9e8     loadcmdline.obj
 0002:00001a00       ??_C@_0M@FMINHJIF@CommandLine?$AA@ 0049ba00     loadcmdline.obj
 0002:00001a0c       ??_C@_0P@GHFPNOJB@bad?5allocation?$AA@ 0049ba0c     map.obj
 0002:00001a1c       ??_C@_0BD@JBACICKJ@Not?5a?5Parse?5error?$CB?$AA@ 0049ba1c     map.obj
 0002:00001a30       ??_C@_0CC@NMNJEPNA@Brush?5?$CFi?3?5?$CFs?6Side?5?$CFi?6Texture?3?5?$CFs@ 0049ba30     map.obj
 0002:00001a54       ??_C@_0BH@MAFNOPPO@Brush?5?$CFi?0?5Side?5?$CFi?3?5?$CFs?6?$AA@ 0049ba54     map.obj
 0002:00001a6c       ??_C@_0BA@GNFEIJEF@func_areaportal?$AA@ 0049ba6c     map.obj
 0002:00001a7c       ??_C@_0CF@HOACDEG@Brush?5?$CFi?3?5no?5visible?5sides?5on?5br@ 0049ba7c     map.obj
 0002:00001aa4       ??_C@_0BP@MBAIJKBK@Brush?5?$CFi?3?5bounds?5out?5of?5range?6?$AA@ 0049baa4     map.obj
 0002:00001ac4       ??_C@_03DMHICLNI@row?$AA@  0049bac4     map.obj
 0002:00001ac8       ??_C@_06INICNAFJ@smooth?$AA@ 0049bac8     map.obj
 0002:00001ad0       ??_C@_07KPOMEPOC@mintess?$AA@ 0049bad0     map.obj
 0002:00001ad8       ??_C@_05GECEPKB@flags?$AA@ 0049bad8     map.obj
 0002:00001ae0       ??_C@_0O@NBIGDJFH@startposition?$AA@ 0049bae0     map.obj
 0002:00001af0       ??_C@_05NKILLMJE@vaxis?$AA@ 0049baf0     map.obj
 0002:00001af8       ??_C@_05FMBPMODK@uaxis?$AA@ 0049baf8     map.obj
 0002:00001b00       ??_C@_05PLIADJJL@power?$AA@ 0049bb00     map.obj
 0002:00001b08       ??_C@_06BMHBIPLB@maxs?4z?$AA@ 0049bb08     map.obj
 0002:00001b10       ??_C@_06DHFMNMHC@maxs?4y?$AA@ 0049bb10     map.obj
 0002:00001b18       ??_C@_06COEHONDD@maxs?4x?$AA@ 0049bb18     map.obj
 0002:00001b20       ??_C@_06BPICGPPO@mins?4z?$AA@ 0049bb20     map.obj
 0002:00001b28       ??_C@_06DEKPDMDN@mins?4y?$AA@ 0049bb28     map.obj
 0002:00001b30       ??_C@_06CNLEANHM@mins?4x?$AA@ 0049bb30     map.obj
 0002:00001b38       ??_C@_05JGBIAEON@?$CF2?42f?$AA@ 0049bb38     map.obj
 0002:00001b40       ??_C@_0L@FEPNPAJD@targetname?$AA@ 0049bb40     map.obj
 0002:00001b4c       ??_C@_0BB@FIHILHEL@BackgroundBModel?$AA@ 0049bb4c     map.obj
 0002:00001b60       ??_C@_06JJLAMBGK@target?$AA@ 0049bb60     map.obj
 0002:00001b68       ??_C@_0BB@OGPBFIKB@smoothing_groups?$AA@ 0049bb68     map.obj
 0002:00001b7c       ??_C@_02EGCJHIOB@id?$AA@   0049bb7c     map.obj
 0002:00001b80       ??_C@_0BA@DFPKDOLK@luxel?5size?5of?50?$AA@ 0049bb80     map.obj
 0002:00001b90       ??_C@_0O@JMIJMGFN@lightmapscale?$AA@ 0049bb90     map.obj
 0002:00001ba0       ??_C@_0BK@EDNAAFKG@parsing?5V?5axis?5definition?$AA@ 0049bba0     map.obj
 0002:00001bbc       ??_C@_0BK@KJFGNIME@parsing?5U?5axis?5definition?$AA@ 0049bbbc     map.obj
 0002:00001bd8       ??_C@_0BB@LHCKFDFE@?$FL?$CFf?5?$CFf?5?$CFf?5?$CFf?$FN?5?$CFf?$AA@ 0049bbd8     map.obj
 0002:00001bec       ??_C@_08KNOEMJMM@material?$AA@ 0049bbec     map.obj
 0002:00001bf8       ??_C@_0BJ@MKMLNGKE@parsing?5plane?5definition?$AA@ 0049bbf8     map.obj
 0002:00001c14       ??_C@_0CB@BIIACPHF@?$CI?$CFf?5?$CFf?5?$CFf?$CJ?5?$CI?$CFf?5?$CFf?5?$CFf?$CJ?5?$CI?$CFf?5?$CFf?5?$CFf?$CJ@ 0049bc14     map.obj
 0002:00001c38       ??_C@_05MAIECAHP@plane?$AA@ 0049bc38     map.obj
 0002:00001c40       ??_C@_01CELHOKLL@?$HN?$AA@ 0049bc40     map.obj
 0002:00001c44       ??_C@_01HCONENDN@?$HL?$AA@ 0049bc44     map.obj
 0002:00001c48       ??_C@_0DG@GPKBCONA@ParseDispInfoChunk?3?5nummapdispin@ 0049bc48     map.obj
 0002:00001c80       ??_C@_0P@OPCJGGAO@MAX_MAP_PLANES?$AA@ 0049bc80     map.obj
 0002:00001c90       ??_C@_0BH@HHAHLGNM@FloatPlane?3?5bad?5normal?$AA@ 0049bc90     map.obj
 0002:00001ca8       __real@3727c5ac            0049bca8     map.obj
 0002:00001cac       ??_C@_0O@LBPCPJAL@triangle_tags?$AA@ 0049bcac     map.obj
 0002:00001cbc       ??_C@_06HKCDBMPA@alphas?$AA@ 0049bcbc     map.obj
 0002:00001cc4       ??_C@_07EALNHAIO@offsets?$AA@ 0049bcc4     map.obj
 0002:00001ccc       ??_C@_09IIHGAIPH@distances?$AA@ 0049bccc     map.obj
 0002:00001cd8       ??_C@_07MDEPDJDC@normals?$AA@ 0049bcd8     map.obj
 0002:00001ce0       ??_C@_0BF@IIALCAPD@plane?5with?5no?5normal?$AA@ 0049bce0     map.obj
 0002:00001cf8       ??_C@_0P@JEIPHHHE@mirrored?5plane?$AA@ 0049bcf8     map.obj
 0002:00001d08       ??_C@_0BA@IDGBHDDK@duplicate?5plane?$AA@ 0049bd08     map.obj
 0002:00001d18       ??_C@_08OAJLBCOI@dispinfo?$AA@ 0049bd18     map.obj
 0002:00001d24       ??_C@_0BD@MGJMIOFL@MAX_MAP_BRUSHSIDES?$AA@ 0049bd24     map.obj
 0002:00001d38       __real@41800000            0049bd38     map.obj
 0002:00001d3c       ??_C@_05KJODHHKF@sides?$AA@ 0049bd3c     map.obj
 0002:00001d44       ??_C@_03CGENABJP@uv3?$AA@  0049bd44     map.obj
 0002:00001d48       ??_C@_03DPFGDANO@uv2?$AA@  0049bd48     map.obj
 0002:00001d4c       ??_C@_03BEHLGDBN@uv1?$AA@  0049bd4c     map.obj
 0002:00001d50       ??_C@_03NGAFCFM@uv0?$AA@   0049bd50     map.obj
 0002:00001d54       ??_C@_0M@CBNMGMHG@BasisNormal?$AA@ 0049bd54     map.obj
 0002:00001d60       ??_C@_06DAKFJGGD@BasisV?$AA@ 0049bd60     map.obj
 0002:00001d68       ??_C@_06BLIIMFKA@BasisU?$AA@ 0049bd68     map.obj
 0002:00001d70       ??_C@_0M@HMELADEK@BasisOrigin?$AA@ 0049bd70     map.obj
 0002:00001d7c       ??_C@_04NBAIMGMF@EndV?$AA@ 0049bd7c     map.obj
 0002:00001d84       ??_C@_06DKGAJAMI@StartV?$AA@ 0049bd84     map.obj
 0002:00001d8c       ??_C@_04PKCFJFAG@EndU?$AA@ 0049bd8c     map.obj
 0002:00001d94       ??_C@_06BBENMDAL@StartU?$AA@ 0049bd94     map.obj
 0002:00001d9c       ??_C@_0DF@DBGEDADE@Overlay?5Material?5Name?5?$CI?$CFs?$CJ?5?$DO?5OVE@ 0049bd9c     map.obj
 0002:00001dd4       ??_C@_0M@GHHOADBD@overlaydata?$AA@ 0049bdd4     map.obj
 0002:00001de0       ??_C@_08DIEBNEND@?$CFi?5?$CFi?5?$CFi?$AA@ 0049bde0     map.obj
 0002:00001dec       ??_C@_0CO@GOILIMJA@Brush?5?$CFi?3?5origin?5brushes?5not?5all@ 0049bdec     map.obj
 0002:00001e1c       ??_C@_04JGNFNGGK@side?$AA@ 0049be1c     map.obj
 0002:00001e24       ??_C@_0CB@FJNNNLDI@nummapbrushes?5?$DN?$DN?5MAX_MAP_BRUSHES@ 0049be24     map.obj
 0002:00001e48       ??_C@_0N@KGPHONEC@portalnumber?$AA@ 0049be48     map.obj
 0002:00001e58       ??_C@_0DG@LEHLNDPI@Entity?5?$CFi?3?5func_areaportal?5can?5o@ 0049be58     map.obj
 0002:00001e90       ??_C@_0BH@NALGDPIA@info_no_dynamic_shadow?$AA@ 0049be90     map.obj
 0002:00001ea8       ??_C@_0BI@OMCMPAEO@info_overlay_transition?$AA@ 0049bea8     map.obj
 0002:00001ec0       ??_C@_09DFIMFMKC@OverlayID?$AA@ 0049bec0     map.obj
 0002:00001ecc       ??_C@_0BG@CNGIAIJF@info_overlay_accessor?$AA@ 0049becc     map.obj
 0002:00001ee4       ??_C@_0N@BGKIAKKP@info_overlay?$AA@ 0049bee4     map.obj
 0002:00001ef4       ??_C@_0O@LNCJIGDK@test_sidelist?$AA@ 0049bef4     map.obj
 0002:00001f04       ??_C@_0M@EDMIMGHH@cubemapsize?$AA@ 0049bf04     map.obj
 0002:00001f10       ??_C@_0M@OEALFABH@info_ladder?$AA@ 0049bf10     map.obj
 0002:00001f1c       ??_C@_0M@OOKLDPAJ@func_ladder?$AA@ 0049bf1c     map.obj
 0002:00001f28       ??_C@_0BA@EEDDHHGA@func_viscluster?$AA@ 0049bf28     map.obj
 0002:00001f38       ??_C@_0M@MMLAJCHD@func_detail?$AA@ 0049bf38     map.obj
 0002:00001f44       ??_C@_0L@BGKEEOJO@maxdxlevel?$AA@ 0049bf44     map.obj
 0002:00001f50       ??_C@_0L@NKKJDFJB@mindxlevel?$AA@ 0049bf50     map.obj
 0002:00001f5c       ??_C@_0BC@FJHAELML@overlaytransition?$AA@ 0049bf5c     map.obj
 0002:00001f70       ??_C@_0M@EAJPACGF@connections?$AA@ 0049bf70     map.obj
 0002:00001f7c       ??_C@_05OPIONHBI@solid?$AA@ 0049bf7c     map.obj
 0002:00001f84       ??_C@_0CB@GIFGAPCN@num_entities?5?$DN?$DN?5MAX_MAP_ENTITIES@ 0049bf84     map.obj
 0002:00001fa8       ??_C@_0CO@GHCPCDGG@size?3?5?$CF5?40f?0?$CF5?40f?0?$CF5?40f?5to?5?$CF5?40f@ 0049bfa8     map.obj
 0002:00001fd8       ??_C@_0BB@PBBAPMMD@?$CF5i?5areaportals?6?$AA@ 0049bfd8     map.obj
 0002:00001fec       ??_C@_0M@FHMKEEFP@?$CF5i?5planes?6?$AA@ 0049bfec     map.obj
 0002:00001ff8       ??_C@_0O@HPNIHHPI@?$CF5i?5entities?6?$AA@ 0049bff8     map.obj
 0002:00002008       ??_C@_0BA@HPIFLHBK@?$CF5i?5edgebevels?6?$AA@ 0049c008     map.obj
 0002:00002018       ??_C@_0P@FECCOIAO@?$CF5i?5boxbevels?6?$AA@ 0049c018     map.obj
 0002:00002028       ??_C@_0BB@LDGJKFDM@?$CF5i?5total?5sides?6?$AA@ 0049c028     map.obj
 0002:0000203c       ??_C@_0BB@HLCBGCLL@?$CF5i?5clipbrushes?6?$AA@ 0049c03c     map.obj
 0002:00002050       ??_C@_0BH@GDLKMEGB@Error?5opening?5?$CFs?3?5?$CFs?4?6?$AA@ 0049c050     map.obj
 0002:00002068       ??_C@_06GOJKNBFM@entity?$AA@ 0049c068     map.obj
 0002:00002070       ??_C@_05MCBCHHEJ@world?$AA@ 0049c070     map.obj
 0002:00002078       ??_C@_0M@LGGMODLI@Loading?5?$CFs?6?$AA@ 0049c078     map.obj
 0002:00002084       ??_C@_0CD@CLEPENAJ@Infinite?5recursion?5in?5patch?5file@ 0049c084     materialpatch.obj
 0002:000020a8       ??_C@_07CLEHDIEJ@replace?$AA@ 0049c0a8     materialpatch.obj
 0002:000020b0       ??_C@_06OAOPNKHP@insert?$AA@ 0049c0b0     materialpatch.obj
 0002:000020b8       ??_C@_03JLLDDLCC@vmt?$AA@  0049c0b8     materialpatch.obj
 0002:000020bc       ??_C@_07FHOHOHLG@include?$AA@ 0049c0bc     materialpatch.obj
 0002:000020c4       ??_C@_05OCKFKOHN@patch?$AA@ 0049c0c4     materialpatch.obj
 0002:000020cc       ??_C@_0BB@LDFMOGIJ@materials?1?$CFs?4vmt?$AA@ 0049c0cc     materialpatch.obj
 0002:000020e0       ??_C@_04EPOOCEMM@blah?$AA@ 0049c0e0     materialpatch.obj
 0002:000020e8       ??_C@_0CG@LIACKKOF@Couldn?8t?5allocate?5KeyValues?5for?5@ 0049c0e8     materialpatch.obj
 0002:00002110       ??_C@_07DPNAEFKO@AllMaps?$AA@ 0049c110     materialsub.obj
 0002:00002118       ??_C@_0CA@HOILNHCB@Failed?5to?5load?5KeyValues?5file?$CB?6?$AA@ 0049c118     materialsub.obj
 0002:00002138       ??_C@_0O@DMIKEJDC@File?5path?3?5?$CFs?$AA@ 0049c138     materialsub.obj
 0002:00002148       ??_C@_0BF@HKOHJKOO@MaterialReplacements?$AA@ 0049c148     materialsub.obj
 0002:00002160       ??_C@_0BG@MMHIEDBE@?$CFscfg?2materialsub?4cfg?$AA@ 0049c160     materialsub.obj
 0002:00002178       ??_C@_0BK@GFEEBONO@Loading?5Replacement?5Keys?6?$AA@ 0049c178     materialsub.obj
 0002:00002198       ??_7bad_alloc@std@@6B@     0049c198     mstristrip.obj
 0002:000021a4       ??_7logic_error@std@@6B@   0049c1a4     mstristrip.obj
 0002:000021b0       ??_7length_error@std@@6B@  0049c1b0     mstristrip.obj
 0002:000021b8       ??_C@_0CN@MHFNKKHI@g_numvertnormals?5?$DN?$DN?5MAX_MAP_VERT@ 0049c1b8     normals.obj
 0002:000021e8       ??_C@_0DJ@NAANFADH@g_numvertnormalindices?5?$DN?$DN?5MAX_MA@ 0049c1e8     normals.obj
 0002:00002228       ??_C@_0FD@LPHBLOPA@Overlay?5touching?5too?5many?5faces?5@ 0049c228     overlay.obj
 0002:0000227c       ??_C@_0CJ@LIPKIIKH@Too?5Many?5Overlays?$CB?6MAX_MAP_OVERL@ 0049c27c     overlay.obj
 0002:000022a8       ??_C@_0FJ@IINLDJCB@Water?5Overlay?5touching?5too?5many?5@ 0049c2a8     overlay.obj
 0002:00002304       ??_C@_0DE@LMCOJDDK@Too?5many?5water?5overlays?$CB?6MAX_MAP@ 0049c304     overlay.obj
 0002:00002338       ??_C@_0DP@LKIFHCNF@Overlay?5Material?5Name?5?$CI?$CFs?$CJ?5too?5l@ 0049c338     overlay.obj
 0002:00002378       ??_C@_0DJ@OHEEDLDK@Overlay?5?$CI?$CFs?$CJ?5at?5?$CFf?5?$CFf?5?$CFf?5has?5inv@ 0049c378     overlay.obj
 0002:000023b4       ??_C@_0M@MCPJDFDC@RenderOrder?$AA@ 0049c3b4     overlay.obj
 0002:000023c0       ??_C@_0M@KKMBKHAJ@fademaxdist?$AA@ 0049c3c0     overlay.obj
 0002:000023cc       ??_C@_0M@EMKBAIOI@fademindist?$AA@ 0049c3cc     overlay.obj
 0002:000023d8       ??_C@_0N@IBCKMFJP@VPHYSICS?4DLL?$AA@ 0049c3d8     physdll.obj
 0002:000023e8       ??_C@_0BP@LIHEBGBH@Portal_EntityFlood?3?5not?5a?5leaf?$AA@ 0049c3e8     portals.obj
 0002:00002408       ??_C@_0CD@JFIEIEKB@AddPortalToNode?3?5allready?5includ@ 0049c408     portals.obj
 0002:0000242c       ??_C@_0CP@CAKEOEAK@RemovePortalFromNode?3?5portal?5not@ 0049c42c     portals.obj
 0002:0000245c       ??_C@_0CJ@IIKHMOPG@RemovePortalFromNode?3?5portal?5not@ 0049c45c     portals.obj
 0002:00002488       ??_C@_0CL@GHKIMALJ@entity?5reached?5from?5outside?5?9?9?5n@ 0049c488     portals.obj
 0002:000024b4       ??_C@_0CD@DNPJGLB@no?5entities?5in?5open?5?9?9?5no?5fillin@ 0049c4b4     portals.obj
 0002:000024d8       ??_C@_0BC@IHPKIKNE@info_player_start?$AA@ 0049c4d8     portals.obj
 0002:000024ec       ??_C@_0BH@HLBIBACP@?9?9?9?5FloodEntities?5?9?9?9?6?$AA@ 0049c4ec     portals.obj
 0002:00002504       ??_C@_0DM@NNFAMLGB@WARNING?3?5areaportal?5entity?5?$CFi?5?$CIb@ 0049c504     portals.obj
 0002:00002540       ??_C@_0DF@LBOOPFLN@?6Brush?5?$CFi?3?5areaportal?5brush?5does@ 0049c540     portals.obj
 0002:00002578       __real@401921fb60000000    0049c578     portals.obj
 0002:00002580       __real@401921fb54442d18    0049c580     portals.obj
 0002:00002588       ??_C@_0DK@BCHHFABC@FindUniquePoints?3?5overflowed?5uni@ 0049c588     portals.obj
 0002:000025c4       __real@459c4000            0049c5c4     portals.obj
 0002:000025c8       ??_C@_0L@PBOEMMBA@?$CF5i?5areas?6?$AA@ 0049c5c8     portals.obj
 0002:000025d4       ??_C@_0BE@NMCFKNEG@Processing?5areas?4?4?4?$AA@ 0049c5d4     portals.obj
 0002:000025e8       ??_C@_0BE@PLEMBIKP@?9?9?9?5FloodAreas?5?9?9?9?6?$AA@ 0049c5e8     portals.obj
 0002:000025fc       ??_C@_0BC@BLMODMPJ@?$CF5i?5inside?5leafs?6?$AA@ 0049c5fc     portals.obj
 0002:00002610       ??_C@_0BC@DDIBNNOE@?$CF5i?5leafs?5filled?6?$AA@ 0049c610     portals.obj
 0002:00002624       ??_C@_0BB@EOCBGIME@?$CF5i?5solid?5leafs?6?$AA@ 0049c624     portals.obj
 0002:00002638       ??_C@_0BF@HAKMMJNB@?9?9?9?5FillOutside?5?9?9?9?6?$AA@ 0049c638     portals.obj
 0002:00002650       ??_C@_0CD@BKLIBDI@CutNodePortals_r?3?5mislinked?5port@ 0049c650     portals.obj
 0002:00002674       __real@41000000            0049c674     portals.obj
 0002:00002678       ??_C@_0EB@FMHMLHFO@WARNING?3?5BSP?5node?5with?5unbounded@ 0049c678     portals.obj
 0002:000026bc       ??_C@_0N@IBDKDIFK@?$CI?$CFf?0?5?$CFf?0?5?$CFf?$CJ?$AA@ 0049c6bc     portals.obj
 0002:000026cc       ??_C@_0L@EKPDOEAF@?$DMNO?5BRUSH?$DO?$AA@ 0049c6cc     portals.obj
 0002:000026d8       __real@46801000            0049c6d8     portals.obj
 0002:000026dc       __real@c6801000            0049c6dc     portals.obj
 0002:000026e0       ??_C@_0CA@LKBBLMDG@WARNING?3?5node?5without?5a?5volume?6?$AA@ 0049c6e0     portals.obj
 0002:00002700       ??_C@_0EH@PAHANHPO@MAX_MAP_PORTALVERTS?5?$CIprobably?5a?5@ 0049c700     portals.obj
 0002:00002748       ??_C@_0DJ@GJPMBHMF@Warning?3?5area?5portal?5has?5?$CFd?5vert@ 0049c748     portals.obj
 0002:00002784       ??_C@_0BE@IDCALIKK@?$CF5i?5numareaportals?6?$AA@ 0049c784     portals.obj
 0002:00002798       ??_C@_0O@GFHNKNIP@?$CF5i?5numareas?6?$AA@ 0049c798     portals.obj
 0002:000027a8       ??_C@_0FB@FBBGELIA@Map?5is?5split?5into?5too?5many?5uniqu@ 0049c7a8     portals.obj
 0002:000027fc       ??_C@_02PHMGELLB@?6?6?$AA@ 0049c7fc     portals.obj
 0002:00002800       ??_C@_0L@MOODCIAB@Brush?5?$CFd?3?5?$AA@ 0049c800     portals.obj
 0002:0000280c       ??_C@_0BG@GECLGKNP@Candidate?5brush?5IDs?3?5?$AA@ 0049c80c     portals.obj
 0002:00002828       ??_C@_0EN@FHDPIEOF@Check?5for?5a?5huge?5brush?5enclosing@ 0049c828     portals.obj
 0002:00002878       ??_C@_0FD@FPKNDADB@This?5means?5that?5none?5of?5the?5brus@ 0049c878     portals.obj
 0002:000028cc       ??_C@_0DF@BEFAKAHB@viscontents?5?$CInode?50?5contents?5?$FO?5n@ 0049c8cc     portals.obj
 0002:00002904       ??_C@_0BF@IKJGHNIN@Leaf?51?5contents?3?5?$CFs?6?$AA@ 0049c904     portals.obj
 0002:0000291c       ??_C@_0BF@CEPOOMBM@Leaf?50?5contents?3?5?$CFs?6?$AA@ 0049c91c     portals.obj
 0002:00002938       ??_C@_0GJ@EOHGFIKL@?6FindPortalSide?3?5Couldn?8t?5find?5a@ 0049c938     portals.obj
 0002:000029a4       ??_C@_0DH@NFIHIFFG@?$CK?$CK?$CK?5Suppressing?5further?5FindPort@ 0049c9a4     portals.obj
 0002:000029dc       ??_C@_0CE@DFFGJHBH@WARNING?3?5side?5not?5found?5for?5port@ 0049c9dc     portals.obj
 0002:00002a00       __real@49742400            0049ca00     portals.obj
 0002:00002a04       ??_C@_0BK@GOPFEKFA@?9?9?9?5MarkVisibleSides?5?9?9?9?6?$AA@ 0049ca04     portals.obj
 0002:00002a20       ??_C@_03JLNFKLOC@?$CFi?5?$AA@ 0049ca20     prtfile.obj
 0002:00002a24       ??_C@_02KCKGHPCA@?$CJ?5?$AA@ 0049ca24     prtfile.obj
 0002:00002a28       ??_C@_01ODHLEDKK@?$CI?$AA@ 0049ca28     prtfile.obj
 0002:00002a2c       ??_C@_09IKGGOGBI@?$CFi?5?$CFi?5?$CFi?5?$AA@ 0049ca2c     prtfile.obj
 0002:00002a38       __real@3fefae147ae147ae    0049ca38     prtfile.obj
 0002:00002a40       ??_C@_0BA@IGLBFDOH@?$CF5i?5visportals?6?$AA@ 0049ca40     prtfile.obj
 0002:00002a50       ??_C@_0BB@EDOGNKFI@?$CF5i?5visclusters?6?$AA@ 0049ca50     prtfile.obj
 0002:00002a64       ??_C@_03OFAPEBGM@?$CFs?6?$AA@ 0049ca64     prtfile.obj
 0002:00002a68       ??_C@_04MNCCIBNO@PRT1?$AA@ 0049ca68     prtfile.obj
 0002:00002a70       ??_C@_0BB@KKAAPNA@Error?5opening?5?$CFs?$AA@ 0049ca70     prtfile.obj
 0002:00002a84       ??_C@_0CB@PPJANFIF@Building?5visibility?5clusters?4?4?4?6@ 0049ca84     prtfile.obj
 0002:00002aa8       ??_C@_0O@LMKEHAHJ@writing?5?$CFs?4?4?4?$AA@ 0049caa8     prtfile.obj
 0002:00002ab8       ??_C@_06HLEIHIOA@?$CFs?4prt?$AA@ 0049cab8     prtfile.obj
 0002:00002ac0       ??_C@_0BJ@PPHGGLDL@?9?9?9?5WritePortalFile?5?9?9?9?6?$AA@ 0049cac0     prtfile.obj
 0002:00002adc       ??_C@_0P@PAEMGLHD@VFileSystem017?$AA@ 0049cadc     scratchpad3d.obj
 0002:00002aec       ??_C@_0BB@DHLFOMEN@filesystem_stdio?$AA@ 0049caec     scratchpad3d.obj
 0002:00002b00       ??_C@_02JDPG@rb?$AA@       0049cb00     scratchpad3d.obj
 0002:00002b04       __real@42c80000            0049cb04     scratchpad3d.obj
 0002:00002b10       ??_C@_0M@IHGNALJG@allowstatic?$AA@ 0049cb10     staticprop.obj
 0002:00002b1c       ??_C@_09OMCEPKNN@prop_data?$AA@ 0049cb1c     staticprop.obj
 0002:00002b28       ??_C@_0CP@JIJCKMIO@Error?5Vertex?5File?5?$CFs?5checksum?5?$CFd@ 0049cb28     staticprop.obj
 0002:00002b58       ??_C@_0CO@EPFJDMKK@Error?5Vertex?5File?5?$CFs?5version?5?$CFd?5@ 0049cb58     staticprop.obj
 0002:00002b88       ??_C@_0CJ@LHDPNPII@Error?5Vertex?5File?5?$CFs?5id?5?$CFd?5shoul@ 0049cb88     staticprop.obj
 0002:00002bb4       ??_C@_0BP@FEBLCPLO@Bad?5size?5for?5vertex?5data?5?$CC?$CFs?$CC?6?$AA@ 0049cbb4     staticprop.obj
 0002:00002bd4       ??_C@_0CB@HKBKLBIF@Unable?5to?5load?5vertex?5data?5?$CC?$CFs?$CC?6@ 0049cbd4     staticprop.obj
 0002:00002bf8       ??_C@_04FIJFNMIG@?4vvd?$AA@ 0049cbf8     staticprop.obj
 0002:00002c00       ??_C@_07FLCBLKFO@models?1?$AA@ 0049cc00     staticprop.obj
 0002:00002c08       ??_C@_0GC@BHCCOAEK@Error?$CB?5?$CFs?5using?5model?5?$CC?$CFs?$CC?0?5whic@ 0049cc08     staticprop.obj
 0002:00002c70       ??_C@_0EP@HKFHEIGH@Error?$CB?5To?5use?5model?5?$CC?$CFs?$CC?6?5?5?5?5?5?5w@ 0049cc70     staticprop.obj
 0002:00002cc0       ??_C@_04LGCIMDIF@IDAG?$AA@ 0049ccc0     staticprop.obj
 0002:00002cc8       ??_C@_04MIGFPFAJ@IDST?$AA@ 0049ccc8     staticprop.obj
 0002:00002cd0       ??_C@_0BD@IMPDAIMD@staticprop?$CF03d?4txt?$AA@ 0049ccd0     staticprop.obj
 0002:00002ce4       ??_C@_0BH@KOMFDDOL@Bad?5geometry?5on?5?$CC?$CFs?$CC?$CB?6?$AA@ 0049cce4     staticprop.obj
 0002:00002cfc       ??_C@_0M@FOINAKII@prop_static?$AA@ 0049ccfc     staticprop.obj
 0002:00002d08       ??_C@_0DD@EDIJEFGC@Static?5prop?5?$CFs?5outside?5the?5map?5?$CI@ 0049cd08     staticprop.obj
 0002:00002d3c       ??_C@_0P@MIILKHBP@lightingorigin?$AA@ 0049cd3c     staticprop.obj
 0002:00002d4c       ??_C@_09IPECPEGI@fadescale?$AA@ 0049cd4c     staticprop.obj
 0002:00002d58       ??_C@_0BA@MNGAFPDH@screenspacefade?$AA@ 0049cd58     staticprop.obj
 0002:00002d68       ??_C@_0BF@JGIMAFIJ@disableselfshadowing?$AA@ 0049cd68     staticprop.obj
 0002:00002d80       ??_C@_0BG@ODLFPOKJ@disablevertexlighting?$AA@ 0049cd80     staticprop.obj
 0002:00002d98       ??_C@_0P@KAMOLJAG@disableshadows?$AA@ 0049cd98     staticprop.obj
 0002:00002da8       ??_C@_0O@MANKHPFF@ignorenormals?$AA@ 0049cda8     staticprop.obj
 0002:00002db8       ??_C@_04NHPAFEHJ@skin?$AA@ 0049cdb8     staticprop.obj
 0002:00002dc0       ??_C@_0M@NGBNJMIL@static_prop?$AA@ 0049cdc0     staticprop.obj
 0002:00002dcc       ??_C@_0O@EJEKIFNM@info_lighting?$AA@ 0049cdcc     staticprop.obj
 0002:00002ddc       ??_C@_01HIHLOKLC@1?$AA@    0049cddc     textures.obj
 0002:00002de0       ??_C@_04LOAJBDKD@true?$AA@ 0049cde0     textures.obj
 0002:00002de8       ??_C@_0O@IFAMPFIH@?$CFcompileSlime?$AA@ 0049cde8     textures.obj
 0002:00002df8       ??_C@_0N@KOCEKFOI@UnlitGeneric?$AA@ 0049cdf8     textures.obj
 0002:00002e08       ??_C@_0BC@CEHNDAAO@?$CFcompileKeepLight?$AA@ 0049ce08     textures.obj
 0002:00002e1c       ??_C@_0P@OENLNILK@?$CFcompileDetail?$AA@ 0049ce1c     textures.obj
 0002:00002e2c       ??_C@_0BB@OCMEMLKF@?$CFcompileBlockLOS?$AA@ 0049ce2c     textures.obj
 0002:00002e40       ??_C@_0BB@NGKLKFOF@?$CFcompileNonsolid?$AA@ 0049ce40     textures.obj
 0002:00002e54       ??_C@_0BC@DEINFPLN@?$CFcompileInvisible?$AA@ 0049ce54     textures.obj
 0002:00002e68       ??_C@_0P@KFJIHOEH@?$CFcompileNoDraw?$AA@ 0049ce68     textures.obj
 0002:00002e78       ??_C@_0BE@PDMIKGIN@?$CFcompilePassBullets?$AA@ 0049ce78     textures.obj
 0002:00002e8c       ??_C@_09BFAOOCNM@?$CFnoPortal?$AA@ 0049ce8c     textures.obj
 0002:00002e98       ??_C@_0P@MGMAHFMA@?$CFcompileLadder?$AA@ 0049ce98     textures.obj
 0002:00002ea8       ??_C@_0O@EPOOCJEM@?$CFcompileWater?$AA@ 0049cea8     textures.obj
 0002:00002eb8       ??_C@_0BA@GKDMGPNA@?$CFcompileNoLight?$AA@ 0049ceb8     textures.obj
 0002:00002ec8       ??_C@_0BA@DHJNKBAM@?$CFcompileTrigger?$AA@ 0049cec8     textures.obj
 0002:00002ed8       ??_C@_0P@GNMDKOGB@?$CFcompileNoChop?$AA@ 0049ced8     textures.obj
 0002:00002ee8       ??_C@_0BA@DEIOCLID@?$CFcompileNpcClip?$AA@ 0049cee8     textures.obj
 0002:00002ef8       ??_C@_0M@FALIBANK@?$CFplayerClip?$AA@ 0049cef8     textures.obj
 0002:00002f04       ??_C@_0N@MLJBDBBL@?$CFcompileClip?$AA@ 0049cf04     textures.obj
 0002:00002f14       ??_C@_0P@HHCCNAAO@?$CFcompileOrigin?$AA@ 0049cf14     textures.obj
 0002:00002f24       ??_C@_0N@DGKGJOCA@?$CFcompileSkip?$AA@ 0049cf24     textures.obj
 0002:00002f34       ??_C@_0N@OKLMCDLJ@?$CFcompileHint?$AA@ 0049cf34     textures.obj
 0002:00002f44       ??_C@_0O@MKHJHEJH@?$CFcompile2DSky?$AA@ 0049cf44     textures.obj
 0002:00002f54       ??_C@_0M@LPBDLFMH@?$CFcompileSky?$AA@ 0049cf54     textures.obj
 0002:00002f60       ??_C@_0BJ@FGKNAKCJ@Material?5not?5found?$CB?3?5?$CFs?6?$AA@ 0049cf60     textures.obj
 0002:00002f7c       ??_C@_0CB@NKDKDMKG@Too?5many?5unique?5textures?0?5max?5?$CFd@ 0049cf7c     textures.obj
 0002:00002fa0       ??_C@_0DK@FPPKOMPC@Can?8t?5find?5surfaceprop?5?$CFs?5for?5ma@ 0049cfa0     textures.obj
 0002:00002fdc       ??_C@_0N@CIFOINKH@$surfaceprop?$AA@ 0049cfdc     textures.obj
 0002:00002fec       ??_C@_0DP@BKEKMNEN@Can?8t?5find?5surfacepropblend?5?$CFs?5f@ 0049cfec     textures.obj
 0002:0000302c       ??_C@_0O@KFOKDMLH@$surfaceprop2?$AA@ 0049d02c     textures.obj
 0002:0000303c       ??_C@_0CD@GMKDFIIB@WARNING?3?5material?5not?5found?3?5?$CC?$CFs@ 0049d03c     textures.obj
 0002:00003060       ??_C@_0CM@BNGGNJNC@Too?5many?5unique?5texture?5mappings@ 0049d060     textures.obj
 0002:0000308c       ??_C@_04DAMGJPCA@file?$AA@ 0049d08c     textures.obj
 0002:00003094       ??_C@_04FOKBGDA@GAME?$AA@  0049d094     textures.obj
 0002:0000309c       ??_C@_0CH@KEKFIONI@scripts?1surfaceproperties_manife@ 0049d09c     textures.obj
 0002:000030c4       ??_C@_0BI@ENHKJIPO@VPhysicsSurfaceProps001?$AA@ 0049d0c4     textures.obj
 0002:000030e0       ??_C@_0GL@JNBMOEPF@FindOrCreateTexInfo?3?5?5Tried?5to?5c@ 0049d0e0     textures.obj
 0002:00003150       __real@400921fb54442d18    0049d150     textures.obj
 0002:00003158       __real@3bb60b61            0049d158     textures.obj
 0002:0000315c       __real@43870000            0049d15c     textures.obj
 0002:00003160       __real@42b40000            0049d160     textures.obj
 0002:00003164       __real@3d800000            0049d164     textures.obj
 0002:00003168       ??_C@_0BM@PHNCGPMA@PruneNodes?3?5node?9?$DObrushlist?$AA@ 0049d168     tree.obj
 0002:00003184       ??_C@_0BL@NPACBAIG@?$CBnode?9?$DOfaces?5with?5children?$AA@ 0049d184     tree.obj
 0002:000031a0       ??_C@_0CG@LNPBEHAO@node?9?$DOfaces?5seperating?5CONTENTS_@ 0049d1a0     tree.obj
 0002:000031c8       ??_C@_0BC@CPHJDNDL@?$CF5i?5pruned?5nodes?6?$AA@ 0049d1c8     tree.obj
 0002:000031dc       ??_C@_0BE@MHMEFPNF@?9?9?9?5PruneNodes?5?9?9?9?6?$AA@ 0049d1dc     tree.obj
 0002:000031f0       __real@48800000            0049d1f0     utilmatlib.obj
 0002:000031f4       __real@c8800000            0049d1f4     utilmatlib.obj
 0002:000031f8       __real@40200000            0049d1f8     utilmatlib.obj
 0002:000031fc       __real@437f0000            0049d1fc     utilmatlib.obj
 0002:00003200       __real@400ccccd            0049d200     utilmatlib.obj
 0002:00003204       ??_C@_0DH@PCDCEHLE@Could?5not?5start?5the?5empty?5shader@ 0049d204     utilmatlib.obj
 0002:0000323c       ??_C@_0BD@PBEAPLLE@shaderapiempty?4dll?$AA@ 0049d23c     utilmatlib.obj
 0002:00003250       ??_C@_0DP@FFDBPPE@Could?5not?5find?5factory?5interface@ 0049d250     utilmatlib.obj
 0002:00003290       ??_C@_0FP@CECICCJC@Could?5not?5get?5the?5material?5syste@ 0049d290     utilmatlib.obj
 0002:000032f0       ??_C@_0BD@JIHPMPMC@VMaterialSystem079?$AA@ 0049d2f0     utilmatlib.obj
 0002:00003304       ??_C@_0BP@LKELEPKN@Can?8t?5load?5MaterialSystem?4dll?6?$AA@ 0049d304     utilmatlib.obj
 0002:00003324       ??_C@_0BD@PEHNKAML@materialsystem?4dll?$AA@ 0049d324     utilmatlib.obj
 0002:00003338       ??_C@_0P@IIPEELKE@Other?5textures?$AA@ 0049d338     utilmatlib.obj
 0002:00003348       ??_C@_0O@BJKHNGF@$reflectivity?$AA@ 0049d348     utilmatlib.obj
 0002:00003358       ??_C@_0CP@HJMGEEJC@?$CD?$CD?$CD?$CD?$CD?$CD?$CD?$CD?$CD?$CD?$CD?$CD?$CD?$CD?$CD?5block?5?$CF2i?0?$CF2i?5?$CD?$CD@ 0049d358     vbsp.obj
 0002:00003388       ??_C@_0DJ@FOPOCIBH@bmodel?5?$CFd?5has?5no?5head?5node?5?$CIclas@ 0049d388     vbsp.obj
 0002:000033c4       ??_C@_0O@HDHPHCPK@func_occluder?$AA@ 0049d3c4     vbsp.obj
 0002:000033d4       ??_C@_0P@NMEBHKDB@occludernumber?$AA@ 0049d3d4     vbsp.obj
 0002:000033e4       ??_C@_0N@FNMJMILG@vphysics?4dll?$AA@ 0049d3e4     vbsp.obj
 0002:000033f4       ??_C@_05NKLPODEL@?$CC?$CFs?$CC?5?$AA@ 0049d3f4     vbsp.obj
 0002:000033fc       ??_C@_0P@IFCDDMDK@Command?5line?3?5?$AA@ 0049d3fc     vbsp.obj
 0002:0000340c       ??_C@_0DK@CNKOIEOA@Occluder?5?$CC?$CFs?$CC?5straddles?5multiple@ 0049d40c     vbsp.obj
 0002:00003448       ??_C@_09GMFECJDN@?$DMno?5name?$DO?$AA@ 0049d448     vbsp.obj
 0002:00003454       ??_C@_0DN@DNJAMNLP@Error?$CB?5Entity?5sky_camera?5in?5soli@ 0049d454     vbsp.obj
 0002:00003494       ??_C@_0L@DFIGMJBA@sky_camera?$AA@ 0049d494     vbsp.obj
 0002:000034a0       ??_C@_0BE@MFAIICKC@?9?9?9?5MAP?5LEAKED?5?9?9?9?6?$AA@ 0049d4a0     vbsp.obj
 0002:000034b4       ??_C@_0N@NOHCKMO@WriteBSP?4?4?4?6?$AA@ 0049d4b4     vbsp.obj
 0002:000034c4       ??_C@_0P@BPJPCEDL@PruneNodes?4?4?4?6?$AA@ 0049d4c4     vbsp.obj
 0002:000034d4       ??_C@_0O@IMCAPANA@FixTjuncs?4?4?4?6?$AA@ 0049d4d4     vbsp.obj
 0002:000034e4       ??_C@_0BC@CLHFLLOE@Building?5Faces?4?4?4?$AA@ 0049d4e4     vbsp.obj
 0002:000034f8       ??_C@_0BC@DGHLLCEI@?$CK?$CK?$CK?$CK?5leaked?5?$CK?$CK?$CK?$CK?6?$AA@ 0049d4f8     vbsp.obj
 0002:0000350c       ??_C@_06KMNNMBLO@?$CF?920s?5?$AA@ 0049d50c     vbsp.obj
 0002:00003514       ??_C@_0BF@PDAKPJJC@ProcessBlock_Thread?3?$AA@ 0049d514     vbsp.obj
 0002:0000352c       ??_C@_0CO@IHAFINE@?9?9?9?9?9?9?9?9?9?9?9?9?9?9?9?9?9?9?9?9?9?9?9?9?9?9?9?9?9?9?9?9@ 0049d52c     vbsp.obj
 0002:0000355c       __real@3a800000            0049d55c     vbsp.obj
 0002:00003560       __real@ff7fffff            0049d560     vbsp.obj
 0002:00003564       ??_C@_0CK@FBCLDLJF@?$CD?$CD?$CD?$CD?$CD?$CD?$CD?$CD?$CD?$CD?$CD?$CD?$CD?$CD?$CD?5model?5?$CFi?5?$CD?$CD?$CD?$CD?$CD?$CD?$CD@ 0049d564     vbsp.obj
 0002:00003590       ??_C@_0M@JMMNIPIN@?$CFs?5elapsed?6?$AA@ 0049d590     vbsp.obj
 0002:0000359c       ??_C@_09CPDHAACC@stale?4txt?$AA@ 0049d59c     vbsp.obj
 0002:000035a8       ??_C@_05BFAEFKPM@stale?$AA@ 0049d5a8     vbsp.obj
 0002:000035b0       ??_C@_04HKNAPCJF@?4vmf?$AA@ 0049d5b0     vbsp.obj
 0002:000035b8       ??_C@_0BC@FEKMMIHD@materialPath?3?5?$CFs?6?$AA@ 0049d5b8     vbsp.obj
 0002:000035cc       ??_C@_0M@OJGAHGGE@?$CFsmaterials?$AA@ 0049d5cc     vbsp.obj
 0002:000035d8       ??_C@_06BEJGOBHG@?$CFs?4log?$AA@ 0049d5d8     vbsp.obj
 0002:000035e0       ??_C@_0KEN@GAFAFBAJ@Other?5options?5?5?3?6?5?5?9novconfig?5?5?5@ 0049d5e0     vbsp.obj
 0002:00004030       ??_C@_0DLF@GKGIKNMN@usage?5?5?3?5vbsp?5?$FLoptions?4?4?4?$FN?5mapfi@ 0049e030     vbsp.obj
 0002:000043e8       ??_C@_0BM@FHMHAFJB@VBSP?3?5Unknown?5option?5?$CC?$CFs?$CC?6?6?$AA@ 0049e3e8     vbsp.obj
 0002:00004404       ??_C@_0BA@CJFLDFHJ@verbose?5?$DN?5true?6?$AA@ 0049e404     vbsp.obj
 0002:00004414       ??_C@_0P@EOOCKJDE@?9FullMinidumps?$AA@ 0049e414     vbsp.obj
 0002:00004424       ??_C@_0BA@MHKJJLPK@?9nodrawtriggers?$AA@ 0049e424     vbsp.obj
 0002:00004434       ??_C@_0BC@ECNPNNFD@?9replacematerials?$AA@ 0049e434     vbsp.obj
 0002:00004448       ??_C@_0P@KNLBLKHC@?9novirtualmesh?$AA@ 0049e448     vbsp.obj
 0002:00004458       ??_C@_0BD@JFEPMFFD@?9allowdetailcracks?$AA@ 0049e458     vbsp.obj
 0002:0000446c       ??_C@_05JOPKDNB@?9xbox?$AA@ 0049e46c     vbsp.obj
 0002:00004474       ??_C@_0O@FEHBJGCK@?9keepstalezip?$AA@ 0049e474     vbsp.obj
 0002:00004484       ??_C@_05FACLEBO@?9game?$AA@ 0049e484     vbsp.obj
 0002:0000448c       ??_C@_09NFNCOJPN@?9vproject?$AA@ 0049e48c     vbsp.obj
 0002:00004498       ??_C@_06NIKDPCHB@?9steam?$AA@ 0049e498     vbsp.obj
 0002:000044a0       ??_C@_0M@OJHILNKA@?9allowdebug?$AA@ 0049e4a0     vbsp.obj
 0002:000044ac       ??_C@_0L@JACELBLD@?9NoVConfig?$AA@ 0049e4ac     vbsp.obj
 0002:000044b8       ??_C@_0BA@HBAANLBK@?9lightifmissing?$AA@ 0049e4b8     vbsp.obj
 0002:000044c8       ??_C@_04FCIJMIMA@?9low?$AA@ 0049e4c8     vbsp.obj
 0002:000044d0       ??_C@_08HBKMCN@?9bumpall?$AA@ 0049e4d0     vbsp.obj
 0002:000044dc       ??_C@_0O@MPJAIIJE@DXLevel?5?$DN?5?$CFd?6?$AA@ 0049e4dc     vbsp.obj
 0002:000044ec       ??_C@_08GIKFLJE@?9dxlevel?$AA@ 0049e4ec     vbsp.obj
 0002:000044f8       ??_C@_0P@HDPEMMMK@?9minluxelscale?$AA@ 0049e4f8     vbsp.obj
 0002:00004508       ??_C@_0M@FOIFAPBE@?9luxelscale?$AA@ 0049e508     vbsp.obj
 0002:00004514       ??_C@_04PBCBKGHJ@?1tmp?$AA@ 0049e514     vbsp.obj
 0002:0000451c       ??_C@_07NHBNKOHO@?9tmpout?$AA@ 0049e51c     vbsp.obj
 0002:00004524       ??_C@_0BK@IBFOGJLN@Enabled?5vis?5in?53d?5skybox?6?$AA@ 0049e524     vbsp.obj
 0002:00004540       ??_C@_0N@EJPCONLA@?9forceskyvis?$AA@ 0049e540     vbsp.obj
 0002:00004550       ??_C@_0CL@HKKFBLKO@Dumping?5static?5props?5to?5staticpr@ 0049e550     vbsp.obj
 0002:0000457c       ??_C@_0BA@PJFEFJJO@?9dumpstaticprop?$AA@ 0049e57c     vbsp.obj
 0002:0000458c       ??_C@_0CM@LBENMKOK@Dumping?5collision?5models?5to?5coll@ 0049e58c     vbsp.obj
 0002:000045b8       ??_C@_0N@GFFGPNIL@?9dumpcollide?$AA@ 0049e5b8     vbsp.obj
 0002:000045c8       ??_C@_0BI@GPFNOONF@blocks?3?5?$CFi?0?$CFi?5to?5?$CFi?0?$CFi?6?$AA@ 0049e5c8     vbsp.obj
 0002:000045e0       ??_C@_07OJNAHDHJ@?9blocks?$AA@ 0049e5e0     vbsp.obj
 0002:000045e8       ??_C@_0O@LDGKLHEB@block?3?5?$CFi?0?$CFi?6?$AA@ 0049e5e8     vbsp.obj
 0002:000045f8       ??_C@_06HKNKGMIA@?9block?$AA@ 0049e5f8     vbsp.obj
 0002:00004600       ??_C@_0BD@BFABFADB@snap?5axial?5?$DN?5true?6?$AA@ 0049e600     vbsp.obj
 0002:00004614       ??_C@_0L@GMPPNCKE@?9snapaxial?$AA@ 0049e614     vbsp.obj
 0002:00004620       ??_C@_0BI@HFJEOMHB@verboseentities?5?$DN?5true?6?$AA@ 0049e620     vbsp.obj
 0002:00004638       ??_C@_0BB@HMBOKPMN@?9verboseentities?$AA@ 0049e638     vbsp.obj
 0002:0000464c       ??_C@_0BB@FBDMOHFN@leaktest?5?$DN?5true?6?$AA@ 0049e64c     vbsp.obj
 0002:00004660       ??_C@_09NGDGFAIL@?9leaktest?$AA@ 0049e660     vbsp.obj
 0002:0000466c       ??_C@_0BC@FCFCFNJN@microvolume?5?$DN?5?$CFf?6?$AA@ 0049e66c     vbsp.obj
 0002:00004680       ??_C@_06HADCOCNO@?9micro?$AA@ 0049e680     vbsp.obj
 0002:00004688       ??_C@_0BC@HELGDFAB@onlyprops?5?$DN?5true?6?$AA@ 0049e688     vbsp.obj
 0002:0000469c       ??_C@_0L@CIBPLCFK@?9onlyprops?$AA@ 0049e69c     vbsp.obj
 0002:000046a8       ??_C@_0BB@PAELMIAC@onlyents?5?$DN?5true?6?$AA@ 0049e6a8     vbsp.obj
 0002:000046bc       ??_C@_09FNJHALDJ@?9onlyents?$AA@ 0049e6bc     vbsp.obj
 0002:000046c8       ??_C@_0BD@MHFIDIPG@fulldetail?5?$DN?5true?6?$AA@ 0049e6c8     vbsp.obj
 0002:000046dc       ??_C@_0M@LBOAMCBH@?9fulldetail?$AA@ 0049e6dc     vbsp.obj
 0002:000046e8       ??_C@_0BB@PCIJEAJB@nodetail?5?$DN?5true?6?$AA@ 0049e6e8     vbsp.obj
 0002:000046fc       ??_C@_09BNPKADLK@?9nodetail?$AA@ 0049e6fc     vbsp.obj
 0002:00004708       ??_C@_0BB@PHJFPDJO@nosubdiv?5?$DN?5true?6?$AA@ 0049e708     vbsp.obj
 0002:0000471c       ??_C@_09NEAGMLKK@?9nosubdiv?$AA@ 0049e71c     vbsp.obj
 0002:00004728       ??_C@_0BF@HBKNCEF@nomergewater?5?$DN?5true?6?$AA@ 0049e728     vbsp.obj
 0002:00004740       ??_C@_0O@IOEPNIGE@?9nomergewater?$AA@ 0049e740     vbsp.obj
 0002:00004750       ??_C@_0BA@BKKNDMCH@nomerge?5?$DN?5true?6?$AA@ 0049e750     vbsp.obj
 0002:00004760       ??_C@_08KDELMOMJ@?9nomerge?$AA@ 0049e760     vbsp.obj
 0002:0000476c       ??_C@_0BA@NEEAHJI@noprune?5?$DN?5true?6?$AA@ 0049e76c     vbsp.obj
 0002:0000477c       ??_C@_08FMMFJHCI@?9noprune?$AA@ 0049e77c     vbsp.obj
 0002:00004788       ??_C@_0O@LDPAGHJG@noopt?5?$DN?5true?6?$AA@ 0049e788     vbsp.obj
 0002:00004798       ??_C@_06JJICMFJM@?9noopt?$AA@ 0049e798     vbsp.obj
 0002:000047a0       ??_C@_0BA@BMLCDGPG@nowater?5?$DN?5true?6?$AA@ 0049e7a0     vbsp.obj
 0002:000047b0       ??_C@_08NHOKEGNA@?9nowater?$AA@ 0049e7b0     vbsp.obj
 0002:000047bc       ??_C@_0BA@PHPCINHD@notjunc?5?$DN?5true?6?$AA@ 0049e7bc     vbsp.obj
 0002:000047cc       ??_C@_08MBJOKOPL@?9notjunc?$AA@ 0049e7cc     vbsp.obj
 0002:000047d8       ??_C@_0BA@FEIPGCDA@noshare?5?$DN?5true?6?$AA@ 0049e7d8     vbsp.obj
 0002:000047e8       ??_C@_08DKEGPAHJ@?9noshare?$AA@ 0049e7e8     vbsp.obj
 0002:000047f4       ??_C@_0O@ODIBHGPN@nocsg?5?$DN?5true?6?$AA@ 0049e7f4     vbsp.obj
 0002:00004804       ??_C@_06LAPNIFOP@?9nocsg?$AA@ 0049e804     vbsp.obj
 0002:0000480c       ??_C@_0P@KLOLGE@noweld?5?$DN?5true?6?$AA@ 0049e80c     vbsp.obj
 0002:0000481c       ??_C@_07NNNDHKCP@?9noweld?$AA@ 0049e81c     vbsp.obj
 0002:00004824       ??_C@_08FBJJFDKJ@?9verbose?$AA@ 0049e824     vbsp.obj
 0002:00004830       ??_C@_02EJEOCNCO@?9v?$AA@  0049e830     vbsp.obj
 0002:00004834       ??_C@_07NHFHKBEH@?9glview?$AA@ 0049e834     vbsp.obj
 0002:0000483c       ??_C@_08CFGFJOBF@?9threads?$AA@ 0049e83c     vbsp.obj
 0002:00004848       ??_C@_0CA@CKNGMBPO@Valve?5Software?5?9?5vbsp?4exe?5?$CI?$CFs?$CJ?6?$AA@ 0049e848     vbsp.obj
 0002:00004868       ??_C@_0M@IBLKNBBI@Feb?515?52008?$AA@ 0049e868     vbsp.obj
 0002:00004874       ??_C@_04KHOIINPK@vbsp?$AA@ 0049e874     vbsp.obj
 0002:0000487c       ??_C@_09DNECJBKD@developer?$AA@ 0049e87c     vbsp.obj
 0002:00004888       ??_C@_0EG@LAHCHCLD@Generated?5worldvertextransition?5@ 0049e888     worldvertextransitionfixup.obj
 0002:000048d0       ??_C@_0BF@LNCGHEFN@maps?1?$CFs?1?$CFs_wvt_patch?$AA@ 0049e8d0     worldvertextransitionfixup.obj
 0002:000048e8       ??_C@_0BL@MBEPANAB@Patching?5WVT?5material?3?5?$CFs?6?$AA@ 0049e8e8     worldvertextransitionfixup.obj
 0002:00004904       ??_C@_0BF@JNPIKMOF@$BASETEXTURENOENVMAP?$AA@ 0049e904     worldvertextransitionfixup.obj
 0002:0000491c       ??_C@_0BA@IEBBPPCM@$maskedblending?$AA@ 0049e91c     worldvertextransitionfixup.obj
 0002:0000492c       ??_C@_0BG@BLNABPGE@$blendmodulatetexture?$AA@ 0049e92c     worldvertextransitionfixup.obj
 0002:00004944       ??_C@_0BG@HFLMEPDJ@$basetexture2noenvmap?$AA@ 0049e944     worldvertextransitionfixup.obj
 0002:0000495c       ??_C@_0M@OGEHLGNN@$bumpframe2?$AA@ 0049e95c     worldvertextransitionfixup.obj
 0002:00004968       ??_C@_09HGBMDNKK@$bumpmap2?$AA@ 0049e968     worldvertextransitionfixup.obj
 0002:00004974       ??_C@_0O@FOMCHCMA@$basetexture2?$AA@ 0049e974     worldvertextransitionfixup.obj
 0002:00004984       ??_C@_0BD@FHIKDCGP@LightmappedGeneric?$AA@ 0049e984     worldvertextransitionfixup.obj
 0002:00004998       ??_C@_0L@LJANLFFK@_wvt_patch?$AA@ 0049e998     worldvertextransitionfixup.obj
 0002:000049a4       ??_C@_0BG@EKOIMHEG@worldvertextransition?$AA@ 0049e9a4     worldvertextransitionfixup.obj
 0002:000049bc       ??_C@_0CH@CABCCPPD@Too?5many?5detail?5brush?5faces?0?5max@ 0049e9bc     writebsp.obj
 0002:000049e4       ??_C@_0N@CHDONEPJ@Bad?5leafface?$AA@ 0049e9e4     writebsp.obj
 0002:000049f4       ??_C@_0CH@JAONPFDO@Too?5many?5brushes?5in?5one?5leaf?0?5ma@ 0049e9f4     writebsp.obj
 0002:00004a1c       ??_C@_0BO@KPBGGBDO@Too?5many?5BSP?5leaves?0?5max?5?$DN?5?$CFd?$AA@ 0049ea1c     writebsp.obj
 0002:00004a40       ??_C@_0EC@KGDDHLOB@Too?5much?5brush?5geometry?5in?5bsp?0?5@ 0049ea40     writebsp.obj
 0002:00004a84       ??_C@_0CA@CIKMMFBO@Too?5many?5faces?5in?5map?0?5max?5?$DN?5?$CFd?$AA@ 0049ea84     writebsp.obj
 0002:00004aa4       ??_C@_03JLINDLFM@?$CK?$CFi?$AA@ 0049eaa4     writebsp.obj
 0002:00004aa8       ??_C@_0N@ODLHJNBO@defaultstyle?$AA@ 0049eaa8     writebsp.obj
 0002:00004ab8       ??_C@_05IAKJCFIM@style?$AA@ 0049eab8     writebsp.obj
 0002:00004ac0       ??_C@_0DH@JBALGJNA@Too?5many?5switched?5lights?5?$CIerror?5@ 0049eac0     writebsp.obj
 0002:00004af8       ??_C@_0O@JOPJPNEO@light_dynamic?$AA@ 0049eaf8     writebsp.obj
 0002:00004b08       ??_C@_05OEPGNJB@light?$AA@ 0049eb08     writebsp.obj
 0002:00004b10       ??_C@_0BG@FCCCHMGD@cheapwaterenddistance?$AA@ 0049eb10     writebsp.obj
 0002:00004b28       ??_C@_04OJDKMIMG@2000?$AA@ 0049eb28     writebsp.obj
 0002:00004b30       ??_C@_0BI@IJDCAKBF@cheapwaterstartdistance?$AA@ 0049eb30     writebsp.obj
 0002:00004b48       ??_C@_04KOJKLCBG@1000?$AA@ 0049eb48     writebsp.obj
 0002:00004b50       ??_C@_0EH@ILOLGID@Water?5found?5with?5no?5water_lod_co@ 0049eb50     writebsp.obj
 0002:00004b98       ??_C@_0BC@NGKELJID@water_lod_control?$AA@ 0049eb98     writebsp.obj
 0002:00004bac       ??_C@_0CH@MFDCAFMG@Too?5many?5brush?5models?5in?5map?0?5ma@ 0049ebac     writebsp.obj
 0002:00004bd4       ??_C@_0L@EHFOKKK@world_maxs?$AA@ 0049ebd4     writebsp.obj
 0002:00004be0       ??_C@_0L@NJGKBNIH@world_mins?$AA@ 0049ebe0     writebsp.obj
 0002:00004bec       ??_C@_0BM@EIABJHKK@NODRAW?5on?5terrain?5surface?$CB?6?$AA@ 0049ebec     writebsp.obj
 0002:00004c08       ??_C@_0BP@NGOCBDLI@WriteDrawNodes_r?3?5odd?5planenum?$AA@ 0049ec08     writebsp.obj
 0002:00004c28       ??_C@_0O@FHHLJHDC@MAX_MAP_NODES?$AA@ 0049ec28     writebsp.obj
 0002:00004c38       ??_C@_0BE@CMKAOOGK@?$CF5i?5original?5faces?6?$AA@ 0049ec38     writebsp.obj
 0002:00004c4c       ??_C@_0L@LBCDOAFM@?$CF5i?5faces?6?$AA@ 0049ec4c     writebsp.obj
 0002:00004c58       ??_C@_0BJ@PODJOBCA@?$CF5i?5nodes?5without?5faces?6?$AA@ 0049ec58     writebsp.obj
 0002:00004c74       ??_C@_0BG@JBDJMDA@?$CF5i?5nodes?5with?5faces?6?$AA@ 0049ec74     writebsp.obj
 0002:00004c8c       ??_C@_0BC@GGMDFDDP@?9?9?9?5WriteBSP?5?9?9?9?6?$AA@ 0049ec8c     writebsp.obj
 0002:00004ca0       ??_C@_0CM@KJJLEJKL@Reduced?5?$CFd?5texdatas?5to?5?$CFd?5?$CI?$CFd?5by@ 0049eca0     writebsp.obj
 0002:00004ccc       ??_C@_0BL@HFNBAJOH@Reduced?5?$CFd?5texinfos?5to?5?$CFd?6?$AA@ 0049eccc     writebsp.obj
 0002:00004ce8       ??_C@_0CH@MNJGFCJ@Compacting?5texture?1material?5tabl@ 0049ece8     writebsp.obj
 0002:00004d10       ??_C@_0BO@MHMPJPKO@?9?9?5DiscoverMacroTextures?3?5?$CFs?6?$AA@ 0049ed10     writebsp.obj
 0002:00004d30       ??_C@_0P@LPPLJJCF@$macro_texture?$AA@ 0049ed30     writebsp.obj
 0002:00004d40       ??_C@_0BK@FBHKPEMJ@ZIP_PreloadDirectoryEntry?$AA@ 0049ed40     zip_utils.obj
 0002:00004d5c       ??_C@_0BC@HEOACHKI@ZIP_PreloadHeader?$AA@ 0049ed5c     zip_utils.obj
 0002:00004d70       ??_C@_0BE@DFBHNPNK@ZIP_LocalFileHeader?$AA@ 0049ed70     zip_utils.obj
 0002:00004d84       ??_C@_0P@DELNDGBJ@ZIP_FileHeader?$AA@ 0049ed84     zip_utils.obj
 0002:00004d94       ??_C@_0BK@HMMNJNAE@ZIP_EndOfCentralDirRecord?$AA@ 0049ed94     zip_utils.obj
 0002:00004db0       ??_C@_0BD@DIHGEHMN@?$CFd_?$CFd_?$CFd_?$CFd_?$CFd?4tmp?$AA@ 0049edb0     zip_utils.obj
 0002:00004dc4       ??_C@_07PDHECPID@_?$CFs?4tmp?$AA@ 0049edc4     zip_utils.obj
 0002:00004dd0       ??_7CFileStream@@6B@       0049edd0     zip_utils.obj
 0002:00004dd8       ??_C@_08CBJJBCAI@XZP?$CFc?5?$CFd?$AA@ 0049edd8     zip_utils.obj
 0002:00004de4       ??_C@_03LJCPBJM@XZP?$AA@   0049ede4     zip_utils.obj
 0002:00004dec       ??_7CBufferStream@@6B@     0049edec     zip_utils.obj
 0002:00004df4       ??_C@_0BK@CAOLELCJ@CUtlLinkedList?5overflow?$CB?6?$AA@ 0049edf4     zip_utils.obj
 0002:00004e10       ??_C@_09CMIIOJHF@signature?$AA@ 0049ee10     zip_utils.obj
 0002:00004e1c       ??_C@_0BB@LEECKDMO@numberOfThisDisk?$AA@ 0049ee1c     zip_utils.obj
 0002:00004e30       ??_C@_0CL@OMGIEOOH@numberOfTheDiskWithStartOfCentra@ 0049ee30     zip_utils.obj
 0002:00004e5c       ??_C@_0CC@CAOEOPLI@nCentralDirectoryEntries_ThisDis@ 0049ee5c     zip_utils.obj
 0002:00004e80       ??_C@_0BP@GOGNIAAK@nCentralDirectoryEntries_Total?$AA@ 0049ee80     zip_utils.obj
 0002:00004ea0       ??_C@_0BF@DGGHGBPA@centralDirectorySize?$AA@ 0049eea0     zip_utils.obj
 0002:00004eb8       ??_C@_0BI@PHNJPAJL@startOfCentralDirOffset?$AA@ 0049eeb8     zip_utils.obj
 0002:00004ed0       ??_C@_0O@PEAODJEB@commentLength?$AA@ 0049eed0     zip_utils.obj
 0002:00004ee0       ??_C@_0O@OABAGKLC@versionMadeBy?$AA@ 0049eee0     zip_utils.obj
 0002:00004ef0       ??_C@_0BH@KAODBOOK@versionNeededToExtract?$AA@ 0049eef0     zip_utils.obj
 0002:00004f08       ??_C@_0BC@JMCGMPDB@compressionMethod?$AA@ 0049ef08     zip_utils.obj
 0002:00004f1c       ??_C@_0BB@LHLABCIP@lastModifiedTime?$AA@ 0049ef1c     zip_utils.obj
 0002:00004f30       ??_C@_0BB@BBDDFBN@lastModifiedDate?$AA@ 0049ef30     zip_utils.obj
 0002:00004f44       ??_C@_05KBIBMHFC@crc32?$AA@ 0049ef44     zip_utils.obj
 0002:00004f4c       ??_C@_0P@IEFIMPBE@compressedSize?$AA@ 0049ef4c     zip_utils.obj
 0002:00004f5c       ??_C@_0BB@BDLNGEJN@uncompressedSize?$AA@ 0049ef5c     zip_utils.obj
 0002:00004f70       ??_C@_0P@GEFKFGAH@fileNameLength?$AA@ 0049ef70     zip_utils.obj
 0002:00004f80       ??_C@_0BB@MBCIFNFD@extraFieldLength?$AA@ 0049ef80     zip_utils.obj
 0002:00004f94       ??_C@_0BC@JLPEPFDC@fileCommentLength?$AA@ 0049ef94     zip_utils.obj
 0002:00004fa8       ??_C@_0BA@EPOPKLNJ@diskNumberStart?$AA@ 0049efa8     zip_utils.obj
 0002:00004fb8       ??_C@_0BE@CBMOBGJC@internalFileAttribs?$AA@ 0049efb8     zip_utils.obj
 0002:00004fcc       ??_C@_0BE@HMGGBLGA@externalFileAttribs?$AA@ 0049efcc     zip_utils.obj
 0002:00004fe0       ??_C@_0BM@OJCDHDKM@relativeOffsetOfLocalHeader?$AA@ 0049efe0     zip_utils.obj
 0002:00004ffc       ??_C@_07NGFJPNPN@Version?$AA@ 0049effc     zip_utils.obj
 0002:00005004       ??_C@_0BB@GFAJHKJ@DirectoryEntries?$AA@ 0049f004     zip_utils.obj
 0002:00005018       ??_C@_0BI@IAOOMPJP@PreloadDirectoryEntries?$AA@ 0049f018     zip_utils.obj
 0002:00005030       ??_C@_09FBMAGD@Alignment?$AA@ 0049f030     zip_utils.obj
 0002:0000503c       ??_C@_06MHCOIGNA@Length?$AA@ 0049f03c     zip_utils.obj
 0002:00005044       ??_C@_0L@HLJLKILN@DataOffset?$AA@ 0049f044     zip_utils.obj
 0002:00005054       ??_7CZip@@6B@              0049f054     zip_utils.obj
 0002:000050a4       ??_C@_0BI@OECFCPNB@swapmoppsurfaceheader_t?$AA@ 0049f0a4     bsplib.obj
 0002:000050bc       ??_C@_0BL@DNFCANOP@swapcompactsurfaceheader_t?$AA@ 0049f0bc     bsplib.obj
 0002:000050d8       ??_C@_0BE@OFLJJEKJ@swapcollideheader_t?$AA@ 0049f0d8     bsplib.obj
 0002:000050ec       ??_C@_0BD@OLKDGEE@LUMP_OVERLAY_FADES?$AA@ 0049f0ec     bsplib.obj
 0002:00005100       ??_C@_0P@IIOJAODF@LUMP_MAP_FLAGS?$AA@ 0049f100     bsplib.obj
 0002:00005110       ??_C@_0P@FDJNLOGC@LUMP_FACES_HDR?$AA@ 0049f110     bsplib.obj
 0002:00005120       ??_C@_0BB@NEDFPAGN@LUMP_XZIPPAKFILE?$AA@ 0049f120     bsplib.obj
 0002:00005134       ??_C@_0BL@BKCBAMMA@LUMP_LEAF_AMBIENT_LIGHTING?$AA@ 0049f134     bsplib.obj
 0002:00005150       ??_C@_0BP@BFFHMJPJ@LUMP_LEAF_AMBIENT_LIGHTING_HDR?$AA@ 0049f150     bsplib.obj
 0002:00005170       ??_C@_0BF@CANCIIGC@LUMP_WORLDLIGHTS_HDR?$AA@ 0049f170     bsplib.obj
 0002:00005188       ??_C@_0BC@KEAACHGA@LUMP_LIGHTING_HDR?$AA@ 0049f188     bsplib.obj
 0002:0000519c       ??_C@_0BI@BMFPOHKD@LUMP_LEAF_AMBIENT_INDEX?$AA@ 0049f19c     bsplib.obj
 0002:000051b4       ??_C@_0BM@MBKMFPBI@LUMP_LEAF_AMBIENT_INDEX_HDR?$AA@ 0049f1b4     bsplib.obj
 0002:000051d0       ??_C@_0BD@CLELFBLI@LUMP_WATEROVERLAYS?$AA@ 0049f1d0     bsplib.obj
 0002:000051e4       ??_C@_0BI@NJJHKFEP@LUMP_PHYSCOLLIDESURFACE?$AA@ 0049f1e4     bsplib.obj
 0002:000051fc       ??_C@_0P@ILJIKKIG@LUMP_DISP_TRIS?$AA@ 0049f1fc     bsplib.obj
 0002:0000520c       ??_C@_0BN@FKFFDEEC@LUMP_FACE_MACRO_TEXTURE_INFO?$AA@ 0049f20c     bsplib.obj
 0002:0000522c       ??_C@_0BI@PEOPPAME@LUMP_LEAFMINDISTTOWATER?$AA@ 0049f22c     bsplib.obj
 0002:00005244       ??_C@_0O@EGIHIGHE@LUMP_OVERLAYS?$AA@ 0049f244     bsplib.obj
 0002:00005254       ??_C@_0BK@HOIMAHNF@LUMP_TEXDATA_STRING_TABLE?$AA@ 0049f254     bsplib.obj
 0002:00005270       ??_C@_0BJ@PGCIOLBP@LUMP_TEXDATA_STRING_DATA?$AA@ 0049f270     bsplib.obj
 0002:0000528c       ??_C@_0O@MHPJGMBB@LUMP_CUBEMAPS?$AA@ 0049f28c     bsplib.obj
 0002:0000529c       ??_C@_0BF@NDALMOFD@LUMP_CLIPPORTALVERTS?$AA@ 0049f29c     bsplib.obj
 0002:000052b4       ??_C@_0N@GNKDOCCI@LUMP_PAKFILE?$AA@ 0049f2b4     bsplib.obj
 0002:000052c4       ??_C@_0BB@KPDLNDCB@LUMP_PRIMINDICES?$AA@ 0049f2c4     bsplib.obj
 0002:000052d8       ??_C@_0P@OELFIIM@LUMP_PRIMVERTS?$AA@ 0049f2d8     bsplib.obj
 0002:000052e8       ??_C@_0BA@IJBIAGAH@LUMP_PRIMITIVES?$AA@ 0049f2e8     bsplib.obj
 0002:000052f8       ??_C@_0BD@ODLDHPKI@LUMP_LEAFWATERDATA?$AA@ 0049f2f8     bsplib.obj
 0002:0000530c       ??_C@_0P@GGMDDMAI@LUMP_GAME_LUMP?$AA@ 0049f30c     bsplib.obj
 0002:0000531c       ??_C@_0CE@CBCIIDNL@LUMP_DISP_LIGHTMAP_SAMPLE_POSITI@ 0049f31c     bsplib.obj
 0002:00005340       ??_C@_0BA@IIJJJMKK@LUMP_DISP_VERTS?$AA@ 0049f340     bsplib.obj
 0002:00005350       ??_C@_0BK@HINDNDEN@LUMP_DISP_LIGHTMAP_ALPHAS?$AA@ 0049f350     bsplib.obj
 0002:0000536c       ??_C@_0BH@FFAKLLAA@LUMP_VERTNORMALINDICES?$AA@ 0049f36c     bsplib.obj
 0002:00005384       ??_C@_0BB@DBIDJPFD@LUMP_VERTNORMALS?$AA@ 0049f384     bsplib.obj
 0002:00005398       ??_C@_0BB@MBCNHCIA@LUMP_PHYSCOLLIDE?$AA@ 0049f398     bsplib.obj
 0002:000053ac       ??_C@_0O@OEJDLIOJ@LUMP_PHYSDISP?$AA@ 0049f3ac     bsplib.obj
 0002:000053bc       ??_C@_0BD@EJIHOJDL@LUMP_ORIGINALFACES?$AA@ 0049f3bc     bsplib.obj
 0002:000053d0       ??_C@_0O@EJABBFOH@LUMP_DISPINFO?$AA@ 0049f3d0     bsplib.obj
 0002:000053e0       ??_C@_0N@HPHHNHMM@LUMP_UNUSED3?$AA@ 0049f3e0     bsplib.obj
 0002:000053f0       ??_C@_0N@GGGMOGIN@LUMP_UNUSED2?$AA@ 0049f3f0     bsplib.obj
 0002:00005400       ??_C@_0N@ENEBLFEO@LUMP_UNUSED1?$AA@ 0049f400     bsplib.obj
 0002:00005410       ??_C@_0N@FEFKIEAP@LUMP_UNUSED0?$AA@ 0049f410     bsplib.obj
 0002:00005420       ??_C@_0BB@OJCKABCN@LUMP_AREAPORTALS?$AA@ 0049f420     bsplib.obj
 0002:00005434       ??_C@_0L@HCKCACPC@LUMP_AREAS?$AA@ 0049f434     bsplib.obj
 0002:00005440       ??_C@_0BA@BNCFENGJ@LUMP_BRUSHSIDES?$AA@ 0049f440     bsplib.obj
 0002:00005450       ??_C@_0N@DPCCMAAJ@LUMP_BRUSHES?$AA@ 0049f450     bsplib.obj
 0002:00005460       ??_C@_0BB@HIKJEPMN@LUMP_LEAFBRUSHES?$AA@ 0049f460     bsplib.obj
 0002:00005474       ??_C@_0P@CJINAEPL@LUMP_LEAFFACES?$AA@ 0049f474     bsplib.obj
 0002:00005484       ??_C@_0BB@LDCFDKDP@LUMP_WORLDLIGHTS?$AA@ 0049f484     bsplib.obj
 0002:00005498       ??_C@_0M@BPMHBODO@LUMP_MODELS?$AA@ 0049f498     bsplib.obj
 0002:000054a4       ??_C@_0P@GAMKMAKO@LUMP_SURFEDGES?$AA@ 0049f4a4     bsplib.obj
 0002:000054b4       ??_C@_0L@KLJDECJB@LUMP_EDGES?$AA@ 0049f4b4     bsplib.obj
 0002:000054c0       ??_C@_0N@GOAPMGFG@LUMP_FACEIDS?$AA@ 0049f4c0     bsplib.obj
 0002:000054d0       ??_C@_0L@JGNBNLGM@LUMP_LEAFS?$AA@ 0049f4d0     bsplib.obj
 0002:000054dc       ??_C@_0P@FFNBCDDI@LUMP_OCCLUSION?$AA@ 0049f4dc     bsplib.obj
 0002:000054ec       ??_C@_0O@ENKADPOO@LUMP_LIGHTING?$AA@ 0049f4ec     bsplib.obj
 0002:000054fc       ??_C@_0L@GKIFCIBI@LUMP_FACES?$AA@ 0049f4fc     bsplib.obj
 0002:00005508       ??_C@_0N@HABLHKMA@LUMP_TEXINFO?$AA@ 0049f508     bsplib.obj
 0002:00005518       ??_C@_0L@KEDBCMKN@LUMP_NODES?$AA@ 0049f518     bsplib.obj
 0002:00005524       ??_C@_0BA@JJJJNMIF@LUMP_VISIBILITY?$AA@ 0049f524     bsplib.obj
 0002:00005534       ??_C@_0O@PFMNCFLL@LUMP_VERTEXES?$AA@ 0049f534     bsplib.obj
 0002:00005544       ??_C@_0N@FBMJPELH@LUMP_TEXDATA?$AA@ 0049f544     bsplib.obj
 0002:00005554       ??_C@_0M@IPGKKCGA@LUMP_PLANES?$AA@ 0049f554     bsplib.obj
 0002:00005560       ??_C@_0O@FEFHONOO@LUMP_ENTITIES?$AA@ 0049f560     bsplib.obj
 0002:00005570       ??_C@_0N@MKKKCKNB@FileHeader_t?$AA@ 0049f570     bsplib.obj
 0002:00005580       ??_C@_0N@OAJJGDEO@MeshHeader_t?$AA@ 0049f580     bsplib.obj
 0002:00005590       ??_C@_0BM@MCIAFPDJ@DetailPropLightstylesLump_t?$AA@ 0049f590     bsplib.obj
 0002:000055ac       ??_C@_0BH@MHMAAGLE@DetailSpriteDictLump_t?$AA@ 0049f5ac     bsplib.obj
 0002:000055c4       ??_C@_0BD@PIOIBHCF@DetailObjectLump_t?$AA@ 0049f5c4     bsplib.obj
 0002:000055d8       ??_C@_0BH@NLNJCPJB@DetailObjectDictLump_t?$AA@ 0049f5d8     bsplib.obj
 0002:000055f0       ??_C@_0BF@EHIAMEIF@StaticPropLeafLump_t?$AA@ 0049f5f0     bsplib.obj
 0002:00005608       ??_C@_0BD@LEBBNIAA@StaticPropLumpV5_t?$AA@ 0049f608     bsplib.obj
 0002:0000561c       ??_C@_0BD@MKNLPGF@StaticPropLumpV4_t?$AA@ 0049f61c     bsplib.obj
 0002:00005630       ??_C@_0BB@KBIEIIMO@StaticPropLump_t?$AA@ 0049f630     bsplib.obj
 0002:00005644       ??_C@_0BF@PHBHNLJO@StaticPropDictLump_t?$AA@ 0049f644     bsplib.obj
 0002:0000565c       ??_C@_0M@OMEEDGMC@dgamelump_t?$AA@ 0049f65c     bsplib.obj
 0002:00005668       ??_C@_0BC@DOHNMHNB@dgamelumpheader_t?$AA@ 0049f668     bsplib.obj
 0002:0000567c       ??_C@_0P@GCGCOJHF@doverlayfade_t?$AA@ 0049f67c     bsplib.obj
 0002:0000568c       ??_C@_0BA@LPAAAJLB@dwateroverlay_t?$AA@ 0049f68c     bsplib.obj
 0002:0000569c       ??_C@_0L@NFDMIKGD@doverlay_t?$AA@ 0049f69c     bsplib.obj
 0002:000056a8       ??_C@_0BB@PEILJHEN@dcubemapsample_t?$AA@ 0049f6a8     bsplib.obj
 0002:000056bc       ??_C@_0BE@LJCKGEBK@doccluderpolydata_t?$AA@ 0049f6bc     bsplib.obj
 0002:000056d0       ??_C@_0BA@DGINHBJN@doccluderdata_t?$AA@ 0049f6d0     bsplib.obj
 0002:000056e0       ??_C@_0BB@LPGCFBAA@dleafwaterdata_t?$AA@ 0049f6e0     bsplib.obj
 0002:000056f4       ??_C@_0O@KHFJINND@dworldlight_t?$AA@ 0049f6f4     bsplib.obj
 0002:00005704       ??_C@_0O@FELKPDKA@dareaportal_t?$AA@ 0049f704     bsplib.obj
 0002:00005714       ??_C@_07FLKMNIGI@darea_t?$AA@ 0049f714     bsplib.obj
 0002:0000571c       ??_C@_0M@EEEPECPF@dphysdisp_t?$AA@ 0049f71c     bsplib.obj
 0002:00005728       ??_C@_0N@JKAKAPKN@dphysmodel_t?$AA@ 0049f728     bsplib.obj
 0002:00005738       ??_C@_08LBJNJKCK@dmodel_t?$AA@ 0049f738     bsplib.obj
 0002:00005744       ??_C@_07IPMONJMK@dedge_t?$AA@ 0049f744     bsplib.obj
 0002:0000574c       ??_C@_0N@DICEINDF@dbrushside_t?$AA@ 0049f74c     bsplib.obj
 0002:0000575c       ??_C@_08MGPMFBMD@dbrush_t?$AA@ 0049f75c     bsplib.obj
 0002:00005768       ??_C@_09BJPDADAO@dfaceid_t?$AA@ 0049f768     bsplib.obj
 0002:00005774       ??_C@_07BLGLPECE@dface_t?$AA@ 0049f774     bsplib.obj
 0002:0000577c       ??_C@_0M@IELDMBMH@dprimvert_t?$AA@ 0049f77c     bsplib.obj
 0002:00005788       ??_C@_0N@JCLKPMCB@dprimitive_t?$AA@ 0049f788     bsplib.obj
 0002:00005798       ??_C@_0BG@DPNAMNGO@CFaceMacroTextureInfo?$AA@ 0049f798     bsplib.obj
 0002:000057b0       ??_C@_08JOFBHKDH@CDispTri?$AA@ 0049f7b0     bsplib.obj
 0002:000057bc       ??_C@_09FEANDIFA@CDispVert?$AA@ 0049f7bc     bsplib.obj
 0002:000057c8       ??_C@_0BB@CINMEECK@CDispSubNeighbor?$AA@ 0049f7c8     bsplib.obj
 0002:000057dc       ??_C@_0BF@GAGKEJIM@CDispCornerNeighbors?$AA@ 0049f7dc     bsplib.obj
 0002:000057f4       ??_C@_0O@KJLBJMCP@CDispNeighbor?$AA@ 0049f7f4     bsplib.obj
 0002:00005804       ??_C@_0M@HCKLBNLM@ddispinfo_t?$AA@ 0049f804     bsplib.obj
 0002:00005810       ??_C@_0L@PNLMHHJK@dtexdata_t?$AA@ 0049f810     bsplib.obj
 0002:0000581c       ??_C@_09PPMCCLHO@texinfo_t?$AA@ 0049f81c     bsplib.obj
 0002:00005828       ??_C@_07KAKOAHCD@dnode_t?$AA@ 0049f828     bsplib.obj
 0002:00005830       ??_C@_09OHGFAMOH@dvertex_t?$AA@ 0049f830     bsplib.obj
 0002:0000583c       ??_C@_0BH@JAMCCGHN@dleafambientlighting_t?$AA@ 0049f83c     bsplib.obj
 0002:00005854       ??_C@_0BE@ILNCIEDE@dleafambientindex_t?$AA@ 0049f854     bsplib.obj
 0002:00005868       ??_C@_0BE@EMOGJPEN@CompressedLightCube?$AA@ 0049f868     bsplib.obj
 0002:0000587c       ??_C@_07EMPPBFPC@dleaf_t?$AA@ 0049f87c     bsplib.obj
 0002:00005884       ??_C@_0BC@EHFLNAFD@dleaf_version_0_t?$AA@ 0049f884     bsplib.obj
 0002:00005898       ??_C@_08DNNOELGF@dplane_t?$AA@ 0049f898     bsplib.obj
 0002:000058a4       ??_C@_0N@LGEPKNAO@dflagslump_t?$AA@ 0049f8a4     bsplib.obj
 0002:000058b4       ??_C@_06FDEEFMHN@lump_t?$AA@ 0049f8b4     bsplib.obj
 0002:000058bc       ??_C@_09LJDKPBKI@dheader_t?$AA@ 0049f8bc     bsplib.obj
 0002:000058c8       ??_C@_07NFANNNEC@UNKNOWN?$AA@ 0049f8c8     bsplib.obj
 0002:000058d0       ??_C@_0CO@EDJFKPFP@ValidateLump?3?5old?5version?5for?5lu@ 0049f8d0     bsplib.obj
 0002:00005900       ??_C@_0CD@HCMHJLHJ@ValidateLump?3?5odd?5size?5for?5lump?5@ 0049f900     bsplib.obj
 0002:00005924       ??_C@_0BJ@EBHLPGFH@?$CFs?5is?5version?5?$CFi?0?5not?5?$CFi?$AA@ 0049f924     bsplib.obj
 0002:00005940       ??_C@_0BG@HLMOFCME@?$CFs?5is?5not?5a?5IBSP?5file?$AA@ 0049f940     bsplib.obj
 0002:00005958       ??_C@_0CM@NMKLEGFP@Error?5opening?5?$CFs?$CB?5?$CICheck?5for?5wri@ 0049f958     bsplib.obj
 0002:00005988       __real@4059000000000000    0049f988     bsplib.obj
 0002:00005990       ??_C@_0M@HBEEPJK@?$CFlf?5?$CFlf?5?$CFlf?$AA@ 0049f990     bsplib.obj
 0002:0000599c       ??_C@_07JNLHAIBP@?$CFlf?5?$CFlf?$AA@ 0049f99c     bsplib.obj
 0002:000059a4       ??_C@_04KPILAJPA@?4bsp?$AA@ 0049f9a4     bsplib.obj
 0002:000059ac       ??_C@_0DJ@IALAKHCH@Unknown?5Static?5Prop?5Lump?5version@ 0049f9ac     bsplib.obj
 0002:000059e8       ??_C@_0CM@DGBFFHA@Unknown?5game?5lump?5?8?$CFs?8?5didn?8t?5ge@ 0049f9e8     bsplib.obj
 0002:00005a14       ??_C@_0CP@MLMNILJJ@?$CB?$CB?$CB?5WARNING?3?5Can?8t?5swap?5the?5phys@ 0049fa14     bsplib.obj
 0002:00005a44       ??_C@_0CF@KAOEHNKC@Writing?5unknown?5lump?5?$CD?$CFd?5?$CI?$CFd?5byt@ 0049fa44     bsplib.obj
 0002:00005a70       ??_C@_0IA@GAOHBJHI@Bad?5surface?5extents?5?9?5surface?5is@ 0049fa70     bsplib.obj
 0002:00005af0       ??_C@_0CF@NFIIJEKN@Bad?5surface?5extents?5point?3?5?$CFf?5?$CFf@ 0049faf0     bsplib.obj
 0002:00005b18       ??_C@_07EMAOIIJD@texdata?$AA@ 0049fb18     bsplib.obj
 0002:00005b20       ??_C@_0CF@BMEFMFJB@Reading?5unknown?5lump?5?$CD?$CFd?5?$CI?$CFd?5byt@ 0049fb20     bsplib.obj
 0002:00005b48       ??_C@_0DJ@MFKFBFPP@Map?5has?5too?5many?5texinfos?5?$CIhas?5?$CF@ 0049fb48     bsplib.obj
 0002:00005b84       ??_C@_05IJGIMKK@ident?$AA@ 0049fb84     bsplib.obj
 0002:00005b8c       ??_C@_07CPCPJPKL@version?$AA@ 0049fb8c     bsplib.obj
 0002:00005b94       ??_C@_05JJJGJDHJ@lumps?$AA@ 0049fb94     bsplib.obj
 0002:00005b9c       ??_C@_0M@HBIBAMBI@mapRevision?$AA@ 0049fb9c     bsplib.obj
 0002:00005ba8       ??_C@_07JHJOMNHC@fileofs?$AA@ 0049fba8     bsplib.obj
 0002:00005bb0       ??_C@_07HIABLANJ@filelen?$AA@ 0049fbb0     bsplib.obj
 0002:00005bb8       ??_C@_06CKNLMMCG@fourCC?$AA@ 0049fbb8     bsplib.obj
 0002:00005bc0       ??_C@_0N@EFAKEOG@m_LevelFlags?$AA@ 0049fbc0     bsplib.obj
 0002:00005bd0       ??_C@_06IKLLLDHL@normal?$AA@ 0049fbd0     bsplib.obj
 0002:00005bd8       ??_C@_04OKFALBN@dist?$AA@  0049fbd8     bsplib.obj
 0002:00005be0       ??_C@_04GPMDFGEJ@type?$AA@ 0049fbe0     bsplib.obj
 0002:00005be8       ??_C@_07NKHKICEG@cluster?$AA@ 0049fbe8     bsplib.obj
 0002:00005bf0       ??_C@_02HIEKPFIC@bf?$AA@   0049fbf0     bsplib.obj
 0002:00005bf4       ??_C@_04FIAKMPII@mins?$AA@ 0049fbf4     bsplib.obj
 0002:00005bfc       ??_C@_04IFBFDIKF@maxs?$AA@ 0049fbfc     bsplib.obj
 0002:00005c04       ??_C@_0O@JFONBDAD@firstleafface?$AA@ 0049fc04     bsplib.obj
 0002:00005c14       ??_C@_0N@BDFNHCAO@numleaffaces?$AA@ 0049fc14     bsplib.obj
 0002:00005c24       ??_C@_0P@OFLACFMD@firstleafbrush?$AA@ 0049fc24     bsplib.obj
 0002:00005c34       ??_C@_0P@FMNNGKO@numleafbrushes?$AA@ 0049fc34     bsplib.obj
 0002:00005c44       ??_C@_0BA@IKLKJAHM@leafWaterDataID?$AA@ 0049fc44     bsplib.obj
 0002:00005c54       ??_C@_0BC@OICOOBDE@m_AmbientLighting?$AA@ 0049fc54     bsplib.obj
 0002:00005c68       ??_C@_07LJHCELCO@m_Color?$AA@ 0049fc68     bsplib.obj
 0002:00005c70       ??_C@_0BD@BFDCJBID@ambientSampleCount?$AA@ 0049fc70     bsplib.obj
 0002:00005c84       ??_C@_0BD@HFMKPMGE@firstAmbientSample?$AA@ 0049fc84     bsplib.obj
 0002:00005c98       ??_C@_04OIHHNFHN@cube?$AA@ 0049fc98     bsplib.obj
 0002:00005ca0       ??_C@_01FJMABOPO@x?$AA@    0049fca0     bsplib.obj
 0002:00005ca4       ??_C@_01EANLCPLP@y?$AA@    0049fca4     bsplib.obj
 0002:00005ca8       ??_C@_01GLPGHMHM@z?$AA@    0049fca8     bsplib.obj
 0002:00005cac       ??_C@_03PNAAIPML@pad?$AA@  0049fcac     bsplib.obj
 0002:00005cb0       ??_C@_05BBEJFBFA@point?$AA@ 0049fcb0     bsplib.obj
 0002:00005cb8       ??_C@_08HJGMHDFH@planenum?$AA@ 0049fcb8     bsplib.obj
 0002:00005cc4       ??_C@_08GOINNFB@children?$AA@ 0049fcc4     bsplib.obj
 0002:00005cd0       ??_C@_09FEPJDPNN@firstface?$AA@ 0049fcd0     bsplib.obj
 0002:00005cdc       ??_C@_08JKOEMKBP@numfaces?$AA@ 0049fcdc     bsplib.obj
 0002:00005ce8       ??_C@_04GOEDGNCF@area?$AA@ 0049fce8     bsplib.obj
 0002:00005cf0       ??_C@_0BP@NMBCBGBE@textureVecsTexelsPerWorldUnits?$AA@ 0049fcf0     bsplib.obj
 0002:00005d10       ??_C@_0CA@IPOFBMEA@lightmapVecsLuxelsPerWorldUnits?$AA@ 0049fd10     bsplib.obj
 0002:00005d30       ??_C@_0N@LJNLFOD@reflectivity?$AA@ 0049fd30     bsplib.obj
 0002:00005d40       ??_C@_0BC@OEOFGALD@nameStringTableID?$AA@ 0049fd40     bsplib.obj
 0002:00005d54       ??_C@_05IGKADHGO@width?$AA@ 0049fd54     bsplib.obj
 0002:00005d5c       ??_C@_06LNLHEAAG@height?$AA@ 0049fd5c     bsplib.obj
 0002:00005d64       ??_C@_0L@CHMFFBH@view_width?$AA@ 0049fd64     bsplib.obj
 0002:00005d70       ??_C@_0M@JEOKFFPM@view_height?$AA@ 0049fd70     bsplib.obj
 0002:00005d7c       ??_C@_0O@FDHHLLPE@startPosition?$AA@ 0049fd7c     bsplib.obj
 0002:00005d8c       ??_C@_0BB@BEGJFCOK@m_iDispVertStart?$AA@ 0049fd8c     bsplib.obj
 0002:00005da0       ??_C@_0BA@EEICBDCB@m_iDispTriStart?$AA@ 0049fda0     bsplib.obj
 0002:00005db0       ??_C@_07GOCNGAOG@minTess?$AA@ 0049fdb0     bsplib.obj
 0002:00005db8       ??_C@_0P@JNKEKPLM@smoothingAngle?$AA@ 0049fdb8     bsplib.obj
 0002:00005dc8       ??_C@_0L@CFKODFKO@m_iMapFace?$AA@ 0049fdc8     bsplib.obj
 0002:00005dd4       ??_C@_0BG@DDOEIFEL@m_iLightmapAlphaStart?$AA@ 0049fdd4     bsplib.obj
 0002:00005dec       ??_C@_0BP@PAFNNLAB@m_iLightmapSamplePositionStart?$AA@ 0049fdec     bsplib.obj
 0002:00005e0c       ??_C@_0BA@KPACCIDF@m_EdgeNeighbors?$AA@ 0049fe0c     bsplib.obj
 0002:00005e1c       ??_C@_0BC@NIPPIPEI@m_CornerNeighbors?$AA@ 0049fe1c     bsplib.obj
 0002:00005e30       ??_C@_0P@LOALHPHF@m_AllowedVerts?$AA@ 0049fe30     bsplib.obj
 0002:00005e40       ??_C@_0P@MHNHNEHJ@m_SubNeighbors?$AA@ 0049fe40     bsplib.obj
 0002:00005e50       ??_C@_0M@PJNEJPND@m_Neighbors?$AA@ 0049fe50     bsplib.obj
 0002:00005e5c       ??_C@_0N@NFFMJJFJ@m_nNeighbors?$AA@ 0049fe5c     bsplib.obj
 0002:00005e6c       ??_C@_0M@BHAIIGNN@m_iNeighbor?$AA@ 0049fe6c     bsplib.obj
 0002:00005e78       ??_C@_0BG@LCLHGLFD@m_NeighborOrientation?$AA@ 0049fe78     bsplib.obj
 0002:00005e90       ??_C@_06NDMNEFDP@m_Span?$AA@ 0049fe90     bsplib.obj
 0002:00005e98       ??_C@_0P@OADNGDCO@m_NeighborSpan?$AA@ 0049fe98     bsplib.obj
 0002:00005ea8       ??_C@_09IDMJOBKC@m_vVector?$AA@ 0049fea8     bsplib.obj
 0002:00005eb4       ??_C@_08FJDFPGMN@m_flDist?$AA@ 0049feb4     bsplib.obj
 0002:00005ec0       ??_C@_09GMODKCE@m_flAlpha?$AA@ 0049fec0     bsplib.obj
 0002:00005ecc       ??_C@_08KOPEMDCL@m_uiTags?$AA@ 0049fecc     bsplib.obj
 0002:00005ed8       ??_C@_0BF@IGHHBDIM@m_MacroTextureNameID?$AA@ 0049fed8     bsplib.obj
 0002:00005ef0       ??_C@_0L@PGKNLMCD@firstIndex?$AA@ 0049fef0     bsplib.obj
 0002:00005efc       ??_C@_0L@PBJJKAHO@indexCount?$AA@ 0049fefc     bsplib.obj
 0002:00005f08       ??_C@_09DEIHPKFL@firstVert?$AA@ 0049ff08     bsplib.obj
 0002:00005f14       ??_C@_09MANBFGEA@vertCount?$AA@ 0049ff14     bsplib.obj
 0002:00005f20       ??_C@_03PCBNCGFH@pos?$AA@  0049ff20     bsplib.obj
 0002:00005f24       ??_C@_06POEBIPME@onNode?$AA@ 0049ff24     bsplib.obj
 0002:00005f2c       ??_C@_09CDIOBNOD@firstedge?$AA@ 0049ff2c     bsplib.obj
 0002:00005f38       ??_C@_08FLPCKAJG@numedges?$AA@ 0049ff38     bsplib.obj
 0002:00005f44       ??_C@_07GNNMAGOE@texinfo?$AA@ 0049ff44     bsplib.obj
 0002:00005f4c       ??_C@_0BD@KHDHNEKP@surfaceFogVolumeID?$AA@ 0049ff4c     bsplib.obj
 0002:00005f60       ??_C@_06OAJMEMBL@styles?$AA@ 0049ff60     bsplib.obj
 0002:00005f68       ??_C@_08OBOMOBNA@lightofs?$AA@ 0049ff68     bsplib.obj
 0002:00005f74       ??_C@_0BO@KLAFEDGH@m_LightmapTextureMinsInLuxels?$AA@ 0049ff74     bsplib.obj
 0002:00005f94       ??_C@_0BO@NBHLKPOL@m_LightmapTextureSizeInLuxels?$AA@ 0049ff94     bsplib.obj
 0002:00005fb4       ??_C@_08HJLENCAJ@origFace?$AA@ 0049ffb4     bsplib.obj
 0002:00005fc0       ??_C@_0L@NCAJFDDK@m_NumPrims?$AA@ 0049ffc0     bsplib.obj
 0002:00005fcc       ??_C@_0M@KIFLCOML@firstPrimID?$AA@ 0049ffcc     bsplib.obj
 0002:00005fd8       ??_C@_0BA@NGBALEKI@smoothingGroups?$AA@ 0049ffd8     bsplib.obj
 0002:00005fe8       ??_C@_0N@OPGHGHFA@hammerfaceid?$AA@ 0049ffe8     bsplib.obj
 0002:00005ff8       ??_C@_09DMACBJEF@firstside?$AA@ 0049fff8     bsplib.obj
 0002:00006004       ??_C@_08GEFICKEP@numsides?$AA@ 004a0004     bsplib.obj
 0002:00006010       ??_C@_05JDNDNKBA@bevel?$AA@ 004a0010     bsplib.obj
 0002:00006018       ??_C@_01MHEDDDHA@v?$AA@    004a0018     bsplib.obj
 0002:0000601c       ??_C@_08MKPBLOEI@headnode?$AA@ 004a001c     bsplib.obj
 0002:00006028       ??_C@_0L@OJKNJKNO@modelIndex?$AA@ 004a0028     bsplib.obj
 0002:00006034       ??_C@_08KHMGMMON@dataSize?$AA@ 004a0034     bsplib.obj
 0002:00006040       ??_C@_0M@EIAFECAC@keydataSize?$AA@ 004a0040     bsplib.obj
 0002:0000604c       ??_C@_0L@BOALBGOC@solidCount?$AA@ 004a004c     bsplib.obj
 0002:00006058       ??_C@_0BB@NNJGKKC@numDisplacements?$AA@ 004a0058     bsplib.obj
 0002:0000606c       ??_C@_0P@JEEOJIEO@numareaportals?$AA@ 004a006c     bsplib.obj
 0002:0000607c       ??_C@_0BA@PNCAMLID@firstareaportal?$AA@ 004a007c     bsplib.obj
 0002:0000608c       ??_C@_0M@HGJDIFIH@m_PortalKey?$AA@ 004a008c     bsplib.obj
 0002:00006098       ??_C@_09FKCCELOM@otherarea?$AA@ 004a0098     bsplib.obj
 0002:000060a4       ??_C@_0BG@GLOJEMCM@m_FirstClipPortalVert?$AA@ 004a00a4     bsplib.obj
 0002:000060bc       ??_C@_0BD@FMOIFBLK@m_nClipPortalVerts?$AA@ 004a00bc     bsplib.obj
 0002:000060d0       ??_C@_09DDBFFAKC@intensity?$AA@ 004a00d0     bsplib.obj
 0002:000060dc       ??_C@_07BMMJEPCG@stopdot?$AA@ 004a00dc     bsplib.obj
 0002:000060e4       ??_C@_08DPGBBIMD@stopdot2?$AA@ 004a00e4     bsplib.obj
 0002:000060f0       ??_C@_08EGJNFMPO@exponent?$AA@ 004a00f0     bsplib.obj
 0002:000060fc       ??_C@_06KGHINEPG@radius?$AA@ 004a00fc     bsplib.obj
 0002:00006104       ??_C@_0O@CNHFALEA@constant_attn?$AA@ 004a0104     bsplib.obj
 0002:00006114       ??_C@_0M@CJNGHEBK@linear_attn?$AA@ 004a0114     bsplib.obj
 0002:00006120       ??_C@_0P@FEPJNKCE@quadratic_attn?$AA@ 004a0120     bsplib.obj
 0002:00006130       ??_C@_05HEIBENID@owner?$AA@ 004a0130     bsplib.obj
 0002:00006138       ??_C@_08BCLLBMPF@surfaceZ?$AA@ 004a0138     bsplib.obj
 0002:00006144       ??_C@_04BMEMFAGD@minZ?$AA@ 004a0144     bsplib.obj
 0002:0000614c       ??_C@_0BB@HHFELCML@surfaceTexInfoID?$AA@ 004a014c     bsplib.obj
 0002:00006160       ??_C@_09LGKNDAKM@firstpoly?$AA@ 004a0160     bsplib.obj
 0002:0000616c       ??_C@_09FHKLOLHG@polycount?$AA@ 004a016c     bsplib.obj
 0002:00006178       ??_C@_0BB@KCKOGCPC@firstvertexindex?$AA@ 004a0178     bsplib.obj
 0002:0000618c       ??_C@_0M@LGFIEHAP@vertexcount?$AA@ 004a018c     bsplib.obj
 0002:00006198       ??_C@_04IAGNFIBA@size?$AA@ 004a0198     bsplib.obj
 0002:000061a0       ??_C@_03HLJILIDP@nId?$AA@  004a01a0     bsplib.obj
 0002:000061a4       ??_C@_08ECOBNKEH@nTexInfo?$AA@ 004a01a4     bsplib.obj
 0002:000061b0       ??_C@_0BL@BMLGJAII@m_nFaceCountAndRenderOrder?$AA@ 004a01b0     bsplib.obj
 0002:000061cc       ??_C@_06FBJMKLEP@aFaces?$AA@ 004a01cc     bsplib.obj
 0002:000061d4       ??_C@_03EGPHBDGJ@flU?$AA@  004a01d4     bsplib.obj
 0002:000061d8       ??_C@_03GNNKEAKK@flV?$AA@  004a01d8     bsplib.obj
 0002:000061dc       ??_C@_0M@DNMEENHI@vecUVPoints?$AA@ 004a01dc     bsplib.obj
 0002:000061e8       ??_C@_09NFLAMELP@vecOrigin?$AA@ 004a01e8     bsplib.obj
 0002:000061f4       ??_C@_0P@BCDLPAHE@vecBasisNormal?$AA@ 004a01f4     bsplib.obj
 0002:00006204       ??_C@_0BA@OHDMMINB@flFadeDistMinSq?$AA@ 004a0204     bsplib.obj
 0002:00006214       ??_C@_0BA@KCDOILFD@flFadeDistMaxSq?$AA@ 004a0214     bsplib.obj
 0002:00006224       ??_C@_09NEJACIE@lumpCount?$AA@ 004a0224     bsplib.obj
 0002:00006230       ??_C@_06EJPGAGFJ@m_Name?$AA@ 004a0230     bsplib.obj
 0002:00006238       ??_C@_08ECNOKJJC@m_Origin?$AA@ 004a0238     bsplib.obj
 0002:00006244       ??_C@_08PILCLMDH@m_Angles?$AA@ 004a0244     bsplib.obj
 0002:00006250       ??_C@_0L@DKADNPBA@m_PropType?$AA@ 004a0250     bsplib.obj
 0002:0000625c       ??_C@_0M@PCPKPBEP@m_FirstLeaf?$AA@ 004a025c     bsplib.obj
 0002:00006268       ??_C@_0M@HIJBBFID@m_LeafCount?$AA@ 004a0268     bsplib.obj
 0002:00006274       ??_C@_07KCLBIANA@m_Solid?$AA@ 004a0274     bsplib.obj
 0002:0000627c       ??_C@_07ELHNBIGJ@m_Flags?$AA@ 004a027c     bsplib.obj
 0002:00006284       ??_C@_06FKMGMEBJ@m_Skin?$AA@ 004a0284     bsplib.obj
 0002:0000628c       ??_C@_0O@NDJEDMNM@m_FadeMinDist?$AA@ 004a028c     bsplib.obj
 0002:0000629c       ??_C@_0O@DFPEJDDN@m_FadeMaxDist?$AA@ 004a029c     bsplib.obj
 0002:000062ac       ??_C@_0BB@LGCHAJAF@m_LightingOrigin?$AA@ 004a02ac     bsplib.obj
 0002:000062c0       ??_C@_0BE@CDLLNLBJ@m_flForcedFadeScale?$AA@ 004a02c0     bsplib.obj
 0002:000062d4       ??_C@_0O@DNAIOLB@m_nMinDXLevel?$AA@ 004a02d4     bsplib.obj
 0002:000062e4       ??_C@_0O@MPNNPFLO@m_nMaxDXLevel?$AA@ 004a02e4     bsplib.obj
 0002:000062f4       ??_C@_06JOGDGIMJ@m_Leaf?$AA@ 004a02f4     bsplib.obj
 0002:000062fc       ??_C@_0O@IFMDLEOF@m_DetailModel?$AA@ 004a02fc     bsplib.obj
 0002:0000630c       ??_C@_0L@DIBKBJPK@m_Lighting?$AA@ 004a030c     bsplib.obj
 0002:00006318       ??_C@_0O@JEEBDPBL@m_LightStyles?$AA@ 004a0318     bsplib.obj
 0002:00006328       ??_C@_0BC@PMMMLGGN@m_LightStyleCount?$AA@ 004a0328     bsplib.obj
 0002:0000633c       ??_C@_0N@OCPKHEBL@m_SwayAmount?$AA@ 004a033c     bsplib.obj
 0002:0000634c       ??_C@_0N@PHKBCMEN@m_ShapeAngle?$AA@ 004a034c     bsplib.obj
 0002:0000635c       ??_C@_0M@LMGIPCHC@m_ShapeSize?$AA@ 004a035c     bsplib.obj
 0002:00006368       ??_C@_0O@IEBBNBA@m_Orientation?$AA@ 004a0368     bsplib.obj
 0002:00006378       ??_C@_0L@CKJLJANI@m_Padding2?$AA@ 004a0378     bsplib.obj
 0002:00006384       ??_C@_06OCPFMGCJ@m_Type?$AA@ 004a0384     bsplib.obj
 0002:0000638c       ??_C@_0L@DDIAKBJJ@m_Padding3?$AA@ 004a038c     bsplib.obj
 0002:00006398       ??_C@_09EBEAFDEH@m_flScale?$AA@ 004a0398     bsplib.obj
 0002:000063a4       ??_C@_04PNKKEILI@m_UL?$AA@ 004a03a4     bsplib.obj
 0002:000063ac       ??_C@_04DKBMOPJI@m_LR?$AA@ 004a03ac     bsplib.obj
 0002:000063b4       ??_C@_07FKFDNKFP@m_TexUL?$AA@ 004a03b4     bsplib.obj
 0002:000063bc       ??_C@_07JNOFHNHP@m_TexLR?$AA@ 004a03bc     bsplib.obj
 0002:000063c4       ??_C@_07MNJGHCEE@m_Style?$AA@ 004a03c4     bsplib.obj
 0002:000063cc       ??_C@_06MAPALLJB@m_nLod?$AA@ 004a03cc     bsplib.obj
 0002:000063d4       ??_C@_0M@NBOPACBB@m_nVertexes?$AA@ 004a03d4     bsplib.obj
 0002:000063e0       ??_C@_09FGLPPFBG@m_nOffset?$AA@ 004a03e0     bsplib.obj
 0002:000063ec       ??_C@_09BEMAELPI@m_nUnused?$AA@ 004a03ec     bsplib.obj
 0002:000063f8       ??_C@_0L@JPACMPLE@m_nVersion?$AA@ 004a03f8     bsplib.obj
 0002:00006404       ??_C@_0M@LAEBCFFC@m_nChecksum?$AA@ 004a0404     bsplib.obj
 0002:00006410       ??_C@_0P@LGPPEEMA@m_nVertexFlags?$AA@ 004a0410     bsplib.obj
 0002:00006420       ??_C@_0O@ONPOBLGK@m_nVertexSize?$AA@ 004a0420     bsplib.obj
 0002:00006430       ??_C@_09CHONMIDK@m_nMeshes?$AA@ 004a0430     bsplib.obj
 0002:0000643c       ??_C@_0CB@HNEIEEGN@Unknown?5occlusion?5lump?5version?$CB?6@ 004a043c     bsplib.obj
 0002:00006460       ??_C@_0L@JODPFALJ@vphysicsID?$AA@ 004a0460     bsplib.obj
 0002:0000646c       ??_C@_09NOHACFLB@modelType?$AA@ 004a046c     bsplib.obj
 0002:00006478       ??_C@_0M@DBJCOOM@surfaceSize?$AA@ 004a0478     bsplib.obj
 0002:00006484       ??_C@_0O@IFELHGBJ@dragAxisAreas?$AA@ 004a0484     bsplib.obj
 0002:00006494       ??_C@_0M@HLOKJILB@axisMapSize?$AA@ 004a0494     bsplib.obj
 0002:000064a0       ??_C@_08CCCKJNKJ@moppSize?$AA@ 004a04a0     bsplib.obj
 0002:000064ac       ??_C@_0BJ@JDOEEAFA@odd?5size?5for?5LUMP_LEAFS?6?$AA@ 004a04ac     bsplib.obj
 0002:000064c8       ??_C@_0BM@KBEAGEDM@Unknown?5LUMP_LEAFS?5version?6?$AA@ 004a04c8     bsplib.obj
 0002:000064e4       ??_C@_0L@KFNFGCAJ@?$CC?$CFs?$CC?5?$CC?$CFs?$CC?6?$AA@ 004a04e4     bsplib.obj
 0002:000064f0       __real@4e6e6b28            004a04f0     builddisp.obj
 0002:000064f4       __real@47c34f80            004a04f4     builddisp.obj
 0002:000064f8       __real@3fe0000000000000    004a04f8     builddisp.obj
 0002:00006500       __real@42fa0000            004a0500     builddisp.obj
 0002:00006508       ??_7CDispUtilsHelper@@6B@  004a0508     builddisp.obj
 0002:0000651c       ??_7CCoreDispInfo@@6B@     004a051c     builddisp.obj
 0002:0000652c       __real@3f800054            004a052c     builddisp.obj
 0002:00006530       __real@3f800008            004a0530     builddisp.obj
 0002:00006538       ??_7ios_base@std@@6B@      004a0538     chunkfile.obj
 0002:0000653c       ??_C@_08HPBFPDOD@error?5?$CFd?$AA@ 004a053c     chunkfile.obj
 0002:00006548       ??_C@_0CH@BEKFMMLP@unterminated?5string?5or?5string?5to@ 004a0548     chunkfile.obj
 0002:00006570       ??_C@_0BH@IIAFKHHE@unexpected?5symbol?5?8?$CFs?8?$AA@ 004a0570     chunkfile.obj
 0002:00006588       ??_C@_0BH@CFIIDOJD@unexpected?5end?5of?5file?$AA@ 004a0588     chunkfile.obj
 0002:000065a0       ??_C@_0L@OGNGFIGA@?$FL?$CFf?5?$CFf?5?$CFf?$FN?$AA@ 004a05a0     chunkfile.obj
 0002:000065ac       ??_C@_02PCIJFNDE@?$AN?6?$AA@ 004a05ac     chunkfile.obj
 0002:000065b4       ??_7?$basic_istream@DU?$char_traits@D@std@@@std@@6B@ 004a05b4     chunkfile.obj
 0002:000065bc       ??_7?$basic_streambuf@DU?$char_traits@D@std@@@std@@6B@ 004a05bc     chunkfile.obj
 0002:000065f8       ??_7?$basic_filebuf@DU?$char_traits@D@std@@@std@@6B@ 004a05f8     chunkfile.obj
 0002:00006634       ??_7facet@locale@std@@6B@  004a0634     chunkfile.obj
 0002:0000663c       ??_7runtime_error@std@@6B@ 004a063c     chunkfile.obj
 0002:00006644       ??_C@_0BA@ELKIONDK@bad?5locale?5name?$AA@ 004a0644     chunkfile.obj
 0002:00006658       ??_7?$codecvt@DDH@std@@6B@ 004a0658     chunkfile.obj
 0002:00006678       ??_C@_01GFHCPBMG@C?$AA@    004a0678     chunkfile.obj
 0002:00006680       ??_7?$basic_ifstream@DU?$char_traits@D@std@@@std@@6B@ 004a0680     chunkfile.obj
 0002:00006684       ??_C@_0BJ@HHDOALOL@?6Press?5any?5key?5to?5quit?4?6?$AA@ 004a0684     cmdlib.obj
 0002:000066a0       ??_C@_01KICIPPFI@?2?$AA@   004a06a0     cmdlib.obj
 0002:000066a4       ??_C@_0M@BBODMOGM@?$CFd?5second?$CFs?$AA@ 004a06a4     cmdlib.obj
 0002:000066b0       ??_C@_0BJ@KMIJFNCM@?$CFd?5minute?$CFs?0?5?$CFd?5second?$CFs?$AA@ 004a06b0     cmdlib.obj
 0002:000066cc       ??_C@_0CE@PALCMKJH@?$CFd?5hour?$CFs?0?5?$CFd?5minute?$CFs?0?5?$CFd?5secon@ 004a06cc     cmdlib.obj
 0002:000066f0       ??_C@_01LKDEMHDF@s?$AA@    004a06f0     cmdlib.obj
 0002:000066f4       ??_C@_0BO@EENJAGHE@CmdLib_InitFileSystem?5failed?4?$AA@ 004a06f4     cmdlib.obj
 0002:00006714       ??_C@_0BC@HMDGJKFB@Error?5opening?5?$CFs?6?$AA@ 004a0714     cmdlib.obj
 0002:00006728       ??_C@_0BC@OGGEBGDM@File?5read?5failure?$AA@ 004a0728     cmdlib.obj
 0002:0000673c       ??_C@_0BD@IHJMODLC@File?5write?5failure?$AA@ 004a073c     cmdlib.obj
 0002:00006750       ??_C@_01OGPIMHDM@?$DP?$AA@ 004a0750     cmdlib.obj
 0002:00006754       ??_C@_01NBENCBCI@?$CK?$AA@ 004a0754     cmdlib.obj
 0002:00006758       ??_C@_0CP@DAHDEIHG@CmdLib_FPrintf?3?5can?8t?5allocate?5s@ 004a0758     cmdlib.obj
 0002:00006788       ??_C@_03EGHOKNNL@?6?6?6?$AA@ 004a0788     cmdlib.obj
 0002:0000678c       ??_C@_0BL@BBEKHHIC@Can?8t?5create?5LogFile?3?$CC?$CFs?$CC?6?$AA@ 004a078c     cmdlib.obj
 0002:000067a8       ??_C@_01MCMALHOG@a?$AA@    004a07a8     cmdlib.obj
 0002:000067ac       ??_C@_05JPPLNOIE@?$CFs?$DN?$CFs?$AA@ 004a07ac     filesystem_init.obj
 0002:000067b4       ??_C@_03HFAIOBFI@?$CFs?$DN?$AA@ 004a07b4     filesystem_init.obj
 0002:000067b8       ??_C@_0BI@HONGKJJH@?$CFs?$CFclocalization?$CFc?$CFs_?$CFs?$AA@ 004a07b8     filesystem_init.obj
 0002:000067d0       ??_C@_06KGBLPGBA@?2game?2?$AA@ 004a07d0     filesystem_init.obj
 0002:000067d8       ??_C@_05ONEOBAM@?$CFs_?$CFs?$AA@ 004a07d8     filesystem_init.obj
 0002:000067e0       ??_C@_07FIIABPFG@GAMEBIN?$AA@ 004a07e0     filesystem_init.obj
 0002:000067e8       ??_C@_07FCGPJGAE@?$CFs?$CFcbin?$AA@ 004a07e8     filesystem_init.obj
 0002:000067f0       ??_C@_0N@GOJIOGBD@User?5Token?53?$AA@ 004a07f0     filesystem_init.obj
 0002:00006800       ??_C@_0N@HHIDNHFC@User?5Token?52?$AA@ 004a0800     filesystem_init.obj
 0002:00006810       ??_C@_0BP@EFOCGGID@Software?2Valve?2Source?2Settings?$AA@ 004a0810     filesystem_init.obj
 0002:00006830       ??_C@_03FIBGOAPP@MOD?$AA@  004a0830     filesystem_init.obj
 0002:00006834       ??_C@_0P@OBDLCKKL@?$CFs_tempcontent?$AA@ 004a0834     filesystem_init.obj
 0002:00006844       ??_C@_0N@MOHILAIK@?9tempcontent?$AA@ 004a0844     filesystem_init.obj
 0002:00006854       ??_C@_05MOIKDAG@?$CFs_lv?$AA@ 004a0854     filesystem_init.obj
 0002:0000685c       ??_C@_04MJNAPEEI@game?$AA@ 004a085c     filesystem_init.obj
 0002:00006868       ??_C@_0EB@JBHGIPO@FileSystem_AddLoadedSearchPath?5?9@ 004a0868     filesystem_init.obj
 0002:000068ac       ??_C@_0BE@MHMPCCEN@SteamUserPassphrase?$AA@ 004a08ac     filesystem_init.obj
 0002:000068c0       ??_C@_0BN@ILMJFDLH@Missing?5SteamAppId?5in?5?$CFs?2?$CFs?4?$AA@ 004a08c0     filesystem_init.obj
 0002:000068e0       ??_C@_0N@DDAKDDIF@gameinfo?4txt?$AA@ 004a08e0     filesystem_init.obj
 0002:000068f0       ??_C@_0L@ECGBBIEJ@SteamAppId?$AA@ 004a08f0     filesystem_init.obj
 0002:000068fc       ??_C@_08FONOGHLN@PLATFORM?$AA@ 004a08fc     filesystem_init.obj
 0002:00006908       ??_C@_0N@MHLNGBBM@?1?4?4?1platform?$AA@ 004a0908     filesystem_init.obj
 0002:00006918       ??_C@_08CBHCFJJK@platform?$AA@ 004a0918     filesystem_init.obj
 0002:00006924       ??_C@_04OJGJKDCG@?2bin?$AA@ 004a0924     filesystem_init.obj
 0002:0000692c       ??_C@_03PDOMKJON@bin?$AA@  004a092c     filesystem_init.obj
 0002:00006930       ??_C@_0M@HIDIPGMM@?$CFs?$CFc?4?4?$CFcbin?$AA@ 004a0930     filesystem_init.obj
 0002:0000693c       ??_C@_08BBHFPNLA@VProject?$AA@ 004a093c     filesystem_init.obj
 0002:00006948       ??_C@_0M@BPBMEHMA@vconfig?4exe?$AA@ 004a0948     filesystem_init.obj
 0002:00006954       ??_C@_09FEGFDDAO@orangebox?$AA@ 004a0954     filesystem_init.obj
 0002:00006960       ??_C@_0DG@DHDKLFGP@Can?8t?5find?5steam?4dll?5relative?5to@ 004a0960     filesystem_init.obj
 0002:00006998       ??_C@_05LKJAIBFI@?$CFs?$DL?$CFs?$AA@ 004a0998     filesystem_init.obj
 0002:000069a0       ??_C@_0DH@CHNFKOPG@Can?8t?5find?5steam?4dll?5relative?5to@ 004a09a0     filesystem_init.obj
 0002:000069d8       ??_C@_0N@KIPMNOMO@steamapp?4cfg?$AA@ 004a09d8     filesystem_init.obj
 0002:000069e8       ??_C@_09OPNECJBP@steam?4dll?$AA@ 004a09e8     filesystem_init.obj
 0002:000069f4       ??_C@_0CE@ICDPACDF@FileSystem_GetExecutableDir?5fail@ 004a09f4     filesystem_init.obj
 0002:00006a18       ??_C@_0DK@HCONFMCF@SetSteamInstallPath?3?5FileSystem_@ 004a0a18     filesystem_init.obj
 0002:00006a54       ??_C@_0BA@PDPKJDAD@EXECUTABLE_PATH?$AA@ 004a0a54     filesystem_init.obj
 0002:00006a64       ??_C@_0BJ@EDPLIIJG@?$CFs?$CFcfilesystem_steam?4dll?$AA@ 004a0a64     filesystem_init.obj
 0002:00006a80       ??_C@_0M@LHJIEJJB@?9steamlocal?$AA@ 004a0a80     filesystem_init.obj
 0002:00006a8c       ??_C@_0BJ@PBHGGHGE@?$CFs?$CFcfilesystem_stdio?4dll?$AA@ 004a0a8c     filesystem_init.obj
 0002:00006aa8       ??_C@_06HPIJBGJD@?1game?1?$AA@ 004a0aa8     filesystem_init.obj
 0002:00006ab0       ??_C@_09EOPDDICB@?1content?1?$AA@ 004a0ab0     filesystem_init.obj
 0002:00006ac0       ??_C@_0OI@HCHEELJO@Unable?5to?5find?5?$CFs?4?5Solutions?3?6?61@ 004a0ac0     filesystem_init.obj
 0002:00006ba8       ??_C@_01LFCBOECM@?4?$AA@   004a0ba8     filesystem_init.obj
 0002:00006bb0       ??_C@_0EA@HIENCNPL@Warning?3?5falling?5back?5to?5auto?5de@ 004a0bb0     filesystem_init.obj
 0002:00006bf0       ??_C@_0GD@JOJOEGKB@Setup?5file?5?8?$CFs?8?5doesn?8t?5exist?5in@ 004a0bf0     filesystem_init.obj
 0002:00006c54       ??_C@_0DB@DMFGMLBG@bOnlyUseDirectoryName?$DN1?5and?5pDir@ 004a0c54     filesystem_init.obj
 0002:00006c88       ??_C@_04LNEJFJGI@path?$AA@ 004a0c88     filesystem_init.obj
 0002:00006c90       ??_C@_0N@JBMCJGB@SteamAppUser?$AA@ 004a0c90     filesystem_init.obj
 0002:00006ca0       ??_C@_0M@OGFGHLLN@SearchPaths?$AA@ 004a0ca0     filesystem_init.obj
 0002:00006cac       ??_C@_0BK@LENANHBB@?$CFs?5is?5not?5a?5valid?5format?4?$AA@ 004a0cac     filesystem_init.obj
 0002:00006cc8       ??_C@_0L@FPFLHALM@FileSystem?$AA@ 004a0cc8     filesystem_init.obj
 0002:00006cd4       ??_C@_0P@BAICOJOC@?$CFs?5is?5missing?4?$AA@ 004a0cd4     filesystem_init.obj
 0002:00006ce4       ??_C@_0DK@HDHHNFK@FileSystem_LoadSearchPaths?3?5Inva@ 004a0ce4     filesystem_init.obj
 0002:00006d20       ??_C@_0BD@BIHGFCAJ@DEFAULT_WRITE_PATH?$AA@ 004a0d20     filesystem_init.obj
 0002:00006d34       ??_C@_03FFONCNID@mod?$AA@  004a0d34     filesystem_init.obj
 0002:00006d38       ??_C@_07KFNNKDNC@gamebin?$AA@ 004a0d38     filesystem_init.obj
 0002:00006d40       ??_C@_0BA@LLOKIJCD@executable_path?$AA@ 004a0d40     filesystem_init.obj
 0002:00006d50       ??_C@_06NKJBFAKB@?4?4?$CFc?$CFs?$AA@ 004a0d50     filesystem_init.obj
 0002:00006d58       ??_C@_0BK@FOIMLNGE@?$HMall_source_engine_paths?$HM?$AA@ 004a0d58     filesystem_init.obj
 0002:00006d74       ??_C@_0BA@MDDINGGJ@?$HMgameinfo_path?$HM?$AA@ 004a0d74     filesystem_init.obj
 0002:00006d84       ??_C@_0BO@DKGHAMPB@FileSystem_GetBaseDir?5failed?4?$AA@ 004a0d84     filesystem_init.obj
 0002:00006da4       ??_C@_0CA@LJBFCIPK@Can?8t?5find?5steam?5app?5user?5info?4?$AA@ 004a0da4     filesystem_init.obj
 0002:00006dc4       ??_C@_0O@JKIHLNMO@AutoLoginUser?$AA@ 004a0dc4     filesystem_init.obj
 0002:00006dd4       ??_C@_0BI@FPAAOPPO@config?2SteamAppData?4vdf?$AA@ 004a0dd4     filesystem_init.obj
 0002:00006dec       ??_C@_0O@GIMNLJAG@steaminfo?4txt?$AA@ 004a0dec     filesystem_init.obj
 0002:00006dfc       ??_C@_0L@INNOAPAJ@ToolsAppId?$AA@ 004a0dfc     filesystem_init.obj
 0002:00006e08       ??_C@_0BN@OJPKFLKO@?$CFs?5IFileSystem?3?3Init?5failed?4?$AA@ 004a0e08     filesystem_init.obj
 0002:00006e28       ??_C@_0CA@KIDODKHJ@?$CFs?5IFileSystem?3?3Connect?5failed?4?$AA@ 004a0e28     filesystem_init.obj
 0002:00006e48       ??_C@_0P@HNMHCAOM@Can?8t?5load?5?$CFs?4?$AA@ 004a0e48     filesystem_init.obj
 0002:00006e58       ??_C@_0DB@IJEHBEGI@Unable?5to?5mount?5Steam?5content?5in@ 004a0e58     filesystem_init.obj
 0002:00006e8c       ??_C@_0M@CHBCHPDB@?4?4?1platform?$AA@ 004a0e8c     filesystem_tools.obj
 0002:00006e98       ??_C@_0L@HEEMIGIK@mapversion?$AA@ 004a0e98     map_shared.obj
 0002:00006ea4       ??_C@_08GKHEJHEP@hammerid?$AA@ 004a0ea4     map_shared.obj
 0002:00006eb0       ??_C@_0L@CGBMHOHE@func_water?$AA@ 004a0eb0     map_shared.obj
 0002:00006ebc       __real@42200000            004a0ebc     pacifier.obj
 0002:00006ec0       ??_C@_0CD@BOFJFDD@FreeWinding?3?5freed?5a?5freed?5windi@ 004a0ec0     polylib.obj
 0002:00006ee4       __real@47800000            004a0ee4     polylib.obj
 0002:00006ee8       ??_C@_0CD@BHBKGNIF@BaseWindingForPlane?3?5no?5axis?5fou@ 004a0ee8     polylib.obj
 0002:00006f0c       ??_C@_0CD@PEDPMDOJ@ClipWinding?3?5MAX_POINTS_ON_WINDI@ 004a0f0c     polylib.obj
 0002:00006f30       ??_C@_0CG@OLJCNKCC@ClipWinding?3?5points?5exceeded?5est@ 004a0f30     polylib.obj
 0002:00006f58       ??_C@_0CK@NIJIDEPG@ReadFileToBuffer?$CI?$CJ?3?5Error?5openin@ 004a0f58     scriplib.obj
 0002:00006f84       ??_C@_06IHDMMOPO@?$CFs?4tmp?$AA@ 004a0f84     scriplib.obj
 0002:00006f8c       ??_C@_04IMHDFGMD@mgd_?$AA@ 004a0f8c     scriplib.obj
 0002:00006f98       ??_7CScriptLib@@6B@        004a0f98     scriplib.obj
 0002:00006fb4       ??_C@_02DJGKEECL@?4?4?$AA@ 004a0fb4     scriplib.obj
 0002:00006fb8       ??_C@_02CEGDFPFP@?4?2?$AA@ 004a0fb8     scriplib.obj
 0002:00006fbc       ??_C@_03FFNGDGKN@tmp?$AA@  004a0fbc     scriplib.obj
 0002:00006fc0       ??_C@_04FGEHGIFJ@temp?$AA@ 004a0fc0     scriplib.obj
 0002:00006fc8       ??_C@_0M@FBLNEIAD@?$CFi?5threads?6?$AA@ 004a0fc8     threads.obj
 0002:00006fd4       ??_C@_0BG@BEEOCMHK@Recursive?5ThreadLock?6?$AA@ 004a0fd4     threads.obj
 0002:00006fec       ??_C@_0BL@HADBLPO@ThreadUnlock?5without?5lock?6?$AA@ 004a0fec     threads.obj
 0002:00007008       ??_C@_06MEKNBDFO@?5?$CI?$CFi?$CJ?6?$AA@ 004a1008     threads.obj
 0002:00007010       __real@4048000000000000    004a1010     tier1:strtools.obj
 0002:00007018       ??_C@_0CH@DNILKGJA@V_AppendSlash?3?5ran?5out?5of?5space?5@ 004a1018     tier1:strtools.obj
 0002:00007040       __real@447a0000            004a1040     tier1:strtools.obj
 0002:00007044       ??_C@_01JOAMLHOP@?9?$AA@   004a1044     tier1:strtools.obj
 0002:00007048       ??_C@_03OOAAEEIB@?4?$CFc?$AA@ 004a1048     tier1:strtools.obj
 0002:0000704c       ??_C@_02CAHBHFGK@?4?1?$AA@ 004a104c     tier1:strtools.obj
 0002:00007050       ??_C@_0DB@FOILCOJM@V_MakeAbsolutePath?3?5tried?5to?5?$CC?4?4@ 004a1050     tier1:strtools.obj
 0002:00007084       ??_C@_0CE@INIPJBEP@V_MakeAbsolutePath?3?5_getcwd?5fail@ 004a1084     tier1:strtools.obj
 0002:000070a8       ??_C@_01GEODFPGF@?8?$AA@   004a10a8     tier1:utlbuffer.obj
 0002:000070ac       ??_C@_01INIBCBCB@f?$AA@    004a10ac     tier1:utlbuffer.obj
 0002:000070b0       ??_C@_01KDCPPGHE@r?$AA@    004a10b0     tier1:utlbuffer.obj
 0002:000070b4       ??_C@_01OJONOECF@b?$AA@    004a10b4     tier1:utlbuffer.obj
 0002:000070b8       ??_C@_01PFHFFBPC@t?$AA@    004a10b8     tier1:utlbuffer.obj
 0002:000070bc       ??_C@_01EFFIKLCJ@n?$AA@    004a10bc     tier1:utlbuffer.obj
 0002:000070c4       ??_7CUtlCharConversion@@6B@ 004a10c4     tier1:utlbuffer.obj
 0002:000070cc       ??_7CUtlNoEscConversion@@6B@ 004a10cc     tier1:utlbuffer.obj
 0002:000070d4       ??_7CUtlCStringConversion@@6B@ 004a10d4     tier1:utlbuffer.obj
 0002:000070d8       ??_C@_02HAOIJKIC@?$CFc?$AA@ 004a10d8     tier1:utlbuffer.obj
 0002:000070dc       ??_C@_07CIFAGBMG@unknown?$AA@ 004a10dc     tier1:KeyValues.obj
 0002:000070e4       ??_C@_04HIBGFPH@NULL?$AA@  004a10e4     tier1:KeyValues.obj
 0002:000070ec       ??_C@_08KKMCJABH@?$CI?$CK?$CFs?$CK?$CJ?0?5?$AA@ 004a10ec     tier1:KeyValues.obj
 0002:000070f8       ??_C@_04ONKFDMMC@?$CFs?0?5?$AA@ 004a10f8     tier1:KeyValues.obj
 0002:00007100       ??_C@_0CA@NDDGCEEP@KeyValues?5Error?3?5?$CFs?5in?5file?5?$CFs?6?$AA@ 004a1100     tier1:KeyValues.obj
 0002:00007120       ??_C@_0BE@CCEENLEF@?5ReadToken?5overflow?$AA@ 004a1120     tier1:KeyValues.obj
 0002:00007134       ??_C@_08HHEPHHEL@?$FL$WIN32?$FN?$AA@ 004a1134     tier1:KeyValues.obj
 0002:00007140       ??_C@_01GPOEFGEJ@?7?$AA@   004a1140     tier1:KeyValues.obj
 0002:00007148       ??_C@_0EE@MCLHPPL@KeyValues?3?3RecursiveSaveToFile?3?5@ 004a1148     tier1:KeyValues.obj
 0002:0000718c       ??_C@_02NJPGOMH@?$CFf?$AA@ 004a118c     tier1:KeyValues.obj
 0002:00007190       ??_C@_0L@BJLDBJPB@0x?$CF016I64X?$AA@ 004a1190     tier1:KeyValues.obj
 0002:0000719c       ??_C@_04FHLHEGKD@?$CC?7?7?$CC?$AA@ 004a119c     tier1:KeyValues.obj
 0002:000071a4       ??_C@_05OKCMKDO@?$CFI64i?$AA@ 004a11a4     tier1:KeyValues.obj
 0002:000071b0       ??_C@_0EA@NBPAKPMP@RecursiveLoadFromBuffer?3?5?5got?5co@ 004a11b0     tier1:KeyValues.obj
 0002:000071f0       ??_C@_0CH@FAEPDIPE@RecursiveLoadFromBuffer?3?5?5got?5?$HN?5@ 004a11f0     tier1:KeyValues.obj
 0002:00007218       ??_C@_0CH@HEKCOJBB@RecursiveLoadFromBuffer?3?5?5got?5NU@ 004a1218     tier1:KeyValues.obj
 0002:00007240       ??_C@_0CM@EGPGDPNF@RecursiveLoadFromBuffer?3?5?5got?5em@ 004a1240     tier1:KeyValues.obj
 0002:0000726c       ??_C@_0DF@BNKODCEE@RecursiveLoadFromBuffer?3?5?5got?5EO@ 004a126c     tier1:KeyValues.obj
 0002:000072a8       ??_C@_0EH@OAIGODPC@KeyValues?3?3ParseIncludedKeys?3?5Co@ 004a12a8     tier1:KeyValues.obj
 0002:000072f0       ??_C@_0BK@NIPBBFNB@LoadFromBuffer?3?5missing?5?$HL?$AA@ 004a12f0     tier1:KeyValues.obj
 0002:0000730c       ??_C@_0P@NHINIODK@?$CDbase?5is?5NULL?5?$AA@ 004a130c     tier1:KeyValues.obj
 0002:0000731c       ??_C@_05OBFANEGE@?$CDbase?$AA@ 004a131c     tier1:KeyValues.obj
 0002:00007324       ??_C@_0BC@NGELGJPP@?$CDinclude?5is?5NULL?5?$AA@ 004a1324     tier1:KeyValues.obj
 0002:00007338       ??_C@_08GPLAJCBH@?$CDinclude?$AA@ 004a1338     tier1:KeyValues.obj
 0002:00007344       ??_C@_04HLONOPDM@?4dll?$AA@ 004a1344     tier1:interface.obj
 0002:0000734c       ??_C@_0BM@OIEJAJOK@Module?5?$CFs?5is?5a?5debug?5build?6?$AA@ 004a134c     tier1:interface.obj
 0002:00007368       ??_C@_0L@EJCNAOMG@BuiltDebug?$AA@ 004a1368     tier1:interface.obj
 0002:00007374       ??_C@_09ILGMALND@?$CFs?1bin?1?$CFs?$AA@ 004a1374     tier1:interface.obj
 0002:00007380       ??_C@_05GFOLEBJA@?$CFs?1?$CFs?$AA@ 004a1380     tier1:interface.obj
 0002:00007388       ??_C@_04MMFEEKAB@bin?1?$AA@ 004a1388     tier1:interface.obj
 0002:00007390       ??_C@_0BA@OBHPCBFP@CreateInterface?$AA@ 004a1390     tier1:interface.obj
 0002:000077a0       ??_C@_0BD@DDNAMMCP@File?5?$CFs?0?5line?5?$CFd?3?5?$AA@ 004a17a0     tier1:tokenreader.obj
 0002:000077b8       ??_7?$basic_ios@DU?$char_traits@D@std@@@std@@6B@ 004a17b8     tier1:tokenreader.obj
 0002:000077c0       ??_7failure@ios_base@std@@6B@ 004a17c0     tier1:tokenreader.obj
 0002:000077cc       ??_7?$ctype@D@std@@6B@     004a17cc     tier1:tokenreader.obj
 0002:000077f8       ??_C@_0BF@OOHOMBOF@ios_base?3?3eofbit?5set?$AA@ 004a17f8     tier1:tokenreader.obj
 0002:00007810       ??_C@_0BG@FMKFHCIL@ios_base?3?3failbit?5set?$AA@ 004a1810     tier1:tokenreader.obj
 0002:00007828       ??_C@_0BF@PHHKMMFD@ios_base?3?3badbit?5set?$AA@ 004a1828     tier1:tokenreader.obj
 0002:00007840       ??_C@_08EPJLHIJG@bad?5cast?$AA@ 004a1840     tier1:tokenreader.obj
 0002:0000784c       ??_8?$basic_ifstream@DU?$char_traits@D@std@@@std@@7B@ 004a184c     tier1:tokenreader.obj
 0002:00007858       ??_7TokenReader@@6B@       004a1858     tier1:tokenreader.obj
 0002:0000785c       ??_8TokenReader@@7B@       004a185c     tier1:tokenreader.obj
 0002:00007864       ?nanmask@@3HB              004a1864     mathlib:mathlib_base.obj
 0002:00007868       __real@34000000            004a1868     mathlib:mathlib_base.obj
 0002:00007870       __real@3f9921fb54442d18    004a1870     mathlib:mathlib_base.obj
 0002:00007878       __real@42652ee1            004a1878     mathlib:mathlib_base.obj
 0002:0000787c       __real@43b40000            004a187c     mathlib:mathlib_base.obj
 0002:00007880       __real@3fd45f306dc9c883    004a1880     mathlib:mathlib_base.obj
 0002:00007888       __real@3c8efa35            004a1888     mathlib:mathlib_base.obj
 0002:00007890       __real@4000000000000000    004a1890     mathlib:mathlib_base.obj
 0002:00007898       __real@3e000000            004a1898     mathlib:mathlib_base.obj
 0002:0000789c       __real@c0000000            004a189c     mathlib:mathlib_base.obj
 0002:000078a0       ?Four_PointFives@@3T__m128@@B 004a18a0     mathlib:sseconst.obj
 0002:000078b0       ?Four_Zeros@@3T__m128@@B   004a18b0     mathlib:sseconst.obj
 0002:000078c0       ?Four_Ones@@3T__m128@@B    004a18c0     mathlib:sseconst.obj
 0002:000078d0       ?Four_Twos@@3T__m128@@B    004a18d0     mathlib:sseconst.obj
 0002:000078e0       ?Four_Threes@@3T__m128@@B  004a18e0     mathlib:sseconst.obj
 0002:000078f0       ?Four_Fours@@3T__m128@@B   004a18f0     mathlib:sseconst.obj
 0002:00007900       ?Four_Origin@@3T__m128@@B  004a1900     mathlib:sseconst.obj
 0002:00007910       ?Four_2ToThe21s@@3T__m128@@B 004a1910     mathlib:sseconst.obj
 0002:00007920       ?Four_2ToThe22s@@3T__m128@@B 004a1920     mathlib:sseconst.obj
 0002:00007930       ?Four_2ToThe23s@@3T__m128@@B 004a1930     mathlib:sseconst.obj
 0002:00007940       ?Four_2ToThe24s@@3T__m128@@B 004a1940     mathlib:sseconst.obj
 0002:00007950       ?Four_Point225s@@3T__m128@@B 004a1950     mathlib:sseconst.obj
 0002:00007960       ?Four_Epsilons@@3T__m128@@B 004a1960     mathlib:sseconst.obj
 0002:00007970       ?Four_FLT_MAX@@3T__m128@@B 004a1970     mathlib:sseconst.obj
 0002:00007980       ?Four_Negative_FLT_MAX@@3T__m128@@B 004a1980     mathlib:sseconst.obj
 0002:00007990       ?g_SIMD_clear_signmask@@3QBHB 004a1990     mathlib:sseconst.obj
 0002:000079a0       ?g_SIMD_signmask@@3QBHB    004a19a0     mathlib:sseconst.obj
 0002:000079b0       ?g_SIMD_lsbmask@@3QBHB     004a19b0     mathlib:sseconst.obj
 0002:000079c0       ?g_SIMD_clear_wmask@@3QBHB 004a19c0     mathlib:sseconst.obj
 0002:000079d0       ?g_SIMD_ComponentMask@@3QAY03$$CBHA 004a19d0     mathlib:sseconst.obj
 0002:00007a10       __real@40019999a0000000    004a1a10     mathlib:color_conversion.obj
 0002:00007a18       __real@3fdd1745c0000000    004a1a18     mathlib:color_conversion.obj
 0002:00007a20       __real@3f50000000000000    004a1a20     mathlib:color_conversion.obj
 0002:00007a28       __real@3fec000000000000    004a1a28     mathlib:color_conversion.obj
 0002:00007a30       __real@3f50040100401004    004a1a30     mathlib:color_conversion.obj
 0002:00007a38       __real@3fc0000000000000    004a1a38     mathlib:color_conversion.obj
 0002:00007a40       __real@3fb3333333333333    004a1a40     mathlib:color_conversion.obj
 0002:00007a48       __real@3d4ccccd            004a1a48     mathlib:color_conversion.obj
 0002:00007b10       ??_C@_0BE@DFJMOMFG@VTFFileHeaderX360_t?$AA@ 004a1b10     vtf:vtf.obj
 0002:00007b24       ??_C@_0BA@PDDLLJA@VTFFileHeader_t?$AA@ 004a1b24     vtf:vtf.obj
 0002:00007b34       ??_C@_0BE@HIKFGPMP@VTFFileHeaderV7_3_t?$AA@ 004a1b34     vtf:vtf.obj
 0002:00007b48       ??_C@_0BE@MABJAIKK@VTFFileHeaderV7_2_t?$AA@ 004a1b48     vtf:vtf.obj
 0002:00007b5c       ??_C@_0BE@NCKMKHEE@VTFFileHeaderV7_1_t?$AA@ 004a1b5c     vtf:vtf.obj
 0002:00007b70       ??_C@_0BE@HCIDAHJO@VTFFileBaseHeader_t?$AA@ 004a1b70     vtf:vtf.obj
 0002:00007b84       __real@3ecccccd            004a1b84     vtf:vtf.obj
 0002:00007b88       ??_C@_0DO@GBPJBKJC@Warning?$CB?5Encountered?5old?5format?5@ 004a1b88     vtf:vtf.obj
 0002:00007bc8       ??_C@_0DJ@LIBGGGAP@?$CK?$CK?$CK?5Encountered?5VTF?5file?5with?5an@ 004a1bc8     vtf:vtf.obj
 0002:00007c04       __real@3e4ccccd            004a1c04     vtf:vtf.obj
 0002:00007c08       ??_C@_0P@DBIAMLO@?5?5?5?$CFc?$DN?$CFd?5?$HO?$CFd?$CF?$CF?$AA@ 004a1c08     vtf:vtf.obj
 0002:00007c18       ??_C@_0BI@BDJEJLNC@Blending?5mip?$CFd?5?$CFdx?$CFd?5to?$AA@ 004a1c18     vtf:vtf.obj
 0002:00007c30       ??_C@_0DF@GPPDIPDC@BlendCubeMapFaceEdges?3?5unsupport@ 004a1c30     vtf:vtf.obj
 0002:00007c68       ??_C@_0DH@FCHKBKML@?$CK?$CK?$CK?5Encountered?5VTF?5file?5with?5an@ 004a1c68     vtf:vtf.obj
 0002:00007ca0       ??_C@_0DD@PIDBFMOO@?$CK?$CK?$CK?5Encountered?5VTF?5file?5with?5an@ 004a1ca0     vtf:vtf.obj
 0002:00007cd4       ??_C@_0DB@LAMDBMNJ@?$CK?$CK?$CK?5Tried?5to?5load?5a?5non?9VTF?5file@ 004a1cd4     vtf:vtf.obj
 0002:00007d08       ??_C@_03PNELBOHC@VTF?$AA@  004a1d08     vtf:vtf.obj
 0002:00007d0c       ??_C@_0DI@LLDOCADD@?$CK?$CK?$CK?5Error?5unserializing?5VTF?5file@ 004a1d0c     vtf:vtf.obj
 0002:00007d4c       ??_7CVTFTexture@@6B@       004a1d4c     vtf:vtf.obj
 0002:00007e28       ??_C@_0DA@JGJBJOIC@?$CK?$CK?$CK?5Unable?5to?5serialize?4?4?4?5have?5@ 004a1e28     vtf:vtf.obj
 0002:00007e58       ??_C@_0P@MLAPKELC@fileTypeString?$AA@ 004a1e58     vtf:vtf.obj
 0002:00007e68       ??_C@_0L@LBANHNIC@headerSize?$AA@ 004a1e68     vtf:vtf.obj
 0002:00007e74       ??_C@_09GEKACOOO@numFrames?$AA@ 004a1e74     vtf:vtf.obj
 0002:00007e80       ??_C@_0L@DAFMKFBI@startFrame?$AA@ 004a1e80     vtf:vtf.obj
 0002:00007e8c       ??_C@_09FKIAOKBL@bumpScale?$AA@ 004a1e8c     vtf:vtf.obj
 0002:00007e98       ??_C@_0M@KCNMOFJC@imageFormat?$AA@ 004a1e98     vtf:vtf.obj
 0002:00007ea4       ??_C@_0N@PAMEODPM@numMipLevels?$AA@ 004a1ea4     vtf:vtf.obj
 0002:00007eb4       ??_C@_0BC@ODLGANAI@lowResImageFormat?$AA@ 004a1eb4     vtf:vtf.obj
 0002:00007ec8       ??_C@_0BB@HCODKAMG@lowResImageWidth?$AA@ 004a1ec8     vtf:vtf.obj
 0002:00007edc       ??_C@_0BC@GFEOCIEL@lowResImageHeight?$AA@ 004a1edc     vtf:vtf.obj
 0002:00007ef0       ??_C@_05BJGJGKJC@depth?$AA@ 004a1ef0     vtf:vtf.obj
 0002:00007ef8       ??_C@_0N@GMGDCOGH@numResources?$AA@ 004a1ef8     vtf:vtf.obj
 0002:00007f08       ??_C@_0BA@NBJOFFPL@preloadDataSize?$AA@ 004a1f08     vtf:vtf.obj
 0002:00007f18       ??_C@_0N@JKABNMJG@mipSkipCount?$AA@ 004a1f18     vtf:vtf.obj
 0002:00007f28       ??_C@_0BC@PHJIOAED@lowResImageSample?$AA@ 004a1f28     vtf:vtf.obj
 0002:00007f3c       ??_C@_0CL@EOJJNAIP@?$CK?$CK?$CK?5Encountered?5VTF?5invalid?5text@ 004a1f3c     vtf:vtf.obj
 0002:00007f68       ??_C@_0CN@NDAFOEKI@?$CK?$CK?$CK?5Encountered?5VTF?5volume?5textu@ 004a1f68     vtf:vtf.obj
 0002:00007f98       ??_C@_0CJ@MFDAKNAJ@?$CK?$CK?$CK?5Encountered?5VTF?5non?9square?5c@ 004a1f98     vtf:vtf.obj
 0002:00007fc4       ??_C@_0CJ@JBJPBPEG@Image?5dimensions?5must?5be?5multipl@ 004a1fc4     vtf:vtf.obj
 0002:00007ff0       ??_C@_0BP@KGAAMOBJ@Depth?5must?5be?51?5for?5cubemaps?$CB?6?$AA@ 004a1ff0     vtf:vtf.obj
 0002:00008010       ??_C@_0CO@IPADFNJN@Height?5and?5width?5must?5be?5equal?5f@ 004a2010     vtf:vtf.obj
 0002:00008040       ??_C@_0CP@BOKKEMAO@GenerateRepresentativePalette?3?5n@ 004a2040     vtf:s3tc_decode.obj
 0002:00008070       __FPinit                   004a2070     LIBCMT:fpinit.obj
 0002:00008074       __FPmtinit                 004a2074     LIBCMT:fpinit.obj
 0002:00008078       __FPmtterm                 004a2078     LIBCMT:fpinit.obj
 0002:00008080       ??_7type_info@@6B@         004a2080     LIBCMT:typinfo.obj
 0002:000080e4       ??_7exception@std@@6B@     004a20e4     LIBCMT:stdexcpt.obj
 0002:000080ec       ??_C@_0BC@EOODALEL@Unknown?5exception?$AA@ 004a20ec     LIBCMT:stdexcpt.obj
 0002:00008104       ??_7bad_cast@std@@6B@      004a2104     LIBCMT:stdexcpt.obj
 0002:0000812c       ??_C@_0P@MIGLKIOC@CorExitProcess?$AA@ 004a212c     LIBCMT:crt0dat.obj
 0002:0000813c       ??_C@_0M@MBOPBNBK@mscoree?4dll?$AA@ 004a213c     LIBCMT:crt0dat.obj
 0002:00008198       ??_C@_0EA@FCLIIPNN@Visual?5C?$CL?$CL?5CRT?3?5Not?5enough?5memor@ 004a2198     LIBCMT:strerror.obj
 0002:000081d8       ??_C@_03FICNPLNB@TMP?$AA@  004a21d8     LIBCMT:tempnam.obj
 0002:000081dc       ??_C@_05KLBDPFGC@e?$CL000?$AA@ 004a21dc     LIBCMT:cvt.obj
 0002:000081e8       __real@4150017ec0000000    004a21e8     LIBCMT:testfdiv.obj
 0002:000081f0       __real@4147ffff80000000    004a21f0     LIBCMT:testfdiv.obj
 0002:000081f8       ??_C@_0BK@NHEOCAHP@IsProcessorFeaturePresent?$AA@ 004a21f8     LIBCMT:testfdiv.obj
 0002:00008214       ??_C@_08CPNIBGIE@KERNEL32?$AA@ 004a2214     LIBCMT:testfdiv.obj
 0002:00008220       ??_C@_1O@CEDCILHN@?$AA?$CI?$AAn?$AAu?$AAl?$AAl?$AA?$CJ?$AA?$AA@ 004a2220     LIBCMT:output.obj
 0002:00008230       ??_C@_06OJHGLDPL@?$CInull?$CJ?$AA@ 004a2230     LIBCMT:output.obj
 0002:00008238       ___lookuptable             004a2238     LIBCMT:output.obj
 0002:000082b8       ??_C@_07EPKMNAGK@?4mixcrt?$AA@ 004a22b8     LIBCMT:tidtable.obj
 0002:000082c0       ??_C@_0O@NLDKAIKN@EncodePointer?$AA@ 004a22c0     LIBCMT:tidtable.obj
 0002:000082d0       ??_C@_0N@NHGLKGEC@KERNEL32?4DLL?$AA@ 004a22d0     LIBCMT:tidtable.obj
 0002:000082e0       ??_C@_0O@KBPMFGHI@DecodePointer?$AA@ 004a22e0     LIBCMT:tidtable.obj
 0002:000082f0       ??_C@_07PEJMOBNF@FlsFree?$AA@ 004a22f0     LIBCMT:tidtable.obj
 0002:000082f8       ??_C@_0M@JCPCPOEF@FlsSetValue?$AA@ 004a22f8     LIBCMT:tidtable.obj
 0002:00008304       ??_C@_0M@GDNOONDI@FlsGetValue?$AA@ 004a2304     LIBCMT:tidtable.obj
 0002:00008310       ??_C@_08KNHFBNJ@FlsAlloc?$AA@ 004a2310     LIBCMT:tidtable.obj
 0002:0000831c       ??_C@_0P@GGKDKEEG@runtime?5error?5?$AA@ 004a231c     LIBCMT:crt0msg.obj
 0002:0000832c       ??_C@_0O@MJNIPGOH@TLOSS?5error?$AN?6?$AA@ 004a232c     LIBCMT:crt0msg.obj
 0002:0000833c       ??_C@_0N@BONNPDHF@SING?5error?$AN?6?$AA@ 004a233c     LIBCMT:crt0msg.obj
 0002:0000834c       ??_C@_0P@MBDAJNE@DOMAIN?5error?$AN?6?$AA@ 004a234c     LIBCMT:crt0msg.obj
 0002:00008360       ??_C@_0JL@DFDOOABL@R6034?$AN?6An?5application?5has?5made?5a@ 004a2360     LIBCMT:crt0msg.obj
 0002:00008400       ??_C@_0PH@EPAFIJ@R6033?$AN?6?9?5Attempt?5to?5use?5MSIL?5cod@ 004a2400     LIBCMT:crt0msg.obj
 0002:000084f8       ??_C@_0DD@BKEEABMM@R6032?$AN?6?9?5not?5enough?5space?5for?5lo@ 004a24f8     LIBCMT:crt0msg.obj
 0002:00008530       ??_C@_0GD@OFKILIED@R6031?$AN?6?9?5Attempt?5to?5initialize?5t@ 004a2530     LIBCMT:crt0msg.obj
 0002:00008594       ??_C@_0BP@LPMHJOKI@R6030?$AN?6?9?5CRT?5not?5initialized?$AN?6?$AA@ 004a2594     LIBCMT:crt0msg.obj
 0002:000085b4       ??_C@_0CF@KJDAIALP@R6028?$AN?6?9?5unable?5to?5initialize?5he@ 004a25b4     LIBCMT:crt0msg.obj
 0002:000085dc       ??_C@_0DF@GAKBPDFP@R6027?$AN?6?9?5not?5enough?5space?5for?5lo@ 004a25dc     LIBCMT:crt0msg.obj
 0002:00008614       ??_C@_0DF@IBLNNAIG@R6026?$AN?6?9?5not?5enough?5space?5for?5st@ 004a2614     LIBCMT:crt0msg.obj
 0002:0000864c       ??_C@_0CG@IOHKGFNJ@R6025?$AN?6?9?5pure?5virtual?5function?5c@ 004a264c     LIBCMT:crt0msg.obj
 0002:00008674       ??_C@_0DF@JIJJFJDC@R6024?$AN?6?9?5not?5enough?5space?5for?5_o@ 004a2674     LIBCMT:crt0msg.obj
 0002:000086ac       ??_C@_0CJ@EGEJHFME@R6019?$AN?6?9?5unable?5to?5open?5console?5@ 004a26ac     LIBCMT:crt0msg.obj
 0002:000086d8       ??_C@_0CB@GNHNIELH@R6018?$AN?6?9?5unexpected?5heap?5error?$AN?6@ 004a26d8     LIBCMT:crt0msg.obj
 0002:000086fc       ??_C@_0CN@FOLDKNG@R6017?$AN?6?9?5unexpected?5multithread?5@ 004a26fc     LIBCMT:crt0msg.obj
 0002:0000872c       ??_C@_0CM@FAHFJNHO@R6016?$AN?6?9?5not?5enough?5space?5for?5th@ 004a272c     LIBCMT:crt0msg.obj
 0002:00008758       ??_C@_0JG@LBKMGKLD@?$AN?6This?5application?5has?5requested@ 004a2758     LIBCMT:crt0msg.obj
 0002:000087f0       ??_C@_0CM@FLCNIPKK@R6009?$AN?6?9?5not?5enough?5space?5for?5en@ 004a27f0     LIBCMT:crt0msg.obj
 0002:0000881c       ??_C@_0CK@KMMJOAPP@R6008?$AN?6?9?5not?5enough?5space?5for?5ar@ 004a281c     LIBCMT:crt0msg.obj
 0002:00008848       ??_C@_0CN@LEKKICBM@R6002?$AN?6?9?5floating?5point?5support?5@ 004a2848     LIBCMT:crt0msg.obj
 0002:00008878       ??_C@_0CF@GOGNBNAK@Microsoft?5Visual?5C?$CL?$CL?5Runtime?5Lib@ 004a2878     LIBCMT:crt0msg.obj
 0002:000088a0       ??_C@_03KHICJKCI@?4?4?4?$AA@ 004a28a0     LIBCMT:crt0msg.obj
 0002:000088a4       ??_C@_0BH@DNAGHKFM@?$DMprogram?5name?5unknown?$DO?$AA@ 004a28a4     LIBCMT:crt0msg.obj
 0002:000088bc       ??_C@_0BK@OFGJDLJJ@Runtime?5Error?$CB?6?6Program?3?5?$AA@ 004a28bc     LIBCMT:crt0msg.obj
 0002:000088d8       ??_C@_07LCBHPJJN@LC_TIME?$AA@ 004a28d8     LIBCMT:setlocal.obj
 0002:000088e0       ??_C@_0L@DLHIECNL@LC_NUMERIC?$AA@ 004a28e0     LIBCMT:setlocal.obj
 0002:000088ec       ??_C@_0M@MIENIKLA@LC_MONETARY?$AA@ 004a28ec     LIBCMT:setlocal.obj
 0002:000088f8       ??_C@_08EADHIDAD@LC_CTYPE?$AA@ 004a28f8     LIBCMT:setlocal.obj
 0002:00008904       ??_C@_0L@KFJHEKIK@LC_COLLATE?$AA@ 004a2904     LIBCMT:setlocal.obj
 0002:00008910       ??_C@_06NEFDFEKB@LC_ALL?$AA@ 004a2910     LIBCMT:setlocal.obj
 0002:00008918       ___lc_category             004a2918     LIBCMT:setlocal.obj
 0002:000089e0       ??_C@_03EGDHDPFD@_?4?0?$AA@ 004a29e0     LIBCMT:setlocal.obj
 0002:000089e4       ??_C@_01ICJEACDI@?$DL?$AA@ 004a29e4     LIBCMT:setlocal.obj
 0002:000089e8       ??_C@_01NEMOKFLO@?$DN?$AA@ 004a29e8     LIBCMT:setlocal.obj
 0002:000089ec       ??_C@_02BALPLPBG@?$DN?$DL?$AA@ 004a29ec     LIBCMT:setlocal.obj
 0002:00008a58       ??_C@_03IIINPABG@tan?$AA@  004a2a58     LIBCMT:libm_error.obj
 0002:00008a5c       ??_C@_03LALBNOCG@cos?$AA@  004a2a5c     LIBCMT:libm_error.obj
 0002:00008a60       ??_C@_03BLEJJJBH@sin?$AA@  004a2a60     LIBCMT:libm_error.obj
 0002:00008a64       ??_C@_04EHEDPDJG@modf?$AA@ 004a2a64     LIBCMT:libm_error.obj
 0002:00008a6c       ??_C@_05PBJFFIGL@floor?$AA@ 004a2a6c     LIBCMT:libm_error.obj
 0002:00008a74       ??_C@_04GFPJNGEK@ceil?$AA@ 004a2a74     LIBCMT:libm_error.obj
 0002:00008a7c       ??_C@_04MLLJIGOK@atan?$AA@ 004a2a7c     LIBCMT:libm_error.obj
 0002:00008a84       ??_C@_05EOHGHCHD@exp10?$AA@ 004a2a84     LIBCMT:libm_error.obj
 0002:00008a8c       ??_C@_04PDIFKINK@acos?$AA@ 004a2a8c     LIBCMT:libm_error.obj
 0002:00008a94       ??_C@_04FIHNOPOL@asin?$AA@ 004a2a94     LIBCMT:libm_error.obj
 0002:00008a9c       ??_C@_03MGHMBJCF@log?$AA@  004a2a9c     LIBCMT:libm_error.obj
 0002:00008aa0       ??_C@_05HGHHAHAP@log10?$AA@ 004a2aa0     LIBCMT:libm_error.obj
 0002:00008aa8       ??_C@_03KHJOGHMM@exp?$AA@  004a2aa8     LIBCMT:libm_error.obj
 0002:00008aac       ??_C@_03JGHBODFD@pow?$AA@  004a2aac     LIBCMT:libm_error.obj
 0002:00008ab0       __pDestructExceptionObject 004a2ab0     LIBCMT:frame.obj
 0002:00008ab8       ??_7bad_exception@std@@6B@ 004a2ab8     LIBCMT:frame.obj
 0002:00008ac0       ??_C@_0O@DPKOEFFH@bad?5exception?$AA@ 004a2ac0     LIBCMT:frame.obj
 0002:00008b00       ??_C@_13NOLLCAOD@?$AA?$AA?$AA?$AA@ 004a2b00     LIBCMT:a_map.obj
 0002:00008b00       __real@00000000            004a2b00     brushbsp.obj
 0002:00008b04       ??_C@_0CG@PKBDLMEO@InitializeCriticalSectionAndSpin@ 004a2b04     LIBCMT:initcrit.obj
 0002:00008b2c       ??_C@_0N@MDJJJHMB@kernel32?4dll?$AA@ 004a2b2c     LIBCMT:initcrit.obj
 0002:00008b3c       ??_C@_0BG@KLEAJEFJ@Illegal?5byte?5sequence?$AA@ 004a2b3c     LIBCMT:syserr.obj
 0002:00008b54       ??_C@_0BE@ICMCHPHH@Directory?5not?5empty?$AA@ 004a2b54     LIBCMT:syserr.obj
 0002:00008b68       ??_C@_0BJ@IHEHINLI@Function?5not?5implemented?$AA@ 004a2b68     LIBCMT:syserr.obj
 0002:00008b84       ??_C@_0BD@CLHBCGPB@No?5locks?5available?$AA@ 004a2b84     LIBCMT:syserr.obj
 0002:00008b98       ??_C@_0BC@BEDIHIDK@Filename?5too?5long?$AA@ 004a2b98     LIBCMT:syserr.obj
 0002:00008bac       ??_C@_0BK@JAEBMJJM@Resource?5deadlock?5avoided?$AA@ 004a2bac     LIBCMT:syserr.obj
 0002:00008bc8       ??_C@_0BB@FCBJFCAJ@Result?5too?5large?$AA@ 004a2bc8     LIBCMT:syserr.obj
 0002:00008bdc       ??_C@_0N@MMJPGLJK@Domain?5error?$AA@ 004a2bdc     LIBCMT:syserr.obj
 0002:00008bec       ??_C@_0M@LHEPIIOM@Broken?5pipe?$AA@ 004a2bec     LIBCMT:syserr.obj
 0002:00008bf8       ??_C@_0P@PKCJJLLM@Too?5many?5links?$AA@ 004a2bf8     LIBCMT:syserr.obj
 0002:00008c08       ??_C@_0BG@DDBFNKBH@Read?9only?5file?5system?$AA@ 004a2c08     LIBCMT:syserr.obj
 0002:00008c20       ??_C@_0N@FEHLOILP@Invalid?5seek?$AA@ 004a2c20     LIBCMT:syserr.obj
 0002:00008c30       ??_C@_0BI@FEALHKLD@No?5space?5left?5on?5device?$AA@ 004a2c30     LIBCMT:syserr.obj
 0002:00008c48       ??_C@_0P@LFMMIPAE@File?5too?5large?$AA@ 004a2c48     LIBCMT:syserr.obj
 0002:00008c58       ??_C@_0CE@ONOKNLPF@Inappropriate?5I?1O?5control?5operat@ 004a2c58     LIBCMT:syserr.obj
 0002:00008c7c       ??_C@_0BE@INBJMKGG@Too?5many?5open?5files?$AA@ 004a2c7c     LIBCMT:syserr.obj
 0002:00008c90       ??_C@_0BO@IIFBODJE@Too?5many?5open?5files?5in?5system?$AA@ 004a2c90     LIBCMT:syserr.obj
 0002:00008cb0       ??_C@_0BB@HMGGCEBG@Invalid?5argument?$AA@ 004a2cb0     LIBCMT:syserr.obj
 0002:00008cc4       ??_C@_0P@NDHGCGKE@Is?5a?5directory?$AA@ 004a2cc4     LIBCMT:syserr.obj
 0002:00008cd4       ??_C@_0BA@CJBACOOL@Not?5a?5directory?$AA@ 004a2cd4     LIBCMT:syserr.obj
 0002:00008ce4       ??_C@_0P@NLEIANHE@No?5such?5device?$AA@ 004a2ce4     LIBCMT:syserr.obj
 0002:00008cf4       ??_C@_0O@OAMDNOCP@Improper?5link?$AA@ 004a2cf4     LIBCMT:syserr.obj
 0002:00008d04       ??_C@_0M@NAAJNNGH@File?5exists?$AA@ 004a2d04     LIBCMT:syserr.obj
 0002:00008d10       ??_C@_0BA@BIBLIOEK@Resource?5device?$AA@ 004a2d10     LIBCMT:syserr.obj
 0002:00008d20       ??_C@_0O@NIPGCINC@Unknown?5error?$AA@ 004a2d20     LIBCMT:syserr.obj
 0002:00008d30       ??_C@_0M@LOEHLCJD@Bad?5address?$AA@ 004a2d30     LIBCMT:syserr.obj
 0002:00008d3c       ??_C@_0BC@HFNFNKAI@Permission?5denied?$AA@ 004a2d3c     LIBCMT:syserr.obj
 0002:00008d50       ??_C@_0BB@IMDKMPFB@Not?5enough?5space?$AA@ 004a2d50     LIBCMT:syserr.obj
 0002:00008d64       ??_C@_0CB@EPFKGNAK@Resource?5temporarily?5unavailable@ 004a2d64     LIBCMT:syserr.obj
 0002:00008d88       ??_C@_0BD@LOHELEP@No?5child?5processes?$AA@ 004a2d88     LIBCMT:syserr.obj
 0002:00008d9c       ??_C@_0BE@NFGDDCEF@Bad?5file?5descriptor?$AA@ 004a2d9c     LIBCMT:syserr.obj
 0002:00008db0       ??_C@_0BC@HKPNECK@Exec?5format?5error?$AA@ 004a2db0     LIBCMT:syserr.obj
 0002:00008dc4       ??_C@_0BC@MFFGCDFL@Arg?5list?5too?5long?$AA@ 004a2dc4     LIBCMT:syserr.obj
 0002:00008dd8       ??_C@_0BK@DPKMCKJ@No?5such?5device?5or?5address?$AA@ 004a2dd8     LIBCMT:syserr.obj
 0002:00008df4       ??_C@_0BD@KKNFOBBD@Input?1output?5error?$AA@ 004a2df4     LIBCMT:syserr.obj
 0002:00008e08       ??_C@_0BK@FJBOAFDK@Interrupted?5function?5call?$AA@ 004a2e08     LIBCMT:syserr.obj
 0002:00008e24       ??_C@_0BA@FKIAIBGA@No?5such?5process?$AA@ 004a2e24     LIBCMT:syserr.obj
 0002:00008e34       ??_C@_0BK@FMDHKPNF@No?5such?5file?5or?5directory?$AA@ 004a2e34     LIBCMT:syserr.obj
 0002:00008e50       ??_C@_0BI@BJFCGOHL@Operation?5not?5permitted?$AA@ 004a2e50     LIBCMT:syserr.obj
 0002:00008e68       ??_C@_08INEPGKHH@No?5error?$AA@ 004a2e68     LIBCMT:syserr.obj
 0002:00008e74       ??_C@_04PNGHFIJN@?4com?$AA@ 004a2e74     LIBCMT:stat.obj
 0002:00008e7c       ??_C@_04NEEFLLOK@?4bat?$AA@ 004a2e7c     LIBCMT:stat.obj
 0002:00008e84       ??_C@_04CPCBDHLK@?4cmd?$AA@ 004a2e84     LIBCMT:stat.obj
 0002:00008e8c       ??_C@_04JLMDILM@?4exe?$AA@ 004a2e8c     LIBCMT:stat.obj
 0002:0000a6c8       __DEFAULT_CW_in_mem        004a46c8     LIBCMT:common.obj
 0002:0000a6ca       __pi_by_2_to_61            004a46ca     LIBCMT:common.obj
 0002:0000f830       ___lookuptable_s           004a9830     LIBCMT:outputs.obj
 0002:0000f894       ??_C@_0BK@CFCOFLF@?5Complete?5Object?5Locator?8?$AA@ 004a9894     LIBCMT:undname.obj
 0002:0000f8b0       ??_C@_0BN@MECKDCOJ@?5Class?5Hierarchy?5Descriptor?8?$AA@ 004a98b0     LIBCMT:undname.obj
 0002:0000f8d0       ??_C@_0BD@LGICGFMM@?5Base?5Class?5Array?8?$AA@ 004a98d0     LIBCMT:undname.obj
 0002:0000f8e4       ??_C@_0BM@LDKODKLH@?5Base?5Class?5Descriptor?5at?5?$CI?$AA@ 004a98e4     LIBCMT:undname.obj
 0002:0000f900       ??_C@_0BC@DAFEJGAK@?5Type?5Descriptor?8?$AA@ 004a9900     LIBCMT:undname.obj
 0002:0000f914       ??_C@_0BM@PMGGMLDN@?$GAlocal?5static?5thread?5guard?8?$AA@ 004a9914     LIBCMT:undname.obj
 0002:0000f930       ??_C@_0CL@FGIJHLCE@?$GAmanaged?5vector?5copy?5constructor@ 004a9930     LIBCMT:undname.obj
 0002:0000f95c       ??_C@_0CJ@GJELGAMM@?$GAvector?5vbase?5copy?5constructor?5i@ 004a995c     LIBCMT:undname.obj
 0002:0000f988       ??_C@_0CD@CGAJBKEJ@?$GAvector?5copy?5constructor?5iterato@ 004a9988     LIBCMT:undname.obj
 0002:0000f9ac       ??_C@_0CB@PDBIFEP@?$GAdynamic?5atexit?5destructor?5for?5?8@ 004a99ac     LIBCMT:undname.obj
 0002:0000f9d0       ??_C@_0BL@CLIPGLGB@?$GAdynamic?5initializer?5for?5?8?$AA@ 004a99d0     LIBCMT:undname.obj
 0002:0000f9ec       ??_C@_0CM@FCBBDIGB@?$GAeh?5vector?5vbase?5copy?5constructo@ 004a99ec     LIBCMT:undname.obj
 0002:0000fa18       ??_C@_0CG@HLDDJMAG@?$GAeh?5vector?5copy?5constructor?5iter@ 004a9a18     LIBCMT:undname.obj
 0002:0000fa40       ??_C@_0CF@IMGKMJNO@?$GAmanaged?5vector?5destructor?5itera@ 004a9a40     LIBCMT:undname.obj
 0002:0000fa68       ??_C@_0CG@CFDHKGGD@?$GAmanaged?5vector?5constructor?5iter@ 004a9a68     LIBCMT:undname.obj
 0002:0000fa90       ??_C@_0BN@CKNJLHMB@?$GAplacement?5delete?$FL?$FN?5closure?8?$AA@ 004a9a90     LIBCMT:undname.obj
 0002:0000fab0       ??_C@_0BL@CNOONJFP@?$GAplacement?5delete?5closure?8?$AA@ 004a9ab0     LIBCMT:undname.obj
 0002:0000facc       ??_C@_0P@HJKNJFNN@?$GAomni?5callsig?8?$AA@ 004a9acc     LIBCMT:undname.obj
 0002:0000fadc       ??_C@_09LBNFPBCA@?5delete?$FL?$FN?$AA@ 004a9adc     LIBCMT:undname.obj
 0002:0000fae8       ??_C@_06FHBGPFGH@?5new?$FL?$FN?$AA@ 004a9ae8     LIBCMT:undname.obj
 0002:0000faf0       ??_C@_0CE@IIHCMGGL@?$GAlocal?5vftable?5constructor?5closu@ 004a9af0     LIBCMT:undname.obj
 0002:0000fb14       ??_C@_0BA@KKLDJDLB@?$GAlocal?5vftable?8?$AA@ 004a9b14     LIBCMT:undname.obj
 0002:0000fb24       ??_C@_05KHLCHHI@?$GARTTI?$AA@ 004a9b24     LIBCMT:undname.obj
 0002:0000fb2c       ??_C@_03KLGMFNMG@?$GAEH?$AA@ 004a9b2c     LIBCMT:undname.obj
 0002:0000fb30       ??_C@_0BA@KBCDOMBN@?$GAudt?5returning?8?$AA@ 004a9b30     LIBCMT:undname.obj
 0002:0000fb40       ??_C@_0BL@LLKPOHJI@?$GAcopy?5constructor?5closure?8?$AA@ 004a9b40     LIBCMT:undname.obj
 0002:0000fb5c       ??_C@_0CH@OOJPLCPH@?$GAeh?5vector?5vbase?5constructor?5ite@ 004a9b5c     LIBCMT:undname.obj
 0002:0000fb84       ??_C@_0CA@GCEOPDGL@?$GAeh?5vector?5destructor?5iterator?8?$AA@ 004a9b84     LIBCMT:undname.obj
 0002:0000fba4       ??_C@_0CB@JONCMFFK@?$GAeh?5vector?5constructor?5iterator?8@ 004a9ba4     LIBCMT:undname.obj
 0002:0000fbc8       ??_C@_0BL@NILFHHPC@?$GAvirtual?5displacement?5map?8?$AA@ 004a9bc8     LIBCMT:undname.obj
 0002:0000fbe4       ??_C@_0CE@IKBNEHA@?$GAvector?5vbase?5constructor?5iterat@ 004a9be4     LIBCMT:undname.obj
 0002:0000fc08       ??_C@_0BN@LFPFMEDL@?$GAvector?5destructor?5iterator?8?$AA@ 004a9c08     LIBCMT:undname.obj
 0002:0000fc28       ??_C@_0BO@PFGOCPJJ@?$GAvector?5constructor?5iterator?8?$AA@ 004a9c28     LIBCMT:undname.obj
 0002:0000fc48       ??_C@_0BN@IMDCHIKM@?$GAscalar?5deleting?5destructor?8?$AA@ 004a9c48     LIBCMT:undname.obj
 0002:0000fc68       ??_C@_0BO@OBMKPJIG@?$GAdefault?5constructor?5closure?8?$AA@ 004a9c68     LIBCMT:undname.obj
 0002:0000fc88       ??_C@_0BN@DEGPLNFK@?$GAvector?5deleting?5destructor?8?$AA@ 004a9c88     LIBCMT:undname.obj
 0002:0000fca8       ??_C@_0BD@JDLKDPAB@?$GAvbase?5destructor?8?$AA@ 004a9ca8     LIBCMT:undname.obj
 0002:0000fcbc       ??_C@_08OBABFOLI@?$GAstring?8?$AA@ 004a9cbc     LIBCMT:undname.obj
 0002:0000fcc8       ??_C@_0BF@KDPPACIK@?$GAlocal?5static?5guard?8?$AA@ 004a9cc8     LIBCMT:undname.obj
 0002:0000fce0       ??_C@_08LLFFHHDJ@?$GAtypeof?8?$AA@ 004a9ce0     LIBCMT:undname.obj
 0002:0000fcec       ??_C@_07FEEIOKP@?$GAvcall?8?$AA@ 004a9cec     LIBCMT:undname.obj
 0002:0000fcf4       ??_C@_09BLBHBJP@?$GAvbtable?8?$AA@ 004a9cf4     LIBCMT:undname.obj
 0002:0000fd00       ??_C@_09IFPLHPGF@?$GAvftable?8?$AA@ 004a9d00     LIBCMT:undname.obj
 0002:0000fd0c       ??_C@_02MHEGNOJ@?$FO?$DN?$AA@ 004a9d0c     LIBCMT:undname.obj
 0002:0000fd10       ??_C@_02DHLNPPGH@?$HM?$DN?$AA@ 004a9d10     LIBCMT:undname.obj
 0002:0000fd14       ??_C@_02FGJGFEAB@?$CG?$DN?$AA@ 004a9d14     LIBCMT:undname.obj
 0002:0000fd18       ??_C@_03CDNPDDLA@?$DM?$DM?$DN?$AA@ 004a9d18     LIBCMT:undname.obj
 0002:0000fd1c       ??_C@_03IKFCCPFF@?$DO?$DO?$DN?$AA@ 004a9d1c     LIBCMT:undname.obj
 0002:0000fd20       ??_C@_02FENAOKFI@?$CF?$DN?$AA@ 004a9d20     LIBCMT:undname.obj
 0002:0000fd24       ??_C@_02FJEHGPIO@?1?$DN?$AA@ 004a9d24     LIBCMT:undname.obj
 0002:0000fd28       ??_C@_02FKMDLLOA@?9?$DN?$AA@ 004a9d28     LIBCMT:undname.obj
 0002:0000fd2c       ??_C@_02FOEOMHFC@?$CL?$DN?$AA@ 004a9d2c     LIBCMT:undname.obj
 0002:0000fd30       ??_C@_02FPIMKNGF@?$CK?$DN?$AA@ 004a9d30     LIBCMT:undname.obj
 0002:0000fd34       ??_C@_02NONPIBCD@?$HM?$HM?$AA@ 004a9d34     LIBCMT:undname.obj
 0002:0000fd38       ??_C@_02PPKAJPJL@?$CG?$CG?$AA@ 004a9d38     LIBCMT:undname.obj
 0002:0000fd3c       ??_C@_01DNKMNLPK@?$HM?$AA@ 004a9d3c     LIBCMT:undname.obj
 0002:0000fd40       ??_C@_01JKBOJNNK@?$FO?$AA@ 004a9d40     LIBCMT:undname.obj
 0002:0000fd44       ??_C@_01PJKLJHI@?$HO?$AA@  004a9d44     LIBCMT:undname.obj
 0002:0000fd48       ??_C@_02HCKGKOFO@?$CI?$CJ?$AA@ 004a9d48     LIBCMT:undname.obj
 0002:0000fd4c       ??_C@_01IHBHIGKO@?0?$AA@   004a9d4c     LIBCMT:undname.obj
 0002:0000fd50       ??_C@_02EEKDKGMJ@?$DO?$DN?$AA@ 004a9d50     LIBCMT:undname.obj
 0002:0000fd54       ??_C@_01PPODPGHN@?$DO?$AA@ 004a9d54     LIBCMT:undname.obj
 0002:0000fd58       ??_C@_02EHCHHCKH@?$DM?$DN?$AA@ 004a9d58     LIBCMT:undname.obj
 0002:0000fd5c       ??_C@_01MNNFJEPP@?$DM?$AA@ 004a9d5c     LIBCMT:undname.obj
 0002:0000fd60       ??_C@_01FGNFDNOH@?$CF?$AA@ 004a9d60     LIBCMT:undname.obj
 0002:0000fd64       ??_C@_01KMDKNFGN@?1?$AA@   004a9d64     LIBCMT:undname.obj
 0002:0000fd68       ??_C@_03MNHNFDLC@?9?$DO?$CK?$AA@ 004a9d68     LIBCMT:undname.obj
 0002:0000fd6c       ??_C@_01HNPIGOCE@?$CG?$AA@ 004a9d6c     LIBCMT:undname.obj
 0002:0000fd70       ??_C@_01MIFGBAGJ@?$CL?$AA@ 004a9d70     LIBCMT:undname.obj
 0002:0000fd74       ??_C@_02BAABKJLB@?9?9?$AA@ 004a9d74     LIBCMT:undname.obj
 0002:0000fd78       ??_C@_02ECNGHCIF@?$CL?$CL?$AA@ 004a9d78     LIBCMT:undname.obj
 0002:0000fd7c       ??_C@_02HBOOOICD@?9?$DO?$AA@ 004a9d7c     LIBCMT:undname.obj
 0002:0000fd80       ??_C@_08LHJFAFGD@operator?$AA@ 004a9d80     LIBCMT:undname.obj
 0002:0000fd8c       ??_C@_02GPECMEKF@?$FL?$FN?$AA@ 004a9d8c     LIBCMT:undname.obj
 0002:0000fd90       ??_C@_02FDNJECIE@?$CB?$DN?$AA@ 004a9d90     LIBCMT:undname.obj
 0002:0000fd94       ??_C@_02EGOFBIJA@?$DN?$DN?$AA@ 004a9d94     LIBCMT:undname.obj
 0002:0000fd98       ??_C@_01DCLJPIOD@?$CB?$AA@ 004a9d98     LIBCMT:undname.obj
 0002:0000fd9c       ??_C@_02FODMEDOG@?$DM?$DM?$AA@ 004a9d9c     LIBCMT:undname.obj
 0002:0000fda0       ??_C@_02GPIOPFAK@?$DO?$DO?$AA@ 004a9da0     LIBCMT:undname.obj
 0002:0000fda4       ??_C@_07FPCDHGMM@?5delete?$AA@ 004a9da4     LIBCMT:undname.obj
 0002:0000fdac       ??_C@_04NIHEBCM@?5new?$AA@ 004a9dac     LIBCMT:undname.obj
 0002:0000fdb4       ??_C@_0M@GFIIJFMG@__unaligned?$AA@ 004a9db4     LIBCMT:undname.obj
 0002:0000fdc0       ??_C@_0L@PILCLIHE@__restrict?$AA@ 004a9dc0     LIBCMT:undname.obj
 0002:0000fdcc       ??_C@_07JOMMBBKO@__ptr64?$AA@ 004a9dcc     LIBCMT:undname.obj
 0002:0000fdd4       ??_C@_09HIJEGCPM@__clrcall?$AA@ 004a9dd4     LIBCMT:undname.obj
 0002:0000fde0       ??_C@_0L@JMKHOMEK@__fastcall?$AA@ 004a9de0     LIBCMT:undname.obj
 0002:0000fdec       ??_C@_0L@NPHFGOKO@__thiscall?$AA@ 004a9dec     LIBCMT:undname.obj
 0002:0000fdf8       ??_C@_09IFJBGAPI@__stdcall?$AA@ 004a9df8     LIBCMT:undname.obj
 0002:0000fe04       ??_C@_08GHMPAG@__pascal?$AA@ 004a9e04     LIBCMT:undname.obj
 0002:0000fe10       ??_C@_07KOLFKCDI@__cdecl?$AA@ 004a9e10     LIBCMT:undname.obj
 0002:0000fe18       ??_C@_08EHJDFFNH@__based?$CI?$AA@ 004a9e18     LIBCMT:undname.obj
 0002:0000ffa8       ??_C@_0BI@DFKBFLJE@GetProcessWindowStation?$AA@ 004a9fa8     LIBCMT:crtmbox.obj
 0002:0000ffc0       ??_C@_0BK@CIDNPOGP@GetUserObjectInformationA?$AA@ 004a9fc0     LIBCMT:crtmbox.obj
 0002:0000ffdc       ??_C@_0BD@HHGDFDBJ@GetLastActivePopup?$AA@ 004a9fdc     LIBCMT:crtmbox.obj
 0002:0000fff0       ??_C@_0BA@HNOPNCHB@GetActiveWindow?$AA@ 004a9ff0     LIBCMT:crtmbox.obj
 0002:00010000       ??_C@_0M@CHKKJDAI@MessageBoxA?$AA@ 004aa000     LIBCMT:crtmbox.obj
 0002:0001000c       ??_C@_0L@NDEGIDAG@USER32?4DLL?$AA@ 004aa00c     LIBCMT:crtmbox.obj
 0002:00010018       ___newctype                004aa018     LIBCMT:ctype.obj
 0002:00010318       __wctype                   004aa318     LIBCMT:ctype.obj
 0002:00010520       ___newclmap                004aa520     LIBCMT:ctype.obj
 0002:000106a0       ___newcumap                004aa6a0     LIBCMT:ctype.obj
 0002:00010820       ??_C@_08JCCMCCIL@HH?3mm?3ss?$AA@ 004aa820     LIBCMT:strftime.obj
 0002:0001082c       ??_C@_0BE@CKGJFCPC@dddd?0?5MMMM?5dd?0?5yyyy?$AA@ 004aa82c     LIBCMT:strftime.obj
 0002:00010840       ??_C@_08BPBNCDIB@MM?1dd?1yy?$AA@ 004aa840     LIBCMT:strftime.obj
 0002:0001084c       ??_C@_02CJNFDJBF@PM?$AA@   004aa84c     LIBCMT:strftime.obj
 0002:00010850       ??_C@_02DEDBPAFC@AM?$AA@   004aa850     LIBCMT:strftime.obj
 0002:00010854       ??_C@_08EDHMEBNP@December?$AA@ 004aa854     LIBCMT:strftime.obj
 0002:00010860       ??_C@_08HCHEGEOA@November?$AA@ 004aa860     LIBCMT:strftime.obj
 0002:0001086c       ??_C@_07JJNFCEND@October?$AA@ 004aa86c     LIBCMT:strftime.obj
 0002:00010874       ??_C@_09BHHEALKD@September?$AA@ 004aa874     LIBCMT:strftime.obj
 0002:00010880       ??_C@_06LBBHFDDG@August?$AA@ 004aa880     LIBCMT:strftime.obj
 0002:00010888       ??_C@_04MIEPOIFP@July?$AA@ 004aa888     LIBCMT:strftime.obj
 0002:00010890       ??_C@_04CNLMGBGM@June?$AA@ 004aa890     LIBCMT:strftime.obj
 0002:00010898       ??_C@_05DMJDNLEJ@April?$AA@ 004aa898     LIBCMT:strftime.obj
 0002:000108a0       ??_C@_05HPCKOFNC@March?$AA@ 004aa8a0     LIBCMT:strftime.obj
 0002:000108a8       ??_C@_08GNJGEPFN@February?$AA@ 004aa8a8     LIBCMT:strftime.obj
 0002:000108b4       ??_C@_07CGJPFGJA@January?$AA@ 004aa8b4     LIBCMT:strftime.obj
 0002:000108bc       ??_C@_03MKABNOCG@Dec?$AA@  004aa8bc     LIBCMT:strftime.obj
 0002:000108c0       ??_C@_03JPJOFNIA@Nov?$AA@  004aa8c0     LIBCMT:strftime.obj
 0002:000108c4       ??_C@_03BMAOKBAD@Oct?$AA@  004aa8c4     LIBCMT:strftime.obj
 0002:000108c8       ??_C@_03GGCAPAJC@Sep?$AA@  004aa8c8     LIBCMT:strftime.obj
 0002:000108cc       ??_C@_03IFJFEIGA@Aug?$AA@  004aa8cc     LIBCMT:strftime.obj
 0002:000108d0       ??_C@_03LBGABGKK@Jul?$AA@  004aa8d0     LIBCMT:strftime.obj
 0002:000108d4       ??_C@_03IDFGHECI@Jun?$AA@  004aa8d4     LIBCMT:strftime.obj
 0002:000108d8       ??_C@_03CNMDKL@May?$AA@    004aa8d8     LIBCMT:strftime.obj
 0002:000108dc       ??_C@_03LEOLGMJP@Apr?$AA@  004aa8dc     LIBCMT:strftime.obj
 0002:000108e0       ??_C@_03ODNJBKGA@Mar?$AA@  004aa8e0     LIBCMT:strftime.obj
 0002:000108e4       ??_C@_03HJBDCHOM@Feb?$AA@  004aa8e4     LIBCMT:strftime.obj
 0002:000108e8       ??_C@_03JIHJHPIE@Jan?$AA@  004aa8e8     LIBCMT:strftime.obj
 0002:000108ec       ??_C@_08INBOOONO@Saturday?$AA@ 004aa8ec     LIBCMT:strftime.obj
 0002:000108f8       ??_C@_06JECMNKMI@Friday?$AA@ 004aa8f8     LIBCMT:strftime.obj
 0002:00010900       ??_C@_08HACCIKIA@Thursday?$AA@ 004aa900     LIBCMT:strftime.obj
 0002:0001090c       ??_C@_09DLIGFAKA@Wednesday?$AA@ 004aa90c     LIBCMT:strftime.obj
 0002:00010918       ??_C@_07BAAGCFCM@Tuesday?$AA@ 004aa918     LIBCMT:strftime.obj
 0002:00010920       ??_C@_06JLEDEDGH@Monday?$AA@ 004aa920     LIBCMT:strftime.obj
 0002:00010928       ??_C@_06OOPIFAJ@Sunday?$AA@ 004aa928     LIBCMT:strftime.obj
 0002:00010930       ??_C@_03FEFJNEK@Sat?$AA@   004aa930     LIBCMT:strftime.obj
 0002:00010934       ??_C@_03IDIOELNC@Fri?$AA@  004aa934     LIBCMT:strftime.obj
 0002:00010938       ??_C@_03IOFIKPDN@Thu?$AA@  004aa938     LIBCMT:strftime.obj
 0002:0001093c       ??_C@_03MHOMLAJA@Wed?$AA@  004aa93c     LIBCMT:strftime.obj
 0002:00010940       ??_C@_03NAGEINEP@Tue?$AA@  004aa940     LIBCMT:strftime.obj
 0002:00010944       ??_C@_03PDAGKDH@Mon?$AA@   004aa944     LIBCMT:strftime.obj
 0002:00010948       ??_C@_03KOEHGMDN@Sun?$AA@  004aa948     LIBCMT:strftime.obj
 0002:0001094c       ??_C@_0O@FMJNFNKE@united?9states?$AA@ 004aa94c     LIBCMT:getqloc.obj
 0002:0001095c       ??_C@_0P@NDHFFKCA@united?9kingdom?$AA@ 004aa95c     LIBCMT:getqloc.obj
 0002:0001096c       ??_C@_0BC@HHDADLGF@trinidad?5?$CG?5tobago?$AA@ 004aa96c     LIBCMT:getqloc.obj
 0002:00010980       ??_C@_0M@IOAEBDAC@south?9korea?$AA@ 004aa980     LIBCMT:getqloc.obj
 0002:0001098c       ??_C@_0N@FIELFKIJ@south?9africa?$AA@ 004aa98c     LIBCMT:getqloc.obj
 0002:0001099c       ??_C@_0M@OPNDHCMC@south?5korea?$AA@ 004aa99c     LIBCMT:getqloc.obj
 0002:000109a8       ??_C@_0N@MDEOEPFI@south?5africa?$AA@ 004aa9a8     LIBCMT:getqloc.obj
 0002:000109b8       ??_C@_06FKAPCJLB@slovak?$AA@ 004aa9b8     LIBCMT:getqloc.obj
 0002:000109c0       ??_C@_0M@EFJANOAL@puerto?9rico?$AA@ 004aa9c0     LIBCMT:getqloc.obj
 0002:000109cc       ??_C@_08PGOJKDAI@pr?9china?$AA@ 004aa9cc     LIBCMT:getqloc.obj
 0002:000109d8       ??_C@_08JHDOMCMI@pr?5china?$AA@ 004aa9d8     LIBCMT:getqloc.obj
 0002:000109e4       ??_C@_02JHCHFBLL@nz?$AA@   004aa9e4     LIBCMT:getqloc.obj
 0002:000109e8       ??_C@_0M@LINHDHKP@new?9zealand?$AA@ 004aa9e8     LIBCMT:getqloc.obj
 0002:000109f4       ??_C@_09IIIPPBDB@hong?9kong?$AA@ 004aa9f4     LIBCMT:getqloc.obj
 0002:00010a00       ??_C@_07HJLCKBG@holland?$AA@ 004aaa00     LIBCMT:getqloc.obj
 0002:00010a08       ??_C@_0O@LEHGMHAG@great?5britain?$AA@ 004aaa08     LIBCMT:getqloc.obj
 0002:00010a18       ??_C@_07FACOMELA@england?$AA@ 004aaa18     LIBCMT:getqloc.obj
 0002:00010a20       ??_C@_05JIHCEICB@czech?$AA@ 004aaa20     LIBCMT:getqloc.obj
 0002:00010a28       ??_C@_05BBJOBLGB@china?$AA@ 004aaa28     LIBCMT:getqloc.obj
 0002:00010a30       ??_C@_07GPKPHICP@britain?$AA@ 004aaa30     LIBCMT:getqloc.obj
 0002:00010a38       ??_C@_07MHIPBHMG@america?$AA@ 004aaa38     LIBCMT:getqloc.obj
 0002:00010a40       ??_C@_03KIALPMKC@usa?$AA@  004aaa40     LIBCMT:getqloc.obj
 0002:00010a44       ??_C@_02FGJGKGGD@us?$AA@   004aaa44     LIBCMT:getqloc.obj
 0002:00010a48       ??_C@_02NEINDODK@uk?$AA@   004aaa48     LIBCMT:getqloc.obj
 0002:00010a4c       ??_C@_05JMPCFJFJ@swiss?$AA@ 004aaa4c     LIBCMT:getqloc.obj
 0002:00010a54       ??_C@_0BA@HLOCPIOD@swedish?9finland?$AA@ 004aaa54     LIBCMT:getqloc.obj
 0002:00010a64       ??_C@_0BC@PKCNIABK@spanish?9venezuela?$AA@ 004aaa64     LIBCMT:getqloc.obj
 0002:00010a78       ??_C@_0BA@GBHHMIJI@spanish?9uruguay?$AA@ 004aaa78     LIBCMT:getqloc.obj
 0002:00010a88       ??_C@_0BE@BHDOHPMC@spanish?9puerto?5rico?$AA@ 004aaa88     LIBCMT:getqloc.obj
 0002:00010a9c       ??_C@_0N@KMOIDGGN@spanish?9peru?$AA@ 004aaa9c     LIBCMT:getqloc.obj
 0002:00010aac       ??_C@_0BB@HMHLPGPH@spanish?9paraguay?$AA@ 004aaaac     LIBCMT:getqloc.obj
 0002:00010ac0       ??_C@_0P@MCPKNGFD@spanish?9panama?$AA@ 004aaac0     LIBCMT:getqloc.obj
 0002:00010ad0       ??_C@_0BC@IHOHGAIL@spanish?9nicaragua?$AA@ 004aaad0     LIBCMT:getqloc.obj
 0002:00010ae4       ??_C@_0P@KLMJDNFJ@spanish?9modern?$AA@ 004aaae4     LIBCMT:getqloc.obj
 0002:00010af4       ??_C@_0BA@BPAPGBCM@spanish?9mexican?$AA@ 004aaaf4     LIBCMT:getqloc.obj
 0002:00010b04       ??_C@_0BB@PDECHHHE@spanish?9honduras?$AA@ 004aab04     LIBCMT:getqloc.obj
 0002:00010b18       ??_C@_0BC@KLHKFGDB@spanish?9guatemala?$AA@ 004aab18     LIBCMT:getqloc.obj
 0002:00010b2c       ??_C@_0BE@MFOOKJAI@spanish?9el?5salvador?$AA@ 004aab2c     LIBCMT:getqloc.obj
 0002:00010b40       ??_C@_0BA@FCOKFPFC@spanish?9ecuador?$AA@ 004aab40     LIBCMT:getqloc.obj
 0002:00010b50       ??_C@_0BL@PLMGIMOO@spanish?9dominican?5republic?$AA@ 004aab50     LIBCMT:getqloc.obj
 0002:00010b6c       ??_C@_0BD@HLGDNMHB@spanish?9costa?5rica?$AA@ 004aab6c     LIBCMT:getqloc.obj
 0002:00010b80       ??_C@_0BB@PKCBKCPE@spanish?9colombia?$AA@ 004aab80     LIBCMT:getqloc.obj
 0002:00010b94       ??_C@_0O@MCBIJGNE@spanish?9chile?$AA@ 004aab94     LIBCMT:getqloc.obj
 0002:00010ba4       ??_C@_0BA@BEFEIGJJ@spanish?9bolivia?$AA@ 004aaba4     LIBCMT:getqloc.obj
 0002:00010bb4       ??_C@_0BC@EMECMPD@spanish?9argentina?$AA@ 004aabb4     LIBCMT:getqloc.obj
 0002:00010bc8       ??_C@_0BF@EALFLENP@portuguese?9brazilian?$AA@ 004aabc8     LIBCMT:getqloc.obj
 0002:00010be0       ??_C@_0BC@HBLEBLNN@norwegian?9nynorsk?$AA@ 004aabe0     LIBCMT:getqloc.obj
 0002:00010bf4       ??_C@_0BB@HMACDDCK@norwegian?9bokmal?$AA@ 004aabf4     LIBCMT:getqloc.obj
 0002:00010c08       ??_C@_09BAFFPPHE@norwegian?$AA@ 004aac08     LIBCMT:getqloc.obj
 0002:00010c14       ??_C@_0O@EAJFJDFG@italian?9swiss?$AA@ 004aac14     LIBCMT:getqloc.obj
 0002:00010c24       ??_C@_0O@CNOMPGD@irish?9english?$AA@ 004aac24     LIBCMT:getqloc.obj
 0002:00010c34       ??_C@_0N@EDHBGCKG@german?9swiss?$AA@ 004aac34     LIBCMT:getqloc.obj
 0002:00010c44       ??_C@_0BC@JACMHNBP@german?9luxembourg?$AA@ 004aac44     LIBCMT:getqloc.obj
 0002:00010c58       ??_C@_0BE@HBGMGFEG@german?9lichtenstein?$AA@ 004aac58     LIBCMT:getqloc.obj
 0002:00010c6c       ??_C@_0BA@HKKBIBKL@german?9austrian?$AA@ 004aac6c     LIBCMT:getqloc.obj
 0002:00010c7c       ??_C@_0N@GCAEPEBK@french?9swiss?$AA@ 004aac7c     LIBCMT:getqloc.obj
 0002:00010c8c       ??_C@_0BC@DJFJJCK@french?9luxembourg?$AA@ 004aac8c     LIBCMT:getqloc.obj
 0002:00010ca0       ??_C@_0BA@NNCEDFIC@french?9canadian?$AA@ 004aaca0     LIBCMT:getqloc.obj
 0002:00010cb0       ??_C@_0P@CMPOCLM@french?9belgian?$AA@ 004aacb0     LIBCMT:getqloc.obj
 0002:00010cc0       ??_C@_0M@GHHDJOK@english?9usa?$AA@ 004aacc0     LIBCMT:getqloc.obj
 0002:00010ccc       ??_C@_0L@PLDJKEIL@english?9us?$AA@ 004aaccc     LIBCMT:getqloc.obj
 0002:00010cd8       ??_C@_0L@HJCCDMNC@english?9uk?$AA@ 004aacd8     LIBCMT:getqloc.obj
 0002:00010ce4       ??_C@_0BK@CKLIAGJB@english?9trinidad?5y?5tobago?$AA@ 004aace4     LIBCMT:getqloc.obj
 0002:00010d00       ??_C@_0BF@JMJMGNNF@english?9south?5africa?$AA@ 004aad00     LIBCMT:getqloc.obj
 0002:00010d18       ??_C@_0L@DKIIFDFD@english?9nz?$AA@ 004aad18     LIBCMT:getqloc.obj
 0002:00010d24       ??_C@_0BA@ONHGJCLH@english?9jamaica?$AA@ 004aad24     LIBCMT:getqloc.obj
 0002:00010d34       ??_C@_0M@HJBGHOPO@english?9ire?$AA@ 004aad34     LIBCMT:getqloc.obj
 0002:00010d40       ??_C@_0BC@LFEKMIFB@english?9caribbean?$AA@ 004aad40     LIBCMT:getqloc.obj
 0002:00010d54       ??_C@_0M@OLDPFKHI@english?9can?$AA@ 004aad54     LIBCMT:getqloc.obj
 0002:00010d60       ??_C@_0P@OMDEHBMP@english?9belize?$AA@ 004aad60     LIBCMT:getqloc.obj
 0002:00010d70       ??_C@_0M@KFHFPFED@english?9aus?$AA@ 004aad70     LIBCMT:getqloc.obj
 0002:00010d7c       ??_C@_0BB@MNMBKDFE@english?9american?$AA@ 004aad7c     LIBCMT:getqloc.obj
 0002:00010d90       ??_C@_0O@KIDLNNBA@dutch?9belgian?$AA@ 004aad90     LIBCMT:getqloc.obj
 0002:00010da0       ??_C@_0BE@JBKABBMH@chinese?9traditional?$AA@ 004aada0     LIBCMT:getqloc.obj
 0002:00010db4       ??_C@_0BC@MJJMPKCG@chinese?9singapore?$AA@ 004aadb4     LIBCMT:getqloc.obj
 0002:00010dc8       ??_C@_0BD@FDKADDCP@chinese?9simplified?$AA@ 004aadc8     LIBCMT:getqloc.obj
 0002:00010ddc       ??_C@_0BB@DBEFDDME@chinese?9hongkong?$AA@ 004aaddc     LIBCMT:getqloc.obj
 0002:00010df0       ??_C@_07DHNMFMCI@chinese?$AA@ 004aadf0     LIBCMT:getqloc.obj
 0002:00010df8       ??_C@_03FNDDCHI@chi?$AA@   004aadf8     LIBCMT:getqloc.obj
 0002:00010dfc       ??_C@_03BMMIADDJ@chh?$AA@  004aadfc     LIBCMT:getqloc.obj
 0002:00010e00       ??_C@_08OAIPJDGI@canadian?$AA@ 004aae00     LIBCMT:getqloc.obj
 0002:00010e0c       ??_C@_07HBPMNPNJ@belgian?$AA@ 004aae0c     LIBCMT:getqloc.obj
 0002:00010e14       ??_C@_0L@OEKOPBEL@australian?$AA@ 004aae14     LIBCMT:getqloc.obj
 0002:00010e20       ??_C@_0BB@MEIMBEDG@american?9english?$AA@ 004aae20     LIBCMT:getqloc.obj
 0002:00010e34       ??_C@_0BB@DFMDPDGB@american?5english?$AA@ 004aae34     LIBCMT:getqloc.obj
 0002:00010e48       ??_C@_08IJLOKOLL@american?$AA@ 004aae48     LIBCMT:getqloc.obj
 0002:00010e58       ___rg_language             004aae58     LIBCMT:getqloc.obj
 0002:00011060       ___rg_country              004ab060     LIBCMT:getqloc.obj
 0002:00011118       ___rglangidNotDefault      004ab118     LIBCMT:getqloc.obj
 0002:0001112c       ??_C@_03NFKLAGEF@OCP?$AA@  004ab12c     LIBCMT:getqloc.obj
 0002:00011130       ??_C@_03DFHEHBHG@ACP?$AA@  004ab130     LIBCMT:getqloc.obj
 0002:00011134       ??_C@_0BC@NFIEMBLL@Norwegian?9Nynorsk?$AA@ 004ab134     LIBCMT:getqloc.obj
 0002:00011148       ??_C@_0L@KDOEJCKC@_nextafter?$AA@ 004ab148     LIBCMT:fpexcept.obj
 0002:00011154       ??_C@_05JGDBENOH@_logb?$AA@ 004ab154     LIBCMT:fpexcept.obj
 0002:0001115c       ??_C@_03ONILCKOB@_yn?$AA@  004ab15c     LIBCMT:fpexcept.obj
 0002:00011160       ??_C@_03NAKIGLHK@_y1?$AA@  004ab160     LIBCMT:fpexcept.obj
 0002:00011164       ??_C@_03MJLDFKDL@_y0?$AA@  004ab164     LIBCMT:fpexcept.obj
 0002:00011168       ??_C@_05GKKHEGJL@frexp?$AA@ 004ab168     LIBCMT:fpexcept.obj
 0002:00011170       ??_C@_04KEPJIHGP@fmod?$AA@ 004ab170     LIBCMT:fpexcept.obj
 0002:00011178       ??_C@_06MEIMCGCF@_hypot?$AA@ 004ab178     LIBCMT:fpexcept.obj
 0002:00011180       ??_C@_05KBKMEMPO@_cabs?$AA@ 004ab180     LIBCMT:fpexcept.obj
 0002:00011188       ??_C@_05CEJMAHNP@ldexp?$AA@ 004ab188     LIBCMT:fpexcept.obj
 0002:00011190       ??_C@_04ODHECPBC@fabs?$AA@ 004ab190     LIBCMT:fpexcept.obj
 0002:00011198       ??_C@_04EIAKFFMI@sqrt?$AA@ 004ab198     LIBCMT:fpexcept.obj
 0002:000111a0       ??_C@_05KNGEOGJB@atan2?$AA@ 004ab1a0     LIBCMT:fpexcept.obj
 0002:000111a8       ??_C@_04FJHINJAO@tanh?$AA@ 004ab1a8     LIBCMT:fpexcept.obj
 0002:000111b0       ??_C@_04HPJJNFIM@cosh?$AA@ 004ab1b0     LIBCMT:fpexcept.obj
 0002:000111b8       ??_C@_04COOMCNPB@sinh?$AA@ 004ab1b8     LIBCMT:fpexcept.obj
 0002:000111c0       ??_C@_02CLFPBFFP@TZ?$AA@   004ab1c0     LIBCMT:tzset.obj
 0002:000111c4       ___dnames                  004ab1c4     LIBCMT:timeset.obj
 0002:000111dc       ___mnames                  004ab1dc     LIBCMT:timeset.obj
 0002:00011204       ??_C@_0L@NKOGAPMJ@SystemRoot?$AA@ 004ab204     LIBCMT:cenvarg.obj
 0002:00011210       ??_C@_06IMKFLFPG@1?$CDQNAN?$AA@ 004ab210     LIBCMT:x10fout.obj
 0002:00011218       ??_C@_05DNEBIAHO@1?$CDINF?$AA@ 004ab218     LIBCMT:x10fout.obj
 0002:00011220       ??_C@_05PHHOCPM@1?$CDIND?$AA@ 004ab220     LIBCMT:x10fout.obj
 0002:00011228       ??_C@_06PGGFOGJG@1?$CDSNAN?$AA@ 004ab228     LIBCMT:x10fout.obj
 0002:00011230       ??_C@_06GDENEHCP@CONIN$?$AA@ 004ab230     LIBCMT:initcon.obj
 0002:00011238       ??_C@_07GPDNMNG@CONOUT$?$AA@ 004ab238     LIBCMT:initcon.obj
 0002:00011244       ??_7out_of_range@std@@6B@  004ab244     libcpmt:string.obj
 0002:0001124c       ??_C@_0BA@JFNIOLAK@string?5too?5long?$AA@ 004ab24c     libcpmt:string.obj
 0002:0001125c       ??_C@_0BI@CFPLBAOH@invalid?5string?5position?$AA@ 004ab25c     libcpmt:string.obj
 0002:00011274       ?_BADOFF@std@@3JB          004ab274     libcpmt:ios.obj
 0002:0001127c       ??_7_Locimp@locale@std@@6B@ 004ab27c     libcpmt:locale0.obj
 0002:00011280       ??_C@_13BPINEIPE@?$AAr?$AA?$AA@ 004ab280     libcpmt:fiopen.obj
 0002:000112c0       ??_C@_13CIFDLIMG@?$AAw?$AA?$AA@ 004ab2c0     libcpmt:fiopen.obj
 0002:000112c4       ??_C@_13FNCBLAIF@?$AAa?$AA?$AA@ 004ab2c4     libcpmt:fiopen.obj
 0002:000112c8       ??_C@_15JJPIMNBO@?$AAr?$AAb?$AA?$AA@ 004ab2c8     libcpmt:fiopen.obj
 0002:000112d0       ??_C@_15MJDFFMKN@?$AAw?$AAb?$AA?$AA@ 004ab2d0     libcpmt:fiopen.obj
 0002:000112d8       ??_C@_15BMLKLNCL@?$AAa?$AAb?$AA?$AA@ 004ab2d8     libcpmt:fiopen.obj
 0002:000112e0       ??_C@_15HPOENKKJ@?$AAr?$AA?$CL?$AA?$AA@ 004ab2e0     libcpmt:fiopen.obj
 0002:000112e8       ??_C@_15CPCJELBK@?$AAw?$AA?$CL?$AA?$AA@ 004ab2e8     libcpmt:fiopen.obj
 0002:000112f0       ??_C@_15PKKGKKJM@?$AAa?$AA?$CL?$AA?$AA@ 004ab2f0     libcpmt:fiopen.obj
 0002:000112f8       ??_C@_17IIOMHMAG@?$AAr?$AA?$CL?$AAb?$AA?$AA@ 004ab2f8     libcpmt:fiopen.obj
 0002:00011300       ??_C@_17MAAMHCGC@?$AAw?$AA?$CL?$AAb?$AA?$AA@ 004ab300     libcpmt:fiopen.obj
 0002:00011308       ??_C@_17HKNIEKMO@?$AAa?$AA?$CL?$AAb?$AA?$AA@ 004ab308     libcpmt:fiopen.obj
 0002:00011310       ??_C@_05OIKDKKFM@ATI2N?$AA@ 004ab310     bitmap:imageformat.obj
 0002:00011318       ??_C@_05OKOFBEAF@ATI1N?$AA@ 004ab318     bitmap:imageformat.obj
 0002:00011320       ??_C@_07CFELPLPD@NV_NULL?$AA@ 004ab320     bitmap:imageformat.obj
 0002:00011328       ??_C@_09JCCMAMGI@ATI_DST24?$AA@ 004ab328     bitmap:imageformat.obj
 0002:00011334       ??_C@_09KCFMNALD@ATI_DST16?$AA@ 004ab334     bitmap:imageformat.obj
 0002:00011340       ??_C@_07FDMLLIPO@NV_RAWZ?$AA@ 004ab340     bitmap:imageformat.obj
 0002:00011348       ??_C@_07BONOLAGC@NV_INTZ?$AA@ 004ab348     bitmap:imageformat.obj
 0002:00011350       ??_C@_08HKKCPHEG@NV_DST24?$AA@ 004ab350     bitmap:imageformat.obj
 0002:0001135c       ??_C@_08EKNCCLJN@NV_DST16?$AA@ 004ab35c     bitmap:imageformat.obj
 0002:00011368       ??_C@_0BL@OLOJPJLN@IMAGE_FORMAT_RGBA32323232F?$AA@ 004ab368     bitmap:imageformat.obj
 0002:00011384       ??_C@_0BI@FLDBGJMJ@IMAGE_FORMAT_RGB323232F?$AA@ 004ab384     bitmap:imageformat.obj
 0002:0001139c       ??_C@_0BC@EJLIBMHN@IMAGE_FORMAT_R32F?$AA@ 004ab39c     bitmap:imageformat.obj
 0002:000113b0       ??_C@_0BG@EPLNNPIA@IMAGE_FORMAT_UVLX8888?$AA@ 004ab3b0     bitmap:imageformat.obj
 0002:000113c8       ??_C@_0N@GBJBEFCM@RGBA16161616?$AA@ 004ab3c8     bitmap:imageformat.obj
 0002:000113d8       ??_C@_0O@JEJKBFCF@RGBA16161616F?$AA@ 004ab3d8     bitmap:imageformat.obj
 0002:000113e8       ??_C@_08KPDDCJI@UVWQ8888?$AA@ 004ab3e8     bitmap:imageformat.obj
 0002:000113f4       ??_C@_04BKKPBAPE@UV88?$AA@ 004ab3f4     bitmap:imageformat.obj
 0002:000113fc       ??_C@_08PAENDFNP@BGRA5551?$AA@ 004ab3fc     bitmap:imageformat.obj
 0002:00011408       ??_C@_0BB@BFEFPFPF@DXT1_ONEBITALPHA?$AA@ 004ab408     bitmap:imageformat.obj
 0002:0001141c       ??_C@_08JCEOFHI@BGRA4444?$AA@ 004ab41c     bitmap:imageformat.obj
 0002:00011428       ??_C@_08NEJEGGIM@BGRX5551?$AA@ 004ab428     bitmap:imageformat.obj
 0002:00011434       ??_C@_06KEKLLBKJ@BGR565?$AA@ 004ab434     bitmap:imageformat.obj
 0002:0001143c       ??_C@_08HHEFCPK@BGRX8888?$AA@ 004ab43c     bitmap:imageformat.obj
 0002:00011448       ??_C@_04FDJDJFPM@DXT5?$AA@ 004ab448     bitmap:imageformat.obj
 0002:00011450       ??_C@_04FMJDCHK@DXT3?$AA@  004ab450     bitmap:imageformat.obj
 0002:00011458       ??_C@_04DHPPFAPI@DXT1?$AA@ 004ab458     bitmap:imageformat.obj
 0002:00011460       ??_C@_08CDKNABKJ@BGRA8888?$AA@ 004ab460     bitmap:imageformat.obj
 0002:0001146c       ??_C@_08JNAJMDOE@ARGB8888?$AA@ 004ab46c     bitmap:imageformat.obj
 0002:00011478       ??_C@_0BC@KDPNAOFO@BGR888_BLUESCREEN?$AA@ 004ab478     bitmap:imageformat.obj
 0002:0001148c       ??_C@_0BC@GLHJGMNI@RGB888_BLUESCREEN?$AA@ 004ab48c     bitmap:imageformat.obj
 0002:000114a0       ??_C@_02GGHJHNOB@A8?$AA@   004ab4a0     bitmap:imageformat.obj
 0002:000114a4       ??_C@_02HLJNLEKG@P8?$AA@   004ab4a4     bitmap:imageformat.obj
 0002:000114a8       ??_C@_04HCHBAFFB@IA88?$AA@ 004ab4a8     bitmap:imageformat.obj
 0002:000114b0       ??_C@_02GIGKCMFJ@I8?$AA@   004ab4b0     bitmap:imageformat.obj
 0002:000114b4       ??_C@_06KDJFLKOF@RGB565?$AA@ 004ab4b4     bitmap:imageformat.obj
 0002:000114bc       ??_C@_06OJPBDKDD@BGR888?$AA@ 004ab4bc     bitmap:imageformat.obj
 0002:000114c4       ??_C@_06OOMPDBHP@RGB888?$AA@ 004ab4c4     bitmap:imageformat.obj
 0002:000114cc       ??_C@_08OCGEPAFE@ABGR8888?$AA@ 004ab4cc     bitmap:imageformat.obj
 0002:000114d8       ??_C@_08OILDNPBG@RGBA8888?$AA@ 004ab4d8     bitmap:imageformat.obj
 0002:000114ec       __real@c77fe000            004ab4ec     bitmap:colorconversion.obj
 0002:000114f0       __real@38800000            004ab4f0     bitmap:colorconversion.obj
 0002:000114f4       __real@3da7ef9e            004ab4f4     bitmap:colorconversion.obj
 0002:000114f8       __real@3f1c01a3            004ab4f8     bitmap:colorconversion.obj
 0002:000114fc       __real@3e9e00d2            004ab4fc     bitmap:colorconversion.obj
 0002:00011500       __real@477fff00            004ab500     bitmap:colorconversion.obj
 0002:00011504       __real@45800000            004ab504     bitmap:colorconversion.obj
 0002:00011508       __real@43000000            004ab508     bitmap:colorconversion.obj
 0002:0001150c       __real@42fe0000            004ab50c     bitmap:colorconversion.obj
 0002:00011510       __real@3c010204            004ab510     bitmap:colorconversion.obj
 0002:00011514       __real@3e991687            004ab514     bitmap:colorconversion.obj
 0002:00011518       __real@3f1645a2            004ab518     bitmap:colorconversion.obj
 0002:0001151c       __real@3de978d5            004ab51c     bitmap:colorconversion.obj
 0002:00011520       __real@37800000            004ab520     bitmap:colorconversion.obj
 0002:00011528       __real@42cc0000            004ab528     bitmap:resample.obj
 0002:0001152c       ??_C@_0P@JPKGKFHD@AlphaThreshold?$AA@ 004ab52c     bitmap:ATI_Compress.obj
 0002:0001153c       ??_C@_0N@PCNBPLHN@DXT1UseAlpha?$AA@ 004ab53c     bitmap:ATI_Compress.obj
 0002:0001154c       ??_C@_0BF@OHABJJJO@UseAdaptiveWeighting?$AA@ 004ab54c     bitmap:ATI_Compress.obj
 0002:00011564       ??_C@_07HHHMHOCD@WeightB?$AA@ 004ab564     bitmap:ATI_Compress.obj
 0002:0001156c       ??_C@_07KALIKGG@WeightG?$AA@ 004ab56c     bitmap:ATI_Compress.obj
 0002:00011574       ??_C@_07DNLOGMHC@WeightR?$AA@ 004ab574     bitmap:ATI_Compress.obj
 0002:00011580       __real@3f847ae140000000    004ab580     bitmap:ATI_Compress.obj
 0002:00011588       ??_C@_0BE@DKLHGILP@UseChannelWeighting?$AA@ 004ab588     bitmap:ATI_Compress.obj
 0002:0001159c       __real@41700000            004ab59c     bitmap:S3_intrf.obj
 0002:000115a0       ??_7CCodec@ATI_Compress@@6B@ 004ab5a0     bitmap:Codec.obj
 0002:000115c8       __real@4060000000000000    004ab5c8     bitmap:Codec.obj
 0002:000115d0       __real@405fc00000000000    004ab5d0     bitmap:Codec.obj
 0002:000115d8       ??_7CCodecBuffer@@6B@      004ab5d8     bitmap:CodecBuffer.obj
 0002:000116b8       __real@40efffe000000000    004ab6b8     bitmap:CodecBuffer.obj
 0002:000116d0       __real@3f40000000000000    004ab6d0     bitmap:S3_quant.obj
 0002:000116d8       __real@400c000000000000    004ab6d8     bitmap:S3_quant.obj
 0002:000116e0       __real@4008000000000000    004ab6e0     bitmap:S3_quant.obj
 0002:000116e8       __real@4014000000000000    004ab6e8     bitmap:S3_quant.obj
 0002:000116f0       __real@4058000000000000    004ab6f0     bitmap:S3_quant.obj
 0002:000116f8       ??_7CCodec_ATI2N_DXT5@@6B@ 004ab6f8     bitmap:Codec_ATI2N_DXT5.obj
 0002:00011778       __real@4f800000            004ab778     bitmap:Codec_ATI2N_DXT5.obj
 0002:00011780       ??_7CCodec_ATI2N@@6B@      004ab780     bitmap:Codec_ATI2N.obj
 0002:00011800       ??_7CCodec_ATI1N@@6B@      004ab800     bitmap:Codec_ATI1N.obj
 0002:00011878       ??_7CCodec_DXT5_xGxR@@6B@  004ab878     bitmap:Codec_DXT5_xGxR.obj
 0002:00011900       ??_7CCodec_DXT5_RGxB@@6B@  004ab900     bitmap:Codec_DXT5_RGxB.obj
 0002:00011988       ??_7CCodec_DXT5_xRBG@@6B@  004ab988     bitmap:Codec_DXT5_xRBG.obj
 0002:00011a10       ??_7CCodec_DXT5_RBxG@@6B@  004aba10     bitmap:Codec_DXT5_RBxG.obj
 0002:00011a98       ??_7CCodec_DXT5_RxBG@@6B@  004aba98     bitmap:Codec_DXT5_RxBG.obj
 0002:00011b20       ??_7CCodec_DXT5_xGBR@@6B@  004abb20     bitmap:Codec_DXT5_xGBR.obj
 0002:00011ba8       ??_7CCodec_DXT5@@6B@       004abba8     bitmap:Codec_DXT5.obj
 0002:00011c20       ??_7CCodec_DXT3@@6B@       004abc20     bitmap:Codec_DXT3.obj
 0002:00011c98       ??_7CCodec_DXT1@@6B@       004abc98     bitmap:Codec_DXT1.obj
 0002:00011d10       ?_toFloat@half@@0QBTuif@1@B 004abd10     bitmap:half.obj
 0002:00051d10       ?_eLut@half@@0QBGB         004ebd10     bitmap:half.obj
 0002:00052110       __real@501502f9            004ec110     bitmap:half.obj
 0002:00052118       ??_7CCodecBuffer_Block@@6B@ 004ec118     bitmap:CodecBuffer_Block.obj
 0002:000521f8       ??_7CCodecBuffer_RGBA32F@@6B@ 004ec1f8     bitmap:CodecBuffer_RGBA32F.obj
 0002:000522e0       ??_7CCodecBuffer_RGBA16F@@6B@ 004ec2e0     bitmap:CodecBuffer_RGBA16F.obj
 0002:000523c8       ??_7CCodecBuffer_RGBA16@@6B@ 004ec3c8     bitmap:CodecBuffer_RGBA16.obj
 0002:000524b0       ??_7CCodecBuffer_RGBA2101010@@6B@ 004ec4b0     bitmap:CodecBuffer_RGBA2101010.obj
 0002:00052598       ??_7CCodecBuffer_RGBA8888@@6B@ 004ec598     bitmap:CodecBuffer_RGBA8888.obj
 0002:00052680       ??_7CCodec_DXTC@@6B@       004ec680     bitmap:Codec_DXTC.obj
 0002:000526f8       ??_C@_0P@GGJMOEEN@ForceFloatPath?$AA@ 004ec6f8     bitmap:Codec_DXTC.obj
 0002:00052708       ??_C@_0BA@FGFEHBI@RefinementSteps?$AA@ 004ec708     bitmap:Codec_DXTC.obj
 0002:00052718       ??_C@_0N@GJGMBLDI@3DRefinement?$AA@ 004ec718     bitmap:Codec_DXTC.obj
 0002:00052728       ??_C@_07DPIIIHGG@UseSSE2?$AA@ 004ec728     bitmap:Codec_DXTC.obj
 0002:00052730       ??_7CCodec_Block_4x4@@6B@  004ec730     bitmap:Codec_Block_4x4.obj
 0002:00052758       __real@401c000000000000    004ec758     bitmap:Codec_DXTC_Alpha.obj
 0002:00052760       __real@4018000000000000    004ec760     bitmap:Codec_DXTC_Alpha.obj
 0002:00052768       __real@3fd0000000000000    004ec768     bitmap:Codec_DXTC_RGBA.obj
 0002:00052770       __real@3fb0000000000000    004ec770     bitmap:Codec_DXTC_RGBA.obj
 0002:00052778       ??_7CCodec_DXT5_Swizzled@@6B@ 004ec778     bitmap:Codec_DXT5_Swizzled.obj
 0002:00052800       ??_7CCodec_Block@@6B@      004ec800     bitmap:Codec_Block.obj
 0002:0005286c       __real@51ba43b7            004ec86c     bitmap:ATiXCodec.obj
 0002:00052870       __real@4b189680            004ec870     bitmap:ATiXCodec.obj
 0002:00052878       __real@3fe3333340000000    004ec878     bitmap:ATiXCodec.obj
 0002:00052880       __real@3f926e9780000000    004ec880     bitmap:ATiXCodec.obj
 0002:00052888       __real@3fb99999a0000000    004ec888     bitmap:ATiXCodec.obj
 0002:00052890       __real@47fa0000            004ec890     bitmap:ATiXCodec.obj
 0002:00052894       __real@43010000            004ec894     bitmap:ATiXCodec.obj
 0002:00052898       __real@c000000000000000    004ec898     bitmap:ATiXCodec.obj
 0002:000528a0       __real@3fefcfcfcfcfcfd0    004ec8a0     bitmap:ATiXCodec.obj
 0002:000528a8       __real@3f78181818181818    004ec8a8     bitmap:ATiXCodec.obj
 0002:000528b0       __real@47c35000            004ec8b0     bitmap:ATiXCodec.obj
 0002:000528b8       __real@3f80101020000000    004ec8b8     bitmap:ATiXCodec.obj
 0002:000528c0       __real@3f999999a0000000    004ec8c0     bitmap:ATiXCodec.obj
 0002:000528c8       __real@3fa99999a0000000    004ec8c8     bitmap:ATiXCodec.obj
 0002:000528d0       __real@c47a0000            004ec8d0     bitmap:ATiXCodec.obj
 0002:00052c98       ??_R3IVirtualMeshEvent@@8  004ecc98     disp_ivp.obj
 0002:00052ca8       ??_R2IVirtualMeshEvent@@8  004ecca8     disp_ivp.obj
 0002:00052cb0       ??_R1A@?0A@EA@IVirtualMeshEvent@@8 004eccb0     disp_ivp.obj
 0002:00052ccc       ??_R4CDispMeshEvent@@6B@   004ecccc     disp_ivp.obj
 0002:00052ce0       ??_R3CDispMeshEvent@@8     004ecce0     disp_ivp.obj
 0002:00052cf0       ??_R2CDispMeshEvent@@8     004eccf0     disp_ivp.obj
 0002:00052cfc       ??_R1A@?0A@EA@CDispMeshEvent@@8 004eccfc     disp_ivp.obj
 0002:00052d18       ??_R3CPhysCollisionEntry@@8 004ecd18     ivp.obj
 0002:00052d28       ??_R2CPhysCollisionEntry@@8 004ecd28     ivp.obj
 0002:00052d30       ??_R1A@?0A@EA@CPhysCollisionEntry@@8 004ecd30     ivp.obj
 0002:00052d4c       ??_R4CPhysCollisionEntrySolid@@6B@ 004ecd4c     ivp.obj
 0002:00052d60       ??_R3CPhysCollisionEntrySolid@@8 004ecd60     ivp.obj
 0002:00052d70       ??_R2CPhysCollisionEntrySolid@@8 004ecd70     ivp.obj
 0002:00052d7c       ??_R1A@?0A@EA@CPhysCollisionEntrySolid@@8 004ecd7c     ivp.obj
 0002:00052d98       ??_R4CPhysCollisionEntryStaticSolid@@6B@ 004ecd98     ivp.obj
 0002:00052dac       ??_R3CPhysCollisionEntryStaticSolid@@8 004ecdac     ivp.obj
 0002:00052dbc       ??_R2CPhysCollisionEntryStaticSolid@@8 004ecdbc     ivp.obj
 0002:00052dc8       ??_R1A@?0A@EA@CPhysCollisionEntryStaticSolid@@8 004ecdc8     ivp.obj
 0002:00052de4       ??_R4CPhysCollisionEntryStaticMesh@@6B@ 004ecde4     ivp.obj
 0002:00052df8       ??_R3CPhysCollisionEntryStaticMesh@@8 004ecdf8     ivp.obj
 0002:00052e08       ??_R2CPhysCollisionEntryStaticMesh@@8 004ece08     ivp.obj
 0002:00052e14       ??_R1A@?0A@EA@CPhysCollisionEntryStaticMesh@@8 004ece14     ivp.obj
 0002:00052e30       ??_R4CPhysCollisionEntryFluid@@6B@ 004ece30     ivp.obj
 0002:00052e44       ??_R3CPhysCollisionEntryFluid@@8 004ece44     ivp.obj
 0002:00052e54       ??_R2CPhysCollisionEntryFluid@@8 004ece54     ivp.obj
 0002:00052e60       ??_R1A@?0A@EA@CPhysCollisionEntryFluid@@8 004ece60     ivp.obj
 0002:00052e7c       ??_R4bad_alloc@std@@6B@    004ece7c     mstristrip.obj
 0002:00052e90       ??_R3bad_alloc@std@@8      004ece90     mstristrip.obj
 0002:00052ea0       ??_R2bad_alloc@std@@8      004ecea0     mstristrip.obj
 0002:00052eac       ??_R1A@?0A@EA@bad_alloc@std@@8 004eceac     mstristrip.obj
 0002:00052ec8       ??_R1A@?0A@EA@exception@std@@8 004ecec8     mstristrip.obj
 0002:00052ee4       ??_R3exception@std@@8      004ecee4     mstristrip.obj
 0002:00052ef4       ??_R2exception@std@@8      004ecef4     mstristrip.obj
 0002:00052efc       ??_R4logic_error@std@@6B@  004ecefc     mstristrip.obj
 0002:00052f10       ??_R3logic_error@std@@8    004ecf10     mstristrip.obj
 0002:00052f20       ??_R2logic_error@std@@8    004ecf20     mstristrip.obj
 0002:00052f2c       ??_R1A@?0A@EA@logic_error@std@@8 004ecf2c     mstristrip.obj
 0002:00052f48       ??_R4length_error@std@@6B@ 004ecf48     mstristrip.obj
 0002:00052f5c       ??_R3length_error@std@@8   004ecf5c     mstristrip.obj
 0002:00052f6c       ??_R2length_error@std@@8   004ecf6c     mstristrip.obj
 0002:00052f7c       ??_R1A@?0A@EA@length_error@std@@8 004ecf7c     mstristrip.obj
 0002:00052f98       ??_R3IWriteStream@@8       004ecf98     zip_utils.obj
 0002:00052fa8       ??_R2IWriteStream@@8       004ecfa8     zip_utils.obj
 0002:00052fb0       ??_R1A@?0A@EA@IWriteStream@@8 004ecfb0     zip_utils.obj
 0002:00052fcc       ??_R4CFileStream@@6B@      004ecfcc     zip_utils.obj
 0002:00052fe0       ??_R3CFileStream@@8        004ecfe0     zip_utils.obj
 0002:00052ff0       ??_R2CFileStream@@8        004ecff0     zip_utils.obj
 0002:00052ffc       ??_R1A@?0A@EA@CFileStream@@8 004ecffc     zip_utils.obj
 0002:00053018       ??_R3IZip@@8               004ed018     zip_utils.obj
 0002:00053028       ??_R2IZip@@8               004ed028     zip_utils.obj
 0002:00053030       ??_R1A@?0A@EA@IZip@@8      004ed030     zip_utils.obj
 0002:0005304c       ??_R4CBufferStream@@6B@    004ed04c     zip_utils.obj
 0002:00053060       ??_R3CBufferStream@@8      004ed060     zip_utils.obj
 0002:00053070       ??_R2CBufferStream@@8      004ed070     zip_utils.obj
 0002:0005307c       ??_R1A@?0A@EA@CBufferStream@@8 004ed07c     zip_utils.obj
 0002:00053098       ??_R4CZip@@6B@             004ed098     zip_utils.obj
 0002:000530ac       ??_R3CZip@@8               004ed0ac     zip_utils.obj
 0002:000530bc       ??_R2CZip@@8               004ed0bc     zip_utils.obj
 0002:000530c8       ??_R1A@?0A@EA@CZip@@8      004ed0c8     zip_utils.obj
 0002:000530e4       ??_R4CDispUtilsHelper@@6B@ 004ed0e4     builddisp.obj
 0002:000530f8       ??_R3CDispUtilsHelper@@8   004ed0f8     builddisp.obj
 0002:00053108       ??_R2CDispUtilsHelper@@8   004ed108     builddisp.obj
 0002:00053110       ??_R1A@?0A@EA@CDispUtilsHelper@@8 004ed110     builddisp.obj
 0002:0005312c       ??_R4CCoreDispInfo@@6B@    004ed12c     builddisp.obj
 0002:00053140       ??_R3CCoreDispInfo@@8      004ed140     builddisp.obj
 0002:00053150       ??_R2CCoreDispInfo@@8      004ed150     builddisp.obj
 0002:0005315c       ??_R1A@?0A@EA@CCoreDispInfo@@8 004ed15c     builddisp.obj
 0002:00053178       ??_R4ios_base@std@@6B@     004ed178     chunkfile.obj
 0002:0005318c       ??_R3ios_base@std@@8       004ed18c     chunkfile.obj
 0002:0005319c       ??_R2ios_base@std@@8       004ed19c     chunkfile.obj
 0002:000531a8       ??_R1A@?0A@EA@ios_base@std@@8 004ed1a8     chunkfile.obj
 0002:000531c4       ??_R13?0A@EA@?$_Iosb@H@std@@8 004ed1c4     chunkfile.obj
 0002:000531e0       ??_R3?$_Iosb@H@std@@8      004ed1e0     chunkfile.obj
 0002:000531f0       ??_R2?$_Iosb@H@std@@8      004ed1f0     chunkfile.obj
 0002:000531f8       ??_R1A@?0A@EA@?$_Iosb@H@std@@8 004ed1f8     chunkfile.obj
 0002:00053214       ??_R4?$basic_istream@DU?$char_traits@D@std@@@std@@6B@ 004ed214     chunkfile.obj
 0002:00053228       ??_R3?$basic_istream@DU?$char_traits@D@std@@@std@@8 004ed228     chunkfile.obj
 0002:00053238       ??_R2?$basic_istream@DU?$char_traits@D@std@@@std@@8 004ed238     chunkfile.obj
 0002:0005324c       ??_R1A@?0A@EA@?$basic_istream@DU?$char_traits@D@std@@@std@@8 004ed24c     chunkfile.obj
 0002:00053268       ??_R1A@A@3FA@?$basic_ios@DU?$char_traits@D@std@@@std@@8 004ed268     chunkfile.obj
 0002:00053284       ??_R3?$basic_ios@DU?$char_traits@D@std@@@std@@8 004ed284     chunkfile.obj
 0002:00053294       ??_R2?$basic_ios@DU?$char_traits@D@std@@@std@@8 004ed294     chunkfile.obj
 0002:000532a4       ??_R1A@?0A@EA@?$basic_ios@DU?$char_traits@D@std@@@std@@8 004ed2a4     chunkfile.obj
 0002:000532c0       ??_R1A@A@3EA@ios_base@std@@8 004ed2c0     chunkfile.obj
 0002:000532dc       ??_R13A@3EA@?$_Iosb@H@std@@8 004ed2dc     chunkfile.obj
 0002:000532f8       ??_R4?$basic_streambuf@DU?$char_traits@D@std@@@std@@6B@ 004ed2f8     chunkfile.obj
 0002:0005330c       ??_R3?$basic_streambuf@DU?$char_traits@D@std@@@std@@8 004ed30c     chunkfile.obj
 0002:0005331c       ??_R2?$basic_streambuf@DU?$char_traits@D@std@@@std@@8 004ed31c     chunkfile.obj
 0002:00053324       ??_R1A@?0A@EA@?$basic_streambuf@DU?$char_traits@D@std@@@std@@8 004ed324     chunkfile.obj
 0002:00053340       ??_R4?$basic_filebuf@DU?$char_traits@D@std@@@std@@6B@ 004ed340     chunkfile.obj
 0002:00053354       ??_R3?$basic_filebuf@DU?$char_traits@D@std@@@std@@8 004ed354     chunkfile.obj
 0002:00053364       ??_R2?$basic_filebuf@DU?$char_traits@D@std@@@std@@8 004ed364     chunkfile.obj
 0002:00053370       ??_R1A@?0A@EA@?$basic_filebuf@DU?$char_traits@D@std@@@std@@8 004ed370     chunkfile.obj
 0002:0005338c       ??_R4facet@locale@std@@6B@ 004ed38c     chunkfile.obj
 0002:000533a0       ??_R3facet@locale@std@@8   004ed3a0     chunkfile.obj
 0002:000533b0       ??_R2facet@locale@std@@8   004ed3b0     chunkfile.obj
 0002:000533b8       ??_R1A@?0A@EA@facet@locale@std@@8 004ed3b8     chunkfile.obj
 0002:000533d4       ??_R3codecvt_base@std@@8   004ed3d4     chunkfile.obj
 0002:000533e4       ??_R2codecvt_base@std@@8   004ed3e4     chunkfile.obj
 0002:000533f0       ??_R1A@?0A@EA@codecvt_base@std@@8 004ed3f0     chunkfile.obj
 0002:0005340c       ??_R4runtime_error@std@@6B@ 004ed40c     chunkfile.obj
 0002:00053420       ??_R3runtime_error@std@@8  004ed420     chunkfile.obj
 0002:00053430       ??_R2runtime_error@std@@8  004ed430     chunkfile.obj
 0002:0005343c       ??_R1A@?0A@EA@runtime_error@std@@8 004ed43c     chunkfile.obj
 0002:00053458       ??_R4?$codecvt@DDH@std@@6B@ 004ed458     chunkfile.obj
 0002:0005346c       ??_R3?$codecvt@DDH@std@@8  004ed46c     chunkfile.obj
 0002:0005347c       ??_R2?$codecvt@DDH@std@@8  004ed47c     chunkfile.obj
 0002:0005348c       ??_R1A@?0A@EA@?$codecvt@DDH@std@@8 004ed48c     chunkfile.obj
 0002:000534a8       ??_R4?$basic_ifstream@DU?$char_traits@D@std@@@std@@6B@ 004ed4a8     chunkfile.obj
 0002:000534bc       ??_R3?$basic_ifstream@DU?$char_traits@D@std@@@std@@8 004ed4bc     chunkfile.obj
 0002:000534cc       ??_R2?$basic_ifstream@DU?$char_traits@D@std@@@std@@8 004ed4cc     chunkfile.obj
 0002:000534e4       ??_R1A@?0A@EA@?$basic_ifstream@DU?$char_traits@D@std@@@std@@8 004ed4e4     chunkfile.obj
 0002:00053500       ??_R3IScriptLib@@8         004ed500     scriplib.obj
 0002:00053510       ??_R2IScriptLib@@8         004ed510     scriplib.obj
 0002:00053518       ??_R1A@?0A@EA@IScriptLib@@8 004ed518     scriplib.obj
 0002:00053534       ??_R4CScriptLib@@6B@       004ed534     scriplib.obj
 0002:00053548       ??_R3CScriptLib@@8         004ed548     scriplib.obj
 0002:00053558       ??_R2CScriptLib@@8         004ed558     scriplib.obj
 0002:00053564       ??_R1A@?0A@EA@CScriptLib@@8 004ed564     scriplib.obj
 0002:00053580       ??_R4CUtlCharConversion@@6B@ 004ed580     tier1:utlbuffer.obj
 0002:00053594       ??_R3CUtlCharConversion@@8 004ed594     tier1:utlbuffer.obj
 0002:000535a4       ??_R2CUtlCharConversion@@8 004ed5a4     tier1:utlbuffer.obj
 0002:000535ac       ??_R1A@?0A@EA@CUtlCharConversion@@8 004ed5ac     tier1:utlbuffer.obj
 0002:000535c8       ??_R4CUtlNoEscConversion@@6B@ 004ed5c8     tier1:utlbuffer.obj
 0002:000535dc       ??_R3CUtlNoEscConversion@@8 004ed5dc     tier1:utlbuffer.obj
 0002:000535ec       ??_R2CUtlNoEscConversion@@8 004ed5ec     tier1:utlbuffer.obj
 0002:000535f8       ??_R1A@?0A@EA@CUtlNoEscConversion@@8 004ed5f8     tier1:utlbuffer.obj
 0002:00053614       ??_R4CUtlCStringConversion@@6B@ 004ed614     tier1:utlbuffer.obj
 0002:00053628       ??_R3CUtlCStringConversion@@8 004ed628     tier1:utlbuffer.obj
 0002:00053638       ??_R2CUtlCStringConversion@@8 004ed638     tier1:utlbuffer.obj
 0002:00053644       ??_R1A@?0A@EA@CUtlCStringConversion@@8 004ed644     tier1:utlbuffer.obj
 0002:00053660       ??_R3ctype_base@std@@8     004ed660     tier1:tokenreader.obj
 0002:00053670       ??_R2ctype_base@std@@8     004ed670     tier1:tokenreader.obj
 0002:0005367c       ??_R1A@?0A@EA@ctype_base@std@@8 004ed67c     tier1:tokenreader.obj
 0002:00053698       ??_R4?$basic_ios@DU?$char_traits@D@std@@@std@@6B@ 004ed698     tier1:tokenreader.obj
 0002:000536ac       ??_R4failure@ios_base@std@@6B@ 004ed6ac     tier1:tokenreader.obj
 0002:000536c0       ??_R3failure@ios_base@std@@8 004ed6c0     tier1:tokenreader.obj
 0002:000536d0       ??_R2failure@ios_base@std@@8 004ed6d0     tier1:tokenreader.obj
 0002:000536e0       ??_R1A@?0A@EA@failure@ios_base@std@@8 004ed6e0     tier1:tokenreader.obj
 0002:000536fc       ??_R4?$ctype@D@std@@6B@    004ed6fc     tier1:tokenreader.obj
 0002:00053710       ??_R3?$ctype@D@std@@8      004ed710     tier1:tokenreader.obj
 0002:00053720       ??_R2?$ctype@D@std@@8      004ed720     tier1:tokenreader.obj
 0002:00053730       ??_R1A@?0A@EA@?$ctype@D@std@@8 004ed730     tier1:tokenreader.obj
 0002:0005374c       ??_R4TokenReader@@6B@      004ed74c     tier1:tokenreader.obj
 0002:00053760       ??_R3TokenReader@@8        004ed760     tier1:tokenreader.obj
 0002:00053770       ??_R2TokenReader@@8        004ed770     tier1:tokenreader.obj
 0002:0005378c       ??_R1A@?0A@EA@TokenReader@@8 004ed78c     tier1:tokenreader.obj
 0002:000537a8       ??_R1A@?0A@EN@?$basic_ifstream@DU?$char_traits@D@std@@@std@@8 004ed7a8     tier1:tokenreader.obj
 0002:000537c4       ??_R1A@?0A@EJ@?$basic_istream@DU?$char_traits@D@std@@@std@@8 004ed7c4     tier1:tokenreader.obj
 0002:000537e0       ??_R1A@A@3FJ@?$basic_ios@DU?$char_traits@D@std@@@std@@8 004ed7e0     tier1:tokenreader.obj
 0002:000537fc       ??_R1A@A@3EJ@ios_base@std@@8 004ed7fc     tier1:tokenreader.obj
 0002:00053818       ??_R13A@3EJ@?$_Iosb@H@std@@8 004ed818     tier1:tokenreader.obj
 0002:00053834       ??_R3IVTFTexture@@8        004ed834     vtf:vtf.obj
 0002:00053844       ??_R2IVTFTexture@@8        004ed844     vtf:vtf.obj
 0002:0005384c       ??_R1A@?0A@EA@IVTFTexture@@8 004ed84c     vtf:vtf.obj
 0002:00053868       ??_R4CVTFTexture@@6B@      004ed868     vtf:vtf.obj
 0002:0005387c       ??_R3CVTFTexture@@8        004ed87c     vtf:vtf.obj
 0002:0005388c       ??_R2CVTFTexture@@8        004ed88c     vtf:vtf.obj
 0002:00053898       ??_R1A@?0A@EA@CVTFTexture@@8 004ed898     vtf:vtf.obj
 0002:000538b4       ??_R4type_info@@6B@        004ed8b4     LIBCMT:typinfo.obj
 0002:000538c8       ??_R3type_info@@8          004ed8c8     LIBCMT:typinfo.obj
 0002:000538d8       ??_R2type_info@@8          004ed8d8     LIBCMT:typinfo.obj
 0002:000538e0       ??_R1A@?0A@EA@type_info@@8 004ed8e0     LIBCMT:typinfo.obj
 0002:000538fc       ??_R4exception@std@@6B@    004ed8fc     LIBCMT:stdexcpt.obj
 0002:00053910       ??_R4bad_cast@std@@6B@     004ed910     LIBCMT:stdexcpt.obj
 0002:00053924       ??_R3bad_cast@std@@8       004ed924     LIBCMT:stdexcpt.obj
 0002:00053934       ??_R2bad_cast@std@@8       004ed934     LIBCMT:stdexcpt.obj
 0002:00053940       ??_R1A@?0A@EA@bad_cast@std@@8 004ed940     LIBCMT:stdexcpt.obj
 0002:0005395c       ??_R4bad_exception@std@@6B@ 004ed95c     LIBCMT:frame.obj
 0002:00053970       ??_R3bad_exception@std@@8  004ed970     LIBCMT:frame.obj
 0002:00053980       ??_R2bad_exception@std@@8  004ed980     LIBCMT:frame.obj
 0002:0005398c       ??_R1A@?0A@EA@bad_exception@std@@8 004ed98c     LIBCMT:frame.obj
 0002:000539a8       ??_R4out_of_range@std@@6B@ 004ed9a8     libcpmt:string.obj
 0002:000539bc       ??_R3out_of_range@std@@8   004ed9bc     libcpmt:string.obj
 0002:000539cc       ??_R2out_of_range@std@@8   004ed9cc     libcpmt:string.obj
 0002:000539dc       ??_R1A@?0A@EA@out_of_range@std@@8 004ed9dc     libcpmt:string.obj
 0002:000539f8       ??_R4_Locimp@locale@std@@6B@ 004ed9f8     libcpmt:locale0.obj
 0002:00053a0c       ??_R3_Locimp@locale@std@@8 004eda0c     libcpmt:locale0.obj
 0002:00053a1c       ??_R2_Locimp@locale@std@@8 004eda1c     libcpmt:locale0.obj
 0002:00053a28       ??_R1A@?0A@EA@_Locimp@locale@std@@8 004eda28     libcpmt:locale0.obj
 0002:00053a44       ___rtc_iaa                 004eda44     LIBCMT:initsect.obj
 0002:00053a48       ___rtc_izz                 004eda48     LIBCMT:initsect.obj
 0002:00053a4c       ___rtc_taa                 004eda4c     LIBCMT:initsect.obj
 0002:00053a50       ___rtc_tzz                 004eda50     LIBCMT:initsect.obj
 0002:00053a58       __TI2?AVbad_alloc@std@@    004eda58     mstristrip.obj
 0002:00053a68       __CTA2?AVbad_alloc@std@@   004eda68     mstristrip.obj
 0002:00053a74       __CT??_R0?AVbad_alloc@std@@@8??0bad_alloc@std@@QAE@ABV01@@Z12 004eda74     mstristrip.obj
 0002:00053a90       __CT??_R0?AVexception@std@@@8??0exception@std@@QAE@ABV01@@Z12 004eda90     mstristrip.obj
 0002:00053b38       __TI3?AVlength_error@std@@ 004edb38     mstristrip.obj
 0002:00053b48       __CTA3?AVlength_error@std@@ 004edb48     mstristrip.obj
 0002:00053b58       __CT??_R0?AVlength_error@std@@@8??0length_error@std@@QAE@ABV01@@Z40 004edb58     mstristrip.obj
 0002:00053b74       __CT??_R0?AVlogic_error@std@@@8??0logic_error@std@@QAE@ABV01@@Z40 004edb74     mstristrip.obj
 0002:00053b90       __TI2?AVruntime_error@std@@ 004edb90     chunkfile.obj
 0002:00053ba0       __CTA2?AVruntime_error@std@@ 004edba0     chunkfile.obj
 0002:00053bac       __CT??_R0?AVruntime_error@std@@@8??0runtime_error@std@@QAE@ABV01@@Z40 004edbac     chunkfile.obj
 0002:00053bc8       __TI3?AVfailure@ios_base@std@@ 004edbc8     tier1:tokenreader.obj
 0002:00053bd8       __CTA3?AVfailure@ios_base@std@@ 004edbd8     tier1:tokenreader.obj
 0002:00053be8       __CT??_R0?AVfailure@ios_base@std@@@8??0failure@ios_base@std@@QAE@ABV012@@Z40 004edbe8     tier1:tokenreader.obj
 0002:00053c04       __TI2?AVbad_cast@std@@     004edc04     tier1:tokenreader.obj
 0002:00053c14       __CTA2?AVbad_cast@std@@    004edc14     tier1:tokenreader.obj
 0002:00053c20       __CT??_R0?AVbad_cast@std@@@8??0bad_cast@std@@QAE@ABV01@@Z12 004edc20     tier1:tokenreader.obj
 0002:000543bc       __TI2?AVbad_exception@std@@ 004ee3bc     LIBCMT:frame.obj
 0002:000543cc       __CTA2?AVbad_exception@std@@ 004ee3cc     LIBCMT:frame.obj
 0002:000543d8       __CT??_R0?AVbad_exception@std@@@8??0bad_exception@std@@QAE@ABV01@@Z12 004ee3d8     LIBCMT:frame.obj
 0002:000546c4       __TI3?AVout_of_range@std@@ 004ee6c4     libcpmt:string.obj
 0002:00054700       __CTA3?AVout_of_range@std@@ 004ee700     libcpmt:string.obj
 0002:00054710       __CT??_R0?AVout_of_range@std@@@8??0out_of_range@std@@QAE@ABV01@@Z40 004ee710     libcpmt:string.obj
 0002:000549e4       __IMPORT_DESCRIPTOR_KERNEL32 004ee9e4     kernel32:KERNEL32.dll
 0002:000549f8       __IMPORT_DESCRIPTOR_ADVAPI32 004ee9f8     advapi32:ADVAPI32.dll
 0002:00054a0c       __IMPORT_DESCRIPTOR_tier0  004eea0c     tier0:tier0.dll
 0002:00054a20       __IMPORT_DESCRIPTOR_vstdlib 004eea20     vstdlib:vstdlib.dll
 0002:00054a34       __NULL_IMPORT_DESCRIPTOR   004eea34     kernel32:KERNEL32.dll
 0003:000000e0       ?g_EdgeDims@@3PAHA         004f00e0     disp_common.obj
 0003:000000f0       ?g_ShiftInfos@@3PAY02VCShiftInfo@@A 004f00f0     disp_common.obj
 0003:0000015c       ?g_EdgeSideLenMul@@3PAHA   004f015c     disp_common.obj
 0003:00000254       ??_R0?AVIVirtualMeshEvent@@@8 004f0254     disp_ivp.obj
 0003:00000274       ??_R0?AVCDispMeshEvent@@@8 004f0274     disp_ivp.obj
 0003:00000320       ?g_TWinding@@3VCTesselateWinding@@A 004f0320     disp_powerinfo.obj
 0003:00000328       ?g_PowerInfos@@3PAPAVCPowerInfo@@A 004f0328     disp_powerinfo.obj
 0003:00000374       ?g_TesselateVerts@@3PAVCTesselateVert@@A 004f0374     disp_powerinfo.obj
 0003:000006a0       ?firstmodeledge@@3HA       004f06a0     faces.obj
 0003:000006a4       ?g_maxLightmapDimension@@3MA 004f06a4     faces.obj
 0003:000006bc       ??_R0?AVCPhysCollisionEntry@@@8 004f06bc     ivp.obj
 0003:000006e0       ??_R0?AVCPhysCollisionEntrySolid@@@8 004f06e0     ivp.obj
 0003:00000708       ??_R0?AVCPhysCollisionEntryStaticSolid@@@8 004f0708     ivp.obj
 0003:00000738       ??_R0?AVCPhysCollisionEntryStaticMesh@@@8 004f0738     ivp.obj
 0003:00000764       ??_R0?AVCPhysCollisionEntryFluid@@@8 004f0764     ivp.obj
 0003:000007e4       ?g_ClipTexinfo@@3HA        004f07e4     map.obj
 0003:000007f8       ?s_MapPatchedMatToOriginalMat@@3V?$CUtlRBTree@UNameTranslationLookup_t@@HP6A_NABU1@0@ZV?$CUtlMemory@U?$UtlRBTreeNode_t@UNameTranslationLookup_t@@H@@H@@@@A 004f07f8     materialpatch.obj
 0003:00000824       __amblksiz                 004f0824     memoverride.obj
 0003:00000828       __crtheap                  004f0828     memoverride.obj
 0003:0000082c       ___active_heap             004f082c     memoverride.obj
 0003:00000830       __crtDbgFlag               004f0830     memoverride.obj
 0003:00000834       __crtAssertBusy            004f0834     memoverride.obj
 0003:0000083c       ??_R0?AVbad_alloc@std@@@8  004f083c     mstristrip.obj
 0003:00000858       ??_R0?AVexception@std@@@8  004f0858     mstristrip.obj
 0003:00000874       ??_R0?AVlogic_error@std@@@8 004f0874     mstristrip.obj
 0003:00000894       ??_R0?AVlength_error@std@@@8 004f0894     mstristrip.obj
 0003:000008fc       ?g_SkyCluster@@3HA         004f08fc     prtfile.obj
 0003:00000978       ?baseaxis@@3PAVVector@@A   004f0978     textures.obj
 0003:00000a70       ?microvolume@@3MA          004f0a70     vbsp.obj
 0003:00000a74       ?g_defaultLuxelSize@@3MA   004f0a74     vbsp.obj
 0003:00000a78       ?g_luxelScale@@3MA         004f0a78     vbsp.obj
 0003:00000a7c       ?g_minLuxelScale@@3MA      004f0a7c     vbsp.obj
 0003:00000a80       ?block_xl@@3HA             004f0a80     vbsp.obj
 0003:00000a84       ?block_xh@@3HA             004f0a84     vbsp.obj
 0003:00000a88       ?block_yl@@3HA             004f0a88     vbsp.obj
 0003:00000a8c       ?block_yh@@3HA             004f0a8c     vbsp.obj
 0003:00000ab8       ?m_DataMap@ZIP_EndOfCentralDirRecord@@2Udatamap_t@@A 004f0ab8     zip_utils.obj
 0003:00000ad0       ?m_DataMap@ZIP_FileHeader@@2Udatamap_t@@A 004f0ad0     zip_utils.obj
 0003:00000ae8       ?m_DataMap@ZIP_LocalFileHeader@@2Udatamap_t@@A 004f0ae8     zip_utils.obj
 0003:00000b00       ?m_DataMap@ZIP_PreloadHeader@@2Udatamap_t@@A 004f0b00     zip_utils.obj
 0003:00000b18       ?m_DataMap@ZIP_PreloadDirectoryEntry@@2Udatamap_t@@A 004f0b18     zip_utils.obj
 0003:00000b54       ??_R0?AVIWriteStream@@@8   004f0b54     zip_utils.obj
 0003:00000b70       ??_R0?AVCFileStream@@@8    004f0b70     zip_utils.obj
 0003:00000b8c       ??_R0?AVIZip@@@8           004f0b8c     zip_utils.obj
 0003:00000ba0       ??_R0?AVCBufferStream@@@8  004f0ba0     zip_utils.obj
 0003:00001554       ??_R0?AVCZip@@@8           004f1554     zip_utils.obj
 0003:00001568       ?m_DataMap@dheader_t@@2Udatamap_t@@A 004f1568     bsplib.obj
 0003:00001580       ?m_DataMap@lump_t@@2Udatamap_t@@A 004f1580     bsplib.obj
 0003:00001598       ?m_DataMap@dflagslump_t@@2Udatamap_t@@A 004f1598     bsplib.obj
 0003:000015b0       ?m_DataMap@dplane_t@@2Udatamap_t@@A 004f15b0     bsplib.obj
 0003:000015c8       ?m_DataMap@dleaf_version_0_t@@2Udatamap_t@@A 004f15c8     bsplib.obj
 0003:000015e0       ?m_DataMap@dleaf_t@@2Udatamap_t@@A 004f15e0     bsplib.obj
 0003:000015f8       ?m_DataMap@CompressedLightCube@@2Udatamap_t@@A 004f15f8     bsplib.obj
 0003:00001610       ?m_DataMap@dleafambientindex_t@@2Udatamap_t@@A 004f1610     bsplib.obj
 0003:00001628       ?m_DataMap@dleafambientlighting_t@@2Udatamap_t@@A 004f1628     bsplib.obj
 0003:00001640       ?m_DataMap@dvertex_t@@2Udatamap_t@@A 004f1640     bsplib.obj
 0003:00001658       ?m_DataMap@dnode_t@@2Udatamap_t@@A 004f1658     bsplib.obj
 0003:00001670       ?m_DataMap@texinfo_s@@2Udatamap_t@@A 004f1670     bsplib.obj
 0003:00001688       ?m_DataMap@dtexdata_t@@2Udatamap_t@@A 004f1688     bsplib.obj
 0003:000016a0       ?m_DataMap@ddispinfo_t@@2Udatamap_t@@A 004f16a0     bsplib.obj
 0003:000016b8       ?m_DataMap@CDispNeighbor@@2Udatamap_t@@A 004f16b8     bsplib.obj
 0003:000016d0       ?m_DataMap@CDispCornerNeighbors@@2Udatamap_t@@A 004f16d0     bsplib.obj
 0003:000016e8       ?m_DataMap@CDispSubNeighbor@@2Udatamap_t@@A 004f16e8     bsplib.obj
 0003:00001700       ?m_DataMap@CDispVert@@2Udatamap_t@@A 004f1700     bsplib.obj
 0003:00001718       ?m_DataMap@CDispTri@@2Udatamap_t@@A 004f1718     bsplib.obj
 0003:00001730       ?m_DataMap@CFaceMacroTextureInfo@@2Udatamap_t@@A 004f1730     bsplib.obj
 0003:00001748       ?m_DataMap@dprimitive_t@@2Udatamap_t@@A 004f1748     bsplib.obj
 0003:00001760       ?m_DataMap@dprimvert_t@@2Udatamap_t@@A 004f1760     bsplib.obj
 0003:00001778       ?m_DataMap@dface_t@@2Udatamap_t@@A 004f1778     bsplib.obj
 0003:00001790       ?m_DataMap@dfaceid_t@@2Udatamap_t@@A 004f1790     bsplib.obj
 0003:000017a8       ?m_DataMap@dbrush_t@@2Udatamap_t@@A 004f17a8     bsplib.obj
 0003:000017c0       ?m_DataMap@dbrushside_t@@2Udatamap_t@@A 004f17c0     bsplib.obj
 0003:000017d8       ?m_DataMap@dedge_t@@2Udatamap_t@@A 004f17d8     bsplib.obj
 0003:000017f0       ?m_DataMap@dmodel_t@@2Udatamap_t@@A 004f17f0     bsplib.obj
 0003:00001808       ?m_DataMap@dphysmodel_t@@2Udatamap_t@@A 004f1808     bsplib.obj
 0003:00001820       ?m_DataMap@dphysdisp_t@@2Udatamap_t@@A 004f1820     bsplib.obj
 0003:00001838       ?m_DataMap@darea_t@@2Udatamap_t@@A 004f1838     bsplib.obj
 0003:00001850       ?m_DataMap@dareaportal_t@@2Udatamap_t@@A 004f1850     bsplib.obj
 0003:00001868       ?m_DataMap@dworldlight_t@@2Udatamap_t@@A 004f1868     bsplib.obj
 0003:00001880       ?m_DataMap@dleafwaterdata_t@@2Udatamap_t@@A 004f1880     bsplib.obj
 0003:00001898       ?m_DataMap@doccluderdata_t@@2Udatamap_t@@A 004f1898     bsplib.obj
 0003:000018b0       ?m_DataMap@doccluderpolydata_t@@2Udatamap_t@@A 004f18b0     bsplib.obj
 0003:000018c8       ?m_DataMap@dcubemapsample_t@@2Udatamap_t@@A 004f18c8     bsplib.obj
 0003:000018e0       ?m_DataMap@doverlay_t@@2Udatamap_t@@A 004f18e0     bsplib.obj
 0003:000018f8       ?m_DataMap@dwateroverlay_t@@2Udatamap_t@@A 004f18f8     bsplib.obj
 0003:00001910       ?m_DataMap@doverlayfade_t@@2Udatamap_t@@A 004f1910     bsplib.obj
 0003:00001928       ?m_DataMap@dgamelumpheader_t@@2Udatamap_t@@A 004f1928     bsplib.obj
 0003:00001940       ?m_DataMap@dgamelump_t@@2Udatamap_t@@A 004f1940     bsplib.obj
 0003:00001958       ?m_DataMap@StaticPropDictLump_t@@2Udatamap_t@@A 004f1958     bsplib.obj
 0003:00001970       ?m_DataMap@StaticPropLump_t@@2Udatamap_t@@A 004f1970     bsplib.obj
 0003:00001988       ?m_DataMap@StaticPropLumpV4_t@@2Udatamap_t@@A 004f1988     bsplib.obj
 0003:000019a0       ?m_DataMap@StaticPropLumpV5_t@@2Udatamap_t@@A 004f19a0     bsplib.obj
 0003:000019b8       ?m_DataMap@StaticPropLeafLump_t@@2Udatamap_t@@A 004f19b8     bsplib.obj
 0003:000019d0       ?m_DataMap@DetailObjectDictLump_t@@2Udatamap_t@@A 004f19d0     bsplib.obj
 0003:000019e8       ?m_DataMap@DetailObjectLump_t@@2Udatamap_t@@A 004f19e8     bsplib.obj
 0003:00001a00       ?m_DataMap@DetailSpriteDictLump_t@@2Udatamap_t@@A 004f1a00     bsplib.obj
 0003:00001a18       ?m_DataMap@DetailPropLightstylesLump_t@@2Udatamap_t@@A 004f1a18     bsplib.obj
 0003:00001a30       ?m_DataMap@MeshHeader_t@HardwareVerts@@2Udatamap_t@@A 004f1a30     bsplib.obj
 0003:00001a48       ?m_DataMap@FileHeader_t@HardwareVerts@@2Udatamap_t@@A 004f1a48     bsplib.obj
 0003:00001b54       ?dvis@@3PAUdvis_t@@A       004f1b54     bsplib.obj
 0003:00001b58       ?pdlightdata@@3PAV?$CUtlVector@EV?$CUtlMemory@EH@@@@A 004f1b58     bsplib.obj
 0003:00001b5c       ?pNumworldlights@@3PAHA    004f1b5c     bsplib.obj
 0003:00001b60       ?dworldlights@@3PAUdworldlight_t@@A 004f1b60     bsplib.obj
 0003:00001b64       ?m_DataMap@swapcollideheader_t@@2Udatamap_t@@A 004f1b64     bsplib.obj
 0003:00001b7c       ?m_DataMap@swapcompactsurfaceheader_t@@2Udatamap_t@@A 004f1b7c     bsplib.obj
 0003:00001b94       ?m_DataMap@swapmoppsurfaceheader_t@@2Udatamap_t@@A 004f1b94     bsplib.obj
 0003:00001bc4       ?texinfo@@3V?$CUtlVector@Utexinfo_s@@V?$CUtlMemory@Utexinfo_s@@H@@@@A 004f1bc4     bsplib.obj
 0003:00001bd8       ?g_OccluderData@@3V?$CUtlVector@Udoccluderdata_t@@V?$CUtlMemory@Udoccluderdata_t@@H@@@@A 004f1bd8     bsplib.obj
 0003:00001bec       ?g_OccluderPolyData@@3V?$CUtlVector@Udoccluderpolydata_t@@V?$CUtlMemory@Udoccluderpolydata_t@@H@@@@A 004f1bec     bsplib.obj
 0003:00001c00       ?g_OccluderVertexIndices@@3V?$CUtlVector@HV?$CUtlMemory@HH@@@@A 004f1c00     bsplib.obj
 0003:00001c14       ?g_GameLumps@@3VCGameLump@@A 004f1c14     bsplib.obj
 0003:00005ec0       ??_R0?AVCDispUtilsHelper@@@8 004f5ec0     builddisp.obj
 0003:00005ee0       ??_R0?AVCCoreDispInfo@@@8  004f5ee0     builddisp.obj
 0003:00005f20       ??_R0?AVios_base@std@@@8   004f5f20     chunkfile.obj
 0003:00005f3c       ??_R0?AV?$_Iosb@H@std@@@8  004f5f3c     chunkfile.obj
 0003:00005f58       ??_R0?AV?$basic_istream@DU?$char_traits@D@std@@@std@@@8 004f5f58     chunkfile.obj
 0003:00005f94       ??_R0?AV?$basic_ios@DU?$char_traits@D@std@@@std@@@8 004f5f94     chunkfile.obj
 0003:00005fcc       ??_R0?AV?$basic_streambuf@DU?$char_traits@D@std@@@std@@@8 004f5fcc     chunkfile.obj
 0003:00006008       ??_R0?AV?$basic_filebuf@DU?$char_traits@D@std@@@std@@@8 004f6008     chunkfile.obj
 0003:00006044       ??_R0?AVfacet@locale@std@@@8 004f6044     chunkfile.obj
 0003:00006064       ??_R0?AVcodecvt_base@std@@@8 004f6064     chunkfile.obj
 0003:00006084       ??_R0?AVruntime_error@std@@@8 004f6084     chunkfile.obj
 0003:000060a4       ??_R0?AV?$codecvt@DDH@std@@@8 004f60a4     chunkfile.obj
 0003:000060c4       ??_R0?AV?$basic_ifstream@DU?$char_traits@D@std@@@std@@@8 004f60c4     chunkfile.obj
 0003:00006118       ?g_CleanupFunctions@@3V?$CUtlLinkedList@P6AXXZG$0A@GV?$CUtlMemory@U?$UtlLinkedListElem_t@P6AXXZG@@G@@@@A 004f6118     cmdlib.obj
 0003:00006134       ?g_ExtraSpewHooks@@3V?$CUtlLinkedList@P6AXPBD@ZG$0A@GV?$CUtlMemory@U?$UtlLinkedListElem_t@P6AXPBD@ZG@@G@@@@A 004f6134     cmdlib.obj
 0003:00006184       ?g_pfnCallback@@3P6AXPBD0H@ZA 004f6184     scriplib.obj
 0003:00006188       ?scriptlib@@3PAVIScriptLib@@A 004f6188     scriplib.obj
 0003:00006198       ??_R0?AVIScriptLib@@@8     004f6198     scriplib.obj
 0003:000061b4       ??_R0?AVCScriptLib@@@8     004f61b4     scriplib.obj
 0003:000061d0       ?numthreads@@3HA           004f61d0     threads.obj
 0003:00006258       ??_R0?AVCUtlCharConversion@@@8 004f6258     tier1:utlbuffer.obj
 0003:0000627c       ??_R0?AVCUtlNoEscConversion@@@8 004f627c     tier1:utlbuffer.obj
 0003:000062a0       ??_R0?AVCUtlCStringConversion@@@8 004f62a0     tier1:utlbuffer.obj
 0003:000062c4       ?s_bAllowStaticSymbolTable@CUtlSymbol@@1_NA 004f62c4     tier1:utlsymbol.obj
 0003:000062e0       ?g_KeyValuesErrorStack@@3VCKeyValuesErrorStack@@A 004f62e0     tier1:KeyValues.obj
 0003:000063f8       ??_R0?AUctype_base@std@@@8 004f63f8     tier1:tokenreader.obj
 0003:00006418       ??_R0?AVfailure@ios_base@std@@@8 004f6418     tier1:tokenreader.obj
 0003:0000643c       ??_R0?AV?$ctype@D@std@@@8  004f643c     tier1:tokenreader.obj
 0003:00006458       ??_R0?AVbad_cast@std@@@8   004f6458     tier1:tokenreader.obj
 0003:00006474       ??_R0?AVTokenReader@@@8    004f6474     tier1:tokenreader.obj
 0003:00006898       ?pfSqrt@@3P6AMM@ZA         004f6898     mathlib:mathlib_base.obj
 0003:0000689c       ?pfRSqrt@@3P6AMM@ZA        004f689c     mathlib:mathlib_base.obj
 0003:000068a0       ?pfRSqrtFast@@3P6AMM@ZA    004f68a0     mathlib:mathlib_base.obj
 0003:000068a4       ?pfVectorNormalize@@3P6IMAAVVector@@@ZA 004f68a4     mathlib:mathlib_base.obj
 0003:000068a8       ?pfVectorNormalizeFast@@3P6IXAAVVector@@@ZA 004f68a8     mathlib:mathlib_base.obj
 0003:000068ac       ?pfInvRSquared@@3P6AMPBM@ZA 004f68ac     mathlib:mathlib_base.obj
 0003:000068b0       ?pfFastSinCos@@3P6AXMPAM0@ZA 004f68b0     mathlib:mathlib_base.obj
 0003:000068b4       ?pfFastCos@@3P6AMM@ZA      004f68b4     mathlib:mathlib_base.obj
 0003:000068c0       ?vec3_invalid@@3VVector@@B 004f68c0     mathlib:mathlib_base.obj
 0003:00006900       ?power2_n@@3PAMA           004f6900     mathlib:color_conversion.obj
 0003:00006d30       ?m_DataMap@VTFFileBaseHeader_t@@2Udatamap_t@@A 004f6d30     vtf:vtf.obj
 0003:00006d48       ?m_DataMap@VTFFileHeaderV7_1_t@@2Udatamap_t@@A 004f6d48     vtf:vtf.obj
 0003:00006d60       ?m_DataMap@VTFFileHeaderV7_2_t@@2Udatamap_t@@A 004f6d60     vtf:vtf.obj
 0003:00006d78       ?m_DataMap@VTFFileHeaderV7_3_t@@2Udatamap_t@@A 004f6d78     vtf:vtf.obj
 0003:00006d90       ?m_DataMap@VTFFileHeader_t@@2Udatamap_t@@A 004f6d90     vtf:vtf.obj
 0003:00006da8       ?m_DataMap@VTFFileHeaderX360_t@@2Udatamap_t@@A 004f6da8     vtf:vtf.obj
 0003:00006dc0       ?g_leftFaceVerts@@3PAHA    004f6dc0     vtf:vtf.obj
 0003:00006dd0       ?g_frontFaceVerts@@3PAHA   004f6dd0     vtf:vtf.obj
 0003:00006de0       ?g_downFaceVerts@@3PAHA    004f6de0     vtf:vtf.obj
 0003:00006df0       ?g_rightFaceVerts@@3PAHA   004f6df0     vtf:vtf.obj
 0003:00006e00       ?g_backFaceVerts@@3PAHA    004f6e00     vtf:vtf.obj
 0003:00006e10       ?g_upFaceVerts@@3PAHA      004f6e10     vtf:vtf.obj
 0003:00006e20       ?g_FaceVerts@@3PAPAHA      004f6e20     vtf:vtf.obj
 0003:00006e38       ?g_skybox_rightFaceVerts@@3PAHA 004f6e38     vtf:vtf.obj
 0003:00006e48       ?g_skybox_leftFaceVerts@@3PAHA 004f6e48     vtf:vtf.obj
 0003:00006e58       ?g_skybox_backFaceVerts@@3PAHA 004f6e58     vtf:vtf.obj
 0003:00006e68       ?g_skybox_frontFaceVerts@@3PAHA 004f6e68     vtf:vtf.obj
 0003:00006e78       ?g_skybox_upFaceVerts@@3PAHA 004f6e78     vtf:vtf.obj
 0003:00006e88       ?g_skybox_downFaceVerts@@3PAHA 004f6e88     vtf:vtf.obj
 0003:00006e98       ?g_skybox_FaceVerts@@3PAPAHA 004f6e98     vtf:vtf.obj
 0003:00006eb8       ??_R0?AVIVTFTexture@@@8    004f6eb8     vtf:vtf.obj
 0003:00006ed4       ??_R0?AVCVTFTexture@@@8    004f6ed4     vtf:vtf.obj
 0003:00007618       __fltused                  004f7618     LIBCMT:fpinit.obj
 0003:0000761c       __ldused                   004f761c     LIBCMT:fpinit.obj
 0003:00007624       ??_R0?AVtype_info@@@8      004f7624     LIBCMT:typinfo.obj
 0003:00007650       __OP_FMODjmptab            004f7650     LIBCMT:87fmod.obj
 0003:000076a0       __aexit_rtn                004f76a0     LIBCMT:crt0dat.obj
 0003:000076b0       __iob                      004f76b0     LIBCMT:_file.obj
 0003:00007aa0       ___app_type                004f7aa0     LIBCMT:crt0.obj
 0003:00007ad0       __half                     004f7ad0     LIBCMT:pow.obj
 0003:00007ae0       __cfltcvt_tab              004f7ae0     LIBCMT:cmiscdat.obj
 0003:00007b08       ___nullstring              004f7b08     LIBCMT:output.obj
 0003:00007b0c       ___wnullstring             004f7b0c     LIBCMT:output.obj
 0003:00007b10       ___badioinfo               004f7b10     LIBCMT:ioinit.obj
 0003:00007b48       ___security_cookie         004f7b48     LIBCMT:gs_cookie.obj
 0003:00007b4c       ___security_cookie_complement 004f7b4c     LIBCMT:gs_cookie.obj
 0003:00007b50       ___flsindex                004f7b50     LIBCMT:tidtable.obj
 0003:00007b54       ___getvalueindex           004f7b54     LIBCMT:tidtable.obj
 0003:00007b60       ___abort_behavior          004f7b60     LIBCMT:abort.obj
 0003:00007c20       ___initialmbcinfo          004f7c20     LIBCMT:mbctype.obj
 0003:00007e40       __mbctype                  004f7e40     LIBCMT:mbctype.obj
 0003:00007f48       __mbcasemap                004f7f48     LIBCMT:mbctype.obj
 0003:00008048       ___ptmbcinfo               004f8048     LIBCMT:mbctype.obj
 0003:00008144       ___globallocalestatus      004f8144     LIBCMT:glstatus.obj
 0003:00008148       ___clocalestr              004f8148     LIBCMT:nlsdata2.obj
 0003:00008150       ___initiallocinfo          004f8150     LIBCMT:nlsdata2.obj
 0003:00008228       ___ptlocinfo               004f8228     LIBCMT:nlsdata2.obj
 0003:0000822c       ___lc_clike                004f822c     LIBCMT:nlsdata2.obj
 0003:00008230       ___initiallocalestructinfo 004f8230     LIBCMT:nlsdata2.obj
 0003:00008240       ??_R0?AVbad_exception@std@@@8 004f8240     LIBCMT:frame.obj
 0003:00008260       __indefinite               004f8260     LIBCMT:87disp.obj
 0003:0000826a       __piby2                    004f826a     LIBCMT:87disp.obj
 0003:00008510       __XcptActTab               004f8510     LIBCMT:winxfltr.obj
 0003:00008588       __First_FPE_Indx           004f8588     LIBCMT:winxfltr.obj
 0003:0000858c       __Num_FPE                  004f858c     LIBCMT:winxfltr.obj
 0003:00008590       __XcptActTabSize           004f8590     LIBCMT:winxfltr.obj
 0003:00008594       __XcptActTabCount          004f8594     LIBCMT:winxfltr.obj
 0003:00008598       __tmpoff                   004f8598     LIBCMT:rmtmp.obj
 0003:0000859c       __tempoff                  004f859c     LIBCMT:rmtmp.obj
 0003:000085a0       __lookuptrailbytes         004f85a0     LIBCMT:read.obj
 0003:000086a8       __sys_errlist              004f86a8     LIBCMT:syserr.obj
 0003:00008758       __sys_nerr                 004f8758     LIBCMT:syserr.obj
 0003:00008770       __HUGE                     004f8770     LIBCMT:huge.obj
 0003:00008780       __infinity                 004f8780     LIBCMT:87tran.obj
 0003:0000878a       __minfinity                004f878a     LIBCMT:87tran.obj
 0003:00008794       __logemax                  004f8794     LIBCMT:87tran.obj
 0003:000087ba       __OP_EXPjmptab             004f87ba     LIBCMT:87tran.obj
 0003:000087e0       __NLG_Destination          004f87e0     LIBCMT:exsup.obj
 0003:000087f0       __pctype                   004f87f0     LIBCMT:ctype.obj
 0003:000087f4       __pwctype                  004f87f4     LIBCMT:ctype.obj
 0003:000087f8       ___lc_time_c               004f87f8     LIBCMT:strftime.obj
 0003:000088b0       ___lc_time_curr            004f88b0     LIBCMT:strftime.obj
 0003:000088b4       ___lconv_static_decimal    004f88b4     LIBCMT:lconv.obj
 0003:000088b8       ___lconv_c                 004f88b8     LIBCMT:lconv.obj
 0003:000088e8       ___lconv                   004f88e8     LIBCMT:lconv.obj
 0003:000088ec       ___mb_cur_max              004f88ec     LIBCMT:nlsdata1.obj
 0003:000088f0       ___decimal_point           004f88f0     LIBCMT:nlsdata1.obj
 0003:000088f4       ___decimal_point_length    004f88f4     LIBCMT:nlsdata1.obj
 0003:00008930       __pow10pos                 004f8930     LIBCMT:constpow.obj
 0003:00008a90       __pow10neg                 004f8a90     LIBCMT:constpow.obj
 0003:00008bf0       __matherr_flag             004f8bf0     LIBCMT:matherr.obj
 0003:00008ce0       __d_inf                    004f8ce0     LIBCMT:util.obj
 0003:00008ce8       __d_ind                    004f8ce8     LIBCMT:util.obj
 0003:00008cf0       __d_max                    004f8cf0     LIBCMT:util.obj
 0003:00008cf8       __d_min                    004f8cf8     LIBCMT:util.obj
 0003:00008d00       __d_mzero                  004f8d00     LIBCMT:util.obj
 0003:00008d40       __timezone                 004f8d40     LIBCMT:timeset.obj
 0003:00008d44       __daylight                 004f8d44     LIBCMT:timeset.obj
 0003:00008d48       __dstbias                  004f8d48     LIBCMT:timeset.obj
 0003:00008dd0       __tzname                   004f8dd0     LIBCMT:timeset.obj
 0003:00008dd8       __lpdays                   004f8dd8     LIBCMT:days.obj
 0003:00008e0c       __days                     004f8e0c     LIBCMT:days.obj
 0003:00008e40       __p_overlay                004f8e40     LIBCMT:dospawn.obj
 0003:00008e44       __coninpfh                 004f8e44     LIBCMT:initcon.obj
 0003:00008e48       __confh                    004f8e48     LIBCMT:initcon.obj
 0003:00008e54       ??_R0?AVout_of_range@std@@@8 004f8e54     libcpmt:string.obj
 0003:00008e7c       ?_Sync@ios_base@std@@0_NA  004f8e7c     libcpmt:ios.obj
 0003:00008e84       ??_R0?AV_Locimp@locale@std@@@8 004f8e84     libcpmt:locale0.obj
 0003:00008ef0       ?_PJP_CPP_Copyright@@3PADA 004f8ef0     libcpmt:iosptrs.obj
 0003:000093ec       ?S3TC_BLOCK_WIDTH@@3HA     004f93ec     bitmap:S3_intrf.obj
 0003:00009790       ?nByteBitsMask@@3PAEA      004f9790     bitmap:ATiXCodec.obj
 0003:0000979c       ?dwRndAmount@@3PAKA        004f979c     bitmap:ATiXCodec.obj
 0003:000097e0       ?c_nonvis@@3HA             004f97e0     brushbsp.obj
 0003:000097e4       ?c_nodes@@3HA              004f97e4     brushbsp.obj
 0003:000097e8       ?c_active_brushes@@3HA     004f97e8     brushbsp.obj
 0003:00009814       ?minplanenums@@3PAHA       004f9814     csg.obj
 0003:00009820       ?maxplanenums@@3PAHA       004f9820     csg.obj
 0003:0002a278       ?s_Sentinel@?1??Links@?$CUtlRBTree@UCubemapInfo_t@@GP6A_NABU1@0@ZV?$CUtlMemory@U?$UtlRBTreeNode_t@UCubemapInfo_t@@G@@G@@@@IBEABU?$UtlRBTreeLinks_t@G@@G@Z@4U3@A 0051a278     cubemap.obj
 0003:0002a280       ??_B?1??Links@?$CUtlRBTree@UCubemapInfo_t@@GP6A_NABU1@0@ZV?$CUtlMemory@U?$UtlRBTreeNode_t@UCubemapInfo_t@@G@@G@@@@IBEABU?$UtlRBTreeLinks_t@G@@G@Z@51 0051a280     cubemap.obj
 0003:0002a2f8       ?s_Sentinel@?1??Links@?$CUtlRBTree@UStaticPropLookup_t@@GP6A_NABU1@0@ZV?$CUtlMemory@U?$UtlRBTreeNode_t@UStaticPropLookup_t@@G@@G@@@@IBEABU?$UtlRBTreeLinks_t@G@@G@Z@4U3@A 0051a2f8     detailobjects.obj
 0003:0002a300       ??_B?1??Links@?$CUtlRBTree@UStaticPropLookup_t@@GP6A_NABU1@0@ZV?$CUtlMemory@U?$UtlRBTreeNode_t@UStaticPropLookup_t@@G@@G@@@@IBEABU?$UtlRBTreeLinks_t@G@@G@Z@51 0051a300     detailobjects.obj
 0003:0002a310       ?dummy@?1??GetNodeInfo@CVBSPTesselateHelper@@QAEAAUDispNodeInfo_t@@H@Z@4U3@A 0051a310     disp_ivp.obj
 0003:00034430       ?nummapdispinfo@@3HA       00524430     disp_vbsp.obj
 0003:0003443c       ?g_CoreDispInfos@@3V?$CUtlVector@PAVCCoreDispInfo@@V?$CUtlMemory@PAVCCoreDispInfo@@H@@@@A 0052443c     disp_vbsp.obj
 0003:00034450       ?mapdispinfo@@3PAUmapdispinfo_t@@A 00524450     disp_vbsp.obj
 0003:014cc450       ?hashverts@@3PAHA          019bc450     faces.obj
 0003:0150c450       ?c_tryedges@@3HA           019fc450     faces.obj
 0003:0150c454       ?num_edge_verts@@3HA       019fc454     faces.obj
 0003:0150c458       ?c_uniqueverts@@3HA        019fc458     faces.obj
 0003:0150c45c       ?c_faces@@3HA              019fc45c     faces.obj
 0003:0150c460       ?c_facecollapse@@3HA       019fc460     faces.obj
 0003:0150c464       ?c_tjunctions@@3HA         019fc464     faces.obj
 0003:0150c468       ?edgefaces@@3PAY01PAUface_t@@A 019fc468     faces.obj
 0003:01700468       ?edge_verts@@3PAHA         01bf0468     faces.obj
 0003:01740468       ?c_nodefaces@@3HA          01c30468     faces.obj
 0003:0174046c       ?c_faceoverflows@@3HA      01c3046c     faces.obj
 0003:01740470       ?numsuperverts@@3HA        01c30470     faces.obj
 0003:01740474       ?edge_len@@3MA             01c30474     faces.obj
 0003:01740478       ?firstmodelface@@3HA       01c30478     faces.obj
 0003:0174047c       ?c_subdivide@@3HA          01c3047c     faces.obj
 0003:01740480       ?superverts@@3PAHA         01c30480     faces.obj
 0003:01740c80       ?vertexchain@@3PAHA        01c30c80     faces.obj
 0003:01780c80       ?c_badstartverts@@3HA      01c70c80     faces.obj
 0003:01780c84       ?c_degenerate@@3HA         01c70c84     faces.obj
 0003:01780c88       ?c_merge@@3HA              01c70c88     faces.obj
 0003:01780c8c       ?c_totalverts@@3HA         01c70c8c     faces.obj
 0003:01780c98       ?edge_dir@@3VVector@@A     01c70c98     faces.obj
 0003:01780ca4       ?edge_start@@3VVector@@A   01c70ca4     faces.obj
 0003:01780cb0       ?g_VertEdgeList@@3PAV?$CUtlVector@HV?$CUtlMemory@HH@@@@A 01c70cb0     faces.obj
 0003:018c0cb4       ?c_glfaces@@3HA            01db0cb4     glfile.obj
 0003:018c0cc0       ?physcollision@@3PAVIPhysicsCollision@@A 01db0cc0     ivp.obj
 0003:018c0d18       ?s_Sentinel@?1??Links@?$CUtlRBTree@UWaterTexInfo@@HP6A_NABU1@0@ZV?$CUtlMemory@U?$UtlRBTreeNode_t@UWaterTexInfo@@H@@H@@@@IBEABU?$UtlRBTreeLinks_t@H@@H@Z@4U3@A 01db0d18     ivp.obj
 0003:018c0d28       ??_B?1??Links@?$CUtlRBTree@UWaterTexInfo@@HP6A_NABU1@0@ZV?$CUtlMemory@U?$UtlRBTreeNode_t@UWaterTexInfo@@H@@H@@@@IBEABU?$UtlRBTreeLinks_t@H@@H@Z@51 01db0d28     ivp.obj
 0003:018c0d48       ?nummapbrushsides@@3HA     01db0d48     map.obj
 0003:018c0d4c       ?nummapbrushes@@3HA        01db0d4c     map.obj
 0003:018c0d50       ?planehash@@3PAPAUplane_t@@A 01db0d50     map.obj
 0003:018c1d50       ?c_edgebevels@@3HA         01db1d50     map.obj
 0003:018c1d54       ?c_areaportals@@3HA        01db1d54     map.obj
 0003:018c1d58       ?nummapplanes@@3HA         01db1d58     map.obj
 0003:018c1d5c       ?c_boxbevels@@3HA          01db1d5c     map.obj
 0003:018c1d60       ?c_clipbrushes@@3HA        01db1d60     map.obj
 0003:018c1d6c       ?map_mins@@3VVector@@A     01db1d6c     map.obj
 0003:018c1d78       ?map_maxs@@3VVector@@A     01db1d78     map.obj
 0003:018c1d84       ?g_NoDynamicShadowSides@@3V?$CUtlVector@HV?$CUtlMemory@HH@@@@A 01db1d84     map.obj
 0003:018c1d98       ?brushsides@@3PAUside_t@@A 01db1d98     map.obj
 0003:01f01d98       ?side_brushtextures@@3PAUbrush_texture_t@@A 023f1d98     map.obj
 0003:02a41d98       ?mapbrushes@@3PAUmapbrush_t@@A 02f31d98     map.obj
 0003:02aa1d98       ?mapplanes@@3PAUplane_t@@A 02f91d98     map.obj
 0003:02c21d98       ?id@?$codecvt@DDH@std@@2V0locale@2@A 03111d98     map.obj
 0003:02c21d9c       ?s_Sentinel@?1??Links@?$CUtlRBTree@UNameTranslationLookup_t@@HP6A_NABU1@0@ZV?$CUtlMemory@U?$UtlRBTreeNode_t@UNameTranslationLookup_t@@H@@H@@@@IBEABU?$UtlRBTreeLinks_t@H@@H@Z@4U3@A 03111d9c     materialpatch.obj
 0003:02c21dac       ??_B?1??Links@?$CUtlRBTree@UNameTranslationLookup_t@@HP6A_NABU1@0@ZV?$CUtlMemory@U?$UtlRBTreeNode_t@UNameTranslationLookup_t@@H@@H@@@@IBEABU?$UtlRBTreeLinks_t@H@@H@Z@51 03111dac     materialpatch.obj
 0003:02c21df0       ?g_ReplaceMaterials@@3_NA  03111df0     materialsub.obj
 0003:02c21e08       __crtBreakAlloc            03111e08     memoverride.obj
 0003:02c21e0c       ___crtDebugCheckCount      03111e0c     memoverride.obj
 0003:02c21e10       ___crtDebugFillThreshold   03111e10     memoverride.obj
 0003:02c21e30       ?draw_maxs@@3VVector@@A    03111e30     nodraw.obj
 0003:02c21e3c       ?draw_mins@@3VVector@@A    03111e3c     nodraw.obj
 0003:02c21e58       ?g_aMapOverlays@@3V?$CUtlVector@Umapoverlay_t@@V?$CUtlMemory@Umapoverlay_t@@H@@@@A 03111e58     overlay.obj
 0003:02c21e6c       ?g_aMapWaterOverlays@@3V?$CUtlVector@Umapoverlay_t@@V?$CUtlMemory@Umapoverlay_t@@H@@@@A 03111e6c     overlay.obj
 0003:02c21e9c       ?c_outside@@3HA            03111e9c     portals.obj
 0003:02c21ea0       ?c_boundary@@3HA           03111ea0     portals.obj
 0003:02c21ea4       ?c_peak_portals@@3HA       03111ea4     portals.obj
 0003:02c21ea8       ?c_solid@@3HA              03111ea8     portals.obj
 0003:02c21eac       ?c_boundary_sides@@3HA     03111eac     portals.obj
 0003:02c21eb0       ?c_tinyportals@@3HA        03111eb0     portals.obj
 0003:02c21eb4       ?c_inside@@3HA             03111eb4     portals.obj
 0003:02c21eb8       ?c_areas@@3HA              03111eb8     portals.obj
 0003:02c21ebc       ?c_active_portals@@3HA     03111ebc     portals.obj
 0003:02c21ee0       ?num_visclusters@@3HA      03111ee0     prtfile.obj
 0003:02c21ee4       ?num_visportals@@3HA       03111ee4     prtfile.obj
 0003:02c21ee8       ?clusterleaf@@3HA          03111ee8     prtfile.obj
 0003:02c21f2c       ?s_pPhysCollision@@3PAVIPhysicsCollision@@A 03111f2c     staticprop.obj
 0003:02c21f98       ?s_Sentinel@?1??Links@?$CUtlRBTree@UModelCollisionLookup_t@@GP6A_NABU1@0@ZV?$CUtlMemory@U?$UtlRBTreeNode_t@UModelCollisionLookup_t@@G@@G@@@@IBEABU?$UtlRBTreeLinks_t@G@@G@Z@4U3@A 03111f98     staticprop.obj
 0003:02c21fa0       ??_B?1??Links@?$CUtlRBTree@UModelCollisionLookup_t@@GP6A_NABU1@0@ZV?$CUtlMemory@U?$UtlRBTreeNode_t@UModelCollisionLookup_t@@G@@G@@@@IBEABU?$UtlRBTreeLinks_t@G@@G@Z@51 03111fa0     staticprop.obj
 0003:02c21fa8       ?nummiptex@@3HA            03111fa8     textures.obj
 0003:02c21fb0       ?g_SurfaceProperties@@3PAHA 03111fb0     textures.obj
 0003:02c23fb0       ?textureref@@3PAUtextureref_t@@A 03113fb0     textures.obj
 0003:02c46fb0       ?physprops@@3PAVIPhysicsSurfaceProps@@A 03136fb0     textures.obj
 0003:02c46fb4       ?g_bHasWater@@3_NA         03136fb4     textures.obj
 0003:02c46fd0       ?c_pruned@@3HA             03136fd0     tree.obj
 0003:02c46ff8       ?nocsg@@3HA                03136ff8     vbsp.obj
 0003:02c46ffc       ?nosubdiv@@3HA             03136ffc     vbsp.obj
 0003:02c47000       ?outbase@@3PADA            03137000     vbsp.obj
 0003:02c47020       ?mapbase@@3PADA            03137020     vbsp.obj
 0003:02c47060       ?fulldetail@@3HA           03137060     vbsp.obj
 0003:02c47064       ?onlyprops@@3_NA           03137064     vbsp.obj
 0003:02c47068       ?nowater@@3HA              03137068     vbsp.obj
 0003:02c4706c       ?brush_end@@3HA            0313706c     vbsp.obj
 0003:02c47070       ?block_nodes@@3PAY0CC@PAUnode_t@@A 03137070     vbsp.obj
 0003:02c48280       ?verboseentities@@3HA      03138280     vbsp.obj
 0003:02c48284       ?onlyents@@3HA             03138284     vbsp.obj
 0003:02c48288       ?noshare@@3HA              03138288     vbsp.obj
 0003:02c4828c       ?nodetail@@3HA             0313828c     vbsp.obj
 0003:02c48290       ?notjunc@@3HA              03138290     vbsp.obj
 0003:02c48294       ?noprune@@3HA              03138294     vbsp.obj
 0003:02c48298       ?noweld@@3HA               03138298     vbsp.obj
 0003:02c4829c       ?nomerge@@3HA              0313829c     vbsp.obj
 0003:02c482a0       ?glview@@3HA               031382a0     vbsp.obj
 0003:02c482a4       ?brush_start@@3HA          031382a4     vbsp.obj
 0003:02c482a8       ?name@@3PADA               031382a8     vbsp.obj
 0003:02c486a8       ?entity_num@@3HA           031386a8     vbsp.obj
 0003:02c486ac       ?noopt@@3HA                031386ac     vbsp.obj
 0003:02c486b0       ?source@@3PADA             031386b0     vbsp.obj
 0003:02c48ab0       ?leaktest@@3HA             03138ab0     vbsp.obj
 0003:02c48ab8       ?materialPath@@3PADA       03138ab8     vbsp.obj
 0003:02c48eb8       ?nomergewater@@3HA         03138eb8     vbsp.obj
 0003:02c48ebc       ?dumpcollide@@3HA          03138ebc     vbsp.obj
 0003:02c48ec0       ?g_bLowPriority@@3HA       03138ec0     vbsp.obj
 0003:02c48ec4       ?g_DumpStaticProps@@3HA    03138ec4     vbsp.obj
 0003:02c48ec8       ?g_bSkyVis@@3HA            03138ec8     vbsp.obj
 0003:02c48ecc       ?g_bLightIfMissing@@3_NA   03138ecc     vbsp.obj
 0003:02c48ecd       ?g_snapAxialPlanes@@3_NA   03138ecd     vbsp.obj
 0003:02c48ece       ?g_bKeepStaleZip@@3_NA     03138ece     vbsp.obj
 0003:02c48ecf       ?g_NodrawTriggers@@3_NA    03138ecf     vbsp.obj
 0003:02c48ed0       ?g_DisableWaterLighting@@3_NA 03138ed0     vbsp.obj
 0003:02c48ed1       ?g_bAllowDetailCracks@@3_NA 03138ed1     vbsp.obj
 0003:02c48ed2       ?g_bNoVirtualMesh@@3_NA    03138ed2     vbsp.obj
 0003:02c48ed3       ?g_BumpAll@@3_NA           03138ed3     vbsp.obj
 0003:02c48ed4       ?g_nDXLevel@@3HA           03138ed4     vbsp.obj
 0003:02c48ef0       ?g_SkyAreas@@3V?$CUtlVector@HV?$CUtlMemory@HH@@@@A 03138ef0     vbsp.obj
 0003:02c48f20       ?firstmodleaf@@3HA         03138f20     writebsp.obj
 0003:02c48f24       ?c_nofaces@@3HA            03138f24     writebsp.obj
 0003:02c48f28       ?pOrigFaceSideList@@3PAPAUside_t@@A 03138f28     writebsp.obj
 0003:02c88f28       ?c_facenodes@@3HA          03178f28     writebsp.obj
 0003:02c88f30       ?dfacenodes@@3PAPAUnode_t@@A 03178f30     writebsp.obj
 0003:02cc8f3c       ?s_Sentinel@?1??Links@?$CUtlRBTree@UNode_t@?$CUtlMap@PBDHH@@HVCKeyLess@2@V?$CUtlMemory@U?$UtlRBTreeNode_t@UNode_t@?$CUtlMap@PBDHH@@H@@H@@@@IBEABU?$UtlRBTreeLinks_t@H@@H@Z@4U3@A 031b8f3c     writebsp.obj
 0003:02cc8f4c       ??_B?1??Links@?$CUtlRBTree@UNode_t@?$CUtlMap@PBDHH@@HVCKeyLess@2@V?$CUtlMemory@U?$UtlRBTreeNode_t@UNode_t@?$CUtlMap@PBDHH@@H@@H@@@@IBEABU?$UtlRBTreeLinks_t@H@@H@Z@51 031b8f4c     writebsp.obj
 0003:02cc8f50       ?s_Sentinel@?1??Links@?$CUtlRBTree@VCZipEntry@CZipFile@@HP6A_NABV12@0@ZV?$CUtlMemory@U?$UtlRBTreeNode_t@VCZipEntry@CZipFile@@H@@H@@@@IBEABU?$UtlRBTreeLinks_t@H@@H@Z@4U3@A 031b8f50     zip_utils.obj
 0003:02cc8f60       ??_B?1??Links@?$CUtlRBTree@VCZipEntry@CZipFile@@HP6A_NABV12@0@ZV?$CUtlMemory@U?$UtlRBTreeNode_t@VCZipEntry@CZipFile@@H@@H@@@@IBEABU?$UtlRBTreeLinks_t@H@@H@Z@51 031b8f60     zip_utils.obj
 0003:02cc900c       ?g_DataMapHolder@ZIP_PreloadDirectoryEntry_DataDescInit@@3PAUdatamap_t@@A 031b900c     zip_utils.obj
 0003:02cc9010       ?g_DataMapHolder@ZIP_PreloadHeader_DataDescInit@@3PAUdatamap_t@@A 031b9010     zip_utils.obj
 0003:02cc9014       ?g_DataMapHolder@ZIP_FileHeader_DataDescInit@@3PAUdatamap_t@@A 031b9014     zip_utils.obj
 0003:02cc9018       ?g_DataMapHolder@ZIP_LocalFileHeader_DataDescInit@@3PAUdatamap_t@@A 031b9018     zip_utils.obj
 0003:02cc901c       ?g_DataMapHolder@ZIP_EndOfCentralDirRecord_DataDescInit@@3PAUdatamap_t@@A 031b901c     zip_utils.obj
 0003:02cc9020       ?numnodes@@3HA             031b9020     bsplib.obj
 0003:02cc9024       ?g_nClipPortalVerts@@3HA   031b9024     bsplib.obj
 0003:02cc9028       ?g_hBSPFile@@3PAXA         031b9028     bsplib.obj
 0003:02cc902c       ?numareaportals@@3HA       031b902c     bsplib.obj
 0003:02cc9030       ?numworldlightsLDR@@3HA    031b9030     bsplib.obj
 0003:02cc9034       ?visdatasize@@3HA          031b9034     bsplib.obj
 0003:02cc9038       ?dleafs@@3PAUdleaf_t@@A    031b9038     bsplib.obj
 0003:02ec9038       ?g_LeafMinDistToWater@@3PAGA 033b9038     bsplib.obj
 0003:02ee9038       ?g_CubemapSamples@@3PAUdcubemapsample_t@@A 033d9038     bsplib.obj
 0003:02eed038       ?dedges@@3PAUdedge_t@@A    033dd038     bsplib.obj
 0003:02fe7038       ?g_Lumps@@3U<unnamed-tag>@@A 034d7038     bsplib.obj
 0003:02fe7278       ?dorigfaces@@3PAUdface_t@@A 034d7278     bsplib.obj
 0003:03367278       ?dareaportals@@3PAUdareaportal_t@@A 03857278     bsplib.obj
 0003:0336a278       ?g_primitives@@3PAUdprimitive_t@@A 0385a278     bsplib.obj
 0003:033ba278       ?nummodels@@3HA            038aa278     bsplib.obj
 0003:033ba27c       ?g_pCompressFunc@@3P6A_NAAVCUtlBuffer@@0@ZA 038aa27c     bsplib.obj
 0003:033ba280       ?dleaffaces@@3PAGA         038aa280     bsplib.obj
 0003:033da280       ?dbrushsides@@3PAUdbrushside_t@@A 038ca280     bsplib.obj
 0003:0345a280       ?numsurfedges@@3HA         0394a280     bsplib.obj
 0003:0345a284       ?g_pBSPHeader@@3PAUdheader_t@@A 0394a284     bsplib.obj
 0003:0345a288       ?dleafwaterdata@@3PAUdleafwaterdata_t@@A 0394a288     bsplib.obj
 0003:034ba288       ?dfaces_hdr@@3PAUdface_t@@A 039aa288     bsplib.obj
 0003:0383a288       ?g_OverlayFades@@3PAUdoverlayfade_t@@A 03d2a288     bsplib.obj
 0003:0383b288       ?numleafbrushes@@3HA       03d2b288     bsplib.obj
 0003:0383b28c       ?g_nOverlayCount@@3HA      03d2b28c     bsplib.obj
 0003:0383b290       ?numplanes@@3HA            03d2b290     bsplib.obj
 0003:0383b294       ?g_numvertnormals@@3HA     03d2b294     bsplib.obj
 0003:0383b298       ?numleafs@@3HA             03d2b298     bsplib.obj
 0003:0383b29c       ?g_pVTFConvertFunc@@3P6A_NPBDAAVCUtlBuffer@@1P6A_N11@Z@ZA 03d2b29c     bsplib.obj
 0003:0383b2a0       ?dsurfedges@@3PAHA         03d2b2a0     bsplib.obj
 0003:03a2f2a0       ?g_numvertnormalindices@@3HA 03f1f2a0     bsplib.obj
 0003:03a2f2a4       ?numleaffaces@@3HA         03f1f2a4     bsplib.obj
 0003:03a2f2a8       ?dvisdata@@3PAEA           03f1f2a8     bsplib.obj
 0003:04a2f2a8       ?numareas@@3HA             04f1f2a8     bsplib.obj
 0003:04a2f2ac       ?numvertexes@@3HA          04f1f2ac     bsplib.obj
 0003:04a2f2b0       ?dfaces@@3PAUdface_t@@A    04f1f2b0     bsplib.obj
 0003:04daf2b0       ?g_pVHVFixupFunc@@3P6A_NPBD0AAVCUtlBuffer@@1@ZA 0529f2b0     bsplib.obj
 0003:04daf2b4       ?numorigfaces@@3HA         0529f2b4     bsplib.obj
 0003:04daf2b8       ?numedges@@3HA             0529f2b8     bsplib.obj
 0003:04daf2bc       ?numbrushes@@3HA           0529f2bc     bsplib.obj
 0003:04daf2c0       ?num_entities@@3HA         0529f2c0     bsplib.obj
 0003:04daf2c4       ?numfaces@@3HA             0529f2c4     bsplib.obj
 0003:04daf2c8       ?dleafbrushes@@3PAGA       0529f2c8     bsplib.obj
 0003:04dcf2c8       ?g_nWaterOverlayCount@@3HA 052bf2c8     bsplib.obj
 0003:04dcf2cc       ?numfaceids@@3HA           052bf2cc     bsplib.obj
 0003:04dcf2d0       ?dareas@@3PAUdarea_t@@A    052bf2d0     bsplib.obj
 0003:04dcfad0       ?dnodes@@3PAUdnode_t@@A    052bfad0     bsplib.obj
 0003:04fcfad0       ?numbrushsides@@3HA        054bfad0     bsplib.obj
 0003:04fcfad4       ?numworldlightsHDR@@3HA    054bfad4     bsplib.obj
 0003:04fcfad8       ?dbrushes@@3PAUdbrush_t@@A 054bfad8     bsplib.obj
 0003:04fe7ad8       ?numfaces_hdr@@3HA         054d7ad8     bsplib.obj
 0003:04fe7adc       ?numtexdata@@3HA           054d7adc     bsplib.obj
 0003:04fe7ae0       ?g_primindices@@3PAGA      054d7ae0     bsplib.obj
 0003:05007ae0       ?g_vertnormalindices@@3PAGA 054f7ae0     bsplib.obj
 0003:05084ae0       ?g_bHDR@@3_NA              05574ae0     bsplib.obj
 0003:05084ae4       ?g_LevelFlags@@3IA         05574ae4     bsplib.obj
 0003:05084ae8       ?g_pLeafAmbientIndex@@3PAV?$CUtlVector@Udleafambientindex_t@@V?$CUtlMemory@Udleafambientindex_t@@H@@@@A 05574ae8     bsplib.obj
 0003:05084aec       ?g_pLeafAmbientLighting@@3PAV?$CUtlVector@Udleafambientlighting_t@@V?$CUtlMemory@Udleafambientlighting_t@@H@@@@A 05574aec     bsplib.obj
 0003:05084af0       ?g_numprimitives@@3HA      05574af0     bsplib.obj
 0003:05084af4       ?g_numprimverts@@3HA       05574af4     bsplib.obj
 0003:05084af8       ?g_numprimindices@@3HA     05574af8     bsplib.obj
 0003:05084afc       ?numleafwaterdata@@3HA     05574afc     bsplib.obj
 0003:05084b00       ?g_nCubemapSamples@@3HA    05574b00     bsplib.obj
 0003:05084b04       ?g_pPhysCollide@@3PAEA     05574b04     bsplib.obj
 0003:05084b08       ?g_PhysCollideSize@@3HA    05574b08     bsplib.obj
 0003:05084b0c       ?g_MapRevision@@3HA        05574b0c     bsplib.obj
 0003:05084b10       ?g_pPhysDisp@@3PAEA        05574b10     bsplib.obj
 0003:05084b14       ?g_PhysDispSize@@3HA       05574b14     bsplib.obj
 0003:05084b34       ?g_DataMapHolder@CompressedLightCube_DataDescInit@@3PAUdatamap_t@@A 05574b34     bsplib.obj
 0003:05084b38       ?g_DataMapHolder@CDispCornerNeighbors_DataDescInit@@3PAUdatamap_t@@A 05574b38     bsplib.obj
 0003:05084b3c       ?g_DataMapHolder@dbrush_t_DataDescInit@@3PAUdatamap_t@@A 05574b3c     bsplib.obj
 0003:05084b40       ?g_DataMapHolder@dgamelumpheader_t_DataDescInit@@3PAUdatamap_t@@A 05574b40     bsplib.obj
 0003:05084b44       ?g_DataMapHolder@StaticPropLumpV4_t_DataDescInit@@3PAUdatamap_t@@A 05574b44     bsplib.obj
 0003:05084b48       ?g_DataMapHolder@doverlay_t_DataDescInit@@3PAUdatamap_t@@A 05574b48     bsplib.obj
 0003:05084b4c       ?g_DataMapHolder@dareaportal_t_DataDescInit@@3PAUdatamap_t@@A 05574b4c     bsplib.obj
 0003:05084b50       ?g_DataMapHolder@dleafambientlighting_t_DataDescInit@@3PAUdatamap_t@@A 05574b50     bsplib.obj
 0003:05084b54       ?g_DataMapHolder@StaticPropDictLump_t_DataDescInit@@3PAUdatamap_t@@A 05574b54     bsplib.obj
 0003:05084b58       ?g_vertnormals@@3PAVVector@@A 05574b58     bsplib.obj
 0003:05372b58       ?g_DataMapHolder@dleafwaterdata_t_DataDescInit@@3PAUdatamap_t@@A 05862b58     bsplib.obj
 0003:05372b5c       ?g_DataMapHolder@dnode_t_DataDescInit@@3PAUdatamap_t@@A 05862b5c     bsplib.obj
 0003:05372b60       ?g_DataMapHolder@dflagslump_t_DataDescInit@@3PAUdatamap_t@@A 05862b60     bsplib.obj
 0003:05372b64       ?g_DataMapHolder@dmodel_t_DataDescInit@@3PAUdatamap_t@@A 05862b64     bsplib.obj
 0003:05372b68       ?dworldlightsHDR@@3PAUdworldlight_t@@A 05862b68     bsplib.obj
 0003:05422b68       ?g_LeafAmbientLightingHDR@@3V?$CUtlVector@Udleafambientlighting_t@@V?$CUtlMemory@Udleafambientlighting_t@@H@@@@A 05912b68     bsplib.obj
 0003:05422b7c       ?g_DataMapHolder@CFaceMacroTextureInfo_DataDescInit@@3PAUdatamap_t@@A 05912b7c     bsplib.obj
 0003:05422b80       ?dtexdata@@3PAUdtexdata_t@@A 05912b80     bsplib.obj
 0003:05432b80       ?g_DataMapHolder@dphysdisp_t_DataDescInit@@3PAUdatamap_t@@A 05922b80     bsplib.obj
 0003:05432b84       ?g_DataMapHolder@DetailObjectLump_t_DataDescInit@@3PAUdatamap_t@@A 05922b84     bsplib.obj
 0003:05432b88       ?g_DataMapHolder@dleaf_version_0_t_DataDescInit@@3PAUdatamap_t@@A 05922b88     bsplib.obj
 0003:05432b8c       ?g_DataMapHolder@dvertex_t_DataDescInit@@3PAUdatamap_t@@A 05922b8c     bsplib.obj
 0003:05432b90       ?g_DataMapHolder@dworldlight_t_DataDescInit@@3PAUdatamap_t@@A 05922b90     bsplib.obj
 0003:05432b94       ?g_DataMapHolder@dprimvert_t_DataDescInit@@3PAUdatamap_t@@A 05922b94     bsplib.obj
 0003:05432b98       ?g_Overlays@@3PAUdoverlay_t@@A 05922b98     bsplib.obj
 0003:0545eb98       ?g_DispLightmapSamplePositions@@3V?$CUtlVector@EV?$CUtlMemory@EH@@@@A 0594eb98     bsplib.obj
 0003:0545ebac       ?g_DataMapHolder@dwateroverlay_t_DataDescInit@@3PAUdatamap_t@@A 0594ebac     bsplib.obj
 0003:0545ebb0       ?g_DataMapHolder@swapcompactsurfaceheader_t_DataDescInit@@3PAUdatamap_t@@A 0594ebb0     bsplib.obj
 0003:0545ebb4       ?g_StaticPropNames@@3V?$CUtlVector@VCUtlString@@V?$CUtlMemory@VCUtlString@@H@@@@A 0594ebb4     bsplib.obj
 0003:0545ebc8       ?dlightdataLDR@@3V?$CUtlVector@EV?$CUtlMemory@EH@@@@A 0594ebc8     bsplib.obj
 0003:0545ebdc       ?g_LeafAmbientIndexHDR@@3V?$CUtlVector@Udleafambientindex_t@@V?$CUtlMemory@Udleafambientindex_t@@H@@@@A 0594ebdc     bsplib.obj
 0003:0545ebf0       ?g_DataMapHolder@ddispinfo_t_DataDescInit@@3PAUdatamap_t@@A 0594ebf0     bsplib.obj
 0003:0545ebf4       ?g_DataMapHolder@dgamelump_t_DataDescInit@@3PAUdatamap_t@@A 0594ebf4     bsplib.obj
 0003:0545ebf8       ?g_DataMapHolder@DetailSpriteDictLump_t_DataDescInit@@3PAUdatamap_t@@A 0594ebf8     bsplib.obj
 0003:0545ebfc       ?g_DataMapHolder@dheader_t_DataDescInit@@3PAUdatamap_t@@A 0594ebfc     bsplib.obj
 0003:0545ec00       ?g_DataMapHolder@swapcollideheader_t_DataDescInit@@3PAUdatamap_t@@A 0594ec00     bsplib.obj
 0003:0545ec04       ?g_LeafAmbientLightingLDR@@3V?$CUtlVector@Udleafambientlighting_t@@V?$CUtlMemory@Udleafambientlighting_t@@H@@@@A 0594ec04     bsplib.obj
 0003:0545ec18       ?g_DataMapHolder@CDispTri_DataDescInit@@3PAUdatamap_t@@A 0594ec18     bsplib.obj
 0003:0545ec1c       ?g_DataMapHolder@dtexdata_t_DataDescInit@@3PAUdatamap_t@@A 0594ec1c     bsplib.obj
 0003:0545ec20       ?g_DataMapHolder@swapmoppsurfaceheader_t_DataDescInit@@3PAUdatamap_t@@A 0594ec20     bsplib.obj
 0003:0545ec24       ?g_ClusterLeaves@@3V?$CUtlVector@Uclusterlist_t@@V?$CUtlMemory@Uclusterlist_t@@H@@@@A 0594ec24     bsplib.obj
 0003:0545ec38       ?g_DataMapHolder@dcubemapsample_t_DataDescInit@@3PAUdatamap_t@@A 0594ec38     bsplib.obj
 0003:0545ec3c       ?g_dispinfo@@3V?$CUtlVector@Vddispinfo_t@@V?$CUtlMemory@Vddispinfo_t@@H@@@@A 0594ec3c     bsplib.obj
 0003:0545ec50       ?entities@@3PAUentity_t@@A 0594ec50     bsplib.obj
 0003:054b6c50       ?g_TexDataStringData@@3V?$CUtlVector@DV?$CUtlMemory@DH@@@@A 059a6c50     bsplib.obj
 0003:054b6c64       ?g_DataMapHolder@dphysmodel_t_DataDescInit@@3PAUdatamap_t@@A 059a6c64     bsplib.obj
 0003:054b6c68       ?dentdata@@3V?$CUtlVector@DV?$CUtlMemory@DH@@@@A 059a6c68     bsplib.obj
 0003:054b6c7c       ?g_DataMapHolder@CDispVert_DataDescInit@@3PAUdatamap_t@@A 059a6c7c     bsplib.obj
 0003:054b6c80       ?g_DataMapHolder@darea_t_DataDescInit@@3PAUdatamap_t@@A 059a6c80     bsplib.obj
 0003:054b6c84       ?g_DataMapHolder@MeshHeader_t_DataDescInit@HardwareVerts@@3PAUdatamap_t@@A 059a6c84     bsplib.obj
 0003:054b6c88       ?g_DataMapHolder@FileHeader_t_DataDescInit@HardwareVerts@@3PAUdatamap_t@@A 059a6c88     bsplib.obj
 0003:054b6c8c       ?g_TexDataStringTable@@3V?$CUtlVector@HV?$CUtlMemory@HH@@@@A 059a6c8c     bsplib.obj
 0003:054b6ca0       ?g_ClipPortalVerts@@3PAVVector@@A 059a6ca0     bsplib.obj
 0003:0562dca0       ?g_DataMapHolder@dleaf_t_DataDescInit@@3PAUdatamap_t@@A 05b1dca0     bsplib.obj
 0003:0562dca4       ?g_DataMapHolder@lump_t_DataDescInit@@3PAUdatamap_t@@A 05b1dca4     bsplib.obj
 0003:0562dca8       ?g_DataMapHolder@dedge_t_DataDescInit@@3PAUdatamap_t@@A 05b1dca8     bsplib.obj
 0003:0562dcac       ?g_DataMapHolder@doccluderpolydata_t_DataDescInit@@3PAUdatamap_t@@A 05b1dcac     bsplib.obj
 0003:0562dcb0       ?g_DataMapHolder@DetailObjectDictLump_t_DataDescInit@@3PAUdatamap_t@@A 05b1dcb0     bsplib.obj
 0003:0562dcb4       ?g_DataMapHolder@dleafambientindex_t_DataDescInit@@3PAUdatamap_t@@A 05b1dcb4     bsplib.obj
 0003:0562dcb8       ?g_DataMapHolder@StaticPropLump_t_DataDescInit@@3PAUdatamap_t@@A 05b1dcb8     bsplib.obj
 0003:0562dcbc       ?g_DataMapHolder@CDispSubNeighbor_DataDescInit@@3PAUdatamap_t@@A 05b1dcbc     bsplib.obj
 0003:0562dcc0       ?g_DataMapHolder@DetailPropLightstylesLump_t_DataDescInit@@3PAUdatamap_t@@A 05b1dcc0     bsplib.obj
 0003:0562dcc4       ?g_DispVerts@@3V?$CUtlVector@VCDispVert@@V?$CUtlMemory@VCDispVert@@H@@@@A 05b1dcc4     bsplib.obj
 0003:0562dcd8       ?g_primverts@@3PAUdprimvert_t@@A 05b1dcd8     bsplib.obj
 0003:056edcd8       ?g_DataMapHolder@dfaceid_t_DataDescInit@@3PAUdatamap_t@@A 05bddcd8     bsplib.obj
 0003:056edcdc       ?g_StaticPropInstances@@3V?$CUtlVector@HV?$CUtlMemory@HH@@@@A 05bddcdc     bsplib.obj
 0003:056edcf0       ?g_DataMapHolder@StaticPropLumpV5_t_DataDescInit@@3PAUdatamap_t@@A 05bddcf0     bsplib.obj
 0003:056edcf4       ?g_DataMapHolder@CDispNeighbor_DataDescInit@@3PAUdatamap_t@@A 05bddcf4     bsplib.obj
 0003:056edcf8       ?dplanes@@3PAUdplane_t@@A  05bddcf8     bsplib.obj
 0003:0582dcf8       ?g_FaceMacroTextureInfos@@3V?$CUtlVector@VCFaceMacroTextureInfo@@V?$CUtlMemory@VCFaceMacroTextureInfo@@H@@@@A 05d1dcf8     bsplib.obj
 0003:0582dd0c       ?g_DataMapHolder@dbrushside_t_DataDescInit@@3PAUdatamap_t@@A 05d1dd0c     bsplib.obj
 0003:0582dd10       ?g_DataMapHolder@doverlayfade_t_DataDescInit@@3PAUdatamap_t@@A 05d1dd10     bsplib.obj
 0003:0582dd14       ?g_DataMapHolder@texinfo_t_DataDescInit@@3PAUdatamap_t@@A 05d1dd14     bsplib.obj
 0003:0582dd18       ?g_DataMapHolder@StaticPropLeafLump_t_DataDescInit@@3PAUdatamap_t@@A 05d1dd18     bsplib.obj
 0003:0582dd1c       ?dfaceids@@3V?$CUtlVector@Udfaceid_t@@V?$CUtlMemory@Udfaceid_t@@H@@@@A 05d1dd1c     bsplib.obj
 0003:0582dd30       ?dworldlightsLDR@@3PAUdworldlight_t@@A 05d1dd30     bsplib.obj
 0003:058ddd30       ?g_DataMapHolder@dprimitive_t_DataDescInit@@3PAUdatamap_t@@A 05dcdd30     bsplib.obj
 0003:058ddd34       ?g_DataMapHolder@dplane_t_DataDescInit@@3PAUdatamap_t@@A 05dcdd34     bsplib.obj
 0003:058ddd38       ?g_LeafAmbientIndexLDR@@3V?$CUtlVector@Udleafambientindex_t@@V?$CUtlMemory@Udleafambientindex_t@@H@@@@A 05dcdd38     bsplib.obj
 0003:058ddd4c       ?g_DispTris@@3V?$CUtlVector@VCDispTri@@V?$CUtlMemory@VCDispTri@@H@@@@A 05dcdd4c     bsplib.obj
 0003:058ddd60       ?g_WaterOverlays@@3PAUdwateroverlay_t@@A 05dcdd60     bsplib.obj
 0003:06a5dd60       ?dmodels@@3PAUdmodel_t@@A  06f4dd60     bsplib.obj
 0003:06a69d60       ?g_Swap@@3VCByteswap@@A    06f59d60     bsplib.obj
 0003:06a69d64       ?g_DataMapHolder@dface_t_DataDescInit@@3PAUdatamap_t@@A 06f59d64     bsplib.obj
 0003:06a69d68       ?dlightdataHDR@@3V?$CUtlVector@EV?$CUtlMemory@EH@@@@A 06f59d68     bsplib.obj
 0003:06a69d7c       ?g_DataMapHolder@doccluderdata_t_DataDescInit@@3PAUdatamap_t@@A 06f59d7c     bsplib.obj
 0003:06a69d80       ?dvertexes@@3PAUdvertex_t@@A 06f59d80     bsplib.obj
 0003:06b2a888       ?_Stinit@?1??_Init@?$basic_filebuf@DU?$char_traits@D@std@@@std@@IAEXPAU_iobuf@@W4_Initfl@23@@Z@4HA 0701a888     chunkfile.obj
 0003:06b2a88c       ?_Psave@?$_Facetptr@V?$codecvt@DDH@std@@@std@@2PBVfacet@locale@2@B 0701a88c     chunkfile.obj
 0003:06b2a8a8       ?ex_argv@@3PAPADA          0701a8a8     cmdlib.obj
 0003:06b2b8a8       ?g_SpewCS@@3U_RTL_CRITICAL_SECTION@@A 0701b8a8     cmdlib.obj
 0003:06b2b8c0       ?com_token@@3PADA          0701b8c0     cmdlib.obj
 0003:06b2bcc0       ?archivedir@@3PADA         0701bcc0     cmdlib.obj
 0003:06b2c0c0       ?myargc@@3HA               0701c0c0     cmdlib.obj
 0003:06b2c0c4       ?ex_argc@@3HA              0701c0c4     cmdlib.obj
 0003:06b2caf0       ?myargv@@3PAPADA           0701caf0     cmdlib.obj
 0003:06b2caf4       ?archive@@3HA              0701caf4     cmdlib.obj
 0003:06b2caf8       ?g_pLogFile@@3PAXA         0701caf8     cmdlib.obj
 0003:06b2cafc       ?g_bStopOnExit@@3_NA       0701cafc     cmdlib.obj
 0003:06b2cafd       ?g_bSpewCSInitted@@3_NA    0701cafd     cmdlib.obj
 0003:06b2cafe       ?g_bSuppressPrintfOutput@@3_NA 0701cafe     cmdlib.obj
 0003:06b2cb00       ?g_ExtraSpewHook@@3P6AXPBD@ZA 0701cb00     cmdlib.obj
 0003:06b2cb04       ?verbose@@3HA              0701cb04     cmdlib.obj
 0003:06b2cb14       ?g_ExitStopper@@3VCExitStopper@@A 0701cb14     cmdlib.obj
 0003:06b2d248       ?qdir@@3PADA               0701d248     filesystem_tools.obj
 0003:06b2d648       ?gamedir@@3PADA            0701d648     filesystem_tools.obj
 0003:06b2da48       ?g_pFileSystem@@3PAVIBaseFileSystem@@A 0701da48     filesystem_tools.obj
 0003:06b2da4c       ?g_pFullFileSystemModule@@3PAVCSysModule@@A 0701da4c     filesystem_tools.obj
 0003:06b2da58       ?g_MapError@@3VCMapError@@A 0701da58     map_shared.obj
 0003:06b2dab0       ?g_nMapFileVersion@@3HA    0701dab0     map_shared.obj
 0003:06b2dac0       ?c_active_windings@@3HA    0701dac0     polylib.obj
 0003:06b2dac4       ?c_removed@@3HA            0701dac4     polylib.obj
 0003:06b2dac8       ?c_peak_windings@@3HA      0701dac8     polylib.obj
 0003:06b2dacc       ?c_winding_allocs@@3HA     0701dacc     polylib.obj
 0003:06b2dad0       ?winding_pool@@3PAPAUwinding_t@@A 0701dad0     polylib.obj
 0003:06b2dbe0       ?c_winding_points@@3HA     0701dbe0     polylib.obj
 0003:06b2dbf0       ?macrolist@@3PAPAUscript_t@@A 0701dbf0     scriplib.obj
 0003:06b2dcf0       ?script@@3PAUscript_t@@A   0701dcf0     scriplib.obj
 0003:06b2dcf4       ?nummacros@@3HA            0701dcf4     scriplib.obj
 0003:06b2dcf8       ?scriptstack@@3PAUscript_t@@A 0701dcf8     scriplib.obj
 0003:06b43e38       ?token@@3PADA              07033e38     scriplib.obj
 0003:06b44238       ?scriptline@@3HA           07034238     scriplib.obj
 0003:06b4423c       ?endofscript@@3HA          0703423c     scriplib.obj
 0003:06b44240       ?tokenready@@3HA           07034240     scriplib.obj
 0003:06b4424c       ?g_definevariable@@3V?$CUtlVector@Uvariable_t@@V?$CUtlMemory@Uvariable_t@@H@@@@A 0703424c     scriplib.obj
 0003:06b44260       ?pacifier@@3HA             07034260     threads.obj
 0003:06b44264       ?crit@@3U_RTL_CRITICAL_SECTION@@A 07034264     threads.obj
 0003:06b4427c       ?workcount@@3HA            0703427c     threads.obj
 0003:06b44280       ?g_RunThreadsData@@3PAVCRunThreadsData@@A 07034280     threads.obj
 0003:06b44340       ?workfunction@@3P6AXHH@ZA  07034340     threads.obj
 0003:06b44344       ?dispatch@@3HA             07034344     threads.obj
 0003:06b44348       ?g_ThreadHandles@@3PAPAXA  07034348     threads.obj
 0003:06b44388       ?threaded@@3HA             07034388     threads.obj
 0003:06b44390       ?g_bLowPriorityThreads@@3_NA 07034390     threads.obj
 0003:06b4439c       ?g_CritInit@@3VCCritInit@@A 0703439c     threads.obj
 0003:06b443b8       ?s_StringCharConversion@@3VCUtlCStringConversion@@A 070343b8     tier1:utlbuffer.obj
 0003:06b44dc8       ?s_NoEscConversion@@3VCUtlNoEscConversion@@A 07034dc8     tier1:utlbuffer.obj
 0003:06b456d8       ?s_pSymbolTable@CUtlSymbol@@1PAVCUtlSymbolTableMT@@A 070356d8     tier1:utlsymbol.obj
 0003:06b456e8       ?s_Sentinel@?1??Links@?$CUtlRBTree@VCStringPoolIndex@CUtlSymbolTable@@GVCLess@2@V?$CUtlMemory@U?$UtlRBTreeNode_t@VCStringPoolIndex@CUtlSymbolTable@@G@@G@@@@IBEABU?$UtlRBTreeLinks_t@G@@G@Z@4U3@A 070356e8     tier1:utlsymbol.obj
 0003:06b456f0       ??_B?1??Links@?$CUtlRBTree@VCStringPoolIndex@CUtlSymbolTable@@GVCLess@2@V?$CUtlMemory@U?$UtlRBTreeNode_t@VCStringPoolIndex@CUtlSymbolTable@@G@@G@@@@IBEABU?$UtlRBTreeLinks_t@G@@G@Z@51 070356f0     tier1:utlsymbol.obj
 0003:06b45f08       ?s_pInterfaceRegs@InterfaceReg@@2PAV1@A 07035f08     tier1:interface.obj
 0003:06b46010       ?_Psave@?$_Facetptr@V?$ctype@D@std@@@std@@2PBVfacet@locale@2@B 07036010     tier1:tokenreader.obj
 0003:06b46020       ?SinCosTable@@3PAMA        07036020     mathlib:mathlib_base.obj
 0003:06b46420       ?s_bMathlibInitialized@@3_NA 07036420     mathlib:mathlib_base.obj
 0003:06b46430       ?vec3_origin@@3VVector@@B  07036430     mathlib:mathlib_base.obj
 0003:06b4643c       ?vec3_angle@@3VQAngle@@B   0703643c     mathlib:mathlib_base.obj
 0003:06b46868       ?lineartolightmap@@3PAEA   07036868     mathlib:color_conversion.obj
 0003:06b4a068       ?lineartovertex@@3PAMA     0703a068     mathlib:color_conversion.obj
 0003:06b4e180       ?g_pFullFileSystem@@3PAVIFileSystem@@A 0703e180     tier2:tier2.obj
 0003:06b4e184       ?materials@@3PAVIMaterialSystem@@A 0703e184     tier2:tier2.obj
 0003:06b4e188       ?g_pMaterialSystem@@3PAVIMaterialSystem@@A 0703e188     tier2:tier2.obj
 0003:06b4e18c       ?g_pInputSystem@@3PAVIInputSystem@@A 0703e18c     tier2:tier2.obj
 0003:06b4e190       ?g_pNetworkSystem@@3PAVINetworkSystem@@A 0703e190     tier2:tier2.obj
 0003:06b4e194       ?g_pMaterialSystemHardwareConfig@@3PAVIMaterialSystemHardwareConfig@@A 0703e194     tier2:tier2.obj
 0003:06b4e198       ?g_pMaterialSystemDebugTextureInfo@@3PAVIDebugTextureInfo@@A 0703e198     tier2:tier2.obj
 0003:06b4e19c       ?g_VBAllocTracker@@3PAVIVBAllocTracker@@A 0703e19c     tier2:tier2.obj
 0003:06b4e1a0       ?colorcorrection@@3PAVIColorCorrectionSystem@@A 0703e1a0     tier2:tier2.obj
 0003:06b4e1a4       ?p4@@3PAVIP4@@A            0703e1a4     tier2:tier2.obj
 0003:06b4e1a8       ?mdllib@@3PAVIMdlLib@@A    0703e1a8     tier2:tier2.obj
 0003:06b4e1ac       ?g_pQueuedLoader@@3PAVIQueuedLoader@@A 0703e1ac     tier2:tier2.obj
 0003:06b4e2c4       ?g_DataMapHolder@VTFFileHeaderV7_3_t_DataDescInit@@3PAUdatamap_t@@A 0703e2c4     vtf:vtf.obj
 0003:06b4e2c8       ?g_DataMapHolder@VTFFileHeaderV7_1_t_DataDescInit@@3PAUdatamap_t@@A 0703e2c8     vtf:vtf.obj
 0003:06b4e2cc       ?g_DataMapHolder@VTFFileBaseHeader_t_DataDescInit@@3PAUdatamap_t@@A 0703e2cc     vtf:vtf.obj
 0003:06b4e2d0       ?g_DataMapHolder@VTFFileHeaderV7_2_t_DataDescInit@@3PAUdatamap_t@@A 0703e2d0     vtf:vtf.obj
 0003:06b4e2d4       ?g_DataMapHolder@VTFFileHeader_t_DataDescInit@@3PAUdatamap_t@@A 0703e2d4     vtf:vtf.obj
 0003:06b4e2d8       ?g_DataMapHolder@VTFFileHeaderX360_t_DataDescInit@@3PAUdatamap_t@@A 0703e2d8     vtf:vtf.obj
 0003:06b4e2e4       ___fastflag                0703e2e4     LIBCMT:fpinit.obj
 0003:06b4e2e8       __adjust_fdiv              0703e2e8     LIBCMT:fpinit.obj
 0003:06b4e2f0       ___pInvalidArgHandler      0703e2f0     LIBCMT:invarg.obj
 0003:06b4e2f4       __umaskval                 0703e2f4     LIBCMT:crt0dat.obj
 0003:06b4e2f8       __osplatform               0703e2f8     LIBCMT:crt0dat.obj
 0003:06b4e2fc       __osver                    0703e2fc     LIBCMT:crt0dat.obj
 0003:06b4e300       __winver                   0703e300     LIBCMT:crt0dat.obj
 0003:06b4e304       __winmajor                 0703e304     LIBCMT:crt0dat.obj
 0003:06b4e308       __winminor                 0703e308     LIBCMT:crt0dat.obj
 0003:06b4e30c       ___argc                    0703e30c     LIBCMT:crt0dat.obj
 0003:06b4e310       ___argv                    0703e310     LIBCMT:crt0dat.obj
 0003:06b4e314       ___wargv                   0703e314     LIBCMT:crt0dat.obj
 0003:06b4e318       __environ                  0703e318     LIBCMT:crt0dat.obj
 0003:06b4e31c       ___initenv                 0703e31c     LIBCMT:crt0dat.obj
 0003:06b4e320       __wenviron                 0703e320     LIBCMT:crt0dat.obj
 0003:06b4e324       ___winitenv                0703e324     LIBCMT:crt0dat.obj
 0003:06b4e328       __pgmptr                   0703e328     LIBCMT:crt0dat.obj
 0003:06b4e32c       __wpgmptr                  0703e32c     LIBCMT:crt0dat.obj
 0003:06b4e330       __exitflag                 0703e330     LIBCMT:crt0dat.obj
 0003:06b4e334       __C_Termination_Done       0703e334     LIBCMT:crt0dat.obj
 0003:06b4e338       __C_Exit_Done              0703e338     LIBCMT:crt0dat.obj
 0003:06b4e374       __cflush                   0703e374     LIBCMT:_file.obj
 0003:06b4e378       ?_pnhHeap@@3P6AHI@ZA       0703e378     LIBCMT:handler.obj
 0003:06b4e37c       __aenvptr                  0703e37c     LIBCMT:crt0.obj
 0003:06b4e380       __wenvptr                  0703e380     LIBCMT:crt0.obj
 0003:06b4e384       ___error_mode              0703e384     LIBCMT:crt0.obj
 0003:06b4e388       __stdbuf                   0703e388     LIBCMT:_sftbuf.obj
 0003:06b4e390       _gpFlsAlloc                0703e390     LIBCMT:tidtable.obj
 0003:06b4e394       _gpFlsGetValue             0703e394     LIBCMT:tidtable.obj
 0003:06b4e398       _gpFlsSetValue             0703e398     LIBCMT:tidtable.obj
 0003:06b4e39c       _gpFlsFree                 0703e39c     LIBCMT:tidtable.obj
 0003:06b4e6c4       ___pPurecall               0703e6c4     LIBCMT:inithelp.obj
 0003:06b4e6cc       ___mbulinfo                0703e6cc     LIBCMT:mbctype.obj
 0003:06b4e6d8       ___mbcodepage              0703e6d8     LIBCMT:mbctype.obj
 0003:06b4e6dc       ___ismbcodepage            0703e6dc     LIBCMT:mbctype.obj
 0003:06b4e6e0       ___mblcid                  0703e6e0     LIBCMT:mbctype.obj
 0003:06b4e6e4       ___locale_changed          0703e6e4     LIBCMT:setlocal.obj
 0003:06b4e6e8       ___lc_handle               0703e6e8     LIBCMT:nlsdata2.obj
 0003:06b4e700       ___lc_codepage             0703e700     LIBCMT:nlsdata2.obj
 0003:06b4e704       ___lc_collate_cp           0703e704     LIBCMT:nlsdata2.obj
 0003:06b4e70c       ?__pInconsistency@@3P6AXXZA 0703e70c     LIBCMT:hooks.obj
 0003:06b4e884       __old_pfxlen               0703e884     LIBCMT:rmtmp.obj
 0003:06b4e888       __commode                  0703e888     LIBCMT:ncommode.obj
 0003:06b4e88c       __newmode                  0703e88c     LIBCMT:_newmode.obj
 0003:06b4e99c       __outputformat             0703e99c     LIBCMT:outputformat.obj
 0003:06b4ecd8       ?pArgList@UnDecorator@@0PAVReplicator@@A 0703ecd8     LIBCMT:undname.obj
 0003:06b4ecdc       ?pZNameList@UnDecorator@@0PAVReplicator@@A 0703ecdc     LIBCMT:undname.obj
 0003:06b4ece0       ?pTemplateArgList@UnDecorator@@0PAVReplicator@@A 0703ece0     LIBCMT:undname.obj
 0003:06b4ece4       ?gName@UnDecorator@@0PBDB  0703ece4     LIBCMT:undname.obj
 0003:06b4ece8       ?name@UnDecorator@@0PBDB   0703ece8     LIBCMT:undname.obj
 0003:06b4ecec       ?outputString@UnDecorator@@0PADA 0703ecec     LIBCMT:undname.obj
 0003:06b4ecf0       ?maxStringLength@UnDecorator@@0HA 0703ecf0     LIBCMT:undname.obj
 0003:06b4ecf4       ?disableFlags@UnDecorator@@0KA 0703ecf4     LIBCMT:undname.obj
 0003:06b4ecf8       ?m_pGetParameter@UnDecorator@@0P6APADJ@ZA 0703ecf8     LIBCMT:undname.obj
 0003:06b4ecfc       ?fExplicitTemplateParams@UnDecorator@@0_NA 0703ecfc     LIBCMT:undname.obj
 0003:06b4ecfd       ?fGetTemplateArgumentList@UnDecorator@@0_NA 0703ecfd     LIBCMT:undname.obj
 0003:06b4ed20       ___lconv_static_null       0703ed20     LIBCMT:lconv.obj
 0003:06b4edec       __fmode                    0703edec     LIBCMT:txtmode.obj
 0003:06b4ee60       ?_Fpz@std@@3_JA            0703ee60     libcpmt:ios.obj
 0003:06b4ee68       ?_Index@ios_base@std@@0HA  0703ee68     libcpmt:ios.obj
 0003:06b4eea8       ?_Clocptr@_Locimp@locale@std@@0PAV123@A 0703eea8     libcpmt:locale0.obj
 0003:06b4eeac       ?_Id_cnt@id@locale@std@@0HA 0703eeac     libcpmt:locale0.obj
 0003:06b4eeb0       ?id@?$ctype@D@std@@2V0locale@2@A 0703eeb0     libcpmt:locale0.obj
 0003:06b4eeb4       ?id@?$codecvt@GDH@std@@2V0locale@2@A 0703eeb4     libcpmt:locale0.obj
 0003:06b4eeb8       ?id@?$ctype@_W@std@@2V0locale@2@A 0703eeb8     libcpmt:locale0.obj
 0003:06b4eebc       ?id@?$codecvt@_WDH@std@@2V0locale@2@A 0703eebc     libcpmt:locale0.obj
 0003:06b4eec4       ?id@?$ctype@G@std@@2V0locale@2@A 0703eec4     libcpmt:locale0.obj
 0003:06b4eecc       ?_Ptr_cin@std@@3PAV?$basic_istream@DU?$char_traits@D@std@@@1@A 0703eecc     libcpmt:iosptrs.obj
 0003:06b4eed0       ?_Ptr_cout@std@@3PAV?$basic_ostream@DU?$char_traits@D@std@@@1@A 0703eed0     libcpmt:iosptrs.obj
 0003:06b4eed4       ?_Ptr_cerr@std@@3PAV?$basic_ostream@DU?$char_traits@D@std@@@1@A 0703eed4     libcpmt:iosptrs.obj
 0003:06b4eed8       ?_Ptr_clog@std@@3PAV?$basic_ostream@DU?$char_traits@D@std@@@1@A 0703eed8     libcpmt:iosptrs.obj
 0003:06b4eedc       ?_Ptr_wcin@std@@3PAV?$basic_istream@_WU?$char_traits@_W@std@@@1@A 0703eedc     libcpmt:iosptrs.obj
 0003:06b4eee0       ?_Ptr_wcout@std@@3PAV?$basic_ostream@_WU?$char_traits@_W@std@@@1@A 0703eee0     libcpmt:iosptrs.obj
 0003:06b4eee4       ?_Ptr_wcerr@std@@3PAV?$basic_ostream@_WU?$char_traits@_W@std@@@1@A 0703eee4     libcpmt:iosptrs.obj
 0003:06b4eee8       ?_Ptr_wclog@std@@3PAV?$basic_ostream@_WU?$char_traits@_W@std@@@1@A 0703eee8     libcpmt:iosptrs.obj
 0003:06b4f608       ?bS3TCForce4@@3_NA         0703f608     bitmap:S3_intrf.obj
 0003:06b58e9c       __debugger_hook_dummy      07048e9c     <common>
 0003:06b58ea0       __pmatherr                 07048ea0     <common>
 0003:06b58ea4       __nhandle                  07048ea4     <common>
 0003:06b58ec0       ___pioinfo                 07048ec0     <common>
 0003:06b58fc0       ___use_sse2_mathfcns       07048fc0     <common>
 0003:06b58fc4       ___sse2_available          07048fc4     <common>
 0003:06b58fc8       __acmdln                   07048fc8     <common>
 0003:06b58fcc       ___piob                    07048fcc     <common>
 0003:06b58fe0       __bufin                    07048fe0     <common>
 0003:06b59fe0       __nstream                  07049fe0     <common>
 0003:06b59fe4       ___env_initialized         07049fe4     <common>
 0003:06b59fe8       ___onexitend               07049fe8     <common>
 0003:06b59fec       ___onexitbegin             07049fec     <common>
 0003:06b59ff0       ___mbctype_initialized     07049ff0     <common>
 0003:06b59ff4       ___dyn_tls_init_callback   07049ff4     <common>

 entry point at        0001:000562c0

 Static symbols

 0001:000026a0       ?CreateClippedBrush@@YAPAUbspbrush_t@@PAUmapbrush_t@@ABVVector@@1@Z 004036a0 f   csg.obj
 0001:00002790       ?ComputeBoundingPlanes@@YAXABVVector@@0@Z 00403790 f   csg.obj
 0001:000030e0       ?CubemapLessFunc@@YA_NABUCubemapInfo_t@@0@Z 004040e0 f   cubemap.obj
 0001:00003150       ?FindSkyboxMaterialName@@YAPBDXZ 00404150 f   cubemap.obj
 0001:000031c0       ?FindDependentMaterial@@YAPBDPBDPAPBD@Z 004041c0 f   cubemap.obj
 0001:00003250       ?GeneratePatchedName@@YAXPBDABUPatchInfo_t@@_NPADH@Z 00404250 f   cubemap.obj
 0001:000032d0       ?PatchEnvmapForMaterialAndDependents@@YA_NPBDABUPatchInfo_t@@0@Z 004042d0 f   cubemap.obj
 0001:000045a0       ?LoadSrcVTFFiles@@YA_NQAPAVIVTFTexture@@PBDPAH_N@Z 004055a0 f   cubemap.obj
 0001:00005140       ?Cubemap_CreateTexInfo@@YAHHQAH@Z 00406140 f   cubemap.obj
 0001:00006160       ?ClipFaceToBrushList@@YAXPAUface_t@@ABV?$CUtlVector@PAUbspbrush_t@@V?$CUtlMemory@PAUbspbrush_t@@H@@@@PAPAU1@@Z 00407160 f   detail.obj
 0001:00006560       ?FindDetailVBSPName@@YAPBDXZ 00407560 f   detailobjects.obj
 0001:000065e0       ?ComputeDetailLeaf@@YAHABVVector@@@Z 004075e0 f   detailobjects.obj
 0001:00006630       ?ComputeDisplacementFaceArea@@YAMPAUdface_t@@@Z 00407630 f   detailobjects.obj
 0001:00006730       ?SortFunc@@YAHPBX0@Z       00407730 f   detailobjects.obj
 0001:00006a90       ?SelectGroup@@YAHABUDetailObject_t@@M@Z 00407a90 f   detailobjects.obj
 0001:00007840       ?SetLumpData@@YAXXZ        00408840 f   detailobjects.obj
 0001:00007ad0       ?AddDetailDictLump@@YAHPBD@Z 00408ad0 f   detailobjects.obj
 0001:00007c40       ?AddDetailSpriteDictLump@@YAHPBVVector2D@@0@Z 00408c40 f   detailobjects.obj
 0001:00007d60       ?AddDetailSpriteToLump@@YAXABVVector@@ABVQAngle@@HPBVVector2D@@2MHHHH@Z 00408d60 f   detailobjects.obj
 0001:00007ef0       ?IsModelValid@@YA_NPBD@Z   00408ef0 f   detailobjects.obj
 0001:00007fb0       ?AddDetailToLump@@YAXPBDABVVector@@ABVQAngle@@H@Z 00408fb0 f   detailobjects.obj
 0001:00008060       ?PlaceDetail@@YAXABUDetailModel_t@@ABVVector@@1@Z 00409060 f   detailobjects.obj
 0001:00008370       ?EmitDetailObjectsOnFace@@YAXPAUdface_t@@AAUDetailObject_t@@@Z 00409370 f   detailobjects.obj
 0001:00008640       ?EmitDetailObjectsOnDisplacementFace@@YAXPAUdface_t@@AAUDetailObject_t@@AAVCCoreDispInfo@@@Z 00409640 f   detailobjects.obj
 0001:00008760       ?ParseDetailGroup@@YAXHPAVKeyValues@@@Z 00409760 f   detailobjects.obj
 0001:000091a0       ?ParseDetailObjectFile@@YAXAAVKeyValues@@@Z 0040a1a0 f   detailobjects.obj
 0001:00009470       ?RotateVertIncrement@@YAXW4NeighborOrientation@@ABVCVertIndex@@AAV2@@Z 0040a470 f   disp_common.obj
 0001:0000c1c0       ?WrapVertIndex@@YA?AVCVertIndex@@ABV1@H@Z 0040d1c0 f   disp_powerinfo.obj
 0001:0000c220       ?AddDependency@@YAXPAVCVertInfo@@HABVCVertIndex@@1H_N2@Z 0040d220 f   disp_powerinfo.obj
 0001:0000c340       ?InitPowerInfo_R@@YAXPAVCPowerInfo@@HABVCVertIndex@@11111H@Z 0040d340 f   disp_powerinfo.obj
 0001:0000c6e0       ?InitPowerInfoTriInfos_R@@YAXPAVCPowerInfo@@ABVCVertIndex@@AAPAVCTriInfo@@HH@Z 0040d6e0 f   disp_powerinfo.obj
 0001:0000fe00       ?AssignBottomWaterMaterialToFace@@YA_NPAUface_t@@@Z 00410e00 f   faces.obj
 0001:000114d0       ?ModelLess@@YA_NABUModelCollisionLookup_t@@0@Z 004124d0 f   ivp.obj
 0001:000114d0       ?StaticLess@@YA_NABUStaticPropLookup_t@@0@Z 004124d0 f   ivp.obj
 0001:000115d0       ?FindOrCreateLeafWaterData@@YAHMMH@Z 004125d0 f   ivp.obj
 0001:00011640       ?BuildWaterLeaf@@YAXPAUnode_t@@AAUwaterleaf_t@@@Z 00412640 f   ivp.obj
 0001:00011790       ?FindBrushSide@@YAPAUdbrushside_t@@HABVVector@@@Z 00412790 f   ivp.obj
 0001:00011e40       ?VisitLeaves_r@@YAXAAVCPlaneList@@H@Z 00412e40 f   ivp.obj
 0001:00011ed0       ?WriteFogVolumeIDs@@YAXPAUdmodel_t@@@Z 00412ed0 f   ivp.obj
 0001:00012d20       ?PropIndex@@YAHAAV?$CUtlVector@HV?$CUtlMemory@HH@@@@H@Z 00413d20 f   ivp.obj
 0001:000131c0       ?InsertSortWaterLeaf@@YAXAAV?$CUtlVector@Uwaterleaf_t@@V?$CUtlMemory@Uwaterleaf_t@@H@@@@ABUwaterleaf_t@@@Z 004141c0 f   ivp.obj
 0001:00013220       ?Flood_FindConnectedWaterVolumes_r@@YAXAAV?$CUtlVector@PAUnode_t@@V?$CUtlMemory@PAUnode_t@@H@@@@PAUnode_t@@AAUwaterleaf_t@@AAV?$CBitVec@$0BAAAA@@@@Z 00414220 f   ivp.obj
 0001:00013340       ?ConvertWaterModelToPhysCollide@@YAXAAV?$CUtlVector@PAVCPhysCollisionEntry@@V?$CUtlMemory@PAVCPhysCollisionEntry@@H@@@@HMM@Z 00414340 f   ivp.obj
 0001:00013650       ?ConvertWorldBrushesToPhysCollide@@YAXAAV?$CUtlVector@PAVCPhysCollisionEntry@@V?$CUtlMemory@PAVCPhysCollisionEntry@@H@@@@MMH@Z 00414650 f   ivp.obj
 0001:00013940       ?BuildWorldPhysModel@@YAXAAV?$CUtlVector@PAVCPhysCollisionEntry@@V?$CUtlMemory@PAVCPhysCollisionEntry@@H@@@@MM@Z 00414940 f   ivp.obj
 0001:00013a00       ?ConvertModelToPhysCollide@@YAXAAV?$CUtlVector@PAVCPhysCollisionEntry@@V?$CUtlMemory@PAVCPhysCollisionEntry@@H@@@@HHMM@Z 00414a00 f   ivp.obj
 0001:00015430       ?AddArguments@@YAXAAHAAPAPADPBD@Z 00416430 f   loadcmdline.obj
 0001:00017540       ?LoadOverlayDataTransitionKeyCallback@@YA?AW4ChunkFileResult_t@@PBD0PAUmapoverlay_t@@@Z 00418540 f   map.obj
 0001:000180f0       ?LoadOverlayDataTransitionCallback@@YA?AW4ChunkFileResult_t@@PAVCChunkFile@@H@Z 004190f0 f   map.obj
 0001:00018140       ?LoadOverlayTransitionCallback@@YA?AW4ChunkFileResult_t@@PAVCChunkFile@@H@Z 00419140 f   map.obj
 0001:00018cf0       ?NameTranslationLessFunc@@YA_NABUNameTranslationLookup_t@@0@Z 00419cf0 f   materialpatch.obj
 0001:00018db0       ?DoesMaterialHaveKey@@YA_NPAVKeyValues@@PBD@Z 00419db0 f   materialpatch.obj
 0001:00018e00       ?DoesMaterialHaveKeyValuePair@@YA_NPAVKeyValues@@PBD1@Z 00419e00 f   materialpatch.obj
 0001:00018e70       ?InsertKeyValues@@YAXAAVKeyValues@@0_N@Z 00419e70 f   materialpatch.obj
 0001:00019550       ?ExpandPatchFile@@YAXAAVKeyValues@@@Z 0041a550 f   materialpatch.obj
 0001:0001ad89       __catch$?_Copy@?$basic_string@DU?$char_traits@D@std@@V?$allocator@D@2@@std@@IAEXII@Z$0 0041bd89 f i mstristrip.obj
 0001:0001ae23       __catch$?_Copy@?$basic_string@DU?$char_traits@D@std@@V?$allocator@D@2@@std@@IAEXII@Z$1 0041be23 f i mstristrip.obj
 0001:0001d310       ?ComputeDistFromPlane@@YAMPAUwinding_t@@PAUplane_t@@M@Z 0041e310 f   portals.obj
 0001:0001e540       ?DisplayPortalError@@YAXPAUportal_t@@H@Z 0041f540 f   portals.obj
 0001:0001fa90       ?TestLeafAgainstCollide@@YA_NHPAHABVVector@@ABVQAngle@@PAVCPhysCollide@@@Z 00420a90 f   staticprop.obj
 0001:0001fe40       ?ComputeConvexHull@@YAPAVCPhysConvex@@PAUmstudiomesh_t@@@Z 00420e40 f   staticprop.obj
 0001:0001fed0       ?ComputeLightingOrigin@@YA_NABUStaticPropBuild_t@@AAVVector@@@Z 00420ed0 f   staticprop.obj
 0001:00020b60       ?SetLumpData@@YAXXZ        00421b60 f   staticprop.obj
 0001:00020d50       ?AddStaticPropDictLump@@YAHPBD@Z 00421d50 f   staticprop.obj
 0001:00021050       ?ComputeConvexHullLeaves_R@@YAXHHPAHABVVector@@11ABVQAngle@@PAVCPhysCollide@@AAV?$CUtlVector@GV?$CUtlMemory@GH@@@@@Z 00422050 f   staticprop.obj
 0001:00021210       ?ComputeStaticPropLeaves@@YAXPAVCPhysCollide@@ABVVector@@ABVQAngle@@AAV?$CUtlVector@GV?$CUtlMemory@GH@@@@@Z 00422210 f   staticprop.obj
 0001:00021340       ?GetCollisionModel@@YAPAVCPhysCollide@@PBD@Z 00422340 f   staticprop.obj
 0001:00021530       ?AddStaticPropToLump@@YAXABUStaticPropBuild_t@@@Z 00422530 f   staticprop.obj
 0001:00021a00       ?StringIsTrue@@YAHPBD@Z    00422a00 f   textures.obj
 0001:00023c80       ?ClipOccluderBrushes@@YAPAUtree_t@@XZ 00424c80 f   vbsp.obj
 0001:00023e80       ?GenerateOccluderSideList@@YAXHAAV?$CUtlVector@PAUside_t@@V?$CUtlMemory@PAUside_t@@H@@@@@Z 00424e80 f   vbsp.obj
 0001:00023f50       ?GenerateOccluderFaceList@@YAXPAUnode_t@@AAV?$CUtlVector@PAUface_t@@V?$CUtlMemory@PAUface_t@@H@@@@@Z 00424f50 f   vbsp.obj
 0001:00023ff0       ?Compute3DSkyboxAreas@@YAXPAUnode_t@@AAV?$CUtlVector@HV?$CUtlMemory@HH@@@@@Z 00424ff0 f   vbsp.obj
 0001:00024500       ?EmitOccluderBrushes@@YAXXZ 00425500 f   vbsp.obj
 0001:000257c0       ?GeneratePatchedMaterialName@@YAXPBDPADH@Z 004267c0 f   worldvertextransitionfixup.obj
 0001:00026b00       ?AddNodeToBounds@@YAXHAAV?$CUtlVector@HV?$CUtlMemory@HH@@@@AAVVector@@1@Z 00427b00 f   writebsp.obj
 0001:00029440       ?CopyTextData@@YAXPADPBDHH@Z 0042a440 f   zip_utils.obj
 0001:0002a080       ?ReadTextData@@YAXPBDHAAVCUtlBuffer@@@Z 0042b080 f   zip_utils.obj
 0001:0002e380       ?AlignFilePosition@@YAIPAXH@Z 0042f380 f   bsplib.obj
 0001:0002e410       ?AddLumpInternal@@YAXHPAXHH@Z 0042f410 f   bsplib.obj
 0001:00030100       ?SwapPhyscollideLump@@YAXPAE0AAI@Z 00431100 f   bsplib.obj
 0001:00030590       ?SwapPhysdispLump@@YAXPAE0H@Z 00431590 f   bsplib.obj
 0001:00030620       ?SwapVisibilityLump@@YAXPAE0H@Z 00431620 f   bsplib.obj
 0001:000312b0       ?AddGameLumps@@YAXXZ       004322b0 f   bsplib.obj
 0001:00031540       ?AddOcclusionLump@@YAXXZ   00432540 f   bsplib.obj
 0001:000317a0       ?WritePakFileLump@@YAXXZ   004327a0 f   bsplib.obj
 0001:00033cd0       ?UnserializeOcclusionLumpV2@@YAXAAVCUtlBuffer@@@Z 00434cd0 f   bsplib.obj
 0001:00033e10       ?LoadOcclusionLump@@YAXXZ  00434e10 f   bsplib.obj
 0001:0003ed90       ?GetInitialColors@@YAXXZ   0043fd90 f   cmdlib.obj
 0001:0003fcf0       ?FileSystem_AddLoadedSearchPath@@YAXAAVCFSSearchPathsInit@@PBDPA_N11_N@Z 00440cf0 f   filesystem_init.obj
 0001:000406e0       ?TryLocateGameInfoFile@@YA?AW4FSReturnCode_t@@PADH_N@Z 004416e0 f   filesystem_init.obj
 0001:000440e0       ?ToolsExceptionFilter@@YGJPAU_EXCEPTION_POINTERS@@@Z 004450e0 f   tools_minidump.obj
 0001:0004a5fd       __catch$?_Ipfx@?$basic_istream@DU?$char_traits@D@std@@@std@@QAE_N_N@Z$0 0044b5fd f i tier1:tokenreader.obj
 0001:0004a79d       __catch$?get@?$basic_istream@DU?$char_traits@D@std@@@std@@QAEHXZ$0 0044b79d f i tier1:tokenreader.obj
 0001:0004a945       __catch$?get@?$basic_istream@DU?$char_traits@D@std@@@std@@QAEAAV12@PADHD@Z$0 0044b945 f i tier1:tokenreader.obj
 0001:0004aa79       __catch$?ignore@?$basic_istream@DU?$char_traits@D@std@@@std@@QAEAAV12@HH@Z$0 0044ba79 f i tier1:tokenreader.obj
 0001:0004ab44       __catch$?peek@?$basic_istream@DU?$char_traits@D@std@@@std@@QAEHXZ$0 0044bb44 f i tier1:tokenreader.obj
 0001:0004aca6       __catch$?putback@?$basic_istream@DU?$char_traits@D@std@@@std@@QAEAAV12@D@Z$0 0044bca6 f i tier1:tokenreader.obj
 0001:0004ca50       ?ReadHeaderFromBufferPastBaseHeader@@YA_NAAVCUtlBuffer@@AAUVTFFileHeader_t@@@Z 0044da50 f   vtf:vtf.obj
 0001:0004d280       ?CalcInit@@YAXPAUSphereCalc_t@@HPAPAEW4LookDir_t@@@Z 0044e280 f   vtf:vtf.obj
 0001:0004d340       ?TransformNormal@@YAXPAUSphereCalc_t@@AAVVector@@@Z 0044e340 f   vtf:vtf.obj
 0001:0004d3f0       ?CalcFaceIndex@@YAHABVVector@@@Z 0044e3f0 f   vtf:vtf.obj
 0001:0004d490       ?CalcColor@@YAXPAUSphereCalc_t@@HABVVector@@PAE@Z 0044e490 f   vtf:vtf.obj
 0001:0004d580       ?CalcSphereColor@@YAXPAUSphereCalc_t@@MM@Z 0044e580 f   vtf:vtf.obj
 0001:0004d670       ?CalcHemisphereColor@@YAXPAUSphereCalc_t@@MM@Z 0044e670 f   vtf:vtf.obj
 0001:0004d930       ?FixCubeMapFacing@@YAXPAEHHW4ImageFormat@@@Z 0044e930 f   vtf:vtf.obj
 0001:00051dfa       _vscan_fn                  00452dfa f   LIBCMT:sscanf.obj
 0001:00051f6c       __onexit_nolock            00452f6c f   LIBCMT:onexit.obj
 0001:000520e0       _swap                      004530e0 f   LIBCMT:qsort.obj
 0001:00052110       _shortsort                 00453110 f   LIBCMT:qsort.obj
 0001:000530a6       ?CatchGuardHandler@@YA?AW4_EXCEPTION_DISPOSITION@@PAUEHExceptionRecord@@PAUCatchGuardRN@@PAX2@Z 004540a6 f   LIBCMT:trnsctrl.obj
 0001:000531ab       ?TranslatorGuardHandler@@YA?AW4_EXCEPTION_DISPOSITION@@PAUEHExceptionRecord@@PAUTranslatorGuardRN@@PAX2@Z 004541ab f   LIBCMT:trnsctrl.obj
 0001:0005381d       __initterm                 0045481d f   LIBCMT:crt0dat.obj
 0001:0005395a       _doexit                    0045495a f   LIBCMT:crt0dat.obj
 0001:00053ba4       _init_namebuf              00454ba4 f   LIBCMT:tmpfile.obj
 0001:00053c69       _genfname                  00454c69 f   LIBCMT:tmpfile.obj
 0001:00054ca1       _flsall                    00455ca1 f   LIBCMT:fflush.obj
 0001:000554e6       __putenv_helper            004564e6 f   LIBCMT:putenv.obj
 0001:000560a5       _fast_error_exit           004570a5 f   LIBCMT:crt0.obj
 0001:000560c9       _check_managed_app         004570c9 f   LIBCMT:crt0.obj
 0001:0005610a       ___tmainCRTStartup         0045710a f   LIBCMT:crt0.obj
 0001:000567e8       ?strtoxl@@YAKPAUlocaleinfo_struct@@PBDPAPBDHH@Z 004577e8 f   LIBCMT:strtol.obj
 0001:0005734f       __shift                    0045834f f   LIBCMT:cvt.obj
 0001:00057388       __cftoe2_l                 00458388 f   LIBCMT:cvt.obj
 0001:00057952       __cftof2_l                 00458952 f   LIBCMT:cvt.obj
 0001:00057d4c       _fastcopy_I                00458d4c f   LIBCMT:p4_memcpy.obj
 0001:00057eca       _fastzero_I                00458eca f   LIBCMT:p4_memset.obj
 0001:0005842b       _write_char                0045942b f   LIBCMT:output.obj
 0001:0005845e       _write_multi_char          0045945e f   LIBCMT:output.obj
 0001:00058482       _write_string              00459482 f   LIBCMT:output.obj
 0001:00059500       __unwind_handler4          0045a500 f   LIBCMT:exsup4.obj
 0001:000597bb       ___check_float_string      0045a7bb f   LIBCMT:input.obj
 0001:0005980f       __inc                      0045a80f f   LIBCMT:input.obj
 0001:00059825       __whiteout                 0045a825 f   LIBCMT:input.obj
 0001:0005a497       __use_encode_pointer       0045b497 f   LIBCMT:tidtable.obj
 0001:0005afb6       ?CPtoLCID@@YAHH@Z          0045bfb6 f   LIBCMT:mbctype.obj
 0001:0005afe5       ?setSBCS@@YAXPAUthreadmbcinfostruct@@@Z 0045bfe5 f   LIBCMT:mbctype.obj
 0001:0005b03a       ?setSBUpLow@@YAXPAUthreadmbcinfostruct@@@Z 0045c03a f   LIBCMT:mbctype.obj
 0001:0005b268       ?getSystemCP@@YAHH@Z       0045c268 f   LIBCMT:mbctype.obj
 0001:0005b8c5       __copytlocinfo_nolock      0045c8c5 f   LIBCMT:setlocal.obj
 0001:0005b8e9       __updatetlocinfoEx_nolock  0045c8e9 f   LIBCMT:setlocal.obj
 0001:0005b99d       _sync_legacy_variables_lk  0045c99d f   LIBCMT:setlocal.obj
 0001:0005bbc2       __setlocale_get_all        0045cbc2 f   LIBCMT:setlocal.obj
 0001:0005bf07       __setlocale_set_cat        0045cf07 f   LIBCMT:setlocal.obj
 0001:0005c1fd       __setlocale_nolock         0045d1fd f   LIBCMT:setlocal.obj
 0001:0005d994       ?ExFilterRethrow@@YAHPAU_EXCEPTION_POINTERS@@@Z 0045e994 f   LIBCMT:frame.obj
 0001:0005da52       ?IsInExceptionSpec@@YAEPAUEHExceptionRecord@@PBU_s_ESTypeList@@@Z 0045ea52 f   LIBCMT:frame.obj
 0001:0005dacb       ?CallUnexpected@@YAXPBU_s_ESTypeList@@@Z 0045eacb f   LIBCMT:frame.obj
 0001:0005dafc       __catch$?CallUnexpected@@YAXPBU_s_ESTypeList@@@Z$0 0045eafc f   LIBCMT:frame.obj
 0001:0005db14       ?CallCatchBlock@@YAPAXPAUEHExceptionRecord@@PAUEHRegistrationNode@@PAU_CONTEXT@@PBU_s_FuncInfo@@PAXHK@Z 0045eb14 f   LIBCMT:frame.obj
 0001:0005dec0       ?CatchIt@@YAXPAUEHExceptionRecord@@PAUEHRegistrationNode@@PAU_CONTEXT@@PAXPBU_s_FuncInfo@@PBU_s_HandlerType@@PBU_s_CatchableType@@PBU_s_TryBlockMapEntry@@H1E@Z 0045eec0 f   LIBCMT:frame.obj
 0001:0005df2c       ?FindHandlerForForeignException@@YAXPAUEHExceptionRecord@@PAUEHRegistrationNode@@PAU_CONTEXT@@PAXPBU_s_FuncInfo@@HH1@Z 0045ef2c f   LIBCMT:frame.obj
 0001:0005e01e       ?FindHandler@@YAXPAUEHExceptionRecord@@PAUEHRegistrationNode@@PAU_CONTEXT@@PAXPBU_s_FuncInfo@@EH1@Z 0045f01e f   LIBCMT:frame.obj
 0001:0005f73b       ?__crtLCMapStringA_stat@@YAHPAUlocaleinfo_struct@@KKPBDHPADHHH@Z 0046073b f   LIBCMT:a_map.obj
 0001:0005ffe3       _siglookup                 00460fe3 f   LIBCMT:winsig.obj
 0001:000601e8       ___crtInitCritSecNoSpinCount@8 004611e8 f   LIBCMT:initcrit.obj
 0001:0006032e       _xtoa_s@20                 0046132e f   LIBCMT:xtoas.obj
 0001:000605cb       __tsopen_nolock            004615cb f   LIBCMT:open.obj
 0001:000621cb       _wfindenv                  004631cb f   LIBCMT:wsetenv.obj
 0001:0006221c       _copy_environ              0046321c f   LIBCMT:wsetenv.obj
 0001:000625f5       _findenv                   004635f5 f   LIBCMT:setenv.obj
 0001:00062642       _copy_environ              00463642 f   LIBCMT:setenv.obj
 0001:00062b50       _comexecmd                 00463b50 f   LIBCMT:spawnve.obj
 0001:00062fbf       _parse_cmdline             00463fbf f   LIBCMT:stdargv.obj
 0001:00063420       ?wcstoxl@@YAKPAUlocaleinfo_struct@@PB_WPAPB_WHH@Z 00464420 f   LIBCMT:wcstol.obj
 0001:00065f32       _has_osfxsr_set            00466f32 f   LIBCMT:cpu_disp.obj
 0001:00066a04       __unwind_handler           00467a04 f   LIBCMT:exsup.obj
 0001:000670e8       ?__crtGetLocaleInfoW_stat@@YAHPAUlocaleinfo_struct@@KKPA_WHH@Z 004680e8 f   LIBCMT:w_loc.obj
 0001:0006725e       ?__crtGetLocaleInfoA_stat@@YAHPAUlocaleinfo_struct@@KKPADHH@Z 0046825e f   LIBCMT:a_loc.obj
 0001:000673d6       ?__crtGetStringTypeA_stat@@YAHPAUlocaleinfo_struct@@KPBDHPAGHHH@Z 004683d6 f   LIBCMT:a_str.obj
 0001:000675f7       __get_lc_time              004685f7 f   LIBCMT:inittime.obj
 0001:00068596       _TranslateName             00469596 f   LIBCMT:getqloc.obj
 0001:000685f6       _ProcessCodePage           004695f6 f   LIBCMT:getqloc.obj
 0001:0006866d       _TestDefaultCountry        0046966d f   LIBCMT:getqloc.obj
 0001:0006868b       _LcidFromHexString         0046968b f   LIBCMT:getqloc.obj
 0001:000686bd       _GetPrimaryLen             004696bd f   LIBCMT:getqloc.obj
 0001:000686d8       _CountryEnumProc@4         004696d8 f   LIBCMT:getqloc.obj
 0001:0006876e       _TestDefaultLanguage       0046976e f   LIBCMT:getqloc.obj
 0001:000687e0       _LangCountryEnumProc@4     004697e0 f   LIBCMT:getqloc.obj
 0001:000689b0       _LanguageEnumProc@4        004699b0 f   LIBCMT:getqloc.obj
 0001:00068a6f       _GetLcidFromLangCountry    00469a6f f   LIBCMT:getqloc.obj
 0001:00068ad4       _GetLcidFromLanguage       00469ad4 f   LIBCMT:getqloc.obj
 0001:0006c01f       __tzset_nolock             0046d01f f   LIBCMT:tzset.obj
 0001:0006c368       _cvtdate                   0046d368 f   LIBCMT:tzset.obj
 0001:0006c55d       __isindst_nolock           0046d55d f   LIBCMT:tzset.obj
 0001:0006cd80       ?__crtCompareStringA_stat@@YAHPAUlocaleinfo_struct@@KKPBDH1HH@Z 0046dd80 f   LIBCMT:a_cmp.obj
 0001:0006d825       ?x_ismbbtype_l@@YAHPAUlocaleinfo_struct@@IHH@Z 0046e825 f   LIBCMT:ismbbyte.obj
 0001:0006da0b       ?__crtGetStringTypeW_stat@@YAHPAUlocaleinfo_struct@@KPB_WHPAGHH@Z 0046ea0b f   LIBCMT:w_str.obj
 0001:0006e5c7       __hw_cw                    0046f5c7 f   LIBCMT:ieee87.obj
 0001:0006e655       ___hw_cw_sse2              0046f655 f   LIBCMT:ieee87.obj
 0001:0006f010       ?wcsncnt@@YAHPB_WH@Z       00470010 f   LIBCMT:w_cmp.obj
 0001:0006f02c       ?__crtCompareStringW_stat@@YAHPAUlocaleinfo_struct@@KKPB_WH1HH@Z 0047002c f   LIBCMT:w_cmp.obj
 0001:0006f765       _tidy_global               00470765 f   libcpmt:locale0.obj
 0001:00070540       ?GetColorBlockColorsBGRA8888@ImageLoader@@YAXPAUDXTColBlock@1@PAUBGRA8888_t@@111AAG@Z 00471540 f   bitmap:colorconversion.obj
 0001:00070700       ?GetDXTCEncodeType@ImageLoader@@YAKW4ImageFormat@@@Z 00471700 f   bitmap:colorconversion.obj
 0001:00071850       ?ABGR8888ToRGBA8888@ImageLoader@@YAXPBEPAEH@Z 00472850 f   bitmap:colorconversion.obj
 0001:00071850       ?RGBA8888ToABGR8888@ImageLoader@@YAXPBEPAEH@Z 00472850 f   bitmap:colorconversion.obj
 0001:00071890       ?RGBA8888ToRGB888@ImageLoader@@YAXPBEPAEH@Z 00472890 f   bitmap:colorconversion.obj
 0001:000718d0       ?RGBA8888ToBGR888@ImageLoader@@YAXPBEPAEH@Z 004728d0 f   bitmap:colorconversion.obj
 0001:00071910       ?RGBA8888ToI8@ImageLoader@@YAXPBEPAEH@Z 00472910 f   bitmap:colorconversion.obj
 0001:000719a0       ?RGBA8888ToIA88@ImageLoader@@YAXPBEPAEH@Z 004729a0 f   bitmap:colorconversion.obj
 0001:00071a40       ?RGBA8888ToA8@ImageLoader@@YAXPBEPAEH@Z 00472a40 f   bitmap:colorconversion.obj
 0001:00071a70       ?RGBA8888ToRGB888_BLUESCREEN@ImageLoader@@YAXPBEPAEH@Z 00472a70 f   bitmap:colorconversion.obj
 0001:00071ac0       ?RGBA8888ToBGR888_BLUESCREEN@ImageLoader@@YAXPBEPAEH@Z 00472ac0 f   bitmap:colorconversion.obj
 0001:00071b10       ?RGBA8888ToARGB8888@ImageLoader@@YAXPBEPAEH@Z 00472b10 f   bitmap:colorconversion.obj
 0001:00071b50       ?RGBA8888ToBGRX8888@ImageLoader@@YAXPBEPAEH@Z 00472b50 f   bitmap:colorconversion.obj
 0001:00071b90       ?RGBA8888ToBGR565@ImageLoader@@YAXPBEPAEH@Z 00472b90 f   bitmap:colorconversion.obj
 0001:00071c00       ?RGBA8888ToBGRX5551@ImageLoader@@YAXPBEPAEH@Z 00472c00 f   bitmap:colorconversion.obj
 0001:00071c60       ?RGBA8888ToBGRA5551@ImageLoader@@YAXPBEPAEH@Z 00472c60 f   bitmap:colorconversion.obj
 0001:00071cd0       ?RGBA8888ToBGRA4444@ImageLoader@@YAXPBEPAEH@Z 00472cd0 f   bitmap:colorconversion.obj
 0001:00071d40       ?RGBA8888ToUV88@ImageLoader@@YAXPBEPAEH@Z 00472d40 f   bitmap:colorconversion.obj
 0001:00071d70       ?UVWQ8888ToRGBA8888@ImageLoader@@YAXPBEPAEH@Z 00472d70 f   bitmap:colorconversion.obj
 0001:00071d70       ?RGBA8888ToUVWQ8888@ImageLoader@@YAXPBEPAEH@Z 00472d70 f   bitmap:colorconversion.obj
 0001:00071d70       ?RGBA8888ToUVLX8888@ImageLoader@@YAXPBEPAEH@Z 00472d70 f   bitmap:colorconversion.obj
 0001:00071d70       ?RGBA8888ToRGBA8888@ImageLoader@@YAXPBEPAEH@Z 00472d70 f   bitmap:colorconversion.obj
 0001:00071d70       ?UVLX8888ToRGBA8888@ImageLoader@@YAXPBEPAEH@Z 00472d70 f   bitmap:colorconversion.obj
 0001:00071d90       ?RGB888ToRGBA8888@ImageLoader@@YAXPBEPAEH@Z 00472d90 f   bitmap:colorconversion.obj
 0001:00071de0       ?BGR888ToRGBA8888@ImageLoader@@YAXPBEPAEH@Z 00472de0 f   bitmap:colorconversion.obj
 0001:00071e30       ?I8ToRGBA8888@ImageLoader@@YAXPBEPAEH@Z 00472e30 f   bitmap:colorconversion.obj
 0001:00071e70       ?IA88ToRGBA8888@ImageLoader@@YAXPBEPAEH@Z 00472e70 f   bitmap:colorconversion.obj
 0001:00071eb0       ?A8ToRGBA8888@ImageLoader@@YAXPBEPAEH@Z 00472eb0 f   bitmap:colorconversion.obj
 0001:00071ef0       ?RGB888_BLUESCREENToRGBA8888@ImageLoader@@YAXPBEPAEH@Z 00472ef0 f   bitmap:colorconversion.obj
 0001:00071f50       ?BGR888_BLUESCREENToRGBA8888@ImageLoader@@YAXPBEPAEH@Z 00472f50 f   bitmap:colorconversion.obj
 0001:00071fb0       ?ARGB8888ToRGBA8888@ImageLoader@@YAXPBEPAEH@Z 00472fb0 f   bitmap:colorconversion.obj
 0001:00071ff0       ?BGRA8888ToRGBA8888@ImageLoader@@YAXPBEPAEH@Z 00472ff0 f   bitmap:colorconversion.obj
 0001:00071ff0       ?RGBA8888ToBGRA8888@ImageLoader@@YAXPBEPAEH@Z 00472ff0 f   bitmap:colorconversion.obj
 0001:00072030       ?BGRX8888ToRGBA8888@ImageLoader@@YAXPBEPAEH@Z 00473030 f   bitmap:colorconversion.obj
 0001:00072080       ?BGR565ToRGBA8888@ImageLoader@@YAXPBEPAEH@Z 00473080 f   bitmap:colorconversion.obj
 0001:00072100       ?BGRX5551ToRGBA8888@ImageLoader@@YAXPBEPAEH@Z 00473100 f   bitmap:colorconversion.obj
 0001:00072170       ?BGRA5551ToRGBA8888@ImageLoader@@YAXPBEPAEH@Z 00473170 f   bitmap:colorconversion.obj
 0001:00072200       ?BGRA4444ToRGBA8888@ImageLoader@@YAXPBEPAEH@Z 00473200 f   bitmap:colorconversion.obj
 0001:00072290       ?UV88ToRGBA8888@ImageLoader@@YAXPBEPAEH@Z 00473290 f   bitmap:colorconversion.obj
 0001:000722d0       ?RGBA16161616ToRGBA8888@ImageLoader@@YAXPBEPAEH@Z 004732d0 f   bitmap:colorconversion.obj
 0001:000723a0       ??$DecodeColorBlock@URGBA8888_t@@@ImageLoader@@YAXPAURGBA8888_t@@PAUDXTColBlock@0@HPAUBGRA8888_t@@222@Z 004733a0 f   bitmap:colorconversion.obj
 0001:000724e0       ??$DecodeColorBlock@UBGRA8888_t@@@ImageLoader@@YAXPAUBGRA8888_t@@PAUDXTColBlock@0@H0000@Z 004734e0 f   bitmap:colorconversion.obj
 0001:000725b0       ??$DecodeColorBlock@URGB888_t@@@ImageLoader@@YAXPAURGB888_t@@PAUDXTColBlock@0@HPAUBGRA8888_t@@222@Z 004735b0 f   bitmap:colorconversion.obj
 0001:000726c0       ??$DecodeColorBlock@UBGR888_t@@@ImageLoader@@YAXPAUBGR888_t@@PAUDXTColBlock@0@HPAUBGRA8888_t@@222@Z 004736c0 f   bitmap:colorconversion.obj
 0001:000727c0       ??$DecodeColorBlock@UBGR565_t@@@ImageLoader@@YAXPAUBGR565_t@@PAUDXTColBlock@0@HPAUBGRA8888_t@@222@Z 004737c0 f   bitmap:colorconversion.obj
 0001:000729b0       ??$DecodeColorBlock@UBGRA5551_t@@@ImageLoader@@YAXPAUBGRA5551_t@@PAUDXTColBlock@0@HPAUBGRA8888_t@@222@Z 004739b0 f   bitmap:colorconversion.obj
 0001:00072a80       ??$DecodeColorBlock@UBGRA4444_t@@@ImageLoader@@YAXPAUBGRA4444_t@@PAUDXTColBlock@0@HPAUBGRA8888_t@@222@Z 00473a80 f   bitmap:colorconversion.obj
 0001:00072b50       ??$DecodeAlpha3BitLinear@UBGRA8888_t@@@ImageLoader@@YAXPAUBGRA8888_t@@PAUDXTAlphaBlock3BitLinear@0@HH@Z 00473b50 f   bitmap:colorconversion.obj
 0001:00072e60       ??$DecodeAlpha3BitLinear@URGBA8888_t@@@ImageLoader@@YAXPAURGBA8888_t@@PAUDXTAlphaBlock3BitLinear@0@HH@Z 00473e60 f   bitmap:colorconversion.obj
 0001:00073170       ??$DecodeAlpha3BitLinear@UBGRA5551_t@@@ImageLoader@@YAXPAUBGRA5551_t@@PAUDXTAlphaBlock3BitLinear@0@HH@Z 00474170 f   bitmap:colorconversion.obj
 0001:000734a0       ??$DecodeAlpha3BitLinear@UBGRA4444_t@@@ImageLoader@@YAXPAUBGRA4444_t@@PAUDXTAlphaBlock3BitLinear@0@HH@Z 004744a0 f   bitmap:colorconversion.obj
 0001:000737e0       ?GetUserFormatToRGBA8888Func_t@ImageLoader@@YAP6AXPBEPAEH@ZW4ImageFormat@@@Z 004747e0 f   bitmap:colorconversion.obj
 0001:000738e0       ?GetRGBA8888ToUserFormatFunc_t@ImageLoader@@YAP6AXPBEPAEH@ZW4ImageFormat@@@Z 004748e0 f   bitmap:colorconversion.obj
 0001:00073cb0       ??$ConvertFromDXT1@URGBA8888_t@@@ImageLoader@@YAXPBEPAURGBA8888_t@@HH@Z 00474cb0 f   bitmap:colorconversion.obj
 0001:00073e00       ??$ConvertFromDXT1@UBGRA8888_t@@@ImageLoader@@YAXPBEPAUBGRA8888_t@@HH@Z 00474e00 f   bitmap:colorconversion.obj
 0001:00073f60       ??$ConvertFromDXT1@URGB888_t@@@ImageLoader@@YAXPBEPAURGB888_t@@HH@Z 00474f60 f   bitmap:colorconversion.obj
 0001:000740c0       ??$ConvertFromDXT1@UBGR888_t@@@ImageLoader@@YAXPBEPAUBGR888_t@@HH@Z 004750c0 f   bitmap:colorconversion.obj
 0001:00074220       ??$ConvertFromDXT1@UBGR565_t@@@ImageLoader@@YAXPBEPAUBGR565_t@@HH@Z 00475220 f   bitmap:colorconversion.obj
 0001:00074360       ??$ConvertFromDXT1@UBGRA5551_t@@@ImageLoader@@YAXPBEPAUBGRA5551_t@@HH@Z 00475360 f   bitmap:colorconversion.obj
 0001:000744b0       ??$ConvertFromDXT1@UBGRA4444_t@@@ImageLoader@@YAXPBEPAUBGRA4444_t@@HH@Z 004754b0 f   bitmap:colorconversion.obj
 0001:00074600       ??$ConvertFromATIxN@UBGRA8888_t@@@ImageLoader@@YAXPBEPAUBGRA8888_t@@HH_N@Z 00475600 f   bitmap:colorconversion.obj
 0001:00074730       ??$ConvertFromDXT5@URGBA8888_t@@@ImageLoader@@YAXPBEPAURGBA8888_t@@HH@Z 00475730 f   bitmap:colorconversion.obj
 0001:000748a0       ??$ConvertFromDXT5@UBGRA8888_t@@@ImageLoader@@YAXPBEPAUBGRA8888_t@@HH@Z 004758a0 f   bitmap:colorconversion.obj
 0001:00074a10       ??$ConvertFromDXT5IgnoreAlpha@URGB888_t@@@ImageLoader@@YAXPBEPAURGB888_t@@HH@Z 00475a10 f   bitmap:colorconversion.obj
 0001:00074b70       ??$ConvertFromDXT5IgnoreAlpha@UBGR888_t@@@ImageLoader@@YAXPBEPAUBGR888_t@@HH@Z 00475b70 f   bitmap:colorconversion.obj
 0001:00074cd0       ??$ConvertFromDXT5IgnoreAlpha@UBGR565_t@@@ImageLoader@@YAXPBEPAUBGR565_t@@HH@Z 00475cd0 f   bitmap:colorconversion.obj
 0001:00074e20       ??$ConvertFromDXT5@UBGRA5551_t@@@ImageLoader@@YAXPBEPAUBGRA5551_t@@HH@Z 00475e20 f   bitmap:colorconversion.obj
 0001:00074f80       ??$ConvertFromDXT5@UBGRA4444_t@@@ImageLoader@@YAXPBEPAUBGRA4444_t@@HH@Z 00475f80 f   bitmap:colorconversion.obj
 0001:000757f0       ?ConstructFloatGammaTable@ImageLoader@@YAXPAMMM@Z 004767f0 f   bitmap:resample.obj
 0001:00075a70       ?GenerateNiceFilter@ImageLoader@@YAXMMMHPAM0@Z 00476a70 f   bitmap:resample.obj
 0001:000815f0       ?getAxis@@YAXHPAY02NQAN@Z  004825f0 f   bitmap:S3_quant.obj
 0001:000819f0       ?getDiameter@@YAXHPAY02NQAN@Z 004829f0 f   bitmap:S3_quant.obj
 0001:00081b00       ?sortProjection@@YAXHPAY02NQANQAHH@Z 00482b00 f   bitmap:S3_quant.obj
 0001:00081c50       ?sameOrder@@YAHHQAH0@Z     00482c50 f   bitmap:S3_quant.obj
 0001:00081cc0       ?search43Mult@@YANPAHHPAY02NPANQAHQAY02NQAN@Z 00482cc0 f   bitmap:S3_quant.obj
 0001:00082360       ?searchClipped43Mult@@YANPAHHPAY02NPANQAHQAY02N4QAN@Z 00483360 f   bitmap:S3_quant.obj
 0001:00082d70       ?allSame@@YANPAHHPAY02NQANQAY02HQAH@Z 00483d70 f   bitmap:S3_quant.obj
 0001:000832c0       ?mapAndRoundMult@@YANPAHHHPAY02NPANQANQAY02NQAY02HQAH@Z 004842c0 f   bitmap:S3_quant.obj
 0001:000834a0       ?roundMult@@YANHHPAY02NPANQANQAY02NQAY02HQAH@Z 004844a0 f   bitmap:S3_quant.obj
 0001:00083fd0       ?quantizeAlpha@@YANHHQANQAH1@Z 00484fd0 f   bitmap:S3_quant.obj
 0001:0008d410       ?QSortIntCmp@@YAHPBX0@Z    0048e410 f   bitmap:ATiXCodec.obj
 0001:0008d420       ?QSortFloatCmp@@YAHPBX0@Z  0048e420 f   bitmap:ATiXCodec.obj
 0001:0008d490       ?ClstrErr@@YAMQAY03MQAMQAY0BA@MHH_NPAM@Z 0048e490 f   bitmap:ATiXCodec.obj
 0001:0008d8c0       ?ClstrIntnl@@YAMQAY03MPAEQAY0BA@MHE_NPAM3@Z 0048e8c0 f   bitmap:ATiXCodec.obj
 0001:0008da40       ?RampSrchWSS2E@@YAMQAM00MMMHE@Z 0048ea40 f   bitmap:ATiXCodec.obj
 0001:0008db30       ?BldRmp1@@YAXQAM0H@Z       0048eb30 f   bitmap:ATiXCodec.obj
 0001:0008dc80       ?GetRmp1@@YAXQAM0H_NHH1@Z  0048ec80 f   bitmap:ATiXCodec.obj
 0001:0008dd90       ?Clstr1@@YAMPAEQAM1HH_NHH2@Z 0048ed90 f   bitmap:ATiXCodec.obj
 0001:0008df00       ?RmpSrch1SSE2@@YAMQAM0MMMHE@Z 0048ef00 f   bitmap:ATiXCodec.obj
 0001:0008dff0       ?RmpSrch1@@YAMQAM0MMMHE@Z  0048eff0 f   bitmap:ATiXCodec.obj
 0001:0008e150       ?Refine1@@YAMQAM0MAAM1MMMHE_N@Z 0048f150 f   bitmap:ATiXCodec.obj
 0001:0008e310       ?QSortFCmp@@YAHPBX0@Z      0048f310 f   bitmap:ATiXCodec.obj
 0001:0008e350       ?CompBlock1@@YAMQAM0HE_NHH11@Z 0048f350 f   bitmap:ATiXCodec.obj
 0001:0008f020       ?MkRmpOnGrid@@YAXQAY01M0MMEEE@Z 00490020 f   bitmap:ATiXCodec.obj
 0001:0008f1f0       ?ClstrBas@@YAMPAEQAY03MQAY01MHEPAM_NEEE@Z 004901f0 f   bitmap:ATiXCodec.obj
 0001:0008f890       ?RampSrchW@@YAMQAM00MMMHH@Z 00490890 f   bitmap:ATiXCodec.obj
 0001:0008fa00       ?FindAxis@@YAXQAY03MQAM1PA_N01HH@Z 00490a00 f   bitmap:ATiXCodec.obj
 0001:000900f0       ?Refine@@YAMQAY01M0QAY03MQAMHEPAMEEEE@Z 004910f0 f   bitmap:ATiXCodec.obj
 0001:00091360       ?Refine3D@@YAMQAY01M0QAY03MQAMHEPAMEEEE@Z 00492360 f   bitmap:ATiXCodec.obj
 0001:00091db0       ?RefineSSE2@@YAMQAY01M0QAY03MQAMHEPAMEEEE@Z 00492db0 f   bitmap:ATiXCodec.obj
 0001:00093140       ?Refine3DSSE2@@YAMQAY01M0QAY03MQAMHEPAMEEEE@Z 00494140 f   bitmap:ATiXCodec.obj
 0001:00094550       ?CompressRGBBlockX@@YAXQAY01MQAY03MQAMHE_NEPAMEEE@Z 00495550 f   bitmap:ATiXCodec.obj
 0001:00095913       _xtoa@16                   00496913 f   LIBCMT:xtoa.obj
 0001:00096775       __tsopen_nolock            00497775 f   LIBCMT:wopen.obj
 0001:0009723b       ?__crtLCMapStringW_stat@@YAHPAUlocaleinfo_struct@@KKPB_WHPA_WHH@Z 0049823b f   LIBCMT:w_map.obj
 0001:000974e0       __ehhandler$?_Copy@?$basic_string@DU?$char_traits@D@std@@V?$allocator@D@2@@std@@IAEXII@Z 004984e0 f   mstristrip.obj
 0001:000974f0       __ehhandler$?_Ipfx@?$basic_istream@DU?$char_traits@D@std@@@std@@QAE_N_N@Z 004984f0 f   tier1:tokenreader.obj
 0001:00097500       __ehhandler$?get@?$basic_istream@DU?$char_traits@D@std@@@std@@QAEHXZ 00498500 f   tier1:tokenreader.obj
 0001:00097510       __ehhandler$?get@?$basic_istream@DU?$char_traits@D@std@@@std@@QAEAAV12@PADHD@Z 00498510 f   tier1:tokenreader.obj
 0001:00097520       __ehhandler$?ignore@?$basic_istream@DU?$char_traits@D@std@@@std@@QAEAAV12@HH@Z 00498520 f   tier1:tokenreader.obj
 0001:00097530       __ehhandler$?peek@?$basic_istream@DU?$char_traits@D@std@@@std@@QAEHXZ 00498530 f   tier1:tokenreader.obj
 0001:00097540       __ehhandler$?putback@?$basic_istream@DU?$char_traits@D@std@@@std@@QAEAAV12@D@Z 00498540 f   tier1:tokenreader.obj
 0001:0009754a       __ehhandler$?CallUnexpected@@YAXPBU_s_ESTypeList@@@Z 0049854a f   LIBCMT:frame.obj
 0001:00097565       __unwindfunclet$?_Xran@_String_base@std@@SAXXZ$0 00498565 f   libcpmt:string.obj
 0001:00097565       __unwindfunclet$?_Xlen@_String_base@std@@SAXXZ$0 00498565 f   libcpmt:string.obj
 0001:0009756d       __ehhandler$?_Xlen@_String_base@std@@SAXXZ 0049856d f   libcpmt:string.obj
 0001:0009756d       __ehhandler$?_Xran@_String_base@std@@SAXXZ 0049856d f   libcpmt:string.obj
 0001:00097588       __unwindfunclet$?_Locimp_dtor@_Locimp@locale@std@@CAXPAV123@@Z$0 00498588 f   libcpmt:locale0.obj
 0001:00097590       __ehhandler$?_Locimp_dtor@_Locimp@locale@std@@CAXPAV123@@Z 00498590 f   libcpmt:locale0.obj
 0001:000975ab       __unwindfunclet$??0_Locimp@locale@std@@AAE@_N@Z$0 004985ab f   libcpmt:locale0.obj
 0001:000975b3       __ehhandler$??0_Locimp@locale@std@@AAE@_N@Z 004985b3 f   libcpmt:locale0.obj
 0001:000975ce       __unwindfunclet$??1_Locimp@locale@std@@MAE@XZ$0 004985ce f   libcpmt:locale0.obj
 0001:000975d6       __unwindfunclet$??1_Locimp@locale@std@@MAE@XZ$1 004985d6 f   libcpmt:locale0.obj
 0001:000975e1       __ehhandler$??1_Locimp@locale@std@@MAE@XZ 004985e1 f   libcpmt:locale0.obj
 0001:000975fc       __unwindfunclet$?_Init@locale@std@@CAPAV_Locimp@12@XZ$0 004985fc f   libcpmt:locale0.obj
 0001:00097604       __unwindfunclet$?_Init@locale@std@@CAPAV_Locimp@12@XZ$1 00498604 f   libcpmt:locale0.obj
 0001:0009760e       __ehhandler$?_Init@locale@std@@CAPAV_Locimp@12@XZ 0049860e f   libcpmt:locale0.obj
 0001:00097630       __unwindfunclet$?ThreadedCompressTexture@@YA?AW4ATI_TC_ERROR@@PBU_ATI_TC_Texture@@PAU2@PBU_ATI_TC_CompressOptions@@P6A_NMKK@ZKKW4_CodecType@@@Z$0 00498630 f   bitmap:ATI_Compress.obj
 0001:00097646       __ehhandler$?ThreadedCompressTexture@@YA?AW4ATI_TC_ERROR@@PBU_ATI_TC_Texture@@PAU2@PBU_ATI_TC_CompressOptions@@P6A_NMKK@ZKKW4_CodecType@@@Z 00498646 f   bitmap:ATI_Compress.obj
 0001:00097670       __unwindfunclet$?CreateCodec@@YAPAVCCodec@ATI_Compress@@W4_CodecType@@@Z$0 00498670 f   bitmap:Codec.obj
 0001:0009767b       __unwindfunclet$?CreateCodec@@YAPAVCCodec@ATI_Compress@@W4_CodecType@@@Z$1 0049867b f   bitmap:Codec.obj
 0001:00097686       __unwindfunclet$?CreateCodec@@YAPAVCCodec@ATI_Compress@@W4_CodecType@@@Z$2 00498686 f   bitmap:Codec.obj
 0001:00097691       __unwindfunclet$?CreateCodec@@YAPAVCCodec@ATI_Compress@@W4_CodecType@@@Z$3 00498691 f   bitmap:Codec.obj
 0001:0009769c       __unwindfunclet$?CreateCodec@@YAPAVCCodec@ATI_Compress@@W4_CodecType@@@Z$4 0049869c f   bitmap:Codec.obj
 0001:000976a7       __unwindfunclet$?CreateCodec@@YAPAVCCodec@ATI_Compress@@W4_CodecType@@@Z$5 004986a7 f   bitmap:Codec.obj
 0001:000976b2       __unwindfunclet$?CreateCodec@@YAPAVCCodec@ATI_Compress@@W4_CodecType@@@Z$6 004986b2 f   bitmap:Codec.obj
 0001:000976bd       __unwindfunclet$?CreateCodec@@YAPAVCCodec@ATI_Compress@@W4_CodecType@@@Z$7 004986bd f   bitmap:Codec.obj
 0001:000976c8       __unwindfunclet$?CreateCodec@@YAPAVCCodec@ATI_Compress@@W4_CodecType@@@Z$8 004986c8 f   bitmap:Codec.obj
 0001:000976d3       __unwindfunclet$?CreateCodec@@YAPAVCCodec@ATI_Compress@@W4_CodecType@@@Z$9 004986d3 f   bitmap:Codec.obj
 0001:000976de       __unwindfunclet$?CreateCodec@@YAPAVCCodec@ATI_Compress@@W4_CodecType@@@Z$10 004986de f   bitmap:Codec.obj
 0001:000976e9       __unwindfunclet$?CreateCodec@@YAPAVCCodec@ATI_Compress@@W4_CodecType@@@Z$11 004986e9 f   bitmap:Codec.obj
 0001:000976f4       __unwindfunclet$?CreateCodec@@YAPAVCCodec@ATI_Compress@@W4_CodecType@@@Z$12 004986f4 f   bitmap:Codec.obj
 0001:000976ff       __ehhandler$?CreateCodec@@YAPAVCCodec@ATI_Compress@@W4_CodecType@@@Z 004986ff f   bitmap:Codec.obj
 0001:00097720       __unwindfunclet$?CreateCodecBuffer@@YAPAVCCodecBuffer@@W4_CodecBufferType@@KKKPAE@Z$0 00498720 f   bitmap:CodecBuffer.obj
 0001:0009772b       __unwindfunclet$?CreateCodecBuffer@@YAPAVCCodecBuffer@@W4_CodecBufferType@@KKKPAE@Z$1 0049872b f   bitmap:CodecBuffer.obj
 0001:00097736       __unwindfunclet$?CreateCodecBuffer@@YAPAVCCodecBuffer@@W4_CodecBufferType@@KKKPAE@Z$2 00498736 f   bitmap:CodecBuffer.obj
 0001:00097741       __unwindfunclet$?CreateCodecBuffer@@YAPAVCCodecBuffer@@W4_CodecBufferType@@KKKPAE@Z$3 00498741 f   bitmap:CodecBuffer.obj
 0001:0009774c       __unwindfunclet$?CreateCodecBuffer@@YAPAVCCodecBuffer@@W4_CodecBufferType@@KKKPAE@Z$4 0049874c f   bitmap:CodecBuffer.obj
 0001:00097757       __unwindfunclet$?CreateCodecBuffer@@YAPAVCCodecBuffer@@W4_CodecBufferType@@KKKPAE@Z$5 00498757 f   bitmap:CodecBuffer.obj
 0001:00097762       __ehhandler$?CreateCodecBuffer@@YAPAVCCodecBuffer@@W4_CodecBufferType@@KKKPAE@Z 00498762 f   bitmap:CodecBuffer.obj
 0001:00097780       __unwindfunclet$??0CCodec_DXTC@@QAE@W4_CodecType@@@Z$0 00498780 f   bitmap:Codec_DXTC.obj
 0001:00097788       __ehhandler$??0CCodec_DXTC@@QAE@W4_CodecType@@@Z 00498788 f   bitmap:Codec_DXTC.obj
 0001:000977b0       ??__Es_EnvCubemapToBrushSides@@YAXXZ 004987b0 f   cubemap.obj
 0001:000977c0       ??__Es_DefaultCubemapNames@@YAXXZ 004987c0 f   cubemap.obj
 0001:000977d0       ??__Es_DetailObjectDict@@YAXXZ 004987d0 f   detailobjects.obj
 0001:000977e0       ??__Es_StaticPropLookup@@YAXXZ 004987e0 f   detailobjects.obj
 0001:00097830       ??__Es_DetailObjectDictLump@@YAXXZ 00498830 f   detailobjects.obj
 0001:00097840       ??__Es_DetailObjectLump@@YAXXZ 00498840 f   detailobjects.obj
 0001:00097850       ??__Es_DetailSpriteDictLump@@YAXXZ 00498850 f   detailobjects.obj
 0001:00097860       ??__EgDispGridList@@YAXXZ  00498860 f   disp_ivp.obj
 0001:00097870       ??__Eg_TesselateVerts@@YAXXZ 00498870 f   disp_powerinfo.obj
 0001:00097930       ??__Eg_VertInfo_5x5@@YAXXZ 00498930 f   disp_powerinfo.obj
 0001:00097960       ??__Eg_VertInfo_9x9@@YAXXZ 00498960 f   disp_powerinfo.obj
 0001:00097990       ??__Eg_VertInfo_17x17@@YAXXZ 00498990 f   disp_powerinfo.obj
 0001:000979c0       ??__Eg_PowerInfoInitializer@@YAXXZ 004989c0 f   disp_powerinfo.obj
 0001:000979d0       ??__Eg_CoreDispInfos@@YAXXZ 004989d0 f   disp_vbsp.obj
 0001:000979e0       ??__Eg_VertEdgeList@@YAXXZ 004989e0 f   faces.obj
 0001:00097a20       ??__Es_WorldPropList@@YAXXZ 00498a20 f   ivp.obj
 0001:00097a30       ??__Eg_WaterTexInfos@@YAXXZ 00498a30 f   ivp.obj
 0001:00097a80       ??__Eg_WaterModels@@YAXXZ  00498a80 f   ivp.obj
 0001:00097a90       ??__Eg_WaterLeafList@@YAXXZ 00498a90 f   ivp.obj
 0001:00097aa0       ??__Ebrushsides@@YAXXZ     00498aa0 f   map.obj
 0001:00097af0       ??__Eside_brushtextures@@YAXXZ 00498af0 f   map.obj
 0001:00097b30       ??__Emapplanes@@YAXXZ      00498b30 f   map.obj
 0001:00097b50       ??__Eg_NoDynamicShadowSides@@YAXXZ 00498b50 f   map.obj
 0001:00097b60       ??__Es_SymbolTable@@YAXXZ  00498b60 f   materialpatch.obj
 0001:00097b80       ??__Es_MapPatchedMatToOriginalMat@@YAXXZ 00498b80 f   materialpatch.obj
 0001:00097bd0       ??__Eg_aMapOverlays@@YAXXZ 00498bd0 f   overlay.obj
 0001:00097be0       ??__Eg_aMapWaterOverlays@@YAXXZ 00498be0 f   overlay.obj
 0001:00097bf0       ??__Eg_VisClusters@@YAXXZ  00498bf0 f   prtfile.obj
 0001:00097c00       ??__Es_StaticPropDictLump@@YAXXZ 00498c00 f   staticprop.obj
 0001:00097c10       ??__Es_StaticPropLump@@YAXXZ 00498c10 f   staticprop.obj
 0001:00097c20       ??__Es_StaticPropLeafLump@@YAXXZ 00498c20 f   staticprop.obj
 0001:00097c30       ??__Es_ModelCollisionCache@@YAXXZ 00498c30 f   staticprop.obj
 0001:00097c80       ??__Es_LightingInfo@@YAXXZ 00498c80 f   staticprop.obj
 0001:00097c90       ??__Eg_SkyAreas@@YAXXZ     00498c90 f   vbsp.obj
 0001:00097ca0       ??__Eg_OccluderInfo@@YAXXZ 00498ca0 f   vbsp.obj
 0001:00097cb0       ??__Eg_DataMapHolder@ZIP_EndOfCentralDirRecord_DataDescInit@@YAXXZ 00498cb0 f   zip_utils.obj
 0001:00097cc0       ??__Eg_DataMapHolder@ZIP_FileHeader_DataDescInit@@YAXXZ 00498cc0 f   zip_utils.obj
 0001:00097cd0       ??__Eg_DataMapHolder@ZIP_LocalFileHeader_DataDescInit@@YAXXZ 00498cd0 f   zip_utils.obj
 0001:00097ce0       ??__Eg_DataMapHolder@ZIP_PreloadHeader_DataDescInit@@YAXXZ 00498ce0 f   zip_utils.obj
 0001:00097cf0       ??__Eg_DataMapHolder@ZIP_PreloadDirectoryEntry_DataDescInit@@YAXXZ 00498cf0 f   zip_utils.obj
 0001:00097d00       ??__Eg_ZipUtils@@YAXXZ     00498d00 f   zip_utils.obj
 0001:00097d10       ??__Eg_DataMapHolder@dheader_t_DataDescInit@@YAXXZ 00498d10 f   bsplib.obj
 0001:00097d20       ??__Eg_DataMapHolder@lump_t_DataDescInit@@YAXXZ 00498d20 f   bsplib.obj
 0001:00097d30       ??__Eg_DataMapHolder@dflagslump_t_DataDescInit@@YAXXZ 00498d30 f   bsplib.obj
 0001:00097d40       ??__Eg_DataMapHolder@dplane_t_DataDescInit@@YAXXZ 00498d40 f   bsplib.obj
 0001:00097d50       ??__Eg_DataMapHolder@dleaf_version_0_t_DataDescInit@@YAXXZ 00498d50 f   bsplib.obj
 0001:00097d60       ??__Eg_DataMapHolder@dleaf_t_DataDescInit@@YAXXZ 00498d60 f   bsplib.obj
 0001:00097d70       ??__Eg_DataMapHolder@CompressedLightCube_DataDescInit@@YAXXZ 00498d70 f   bsplib.obj
 0001:00097d80       ??__Eg_DataMapHolder@dleafambientindex_t_DataDescInit@@YAXXZ 00498d80 f   bsplib.obj
 0001:00097d90       ??__Eg_DataMapHolder@dleafambientlighting_t_DataDescInit@@YAXXZ 00498d90 f   bsplib.obj
 0001:00097da0       ??__Eg_DataMapHolder@dvertex_t_DataDescInit@@YAXXZ 00498da0 f   bsplib.obj
 0001:00097db0       ??__Eg_DataMapHolder@dnode_t_DataDescInit@@YAXXZ 00498db0 f   bsplib.obj
 0001:00097dc0       ??__Eg_DataMapHolder@texinfo_t_DataDescInit@@YAXXZ 00498dc0 f   bsplib.obj
 0001:00097dd0       ??__Eg_DataMapHolder@dtexdata_t_DataDescInit@@YAXXZ 00498dd0 f   bsplib.obj
 0001:00097de0       ??__Eg_DataMapHolder@ddispinfo_t_DataDescInit@@YAXXZ 00498de0 f   bsplib.obj
 0001:00097df0       ??__Eg_DataMapHolder@CDispNeighbor_DataDescInit@@YAXXZ 00498df0 f   bsplib.obj
 0001:00097e00       ??__Eg_DataMapHolder@CDispCornerNeighbors_DataDescInit@@YAXXZ 00498e00 f   bsplib.obj
 0001:00097e10       ??__Eg_DataMapHolder@CDispSubNeighbor_DataDescInit@@YAXXZ 00498e10 f   bsplib.obj
 0001:00097e20       ??__Eg_DataMapHolder@CDispVert_DataDescInit@@YAXXZ 00498e20 f   bsplib.obj
 0001:00097e30       ??__Eg_DataMapHolder@CDispTri_DataDescInit@@YAXXZ 00498e30 f   bsplib.obj
 0001:00097e40       ??__Eg_DataMapHolder@CFaceMacroTextureInfo_DataDescInit@@YAXXZ 00498e40 f   bsplib.obj
 0001:00097e50       ??__Eg_DataMapHolder@dprimitive_t_DataDescInit@@YAXXZ 00498e50 f   bsplib.obj
 0001:00097e60       ??__Eg_DataMapHolder@dprimvert_t_DataDescInit@@YAXXZ 00498e60 f   bsplib.obj
 0001:00097e70       ??__Eg_DataMapHolder@dface_t_DataDescInit@@YAXXZ 00498e70 f   bsplib.obj
 0001:00097e80       ??__Eg_DataMapHolder@dfaceid_t_DataDescInit@@YAXXZ 00498e80 f   bsplib.obj
 0001:00097e90       ??__Eg_DataMapHolder@dbrush_t_DataDescInit@@YAXXZ 00498e90 f   bsplib.obj
 0001:00097ea0       ??__Eg_DataMapHolder@dbrushside_t_DataDescInit@@YAXXZ 00498ea0 f   bsplib.obj
 0001:00097eb0       ??__Eg_DataMapHolder@dedge_t_DataDescInit@@YAXXZ 00498eb0 f   bsplib.obj
 0001:00097ec0       ??__Eg_DataMapHolder@dmodel_t_DataDescInit@@YAXXZ 00498ec0 f   bsplib.obj
 0001:00097ed0       ??__Eg_DataMapHolder@dphysmodel_t_DataDescInit@@YAXXZ 00498ed0 f   bsplib.obj
 0001:00097ee0       ??__Eg_DataMapHolder@dphysdisp_t_DataDescInit@@YAXXZ 00498ee0 f   bsplib.obj
 0001:00097ef0       ??__Eg_DataMapHolder@darea_t_DataDescInit@@YAXXZ 00498ef0 f   bsplib.obj
 0001:00097f00       ??__Eg_DataMapHolder@dareaportal_t_DataDescInit@@YAXXZ 00498f00 f   bsplib.obj
 0001:00097f10       ??__Eg_DataMapHolder@dworldlight_t_DataDescInit@@YAXXZ 00498f10 f   bsplib.obj
 0001:00097f20       ??__Eg_DataMapHolder@dleafwaterdata_t_DataDescInit@@YAXXZ 00498f20 f   bsplib.obj
 0001:00097f30       ??__Eg_DataMapHolder@doccluderdata_t_DataDescInit@@YAXXZ 00498f30 f   bsplib.obj
 0001:00097f40       ??__Eg_DataMapHolder@doccluderpolydata_t_DataDescInit@@YAXXZ 00498f40 f   bsplib.obj
 0001:00097f50       ??__Eg_DataMapHolder@dcubemapsample_t_DataDescInit@@YAXXZ 00498f50 f   bsplib.obj
 0001:00097f60       ??__Eg_DataMapHolder@doverlay_t_DataDescInit@@YAXXZ 00498f60 f   bsplib.obj
 0001:00097f70       ??__Eg_DataMapHolder@dwateroverlay_t_DataDescInit@@YAXXZ 00498f70 f   bsplib.obj
 0001:00097f80       ??__Eg_DataMapHolder@doverlayfade_t_DataDescInit@@YAXXZ 00498f80 f   bsplib.obj
 0001:00097f90       ??__Eg_DataMapHolder@dgamelumpheader_t_DataDescInit@@YAXXZ 00498f90 f   bsplib.obj
 0001:00097fa0       ??__Eg_DataMapHolder@dgamelump_t_DataDescInit@@YAXXZ 00498fa0 f   bsplib.obj
 0001:00097fb0       ??__Eg_DataMapHolder@StaticPropDictLump_t_DataDescInit@@YAXXZ 00498fb0 f   bsplib.obj
 0001:00097fc0       ??__Eg_DataMapHolder@StaticPropLump_t_DataDescInit@@YAXXZ 00498fc0 f   bsplib.obj
 0001:00097fd0       ??__Eg_DataMapHolder@StaticPropLumpV4_t_DataDescInit@@YAXXZ 00498fd0 f   bsplib.obj
 0001:00097fe0       ??__Eg_DataMapHolder@StaticPropLumpV5_t_DataDescInit@@YAXXZ 00498fe0 f   bsplib.obj
 0001:00097ff0       ??__Eg_DataMapHolder@StaticPropLeafLump_t_DataDescInit@@YAXXZ 00498ff0 f   bsplib.obj
 0001:00098000       ??__Eg_DataMapHolder@DetailObjectDictLump_t_DataDescInit@@YAXXZ 00499000 f   bsplib.obj
 0001:00098010       ??__Eg_DataMapHolder@DetailObjectLump_t_DataDescInit@@YAXXZ 00499010 f   bsplib.obj
 0001:00098020       ??__Eg_DataMapHolder@DetailSpriteDictLump_t_DataDescInit@@YAXXZ 00499020 f   bsplib.obj
 0001:00098030       ??__Eg_DataMapHolder@DetailPropLightstylesLump_t_DataDescInit@@YAXXZ 00499030 f   bsplib.obj
 0001:00098040       ??__Eg_DataMapHolder@MeshHeader_t_DataDescInit@HardwareVerts@@YAXXZ 00499040 f   bsplib.obj
 0001:00098050       ??__Eg_DataMapHolder@FileHeader_t_DataDescInit@HardwareVerts@@YAXXZ 00499050 f   bsplib.obj
 0001:00098060       ??__Eg_StaticPropNames@@YAXXZ 00499060 f   bsplib.obj
 0001:00098070       ??__Eg_StaticPropInstances@@YAXXZ 00499070 f   bsplib.obj
 0001:00098080       ??__Eg_Swap@@YAXXZ         00499080 f   bsplib.obj
 0001:00098090       ??__EdlightdataHDR@@YAXXZ  00499090 f   bsplib.obj
 0001:000980a0       ??__EdlightdataLDR@@YAXXZ  004990a0 f   bsplib.obj
 0001:000980b0       ??__Edentdata@@YAXXZ       004990b0 f   bsplib.obj
 0001:000980c0       ??__Eg_LeafAmbientIndexLDR@@YAXXZ 004990c0 f   bsplib.obj
 0001:000980d0       ??__Eg_LeafAmbientIndexHDR@@YAXXZ 004990d0 f   bsplib.obj
 0001:000980e0       ??__Eg_LeafAmbientLightingLDR@@YAXXZ 004990e0 f   bsplib.obj
 0001:000980f0       ??__Eg_LeafAmbientLightingHDR@@YAXXZ 004990f0 f   bsplib.obj
 0001:00098100       ??__Etexinfo@@YAXXZ        00499100 f   bsplib.obj
 0001:00098110       ??__Eg_dispinfo@@YAXXZ     00499110 f   bsplib.obj
 0001:00098120       ??__Eg_DispVerts@@YAXXZ    00499120 f   bsplib.obj
 0001:00098130       ??__Eg_DispTris@@YAXXZ     00499130 f   bsplib.obj
 0001:00098140       ??__Eg_DispLightmapSamplePositions@@YAXXZ 00499140 f   bsplib.obj
 0001:00098150       ??__Edfaceids@@YAXXZ       00499150 f   bsplib.obj
 0001:00098160       ??__Eg_FaceMacroTextureInfos@@YAXXZ 00499160 f   bsplib.obj
 0001:00098170       ??__Eg_TexDataStringData@@YAXXZ 00499170 f   bsplib.obj
 0001:00098180       ??__Eg_TexDataStringTable@@YAXXZ 00499180 f   bsplib.obj
 0001:00098190       ??__Eg_OccluderData@@YAXXZ 00499190 f   bsplib.obj
 0001:000981d0       ??__Eg_OccluderPolyData@@YAXXZ 004991d0 f   bsplib.obj
 0001:00098210       ??__Eg_OccluderVertexIndices@@YAXXZ 00499210 f   bsplib.obj
 0001:00098250       ??__Eg_GameLumps@@YAXXZ    00499250 f   bsplib.obj
 0001:00098260       ??__Eg_DataMapHolder@swapcollideheader_t_DataDescInit@@YAXXZ 00499260 f   bsplib.obj
 0001:00098270       ??__Eg_DataMapHolder@swapcompactsurfaceheader_t_DataDescInit@@YAXXZ 00499270 f   bsplib.obj
 0001:00098280       ??__Eg_DataMapHolder@swapmoppsurfaceheader_t_DataDescInit@@YAXXZ 00499280 f   bsplib.obj
 0001:00098290       ??__Eg_ClusterLeaves@@YAXXZ 00499290 f   bsplib.obj
 0001:000982a0       ??__Eg_CleanupFunctions@@YAXXZ 004992a0 f   cmdlib.obj
 0001:000982b0       ??__Eg_ExtraSpewHooks@@YAXXZ 004992b0 f   cmdlib.obj
 0001:000982c0       ??__Eg_ExitStopper@@YAXXZ  004992c0 f   cmdlib.obj
 0001:000982d0       ??__Eg_definevariable@@YAXXZ 004992d0 f   scriplib.obj
 0001:000982e0       ??__Eg_CritInit@@YAXXZ     004992e0 f   threads.obj
 0001:000982f0       ??__Es_StringCharConversion@@YAXXZ 004992f0 f   tier1:utlbuffer.obj
 0001:00098350       ??__Es_NoEscConversion@@YAXXZ 00499350 f   tier1:utlbuffer.obj
 0001:00098380       ??__Eg_CleanupSymbolTable@@YAXXZ 00499380 f   tier1:utlsymbol.obj
 0001:00098390       ??__Eg_DataMapHolder@VTFFileBaseHeader_t_DataDescInit@@YAXXZ 00499390 f   vtf:vtf.obj
 0001:000983a0       ??__Eg_DataMapHolder@VTFFileHeaderV7_1_t_DataDescInit@@YAXXZ 004993a0 f   vtf:vtf.obj
 0001:000983b0       ??__Eg_DataMapHolder@VTFFileHeaderV7_2_t_DataDescInit@@YAXXZ 004993b0 f   vtf:vtf.obj
 0001:000983c0       ??__Eg_DataMapHolder@VTFFileHeaderV7_3_t_DataDescInit@@YAXXZ 004993c0 f   vtf:vtf.obj
 0001:000983d0       ??__Eg_DataMapHolder@VTFFileHeader_t_DataDescInit@@YAXXZ 004993d0 f   vtf:vtf.obj
 0001:000983e0       ??__Eg_DataMapHolder@VTFFileHeaderX360_t_DataDescInit@@YAXXZ 004993e0 f   vtf:vtf.obj
 0001:000983f0       ??__Einitlocks@std@@YAXXZ  004993f0 f   libcpmt:xlock.obj
 0001:00098406       ??__Eclassic_locale@std@@YAXXZ 00499406 f   libcpmt:locale0.obj
 0001:00098412       ??__Einitlocks@std@@YAXXZ  00499412 f   libcpmt:iosptrs.obj
 0001:00098428       ??__Einit_atexit@@YAXXZ    00499428 f   libcpmt:iosptrs.obj
 0001:00098440       ??__Ef_dwProcessorCount@@YAXXZ 00499440 f   bitmap:ATI_Compress.obj
 0001:00098460       ??__Fs_DefaultCubemapNames@@YAXXZ 00499460 f   cubemap.obj
 0001:00098470       ??__Fs_EnvCubemapToBrushSides@@YAXXZ 00499470 f   cubemap.obj
 0001:00098480       ??__Fs_DetailObjectDictLump@@YAXXZ 00499480 f   detailobjects.obj
 0001:00098490       ??__Fs_DetailObjectLump@@YAXXZ 00499490 f   detailobjects.obj
 0001:000984a0       ??__Fs_DetailSpriteDictLump@@YAXXZ 004994a0 f   detailobjects.obj
 0001:000984b0       ??__Fs_StaticPropLookup@@YAXXZ 004994b0 f   detailobjects.obj
 0001:000984c0       ??__Fs_DetailObjectDict@@YAXXZ 004994c0 f   detailobjects.obj
 0001:000984d0       ??__FgDispGridList@@YAXXZ  004994d0 f   disp_ivp.obj
 0001:000984e0       ??__Fg_CoreDispInfos@@YAXXZ 004994e0 f   disp_vbsp.obj
 0001:000984f0       ??__Fg_VertEdgeList@@YAXXZ 004994f0 f   faces.obj
 0001:00098560       ??__Fg_WaterModels@@YAXXZ  00499560 f   ivp.obj
 0001:00098570       ??__Fs_WorldPropList@@YAXXZ 00499570 f   ivp.obj
 0001:00098580       ??__Fg_WaterLeafList@@YAXXZ 00499580 f   ivp.obj
 0001:00098590       ??__Fg_WaterTexInfos@@YAXXZ 00499590 f   ivp.obj
 0001:000985a0       ??__Fg_NoDynamicShadowSides@@YAXXZ 004995a0 f   map.obj
 0001:000985b0       ??__Fbrushsides@@YAXXZ     004995b0 f   map.obj
 0001:00098650       ??__Fs_SymbolTable@@YAXXZ  00499650 f   materialpatch.obj
 0001:00098660       ??__Fs_MapPatchedMatToOriginalMat@@YAXXZ 00499660 f   materialpatch.obj
 0001:00098670       ??__Fg_aMapOverlays@@YAXXZ 00499670 f   overlay.obj
 0001:00098680       ??__Fg_aMapWaterOverlays@@YAXXZ 00499680 f   overlay.obj
 0001:00098690       ??__Fg_VisClusters@@YAXXZ  00499690 f   prtfile.obj
 0001:000986a0       ??__Fs_StaticPropDictLump@@YAXXZ 004996a0 f   staticprop.obj
 0001:000986b0       ??__Fs_StaticPropLump@@YAXXZ 004996b0 f   staticprop.obj
 0001:000986c0       ??__Fs_StaticPropLeafLump@@YAXXZ 004996c0 f   staticprop.obj
 0001:000986d0       ??__Fs_LightingInfo@@YAXXZ 004996d0 f   staticprop.obj
 0001:000986e0       ??__Fs_ModelCollisionCache@@YAXXZ 004996e0 f   staticprop.obj
 0001:000986f0       ??__Fg_SkyAreas@@YAXXZ     004996f0 f   vbsp.obj
 0001:00098700       ??__Fg_OccluderInfo@@YAXXZ 00499700 f   vbsp.obj
 0001:00098710       ??__FnameHolder@?1???$DataMapInit@UZIP_EndOfCentralDirRecord@@@@YAPAUdatamap_t@@PAUZIP_EndOfCentralDirRecord@@@Z@YAXXZ 00499710 f   zip_utils.obj
 0001:00098720       ??__FnameHolder@?1???$DataMapInit@UZIP_FileHeader@@@@YAPAUdatamap_t@@PAUZIP_FileHeader@@@Z@YAXXZ 00499720 f   zip_utils.obj
 0001:00098730       ??__FnameHolder@?1???$DataMapInit@UZIP_LocalFileHeader@@@@YAPAUdatamap_t@@PAUZIP_LocalFileHeader@@@Z@YAXXZ 00499730 f   zip_utils.obj
 0001:00098740       ??__FnameHolder@?1???$DataMapInit@UZIP_PreloadHeader@@@@YAPAUdatamap_t@@PAUZIP_PreloadHeader@@@Z@YAXXZ 00499740 f   zip_utils.obj
 0001:00098750       ??__FnameHolder@?1???$DataMapInit@UZIP_PreloadDirectoryEntry@@@@YAPAUdatamap_t@@PAUZIP_PreloadDirectoryEntry@@@Z@YAXXZ 00499750 f   zip_utils.obj
 0001:00098760       ??__Fg_ZipUtils@@YAXXZ     00499760 f   zip_utils.obj
 0001:000987b0       ??__FnameHolder@?1???$DataMapInit@Udheader_t@@@@YAPAUdatamap_t@@PAUdheader_t@@@Z@YAXXZ 004997b0 f   bsplib.obj
 0001:000987c0       ??__FnameHolder@?1???$DataMapInit@Ulump_t@@@@YAPAUdatamap_t@@PAUlump_t@@@Z@YAXXZ 004997c0 f   bsplib.obj
 0001:000987d0       ??__FnameHolder@?1???$DataMapInit@Udflagslump_t@@@@YAPAUdatamap_t@@PAUdflagslump_t@@@Z@YAXXZ 004997d0 f   bsplib.obj
 0001:000987e0       ??__FnameHolder@?1???$DataMapInit@Udplane_t@@@@YAPAUdatamap_t@@PAUdplane_t@@@Z@YAXXZ 004997e0 f   bsplib.obj
 0001:000987f0       ??__FnameHolder@?1???$DataMapInit@Udleaf_version_0_t@@@@YAPAUdatamap_t@@PAUdleaf_version_0_t@@@Z@YAXXZ 004997f0 f   bsplib.obj
 0001:00098800       ??__FnameHolder@?1???$DataMapInit@Udleaf_t@@@@YAPAUdatamap_t@@PAUdleaf_t@@@Z@YAXXZ 00499800 f   bsplib.obj
 0001:00098810       ??__FnameHolder@?1???$DataMapInit@UCompressedLightCube@@@@YAPAUdatamap_t@@PAUCompressedLightCube@@@Z@YAXXZ 00499810 f   bsplib.obj
 0001:00098820       ??__FnameHolder@?1???$DataMapInit@Udleafambientindex_t@@@@YAPAUdatamap_t@@PAUdleafambientindex_t@@@Z@YAXXZ 00499820 f   bsplib.obj
 0001:00098830       ??__FnameHolder@?1???$DataMapInit@Udleafambientlighting_t@@@@YAPAUdatamap_t@@PAUdleafambientlighting_t@@@Z@YAXXZ 00499830 f   bsplib.obj
 0001:00098840       ??__FnameHolder@?1???$DataMapInit@Udvertex_t@@@@YAPAUdatamap_t@@PAUdvertex_t@@@Z@YAXXZ 00499840 f   bsplib.obj
 0001:00098850       ??__FnameHolder@?1???$DataMapInit@Udnode_t@@@@YAPAUdatamap_t@@PAUdnode_t@@@Z@YAXXZ 00499850 f   bsplib.obj
 0001:00098860       ??__FnameHolder@?1???$DataMapInit@Utexinfo_s@@@@YAPAUdatamap_t@@PAUtexinfo_s@@@Z@YAXXZ 00499860 f   bsplib.obj
 0001:00098870       ??__FnameHolder@?1???$DataMapInit@Udtexdata_t@@@@YAPAUdatamap_t@@PAUdtexdata_t@@@Z@YAXXZ 00499870 f   bsplib.obj
 0001:00098880       ??__FnameHolder@?1???$DataMapInit@Vddispinfo_t@@@@YAPAUdatamap_t@@PAVddispinfo_t@@@Z@YAXXZ 00499880 f   bsplib.obj
 0001:00098890       ??__FnameHolder@?1???$DataMapInit@VCDispNeighbor@@@@YAPAUdatamap_t@@PAVCDispNeighbor@@@Z@YAXXZ 00499890 f   bsplib.obj
 0001:000988a0       ??__FnameHolder@?1???$DataMapInit@VCDispCornerNeighbors@@@@YAPAUdatamap_t@@PAVCDispCornerNeighbors@@@Z@YAXXZ 004998a0 f   bsplib.obj
 0001:000988b0       ??__FnameHolder@?1???$DataMapInit@UCDispSubNeighbor@@@@YAPAUdatamap_t@@PAUCDispSubNeighbor@@@Z@YAXXZ 004998b0 f   bsplib.obj
 0001:000988c0       ??__FnameHolder@?1???$DataMapInit@VCDispVert@@@@YAPAUdatamap_t@@PAVCDispVert@@@Z@YAXXZ 004998c0 f   bsplib.obj
 0001:000988d0       ??__FnameHolder@?1???$DataMapInit@VCDispTri@@@@YAPAUdatamap_t@@PAVCDispTri@@@Z@YAXXZ 004998d0 f   bsplib.obj
 0001:000988e0       ??__FnameHolder@?1???$DataMapInit@VCFaceMacroTextureInfo@@@@YAPAUdatamap_t@@PAVCFaceMacroTextureInfo@@@Z@YAXXZ 004998e0 f   bsplib.obj
 0001:000988f0       ??__FnameHolder@?1???$DataMapInit@Udprimitive_t@@@@YAPAUdatamap_t@@PAUdprimitive_t@@@Z@YAXXZ 004998f0 f   bsplib.obj
 0001:00098900       ??__FnameHolder@?1???$DataMapInit@Udprimvert_t@@@@YAPAUdatamap_t@@PAUdprimvert_t@@@Z@YAXXZ 00499900 f   bsplib.obj
 0001:00098910       ??__FnameHolder@?1???$DataMapInit@Udface_t@@@@YAPAUdatamap_t@@PAUdface_t@@@Z@YAXXZ 00499910 f   bsplib.obj
 0001:00098920       ??__FnameHolder@?1???$DataMapInit@Udfaceid_t@@@@YAPAUdatamap_t@@PAUdfaceid_t@@@Z@YAXXZ 00499920 f   bsplib.obj
 0001:00098930       ??__FnameHolder@?1???$DataMapInit@Udbrush_t@@@@YAPAUdatamap_t@@PAUdbrush_t@@@Z@YAXXZ 00499930 f   bsplib.obj
 0001:00098940       ??__FnameHolder@?1???$DataMapInit@Udbrushside_t@@@@YAPAUdatamap_t@@PAUdbrushside_t@@@Z@YAXXZ 00499940 f   bsplib.obj
 0001:00098950       ??__FnameHolder@?1???$DataMapInit@Udedge_t@@@@YAPAUdatamap_t@@PAUdedge_t@@@Z@YAXXZ 00499950 f   bsplib.obj
 0001:00098960       ??__FnameHolder@?1???$DataMapInit@Udmodel_t@@@@YAPAUdatamap_t@@PAUdmodel_t@@@Z@YAXXZ 00499960 f   bsplib.obj
 0001:00098970       ??__FnameHolder@?1???$DataMapInit@Udphysmodel_t@@@@YAPAUdatamap_t@@PAUdphysmodel_t@@@Z@YAXXZ 00499970 f   bsplib.obj
 0001:00098980       ??__FnameHolder@?1???$DataMapInit@Udphysdisp_t@@@@YAPAUdatamap_t@@PAUdphysdisp_t@@@Z@YAXXZ 00499980 f   bsplib.obj
 0001:00098990       ??__FnameHolder@?1???$DataMapInit@Udarea_t@@@@YAPAUdatamap_t@@PAUdarea_t@@@Z@YAXXZ 00499990 f   bsplib.obj
 0001:000989a0       ??__FnameHolder@?1???$DataMapInit@Udareaportal_t@@@@YAPAUdatamap_t@@PAUdareaportal_t@@@Z@YAXXZ 004999a0 f   bsplib.obj
 0001:000989b0       ??__FnameHolder@?1???$DataMapInit@Udworldlight_t@@@@YAPAUdatamap_t@@PAUdworldlight_t@@@Z@YAXXZ 004999b0 f   bsplib.obj
 0001:000989c0       ??__FnameHolder@?1???$DataMapInit@Udleafwaterdata_t@@@@YAPAUdatamap_t@@PAUdleafwaterdata_t@@@Z@YAXXZ 004999c0 f   bsplib.obj
 0001:000989d0       ??__FnameHolder@?1???$DataMapInit@Udoccluderdata_t@@@@YAPAUdatamap_t@@PAUdoccluderdata_t@@@Z@YAXXZ 004999d0 f   bsplib.obj
 0001:000989e0       ??__FnameHolder@?1???$DataMapInit@Udoccluderpolydata_t@@@@YAPAUdatamap_t@@PAUdoccluderpolydata_t@@@Z@YAXXZ 004999e0 f   bsplib.obj
 0001:000989f0       ??__FnameHolder@?1???$DataMapInit@Udcubemapsample_t@@@@YAPAUdatamap_t@@PAUdcubemapsample_t@@@Z@YAXXZ 004999f0 f   bsplib.obj
 0001:00098a00       ??__FnameHolder@?1???$DataMapInit@Udoverlay_t@@@@YAPAUdatamap_t@@PAUdoverlay_t@@@Z@YAXXZ 00499a00 f   bsplib.obj
 0001:00098a10       ??__FnameHolder@?1???$DataMapInit@Udwateroverlay_t@@@@YAPAUdatamap_t@@PAUdwateroverlay_t@@@Z@YAXXZ 00499a10 f   bsplib.obj
 0001:00098a20       ??__FnameHolder@?1???$DataMapInit@Udoverlayfade_t@@@@YAPAUdatamap_t@@PAUdoverlayfade_t@@@Z@YAXXZ 00499a20 f   bsplib.obj
 0001:00098a30       ??__FnameHolder@?1???$DataMapInit@Udgamelumpheader_t@@@@YAPAUdatamap_t@@PAUdgamelumpheader_t@@@Z@YAXXZ 00499a30 f   bsplib.obj
 0001:00098a40       ??__FnameHolder@?1???$DataMapInit@Udgamelump_t@@@@YAPAUdatamap_t@@PAUdgamelump_t@@@Z@YAXXZ 00499a40 f   bsplib.obj
 0001:00098a50       ??__FnameHolder@?1???$DataMapInit@UStaticPropDictLump_t@@@@YAPAUdatamap_t@@PAUStaticPropDictLump_t@@@Z@YAXXZ 00499a50 f   bsplib.obj
 0001:00098a60       ??__FnameHolder@?1???$DataMapInit@UStaticPropLump_t@@@@YAPAUdatamap_t@@PAUStaticPropLump_t@@@Z@YAXXZ 00499a60 f   bsplib.obj
 0001:00098a70       ??__FnameHolder@?1???$DataMapInit@UStaticPropLumpV4_t@@@@YAPAUdatamap_t@@PAUStaticPropLumpV4_t@@@Z@YAXXZ 00499a70 f   bsplib.obj
 0001:00098a80       ??__FnameHolder@?1???$DataMapInit@UStaticPropLumpV5_t@@@@YAPAUdatamap_t@@PAUStaticPropLumpV5_t@@@Z@YAXXZ 00499a80 f   bsplib.obj
 0001:00098a90       ??__FnameHolder@?1???$DataMapInit@UStaticPropLeafLump_t@@@@YAPAUdatamap_t@@PAUStaticPropLeafLump_t@@@Z@YAXXZ 00499a90 f   bsplib.obj
 0001:00098aa0       ??__FnameHolder@?1???$DataMapInit@UDetailObjectDictLump_t@@@@YAPAUdatamap_t@@PAUDetailObjectDictLump_t@@@Z@YAXXZ 00499aa0 f   bsplib.obj
 0001:00098ab0       ??__FnameHolder@?1???$DataMapInit@UDetailObjectLump_t@@@@YAPAUdatamap_t@@PAUDetailObjectLump_t@@@Z@YAXXZ 00499ab0 f   bsplib.obj
 0001:00098ac0       ??__FnameHolder@?1???$DataMapInit@UDetailSpriteDictLump_t@@@@YAPAUdatamap_t@@PAUDetailSpriteDictLump_t@@@Z@YAXXZ 00499ac0 f   bsplib.obj
 0001:00098ad0       ??__FnameHolder@?1???$DataMapInit@UDetailPropLightstylesLump_t@@@@YAPAUdatamap_t@@PAUDetailPropLightstylesLump_t@@@Z@YAXXZ 00499ad0 f   bsplib.obj
 0001:00098ae0       ??__FnameHolder@?1???$DataMapInit@UMeshHeader_t@HardwareVerts@@@HardwareVerts@@YAPAUdatamap_t@@PAUMeshHeader_t@0@@Z@YAXXZ 00499ae0 f   bsplib.obj
 0001:00098af0       ??__FnameHolder@?1???$DataMapInit@UFileHeader_t@HardwareVerts@@@HardwareVerts@@YAPAUdatamap_t@@PAUFileHeader_t@0@@Z@YAXXZ 00499af0 f   bsplib.obj
 0001:00098b00       ??__Fg_StaticPropInstances@@YAXXZ 00499b00 f   bsplib.obj
 0001:00098b10       ??__FdlightdataHDR@@YAXXZ  00499b10 f   bsplib.obj
 0001:00098b20       ??__FdlightdataLDR@@YAXXZ  00499b20 f   bsplib.obj
 0001:00098b30       ??__Fdentdata@@YAXXZ       00499b30 f   bsplib.obj
 0001:00098b40       ??__Fg_LeafAmbientIndexLDR@@YAXXZ 00499b40 f   bsplib.obj
 0001:00098b50       ??__Fg_LeafAmbientIndexHDR@@YAXXZ 00499b50 f   bsplib.obj
 0001:00098b60       ??__Fg_LeafAmbientLightingLDR@@YAXXZ 00499b60 f   bsplib.obj
 0001:00098b70       ??__Fg_LeafAmbientLightingHDR@@YAXXZ 00499b70 f   bsplib.obj
 0001:00098b80       ??__Ftexinfo@@YAXXZ        00499b80 f   bsplib.obj
 0001:00098b90       ??__Fg_DispLightmapSamplePositions@@YAXXZ 00499b90 f   bsplib.obj
 0001:00098ba0       ??__Fg_TexDataStringData@@YAXXZ 00499ba0 f   bsplib.obj
 0001:00098bb0       ??__Fg_TexDataStringTable@@YAXXZ 00499bb0 f   bsplib.obj
 0001:00098bc0       ??__Fg_OccluderData@@YAXXZ 00499bc0 f   bsplib.obj
 0001:00098bd0       ??__Fg_OccluderPolyData@@YAXXZ 00499bd0 f   bsplib.obj
 0001:00098be0       ??__Fg_OccluderVertexIndices@@YAXXZ 00499be0 f   bsplib.obj
 0001:00098bf0       ??__FnameHolder@?1???$DataMapInit@Uswapcollideheader_t@@@@YAPAUdatamap_t@@PAUswapcollideheader_t@@@Z@YAXXZ 00499bf0 f   bsplib.obj
 0001:00098c00       ??__FnameHolder@?1???$DataMapInit@Uswapcompactsurfaceheader_t@@@@YAPAUdatamap_t@@PAUswapcompactsurfaceheader_t@@@Z@YAXXZ 00499c00 f   bsplib.obj
 0001:00098c10       ??__FnameHolder@?1???$DataMapInit@Uswapmoppsurfaceheader_t@@@@YAPAUdatamap_t@@PAUswapmoppsurfaceheader_t@@@Z@YAXXZ 00499c10 f   bsplib.obj
 0001:00098c20       ??__Fg_dispinfo@@YAXXZ     00499c20 f   bsplib.obj
 0001:00098c30       ??__Fg_DispVerts@@YAXXZ    00499c30 f   bsplib.obj
 0001:00098c40       ??__Fg_DispTris@@YAXXZ     00499c40 f   bsplib.obj
 0001:00098c50       ??__Fdfaceids@@YAXXZ       00499c50 f   bsplib.obj
 0001:00098c60       ??__Fg_FaceMacroTextureInfos@@YAXXZ 00499c60 f   bsplib.obj
 0001:00098c70       ??__Fg_GameLumps@@YAXXZ    00499c70 f   bsplib.obj
 0001:00098cc0       ??__Fg_ClusterLeaves@@YAXXZ 00499cc0 f   bsplib.obj
 0001:00098cd0       ??__Fg_StaticPropNames@@YAXXZ 00499cd0 f   bsplib.obj
 0001:00098ce0       ??__Fg_ExitStopper@@YAXXZ  00499ce0 f   cmdlib.obj
 0001:00098d00       ??__Fg_CleanupFunctions@@YAXXZ 00499d00 f   cmdlib.obj
 0001:00098d50       ??__Fg_ExtraSpewHooks@@YAXXZ 00499d50 f   cmdlib.obj
 0001:00098da0       ??__Fbuf@?1??CmdLib_FPrintf@@YAXPAXPBDZZ@YAXXZ 00499da0 f   cmdlib.obj
 0001:00098db0       ??__Fg_definevariable@@YAXXZ 00499db0 f   scriplib.obj
 0001:00098dc0       ??__Fg_CleanupSymbolTable@@YAXXZ 00499dc0 f   tier1:utlsymbol.obj
 0001:00098e00       ??__FnameHolder@?1???$DataMapInit@UVTFFileBaseHeader_t@@@@YAPAUdatamap_t@@PAUVTFFileBaseHeader_t@@@Z@YAXXZ 00499e00 f   vtf:vtf.obj
 0001:00098e10       ??__FnameHolder@?1???$DataMapInit@UVTFFileHeaderV7_1_t@@@@YAPAUdatamap_t@@PAUVTFFileHeaderV7_1_t@@@Z@YAXXZ 00499e10 f   vtf:vtf.obj
 0001:00098e20       ??__FnameHolder@?1???$DataMapInit@UVTFFileHeaderV7_2_t@@@@YAPAUdatamap_t@@PAUVTFFileHeaderV7_2_t@@@Z@YAXXZ 00499e20 f   vtf:vtf.obj
 0001:00098e30       ??__FnameHolder@?1???$DataMapInit@UVTFFileHeaderV7_3_t@@@@YAPAUdatamap_t@@PAUVTFFileHeaderV7_3_t@@@Z@YAXXZ 00499e30 f   vtf:vtf.obj
 0001:00098e40       ??__FnameHolder@?1???$DataMapInit@UVTFFileHeader_t@@@@YAPAUdatamap_t@@PAUVTFFileHeader_t@@@Z@YAXXZ 00499e40 f   vtf:vtf.obj
 0001:00098e50       ??__FnameHolder@?1???$DataMapInit@UVTFFileHeaderX360_t@@@@YAPAUdatamap_t@@PAUVTFFileHeaderX360_t@@@Z@YAXXZ 00499e50 f   vtf:vtf.obj
 0001:00098e5a       ??__Finitlocks@std@@YAXXZ  00499e5a f   libcpmt:xlock.obj
 0001:00098e64       ??__Fclassic_locale@std@@YAXXZ 00499e64 f   libcpmt:locale0.obj
 0001:00098e6e       ??__Finitlocks@std@@YAXXZ  00499e6e f   libcpmt:iosptrs.obj
 0001:00098e78       ??__Finit_atexit@@YAXXZ    00499e78 f   libcpmt:iosptrs.obj
